Archive member included because of file (symbol)

c:/program files (x86)/microchip/xc32/v1.21/bin/../lib/gcc/pic32mx/4.5.2/../../../../pic32mx/lib/size\libmchp_peripheral.a(open_core_timer_lib.o)
                              build/WiFIG/production/_ext/365611741/system_services.o (OpenCoreTimer)
c:/program files (x86)/microchip/xc32/v1.21/bin/../lib/gcc/pic32mx/4.5.2/../../../../pic32mx/lib/size\libmchp_peripheral_32MX695F512H.a(soft_reset_lib.o)
                              build/WiFIG/production/_ext/365611741/system_services.o (SoftReset)
c:/program files (x86)/microchip/xc32/v1.21/bin/../lib/gcc/pic32mx/4.5.2/../../../../pic32mx/lib/size\libmchp_peripheral_32MX695F512H.a(pcache.o)
                              build/WiFIG/production/_ext/365611741/system_services.o (CheKseg0CacheOn)
c:/program files (x86)/microchip/xc32/v1.21/bin/../lib/gcc/pic32mx/4.5.2/../../../../pic32mx/lib/size\libmchp_peripheral_32MX695F512H.a(int_disable_interrupts_lib.o)
                              build/WiFIG/production/_ext/365611741/system_services.o (INTDisableInterrupts)
c:/program files (x86)/microchip/xc32/v1.21/bin/../lib/gcc/pic32mx/4.5.2/../../../../pic32mx/lib/size\libmchp_peripheral_32MX695F512H.a(int_restore_interrupts_lib.o)
                              build/WiFIG/production/_ext/365611741/system_services.o (INTRestoreInterrupts)
c:/program files (x86)/microchip/xc32/v1.21/bin/../lib/gcc/pic32mx/4.5.2/../../../../pic32mx/lib/size\libmchp_peripheral_32MX695F512H.a(int_enable_mv_int_lib.o)
                              build/WiFIG/production/_ext/365611741/system_services.o (INTEnableSystemMultiVectoredInt)
c:/program files (x86)/microchip/xc32/v1.21/bin/../lib/gcc/pic32mx/4.5.2/../../../../pic32mx/lib/size\libmchp_peripheral_32MX695F512H.a(int_tbl_lib.o)
                              build/WiFIG/production/_ext/365611741/system_services.o (INTClearFlag)
c:/program files (x86)/microchip/xc32/v1.21/bin/../lib/gcc/pic32mx/4.5.2/../../../../pic32mx/lib/size\libmchp_peripheral_32MX695F512H.a(rtcc_init_lib.o)
                              build/WiFIG/production/_ext/365611741/system_services.o (RtccInit)
c:/program files (x86)/microchip/xc32/v1.21/bin/../lib/gcc/pic32mx/4.5.2/../../../../pic32mx/lib/size\libmchp_peripheral_32MX695F512H.a(rtcc_open_lib.o)
                              build/WiFIG/production/_ext/365611741/system_services.o (RtccOpen)
c:/program files (x86)/microchip/xc32/v1.21/bin/../lib/gcc/pic32mx/4.5.2/../../../../pic32mx/lib/size\libmchp_peripheral_32MX695F512H.a(spi_chn_data_rdy_lib.o)
                              build/WiFIG/production/_ext/792872985/drv_spi.o (SpiChnDataRdy)
c:/program files (x86)/microchip/xc32/v1.21/bin/../lib/gcc/pic32mx/4.5.2/../../../../pic32mx/lib/size\libmchp_peripheral_32MX695F512H.a(spi_chn_getc_lib.o)
                              build/WiFIG/production/_ext/792872985/drv_spi.o (SpiChnReadC)
c:/program files (x86)/microchip/xc32/v1.21/bin/../lib/gcc/pic32mx/4.5.2/../../../../pic32mx/lib/size\libmchp_peripheral_32MX695F512H.a(spi_chn_open_lib.o)
                              build/WiFIG/production/_ext/792872985/drv_spi.o (SpiChnOpen)
c:/program files (x86)/microchip/xc32/v1.21/bin/../lib/gcc/pic32mx/4.5.2/../../../../pic32mx/lib/size\libmchp_peripheral_32MX695F512H.a(spi_chn_putc_lib.o)
                              build/WiFIG/production/_ext/792872985/drv_spi.o (SpiChnWriteC)
c:/program files (x86)/microchip/xc32/v1.21/bin/../lib/gcc/pic32mx/4.5.2/../../../../pic32mx/lib/size\libmchp_peripheral_32MX695F512H.a(spi_chn_tx_buff_empty_lib.o)
                              build/WiFIG/production/_ext/792872985/drv_spi.o (SpiChnTxBuffEmpty)
c:/program files (x86)/microchip/xc32/v1.21/bin/../lib/gcc/pic32mx/4.5.2/../../../../pic32mx/lib/size\libmchp_peripheral_32MX695F512H.a(spi_io_tbl_libp.o)
                              c:/program files (x86)/microchip/xc32/v1.21/bin/../lib/gcc/pic32mx/4.5.2/../../../../pic32mx/lib/size\libmchp_peripheral_32MX695F512H.a(spi_chn_open_lib.o) (_SpiIoTbl)
c:/program files (x86)/microchip/xc32/v1.21/bin/../lib/gcc/pic32mx/4.5.2/../../../../pic32mx/lib/size\libmchp_peripheral_32MX695F512H.a(spi_map_tbl_libp.o)
                              c:/program files (x86)/microchip/xc32/v1.21/bin/../lib/gcc/pic32mx/4.5.2/../../../../pic32mx/lib/size\libmchp_peripheral_32MX695F512H.a(spi_chn_data_rdy_lib.o) (_SpiMapTbl)
c:/program files (x86)/microchip/xc32/v1.21/bin/../lib/gcc/pic32mx/4.5.2/../../../../pic32mx/lib/size\libmchp_peripheral_32MX695F512H.a(port_set_pins_digital_in_lib.o)
                              c:/program files (x86)/microchip/xc32/v1.21/bin/../lib/gcc/pic32mx/4.5.2/../../../../pic32mx/lib/size\libmchp_peripheral_32MX695F512H.a(spi_chn_open_lib.o) (PORTSetPinsDigitalIn)
c:/program files (x86)/microchip/xc32/v1.21/bin/../lib/gcc/pic32mx/4.5.2/../../../../pic32mx/lib/size\libmchp_peripheral_32MX695F512H.a(port_set_pins_digital_out_lib.o)
                              c:/program files (x86)/microchip/xc32/v1.21/bin/../lib/gcc/pic32mx/4.5.2/../../../../pic32mx/lib/size\libmchp_peripheral_32MX695F512H.a(spi_chn_open_lib.o) (PORTSetPinsDigitalOut)
c:/program files (x86)/microchip/xc32/v1.21/bin/../lib/gcc/pic32mx/4.5.2/../../../../pic32mx/lib/size\libmchp_peripheral_32MX695F512H.a(_ports_tbl_libp.o)
                              c:/program files (x86)/microchip/xc32/v1.21/bin/../lib/gcc/pic32mx/4.5.2/../../../../pic32mx/lib/size\libmchp_peripheral_32MX695F512H.a(port_set_pins_digital_in_lib.o) (PortRegTbl)
c:/program files (x86)/microchip/xc32/v1.21/bin/../lib/gcc/pic32mx/4.5.2/../../../../pic32mx/lib/size\libmchp_peripheral_32MX695F512H.a(int_enable_interrupts_lib.o)
                              c:/program files (x86)/microchip/xc32/v1.21/bin/../lib/gcc/pic32mx/4.5.2/../../../../pic32mx/lib/size\libmchp_peripheral_32MX695F512H.a(int_enable_mv_int_lib.o) (INTEnableInterrupts)
c:/program files (x86)/microchip/xc32/v1.21/bin/../lib/gcc/pic32mx/4.5.2/../../../../pic32mx/lib/size\libmchp_peripheral_32MX695F512H.a(_rtcc_wait_clock_off_lib.o)
                              c:/program files (x86)/microchip/xc32/v1.21/bin/../lib/gcc/pic32mx/4.5.2/../../../../pic32mx/lib/size\libmchp_peripheral_32MX695F512H.a(rtcc_init_lib.o) (_RtccWaitClockOff)
c:/program files (x86)/microchip/xc32/v1.21/bin/../lib/gcc/pic32mx/4.5.2/../../../../pic32mx/lib/size\libmchp_peripheral_32MX695F512H.a(read_core_timer_lib.o)
                              c:/program files (x86)/microchip/xc32/v1.21/bin/../lib/gcc/pic32mx/4.5.2/../../../../pic32mx/lib/size\libmchp_peripheral_32MX695F512H.a(_rtcc_wait_clock_off_lib.o) (ReadCoreTimer)
c:/program files (x86)/microchip/xc32/v1.21/bin/../lib/gcc/pic32mx/4.5.2/size\libgcc.a(_udivdi3.o)
                              build/WiFIG/production/_ext/101875047/big_int.o (__udivdi3)
c:/program files (x86)/microchip/xc32/v1.21/bin/../lib/gcc/pic32mx/4.5.2/../../../../pic32mx/lib/size\libpic32.a(memcmp.o)
                              build/WiFIG/production/_ext/427700826/dhcp.o (memcmp)
c:/program files (x86)/microchip/xc32/v1.21/bin/../lib/gcc/pic32mx/4.5.2/../../../../pic32mx/lib/size\libpic32.a(memcpy.o)
                              build/WiFIG/production/_ext/101875047/hashes.o (memcpy)
c:/program files (x86)/microchip/xc32/v1.21/bin/../lib/gcc/pic32mx/4.5.2/../../../../pic32mx/lib/size\libpic32.a(memset.o)
                              build/WiFIG/production/_ext/427700826/ipv4.o (memset)
c:/program files (x86)/microchip/xc32/v1.21/bin/../lib/gcc/pic32mx/4.5.2/../../../../pic32mx/lib/size\libpic32.a(strcmp.o)
                              build/WiFIG/production/_ext/427700826/dns.o (strcmp)
c:/program files (x86)/microchip/xc32/v1.21/bin/../lib/gcc/pic32mx/4.5.2/../../../../pic32mx/lib/size\libpic32.a(strcpy.o)
                              build/WiFIG/production/_ext/427700826/tcpip_helpers.o (strcpy)
c:/program files (x86)/microchip/xc32/v1.21/bin/../lib/gcc/pic32mx/4.5.2/../../../../pic32mx/lib/size\libpic32.a(strlen.o)
                              build/WiFIG/production/_ext/101875047/helpers.o (strlen)
c:/program files (x86)/microchip/xc32/v1.21/bin/../lib/gcc/pic32mx/4.5.2/../../../../pic32mx/lib/size\libpic32.a(default-bootstrap-exception-handler.o)
                              c:/program files (x86)/microchip/xc32/v1.21/bin/../lib/gcc/pic32mx/4.5.2/../../../../pic32mx/lib/size/crt0.o (_bootstrap_exception_handler)
c:/program files (x86)/microchip/xc32/v1.21/bin/../lib/gcc/pic32mx/4.5.2/../../../../pic32mx/lib/size\libpic32.a(default-on-reset.o)
                              c:/program files (x86)/microchip/xc32/v1.21/bin/../lib/gcc/pic32mx/4.5.2/../../../../pic32mx/lib/size/crt0.o (_on_reset)
c:/program files (x86)/microchip/xc32/v1.21/bin/../lib/gcc/pic32mx/4.5.2/../../../../pic32mx/lib/size\libpic32.a(default-on-bootstrap.o)
                              c:/program files (x86)/microchip/xc32/v1.21/bin/../lib/gcc/pic32mx/4.5.2/../../../../pic32mx/lib/size/crt0.o (_on_bootstrap)
c:/program files (x86)/microchip/xc32/v1.21/bin/../lib/gcc/pic32mx/4.5.2/../../../../pic32mx/lib/size\libpic32.a(default-nmi-handler.o)
                              c:/program files (x86)/microchip/xc32/v1.21/bin/../lib/gcc/pic32mx/4.5.2/../../../../pic32mx/lib/size/crt0.o (_nmi_handler)
c:/program files (x86)/microchip/xc32/v1.21/bin/../lib/gcc/pic32mx/4.5.2/../../../../pic32mx/lib/size\libpic32.a(general-exception.o)
                              c:/program files (x86)/microchip/xc32/v1.21/bin/../lib/gcc/pic32mx/4.5.2/../../../../pic32mx/lib/size/crt0.o (_general_exception_context)
c:/program files (x86)/microchip/xc32/v1.21/bin/../lib/gcc/pic32mx/4.5.2/../../../../pic32mx/lib/size\libpic32.a(vector1.o)
                              c:/program files (x86)/microchip/xc32/v1.21/bin/../lib/gcc/pic32mx/4.5.2/../../../../pic32mx/lib/./proc/32MX695F512H\default_isr_vectors.o (__vector_dispatch_1)
c:/program files (x86)/microchip/xc32/v1.21/bin/../lib/gcc/pic32mx/4.5.2/../../../../pic32mx/lib/size\libpic32.a(vector2.o)
                              c:/program files (x86)/microchip/xc32/v1.21/bin/../lib/gcc/pic32mx/4.5.2/../../../../pic32mx/lib/./proc/32MX695F512H\default_isr_vectors.o (__vector_dispatch_2)
c:/program files (x86)/microchip/xc32/v1.21/bin/../lib/gcc/pic32mx/4.5.2/../../../../pic32mx/lib/size\libpic32.a(vector3.o)
                              c:/program files (x86)/microchip/xc32/v1.21/bin/../lib/gcc/pic32mx/4.5.2/../../../../pic32mx/lib/./proc/32MX695F512H\default_isr_vectors.o (__vector_dispatch_3)
c:/program files (x86)/microchip/xc32/v1.21/bin/../lib/gcc/pic32mx/4.5.2/../../../../pic32mx/lib/size\libpic32.a(vector4.o)
                              c:/program files (x86)/microchip/xc32/v1.21/bin/../lib/gcc/pic32mx/4.5.2/../../../../pic32mx/lib/./proc/32MX695F512H\default_isr_vectors.o (__vector_dispatch_4)
c:/program files (x86)/microchip/xc32/v1.21/bin/../lib/gcc/pic32mx/4.5.2/../../../../pic32mx/lib/size\libpic32.a(vector5.o)
                              c:/program files (x86)/microchip/xc32/v1.21/bin/../lib/gcc/pic32mx/4.5.2/../../../../pic32mx/lib/./proc/32MX695F512H\default_isr_vectors.o (__vector_dispatch_5)
c:/program files (x86)/microchip/xc32/v1.21/bin/../lib/gcc/pic32mx/4.5.2/../../../../pic32mx/lib/size\libpic32.a(vector6.o)
                              c:/program files (x86)/microchip/xc32/v1.21/bin/../lib/gcc/pic32mx/4.5.2/../../../../pic32mx/lib/./proc/32MX695F512H\default_isr_vectors.o (__vector_dispatch_6)
c:/program files (x86)/microchip/xc32/v1.21/bin/../lib/gcc/pic32mx/4.5.2/../../../../pic32mx/lib/size\libpic32.a(vector8.o)
                              c:/program files (x86)/microchip/xc32/v1.21/bin/../lib/gcc/pic32mx/4.5.2/../../../../pic32mx/lib/./proc/32MX695F512H\default_isr_vectors.o (__vector_dispatch_8)
c:/program files (x86)/microchip/xc32/v1.21/bin/../lib/gcc/pic32mx/4.5.2/../../../../pic32mx/lib/size\libpic32.a(vector9.o)
                              c:/program files (x86)/microchip/xc32/v1.21/bin/../lib/gcc/pic32mx/4.5.2/../../../../pic32mx/lib/./proc/32MX695F512H\default_isr_vectors.o (__vector_dispatch_9)
c:/program files (x86)/microchip/xc32/v1.21/bin/../lib/gcc/pic32mx/4.5.2/../../../../pic32mx/lib/size\libpic32.a(vector10.o)
                              c:/program files (x86)/microchip/xc32/v1.21/bin/../lib/gcc/pic32mx/4.5.2/../../../../pic32mx/lib/./proc/32MX695F512H\default_isr_vectors.o (__vector_dispatch_10)
c:/program files (x86)/microchip/xc32/v1.21/bin/../lib/gcc/pic32mx/4.5.2/../../../../pic32mx/lib/size\libpic32.a(vector11.o)
                              c:/program files (x86)/microchip/xc32/v1.21/bin/../lib/gcc/pic32mx/4.5.2/../../../../pic32mx/lib/./proc/32MX695F512H\default_isr_vectors.o (__vector_dispatch_11)
c:/program files (x86)/microchip/xc32/v1.21/bin/../lib/gcc/pic32mx/4.5.2/../../../../pic32mx/lib/size\libpic32.a(vector12.o)
                              c:/program files (x86)/microchip/xc32/v1.21/bin/../lib/gcc/pic32mx/4.5.2/../../../../pic32mx/lib/./proc/32MX695F512H\default_isr_vectors.o (__vector_dispatch_12)
c:/program files (x86)/microchip/xc32/v1.21/bin/../lib/gcc/pic32mx/4.5.2/../../../../pic32mx/lib/size\libpic32.a(vector13.o)
                              c:/program files (x86)/microchip/xc32/v1.21/bin/../lib/gcc/pic32mx/4.5.2/../../../../pic32mx/lib/./proc/32MX695F512H\default_isr_vectors.o (__vector_dispatch_13)
c:/program files (x86)/microchip/xc32/v1.21/bin/../lib/gcc/pic32mx/4.5.2/../../../../pic32mx/lib/size\libpic32.a(vector14.o)
                              c:/program files (x86)/microchip/xc32/v1.21/bin/../lib/gcc/pic32mx/4.5.2/../../../../pic32mx/lib/./proc/32MX695F512H\default_isr_vectors.o (__vector_dispatch_14)
c:/program files (x86)/microchip/xc32/v1.21/bin/../lib/gcc/pic32mx/4.5.2/../../../../pic32mx/lib/size\libpic32.a(vector16.o)
                              c:/program files (x86)/microchip/xc32/v1.21/bin/../lib/gcc/pic32mx/4.5.2/../../../../pic32mx/lib/./proc/32MX695F512H\default_isr_vectors.o (__vector_dispatch_16)
c:/program files (x86)/microchip/xc32/v1.21/bin/../lib/gcc/pic32mx/4.5.2/../../../../pic32mx/lib/size\libpic32.a(vector17.o)
                              c:/program files (x86)/microchip/xc32/v1.21/bin/../lib/gcc/pic32mx/4.5.2/../../../../pic32mx/lib/./proc/32MX695F512H\default_isr_vectors.o (__vector_dispatch_17)
c:/program files (x86)/microchip/xc32/v1.21/bin/../lib/gcc/pic32mx/4.5.2/../../../../pic32mx/lib/size\libpic32.a(vector18.o)
                              c:/program files (x86)/microchip/xc32/v1.21/bin/../lib/gcc/pic32mx/4.5.2/../../../../pic32mx/lib/./proc/32MX695F512H\default_isr_vectors.o (__vector_dispatch_18)
c:/program files (x86)/microchip/xc32/v1.21/bin/../lib/gcc/pic32mx/4.5.2/../../../../pic32mx/lib/size\libpic32.a(vector19.o)
                              c:/program files (x86)/microchip/xc32/v1.21/bin/../lib/gcc/pic32mx/4.5.2/../../../../pic32mx/lib/./proc/32MX695F512H\default_isr_vectors.o (__vector_dispatch_19)
c:/program files (x86)/microchip/xc32/v1.21/bin/../lib/gcc/pic32mx/4.5.2/../../../../pic32mx/lib/size\libpic32.a(vector20.o)
                              c:/program files (x86)/microchip/xc32/v1.21/bin/../lib/gcc/pic32mx/4.5.2/../../../../pic32mx/lib/./proc/32MX695F512H\default_isr_vectors.o (__vector_dispatch_20)
c:/program files (x86)/microchip/xc32/v1.21/bin/../lib/gcc/pic32mx/4.5.2/../../../../pic32mx/lib/size\libpic32.a(vector21.o)
                              c:/program files (x86)/microchip/xc32/v1.21/bin/../lib/gcc/pic32mx/4.5.2/../../../../pic32mx/lib/./proc/32MX695F512H\default_isr_vectors.o (__vector_dispatch_21)
c:/program files (x86)/microchip/xc32/v1.21/bin/../lib/gcc/pic32mx/4.5.2/../../../../pic32mx/lib/size\libpic32.a(vector22.o)
                              c:/program files (x86)/microchip/xc32/v1.21/bin/../lib/gcc/pic32mx/4.5.2/../../../../pic32mx/lib/./proc/32MX695F512H\default_isr_vectors.o (__vector_dispatch_22)
c:/program files (x86)/microchip/xc32/v1.21/bin/../lib/gcc/pic32mx/4.5.2/../../../../pic32mx/lib/size\libpic32.a(vector23.o)
                              c:/program files (x86)/microchip/xc32/v1.21/bin/../lib/gcc/pic32mx/4.5.2/../../../../pic32mx/lib/./proc/32MX695F512H\default_isr_vectors.o (__vector_dispatch_23)
c:/program files (x86)/microchip/xc32/v1.21/bin/../lib/gcc/pic32mx/4.5.2/../../../../pic32mx/lib/size\libpic32.a(vector24.o)
                              c:/program files (x86)/microchip/xc32/v1.21/bin/../lib/gcc/pic32mx/4.5.2/../../../../pic32mx/lib/./proc/32MX695F512H\default_isr_vectors.o (__vector_dispatch_24)
c:/program files (x86)/microchip/xc32/v1.21/bin/../lib/gcc/pic32mx/4.5.2/../../../../pic32mx/lib/size\libpic32.a(vector25.o)
                              c:/program files (x86)/microchip/xc32/v1.21/bin/../lib/gcc/pic32mx/4.5.2/../../../../pic32mx/lib/./proc/32MX695F512H\default_isr_vectors.o (__vector_dispatch_25)
c:/program files (x86)/microchip/xc32/v1.21/bin/../lib/gcc/pic32mx/4.5.2/../../../../pic32mx/lib/size\libpic32.a(vector27.o)
                              c:/program files (x86)/microchip/xc32/v1.21/bin/../lib/gcc/pic32mx/4.5.2/../../../../pic32mx/lib/./proc/32MX695F512H\default_isr_vectors.o (__vector_dispatch_27)
c:/program files (x86)/microchip/xc32/v1.21/bin/../lib/gcc/pic32mx/4.5.2/../../../../pic32mx/lib/size\libpic32.a(vector28.o)
                              c:/program files (x86)/microchip/xc32/v1.21/bin/../lib/gcc/pic32mx/4.5.2/../../../../pic32mx/lib/./proc/32MX695F512H\default_isr_vectors.o (__vector_dispatch_28)
c:/program files (x86)/microchip/xc32/v1.21/bin/../lib/gcc/pic32mx/4.5.2/../../../../pic32mx/lib/size\libpic32.a(vector29.o)
                              c:/program files (x86)/microchip/xc32/v1.21/bin/../lib/gcc/pic32mx/4.5.2/../../../../pic32mx/lib/./proc/32MX695F512H\default_isr_vectors.o (__vector_dispatch_29)
c:/program files (x86)/microchip/xc32/v1.21/bin/../lib/gcc/pic32mx/4.5.2/../../../../pic32mx/lib/size\libpic32.a(vector30.o)
                              c:/program files (x86)/microchip/xc32/v1.21/bin/../lib/gcc/pic32mx/4.5.2/../../../../pic32mx/lib/./proc/32MX695F512H\default_isr_vectors.o (__vector_dispatch_30)
c:/program files (x86)/microchip/xc32/v1.21/bin/../lib/gcc/pic32mx/4.5.2/../../../../pic32mx/lib/size\libpic32.a(vector31.o)
                              c:/program files (x86)/microchip/xc32/v1.21/bin/../lib/gcc/pic32mx/4.5.2/../../../../pic32mx/lib/./proc/32MX695F512H\default_isr_vectors.o (__vector_dispatch_31)
c:/program files (x86)/microchip/xc32/v1.21/bin/../lib/gcc/pic32mx/4.5.2/../../../../pic32mx/lib/size\libpic32.a(vector32.o)
                              c:/program files (x86)/microchip/xc32/v1.21/bin/../lib/gcc/pic32mx/4.5.2/../../../../pic32mx/lib/./proc/32MX695F512H\default_isr_vectors.o (__vector_dispatch_32)
c:/program files (x86)/microchip/xc32/v1.21/bin/../lib/gcc/pic32mx/4.5.2/../../../../pic32mx/lib/size\libpic32.a(vector33.o)
                              c:/program files (x86)/microchip/xc32/v1.21/bin/../lib/gcc/pic32mx/4.5.2/../../../../pic32mx/lib/./proc/32MX695F512H\default_isr_vectors.o (__vector_dispatch_33)
c:/program files (x86)/microchip/xc32/v1.21/bin/../lib/gcc/pic32mx/4.5.2/../../../../pic32mx/lib/size\libpic32.a(vector34.o)
                              c:/program files (x86)/microchip/xc32/v1.21/bin/../lib/gcc/pic32mx/4.5.2/../../../../pic32mx/lib/./proc/32MX695F512H\default_isr_vectors.o (__vector_dispatch_34)
c:/program files (x86)/microchip/xc32/v1.21/bin/../lib/gcc/pic32mx/4.5.2/../../../../pic32mx/lib/size\libpic32.a(vector35.o)
                              c:/program files (x86)/microchip/xc32/v1.21/bin/../lib/gcc/pic32mx/4.5.2/../../../../pic32mx/lib/./proc/32MX695F512H\default_isr_vectors.o (__vector_dispatch_35)
c:/program files (x86)/microchip/xc32/v1.21/bin/../lib/gcc/pic32mx/4.5.2/../../../../pic32mx/lib/size\libpic32.a(vector36.o)
                              c:/program files (x86)/microchip/xc32/v1.21/bin/../lib/gcc/pic32mx/4.5.2/../../../../pic32mx/lib/./proc/32MX695F512H\default_isr_vectors.o (__vector_dispatch_36)
c:/program files (x86)/microchip/xc32/v1.21/bin/../lib/gcc/pic32mx/4.5.2/../../../../pic32mx/lib/size\libpic32.a(vector37.o)
                              c:/program files (x86)/microchip/xc32/v1.21/bin/../lib/gcc/pic32mx/4.5.2/../../../../pic32mx/lib/./proc/32MX695F512H\default_isr_vectors.o (__vector_dispatch_37)
c:/program files (x86)/microchip/xc32/v1.21/bin/../lib/gcc/pic32mx/4.5.2/../../../../pic32mx/lib/size\libpic32.a(vector38.o)
                              c:/program files (x86)/microchip/xc32/v1.21/bin/../lib/gcc/pic32mx/4.5.2/../../../../pic32mx/lib/./proc/32MX695F512H\default_isr_vectors.o (__vector_dispatch_38)
c:/program files (x86)/microchip/xc32/v1.21/bin/../lib/gcc/pic32mx/4.5.2/../../../../pic32mx/lib/size\libpic32.a(vector39.o)
                              c:/program files (x86)/microchip/xc32/v1.21/bin/../lib/gcc/pic32mx/4.5.2/../../../../pic32mx/lib/./proc/32MX695F512H\default_isr_vectors.o (__vector_dispatch_39)
c:/program files (x86)/microchip/xc32/v1.21/bin/../lib/gcc/pic32mx/4.5.2/../../../../pic32mx/lib/size\libpic32.a(vector40.o)
                              c:/program files (x86)/microchip/xc32/v1.21/bin/../lib/gcc/pic32mx/4.5.2/../../../../pic32mx/lib/./proc/32MX695F512H\default_isr_vectors.o (__vector_dispatch_40)
c:/program files (x86)/microchip/xc32/v1.21/bin/../lib/gcc/pic32mx/4.5.2/../../../../pic32mx/lib/size\libpic32.a(vector41.o)
                              c:/program files (x86)/microchip/xc32/v1.21/bin/../lib/gcc/pic32mx/4.5.2/../../../../pic32mx/lib/./proc/32MX695F512H\default_isr_vectors.o (__vector_dispatch_41)
c:/program files (x86)/microchip/xc32/v1.21/bin/../lib/gcc/pic32mx/4.5.2/../../../../pic32mx/lib/size\libpic32.a(vector42.o)
                              c:/program files (x86)/microchip/xc32/v1.21/bin/../lib/gcc/pic32mx/4.5.2/../../../../pic32mx/lib/./proc/32MX695F512H\default_isr_vectors.o (__vector_dispatch_42)
c:/program files (x86)/microchip/xc32/v1.21/bin/../lib/gcc/pic32mx/4.5.2/../../../../pic32mx/lib/size\libpic32.a(vector43.o)
                              c:/program files (x86)/microchip/xc32/v1.21/bin/../lib/gcc/pic32mx/4.5.2/../../../../pic32mx/lib/./proc/32MX695F512H\default_isr_vectors.o (__vector_dispatch_43)
c:/program files (x86)/microchip/xc32/v1.21/bin/../lib/gcc/pic32mx/4.5.2/../../../../pic32mx/lib/size\libpic32.a(vector44.o)
                              c:/program files (x86)/microchip/xc32/v1.21/bin/../lib/gcc/pic32mx/4.5.2/../../../../pic32mx/lib/./proc/32MX695F512H\default_isr_vectors.o (__vector_dispatch_44)
c:/program files (x86)/microchip/xc32/v1.21/bin/../lib/gcc/pic32mx/4.5.2/../../../../pic32mx/lib/size\libpic32.a(vector45.o)
                              c:/program files (x86)/microchip/xc32/v1.21/bin/../lib/gcc/pic32mx/4.5.2/../../../../pic32mx/lib/./proc/32MX695F512H\default_isr_vectors.o (__vector_dispatch_45)
c:/program files (x86)/microchip/xc32/v1.21/bin/../lib/gcc/pic32mx/4.5.2/../../../../pic32mx/lib/size\libpic32.a(vector46.o)
                              c:/program files (x86)/microchip/xc32/v1.21/bin/../lib/gcc/pic32mx/4.5.2/../../../../pic32mx/lib/./proc/32MX695F512H\default_isr_vectors.o (__vector_dispatch_46)
c:/program files (x86)/microchip/xc32/v1.21/bin/../lib/gcc/pic32mx/4.5.2/../../../../pic32mx/lib/size\libpic32.a(vector47.o)
                              c:/program files (x86)/microchip/xc32/v1.21/bin/../lib/gcc/pic32mx/4.5.2/../../../../pic32mx/lib/./proc/32MX695F512H\default_isr_vectors.o (__vector_dispatch_47)
c:/program files (x86)/microchip/xc32/v1.21/bin/../lib/gcc/pic32mx/4.5.2/../../../../pic32mx/lib/size\libpic32.a(vector48.o)
                              c:/program files (x86)/microchip/xc32/v1.21/bin/../lib/gcc/pic32mx/4.5.2/../../../../pic32mx/lib/./proc/32MX695F512H\default_isr_vectors.o (__vector_dispatch_48)
c:/program files (x86)/microchip/xc32/v1.21/bin/../lib/gcc/pic32mx/4.5.2/../../../../pic32mx/lib/size\libpic32.a(vector49.o)
                              c:/program files (x86)/microchip/xc32/v1.21/bin/../lib/gcc/pic32mx/4.5.2/../../../../pic32mx/lib/./proc/32MX695F512H\default_isr_vectors.o (__vector_dispatch_49)
c:/program files (x86)/microchip/xc32/v1.21/bin/../lib/gcc/pic32mx/4.5.2/../../../../pic32mx/lib/size\libpic32.a(vector50.o)
                              c:/program files (x86)/microchip/xc32/v1.21/bin/../lib/gcc/pic32mx/4.5.2/../../../../pic32mx/lib/./proc/32MX695F512H\default_isr_vectors.o (__vector_dispatch_50)
c:/program files (x86)/microchip/xc32/v1.21/bin/../lib/gcc/pic32mx/4.5.2/../../../../pic32mx/lib/size\libpic32.a(vector51.o)
                              c:/program files (x86)/microchip/xc32/v1.21/bin/../lib/gcc/pic32mx/4.5.2/../../../../pic32mx/lib/./proc/32MX695F512H\default_isr_vectors.o (__vector_dispatch_51)
c:/program files (x86)/microchip/xc32/v1.21/bin/../lib/gcc/pic32mx/4.5.2/../../../../pic32mx/lib/size\libpic32.a(vector52.o)
                              c:/program files (x86)/microchip/xc32/v1.21/bin/../lib/gcc/pic32mx/4.5.2/../../../../pic32mx/lib/./proc/32MX695F512H\default_isr_vectors.o (__vector_dispatch_52)
c:/program files (x86)/microchip/xc32/v1.21/bin/../lib/gcc/pic32mx/4.5.2/../../../../pic32mx/lib/size\libpic32.a(vector53.o)
                              c:/program files (x86)/microchip/xc32/v1.21/bin/../lib/gcc/pic32mx/4.5.2/../../../../pic32mx/lib/./proc/32MX695F512H\default_isr_vectors.o (__vector_dispatch_53)
c:/program files (x86)/microchip/xc32/v1.21/bin/../lib/gcc/pic32mx/4.5.2/../../../../pic32mx/lib/size\libpic32.a(vector54.o)
                              c:/program files (x86)/microchip/xc32/v1.21/bin/../lib/gcc/pic32mx/4.5.2/../../../../pic32mx/lib/./proc/32MX695F512H\default_isr_vectors.o (__vector_dispatch_54)
c:/program files (x86)/microchip/xc32/v1.21/bin/../lib/gcc/pic32mx/4.5.2/../../../../pic32mx/lib/size\libpic32.a(vector55.o)
                              c:/program files (x86)/microchip/xc32/v1.21/bin/../lib/gcc/pic32mx/4.5.2/../../../../pic32mx/lib/./proc/32MX695F512H\default_isr_vectors.o (__vector_dispatch_55)
c:/program files (x86)/microchip/xc32/v1.21/bin/../lib/gcc/pic32mx/4.5.2/../../../../pic32mx/lib/size\libpic32.a(vector56.o)
                              c:/program files (x86)/microchip/xc32/v1.21/bin/../lib/gcc/pic32mx/4.5.2/../../../../pic32mx/lib/./proc/32MX695F512H\default_isr_vectors.o (__vector_dispatch_56)
c:/program files (x86)/microchip/xc32/v1.21/bin/../lib/gcc/pic32mx/4.5.2/../../../../pic32mx/lib/size\libpic32.a(vector57.o)
                              c:/program files (x86)/microchip/xc32/v1.21/bin/../lib/gcc/pic32mx/4.5.2/../../../../pic32mx/lib/./proc/32MX695F512H\default_isr_vectors.o (__vector_dispatch_57)
c:/program files (x86)/microchip/xc32/v1.21/bin/../lib/gcc/pic32mx/4.5.2/../../../../pic32mx/lib/size\libpic32.a(vector58.o)
                              c:/program files (x86)/microchip/xc32/v1.21/bin/../lib/gcc/pic32mx/4.5.2/../../../../pic32mx/lib/./proc/32MX695F512H\default_isr_vectors.o (__vector_dispatch_58)
c:/program files (x86)/microchip/xc32/v1.21/bin/../lib/gcc/pic32mx/4.5.2/../../../../pic32mx/lib/size\libpic32.a(vector59.o)
                              c:/program files (x86)/microchip/xc32/v1.21/bin/../lib/gcc/pic32mx/4.5.2/../../../../pic32mx/lib/./proc/32MX695F512H\default_isr_vectors.o (__vector_dispatch_59)
c:/program files (x86)/microchip/xc32/v1.21/bin/../lib/gcc/pic32mx/4.5.2/../../../../pic32mx/lib/size\libpic32.a(vector60.o)
                              c:/program files (x86)/microchip/xc32/v1.21/bin/../lib/gcc/pic32mx/4.5.2/../../../../pic32mx/lib/./proc/32MX695F512H\default_isr_vectors.o (__vector_dispatch_60)
c:/program files (x86)/microchip/xc32/v1.21/bin/../lib/gcc/pic32mx/4.5.2/../../../../pic32mx/lib/size\libpic32.a(vector61.o)
                              c:/program files (x86)/microchip/xc32/v1.21/bin/../lib/gcc/pic32mx/4.5.2/../../../../pic32mx/lib/./proc/32MX695F512H\default_isr_vectors.o (__vector_dispatch_61)
c:/program files (x86)/microchip/xc32/v1.21/bin/../lib/gcc/pic32mx/4.5.2/../../../../pic32mx/lib/size\libpic32.a(vector62.o)
                              c:/program files (x86)/microchip/xc32/v1.21/bin/../lib/gcc/pic32mx/4.5.2/../../../../pic32mx/lib/./proc/32MX695F512H\default_isr_vectors.o (__vector_dispatch_62)
c:/program files (x86)/microchip/xc32/v1.21/bin/../lib/gcc/pic32mx/4.5.2/../../../../pic32mx/lib/size\libpic32.a(vector63.o)
                              c:/program files (x86)/microchip/xc32/v1.21/bin/../lib/gcc/pic32mx/4.5.2/../../../../pic32mx/lib/./proc/32MX695F512H\default_isr_vectors.o (__vector_dispatch_63)
c:/program files (x86)/microchip/xc32/v1.21/bin/../lib/gcc/pic32mx/4.5.2/../../../../pic32mx/lib/size\libpic32.a(defaultinterrupt.o)
                              c:/program files (x86)/microchip/xc32/v1.21/bin/../lib/gcc/pic32mx/4.5.2/../../../../pic32mx/lib/size\libpic32.a(vector1.o) (_DefaultInterrupt)
c:/program files (x86)/microchip/xc32/v1.21/bin/../lib/gcc/pic32mx/4.5.2/../../../../pic32mx/lib/size\libc.a(atoi.o)
                              build/WiFIG/production/_ext/334706090/wf_commands.o (atoi)
c:/program files (x86)/microchip/xc32/v1.21/bin/../lib/gcc/pic32mx/4.5.2/../../../../pic32mx/lib/size\libc.a(ctype.o)
                              build/WiFIG/production/_ext/427700826/tcpip_helpers.o (_ctype)
c:/program files (x86)/microchip/xc32/v1.21/bin/../lib/gcc/pic32mx/4.5.2/../../../../pic32mx/lib/size\libc.a(malloc.o)
                              build/WiFIG/production/_ext/365611741/system_services.o (malloc)
c:/program files (x86)/microchip/xc32/v1.21/bin/../lib/gcc/pic32mx/4.5.2/../../../../pic32mx/lib/size\libc.a(rand.o)
                              build/WiFIG/production/_ext/427700826/dhcp.o (rand)
c:/program files (x86)/microchip/xc32/v1.21/bin/../lib/gcc/pic32mx/4.5.2/../../../../pic32mx/lib/size\libc.a(strcat.o)
                              build/WiFIG/production/_ext/1472/ping_demo.o (strcat)
c:/program files (x86)/microchip/xc32/v1.21/bin/../lib/gcc/pic32mx/4.5.2/../../../../pic32mx/lib/size\libc.a(strchr.o)
                              build/WiFIG/production/_ext/334706090/wf_commands.o (strchr)
c:/program files (x86)/microchip/xc32/v1.21/bin/../lib/gcc/pic32mx/4.5.2/../../../../pic32mx/lib/size\libc.a(strncat.o)
                              build/WiFIG/production/_ext/1472/tcp6_demo_app.o (strncat)
c:/program files (x86)/microchip/xc32/v1.21/bin/../lib/gcc/pic32mx/4.5.2/../../../../pic32mx/lib/size\libc.a(strncpy.o)
                              build/WiFIG/production/_ext/101875047/helpers.o (strncpy)
c:/program files (x86)/microchip/xc32/v1.21/bin/../lib/gcc/pic32mx/4.5.2/../../../../pic32mx/lib/size\libc.a(strstr.o)
                              build/WiFIG/production/_ext/1472/tcp6_demo_app.o (strstr)
c:/program files (x86)/microchip/xc32/v1.21/bin/../lib/gcc/pic32mx/4.5.2/../../../../pic32mx/lib/size\libc.a(strtol.o)
                              build/WiFIG/production/_ext/1472/tcp6_demo_app.o (strtol)
c:/program files (x86)/microchip/xc32/v1.21/bin/../lib/gcc/pic32mx/4.5.2/../../../../pic32mx/lib/size\libc.a(snprintf_cdnopsuxX.eo)
                              build/WiFIG/production/_ext/365611741/system_debug.o (_snprintf_cdnopsuxX)
c:/program files (x86)/microchip/xc32/v1.21/bin/../lib/gcc/pic32mx/4.5.2/../../../../pic32mx/lib/size\libc.a(sprintf_cdnopsuxX.eo)
                              build/WiFIG/production/_ext/334706090/wf_configData.o (_sprintf_cdnopsuxX)
c:/program files (x86)/microchip/xc32/v1.21/bin/../lib/gcc/pic32mx/4.5.2/../../../../pic32mx/lib/size\libc.a(sprintf_cdnopuxX.eo)
                              build/WiFIG/production/_ext/427700826/tcpip_helpers.o (_sprintf_cdnopuxX)
c:/program files (x86)/microchip/xc32/v1.21/bin/../lib/gcc/pic32mx/4.5.2/../../../../pic32mx/lib/size\libc.a(vsnprintf_cdnopsuxX.eo)
                              c:/program files (x86)/microchip/xc32/v1.21/bin/../lib/gcc/pic32mx/4.5.2/../../../../pic32mx/lib/size\libc.a(snprintf_cdnopsuxX.eo) (_vsnprintf_cdnopsuxX)
c:/program files (x86)/microchip/xc32/v1.21/bin/../lib/gcc/pic32mx/4.5.2/../../../../pic32mx/lib/size\libc.a(vsnprintf.o)
                              build/WiFIG/production/_ext/365611741/system_debug.o (vsnprintf)
c:/program files (x86)/microchip/xc32/v1.21/bin/../lib/gcc/pic32mx/4.5.2/../../../../pic32mx/lib/size\libc.a(ctypef.o)
                              c:/program files (x86)/microchip/xc32/v1.21/bin/../lib/gcc/pic32mx/4.5.2/../../../../pic32mx/lib/size\libc.a(strtol.o) (toupper)
c:/program files (x86)/microchip/xc32/v1.21/bin/../lib/gcc/pic32mx/4.5.2/../../../../pic32mx/lib/size\libc.a(errno.o)
                              c:/program files (x86)/microchip/xc32/v1.21/bin/../lib/gcc/pic32mx/4.5.2/../../../../pic32mx/lib/size\libc.a(strtol.o) (errno)
c:/program files (x86)/microchip/xc32/v1.21/bin/../lib/gcc/pic32mx/4.5.2/../../../../pic32mx/lib/size\libc.a(strncmp.o)
                              c:/program files (x86)/microchip/xc32/v1.21/bin/../lib/gcc/pic32mx/4.5.2/../../../../pic32mx/lib/size\libc.a(strstr.o) (strncmp)
c:/program files (x86)/microchip/xc32/v1.21/bin/../lib/gcc/pic32mx/4.5.2/../../../../pic32mx/lib/size\libc.a(doprnt_cdnopsuxX.eo)
                              c:/program files (x86)/microchip/xc32/v1.21/bin/../lib/gcc/pic32mx/4.5.2/../../../../pic32mx/lib/size\libc.a(sprintf_cdnopsuxX.eo) (_vfprintf_cdnopsuxX)
c:/program files (x86)/microchip/xc32/v1.21/bin/../lib/gcc/pic32mx/4.5.2/../../../../pic32mx/lib/size\libc.a(doprnt_cdnopuxX.eo)
                              c:/program files (x86)/microchip/xc32/v1.21/bin/../lib/gcc/pic32mx/4.5.2/../../../../pic32mx/lib/size\libc.a(sprintf_cdnopuxX.eo) (_vfprintf_cdnopuxX)
c:/program files (x86)/microchip/xc32/v1.21/bin/../lib/gcc/pic32mx/4.5.2/../../../../pic32mx/lib/size\libc.a(doprnt.o)
                              c:/program files (x86)/microchip/xc32/v1.21/bin/../lib/gcc/pic32mx/4.5.2/../../../../pic32mx/lib/size\libc.a(vsnprintf.o) (vfprintf)
c:/program files (x86)/microchip/xc32/v1.21/bin/../lib/gcc/pic32mx/4.5.2/../../../../pic32mx/lib/size\libc.a(_fputc_simple.o)
                              c:/program files (x86)/microchip/xc32/v1.21/bin/../lib/gcc/pic32mx/4.5.2/../../../../pic32mx/lib/size\libc.a(doprnt_cdnopsuxX.eo) (fputc)
c:/program files (x86)/microchip/xc32/v1.21/bin/../lib/gcc/pic32mx/4.5.2/../../../../pic32mx/lib/size\libc.a(powersf.o)
                              c:/program files (x86)/microchip/xc32/v1.21/bin/../lib/gcc/pic32mx/4.5.2/../../../../pic32mx/lib/size\libc.a(doprnt.o) (_powers_f)
c:/program files (x86)/microchip/xc32/v1.21/bin/../lib/gcc/pic32mx/4.5.2/../../../../pic32mx/lib/size\libc.a(_iob.o)
                              c:/program files (x86)/microchip/xc32/v1.21/bin/../lib/gcc/pic32mx/4.5.2/../../../../pic32mx/lib/size\libc.a(_fputc_simple.o) (_outdone)
c:/program files (x86)/microchip/xc32/v1.21/bin/../lib/gcc/pic32mx/4.5.2/../../../../pic32mx/lib/size\libc.a(_flsbuf_simple.o)
                              c:/program files (x86)/microchip/xc32/v1.21/bin/../lib/gcc/pic32mx/4.5.2/../../../../pic32mx/lib/size\libc.a(_fputc_simple.o) (_flsbuf)
c:/program files (x86)/microchip/xc32/v1.21/bin/../lib/gcc/pic32mx/4.5.2/../../../../pic32mx/lib/size\libpic32.a(sbrk.o)
                              c:/program files (x86)/microchip/xc32/v1.21/bin/../lib/gcc/pic32mx/4.5.2/../../../../pic32mx/lib/size\libc.a(malloc.o) (sbrk)
c:/program files (x86)/microchip/xc32/v1.21/bin/../lib/gcc/pic32mx/4.5.2/../../../../pic32mx/lib/size\libpic32.a(write.o)
                              c:/program files (x86)/microchip/xc32/v1.21/bin/../lib/gcc/pic32mx/4.5.2/../../../../pic32mx/lib/size\libc.a(_fputc_simple.o) (write)
c:/program files (x86)/microchip/xc32/v1.21/bin/../lib/gcc/pic32mx/4.5.2/../../../../pic32mx/lib/size\libpic32.a(_mon_putc.o)
                              c:/program files (x86)/microchip/xc32/v1.21/bin/../lib/gcc/pic32mx/4.5.2/../../../../pic32mx/lib/size\libpic32.a(write.o) (_mon_putc)
c:/program files (x86)/microchip/xc32/v1.21/bin/../lib/gcc/pic32mx/4.5.2/../../../../pic32mx/lib/size\libpic32.a(xc32_uart.o)
                              c:/program files (x86)/microchip/xc32/v1.21/bin/../lib/gcc/pic32mx/4.5.2/../../../../pic32mx/lib/size\libpic32.a(_mon_putc.o) (__XC_UART)
c:/program files (x86)/microchip/xc32/v1.21/bin/../lib/gcc/pic32mx/4.5.2/../../../../pic32mx/lib/size\libm.a(fpmod32.o)
                              c:/program files (x86)/microchip/xc32/v1.21/bin/../lib/gcc/pic32mx/4.5.2/../../../../pic32mx/lib/size\libc.a(doprnt.o) (frexpf)
c:/program files (x86)/microchip/xc32/v1.21/bin/../lib/gcc/pic32mx/4.5.2/../../../../pic32mx/lib/size\libm.a(fp32.o)
                              c:/program files (x86)/microchip/xc32/v1.21/bin/../lib/gcc/pic32mx/4.5.2/../../../../pic32mx/lib/size\libc.a(doprnt.o) (fpsub)
c:/program files (x86)/microchip/xc32/v1.21/bin/../lib/gcc/pic32mx/4.5.2/../../../../pic32mx/lib/size\libe.a(_floatdisf.o)
                              c:/program files (x86)/microchip/xc32/v1.21/bin/../lib/gcc/pic32mx/4.5.2/../../../../pic32mx/lib/size\libc.a(doprnt.o) (__floatdisf)
c:/program files (x86)/microchip/xc32/v1.21/bin/../lib/gcc/pic32mx/4.5.2/size\libgcc.a(_lshrdi3.o)
                              c:/program files (x86)/microchip/xc32/v1.21/bin/../lib/gcc/pic32mx/4.5.2/../../../../pic32mx/lib/size\libc.a(doprnt_cdnopsuxX.eo) (__lshrdi3)
c:/program files (x86)/microchip/xc32/v1.21/bin/../lib/gcc/pic32mx/4.5.2/size\libgcc.a(_floatundisf.o)
                              c:/program files (x86)/microchip/xc32/v1.21/bin/../lib/gcc/pic32mx/4.5.2/../../../../pic32mx/lib/size\libc.a(doprnt.o) (__floatundisf)
c:/program files (x86)/microchip/xc32/v1.21/bin/../lib/gcc/pic32mx/4.5.2/size\libgcc.a(_umoddi3.o)
                              c:/program files (x86)/microchip/xc32/v1.21/bin/../lib/gcc/pic32mx/4.5.2/../../../../pic32mx/lib/size\libc.a(doprnt_cdnopsuxX.eo) (__umoddi3)
c:/program files (x86)/microchip/xc32/v1.21/bin/../lib/gcc/pic32mx/4.5.2/size\libgcc.a(floatunsisf.o)
                              c:/program files (x86)/microchip/xc32/v1.21/bin/../lib/gcc/pic32mx/4.5.2/../../../../pic32mx/lib/size\libc.a(doprnt.o) (__floatunsisf)

Allocating common symbols
Common symbol       size              file

httpTransaction     0x4b0             build/WiFIG/production/_ext/1472/tcp6_demo_app.o
pingTimer           0x4               build/WiFIG/production/_ext/1472/ping_demo.o
serverIP            0x4               build/WiFIG/production/_ext/1472/tcp6_demo_app.o
j                   0x4               build/WiFIG/production/_ext/1472/tcp6_demo_app.o
stackNotifyHandle   0x4               build/WiFIG/production/_ext/1472/main_demo.o
TCPReadByte         0x1               build/WiFIG/production/_ext/1472/tcp6_demo_app.o
g_rxBufferLength    0x2               build/WiFIG/production/_ext/334706090/wf_mac_24g.o
dnsRes              0x4               build/WiFIG/production/_ext/1472/tcp6_demo_app.o
targetHostName      0x4               build/WiFIG/production/_ext/1472/ping_demo.o
targetMACAddr       0x6               build/WiFIG/production/_ext/1472/ping_demo.o
TCPInBuffer         0x1000            build/WiFIG/production/_ext/1472/tcp6_demo_app.o
mac_addr_string     0x10              build/WiFIG/production/_ext/1472/tcp6_demo_app.o
TCPOutBuffer        0x200             build/WiFIG/production/_ext/1472/tcp6_demo_app.o
mac_addr            0x6               build/WiFIG/production/_ext/1472/tcp6_demo_app.o
g_pNetIf            0x4               build/WiFIG/production/_ext/334706090/wf_mac_24g.o
mysrc               0x80              build/WiFIG/production/_ext/1472/tcp6_demo_app.o
myb64               0x80              build/WiFIG/production/_ext/1472/tcp6_demo_app.o
RawWindowState      0x2               build/WiFIG/production/_ext/334706090/wf_driver_raw_24g.o
iwconfigCb          0x3               build/WiFIG/production/_ext/334706090/wf_commands.o
temp                0x50              build/WiFIG/production/_ext/1472/tcp6_demo_app.o
g_easyConfigCtx     0x98              build/WiFIG/production/_ext/334706090/wf_easy_config.o
pingCount           0x1               build/WiFIG/production/_ext/1472/ping_demo.o
OutString           0x200             build/WiFIG/production/_ext/1472/tcp6_demo_app.o
clientTimer         0x4               build/WiFIG/production/_ext/1472/tcp6_demo_app.o
remoteNode          0xa               build/WiFIG/production/_ext/427700826/tcpip_manager.o
RawMoveState        0x2               build/WiFIG/production/_ext/334706090/wf_driver_com_24g.o
myNetHandle         0x4               build/WiFIG/production/_ext/1472/tcp6_demo_app.o
i                   0x4               build/WiFIG/production/_ext/1472/tcp6_demo_app.o
toggleLed           0x4               build/WiFIG/production/_ext/1472/tcp6_demo_app.o
g_softAPEvent       0x8               build/WiFIG/production/_ext/334706090/wf_event_handler.o
mySocketInfo        0x28              build/WiFIG/production/_ext/1472/tcp6_demo_app.o
targetAddressIPv4   0x4               build/WiFIG/production/_ext/1472/ping_demo.o
TCPIsPutReadyCnt    0x2               build/WiFIG/production/_ext/1472/tcp6_demo_app.o
myResourceState     0xb4              build/WiFIG/production/_ext/1472/tcp6_demo_app.o
wifi_ConfigData     0x8a              build/WiFIG/production/_ext/334706090/wf_configData.o
firstHopAddress     0x4               build/WiFIG/production/_ext/1472/ping_demo.o
lastBlock           0x40              build/WiFIG/production/_ext/101875047/hashes.o
serverPort          0x2               build/WiFIG/production/_ext/1472/tcp6_demo_app.o
g_powerSaveState    0x1               build/WiFIG/production/_ext/334706090/wf_driver_com_24g.o
TCPInBufPtr         0x4               build/WiFIG/production/_ext/1472/tcp6_demo_app.o
g_gratArpContext    0x8               build/WiFIG/production/_ext/334706090/wf_mac_24g.o
TCPInBufferIndex    0x4               build/WiFIG/production/_ext/1472/tcp6_demo_app.o
pNetIf              0x4               build/WiFIG/production/_ext/1472/ping_demo.o
hMac_softap_connect
                    0x4               build/WiFIG/production/_ext/334706090/wf_scan.o
HTTPReplyDelay      0x4               build/WiFIG/production/_ext/1472/tcp6_demo_app.o
HTTPReplyLineCnt    0x4               build/WiFIG/production/_ext/1472/tcp6_demo_app.o
g_savedPsPollContext
                    0x6               build/WiFIG/production/_ext/334706090/wf_power_save.o
mac_addr_ptr        0x4               build/WiFIG/production/_ext/1472/tcp6_demo_app.o

Microchip PIC32 Memory-Usage Report

kseg0 Program-Memory Usage
section                    address  length [bytes]      (dec)  Description
-------                 ----------  -------------------------  -----------
.text._TcpHandleSeg     0x9d000020         0x1778        6008   
.text.vfprintf          0x9d001798         0x15a8        5544   
.text.DNSClientTask     0x9d002d40         0x1144        4420   
.text.tcp6_demo_app_tas 0x9d003e84         0x10f0        4336   
.rodata                 0x9d004f74         0x1084        4228  Read-only const 
.text.DHCPTask          0x9d005ff8          0xa74        2676   
.text._TcpSend          0x9d006a6c          0xa40        2624   
.text                   0x9d0074ac          0x8ec        2284  App's exec code 
.text._vfprintf_cdnopsu 0x9d007d98          0x8b8        2232   
.text.TCPTick           0x9d008650          0x890        2192   
.rodata                 0x9d008ee0          0x7d4        2004  Read-only const 
.text._DHCPReceive      0x9d0096b4          0x748        1864   
.text.NBNSTask          0x9d009dfc          0x73c        1852   
.dinit                  0x9d00a538          0x6d0        1744   
.text._DHCPSend         0x9d00ac08          0x5c8        1480   
.text.SHA1HashBlock     0x9d00b1d0          0x4fc        1276   
.rodata                 0x9d00b6cc          0x4f4        1268  Read-only const 
.text.TCPIP_ANNOUNCE_Se 0x9d00bbc0          0x490        1168   
.text._TCPIP_HEAP_Free  0x9d00c050          0x490        1168   
.text.TCPIP_STACK_Init  0x9d00c4e0          0x464        1124   
.text                   0x9d00c944          0x8a0        2208  App's exec code 
.text.TCPIP_STACK_Bring 0x9d00d1e4          0x438        1080   
.text.TCPOpen           0x9d00d61c          0x420        1056   
.rodata                 0x9d00da3c          0x3fc        1020  Read-only const 
.text.ARPInitialize     0x9d00de38          0x3f4        1012   
.text._TcpFindMatchingS 0x9d00e22c          0x3e8        1000   
.text                   0x9d00e614          0x3dc         988  App's exec code 
.text.WFProcessMgmtIndi 0x9d00e9f0          0x3b0         944   
.text.SYS_Initialize    0x9d00eda0          0x3a8         936   
.text.FindMatchingSocke 0x9d00f148          0x39c         924   
.text.OutputSecurityMod 0x9d00f4e4          0x38c         908   
.text.TCPIP_STACK_Task  0x9d00f870          0x35c         860   
.text.main              0x9d00fbcc          0x358         856   
.text.UDPOpen           0x9d00ff24          0x330         816   
.text.TCPIP_HELPER_Stri 0x9d010254          0x31c         796   
.text.OutputConnectionF 0x9d010570          0x31c         796   
.text.ARPTask           0x9d01088c          0x310         784   
.text.TCPIP_IPV4_PutArr 0x9d010b9c          0x310         784   
.text.UDPInit           0x9d010eac          0x300         768   
.text.tcp6_demo_app_ini 0x9d0111ac          0x2c4         708   
.text.ICMPProcess       0x9d011470          0x2ac         684   
.text.TCPPutArray       0x9d01171c          0x2ac         684   
.text.Wifi_Connect      0x9d0119c8          0x284         644   
.text.UDPProcessIPv4    0x9d011c4c          0x278         632   
.text.SyncENCPtrRAWStat 0x9d011ec4          0x278         632   
.text.GetMaxSegSizeOpti 0x9d01213c          0x274         628   
.text.WriteAnalogRegist 0x9d0123b0          0x270         624   
.text.TCPIP_IPV4_Calcul 0x9d012620          0x268         616   
.text.TCPGetArray       0x9d012888          0x260         608   
.text.SYS_GENERATE_RAND 0x9d012ae8          0x25c         604   
.text.SYS_CLK_OscClockG 0x9d012d44          0x254         596   
.text.TCPIP_IPV4_CopyTx 0x9d012f98          0x250         592   
.text                   0x9d0131e8          0x248         584  App's exec code 
.text.LoadDefaultConfig 0x9d013430          0x244         580   
.text.ProcessTCPIPMacEv 0x9d013674          0x240         576   
.text.malloc            0x9d0138b4          0x240         576   
.text.ARPEntryRemoveNet 0x9d013af4          0x224         548   
.text.TCPIP_IPV4_GetDat 0x9d013d18          0x224         548   
.text.__floatdisf       0x9d013f3c          0x220         544   
.text.TCPInit           0x9d01415c          0x210         528   
.text.DHCPInit          0x9d01436c          0x204         516   
.text._TcpDisconnect    0x9d014570          0x204         516   
.text.UDPTask           0x9d014774          0x200         512   
.text.TCPIP_ANNOUNCE_Ta 0x9d014974          0x1f8         504   
.text.ARPProcess        0x9d014b6c          0x1f0         496   
.text.TCPIP_IPV4_Flush  0x9d014d5c          0x1ec         492   
.text._TCPIP_HEAP_Mallo 0x9d014f48          0x1e0         480   
.text.TCPProcessIPv4    0x9d015128          0x1dc         476   
.text.TCPIP_IPV4_IsTxPu 0x9d015304          0x1d8         472   
.text.UDPv4IsTxPutReady 0x9d0154dc          0x1d0         464   
.text._TCPIsPutReady    0x9d0156ac          0x1cc         460   
.text.UDPDeInit         0x9d015878          0x1cc         460   
.text.strtoul           0x9d015a44          0x1cc         460   
.text._TcpSocketSetIdle 0x9d015c10          0x1c8         456   
.text.MRF24W_MACGetHead 0x9d015dd8          0x1b8         440   
.text.WF_ProcessEvent   0x9d015f90          0x1b4         436   
.text._SystemTickIntHan 0x9d016144          0x1b0         432   
.text.isNotifyApp       0x9d0162f4          0x1a8         424   
.rodata                 0x9d01649c          0x1a8         424  Read-only const 
.text                   0x9d016644          0x1a0         416  App's exec code 
.text._TcpCloseSocket   0x9d0167e4          0x198         408   
.text.NBNSGetName       0x9d01697c          0x194         404   
.text._Sys_Ext1_Isr     0x9d016b10          0x190         400   
.text._Sys_Ext3_Isr     0x9d016ca0          0x190         400   
.text._Sys_CN_Isr       0x9d016e30          0x190         400   
.text.MRF24W_ChipReset  0x9d016fc0          0x190         400   
.text.RawMove           0x9d017150          0x190         400   
.text.TCPIP_HELPER_Stri 0x9d0172e0          0x18c         396   
.text.WaitForRawMoveCom 0x9d01746c          0x18c         396   
.text.UDPGetArray       0x9d0175f8          0x188         392   
.text.OutputBeaconTimeo 0x9d017780          0x188         392   
.text._OAHashFindBkt    0x9d017908          0x180         384   
.text.ARPIsResolved     0x9d017a88          0x178         376   
.text.TCPIP_IPV4_Alloca 0x9d017c00          0x178         376   
.text.TCPIP_HEAP_Create 0x9d017d78          0x178         376   
.text._ARPProbeAddress  0x9d017ef0          0x170         368   
.text.SpiChnOpen        0x9d018060          0x170         368   
.text.OAHashLookUpInser 0x9d0181d0          0x16c         364   
.text.UDPv4Flush        0x9d01833c          0x16c         364   
.text.WFHardwareInit    0x9d0184a8          0x168         360   
.text.RawSetIndex       0x9d018610          0x168         360   
.text                   0x9d018778          0x2d0         720  App's exec code 
.text.SYS_TICK_TimerDel 0x9d018a48          0x160         352   
.text.USART_INIT        0x9d018ba8          0x160         352   
.text.DRV_SPI_TxRx      0x9d018d08          0x160         352   
.text.DNSPutString      0x9d018e68          0x160         352   
.text.TCPIP_IPV4_Transm 0x9d018fc8          0x160         352   
.text.UDPBind           0x9d019128          0x160         352   
.text.WFEintHandler     0x9d019288          0x160         352   
.text.encodeblock       0x9d0193e8          0x160         352   
.text.ARP_SendIfPkt     0x9d019548          0x15c         348   
.text.TCPIP_IPV4_GetHea 0x9d0196a4          0x15c         348   
.text.ProcessInterruptS 0x9d019800          0x154         340   
.rodata                 0x9d019954          0x150         336  Read-only const 
.text._TCPIPStackIsLoca 0x9d019aa4          0x150         336   
.text.TCPIP_Helper_Calc 0x9d019bf4          0x150         336   
.text.OutputChannelList 0x9d019d44          0x150         336   
.text.scale             0x9d019e94          0x150         336   
.text._sbrk_init        0x9d019fe4          0x14c         332   
.text.TCPIP_STACK_DeIni 0x9d01a130          0x148         328   
.text.OutputConnectionT 0x9d01a278          0x148         328   
.text.OutputConnectionP 0x9d01a3c0          0x148         328   
.text.SendMgmtMsg       0x9d01a508          0x148         328   
.text.OAHashLookUp      0x9d01a650          0x144         324   
.text.UDPSocketSetNet   0x9d01a794          0x140         320   
.text._WF_OutputConnect 0x9d01a8d4          0x140         320   
.text.PowerSaveTask     0x9d01aa14          0x140         320   
.text.WF_SetMultiCastFi 0x9d01ab54          0x13c         316   
.text._ARPUpdateEntry   0x9d01ac90          0x138         312   
.text.TCPIP_IPV4_Queued 0x9d01adc8          0x138         312   
.text.UDPIsGetReady     0x9d01af00          0x138         312   
.text._general_exceptio 0x9d01b038          0x134         308   
.text.TCPIP_IPV4_Insert 0x9d01b16c          0x134         308   
.text.SetSecurity       0x9d01b2a0          0x134         308   
.text.uitoa             0x9d01b3d4          0x130         304   
.text.UDPSetBcastIPV4Ad 0x9d01b504          0x130         304   
.text.WF_ConfigDataLoad 0x9d01b634          0x12c         300   
.text.DNSBeginUsage     0x9d01b760          0x128         296   
.text.fputc             0x9d01b888          0x128         296   
.text.SYS_USERIO_Initia 0x9d01b9b0          0x124         292   
.text._TCPSendWinIncUpd 0x9d01bad4          0x124         292   
.text.WaitForMgmtRespon 0x9d01bbf8          0x124         292   
.text.strtol            0x9d01bd1c          0x124         292   
.text.TCPIP_IPV4_QueueP 0x9d01be40          0x120         288   
.text.UDPOpenServer     0x9d01bf60          0x120         288   
.text                   0x9d01c080          0x120         288  App's exec code 
.text.fround            0x9d01c1a0          0x120         288   
.text.SHA1AddData       0x9d01c2c0          0x11c         284   
.text.b64_encode        0x9d01c3dc          0x11c         284   
.text.TCPIP_IPV4_Initia 0x9d01c4f8          0x118         280   
.text.TCPIP_IPV4_PutHea 0x9d01c610          0x114         276   
.text.WiFiAsyncTask     0x9d01c724          0x110         272   
.text.WF_PsPollEnable   0x9d01c834          0x110         272   
.text._flsbuf           0x9d01c944          0x110         272   
.text._TcpSwapHeader    0x9d01ca54          0x10c         268   
.text.TCPIP_STACK_Bring 0x9d01cb60          0x108         264   
.text.OutputNetworkType 0x9d01cc68          0x108         264   
.text._DHCPClose        0x9d01cd70          0x104         260   
.text.WF_ScanContextGet 0x9d01ce74          0x104         260   
.rodata                 0x9d01cf78          0x208         520  Read-only const 
.text.hexatob           0x9d01d180          0x100         256   
.text.DisplayIPValue    0x9d01d280          0x100         256   
.text.WaitForMgmtRespon 0x9d01d380           0xfc         252   
.text._TCPIPStackAddres 0x9d01d47c           0xf8         248   
.text.SingleListRemoveN 0x9d01d574           0xf8         248   
.text.WF_Init           0x9d01d66c           0xf8         248   
.text.SYS_USERIO_Device 0x9d01d764           0xf4         244   
.text.UDPSetSourceIPAdd 0x9d01d858           0xf4         244   
.text.UDPSetDestination 0x9d01d94c           0xf4         244   
.text.WF_SecurityGet    0x9d01da40           0xf4         244   
.text.MRF24W_MACInitial 0x9d01db34           0xf4         244   
.text._ARPAddCompleteEn 0x9d01dc28           0xf0         240   
.text.UDPDiscard        0x9d01dd18           0xf0         240   
.text.WF_ScanContextSet 0x9d01de08           0xf0         240   
.text.NBNSPutName       0x9d01def8           0xec         236   
.text.TCPIsPutReady     0x9d01dfe4           0xec         236   
.text._TCPIP_HEAP_Callo 0x9d01e0d0           0xec         236   
.text.AllocateDataTxBuf 0x9d01e1bc           0xec         236   
.text.DNSIsResolved     0x9d01e2a8           0xe8         232   
.text.TCPIP_IPV4_PutUpp 0x9d01e390           0xe8         232   
.text.UDPSetRxOffset    0x9d01e478           0xe8         232   
.text.ProcessTCPIPTickE 0x9d01e560           0xe8         232   
.text.WF_GetDeviceInfo  0x9d01e648           0xe8         232   
.rodata                 0x9d01e730           0xe8         232  Read-only const 
.text.TCPIP_IPV4_ResetT 0x9d01e818           0xe4         228   
.text.TCPIP_IPV4_Alloca 0x9d01e8fc           0xe4         228   
.text.TCPDeInit         0x9d01e9e0           0xe4         228   
.text.TCPIP_HEAP_Delete 0x9d01eac4           0xe4         228   
.text.SYS_TICK_TimerCre 0x9d01eba8           0xe0         224   
.text._ARPSetEntry      0x9d01ec88           0xe0         224   
.text.ARPResolve        0x9d01ed68           0xe0         224   
.text.UDPPutArray       0x9d01ee48           0xe0         224   
.text.TCPIPMacEventCB   0x9d01ef28           0xe0         224   
.text.ProcessNotificati 0x9d01f008           0xe0         224   
.text._SYS_ERROR_PRINT  0x9d01f0e8           0xdc         220   
.text.ARPHashDeleteEntr 0x9d01f1c4           0xdc         220   
.text.DHCPConnectionHan 0x9d01f2a0           0xdc         220   
.text._TcpCleanup       0x9d01f37c           0xdc         220   
.text.TCPOpenClient     0x9d01f458           0xdc         220   
.text.TcpAllocateEpheme 0x9d01f534           0xdc         220   
.text.UDPOpenClient     0x9d01f610           0xdc         220   
.text.UdpAllocateEpheme 0x9d01f6ec           0xdc         220   
.text.OutputTxMode      0x9d01f7c8           0xdc         220   
.text.MACIFService      0x9d01f8a4           0xdc         220   
.text.DHCPEnable        0x9d01f980           0xd8         216   
.text.TCPIP_IPV4_GetPse 0x9d01fa58           0xd8         216   
.text._TCPIP_HEAP_Mallo 0x9d01fb30           0xd8         216   
.text._SYS_RANDOM_INIT  0x9d01fc08           0xd4         212   
.text.TCPIP_ANNOUNCE_In 0x9d01fcdc           0xd4         212   
.text._TcpAbort         0x9d01fdb0           0xd4         212   
.text.TCPClose          0x9d01fe84           0xd4         212   
.text.OutputDomain      0x9d01ff58           0xd4         212   
.text.AllocateMgmtTxBuf 0x9d02002c           0xd4         212   
.text                   0x9d020100           0xd4         212  App's exec code 
.text.SYS_USERIO_SetLED 0x9d0201d4           0xd0         208   
.text._ARPDeleteResourc 0x9d0202a4           0xd0         208   
.text.fnv_32_hash       0x9d020374           0xd0         208   
.text._TcpSocketInitial 0x9d020444           0xd0         208   
.text.UDPSetOptions     0x9d020514           0xd0         208   
.text.TCPIP_STACK_Regis 0x9d0205e4           0xd0         208   
.text.DhcpConfigTask    0x9d0206b4           0xd0         208   
.text.OutputDeviceInfo  0x9d020784           0xd0         208   
.text.MRF24W_MACPutHead 0x9d020854           0xd0         208   
.text.general_exception 0x9d020924           0xd0         208   
.rodata                 0x9d0209f4            0x4           4  Read-only const 
.rodata                 0x9d0209f8           0xd0         208  Read-only const 
.text.TCPIP_IPV4_SetPay 0x9d020ac8           0xcc         204   
.text.BSP_Initialize    0x9d020b94           0xc8         200   
.text.DNSRetry          0x9d020c5c           0xc8         200   
.text.DNSDiscardName    0x9d020d24           0xc8         200   
.text.UDPClose          0x9d020dec           0xc8         200   
.text.UDPSetTxOffset    0x9d020eb4           0xc8         200   
.text.InitNetConfig     0x9d020f7c           0xc8         200   
.text.TCPIP_Helper_Form 0x9d021044           0xc8         200   
.text.OutputDemoHeader  0x9d02110c           0xc8         200   
.text.HostInterruptRegI 0x9d0211d4           0xc8         200   
.text._DHCPEnable       0x9d02129c           0xc4         196   
.text.MRF24W_MACGetArra 0x9d021360           0xc4         196   
.text.SYS_TICK_Initiali 0x9d021424           0xc0         192   
.text.LowLevel_CPGetEle 0x9d0214e4           0xc0         192   
.text.ProcessMgmtRxMsg  0x9d0215a4           0xc0         192   
.rodata                 0x9d021664           0xbc         188  Read-only const 
.text.SYS_INT_DynamicRe 0x9d021720           0xbc         188   
.text._ARPRemoveEntry   0x9d0217dc           0xbc         188   
.text.OAHashRemoveAll   0x9d021898           0xbc         188   
.text.UDPDiscardNet     0x9d021954           0xbc         188   
.text.TCPIP_Helper_Stri 0x9d021a10           0xbc         188   
.text.LowLevel_CAGetEle 0x9d021acc           0xbc         188   
.text.MRF24W_MACEventSe 0x9d021b88           0xbc         188   
.text.OutputMacAddress  0x9d021c44           0xbc         188   
.text._SYS_DEBUG_INIT   0x9d021d00           0xb8         184   
.text._SYS_CONSOLE_INIT 0x9d021db8           0xb8         184   
.text.TCPv4AllocateTxPa 0x9d021e70           0xb8         184   
.text._TCPIsGetReady    0x9d021f28           0xb8         184   
.text.UDPGetTxCount     0x9d021fe0           0xb8         184   
.text.OutputScanType    0x9d022098           0xb8         184   
.text.RawGetByte        0x9d022150           0xb8         184   
.text.RawSetByte        0x9d022208           0xb8         184   
.text._TcpMac2RamCopy   0x9d0222c0           0xb4         180   
.text.UDPv4AllocateTxPa 0x9d022374           0xb4         180   
.text.UDPIsTxPutReady   0x9d022428           0xb4         180   
.text.WF_SsidSet        0x9d0224dc           0xb4         180   
.text.MRF24W_MACEventIn 0x9d022590           0xb4         180   
.text._mon_putc         0x9d022644           0xb4         180   
.text.TCPIP_ANNOUNCE_De 0x9d0226f8           0xb0         176   
.text._ARPRemoveCacheEn 0x9d0227a8           0xb0         176   
.text._ARPNotifyClients 0x9d022858           0xb0         176   
.text._Tcpv4AckFnc      0x9d022908           0xb0         176   
.text._TCPIPStackSetNet 0x9d0229b8           0xb0         176   
.text._TCPIPStackIsBcas 0x9d022a68           0xb0         176   
.text.HostInterrupt2Reg 0x9d022b18           0xb0         176   
.rodata                 0x9d022bc8           0xac         172  Read-only const 
.text.TCPIsConnected    0x9d022c74           0xac         172   
.text._SYS_ERROR        0x9d022d20           0xa8         168   
.text.ARPDeinitialize   0x9d022dc8           0xa8         168   
.text._TCPIPStackString 0x9d022e70           0xa8         168   
.text.WFConfigureLowPow 0x9d022f18           0xa8         168   
.text.WF_OutputConnecti 0x9d022fc0           0xa8         168   
.text                   0x9d023068           0xa8         168  App's exec code 
.text.SYS_USERIO_ReadIO 0x9d023110           0xa4         164   
.text.DNSResolve        0x9d0231b4           0xa4         164   
.text._ICMPAllocateTxPa 0x9d023258           0xa4         164   
.text.TCPIP_IPV4_DeInit 0x9d0232fc           0xa4         164   
.text._TCPIPStackNetByA 0x9d0233a0           0xa4         164   
.text.WF_ReconnectModeS 0x9d023444           0xa4         164   
.text.WF_LibInitialize  0x9d0234e8           0xa4         164   
.text._sbrk             0x9d02358c           0xa4         164   
.text.USART_GETS        0x9d023630           0xa0         160   
.text._DHCPDiscard      0x9d0236d0           0xa0         160   
.text._DHCPNotifyClient 0x9d023770           0xa0         160   
.text._UdpSocketDcpt    0x9d023810           0xa0         160   
.rodata                 0x9d0238b0           0xa0         160  Read-only const 
.text.strupr            0x9d023950           0x9c         156   
.text.ANNOUNCE_Notify   0x9d0239ec           0x9c         156   
.text.DHCPRegisterHandl 0x9d023a88           0x9c         156   
.text._TcpSocketKill    0x9d023b24           0x9c         156   
.text.TCPIsAvailablePor 0x9d023bc0           0x9c         156   
.text.UdpIsAvailablePor 0x9d023c5c           0x9c         156   
.text._TCPIPStackMacIdT 0x9d023cf8           0x9c         156   
.text.SingleListRemoveH 0x9d023d94           0x9c         156   
.text.SetWpsSecurity    0x9d023e30           0x9c         156   
.text.WF_SpiTxRx        0x9d023ecc           0x9c         156   
.text.OutputIpAddress   0x9d023f68           0x9c         156   
.text.GetSpiPortWithBit 0x9d024004           0x9c         156   
.text._SYS_DEBUG_OPEN   0x9d0240a0           0x98         152   
.text._SYS_ASSERT       0x9d024138           0x98         152   
.text._SYS_CONSOLE_OPEN 0x9d0241d0           0x98         152   
.text.TCPIP_STACK_Verif 0x9d024268           0x98         152   
.text.WF_ReconnectModeG 0x9d024300           0x98         152   
.text.WF_ChannelListGet 0x9d024398           0x98         152   
.text                   0x9d024430           0x98         152  App's exec code 
.text.TCP_PutArray      0x9d0244c8           0x94         148   
.text.SingleListAddTail 0x9d02455c           0x94         148   
.text.LowLevel_CPSetEle 0x9d0245f0           0x94         148   
.text.MRF24W_SetUserEve 0x9d024684           0x94         148   
.text.RawMountRxBuffer  0x9d024718           0x94         148   
.text.MRF24W_MACCalcRxC 0x9d0247ac           0x94         148   
.text.USART_PRINT       0x9d024840           0x90         144   
.text.DHCPIsBound       0x9d0248d0           0x90         144   
.text.TCPIP_IPV4_FreePa 0x9d024960           0x90         144   
.text.NBNSDeInit        0x9d0249f0           0x90         144   
.text.TCP_SetPayload    0x9d024a80           0x90         144   
.text._TCPIPStackIsNetB 0x9d024b10           0x90         144   
.text.OutputSsid        0x9d024ba0           0x90         144   
.text.ReadWFArray       0x9d024c30           0x90         144   
.text.SendGetParamMsg   0x9d024cc0           0x90         144   
.text.SwapARPPacket     0x9d024d50           0x8c         140   
.text.DHCPDisable       0x9d024ddc           0x8c         140   
.text.DNSClientInit     0x9d024e68           0x8c         140   
.text.SwapIPV4Header    0x9d024ef4           0x8c         140   
.text.UDPFlush          0x9d024f80           0x8c         140   
.text.UDPRemoteBind     0x9d02500c           0x8c         140   
.text.LowLevel_CASetEle 0x9d025098           0x8c         140   
.text.write             0x9d025124           0x8c         140   
.text.SHA1Initialize    0x9d0251b0           0x88         136   
.text._SysGetCDevEntry  0x9d025238           0x88         136   
.text.DHCPDeInit        0x9d0252c0           0x88         136   
.text.TCP_IsTxPutReady  0x9d025348           0x88         136   
.text.TCP_PutHeader     0x9d0253d0           0x88         136   
.text._TCPIPStackIpAddT 0x9d025458           0x88         136   
.text._TCPIPStackMACIdT 0x9d0254e0           0x88         136   
.text.TCPIP_STACK_NetBc 0x9d025568           0x88         136   
.text.Read16BitWFRegist 0x9d0255f0           0x88         136   
.text.Write16BitWFRegis 0x9d025678           0x88         136   
.text.WriteWFArray      0x9d025700           0x88         136   
.text.SendSetParamMsg   0x9d025788           0x88         136   
.text.LFSRSeedRand      0x9d025810           0x84         132   
.text._SYS_CONSOLE_PRIN 0x9d025894           0x84         132   
.text.OAHashInit        0x9d025918           0x84         132   
.text._TCPIP_HEAP_Callo 0x9d02599c           0x84         132   
.text.TcpipStackFindMod 0x9d025a20           0x84         132   
.text.TcpipStackFindMac 0x9d025aa4           0x84         132   
.text.mrf24w_MACPowerMo 0x9d025b28           0x84         132   
.text.MRF24W_ISR        0x9d025bac           0x84         132   
.rodata                 0x9d025c30           0x84         132  Read-only const 
.text.atoi              0x9d025cb4           0x84         132   
.text.TCPIP_IPV4_FlushD 0x9d025d38           0x80         128   
.text.TCP_IsTxReady     0x9d025db8           0x80         128   
.text.TCP_CopyTxPacketS 0x9d025e38           0x80         128   
.text._Udpv4AckFnc      0x9d025eb8           0x80         128   
.text.SetWpaSecurity    0x9d025f38           0x80         128   
.text.ValidateConfig    0x9d025fb8           0x80         128   
.text.ScratchMount      0x9d026038           0x80         128   
.text.TCP_Flush         0x9d0260b8           0x7c         124   
.text._TCPIPStackAddres 0x9d026134           0x7c         124   
.text.MRF24W_MACGetConf 0x9d0261b0           0x7c         124   
.text.DeallocateDataRxB 0x9d02622c           0x7c         124   
.text.LFSRRand          0x9d0262a8           0x78         120   
.text.SYS_TICK_TimerSet 0x9d026320           0x78         120   
.text.DHCPDeRegisterHan 0x9d026398           0x78         120   
.text.DNSClientDeInit   0x9d026410           0x78         120   
.text.SetWepSecurity    0x9d026488           0x78         120   
.text.ResetPll          0x9d026500           0x78         120   
.text.SendRAWDataFrame  0x9d026578           0x78         120   
.text.MRF24W_MACFlush   0x9d0265f0           0x78         120   
.text.rand              0x9d026668           0x78         120   
.text.strstr            0x9d0266e0           0x78         120   
.text.SYS_RANDOM_ADD    0x9d026758           0x74         116   
.text.TCPIP_IPV4_SetTxB 0x9d0267cc           0x74         116   
.text.TCP_GetUpperLayer 0x9d026840           0x74         116   
.text.TCP_IsPacketQueue 0x9d0268b4           0x74         116   
.text.TCP_ResetTransmit 0x9d026928           0x74         116   
.text._TCPIP_HEAP_FreeD 0x9d02699c           0x74         116   
.text.UDPIsConnected    0x9d026a10           0x74         116   
.text._TCPIPStackIsAddr 0x9d026a84           0x74         116   
.text.WF_PsPollDisable  0x9d026af8           0x74         116   
.text.EnsureWFisAwake   0x9d026b6c           0x74         116   
.text.RawRead           0x9d026be0           0x74         116   
.text.RawWrite          0x9d026c54           0x74         116   
.text.RawInit           0x9d026cc8           0x74         116   
.text.SYS_INT_SourceRes 0x9d026d3c           0x70         112   
.text._ARPDeleteCache   0x9d026dac           0x70         112   
.text.ICMPInitialize    0x9d026e1c           0x70         112   
.text.TCPIP_IPV4_Single 0x9d026e8c           0x70         112   
.text.NBNSInit          0x9d026efc           0x70         112   
.text.TCPPutString      0x9d026f6c           0x70         112   
.text.WF_Connect        0x9d026fdc           0x70         112   
.text.MRF24W_MACOpen    0x9d02704c           0x70         112   
.text.Write8BitWFRegist 0x9d0270bc           0x70         112   
.text._ARPRefreshEntry  0x9d02712c           0x6c         108   
.text._TCPGetRxFIFOFree 0x9d027198           0x6c         108   
.text.TcpClientIpv4Remo 0x9d027204           0x6c         108   
.text.TCPIP_HEAP_FreeSi 0x9d027270           0x6c         108   
.rodata                 0x9d0272dc           0x6c         108  Read-only const 
.text.ProcessTCPIPMacGe 0x9d027348           0x6c         108   
.text.TCPIP_STACK_NetBI 0x9d0273b4           0x6c         108   
.text.TCPIP_STACK_Filte 0x9d027420           0x6c         108   
.text.TCPIP_Notificatio 0x9d02748c           0x6c         108   
.text.SendPowerModeMsg  0x9d0274f8           0x6c         108   
.text.Read8BitWFRegiste 0x9d027564           0x6c         108   
.text.MRF24W_MACInit    0x9d0275d0           0x6c         108   
.text.OAHashGetEntry    0x9d02763c           0x68         104   
.text.TCPIP_IPV4_FreePa 0x9d0276a4           0x68         104   
.text._TcpSocketBind    0x9d02770c           0x68         104   
.text._TcpSocketChk     0x9d027774           0x68         104   
.text._TcpFlush         0x9d0277dc           0x68         104   
.text._UdpSocketBind    0x9d027844           0x68         104   
.text.MACPutHeader      0x9d0278ac           0x68         104   
.text.TCPIP_STACK_NetNa 0x9d027914           0x68         104   
.text.TCPIP_Notificatio 0x9d02797c           0x68         104   
.rodata                 0x9d0279e4           0x68         104  Read-only const 
.text.MRF24W_MACEventDe 0x9d027a4c           0x68         104   
.text.RawCalculateCheck 0x9d027ab4           0x68         104   
.text.MRF24W_MACPutArra 0x9d027b1c           0x68         104   
.rodata                 0x9d027b84           0x68         104  Read-only const 
.text.TCPIP_IPV4_GetDat 0x9d027bec           0x64         100   
.text._TCPIPStackIsNetL 0x9d027c50           0x64         100   
.text.TCPIP_Notificatio 0x9d027cb4           0x64         100   
.text.WF_CPCreate       0x9d027d18           0x64         100   
.text.MRF24W_MACEventSe 0x9d027d7c           0x64         100   
.text._sprintf_cdnopsux 0x9d027de0           0x64         100   
.text.USART_PUTC        0x9d027e44           0x60          96   
.text.ICMPDeinitialize  0x9d027ea4           0x60          96   
.text.TCPIP_IPV4_SetRxB 0x9d027f04           0x60          96   
.text.TCP_FreePacket    0x9d027f64           0x60          96   
.text.MACCalcRxChecksum 0x9d027fc4           0x60          96   
.rodata                 0x9d028024           0x60          96  Read-only const 
.text.ConfigureSpiMRF24 0x9d028084           0x60          96   
.text.MRF24W_MACDeiniti 0x9d0280e4           0x60          96   
.text.mrf24w_MACSetRXHa 0x9d028144           0x60          96   
.text.WiFi_EintTask     0x9d0281a4           0x60          96   
.text.SYS_INT_SourceDis 0x9d028204           0x5c          92   
.text.SYS_INT_PriorityS 0x9d028260           0x5c          92   
.text.SYS_INT_Subpriori 0x9d0282bc           0x5c          92   
.text._DHCPCleanup      0x9d028318           0x5c          92   
.text.OAHashRemoveEntry 0x9d028374           0x5c          92   
.text.TCPFlush          0x9d0283d0           0x5c          92   
.text.MACGetArray       0x9d02842c           0x5c          92   
.text.MACPutArray       0x9d028488           0x5c          92   
.text.MACEventSetNotify 0x9d0284e4           0x5c          92   
.text._TCPIPStackNetAdd 0x9d028540           0x5c          92   
.text._TCPIPStackNetMas 0x9d02859c           0x5c          92   
.text._TCPIPStackNetMac 0x9d0285f8           0x5c          92   
.text.SetListenInterval 0x9d028654           0x5c          92   
.text.SetDtimInterval   0x9d0286b0           0x5c          92   
.text.WF_SecurityWepSet 0x9d02870c           0x5c          92   
.text.WF_SecurityWpaSet 0x9d028768           0x5c          92   
.text.WF_SecurityWpsSet 0x9d0287c4           0x5c          92   
.text.WF_EintIsPending  0x9d028820           0x5c          92   
.text.mrf24w_MACPutHead 0x9d02887c           0x5c          92   
.text.SignalWiFiConnect 0x9d0288d8           0x5c          92   
.text.WF_StartGratuitou 0x9d028934           0x5c          92   
.text.MRF24W_MACIsTxRea 0x9d028990           0x5c          92   
.text.SYS_INT_SourceEna 0x9d0289ec           0x58          88   
.text.USART_OPEN        0x9d028a44           0x58          88   
.text.USART_GETC        0x9d028a9c           0x58          88   
.text.WaitForDataByte   0x9d028af4           0x58          88   
.text.ARPHashKeyHash    0x9d028b4c           0x58          88   
.text._TcpipHeapHandleT 0x9d028ba4           0x58          88   
.text.TCPIP_STACK_IxToN 0x9d028bfc           0x58          88   
.text._TCPIPStackIsNetU 0x9d028c54           0x58          88   
.text.WF_NetworkTypeSet 0x9d028cac           0x58          88   
.text.mrf24w_MACCalcRxC 0x9d028d04           0x58          88   
.text.MRF24W_MACCalcIPB 0x9d028d5c           0x58          88   
.text.SYS_INT_SourceSta 0x9d028db4           0x54          84   
.text._ICMPAckPacket    0x9d028e08           0x54          84   
.text._TcpDiscardTx     0x9d028e5c           0x54          84   
.text._UdpSocketInit    0x9d028eb0           0x54          84   
.text.UDPPut            0x9d028f04           0x54          84   
.text.MACGetHeader      0x9d028f58           0x54          84   
.text.MACSetReadPtrInRx 0x9d028fac           0x54          84   
.text.MACCalcIPBufferCh 0x9d029000           0x54          84   
.text.MACEventSetNotify 0x9d029054           0x54          84   
.text.MACEventAck       0x9d0290a8           0x54          84   
.text._TCPIPStackAddres 0x9d0290fc           0x54          84   
.text._TCPIPStackAddres 0x9d029150           0x54          84   
.text.mrf24w_MACDeiniti 0x9d0291a4           0x54          84   
.text.GratuitousArpHand 0x9d0291f8           0x54          84   
.text._vsnprintf_cdnops 0x9d02924c           0x54          84   
.text.vsnprintf         0x9d0292a0           0x54          84   
.text._SYS_CONSOLE_MESS 0x9d0292f4           0x50          80   
.text._TCPIP_AnnounceCl 0x9d029344           0x50          80   
.text.ARPHashKeyCompare 0x9d029394           0x50          80   
.text._DNSReleaseSocket 0x9d0293e4           0x50          80   
.text.WF_EintInit       0x9d029434           0x50          80   
.text.WF_SpiInit        0x9d029484           0x50          80   
.text.mrf24w_MACEventSe 0x9d0294d4           0x50          80   
.text.MRF24W_GetTraffic 0x9d029524           0x50          80   
.text.MRF24W_GetMgmtEve 0x9d029574           0x50          80   
.text.SignalDHCPSuccess 0x9d0295c4           0x50          80   
.text.InitGratuitousArp 0x9d029614           0x50          80   
.text.MRF24W_MACSetWrit 0x9d029664           0x50          80   
.text.MRF24W_MACSetRead 0x9d0296b4           0x50          80   
.text.MRF24W_MACSetBase 0x9d029704           0x50          80   
.text.StackNotification 0x9d029754           0x50          80   
.text.DRV_SPI_Initializ 0x9d0297a4           0x4c          76   
.text.TCPGet            0x9d0297f0           0x4c          76   
.text.UDPGet            0x9d02983c           0x4c          76   
.text.MACSetWritePtr    0x9d029888           0x4c          76   
.text.MACSetReadPtr     0x9d0298d4           0x4c          76   
.text.MACEventGetPendin 0x9d029920           0x4c          76   
.text.WF_ChannelListSet 0x9d02996c           0x4c          76   
.text.WF_EintEnable     0x9d0299b8           0x4c          76   
.text.DhcpEventHandler  0x9d029a04           0x4c          76   
.text.mrf24w_MACPutArra 0x9d029a50           0x4c          76   
.text.mrf24w_MACGetArra 0x9d029a9c           0x4c          76   
.text.MRF24W_MACEventAc 0x9d029ae8           0x4c          76   
.text.SendRAWManagement 0x9d029b34           0x4c          76   
.text.ScratchUnmount    0x9d029b80           0x4c          76   
.text.MRF24W_MACSetRead 0x9d029bcc           0x4c          76   
.text.INTEnable         0x9d029c18           0x4c          76   
.text                   0x9d029c64           0x4c          76  App's exec code 
.text.SYS_CLK_Periphera 0x9d029cb0           0x48          72   
.text.ARPHashKeyCopy    0x9d029cf8           0x48          72   
.text.DNSEndUsage       0x9d029d40           0x48          72   
.text.TCPIP_IPV4_SetSou 0x9d029d88           0x48          72   
.text.TCPIP_STACK_NetAd 0x9d029dd0           0x48          72   
.text.TCPIP_STACK_NetMa 0x9d029e18           0x48          72   
.text.isEventNotifyBitS 0x9d029e60           0x48          72   
.rodata                 0x9d029ea8           0x48          72  Read-only const 
.text.mrf24w_MACCalcIPB 0x9d029ef0           0x48          72   
.text.mrf24w_MACEventSe 0x9d029f38           0x48          72   
.text.mrf24w_MACEventCl 0x9d029f80           0x48          72   
.text.mrf24w_MACEventAc 0x9d029fc8           0x48          72   
.text.MRF24W_MACEventCl 0x9d02a010           0x48          72   
.text.OutputPowerSaveMo 0x9d02a058           0x48          72   
.text.WFEnableMRF24WMod 0x9d02a0a0           0x48          72   
.rodata                 0x9d02a0e8           0x48          72  Read-only const 
.text._DefaultInterrupt 0x9d02a130           0x48          72   
.text.sbrk              0x9d02a178           0x48          72   
.text.SYS_CLK_ClockGet  0x9d02a1c0           0x44          68   
.text.USART_DATA_RDY    0x9d02a204           0x44          68   
.text.TCPIP_IPV4_SetPac 0x9d02a248           0x44          68   
.text.MACClose          0x9d02a28c           0x44          68   
.text.MACDiscardRx      0x9d02a2d0           0x44          68   
.text.MACIsTxReady      0x9d02a314           0x44          68   
.text.MACFlush          0x9d02a358           0x44          68   
.text.MACCheckLink      0x9d02a39c           0x44          68   
.text.MACGetTxBaseAddr  0x9d02a3e0           0x44          68   
.text.TCPIP_STACK_NetHa 0x9d02a424           0x44          68   
.text._TCPIPStackNetIx  0x9d02a468           0x44          68   
.text._TCPIPStackSetGat 0x9d02a4ac           0x44          68   
.text._TCPIPStackSetPri 0x9d02a4f0           0x44          68   
.text._TCPIPStackSetSec 0x9d02a534           0x44          68   
.text._TCPIPStackNetToM 0x9d02a578           0x44          68   
.text.SingleListInit    0x9d02a5bc           0x44          68   
.text.WF_ConnectContext 0x9d02a600           0x44          68   
.rodata                 0x9d02a644           0x44          68  Read-only const 
.text.WF_NetworkTypeGet 0x9d02a688           0x44          68   
.text.WF_WepKeyTypeGet  0x9d02a6cc           0x44          68   
.text.mrf24w_MACGetHead 0x9d02a710           0x44          68   
.text.mrf24w_MACSetRead 0x9d02a754           0x44          68   
.text.WiFi_GratuitousAr 0x9d02a798           0x44          68   
.text.MRF24W_MACProcess 0x9d02a7dc           0x44          68   
.text.RawGetMgmtRxBuffe 0x9d02a820           0x44          68   
.text.WF_SetWPATimeout  0x9d02a864           0x44          68   
.text.WF_SetTxMode      0x9d02a8a8           0x44          68   
.text.WF_SetTxDataConfi 0x9d02a8ec           0x44          68   
.text.strncat           0x9d02a930           0x44          68   
.text.strncmp           0x9d02a974           0x44          68   
.text                   0x9d02a9b8           0x44          68  App's exec code 
.text.TCPIP_IPV4_Task   0x9d02a9fc           0x40          64   
.text.UDPResetHeader    0x9d02aa3c           0x40          64   
.text.WF_CASetEventNoti 0x9d02aa7c           0x40          64   
.text.WF_SecurityOpenSe 0x9d02aabc           0x40          64   
.text.MRF24W_MACConnect 0x9d02aafc           0x40          64   
.text.mrf24w_MACEventGe 0x9d02ab3c           0x40          64   
.text.DeallocateMgmtRxB 0x9d02ab7c           0x40          64   
.text.MRF24W_MACDiscard 0x9d02abbc           0x40          64   
.text.WF_GetTxMode      0x9d02abfc           0x40          64   
.text.WF_MacAddressSet  0x9d02ac3c           0x40          64   
.text.WF_MacAddressGet  0x9d02ac7c           0x40          64   
.text.WF_RegionalDomain 0x9d02acbc           0x40          64   
.text.SpiChnDataRdy     0x9d02acfc           0x40          64   
.text._ARPDeleteClients 0x9d02ad3c           0x3c          60   
.text.ARPTmoHandler     0x9d02ad78           0x3c          60   
.text.TCPIP_IPV4_GetUpp 0x9d02adb4           0x3c          60   
.text.TCPIP_IPV4_GetPay 0x9d02adf0           0x3c          60   
.rodata                 0x9d02ae2c           0x3c          60  Read-only const 
.text.WifiAsyncSetEvent 0x9d02ae68           0x3c          60   
.text.mrf24w_MACSetWrit 0x9d02aea4           0x3c          60   
.text.mrf24w_MACSetRead 0x9d02aee0           0x3c          60   
.text.mrf24w_MACSetBase 0x9d02af1c           0x3c          60   
.text.PORTSetPinsDigita 0x9d02af58           0x3c          60   
.text.PORTSetPinsDigita 0x9d02af94           0x3c          60   
.text                   0x9d02afd0           0x38          56  App's exec code 
.text._OAHashProbeStep  0x9d02b008           0x38          56   
.rodata                 0x9d02b040           0x38          56  Read-only const 
.text.RenewDhcp         0x9d02b078           0x38          56   
.text.mrf24w_MACClose   0x9d02b0b0           0x38          56   
.rodata                 0x9d02b0e8           0x70         112  Read-only const 
.text.INTSetVectorPrior 0x9d02b158           0x38          56   
.text.INTSetVectorSubPr 0x9d02b190           0x38          56   
.text.TCPIP_IPV4_SetDes 0x9d02b1c8           0x34          52   
.text.TCPIP_IPV4_GetDes 0x9d02b1fc           0x34          52   
.text.TCPIP_IPV4_GetSou 0x9d02b230           0x34          52   
.text.ProcessTCPIPMacEr 0x9d02b264           0x34          52   
.rodata                 0x9d02b298           0x34          52  Read-only const 
.text.WF_EintIsDisabled 0x9d02b2cc           0x34          52   
.text.WF_DeInit         0x9d02b300           0x34          52   
.text.WF_SpiDisableChip 0x9d02b334           0x34          52   
.text.mrf24w_MACGetRead 0x9d02b368           0x34          52   
.text.mrf24w_MACIsTxRea 0x9d02b39c           0x34          52   
.text.mrf24w_MACFlush   0x9d02b3d0           0x34          52   
.text.mrf24w_MACDiscard 0x9d02b404           0x34          52   
.text.mrf24w_MACCheckLi 0x9d02b438           0x34          52   
.text.SetNetworkConfig  0x9d02b46c           0x34          52   
.rodata                 0x9d02b4a0           0x34          52  Read-only const 
.text.INTEnableSystemMu 0x9d02b4d4           0x34          52   
.text.SYS_Tasks         0x9d02b508           0x30          48   
.text.SYS_USERIO_Tasks  0x9d02b538           0x30          48   
.text.TCPIP_IPV4_TmoHan 0x9d02b568           0x30          48   
.text._TcpTmoHandler    0x9d02b598           0x30          48   
.text.TCPIP_STACK_TickH 0x9d02b5c8           0x30          48   
.text.SetEventNotificat 0x9d02b5f8           0x30          48   
.text.SetLogicalConnect 0x9d02b628           0x30          48   
.text.SetAppPowerSaveMo 0x9d02b658           0x30          48   
.text.WF_GetPowerSaveSt 0x9d02b688           0x30          48   
.text.SetPowerSaveState 0x9d02b6b8           0x30          48   
.text.WF_SpiEnableChipS 0x9d02b6e8           0x30          48   
.rodata                 0x9d02b718           0x30          48  Read-only const 
.text.MRF24W_MACCheckLi 0x9d02b748           0x30          48   
.text.WFStateNotify     0x9d02b778           0x30          48   
.text.strcat            0x9d02b7a8           0x30          48   
.text.SYS_WDT_Clear     0x9d02b7d8           0x2c          44   
.text.TCPIP_ANNOUNCE_Ta 0x9d02b804           0x2c          44   
.text.ARPTaskPending    0x9d02b830           0x2c          44   
.text.TCPIP_IPV4_TaskPe 0x9d02b85c           0x2c          44   
.text.TCPTaskPending    0x9d02b888           0x2c          44   
.text.WF_EintDisable    0x9d02b8b4           0x2c          44   
.text.WiFiAsyncTaskPend 0x9d02b8e0           0x2c          44   
.rodata                 0x9d02b90c           0x2c          44  Read-only const 
.text.MRF24W_MACEventGe 0x9d02b938           0x2c          44   
.text.strchr            0x9d02b964           0x2c          44   
.text._stub_sbd_memlayo 0x9d02b990           0x2c          44   
.rodata                 0x9d02b9bc           0x28          40  Read-only const 
.text.DHCPServerDisable 0x9d02b9e4           0x28          40   
.text.DHCPServerEnable  0x9d02ba0c           0x28          40   
.text.ZCLLEnable        0x9d02ba34           0x28          40   
.text.SetSleepNeeded    0x9d02ba5c           0x28          40   
.text.mrf24w_MACGetTxBa 0x9d02ba84           0x28          40   
.text.WF_OutputConnecti 0x9d02baac           0x28          40   
.text.SetDhcpProgressSt 0x9d02bad4           0x28          40   
.text.SignalMgmtConfirm 0x9d02bafc           0x28          40   
.text.WiFiMemory_read   0x9d02bb24           0x28          40   
.text.INTClearFlag      0x9d02bb4c           0x28          40   
.text.SYS_DRIVERS_Initi 0x9d02bb74           0x24          36   
.text.TCPIP_STACK_GetDe 0x9d02bb98           0x24          36   
.text.TCPIP_STACK_Netwo 0x9d02bbbc           0x24          36   
.text.GetEventNotificat 0x9d02bbe0           0x24          36   
.text.WFisConnected     0x9d02bc04           0x24          36   
.text.GetWiFiNetworkTyp 0x9d02bc28           0x24          36   
.text.WifiAsyncClearAll 0x9d02bc4c           0x24          36   
.text.WF_ConfigDataSave 0x9d02bc70           0x24          36   
.text.isSleepNeeded     0x9d02bc94           0x24          36   
.text.ClearSleepNeeded  0x9d02bcb8           0x24          36   
.text.GetAppPowerSaveMo 0x9d02bcdc           0x24          36   
.text.InitPowerSaveTask 0x9d02bd00           0x24          36   
.text.isDhcpInProgress  0x9d02bd24           0x24          36   
.text.GetReadPtrRawWind 0x9d02bd48           0x24          36   
.text.GetNetworkConfig  0x9d02bd6c           0x24          36   
.text.MRF24W_MACGetRead 0x9d02bd90           0x24          36   
.text._snprintf_cdnopsu 0x9d02bdb4           0x24          36   
.text.toupper           0x9d02bdd8           0x24          36   
.rodata                 0x9d02bdfc           0x20          32  Read-only const 
.text.SetEapSecurity    0x9d02be1c           0x20          32   
.text.MRF24W_MACPowerDo 0x9d02be3c           0x20          32   
.text.MRF24W_MACPowerUp 0x9d02be5c           0x20          32   
.text.SpiChnReadC       0x9d02be7c           0x20          32   
.text.SpiChnWriteC      0x9d02be9c           0x20          32   
.text.SpiChnTxBuffEmpty 0x9d02bebc           0x20          32   
.text.INTRestoreInterru 0x9d02bedc           0x1c          28   
.text.free              0x9d02bef8           0x1c          28   
.text.srand             0x9d02bf14           0x1c          28   
.text.CheKseg0CacheOn   0x9d02bf30           0x18          24   
.text                   0x9d02bf48           0x18          24  App's exec code 
.rodata                 0x9d02bf60           0x24          36  Read-only const 
.text.OpenCoreTimer     0x9d02bf84            0xc          12   
.text._bootstrap_except 0x9d02bf90            0xc          12   
.text.INTDisableInterru 0x9d02bf9c            0x8           8   
.text.INTEnableInterrup 0x9d02bfa4            0x8           8   
.text._on_reset         0x9d02bfac            0x8           8   
.text._on_bootstrap     0x9d02bfb4            0x8           8   
.rodata                 0x9d02bfbc            0x8           8  Read-only const 
      Total kseg0_program_mem used  :     0x2bfa4      180132  34.4% of 0x80000

kseg0 Boot-Memory Usage
section                    address  length [bytes]      (dec)  Description
-------                 ----------  -------------------------  -----------
         Total kseg0_boot_mem used  :           0           0  <1% of 0x970

Exception-Memory Usage 
section                    address  length [bytes]      (dec)  Description
-------                 ----------  -------------------------  -----------
.app_excpt              0x9fc01180           0x10          16  General-Exception 
.vector_0               0x9fc01200            0x8           8  Interrupt Vector 0 
.vector_1               0x9fc01220            0x8           8  Interrupt Vector 1 
.vector_2               0x9fc01240            0x8           8  Interrupt Vector 2 
.vector_3               0x9fc01260            0x8           8  Interrupt Vector 3 
.vector_4               0x9fc01280            0x8           8  Interrupt Vector 4 
.vector_5               0x9fc012a0            0x8           8  Interrupt Vector 5 
.vector_6               0x9fc012c0            0x8           8  Interrupt Vector 6 
.vector_7               0x9fc012e0            0x8           8  Interrupt Vector 7 
.vector_8               0x9fc01300            0x8           8  Interrupt Vector 8 
.vector_9               0x9fc01320            0x8           8  Interrupt Vector 9 
.vector_10              0x9fc01340            0x8           8  Interrupt Vector 10 
.vector_11              0x9fc01360            0x8           8  Interrupt Vector 11 
.vector_12              0x9fc01380            0x8           8  Interrupt Vector 12 
.vector_13              0x9fc013a0            0x8           8  Interrupt Vector 13 
.vector_14              0x9fc013c0            0x8           8  Interrupt Vector 14 
.vector_15              0x9fc013e0            0x8           8  Interrupt Vector 15 
.vector_16              0x9fc01400            0x8           8  Interrupt Vector 16 
.vector_17              0x9fc01420            0x8           8  Interrupt Vector 17 
.vector_18              0x9fc01440            0x8           8  Interrupt Vector 18 
.vector_19              0x9fc01460            0x8           8  Interrupt Vector 19 
.vector_20              0x9fc01480            0x8           8  Interrupt Vector 20 
.vector_21              0x9fc014a0            0x8           8  Interrupt Vector 21 
.vector_22              0x9fc014c0            0x8           8  Interrupt Vector 22 
.vector_23              0x9fc014e0            0x8           8  Interrupt Vector 23 
.vector_24              0x9fc01500            0x8           8  Interrupt Vector 24 
.vector_25              0x9fc01520            0x8           8  Interrupt Vector 25 
.vector_26              0x9fc01540            0x8           8  Interrupt Vector 26 
.vector_27              0x9fc01560            0x8           8  Interrupt Vector 27 
.vector_28              0x9fc01580            0x8           8  Interrupt Vector 28 
.vector_29              0x9fc015a0            0x8           8  Interrupt Vector 29 
.vector_30              0x9fc015c0            0x8           8  Interrupt Vector 30 
.vector_31              0x9fc015e0            0x8           8  Interrupt Vector 31 
.vector_32              0x9fc01600            0x8           8  Interrupt Vector 32 
.vector_33              0x9fc01620            0x8           8  Interrupt Vector 33 
.vector_34              0x9fc01640            0x8           8  Interrupt Vector 34 
.vector_35              0x9fc01660            0x8           8  Interrupt Vector 35 
.vector_36              0x9fc01680            0x8           8  Interrupt Vector 36 
.vector_37              0x9fc016a0            0x8           8  Interrupt Vector 37 
.vector_38              0x9fc016c0            0x8           8  Interrupt Vector 38 
.vector_39              0x9fc016e0            0x8           8  Interrupt Vector 39 
.vector_40              0x9fc01700            0x8           8  Interrupt Vector 40 
.vector_41              0x9fc01720            0x8           8  Interrupt Vector 41 
.vector_42              0x9fc01740            0x8           8  Interrupt Vector 42 
.vector_43              0x9fc01760            0x8           8  Interrupt Vector 43 
.vector_44              0x9fc01780            0x8           8  Interrupt Vector 44 
.vector_45              0x9fc017a0            0x8           8  Interrupt Vector 45 
.vector_46              0x9fc017c0            0x8           8  Interrupt Vector 46 
.vector_47              0x9fc017e0            0x8           8  Interrupt Vector 47 
.vector_48              0x9fc01800            0x8           8  Interrupt Vector 48 
.vector_49              0x9fc01820            0x8           8  Interrupt Vector 49 
.vector_50              0x9fc01840            0x8           8  Interrupt Vector 50 
.vector_51              0x9fc01860            0x8           8  Interrupt Vector 51 
.vector_52              0x9fc01880            0x8           8  Interrupt Vector 52 
.vector_53              0x9fc018a0            0x8           8  Interrupt Vector 53 
.vector_54              0x9fc018c0            0x8           8  Interrupt Vector 54 
.vector_55              0x9fc018e0            0x8           8  Interrupt Vector 55 
.vector_56              0x9fc01900            0x8           8  Interrupt Vector 56 
.vector_57              0x9fc01920            0x8           8  Interrupt Vector 57 
.vector_58              0x9fc01940            0x8           8  Interrupt Vector 58 
.vector_59              0x9fc01960            0x8           8  Interrupt Vector 59 
.vector_60              0x9fc01980            0x8           8  Interrupt Vector 60 
.vector_61              0x9fc019a0            0x8           8  Interrupt Vector 61 
.vector_62              0x9fc019c0            0x8           8  Interrupt Vector 62 
.vector_63              0x9fc019e0            0x8           8  Interrupt Vector 63 
          Total exception_mem used  :       0x210         528  12.9% of 0x1000

kseg1 Boot-Memory Usage
section                    address  length [bytes]      (dec)  Description
-------                 ----------  -------------------------  -----------
.reset                  0xbfc00000          0x1f4         500  Reset handler 
.bev_excpt              0xbfc00380           0x10          16  BEV-Exception 
         Total kseg1_boot_mem used  :       0x204         516  44.2% of 0x490
        --------------------------------------------------------------------------
         Total Program Memory used  :     0x2c3b8      181176  34.1% of 0x81e00
        --------------------------------------------------------------------------


kseg1 Data-Memory Usage
section                    address  length [bytes]      (dec)  Description
-------                 ----------  -------------------------  -----------
.eh_frame               0xa0000000           0x30          48   
.sdata                  0xa0000030          0x1bc         444  Small init data 
.sbss                   0xa00001ec          0x310         784  Small uninit data 
.bss                    0xa00004fc         0x1bc4        7108  Uninitialized data 
.data                   0xa00020c0          0x208         520  Initialized data 
.bss                    0xa00022c8          0x128         296  Uninitialized data 
         Total kseg1_data_mem used  :      0x23f0        9200  7.0% of 0x20000
        --------------------------------------------------------------------------
            Total Data Memory used  :      0x23f0        9200  7.0% of 0x20000
        --------------------------------------------------------------------------


Dynamic Data-Memory Reservation
section                    address  length [bytes]      (dec)  Description
-------                 ----------  -------------------------  -----------
heap                    0xa00023f8         0x5208       21000  Reserved for heap 
stack                   0xa0007618        0x189e0      100832  Reserved for stack 

        --------------------------------------------------------------------------

Discarded input sections

 .data          0x00000000        0x0 c:/program files (x86)/microchip/xc32/v1.21/bin/../lib/gcc/pic32mx/4.5.2/../../../../pic32mx/lib/size/crt0.o
 .bss           0x00000000        0x0 c:/program files (x86)/microchip/xc32/v1.21/bin/../lib/gcc/pic32mx/4.5.2/../../../../pic32mx/lib/size/crt0.o
 .pdr           0x00000000       0xa0 c:/program files (x86)/microchip/xc32/v1.21/bin/../lib/gcc/pic32mx/4.5.2/../../../../pic32mx/lib/size/crt0.o
 .text          0x00000000        0x0 build/WiFIG/production/_ext/1293749816/bsp.o
 .data          0x00000000        0x0 build/WiFIG/production/_ext/1293749816/bsp.o
 .bss           0x00000000        0x0 build/WiFIG/production/_ext/1293749816/bsp.o
 .reginfo       0x00000000       0x18 build/WiFIG/production/_ext/1293749816/bsp.o
 .pdr           0x00000000       0x20 build/WiFIG/production/_ext/1293749816/bsp.o
 .text          0x00000000        0x0 build/WiFIG/production/_ext/101875047/hashes.o
 .data          0x00000000        0x0 build/WiFIG/production/_ext/101875047/hashes.o
 .bss           0x00000000        0x0 build/WiFIG/production/_ext/101875047/hashes.o
 .reginfo       0x00000000       0x18 build/WiFIG/production/_ext/101875047/hashes.o
 .pdr           0x00000000      0x120 build/WiFIG/production/_ext/101875047/hashes.o
 .text.HashAddData
                0x00000000       0x94 build/WiFIG/production/_ext/101875047/hashes.o
 .rodata        0x00000000      0x140 build/WiFIG/production/_ext/101875047/hashes.o
 .text.MD5Initialize
                0x00000000       0x74 build/WiFIG/production/_ext/101875047/hashes.o
 .text.MD5AddData
                0x00000000      0x110 build/WiFIG/production/_ext/101875047/hashes.o
 .text.MD5HashBlock
                0x00000000      0x2bc build/WiFIG/production/_ext/101875047/hashes.o
 .text.MD5Calculate
                0x00000000      0x2a8 build/WiFIG/production/_ext/101875047/hashes.o
 .text.SHA1Calculate
                0x00000000      0x4b8 build/WiFIG/production/_ext/101875047/hashes.o
 .text          0x00000000        0x0 build/WiFIG/production/_ext/101875047/lfsr.o
 .data          0x00000000        0x0 build/WiFIG/production/_ext/101875047/lfsr.o
 .bss           0x00000000        0x0 build/WiFIG/production/_ext/101875047/lfsr.o
 .reginfo       0x00000000       0x18 build/WiFIG/production/_ext/101875047/lfsr.o
 .pdr           0x00000000       0x40 build/WiFIG/production/_ext/101875047/lfsr.o
 .text          0x00000000        0x0 build/WiFIG/production/_ext/101875047/big_int.o
 .data          0x00000000        0x0 build/WiFIG/production/_ext/101875047/big_int.o
 .bss           0x00000000        0x0 build/WiFIG/production/_ext/101875047/big_int.o
 .reginfo       0x00000000       0x18 build/WiFIG/production/_ext/101875047/big_int.o
 .pdr           0x00000000      0x1a0 build/WiFIG/production/_ext/101875047/big_int.o
 .text.BigInt   0x00000000       0x70 build/WiFIG/production/_ext/101875047/big_int.o
 .text.BigIntZero
                0x00000000       0x68 build/WiFIG/production/_ext/101875047/big_int.o
 .text.BigIntMod
                0x00000000      0x220 build/WiFIG/production/_ext/101875047/big_int.o
 .text.BigIntCompare
                0x00000000      0x16c build/WiFIG/production/_ext/101875047/big_int.o
 .text.BigIntMagnitudeDifference
                0x00000000       0x58 build/WiFIG/production/_ext/101875047/big_int.o
 .text.BigIntMagnitude
                0x00000000       0x50 build/WiFIG/production/_ext/101875047/big_int.o
 .text.BigIntMSB
                0x00000000       0xac build/WiFIG/production/_ext/101875047/big_int.o
 .text.BigIntMultiply
                0x00000000       0x94 build/WiFIG/production/_ext/101875047/big_int.o
 .text.BigIntSquare
                0x00000000       0x74 build/WiFIG/production/_ext/101875047/big_int.o
 .text.BigIntAdd
                0x00000000       0x74 build/WiFIG/production/_ext/101875047/big_int.o
 .text.BigIntSubtract
                0x00000000       0x74 build/WiFIG/production/_ext/101875047/big_int.o
 .text.BigIntCopy
                0x00000000       0x70 build/WiFIG/production/_ext/101875047/big_int.o
 .text.BigIntSwapEndianness
                0x00000000       0x9c build/WiFIG/production/_ext/101875047/big_int.o
 .text          0x00000000      0x400 build/WiFIG/production/_ext/101875047/big_int_helper_c32.o
 .data          0x00000000        0x0 build/WiFIG/production/_ext/101875047/big_int_helper_c32.o
 .bss           0x00000000       0x20 build/WiFIG/production/_ext/101875047/big_int_helper_c32.o
 .reginfo       0x00000000       0x18 build/WiFIG/production/_ext/101875047/big_int_helper_c32.o
 .pdr           0x00000000      0x100 build/WiFIG/production/_ext/101875047/big_int_helper_c32.o
 .text          0x00000000        0x0 build/WiFIG/production/_ext/101875047/helpers.o
 .data          0x00000000        0x0 build/WiFIG/production/_ext/101875047/helpers.o
 .bss           0x00000000        0x0 build/WiFIG/production/_ext/101875047/helpers.o
 .reginfo       0x00000000       0x18 build/WiFIG/production/_ext/101875047/helpers.o
 .pdr           0x00000000      0x100 build/WiFIG/production/_ext/101875047/helpers.o
 .text.btohexa_high
                0x00000000       0x64 build/WiFIG/production/_ext/101875047/helpers.o
 .text.btohexa_low
                0x00000000       0x64 build/WiFIG/production/_ext/101875047/helpers.o
 .text.strnchr  0x00000000       0xb4 build/WiFIG/production/_ext/101875047/helpers.o
 .text.strncpy_m
                0x00000000      0x10c build/WiFIG/production/_ext/101875047/helpers.o
 .text.stricmppgm2ram
                0x00000000      0x16c build/WiFIG/production/_ext/101875047/helpers.o
 .text          0x00000000        0x0 build/WiFIG/production/_ext/1472/berkeley_tcp_client_demo.o
 .data          0x00000000        0x0 build/WiFIG/production/_ext/1472/berkeley_tcp_client_demo.o
 .bss           0x00000000        0x0 build/WiFIG/production/_ext/1472/berkeley_tcp_client_demo.o
 .reginfo       0x00000000       0x18 build/WiFIG/production/_ext/1472/berkeley_tcp_client_demo.o
 .pdr           0x00000000        0x0 build/WiFIG/production/_ext/1472/berkeley_tcp_client_demo.o
 .text          0x00000000        0x0 build/WiFIG/production/_ext/1472/berkeley_tcp_server_demo.o
 .data          0x00000000        0x0 build/WiFIG/production/_ext/1472/berkeley_tcp_server_demo.o
 .bss           0x00000000        0x0 build/WiFIG/production/_ext/1472/berkeley_tcp_server_demo.o
 .reginfo       0x00000000       0x18 build/WiFIG/production/_ext/1472/berkeley_tcp_server_demo.o
 .pdr           0x00000000        0x0 build/WiFIG/production/_ext/1472/berkeley_tcp_server_demo.o
 .text          0x00000000        0x0 build/WiFIG/production/_ext/1472/berkeley_udp_client_demo.o
 .data          0x00000000        0x0 build/WiFIG/production/_ext/1472/berkeley_udp_client_demo.o
 .bss           0x00000000        0x0 build/WiFIG/production/_ext/1472/berkeley_udp_client_demo.o
 .reginfo       0x00000000       0x18 build/WiFIG/production/_ext/1472/berkeley_udp_client_demo.o
 .pdr           0x00000000        0x0 build/WiFIG/production/_ext/1472/berkeley_udp_client_demo.o
 .text          0x00000000        0x0 build/WiFIG/production/_ext/1472/generic_tcp_client.o
 .data          0x00000000        0x0 build/WiFIG/production/_ext/1472/generic_tcp_client.o
 .bss           0x00000000        0x0 build/WiFIG/production/_ext/1472/generic_tcp_client.o
 .reginfo       0x00000000       0x18 build/WiFIG/production/_ext/1472/generic_tcp_client.o
 .pdr           0x00000000        0x0 build/WiFIG/production/_ext/1472/generic_tcp_client.o
 .text          0x00000000        0x0 build/WiFIG/production/_ext/1472/generic_tcp_server.o
 .data          0x00000000        0x0 build/WiFIG/production/_ext/1472/generic_tcp_server.o
 .bss           0x00000000        0x0 build/WiFIG/production/_ext/1472/generic_tcp_server.o
 .reginfo       0x00000000       0x18 build/WiFIG/production/_ext/1472/generic_tcp_server.o
 .pdr           0x00000000        0x0 build/WiFIG/production/_ext/1472/generic_tcp_server.o
 .text          0x00000000        0x0 build/WiFIG/production/_ext/1472/ping_demo.o
 .data          0x00000000        0x0 build/WiFIG/production/_ext/1472/ping_demo.o
 .bss           0x00000000        0x0 build/WiFIG/production/_ext/1472/ping_demo.o
 .reginfo       0x00000000       0x18 build/WiFIG/production/_ext/1472/ping_demo.o
 .pdr           0x00000000       0x60 build/WiFIG/production/_ext/1472/ping_demo.o
 .sbss          0x00000000        0x8 build/WiFIG/production/_ext/1472/ping_demo.o
 .sdata         0x00000000        0x4 build/WiFIG/production/_ext/1472/ping_demo.o
 .text.Ping4    0x00000000       0x90 build/WiFIG/production/_ext/1472/ping_demo.o
 .text.PingDemoTask
                0x00000000       0x20 build/WiFIG/production/_ext/1472/ping_demo.o
 .rodata        0x00000000        0xc build/WiFIG/production/_ext/1472/ping_demo.o
 .text.PingProcessIPv4
                0x00000000      0x188 build/WiFIG/production/_ext/1472/ping_demo.o
 .text          0x00000000        0x0 build/WiFIG/production/_ext/1472/smtp_demo.o
 .data          0x00000000        0x0 build/WiFIG/production/_ext/1472/smtp_demo.o
 .bss           0x00000000        0x0 build/WiFIG/production/_ext/1472/smtp_demo.o
 .reginfo       0x00000000       0x18 build/WiFIG/production/_ext/1472/smtp_demo.o
 .pdr           0x00000000        0x0 build/WiFIG/production/_ext/1472/smtp_demo.o
 .text          0x00000000        0x0 build/WiFIG/production/_ext/365611741/system_services.o
 .data          0x00000000        0x0 build/WiFIG/production/_ext/365611741/system_services.o
 .bss           0x00000000        0x0 build/WiFIG/production/_ext/365611741/system_services.o
 .reginfo       0x00000000       0x18 build/WiFIG/production/_ext/365611741/system_services.o
 .pdr           0x00000000      0x420 build/WiFIG/production/_ext/365611741/system_services.o
 .text.SYS_Reboot
                0x00000000       0x18 build/WiFIG/production/_ext/365611741/system_services.o
 .text.SYS_RTCC_Initialize
                0x00000000       0xf4 build/WiFIG/production/_ext/365611741/system_services.o
 .text.SYS_RTCC_DateGet
                0x00000000       0x4c build/WiFIG/production/_ext/365611741/system_services.o
 .text.SYS_RTCC_TimeGet
                0x00000000       0x4c build/WiFIG/production/_ext/365611741/system_services.o
 .text.SYS_TICK_MsDelay
                0x00000000       0x8c build/WiFIG/production/_ext/365611741/system_services.o
 .text.SYS_TICK_UsDelay
                0x00000000       0x8c build/WiFIG/production/_ext/365611741/system_services.o
 .text.SYS_TICK_NsDelay
                0x00000000       0xa4 build/WiFIG/production/_ext/365611741/system_services.o
 .text          0x00000000        0x0 build/WiFIG/production/_ext/365611741/system_debug.o
 .data          0x00000000        0x0 build/WiFIG/production/_ext/365611741/system_debug.o
 .bss           0x00000000        0x0 build/WiFIG/production/_ext/365611741/system_debug.o
 .reginfo       0x00000000       0x18 build/WiFIG/production/_ext/365611741/system_debug.o
 .pdr           0x00000000      0x220 build/WiFIG/production/_ext/365611741/system_debug.o
 .text.__sys_assert
                0x00000000       0x3c build/WiFIG/production/_ext/365611741/system_debug.o
 .text._SYS_PRINT
                0x00000000       0xcc build/WiFIG/production/_ext/365611741/system_debug.o
 .text._SYS_CONSOLE_DATA_RDY
                0x00000000       0x48 build/WiFIG/production/_ext/365611741/system_debug.o
 .text._SYS_CONSOLE_GETC
                0x00000000       0x48 build/WiFIG/production/_ext/365611741/system_debug.o
 .text._SYS_CONSOLE_PUTC
                0x00000000       0x54 build/WiFIG/production/_ext/365611741/system_debug.o
 .text._SYS_CONSOLE_GETLINE
                0x00000000       0x58 build/WiFIG/production/_ext/365611741/system_debug.o
 .text          0x00000000        0x0 build/WiFIG/production/_ext/365611741/system_random.o
 .data          0x00000000        0x0 build/WiFIG/production/_ext/365611741/system_random.o
 .reginfo       0x00000000       0x18 build/WiFIG/production/_ext/365611741/system_random.o
 .pdr           0x00000000       0xa0 build/WiFIG/production/_ext/365611741/system_random.o
 .text.SYS_RANDOM_GET
                0x00000000       0x84 build/WiFIG/production/_ext/365611741/system_random.o
 .text._SYS_RANDOM_DE_INIT
                0x00000000       0x20 build/WiFIG/production/_ext/365611741/system_random.o
 .text          0x00000000        0x0 build/WiFIG/production/_ext/365611741/system_command.o
 .data          0x00000000        0x0 build/WiFIG/production/_ext/365611741/system_command.o
 .bss           0x00000000        0x0 build/WiFIG/production/_ext/365611741/system_command.o
 .reginfo       0x00000000       0x18 build/WiFIG/production/_ext/365611741/system_command.o
 .pdr           0x00000000        0x0 build/WiFIG/production/_ext/365611741/system_command.o
 .text          0x00000000        0x0 build/WiFIG/production/_ext/365611741/system_userio.o
 .data          0x00000000        0x0 build/WiFIG/production/_ext/365611741/system_userio.o
 .reginfo       0x00000000       0x18 build/WiFIG/production/_ext/365611741/system_userio.o
 .pdr           0x00000000      0x100 build/WiFIG/production/_ext/365611741/system_userio.o
 .text.SYS_USERIO_ButtonGetBitMap
                0x00000000       0x68 build/WiFIG/production/_ext/365611741/system_userio.o
 .text.SYS_USERIO_ButtonGet
                0x00000000      0x140 build/WiFIG/production/_ext/365611741/system_userio.o
 .text.SYS_USERIO_ButtonsTest
                0x00000000       0xa8 build/WiFIG/production/_ext/365611741/system_userio.o
 .text          0x00000000        0x0 build/WiFIG/production/_ext/97638081/sys_fs.o
 .data          0x00000000        0x0 build/WiFIG/production/_ext/97638081/sys_fs.o
 .bss           0x00000000        0x0 build/WiFIG/production/_ext/97638081/sys_fs.o
 .reginfo       0x00000000       0x18 build/WiFIG/production/_ext/97638081/sys_fs.o
 .pdr           0x00000000        0x0 build/WiFIG/production/_ext/97638081/sys_fs.o
 .text          0x00000000        0x0 build/WiFIG/production/_ext/97638081/mpfs2.o
 .data          0x00000000        0x0 build/WiFIG/production/_ext/97638081/mpfs2.o
 .bss           0x00000000        0x0 build/WiFIG/production/_ext/97638081/mpfs2.o
 .reginfo       0x00000000       0x18 build/WiFIG/production/_ext/97638081/mpfs2.o
 .pdr           0x00000000        0x0 build/WiFIG/production/_ext/97638081/mpfs2.o
 .text          0x00000000        0x0 build/WiFIG/production/_ext/792872985/usart.o
 .data          0x00000000        0x0 build/WiFIG/production/_ext/792872985/usart.o
 .bss           0x00000000        0x0 build/WiFIG/production/_ext/792872985/usart.o
 .reginfo       0x00000000       0x18 build/WiFIG/production/_ext/792872985/usart.o
 .pdr           0x00000000       0xe0 build/WiFIG/production/_ext/792872985/usart.o
 .text          0x00000000        0x0 build/WiFIG/production/_ext/792872985/lcd.o
 .data          0x00000000        0x0 build/WiFIG/production/_ext/792872985/lcd.o
 .bss           0x00000000        0x0 build/WiFIG/production/_ext/792872985/lcd.o
 .reginfo       0x00000000       0x18 build/WiFIG/production/_ext/792872985/lcd.o
 .pdr           0x00000000        0x0 build/WiFIG/production/_ext/792872985/lcd.o
 .text          0x00000000        0x0 build/WiFIG/production/_ext/792872985/drv_spi.o
 .data          0x00000000        0x0 build/WiFIG/production/_ext/792872985/drv_spi.o
 .bss           0x00000000        0x0 build/WiFIG/production/_ext/792872985/drv_spi.o
 .reginfo       0x00000000       0x18 build/WiFIG/production/_ext/792872985/drv_spi.o
 .pdr           0x00000000       0x60 build/WiFIG/production/_ext/792872985/drv_spi.o
 .text          0x00000000        0x0 build/WiFIG/production/_ext/792872985/db_appio.o
 .data          0x00000000        0x0 build/WiFIG/production/_ext/792872985/db_appio.o
 .bss           0x00000000        0x0 build/WiFIG/production/_ext/792872985/db_appio.o
 .reginfo       0x00000000       0x18 build/WiFIG/production/_ext/792872985/db_appio.o
 .pdr           0x00000000        0x0 build/WiFIG/production/_ext/792872985/db_appio.o
 .text          0x00000000        0x0 build/WiFIG/production/_ext/792872985/spi_ram.o
 .data          0x00000000        0x0 build/WiFIG/production/_ext/792872985/spi_ram.o
 .bss           0x00000000        0x0 build/WiFIG/production/_ext/792872985/spi_ram.o
 .reginfo       0x00000000       0x18 build/WiFIG/production/_ext/792872985/spi_ram.o
 .pdr           0x00000000        0x0 build/WiFIG/production/_ext/792872985/spi_ram.o
 .text          0x00000000        0x0 build/WiFIG/production/_ext/792872985/spi_eeprom.o
 .data          0x00000000        0x0 build/WiFIG/production/_ext/792872985/spi_eeprom.o
 .bss           0x00000000        0x0 build/WiFIG/production/_ext/792872985/spi_eeprom.o
 .reginfo       0x00000000       0x18 build/WiFIG/production/_ext/792872985/spi_eeprom.o
 .pdr           0x00000000        0x0 build/WiFIG/production/_ext/792872985/spi_eeprom.o
 .text          0x00000000        0x0 build/WiFIG/production/_ext/792872985/spi_flash.o
 .data          0x00000000        0x0 build/WiFIG/production/_ext/792872985/spi_flash.o
 .bss           0x00000000        0x0 build/WiFIG/production/_ext/792872985/spi_flash.o
 .reginfo       0x00000000       0x18 build/WiFIG/production/_ext/792872985/spi_flash.o
 .pdr           0x00000000        0x0 build/WiFIG/production/_ext/792872985/spi_flash.o
 .text          0x00000000        0x0 build/WiFIG/production/_ext/792872985/drv_media.o
 .data          0x00000000        0x0 build/WiFIG/production/_ext/792872985/drv_media.o
 .bss           0x00000000        0x0 build/WiFIG/production/_ext/792872985/drv_media.o
 .reginfo       0x00000000       0x18 build/WiFIG/production/_ext/792872985/drv_media.o
 .pdr           0x00000000        0x0 build/WiFIG/production/_ext/792872985/drv_media.o
 .text          0x00000000        0x0 build/WiFIG/production/_ext/427700826/tcpip_announce.o
 .data          0x00000000        0x0 build/WiFIG/production/_ext/427700826/tcpip_announce.o
 .bss           0x00000000        0x0 build/WiFIG/production/_ext/427700826/tcpip_announce.o
 .reginfo       0x00000000       0x18 build/WiFIG/production/_ext/427700826/tcpip_announce.o
 .pdr           0x00000000       0xe0 build/WiFIG/production/_ext/427700826/tcpip_announce.o
 .text          0x00000000        0x0 build/WiFIG/production/_ext/427700826/http2.o
 .data          0x00000000        0x0 build/WiFIG/production/_ext/427700826/http2.o
 .bss           0x00000000        0x0 build/WiFIG/production/_ext/427700826/http2.o
 .reginfo       0x00000000       0x18 build/WiFIG/production/_ext/427700826/http2.o
 .pdr           0x00000000        0x0 build/WiFIG/production/_ext/427700826/http2.o
 .text          0x00000000        0x0 build/WiFIG/production/_ext/427700826/arcfour.o
 .data          0x00000000        0x0 build/WiFIG/production/_ext/427700826/arcfour.o
 .bss           0x00000000        0x0 build/WiFIG/production/_ext/427700826/arcfour.o
 .reginfo       0x00000000       0x18 build/WiFIG/production/_ext/427700826/arcfour.o
 .pdr           0x00000000        0x0 build/WiFIG/production/_ext/427700826/arcfour.o
 .text          0x00000000        0x0 build/WiFIG/production/_ext/427700826/arp.o
 .data          0x00000000        0x0 build/WiFIG/production/_ext/427700826/arp.o
 .bss           0x00000000        0x0 build/WiFIG/production/_ext/427700826/arp.o
 .reginfo       0x00000000       0x18 build/WiFIG/production/_ext/427700826/arp.o
 .pdr           0x00000000      0x480 build/WiFIG/production/_ext/427700826/arp.o
 .text.ARPRegisterHandler
                0x00000000       0x9c build/WiFIG/production/_ext/427700826/arp.o
 .text.ARPDeRegisterHandler
                0x00000000       0x78 build/WiFIG/production/_ext/427700826/arp.o
 .text.ARPProbe
                0x00000000       0x5c build/WiFIG/production/_ext/427700826/arp.o
 .text.ARPEntrySet
                0x00000000      0x24c build/WiFIG/production/_ext/427700826/arp.o
 .text.ARPEntryGet
                0x00000000       0x7c build/WiFIG/production/_ext/427700826/arp.o
 .text.ARPEntryRemove
                0x00000000       0xd0 build/WiFIG/production/_ext/427700826/arp.o
 .text.ARPEntryRemoveAll
                0x00000000       0x90 build/WiFIG/production/_ext/427700826/arp.o
 .text.ARPEntryQuery
                0x00000000      0x1a8 build/WiFIG/production/_ext/427700826/arp.o
 .text.ARPCacheGetEntriesNo
                0x00000000      0x15c build/WiFIG/production/_ext/427700826/arp.o
 .text.ARPCacheSetThreshold
                0x00000000       0xcc build/WiFIG/production/_ext/427700826/arp.o
 .text          0x00000000        0x0 build/WiFIG/production/_ext/427700826/berkeley_api.o
 .data          0x00000000        0x0 build/WiFIG/production/_ext/427700826/berkeley_api.o
 .bss           0x00000000        0x0 build/WiFIG/production/_ext/427700826/berkeley_api.o
 .reginfo       0x00000000       0x18 build/WiFIG/production/_ext/427700826/berkeley_api.o
 .pdr           0x00000000        0x0 build/WiFIG/production/_ext/427700826/berkeley_api.o
 .text          0x00000000        0x0 build/WiFIG/production/_ext/427700826/dhcp.o
 .data          0x00000000        0x0 build/WiFIG/production/_ext/427700826/dhcp.o
 .bss           0x00000000        0x0 build/WiFIG/production/_ext/427700826/dhcp.o
 .reginfo       0x00000000       0x18 build/WiFIG/production/_ext/427700826/dhcp.o
 .pdr           0x00000000      0x260 build/WiFIG/production/_ext/427700826/dhcp.o
 .text.DHCPIsEnabled
                0x00000000       0x64 build/WiFIG/production/_ext/427700826/dhcp.o
 .text.DHCPIsServerDetected
                0x00000000       0x90 build/WiFIG/production/_ext/427700826/dhcp.o
 .text.DHCPSetRequestTimeout
                0x00000000       0x2c build/WiFIG/production/_ext/427700826/dhcp.o
 .text          0x00000000        0x0 build/WiFIG/production/_ext/427700826/dhcps.o
 .data          0x00000000        0x0 build/WiFIG/production/_ext/427700826/dhcps.o
 .bss           0x00000000        0x0 build/WiFIG/production/_ext/427700826/dhcps.o
 .reginfo       0x00000000       0x18 build/WiFIG/production/_ext/427700826/dhcps.o
 .pdr           0x00000000       0x60 build/WiFIG/production/_ext/427700826/dhcps.o
 .text.DHCPServerIsEnabled
                0x00000000       0x28 build/WiFIG/production/_ext/427700826/dhcps.o
 .text          0x00000000        0x0 build/WiFIG/production/_ext/427700826/dns.o
 .data          0x00000000        0x0 build/WiFIG/production/_ext/427700826/dns.o
 .bss           0x00000000        0x0 build/WiFIG/production/_ext/427700826/dns.o
 .reginfo       0x00000000       0x18 build/WiFIG/production/_ext/427700826/dns.o
 .pdr           0x00000000      0x160 build/WiFIG/production/_ext/427700826/dns.o
 .text          0x00000000        0x0 build/WiFIG/production/_ext/427700826/dnss.o
 .data          0x00000000        0x0 build/WiFIG/production/_ext/427700826/dnss.o
 .bss           0x00000000        0x0 build/WiFIG/production/_ext/427700826/dnss.o
 .reginfo       0x00000000       0x18 build/WiFIG/production/_ext/427700826/dnss.o
 .pdr           0x00000000        0x0 build/WiFIG/production/_ext/427700826/dnss.o
 .text          0x00000000        0x0 build/WiFIG/production/_ext/427700826/dyn_dns.o
 .data          0x00000000        0x0 build/WiFIG/production/_ext/427700826/dyn_dns.o
 .bss           0x00000000        0x0 build/WiFIG/production/_ext/427700826/dyn_dns.o
 .reginfo       0x00000000       0x18 build/WiFIG/production/_ext/427700826/dyn_dns.o
 .pdr           0x00000000        0x0 build/WiFIG/production/_ext/427700826/dyn_dns.o
 .text          0x00000000        0x0 build/WiFIG/production/_ext/427700826/enc28_mac.o
 .data          0x00000000        0x0 build/WiFIG/production/_ext/427700826/enc28_mac.o
 .bss           0x00000000        0x0 build/WiFIG/production/_ext/427700826/enc28_mac.o
 .reginfo       0x00000000       0x18 build/WiFIG/production/_ext/427700826/enc28_mac.o
 .pdr           0x00000000        0x0 build/WiFIG/production/_ext/427700826/enc28_mac.o
 .text          0x00000000        0x0 build/WiFIG/production/_ext/427700826/enc28j60.o
 .data          0x00000000        0x0 build/WiFIG/production/_ext/427700826/enc28j60.o
 .bss           0x00000000        0x0 build/WiFIG/production/_ext/427700826/enc28j60.o
 .reginfo       0x00000000       0x18 build/WiFIG/production/_ext/427700826/enc28j60.o
 .pdr           0x00000000        0x0 build/WiFIG/production/_ext/427700826/enc28j60.o
 .text          0x00000000        0x0 build/WiFIG/production/_ext/427700826/encs24j600.o
 .data          0x00000000        0x0 build/WiFIG/production/_ext/427700826/encs24j600.o
 .bss           0x00000000        0x0 build/WiFIG/production/_ext/427700826/encs24j600.o
 .reginfo       0x00000000       0x18 build/WiFIG/production/_ext/427700826/encs24j600.o
 .pdr           0x00000000        0x0 build/WiFIG/production/_ext/427700826/encs24j600.o
 .text          0x00000000        0x0 build/WiFIG/production/_ext/427700826/encx24_mac.o
 .data          0x00000000        0x0 build/WiFIG/production/_ext/427700826/encx24_mac.o
 .bss           0x00000000        0x0 build/WiFIG/production/_ext/427700826/encx24_mac.o
 .reginfo       0x00000000       0x18 build/WiFIG/production/_ext/427700826/encx24_mac.o
 .pdr           0x00000000        0x0 build/WiFIG/production/_ext/427700826/encx24_mac.o
 .text          0x00000000        0x0 build/WiFIG/production/_ext/427700826/eth_pic32_ext_phy.o
 .data          0x00000000        0x0 build/WiFIG/production/_ext/427700826/eth_pic32_ext_phy.o
 .bss           0x00000000        0x0 build/WiFIG/production/_ext/427700826/eth_pic32_ext_phy.o
 .reginfo       0x00000000       0x18 build/WiFIG/production/_ext/427700826/eth_pic32_ext_phy.o
 .pdr           0x00000000        0x0 build/WiFIG/production/_ext/427700826/eth_pic32_ext_phy.o
 .text          0x00000000        0x0 build/WiFIG/production/_ext/427700826/eth_pic32_ext_phy_dp83848.o
 .data          0x00000000        0x0 build/WiFIG/production/_ext/427700826/eth_pic32_ext_phy_dp83848.o
 .bss           0x00000000        0x0 build/WiFIG/production/_ext/427700826/eth_pic32_ext_phy_dp83848.o
 .reginfo       0x00000000       0x18 build/WiFIG/production/_ext/427700826/eth_pic32_ext_phy_dp83848.o
 .pdr           0x00000000        0x0 build/WiFIG/production/_ext/427700826/eth_pic32_ext_phy_dp83848.o
 .text          0x00000000        0x0 build/WiFIG/production/_ext/427700826/eth_pic32_int_mac.o
 .data          0x00000000        0x0 build/WiFIG/production/_ext/427700826/eth_pic32_int_mac.o
 .bss           0x00000000        0x0 build/WiFIG/production/_ext/427700826/eth_pic32_int_mac.o
 .reginfo       0x00000000       0x18 build/WiFIG/production/_ext/427700826/eth_pic32_int_mac.o
 .pdr           0x00000000        0x0 build/WiFIG/production/_ext/427700826/eth_pic32_int_mac.o
 .text          0x00000000        0x0 build/WiFIG/production/_ext/427700826/ftp.o
 .data          0x00000000        0x0 build/WiFIG/production/_ext/427700826/ftp.o
 .bss           0x00000000        0x0 build/WiFIG/production/_ext/427700826/ftp.o
 .reginfo       0x00000000       0x18 build/WiFIG/production/_ext/427700826/ftp.o
 .pdr           0x00000000        0x0 build/WiFIG/production/_ext/427700826/ftp.o
 .text          0x00000000        0x0 build/WiFIG/production/_ext/427700826/hash_fnv.o
 .data          0x00000000        0x0 build/WiFIG/production/_ext/427700826/hash_fnv.o
 .bss           0x00000000        0x0 build/WiFIG/production/_ext/427700826/hash_fnv.o
 .reginfo       0x00000000       0x18 build/WiFIG/production/_ext/427700826/hash_fnv.o
 .pdr           0x00000000       0x40 build/WiFIG/production/_ext/427700826/hash_fnv.o
 .text.fnv_32a_hash
                0x00000000       0xd0 build/WiFIG/production/_ext/427700826/hash_fnv.o
 .text          0x00000000        0x0 build/WiFIG/production/_ext/427700826/hash_tbl.o
 .data          0x00000000        0x0 build/WiFIG/production/_ext/427700826/hash_tbl.o
 .bss           0x00000000        0x0 build/WiFIG/production/_ext/427700826/hash_tbl.o
 .reginfo       0x00000000       0x18 build/WiFIG/production/_ext/427700826/hash_tbl.o
 .pdr           0x00000000      0x100 build/WiFIG/production/_ext/427700826/hash_tbl.o
 .text          0x00000000        0x0 build/WiFIG/production/_ext/427700826/icmp.o
 .data          0x00000000        0x0 build/WiFIG/production/_ext/427700826/icmp.o
 .bss           0x00000000        0x0 build/WiFIG/production/_ext/427700826/icmp.o
 .reginfo       0x00000000       0x18 build/WiFIG/production/_ext/427700826/icmp.o
 .pdr           0x00000000       0xe0 build/WiFIG/production/_ext/427700826/icmp.o
 .text.ICMPRegisterCallback
                0x00000000       0x28 build/WiFIG/production/_ext/427700826/icmp.o
 .text.ICMPDeRegisterCallback
                0x00000000       0x28 build/WiFIG/production/_ext/427700826/icmp.o
 .text          0x00000000        0x0 build/WiFIG/production/_ext/427700826/icmpv6.o
 .data          0x00000000        0x0 build/WiFIG/production/_ext/427700826/icmpv6.o
 .bss           0x00000000        0x0 build/WiFIG/production/_ext/427700826/icmpv6.o
 .reginfo       0x00000000       0x18 build/WiFIG/production/_ext/427700826/icmpv6.o
 .pdr           0x00000000        0x0 build/WiFIG/production/_ext/427700826/icmpv6.o
 .text          0x00000000        0x0 build/WiFIG/production/_ext/427700826/ipv4.o
 .data          0x00000000        0x0 build/WiFIG/production/_ext/427700826/ipv4.o
 .bss           0x00000000        0x0 build/WiFIG/production/_ext/427700826/ipv4.o
 .reginfo       0x00000000       0x18 build/WiFIG/production/_ext/427700826/ipv4.o
 .pdr           0x00000000      0x4e0 build/WiFIG/production/_ext/427700826/ipv4.o
 .text.TCPIP_IPV4_Put
                0x00000000       0x5c build/WiFIG/production/_ext/427700826/ipv4.o
 .text          0x00000000        0x0 build/WiFIG/production/_ext/427700826/ipv6.o
 .data          0x00000000        0x0 build/WiFIG/production/_ext/427700826/ipv6.o
 .bss           0x00000000        0x0 build/WiFIG/production/_ext/427700826/ipv6.o
 .reginfo       0x00000000       0x18 build/WiFIG/production/_ext/427700826/ipv6.o
 .pdr           0x00000000        0x0 build/WiFIG/production/_ext/427700826/ipv6.o
 .text          0x00000000        0x0 build/WiFIG/production/_ext/427700826/mac_events_pic32.o
 .data          0x00000000        0x0 build/WiFIG/production/_ext/427700826/mac_events_pic32.o
 .bss           0x00000000        0x0 build/WiFIG/production/_ext/427700826/mac_events_pic32.o
 .reginfo       0x00000000       0x18 build/WiFIG/production/_ext/427700826/mac_events_pic32.o
 .pdr           0x00000000        0x0 build/WiFIG/production/_ext/427700826/mac_events_pic32.o
 .text          0x00000000        0x0 build/WiFIG/production/_ext/427700826/nbns.o
 .data          0x00000000        0x0 build/WiFIG/production/_ext/427700826/nbns.o
 .bss           0x00000000        0x0 build/WiFIG/production/_ext/427700826/nbns.o
 .reginfo       0x00000000       0x18 build/WiFIG/production/_ext/427700826/nbns.o
 .pdr           0x00000000       0xa0 build/WiFIG/production/_ext/427700826/nbns.o
 .text          0x00000000        0x0 build/WiFIG/production/_ext/427700826/ndp.o
 .data          0x00000000        0x0 build/WiFIG/production/_ext/427700826/ndp.o
 .bss           0x00000000        0x0 build/WiFIG/production/_ext/427700826/ndp.o
 .reginfo       0x00000000       0x18 build/WiFIG/production/_ext/427700826/ndp.o
 .pdr           0x00000000        0x0 build/WiFIG/production/_ext/427700826/ndp.o
 .text          0x00000000        0x0 build/WiFIG/production/_ext/427700826/tcpip_reboot.o
 .data          0x00000000        0x0 build/WiFIG/production/_ext/427700826/tcpip_reboot.o
 .bss           0x00000000        0x0 build/WiFIG/production/_ext/427700826/tcpip_reboot.o
 .reginfo       0x00000000       0x18 build/WiFIG/production/_ext/427700826/tcpip_reboot.o
 .pdr           0x00000000        0x0 build/WiFIG/production/_ext/427700826/tcpip_reboot.o
 .text          0x00000000        0x0 build/WiFIG/production/_ext/427700826/rsa.o
 .data          0x00000000        0x0 build/WiFIG/production/_ext/427700826/rsa.o
 .bss           0x00000000        0x0 build/WiFIG/production/_ext/427700826/rsa.o
 .reginfo       0x00000000       0x18 build/WiFIG/production/_ext/427700826/rsa.o
 .pdr           0x00000000        0x0 build/WiFIG/production/_ext/427700826/rsa.o
 .text          0x00000000        0x0 build/WiFIG/production/_ext/427700826/smtp.o
 .data          0x00000000        0x0 build/WiFIG/production/_ext/427700826/smtp.o
 .bss           0x00000000        0x0 build/WiFIG/production/_ext/427700826/smtp.o
 .reginfo       0x00000000       0x18 build/WiFIG/production/_ext/427700826/smtp.o
 .pdr           0x00000000        0x0 build/WiFIG/production/_ext/427700826/smtp.o
 .text          0x00000000        0x0 build/WiFIG/production/_ext/427700826/snmp.o
 .data          0x00000000        0x0 build/WiFIG/production/_ext/427700826/snmp.o
 .bss           0x00000000        0x0 build/WiFIG/production/_ext/427700826/snmp.o
 .reginfo       0x00000000       0x18 build/WiFIG/production/_ext/427700826/snmp.o
 .pdr           0x00000000        0x0 build/WiFIG/production/_ext/427700826/snmp.o
 .text          0x00000000        0x0 build/WiFIG/production/_ext/427700826/snmpv3.o
 .data          0x00000000        0x0 build/WiFIG/production/_ext/427700826/snmpv3.o
 .bss           0x00000000        0x0 build/WiFIG/production/_ext/427700826/snmpv3.o
 .reginfo       0x00000000       0x18 build/WiFIG/production/_ext/427700826/snmpv3.o
 .pdr           0x00000000        0x0 build/WiFIG/production/_ext/427700826/snmpv3.o
 .text          0x00000000        0x0 build/WiFIG/production/_ext/427700826/snmpv3_usm.o
 .data          0x00000000        0x0 build/WiFIG/production/_ext/427700826/snmpv3_usm.o
 .bss           0x00000000        0x0 build/WiFIG/production/_ext/427700826/snmpv3_usm.o
 .reginfo       0x00000000       0x18 build/WiFIG/production/_ext/427700826/snmpv3_usm.o
 .pdr           0x00000000        0x0 build/WiFIG/production/_ext/427700826/snmpv3_usm.o
 .text          0x00000000        0x0 build/WiFIG/production/_ext/427700826/sntp.o
 .data          0x00000000        0x0 build/WiFIG/production/_ext/427700826/sntp.o
 .bss           0x00000000        0x0 build/WiFIG/production/_ext/427700826/sntp.o
 .reginfo       0x00000000       0x18 build/WiFIG/production/_ext/427700826/sntp.o
 .pdr           0x00000000        0x0 build/WiFIG/production/_ext/427700826/sntp.o
 .text          0x00000000        0x0 build/WiFIG/production/_ext/427700826/ssl.o
 .data          0x00000000        0x0 build/WiFIG/production/_ext/427700826/ssl.o
 .bss           0x00000000        0x0 build/WiFIG/production/_ext/427700826/ssl.o
 .reginfo       0x00000000       0x18 build/WiFIG/production/_ext/427700826/ssl.o
 .pdr           0x00000000        0x0 build/WiFIG/production/_ext/427700826/ssl.o
 .text          0x00000000        0x0 build/WiFIG/production/_ext/427700826/tcp.o
 .data          0x00000000        0x0 build/WiFIG/production/_ext/427700826/tcp.o
 .bss           0x00000000        0x0 build/WiFIG/production/_ext/427700826/tcp.o
 .reginfo       0x00000000       0x18 build/WiFIG/production/_ext/427700826/tcp.o
 .pdr           0x00000000      0x9c0 build/WiFIG/production/_ext/427700826/tcp.o
 .text.TCPSetConnectionMSS
                0x00000000       0x44 build/WiFIG/production/_ext/427700826/tcp.o
 .text.TCPOpenServer
                0x00000000      0x120 build/WiFIG/production/_ext/427700826/tcp.o
 .text.TCPWasReset
                0x00000000       0x94 build/WiFIG/production/_ext/427700826/tcp.o
 .text.TCPDisconnect
                0x00000000       0x80 build/WiFIG/production/_ext/427700826/tcp.o
 .text.TCPAbort
                0x00000000       0x6c build/WiFIG/production/_ext/427700826/tcp.o
 .text.TCPGetSocketInfo
                0x00000000       0xfc build/WiFIG/production/_ext/427700826/tcp.o
 .text.TCPSocketsNo
                0x00000000       0x24 build/WiFIG/production/_ext/427700826/tcp.o
 .text.TCPPut   0x00000000       0x54 build/WiFIG/production/_ext/427700826/tcp.o
 .text.TCPGetTxFIFOFull
                0x00000000       0xa4 build/WiFIG/production/_ext/427700826/tcp.o
 .text.TCPDiscard
                0x00000000       0x90 build/WiFIG/production/_ext/427700826/tcp.o
 .text.TCPIsGetReady
                0x00000000       0x68 build/WiFIG/production/_ext/427700826/tcp.o
 .text.TCPGetRxFIFOFree
                0x00000000       0x68 build/WiFIG/production/_ext/427700826/tcp.o
 .text.TCPPeekArray
                0x00000000      0x1ac build/WiFIG/production/_ext/427700826/tcp.o
 .text.TCPPeek  0x00000000       0x60 build/WiFIG/production/_ext/427700826/tcp.o
 .text.TCPFindArray
                0x00000000      0x578 build/WiFIG/production/_ext/427700826/tcp.o
 .text.TCPFind  0x00000000       0x7c build/WiFIG/production/_ext/427700826/tcp.o
 .text.TCPAdjustFIFOSize
                0x00000000      0x974 build/WiFIG/production/_ext/427700826/tcp.o
 .text.TCPSocketSetNet
                0x00000000       0x80 build/WiFIG/production/_ext/427700826/tcp.o
 .text.TCPSocketGetNet
                0x00000000       0x64 build/WiFIG/production/_ext/427700826/tcp.o
 .text.TCPBind  0x00000000      0x1c4 build/WiFIG/production/_ext/427700826/tcp.o
 .text.TCPRemoteBind
                0x00000000       0x9c build/WiFIG/production/_ext/427700826/tcp.o
 .text.TCPSetOptions
                0x00000000      0x1b8 build/WiFIG/production/_ext/427700826/tcp.o
 .text.TCPGetOptions
                0x00000000      0x1b8 build/WiFIG/production/_ext/427700826/tcp.o
 .text.TCPSetDestinationIPAddress
                0x00000000       0xc4 build/WiFIG/production/_ext/427700826/tcp.o
 .text.TCPSetSourceIPAddress
                0x00000000       0xc4 build/WiFIG/production/_ext/427700826/tcp.o
 .text          0x00000000        0x0 build/WiFIG/production/_ext/427700826/tcpip_heap_alloc.o
 .data          0x00000000        0x0 build/WiFIG/production/_ext/427700826/tcpip_heap_alloc.o
 .bss           0x00000000        0x0 build/WiFIG/production/_ext/427700826/tcpip_heap_alloc.o
 .reginfo       0x00000000       0x18 build/WiFIG/production/_ext/427700826/tcpip_heap_alloc.o
 .pdr           0x00000000      0x200 build/WiFIG/production/_ext/427700826/tcpip_heap_alloc.o
 .text.TCPIP_HEAP_Size
                0x00000000       0x60 build/WiFIG/production/_ext/427700826/tcpip_heap_alloc.o
 .text.TCPIP_HEAP_MaxSize
                0x00000000       0xb0 build/WiFIG/production/_ext/427700826/tcpip_heap_alloc.o
 .text.TCPIP_HEAP_LastError
                0x00000000       0x6c build/WiFIG/production/_ext/427700826/tcpip_heap_alloc.o
 .text.TCPIP_HEAP_SetNoMemHandler
                0x00000000       0x5c build/WiFIG/production/_ext/427700826/tcpip_heap_alloc.o
 .text.TCPIP_HEAP_TraceGetEntry
                0x00000000       0x30 build/WiFIG/production/_ext/427700826/tcpip_heap_alloc.o
 .text.TCPIP_HEAP_TraceGetEntriesNo
                0x00000000       0x30 build/WiFIG/production/_ext/427700826/tcpip_heap_alloc.o
 .text          0x00000000        0x0 build/WiFIG/production/_ext/427700826/tcpip_storage.o
 .data          0x00000000        0x0 build/WiFIG/production/_ext/427700826/tcpip_storage.o
 .bss           0x00000000        0x0 build/WiFIG/production/_ext/427700826/tcpip_storage.o
 .reginfo       0x00000000       0x18 build/WiFIG/production/_ext/427700826/tcpip_storage.o
 .pdr           0x00000000        0x0 build/WiFIG/production/_ext/427700826/tcpip_storage.o
 .text          0x00000000        0x0 build/WiFIG/production/_ext/427700826/telnet.o
 .data          0x00000000        0x0 build/WiFIG/production/_ext/427700826/telnet.o
 .bss           0x00000000        0x0 build/WiFIG/production/_ext/427700826/telnet.o
 .reginfo       0x00000000       0x18 build/WiFIG/production/_ext/427700826/telnet.o
 .pdr           0x00000000        0x0 build/WiFIG/production/_ext/427700826/telnet.o
 .text          0x00000000        0x0 build/WiFIG/production/_ext/427700826/tftpc.o
 .data          0x00000000        0x0 build/WiFIG/production/_ext/427700826/tftpc.o
 .bss           0x00000000        0x0 build/WiFIG/production/_ext/427700826/tftpc.o
 .reginfo       0x00000000       0x18 build/WiFIG/production/_ext/427700826/tftpc.o
 .pdr           0x00000000        0x0 build/WiFIG/production/_ext/427700826/tftpc.o
 .text          0x00000000        0x0 build/WiFIG/production/_ext/427700826/udp.o
 .data          0x00000000        0x0 build/WiFIG/production/_ext/427700826/udp.o
 .bss           0x00000000        0x0 build/WiFIG/production/_ext/427700826/udp.o
 .reginfo       0x00000000       0x18 build/WiFIG/production/_ext/427700826/udp.o
 .pdr           0x00000000      0x560 build/WiFIG/production/_ext/427700826/udp.o
 .text.UDPGetSocketInfo
                0x00000000      0x100 build/WiFIG/production/_ext/427700826/udp.o
 .text.UDPPutString
                0x00000000       0xa0 build/WiFIG/production/_ext/427700826/udp.o
 .text.UDPSocketGetNet
                0x00000000       0x68 build/WiFIG/production/_ext/427700826/udp.o
 .text.UDPGetOptions
                0x00000000       0xdc build/WiFIG/production/_ext/427700826/udp.o
 .text          0x00000000        0x0 build/WiFIG/production/_ext/427700826/tcpip_mac_object.o
 .data          0x00000000        0x0 build/WiFIG/production/_ext/427700826/tcpip_mac_object.o
 .bss           0x00000000        0x0 build/WiFIG/production/_ext/427700826/tcpip_mac_object.o
 .reginfo       0x00000000       0x18 build/WiFIG/production/_ext/427700826/tcpip_mac_object.o
 .pdr           0x00000000      0x300 build/WiFIG/production/_ext/427700826/tcpip_mac_object.o
 .text.MACGetReadPtrInRx
                0x00000000       0x44 build/WiFIG/production/_ext/427700826/tcpip_mac_object.o
 .text.MACSetBaseReadPtr
                0x00000000       0x4c build/WiFIG/production/_ext/427700826/tcpip_mac_object.o
 .text.MACSetRXHashTableEntry
                0x00000000       0x54 build/WiFIG/production/_ext/427700826/tcpip_mac_object.o
 .text.MACPowerMode
                0x00000000       0x4c build/WiFIG/production/_ext/427700826/tcpip_mac_object.o
 .text.MACEventClearNotifyEvents
                0x00000000       0x54 build/WiFIG/production/_ext/427700826/tcpip_mac_object.o
 .text          0x00000000        0x0 build/WiFIG/production/_ext/427700826/tcpip_manager.o
 .data          0x00000000        0x0 build/WiFIG/production/_ext/427700826/tcpip_manager.o
 .bss           0x00000000        0x0 build/WiFIG/production/_ext/427700826/tcpip_manager.o
 .reginfo       0x00000000       0x18 build/WiFIG/production/_ext/427700826/tcpip_manager.o
 .pdr           0x00000000      0xa00 build/WiFIG/production/_ext/427700826/tcpip_manager.o
 .text.TCPIP_STACK_NetUp
                0x00000000      0x1c0 build/WiFIG/production/_ext/427700826/tcpip_manager.o
 .text.TCPIP_STACK_NetDown
                0x00000000      0x134 build/WiFIG/production/_ext/427700826/tcpip_manager.o
 .text.TCPIP_STACK_SetDefaultNet
                0x00000000       0x70 build/WiFIG/production/_ext/427700826/tcpip_manager.o
 .text._TCPIPStackIpAddFromNet
                0x00000000       0xec build/WiFIG/production/_ext/427700826/tcpip_manager.o
 .text._TCPIPStackMacToNet
                0x00000000       0x88 build/WiFIG/production/_ext/427700826/tcpip_manager.o
 .text._TCPIPStackMacToNetIx
                0x00000000       0x88 build/WiFIG/production/_ext/427700826/tcpip_manager.o
 .text.TCPIP_STACK_NetIx
                0x00000000       0x48 build/WiFIG/production/_ext/427700826/tcpip_manager.o
 .text.TCPIP_STACK_SetNetAddress
                0x00000000       0x80 build/WiFIG/production/_ext/427700826/tcpip_manager.o
 .text.TCPIP_STACK_SetNetGatewayAddress
                0x00000000       0x5c build/WiFIG/production/_ext/427700826/tcpip_manager.o
 .text.TCPIP_STACK_NetGatewayAddress
                0x00000000       0x6c build/WiFIG/production/_ext/427700826/tcpip_manager.o
 .text.TCPIP_STACK_NetPriDNSAddress
                0x00000000       0x6c build/WiFIG/production/_ext/427700826/tcpip_manager.o
 .text.TCPIP_STACK_NetSecondDNSAddress
                0x00000000       0x6c build/WiFIG/production/_ext/427700826/tcpip_manager.o
 .text.TCPIP_STACK_SetNetPriDNSAddress
                0x00000000       0x5c build/WiFIG/production/_ext/427700826/tcpip_manager.o
 .text.TCPIP_STACK_SetNetSecondDNSAddress
                0x00000000       0x5c build/WiFIG/production/_ext/427700826/tcpip_manager.o
 .text.TCPIP_STACK_NetMask
                0x00000000       0x48 build/WiFIG/production/_ext/427700826/tcpip_manager.o
 .text.TCPIP_STACK_SetNetMacAddress
                0x00000000       0x7c build/WiFIG/production/_ext/427700826/tcpip_manager.o
 .text.TCPIP_STACK_SetNetBIOSName
                0x00000000       0x8c build/WiFIG/production/_ext/427700826/tcpip_manager.o
 .text.TCPIP_STACK_SetLocalMasksType
                0x00000000       0x98 build/WiFIG/production/_ext/427700826/tcpip_manager.o
 .text.TCPIP_STACK_SetLocalMasks
                0x00000000       0x70 build/WiFIG/production/_ext/427700826/tcpip_manager.o
 .text.TCPIP_STACK_NetMACId
                0x00000000       0x44 build/WiFIG/production/_ext/427700826/tcpip_manager.o
 .text.TCPIP_STACK_ModuleGetConfig
                0x00000000       0xc0 build/WiFIG/production/_ext/427700826/tcpip_manager.o
 .text.TCPIP_STACK_NetConfigGet
                0x00000000      0x10c build/WiFIG/production/_ext/427700826/tcpip_manager.o
 .text.NetConfigStringToBuffer
                0x00000000       0xf0 build/WiFIG/production/_ext/427700826/tcpip_manager.o
 .text.TCPIP_STACK_NetConfigSet
                0x00000000      0x4d8 build/WiFIG/production/_ext/427700826/tcpip_manager.o
 .text.TCPIP_STACK_IsNetUp
                0x00000000       0x48 build/WiFIG/production/_ext/427700826/tcpip_manager.o
 .text.TCPIP_STACK_IsNetLinked
                0x00000000       0x48 build/WiFIG/production/_ext/427700826/tcpip_manager.o
 .text.TCPIP_STACK_GetPendingEvents
                0x00000000       0x6c build/WiFIG/production/_ext/427700826/tcpip_manager.o
 .text.TCPIP_STACK_DeRegisterHandler
                0x00000000       0x7c build/WiFIG/production/_ext/427700826/tcpip_manager.o
 .text._TCPIPStackNetMacId
                0x00000000       0x44 build/WiFIG/production/_ext/427700826/tcpip_manager.o
 .text          0x00000000        0x0 build/WiFIG/production/_ext/427700826/tcpip_helpers.o
 .data          0x00000000        0x0 build/WiFIG/production/_ext/427700826/tcpip_helpers.o
 .bss           0x00000000        0x0 build/WiFIG/production/_ext/427700826/tcpip_helpers.o
 .reginfo       0x00000000       0x18 build/WiFIG/production/_ext/427700826/tcpip_helpers.o
 .pdr           0x00000000      0x340 build/WiFIG/production/_ext/427700826/tcpip_helpers.o
 .text.TCPIP_HELPER_IPAddressToString
                0x00000000       0xec build/WiFIG/production/_ext/427700826/tcpip_helpers.o
 .text.TCPIP_HELPER_MACAddressToString
                0x00000000       0xf4 build/WiFIG/production/_ext/427700826/tcpip_helpers.o
 .text.TCPIP_HELPER_PowerModeToString
                0x00000000       0x58 build/WiFIG/production/_ext/427700826/tcpip_helpers.o
 .text.TCPIP_Helper_Base64Decode
                0x00000000      0x394 build/WiFIG/production/_ext/427700826/tcpip_helpers.o
 .text.TCPIP_Helper_FindCommonPrefix
                0x00000000      0x110 build/WiFIG/production/_ext/427700826/tcpip_helpers.o
 .text.SingleListAddHead
                0x00000000       0x74 build/WiFIG/production/_ext/427700826/tcpip_helpers.o
 .text.SingleListAddMid
                0x00000000       0x5c build/WiFIG/production/_ext/427700826/tcpip_helpers.o
 .text.SingleListRemoveNext
                0x00000000       0xb0 build/WiFIG/production/_ext/427700826/tcpip_helpers.o
 .text.SingleListAppendList
                0x00000000       0x64 build/WiFIG/production/_ext/427700826/tcpip_helpers.o
 .text.DoubleListInit
                0x00000000       0x44 build/WiFIG/production/_ext/427700826/tcpip_helpers.o
 .text.DoubleListAddHead
                0x00000000       0xbc build/WiFIG/production/_ext/427700826/tcpip_helpers.o
 .text.DoubleListAddTail
                0x00000000       0xbc build/WiFIG/production/_ext/427700826/tcpip_helpers.o
 .text.DoubleListAddMid
                0x00000000       0x78 build/WiFIG/production/_ext/427700826/tcpip_helpers.o
 .text.DoubleListRemoveHead
                0x00000000       0xa8 build/WiFIG/production/_ext/427700826/tcpip_helpers.o
 .text.DoubleListRemoveTail
                0x00000000       0xa8 build/WiFIG/production/_ext/427700826/tcpip_helpers.o
 .text.DoubleListRemoveMid
                0x00000000       0x64 build/WiFIG/production/_ext/427700826/tcpip_helpers.o
 .text.DoubleListRemoveNode
                0x00000000       0x90 build/WiFIG/production/_ext/427700826/tcpip_helpers.o
 .text          0x00000000        0x0 build/WiFIG/production/_ext/427700826/tcpip_commands.o
 .data          0x00000000        0x0 build/WiFIG/production/_ext/427700826/tcpip_commands.o
 .bss           0x00000000        0x0 build/WiFIG/production/_ext/427700826/tcpip_commands.o
 .reginfo       0x00000000       0x18 build/WiFIG/production/_ext/427700826/tcpip_commands.o
 .pdr           0x00000000        0x0 build/WiFIG/production/_ext/427700826/tcpip_commands.o
 .text          0x00000000        0x0 build/WiFIG/production/_ext/427700826/iperf.o
 .data          0x00000000        0x0 build/WiFIG/production/_ext/427700826/iperf.o
 .bss           0x00000000        0x0 build/WiFIG/production/_ext/427700826/iperf.o
 .reginfo       0x00000000       0x18 build/WiFIG/production/_ext/427700826/iperf.o
 .pdr           0x00000000        0x0 build/WiFIG/production/_ext/427700826/iperf.o
 .data          0x00000000        0x0 build/WiFIG/production/_ext/427700826/tcpip_helper_c32.o
 .bss           0x00000000        0x0 build/WiFIG/production/_ext/427700826/tcpip_helper_c32.o
 .reginfo       0x00000000       0x18 build/WiFIG/production/_ext/427700826/tcpip_helper_c32.o
 .pdr           0x00000000       0x60 build/WiFIG/production/_ext/427700826/tcpip_helper_c32.o
 .text          0x00000000        0x0 build/WiFIG/production/_ext/427700826/tcpip_notify.o
 .data          0x00000000        0x0 build/WiFIG/production/_ext/427700826/tcpip_notify.o
 .bss           0x00000000        0x0 build/WiFIG/production/_ext/427700826/tcpip_notify.o
 .reginfo       0x00000000       0x18 build/WiFIG/production/_ext/427700826/tcpip_notify.o
 .pdr           0x00000000       0x60 build/WiFIG/production/_ext/427700826/tcpip_notify.o
 .text          0x00000000        0x0 build/WiFIG/production/_ext/427700826/zero_conf_helper.o
 .data          0x00000000        0x0 build/WiFIG/production/_ext/427700826/zero_conf_helper.o
 .bss           0x00000000        0x0 build/WiFIG/production/_ext/427700826/zero_conf_helper.o
 .reginfo       0x00000000       0x18 build/WiFIG/production/_ext/427700826/zero_conf_helper.o
 .pdr           0x00000000        0x0 build/WiFIG/production/_ext/427700826/zero_conf_helper.o
 .text          0x00000000        0x0 build/WiFIG/production/_ext/427700826/zero_conf_link_local.o
 .data          0x00000000        0x0 build/WiFIG/production/_ext/427700826/zero_conf_link_local.o
 .bss           0x00000000        0x0 build/WiFIG/production/_ext/427700826/zero_conf_link_local.o
 .reginfo       0x00000000       0x18 build/WiFIG/production/_ext/427700826/zero_conf_link_local.o
 .pdr           0x00000000       0x60 build/WiFIG/production/_ext/427700826/zero_conf_link_local.o
 .text.ZCLLDisable
                0x00000000       0x28 build/WiFIG/production/_ext/427700826/zero_conf_link_local.o
 .text.ZCLLIsEnabled
                0x00000000       0x28 build/WiFIG/production/_ext/427700826/zero_conf_link_local.o
 .text          0x00000000        0x0 build/WiFIG/production/_ext/427700826/zero_conf_multicast_dns.o
 .data          0x00000000        0x0 build/WiFIG/production/_ext/427700826/zero_conf_multicast_dns.o
 .bss           0x00000000        0x0 build/WiFIG/production/_ext/427700826/zero_conf_multicast_dns.o
 .reginfo       0x00000000       0x18 build/WiFIG/production/_ext/427700826/zero_conf_multicast_dns.o
 .pdr           0x00000000        0x0 build/WiFIG/production/_ext/427700826/zero_conf_multicast_dns.o
 .text          0x00000000        0x0 build/WiFIG/production/_ext/334706090/wf_tx_power.o
 .data          0x00000000        0x0 build/WiFIG/production/_ext/334706090/wf_tx_power.o
 .bss           0x00000000        0x0 build/WiFIG/production/_ext/334706090/wf_tx_power.o
 .reginfo       0x00000000       0x18 build/WiFIG/production/_ext/334706090/wf_tx_power.o
 .pdr           0x00000000       0x60 build/WiFIG/production/_ext/334706090/wf_tx_power.o
 .rodata        0x00000000       0x30 build/WiFIG/production/_ext/334706090/wf_tx_power.o
 .text.WF_TxPowerSetMax
                0x00000000       0xb0 build/WiFIG/production/_ext/334706090/wf_tx_power.o
 .text.WF_TxPowerGetMax
                0x00000000       0x74 build/WiFIG/production/_ext/334706090/wf_tx_power.o
 .text.WF_TxPowerGetFactoryMax
                0x00000000       0x54 build/WiFIG/production/_ext/334706090/wf_tx_power.o
 .text          0x00000000        0x0 build/WiFIG/production/_ext/334706090/wf_connect.o
 .data          0x00000000        0x0 build/WiFIG/production/_ext/334706090/wf_connect.o
 .bss           0x00000000        0x0 build/WiFIG/production/_ext/334706090/wf_connect.o
 .reginfo       0x00000000       0x18 build/WiFIG/production/_ext/334706090/wf_connect.o
 .pdr           0x00000000       0xa0 build/WiFIG/production/_ext/334706090/wf_connect.o
 .text          0x00000000        0x0 build/WiFIG/production/_ext/334706090/wf_connection_algorithm.o
 .data          0x00000000        0x0 build/WiFIG/production/_ext/334706090/wf_connection_algorithm.o
 .bss           0x00000000        0x0 build/WiFIG/production/_ext/334706090/wf_connection_algorithm.o
 .reginfo       0x00000000       0x18 build/WiFIG/production/_ext/334706090/wf_connection_algorithm.o
 .pdr           0x00000000      0x240 build/WiFIG/production/_ext/334706090/wf_connection_algorithm.o
 .text.WF_RssiSet
                0x00000000       0x44 build/WiFIG/production/_ext/334706090/wf_connection_algorithm.o
 .text.WF_RssiGet
                0x00000000       0x44 build/WiFIG/production/_ext/334706090/wf_connection_algorithm.o
 .text.WF_CAGetEventNotificationAction
                0x00000000       0x40 build/WiFIG/production/_ext/334706090/wf_connection_algorithm.o
 .text.WF_AdhocContextSet
                0x00000000       0x84 build/WiFIG/production/_ext/334706090/wf_connection_algorithm.o
 .text.WF_AdhocContextGet
                0x00000000       0x98 build/WiFIG/production/_ext/334706090/wf_connection_algorithm.o
 .text          0x00000000        0x0 build/WiFIG/production/_ext/334706090/wf_connection_manager.o
 .data          0x00000000        0x0 build/WiFIG/production/_ext/334706090/wf_connection_manager.o
 .bss           0x00000000        0x0 build/WiFIG/production/_ext/334706090/wf_connection_manager.o
 .reginfo       0x00000000       0x18 build/WiFIG/production/_ext/334706090/wf_connection_manager.o
 .pdr           0x00000000       0xe0 build/WiFIG/production/_ext/334706090/wf_connection_manager.o
 .text.isDisconnectAllowed
                0x00000000       0x68 build/WiFIG/production/_ext/334706090/wf_connection_manager.o
 .text.WF_Disconnect
                0x00000000       0x8c build/WiFIG/production/_ext/334706090/wf_connection_manager.o
 .text.WF_ConnectionStateGet
                0x00000000       0xc8 build/WiFIG/production/_ext/334706090/wf_connection_manager.o
 .text          0x00000000        0x0 build/WiFIG/production/_ext/334706090/wf_connection_profile.o
 .data          0x00000000        0x0 build/WiFIG/production/_ext/334706090/wf_connection_profile.o
 .bss           0x00000000        0x0 build/WiFIG/production/_ext/334706090/wf_connection_profile.o
 .reginfo       0x00000000       0x18 build/WiFIG/production/_ext/334706090/wf_connection_profile.o
 .pdr           0x00000000      0x300 build/WiFIG/production/_ext/334706090/wf_connection_profile.o
 .text.WF_SsidGet
                0x00000000       0x98 build/WiFIG/production/_ext/334706090/wf_connection_profile.o
 .text.WF_BssidSet
                0x00000000       0x40 build/WiFIG/production/_ext/334706090/wf_connection_profile.o
 .text.WF_BssidGet
                0x00000000       0x44 build/WiFIG/production/_ext/334706090/wf_connection_profile.o
 .text.WF_CPSetWepKeyType
                0x00000000       0x50 build/WiFIG/production/_ext/334706090/wf_connection_profile.o
 .text.WF_WPSCredentialsGet
                0x00000000       0x48 build/WiFIG/production/_ext/334706090/wf_connection_profile.o
 .text.SetHiddenSsid
                0x00000000       0x48 build/WiFIG/production/_ext/334706090/wf_connection_profile.o
 .text.GetHiddenSsid
                0x00000000       0x48 build/WiFIG/production/_ext/334706090/wf_connection_profile.o
 .text.SetAdHocMode
                0x00000000       0x44 build/WiFIG/production/_ext/334706090/wf_connection_profile.o
 .text.GetAdHocMode
                0x00000000       0x48 build/WiFIG/production/_ext/334706090/wf_connection_profile.o
 .text          0x00000000        0x0 build/WiFIG/production/_ext/334706090/wf_easy_config.o
 .data          0x00000000        0x0 build/WiFIG/production/_ext/334706090/wf_easy_config.o
 .bss           0x00000000        0x0 build/WiFIG/production/_ext/334706090/wf_easy_config.o
 .reginfo       0x00000000       0x18 build/WiFIG/production/_ext/334706090/wf_easy_config.o
 .pdr           0x00000000       0x20 build/WiFIG/production/_ext/334706090/wf_easy_config.o
 .rodata        0x00000000       0x7c build/WiFIG/production/_ext/334706090/wf_easy_config.o
 .text.WFDisplayScanMgr
                0x00000000      0x308 build/WiFIG/production/_ext/334706090/wf_easy_config.o
 COMMON         0x00000000       0x98 build/WiFIG/production/_ext/334706090/wf_easy_config.o
 .text          0x00000000        0x0 build/WiFIG/production/_ext/334706090/wf_eint.o
 .data          0x00000000        0x0 build/WiFIG/production/_ext/334706090/wf_eint.o
 .bss           0x00000000        0x0 build/WiFIG/production/_ext/334706090/wf_eint.o
 .reginfo       0x00000000       0x18 build/WiFIG/production/_ext/334706090/wf_eint.o
 .pdr           0x00000000       0xa0 build/WiFIG/production/_ext/334706090/wf_eint.o
 .text          0x00000000        0x0 build/WiFIG/production/_ext/334706090/wf_event_handler.o
 .data          0x00000000        0x0 build/WiFIG/production/_ext/334706090/wf_event_handler.o
 .bss           0x00000000        0x0 build/WiFIG/production/_ext/334706090/wf_event_handler.o
 .reginfo       0x00000000       0x18 build/WiFIG/production/_ext/334706090/wf_event_handler.o
 .pdr           0x00000000      0x140 build/WiFIG/production/_ext/334706090/wf_event_handler.o
 .text.WF_GetSoftApEventInfo
                0x00000000       0x24 build/WiFIG/production/_ext/334706090/wf_event_handler.o
 .text          0x00000000        0x0 build/WiFIG/production/_ext/334706090/wf_init.o
 .data          0x00000000        0x0 build/WiFIG/production/_ext/334706090/wf_init.o
 .bss           0x00000000        0x0 build/WiFIG/production/_ext/334706090/wf_init.o
 .reginfo       0x00000000       0x18 build/WiFIG/production/_ext/334706090/wf_init.o
 .pdr           0x00000000       0xa0 build/WiFIG/production/_ext/334706090/wf_init.o
 .text          0x00000000        0x0 build/WiFIG/production/_ext/334706090/wf_power_save.o
 .data          0x00000000        0x0 build/WiFIG/production/_ext/334706090/wf_power_save.o
 .bss           0x00000000        0x0 build/WiFIG/production/_ext/334706090/wf_power_save.o
 .reginfo       0x00000000       0x18 build/WiFIG/production/_ext/334706090/wf_power_save.o
 .pdr           0x00000000      0x1e0 build/WiFIG/production/_ext/334706090/wf_power_save.o
 .text.WFisPsPollEnabled
                0x00000000       0x50 build/WiFIG/production/_ext/334706090/wf_power_save.o
 .text.WFIsPsPollActive
                0x00000000       0x24 build/WiFIG/production/_ext/334706090/wf_power_save.o
 .text.WF_HibernateEnable
                0x00000000       0x44 build/WiFIG/production/_ext/334706090/wf_power_save.o
 .text          0x00000000        0x0 build/WiFIG/production/_ext/334706090/wf_scan.o
 .data          0x00000000        0x0 build/WiFIG/production/_ext/334706090/wf_scan.o
 .bss           0x00000000        0x0 build/WiFIG/production/_ext/334706090/wf_scan.o
 .reginfo       0x00000000       0x18 build/WiFIG/production/_ext/334706090/wf_scan.o
 .pdr           0x00000000       0x60 build/WiFIG/production/_ext/334706090/wf_scan.o
 .text.isHostScanAllowed
                0x00000000       0x68 build/WiFIG/production/_ext/334706090/wf_scan.o
 .text.WF_Scan  0x00000000       0xb8 build/WiFIG/production/_ext/334706090/wf_scan.o
 .text.WF_ScanGetResult
                0x00000000       0xcc build/WiFIG/production/_ext/334706090/wf_scan.o
 .text          0x00000000        0x0 build/WiFIG/production/_ext/334706090/wf_spi.o
 .data          0x00000000        0x0 build/WiFIG/production/_ext/334706090/wf_spi.o
 .bss           0x00000000        0x0 build/WiFIG/production/_ext/334706090/wf_spi.o
 .reginfo       0x00000000       0x18 build/WiFIG/production/_ext/334706090/wf_spi.o
 .pdr           0x00000000       0xa0 build/WiFIG/production/_ext/334706090/wf_spi.o
 .text          0x00000000        0x0 build/WiFIG/production/_ext/334706090/mrf24w_mac_pic32.o
 .data          0x00000000        0x0 build/WiFIG/production/_ext/334706090/mrf24w_mac_pic32.o
 .bss           0x00000000        0x0 build/WiFIG/production/_ext/334706090/mrf24w_mac_pic32.o
 .reginfo       0x00000000       0x18 build/WiFIG/production/_ext/334706090/mrf24w_mac_pic32.o
 .pdr           0x00000000      0x3c0 build/WiFIG/production/_ext/334706090/mrf24w_mac_pic32.o
 .text          0x00000000        0x0 build/WiFIG/production/_ext/334706090/mrf24w_events.o
 .data          0x00000000        0x0 build/WiFIG/production/_ext/334706090/mrf24w_events.o
 .bss           0x00000000        0x0 build/WiFIG/production/_ext/334706090/mrf24w_events.o
 .reginfo       0x00000000       0x18 build/WiFIG/production/_ext/334706090/mrf24w_events.o
 .pdr           0x00000000      0x160 build/WiFIG/production/_ext/334706090/mrf24w_events.o
 .text          0x00000000        0x0 build/WiFIG/production/_ext/334706090/wf_debug_output.o
 .bss           0x00000000        0x0 build/WiFIG/production/_ext/334706090/wf_debug_output.o
 .reginfo       0x00000000       0x18 build/WiFIG/production/_ext/334706090/wf_debug_output.o
 .pdr           0x00000000      0x280 build/WiFIG/production/_ext/334706090/wf_debug_output.o
 .text          0x00000000        0x0 build/WiFIG/production/_ext/334706090/wf_commands.o
 .data          0x00000000        0x0 build/WiFIG/production/_ext/334706090/wf_commands.o
 .bss           0x00000000        0x0 build/WiFIG/production/_ext/334706090/wf_commands.o
 .reginfo       0x00000000       0x18 build/WiFIG/production/_ext/334706090/wf_commands.o
 .pdr           0x00000000      0x1e0 build/WiFIG/production/_ext/334706090/wf_commands.o
 .sbss          0x00000000        0x3 build/WiFIG/production/_ext/334706090/wf_commands.o
 .rodata        0x00000000      0x5d4 build/WiFIG/production/_ext/334706090/wf_commands.o
 .text.WIFICommandsInit
                0x00000000       0x6c build/WiFIG/production/_ext/334706090/wf_commands.o
 .text.CommandIwConfig
                0x00000000      0x4bc build/WiFIG/production/_ext/334706090/wf_commands.o
 .text.iwconfigUpdateCb
                0x00000000       0xf0 build/WiFIG/production/_ext/334706090/wf_commands.o
 .text.iwconfigDisplayStatus
                0x00000000      0x7f0 build/WiFIG/production/_ext/334706090/wf_commands.o
 .text.iwconfigSetSsid
                0x00000000      0x104 build/WiFIG/production/_ext/334706090/wf_commands.o
 .text.iwconfigSetMode
                0x00000000      0x2e0 build/WiFIG/production/_ext/334706090/wf_commands.o
 .text.iwconfigSetChannel
                0x00000000      0x2a8 build/WiFIG/production/_ext/334706090/wf_commands.o
 .text.iwconfigSetPower
                0x00000000      0x204 build/WiFIG/production/_ext/334706090/wf_commands.o
 .text.iwconfigSetRTS
                0x00000000       0xc4 build/WiFIG/production/_ext/334706090/wf_commands.o
 .text.CommandIw_eraseConfig
                0x00000000       0x68 build/WiFIG/production/_ext/334706090/wf_commands.o
 .text.CommandIw_saveConfig
                0x00000000       0x7c build/WiFIG/production/_ext/334706090/wf_commands.o
 .text.CommandIw_readConfig
                0x00000000       0x68 build/WiFIG/production/_ext/334706090/wf_commands.o
 .text.HexToBin
                0x00000000       0x9c build/WiFIG/production/_ext/334706090/wf_commands.o
 .text.ConvertASCIIHexToBinary
                0x00000000      0x144 build/WiFIG/production/_ext/334706090/wf_commands.o
 .text.convertAsciiToHexInPlace
                0x00000000      0x134 build/WiFIG/production/_ext/334706090/wf_commands.o
 .text          0x00000000        0x0 build/WiFIG/production/_ext/334706090/wf_pbkdf2.o
 .data          0x00000000        0x0 build/WiFIG/production/_ext/334706090/wf_pbkdf2.o
 .bss           0x00000000        0x0 build/WiFIG/production/_ext/334706090/wf_pbkdf2.o
 .reginfo       0x00000000       0x18 build/WiFIG/production/_ext/334706090/wf_pbkdf2.o
 .pdr           0x00000000        0x0 build/WiFIG/production/_ext/334706090/wf_pbkdf2.o
 .text          0x00000000        0x0 build/WiFIG/production/_ext/334706090/wf_driver_com_24g.o
 .data          0x00000000        0x0 build/WiFIG/production/_ext/334706090/wf_driver_com_24g.o
 .bss           0x00000000        0x0 build/WiFIG/production/_ext/334706090/wf_driver_com_24g.o
 .reginfo       0x00000000       0x18 build/WiFIG/production/_ext/334706090/wf_driver_com_24g.o
 .pdr           0x00000000      0x300 build/WiFIG/production/_ext/334706090/wf_driver_com_24g.o
 .text.ReenablePowerSaveMode
                0x00000000       0x28 build/WiFIG/production/_ext/334706090/wf_driver_com_24g.o
 .text          0x00000000        0x0 build/WiFIG/production/_ext/334706090/wf_driver_raw_24g.o
 .data          0x00000000        0x0 build/WiFIG/production/_ext/334706090/wf_driver_raw_24g.o
 .bss           0x00000000        0x0 build/WiFIG/production/_ext/334706090/wf_driver_raw_24g.o
 .reginfo       0x00000000       0x18 build/WiFIG/production/_ext/334706090/wf_driver_raw_24g.o
 .pdr           0x00000000      0x2a0 build/WiFIG/production/_ext/334706090/wf_driver_raw_24g.o
 .text.RawToRawCopy
                0x00000000       0x98 build/WiFIG/production/_ext/334706090/wf_driver_raw_24g.o
 .text.PushRawWindow
                0x00000000       0x4c build/WiFIG/production/_ext/334706090/wf_driver_raw_24g.o
 .text.PopRawWindow
                0x00000000       0x54 build/WiFIG/production/_ext/334706090/wf_driver_raw_24g.o
 .text.RawGetIndex
                0x00000000       0x60 build/WiFIG/production/_ext/334706090/wf_driver_raw_24g.o
 .text          0x00000000        0x0 build/WiFIG/production/_ext/334706090/wf_mac_24g.o
 .data          0x00000000        0x0 build/WiFIG/production/_ext/334706090/wf_mac_24g.o
 .bss           0x00000000        0x0 build/WiFIG/production/_ext/334706090/wf_mac_24g.o
 .reginfo       0x00000000       0x18 build/WiFIG/production/_ext/334706090/wf_mac_24g.o
 .pdr           0x00000000      0x3e0 build/WiFIG/production/_ext/334706090/wf_mac_24g.o
 .text.WF_StopGratuitousArp
                0x00000000       0x40 build/WiFIG/production/_ext/334706090/wf_mac_24g.o
 .text          0x00000000        0x0 build/WiFIG/production/_ext/334706090/wf_mgmt_msg_24g.o
 .data          0x00000000        0x0 build/WiFIG/production/_ext/334706090/wf_mgmt_msg_24g.o
 .bss           0x00000000        0x0 build/WiFIG/production/_ext/334706090/wf_mgmt_msg_24g.o
 .reginfo       0x00000000       0x18 build/WiFIG/production/_ext/334706090/wf_mgmt_msg_24g.o
 .pdr           0x00000000       0xa0 build/WiFIG/production/_ext/334706090/wf_mgmt_msg_24g.o
 .text.WFSetFuncState
                0x00000000       0x80 build/WiFIG/production/_ext/334706090/wf_mgmt_msg_24g.o
 .text          0x00000000        0x0 build/WiFIG/production/_ext/334706090/wf_param_msg_24g.o
 .data          0x00000000        0x0 build/WiFIG/production/_ext/334706090/wf_param_msg_24g.o
 .bss           0x00000000        0x0 build/WiFIG/production/_ext/334706090/wf_param_msg_24g.o
 .reginfo       0x00000000       0x18 build/WiFIG/production/_ext/334706090/wf_param_msg_24g.o
 .pdr           0x00000000      0x340 build/WiFIG/production/_ext/334706090/wf_param_msg_24g.o
 .text.WFEnableBroadcastProbeResponse
                0x00000000       0x48 build/WiFIG/production/_ext/334706090/wf_param_msg_24g.o
 .text.WF_SetLinkDownThreshold
                0x00000000       0x44 build/WiFIG/production/_ext/334706090/wf_param_msg_24g.o
 .text.WF_SetStackVersion
                0x00000000       0x7c build/WiFIG/production/_ext/334706090/wf_param_msg_24g.o
 .text.WF_GetWPATimeout
                0x00000000       0x44 build/WiFIG/production/_ext/334706090/wf_param_msg_24g.o
 .text.WF_GetMultiCastFilter
                0x00000000      0x120 build/WiFIG/production/_ext/334706090/wf_param_msg_24g.o
 .text.WF_MulticastSetConfig
                0x00000000      0x194 build/WiFIG/production/_ext/334706090/wf_param_msg_24g.o
 .text.WF_MulticastGetConfig
                0x00000000       0xf8 build/WiFIG/production/_ext/334706090/wf_param_msg_24g.o
 .text.WF_GetTxDataConfirm
                0x00000000       0x40 build/WiFIG/production/_ext/334706090/wf_param_msg_24g.o
 .text.WF_RtsThresholdSet
                0x00000000       0x88 build/WiFIG/production/_ext/334706090/wf_param_msg_24g.o
 .text.WF_RtsThresholdGet
                0x00000000       0x64 build/WiFIG/production/_ext/334706090/wf_param_msg_24g.o
 .text.WF_EnableSWMultiCastFilter
                0x00000000       0x48 build/WiFIG/production/_ext/334706090/wf_param_msg_24g.o
 .text.WF_GetMacStats
                0x00000000       0xac build/WiFIG/production/_ext/334706090/wf_param_msg_24g.o
 .text.WF_YieldPassphrase2Host
                0x00000000       0x48 build/WiFIG/production/_ext/334706090/wf_param_msg_24g.o
 .text.WF_SetPSK
                0x00000000       0x40 build/WiFIG/production/_ext/334706090/wf_param_msg_24g.o
 .text          0x00000000        0x0 build/WiFIG/production/_ext/334706090/wf_configData.o
 .data          0x00000000        0x0 build/WiFIG/production/_ext/334706090/wf_configData.o
 .bss           0x00000000        0x0 build/WiFIG/production/_ext/334706090/wf_configData.o
 .reginfo       0x00000000       0x18 build/WiFIG/production/_ext/334706090/wf_configData.o
 .pdr           0x00000000       0x80 build/WiFIG/production/_ext/334706090/wf_configData.o
 .text.WiFiMemory_write
                0x00000000       0x28 build/WiFIG/production/_ext/334706090/wf_configData.o
 .rodata        0x00000000      0x190 build/WiFIG/production/_ext/334706090/wf_configData.o
 .text.WF_ConfigDataPrint
                0x00000000      0x4b8 build/WiFIG/production/_ext/334706090/wf_configData.o
 .text.WF_ConfigDataErase
                0x00000000       0x58 build/WiFIG/production/_ext/334706090/wf_configData.o
 .text          0x00000000        0x0 build/WiFIG/production/_ext/1472/main_demo.o
 .data          0x00000000        0x0 build/WiFIG/production/_ext/1472/main_demo.o
 .bss           0x00000000        0x0 build/WiFIG/production/_ext/1472/main_demo.o
 .reginfo       0x00000000       0x18 build/WiFIG/production/_ext/1472/main_demo.o
 .pdr           0x00000000       0x80 build/WiFIG/production/_ext/1472/main_demo.o
 .text          0x00000000        0x0 build/WiFIG/production/_ext/1472/custom_snmp_app.o
 .data          0x00000000        0x0 build/WiFIG/production/_ext/1472/custom_snmp_app.o
 .bss           0x00000000        0x0 build/WiFIG/production/_ext/1472/custom_snmp_app.o
 .reginfo       0x00000000       0x18 build/WiFIG/production/_ext/1472/custom_snmp_app.o
 .pdr           0x00000000        0x0 build/WiFIG/production/_ext/1472/custom_snmp_app.o
 .text          0x00000000        0x0 build/WiFIG/production/_ext/1472/custom_ssl_cert.o
 .data          0x00000000        0x0 build/WiFIG/production/_ext/1472/custom_ssl_cert.o
 .bss           0x00000000        0x0 build/WiFIG/production/_ext/1472/custom_ssl_cert.o
 .reginfo       0x00000000       0x18 build/WiFIG/production/_ext/1472/custom_ssl_cert.o
 .pdr           0x00000000        0x0 build/WiFIG/production/_ext/1472/custom_ssl_cert.o
 .text          0x00000000        0x0 build/WiFIG/production/_ext/1472/mpfs_img2.o
 .data          0x00000000        0x0 build/WiFIG/production/_ext/1472/mpfs_img2.o
 .bss           0x00000000        0x0 build/WiFIG/production/_ext/1472/mpfs_img2.o
 .reginfo       0x00000000       0x18 build/WiFIG/production/_ext/1472/mpfs_img2.o
 .pdr           0x00000000        0x0 build/WiFIG/production/_ext/1472/mpfs_img2.o
 .text          0x00000000        0x0 build/WiFIG/production/_ext/1472/wf_config.o
 .data          0x00000000        0x0 build/WiFIG/production/_ext/1472/wf_config.o
 .bss           0x00000000        0x0 build/WiFIG/production/_ext/1472/wf_config.o
 .reginfo       0x00000000       0x18 build/WiFIG/production/_ext/1472/wf_config.o
 .pdr           0x00000000       0x20 build/WiFIG/production/_ext/1472/wf_config.o
 .text          0x00000000        0x0 build/WiFIG/production/_ext/1472/custom_http_app.o
 .data          0x00000000        0x0 build/WiFIG/production/_ext/1472/custom_http_app.o
 .bss           0x00000000        0x0 build/WiFIG/production/_ext/1472/custom_http_app.o
 .reginfo       0x00000000       0x18 build/WiFIG/production/_ext/1472/custom_http_app.o
 .pdr           0x00000000        0x0 build/WiFIG/production/_ext/1472/custom_http_app.o
 .text          0x00000000        0x0 build/WiFIG/production/_ext/1472/tcp6_demo_app.o
 .bss           0x00000000        0x0 build/WiFIG/production/_ext/1472/tcp6_demo_app.o
 .reginfo       0x00000000       0x18 build/WiFIG/production/_ext/1472/tcp6_demo_app.o
 .pdr           0x00000000       0xa0 build/WiFIG/production/_ext/1472/tcp6_demo_app.o
 .text          0x00000000        0x0 c:/program files (x86)/microchip/xc32/v1.21/bin/../lib/gcc/pic32mx/4.5.2/../../../../pic32mx/lib/./proc/32MX695F512H\default_isr_vectors.o
 .data          0x00000000        0x0 c:/program files (x86)/microchip/xc32/v1.21/bin/../lib/gcc/pic32mx/4.5.2/../../../../pic32mx/lib/./proc/32MX695F512H\default_isr_vectors.o
 .bss           0x00000000        0x0 c:/program files (x86)/microchip/xc32/v1.21/bin/../lib/gcc/pic32mx/4.5.2/../../../../pic32mx/lib/./proc/32MX695F512H\default_isr_vectors.o
 .reginfo       0x00000000       0x18 c:/program files (x86)/microchip/xc32/v1.21/bin/../lib/gcc/pic32mx/4.5.2/../../../../pic32mx/lib/./proc/32MX695F512H\default_isr_vectors.o
 .pdr           0x00000000        0x0 c:/program files (x86)/microchip/xc32/v1.21/bin/../lib/gcc/pic32mx/4.5.2/../../../../pic32mx/lib/./proc/32MX695F512H\default_isr_vectors.o
 .discard       0x00000000      0x100 c:/program files (x86)/microchip/xc32/v1.21/bin/../lib/gcc/pic32mx/4.5.2/../../../../pic32mx/lib/./proc/32MX695F512H\default_isr_vectors.o
 .text          0x00000000        0x0 c:/program files (x86)/microchip/xc32/v1.21/bin/../lib/gcc/pic32mx/4.5.2/../../../../pic32mx/lib/./proc/32MX695F512H\processor.o
 .data          0x00000000        0x0 c:/program files (x86)/microchip/xc32/v1.21/bin/../lib/gcc/pic32mx/4.5.2/../../../../pic32mx/lib/./proc/32MX695F512H\processor.o
 .bss           0x00000000        0x0 c:/program files (x86)/microchip/xc32/v1.21/bin/../lib/gcc/pic32mx/4.5.2/../../../../pic32mx/lib/./proc/32MX695F512H\processor.o
 .reginfo       0x00000000       0x18 c:/program files (x86)/microchip/xc32/v1.21/bin/../lib/gcc/pic32mx/4.5.2/../../../../pic32mx/lib/./proc/32MX695F512H\processor.o
 .pdr           0x00000000        0x0 c:/program files (x86)/microchip/xc32/v1.21/bin/../lib/gcc/pic32mx/4.5.2/../../../../pic32mx/lib/./proc/32MX695F512H\processor.o
 .text          0x00000000        0x0 c:/program files (x86)/microchip/xc32/v1.21/bin/../lib/gcc/pic32mx/4.5.2/../../../../pic32mx/lib/size\libmchp_peripheral.a(open_core_timer_lib.o)
 .data          0x00000000        0x0 c:/program files (x86)/microchip/xc32/v1.21/bin/../lib/gcc/pic32mx/4.5.2/../../../../pic32mx/lib/size\libmchp_peripheral.a(open_core_timer_lib.o)
 .bss           0x00000000        0x0 c:/program files (x86)/microchip/xc32/v1.21/bin/../lib/gcc/pic32mx/4.5.2/../../../../pic32mx/lib/size\libmchp_peripheral.a(open_core_timer_lib.o)
 .reginfo       0x00000000       0x18 c:/program files (x86)/microchip/xc32/v1.21/bin/../lib/gcc/pic32mx/4.5.2/../../../../pic32mx/lib/size\libmchp_peripheral.a(open_core_timer_lib.o)
 .pdr           0x00000000       0x20 c:/program files (x86)/microchip/xc32/v1.21/bin/../lib/gcc/pic32mx/4.5.2/../../../../pic32mx/lib/size\libmchp_peripheral.a(open_core_timer_lib.o)
 .text          0x00000000        0x0 c:/program files (x86)/microchip/xc32/v1.21/bin/../lib/gcc/pic32mx/4.5.2/../../../../pic32mx/lib/size\libmchp_peripheral_32MX695F512H.a(soft_reset_lib.o)
 .data          0x00000000        0x0 c:/program files (x86)/microchip/xc32/v1.21/bin/../lib/gcc/pic32mx/4.5.2/../../../../pic32mx/lib/size\libmchp_peripheral_32MX695F512H.a(soft_reset_lib.o)
 .bss           0x00000000        0x0 c:/program files (x86)/microchip/xc32/v1.21/bin/../lib/gcc/pic32mx/4.5.2/../../../../pic32mx/lib/size\libmchp_peripheral_32MX695F512H.a(soft_reset_lib.o)
 .reginfo       0x00000000       0x18 c:/program files (x86)/microchip/xc32/v1.21/bin/../lib/gcc/pic32mx/4.5.2/../../../../pic32mx/lib/size\libmchp_peripheral_32MX695F512H.a(soft_reset_lib.o)
 .pdr           0x00000000       0x20 c:/program files (x86)/microchip/xc32/v1.21/bin/../lib/gcc/pic32mx/4.5.2/../../../../pic32mx/lib/size\libmchp_peripheral_32MX695F512H.a(soft_reset_lib.o)
 .text.SoftReset
                0x00000000       0x78 c:/program files (x86)/microchip/xc32/v1.21/bin/../lib/gcc/pic32mx/4.5.2/../../../../pic32mx/lib/size\libmchp_peripheral_32MX695F512H.a(soft_reset_lib.o)
 .text          0x00000000        0x0 c:/program files (x86)/microchip/xc32/v1.21/bin/../lib/gcc/pic32mx/4.5.2/../../../../pic32mx/lib/size\libmchp_peripheral_32MX695F512H.a(pcache.o)
 .data          0x00000000        0x0 c:/program files (x86)/microchip/xc32/v1.21/bin/../lib/gcc/pic32mx/4.5.2/../../../../pic32mx/lib/size\libmchp_peripheral_32MX695F512H.a(pcache.o)
 .bss           0x00000000        0x0 c:/program files (x86)/microchip/xc32/v1.21/bin/../lib/gcc/pic32mx/4.5.2/../../../../pic32mx/lib/size\libmchp_peripheral_32MX695F512H.a(pcache.o)
 .reginfo       0x00000000       0x18 c:/program files (x86)/microchip/xc32/v1.21/bin/../lib/gcc/pic32mx/4.5.2/../../../../pic32mx/lib/size\libmchp_peripheral_32MX695F512H.a(pcache.o)
 .pdr           0x00000000       0x40 c:/program files (x86)/microchip/xc32/v1.21/bin/../lib/gcc/pic32mx/4.5.2/../../../../pic32mx/lib/size\libmchp_peripheral_32MX695F512H.a(pcache.o)
 .text.CheKseg0CacheOff
                0x00000000       0x18 c:/program files (x86)/microchip/xc32/v1.21/bin/../lib/gcc/pic32mx/4.5.2/../../../../pic32mx/lib/size\libmchp_peripheral_32MX695F512H.a(pcache.o)
 .text          0x00000000        0x0 c:/program files (x86)/microchip/xc32/v1.21/bin/../lib/gcc/pic32mx/4.5.2/../../../../pic32mx/lib/size\libmchp_peripheral_32MX695F512H.a(int_disable_interrupts_lib.o)
 .data          0x00000000        0x0 c:/program files (x86)/microchip/xc32/v1.21/bin/../lib/gcc/pic32mx/4.5.2/../../../../pic32mx/lib/size\libmchp_peripheral_32MX695F512H.a(int_disable_interrupts_lib.o)
 .bss           0x00000000        0x0 c:/program files (x86)/microchip/xc32/v1.21/bin/../lib/gcc/pic32mx/4.5.2/../../../../pic32mx/lib/size\libmchp_peripheral_32MX695F512H.a(int_disable_interrupts_lib.o)
 .reginfo       0x00000000       0x18 c:/program files (x86)/microchip/xc32/v1.21/bin/../lib/gcc/pic32mx/4.5.2/../../../../pic32mx/lib/size\libmchp_peripheral_32MX695F512H.a(int_disable_interrupts_lib.o)
 .pdr           0x00000000       0x20 c:/program files (x86)/microchip/xc32/v1.21/bin/../lib/gcc/pic32mx/4.5.2/../../../../pic32mx/lib/size\libmchp_peripheral_32MX695F512H.a(int_disable_interrupts_lib.o)
 .text          0x00000000        0x0 c:/program files (x86)/microchip/xc32/v1.21/bin/../lib/gcc/pic32mx/4.5.2/../../../../pic32mx/lib/size\libmchp_peripheral_32MX695F512H.a(int_restore_interrupts_lib.o)
 .data          0x00000000        0x0 c:/program files (x86)/microchip/xc32/v1.21/bin/../lib/gcc/pic32mx/4.5.2/../../../../pic32mx/lib/size\libmchp_peripheral_32MX695F512H.a(int_restore_interrupts_lib.o)
 .bss           0x00000000        0x0 c:/program files (x86)/microchip/xc32/v1.21/bin/../lib/gcc/pic32mx/4.5.2/../../../../pic32mx/lib/size\libmchp_peripheral_32MX695F512H.a(int_restore_interrupts_lib.o)
 .reginfo       0x00000000       0x18 c:/program files (x86)/microchip/xc32/v1.21/bin/../lib/gcc/pic32mx/4.5.2/../../../../pic32mx/lib/size\libmchp_peripheral_32MX695F512H.a(int_restore_interrupts_lib.o)
 .pdr           0x00000000       0x20 c:/program files (x86)/microchip/xc32/v1.21/bin/../lib/gcc/pic32mx/4.5.2/../../../../pic32mx/lib/size\libmchp_peripheral_32MX695F512H.a(int_restore_interrupts_lib.o)
 .text          0x00000000        0x0 c:/program files (x86)/microchip/xc32/v1.21/bin/../lib/gcc/pic32mx/4.5.2/../../../../pic32mx/lib/size\libmchp_peripheral_32MX695F512H.a(int_enable_mv_int_lib.o)
 .data          0x00000000        0x0 c:/program files (x86)/microchip/xc32/v1.21/bin/../lib/gcc/pic32mx/4.5.2/../../../../pic32mx/lib/size\libmchp_peripheral_32MX695F512H.a(int_enable_mv_int_lib.o)
 .bss           0x00000000        0x0 c:/program files (x86)/microchip/xc32/v1.21/bin/../lib/gcc/pic32mx/4.5.2/../../../../pic32mx/lib/size\libmchp_peripheral_32MX695F512H.a(int_enable_mv_int_lib.o)
 .reginfo       0x00000000       0x18 c:/program files (x86)/microchip/xc32/v1.21/bin/../lib/gcc/pic32mx/4.5.2/../../../../pic32mx/lib/size\libmchp_peripheral_32MX695F512H.a(int_enable_mv_int_lib.o)
 .pdr           0x00000000       0x20 c:/program files (x86)/microchip/xc32/v1.21/bin/../lib/gcc/pic32mx/4.5.2/../../../../pic32mx/lib/size\libmchp_peripheral_32MX695F512H.a(int_enable_mv_int_lib.o)
 .text          0x00000000        0x0 c:/program files (x86)/microchip/xc32/v1.21/bin/../lib/gcc/pic32mx/4.5.2/../../../../pic32mx/lib/size\libmchp_peripheral_32MX695F512H.a(int_tbl_lib.o)
 .data          0x00000000        0x0 c:/program files (x86)/microchip/xc32/v1.21/bin/../lib/gcc/pic32mx/4.5.2/../../../../pic32mx/lib/size\libmchp_peripheral_32MX695F512H.a(int_tbl_lib.o)
 .bss           0x00000000        0x0 c:/program files (x86)/microchip/xc32/v1.21/bin/../lib/gcc/pic32mx/4.5.2/../../../../pic32mx/lib/size\libmchp_peripheral_32MX695F512H.a(int_tbl_lib.o)
 .reginfo       0x00000000       0x18 c:/program files (x86)/microchip/xc32/v1.21/bin/../lib/gcc/pic32mx/4.5.2/../../../../pic32mx/lib/size\libmchp_peripheral_32MX695F512H.a(int_tbl_lib.o)
 .pdr           0x00000000      0x120 c:/program files (x86)/microchip/xc32/v1.21/bin/../lib/gcc/pic32mx/4.5.2/../../../../pic32mx/lib/size\libmchp_peripheral_32MX695F512H.a(int_tbl_lib.o)
 .text.INTSetFlag
                0x00000000       0x28 c:/program files (x86)/microchip/xc32/v1.21/bin/../lib/gcc/pic32mx/4.5.2/../../../../pic32mx/lib/size\libmchp_peripheral_32MX695F512H.a(int_tbl_lib.o)
 .text.INTGetFlag
                0x00000000       0x28 c:/program files (x86)/microchip/xc32/v1.21/bin/../lib/gcc/pic32mx/4.5.2/../../../../pic32mx/lib/size\libmchp_peripheral_32MX695F512H.a(int_tbl_lib.o)
 .text.INTGetEnable
                0x00000000       0x28 c:/program files (x86)/microchip/xc32/v1.21/bin/../lib/gcc/pic32mx/4.5.2/../../../../pic32mx/lib/size\libmchp_peripheral_32MX695F512H.a(int_tbl_lib.o)
 .text.INTGetVectorPriority
                0x00000000       0x2c c:/program files (x86)/microchip/xc32/v1.21/bin/../lib/gcc/pic32mx/4.5.2/../../../../pic32mx/lib/size\libmchp_peripheral_32MX695F512H.a(int_tbl_lib.o)
 .text.INTGetVectorSubPriority
                0x00000000       0x2c c:/program files (x86)/microchip/xc32/v1.21/bin/../lib/gcc/pic32mx/4.5.2/../../../../pic32mx/lib/size\libmchp_peripheral_32MX695F512H.a(int_tbl_lib.o)
 .text          0x00000000        0x0 c:/program files (x86)/microchip/xc32/v1.21/bin/../lib/gcc/pic32mx/4.5.2/../../../../pic32mx/lib/size\libmchp_peripheral_32MX695F512H.a(rtcc_init_lib.o)
 .data          0x00000000        0x0 c:/program files (x86)/microchip/xc32/v1.21/bin/../lib/gcc/pic32mx/4.5.2/../../../../pic32mx/lib/size\libmchp_peripheral_32MX695F512H.a(rtcc_init_lib.o)
 .bss           0x00000000        0x0 c:/program files (x86)/microchip/xc32/v1.21/bin/../lib/gcc/pic32mx/4.5.2/../../../../pic32mx/lib/size\libmchp_peripheral_32MX695F512H.a(rtcc_init_lib.o)
 .reginfo       0x00000000       0x18 c:/program files (x86)/microchip/xc32/v1.21/bin/../lib/gcc/pic32mx/4.5.2/../../../../pic32mx/lib/size\libmchp_peripheral_32MX695F512H.a(rtcc_init_lib.o)
 .pdr           0x00000000       0x20 c:/program files (x86)/microchip/xc32/v1.21/bin/../lib/gcc/pic32mx/4.5.2/../../../../pic32mx/lib/size\libmchp_peripheral_32MX695F512H.a(rtcc_init_lib.o)
 .text.RtccInit
                0x00000000      0x170 c:/program files (x86)/microchip/xc32/v1.21/bin/../lib/gcc/pic32mx/4.5.2/../../../../pic32mx/lib/size\libmchp_peripheral_32MX695F512H.a(rtcc_init_lib.o)
 .text          0x00000000        0x0 c:/program files (x86)/microchip/xc32/v1.21/bin/../lib/gcc/pic32mx/4.5.2/../../../../pic32mx/lib/size\libmchp_peripheral_32MX695F512H.a(rtcc_open_lib.o)
 .data          0x00000000        0x0 c:/program files (x86)/microchip/xc32/v1.21/bin/../lib/gcc/pic32mx/4.5.2/../../../../pic32mx/lib/size\libmchp_peripheral_32MX695F512H.a(rtcc_open_lib.o)
 .bss           0x00000000        0x0 c:/program files (x86)/microchip/xc32/v1.21/bin/../lib/gcc/pic32mx/4.5.2/../../../../pic32mx/lib/size\libmchp_peripheral_32MX695F512H.a(rtcc_open_lib.o)
 .reginfo       0x00000000       0x18 c:/program files (x86)/microchip/xc32/v1.21/bin/../lib/gcc/pic32mx/4.5.2/../../../../pic32mx/lib/size\libmchp_peripheral_32MX695F512H.a(rtcc_open_lib.o)
 .pdr           0x00000000       0x20 c:/program files (x86)/microchip/xc32/v1.21/bin/../lib/gcc/pic32mx/4.5.2/../../../../pic32mx/lib/size\libmchp_peripheral_32MX695F512H.a(rtcc_open_lib.o)
 .text.RtccOpen
                0x00000000      0x1b0 c:/program files (x86)/microchip/xc32/v1.21/bin/../lib/gcc/pic32mx/4.5.2/../../../../pic32mx/lib/size\libmchp_peripheral_32MX695F512H.a(rtcc_open_lib.o)
 .text          0x00000000        0x0 c:/program files (x86)/microchip/xc32/v1.21/bin/../lib/gcc/pic32mx/4.5.2/../../../../pic32mx/lib/size\libmchp_peripheral_32MX695F512H.a(spi_chn_data_rdy_lib.o)
 .data          0x00000000        0x0 c:/program files (x86)/microchip/xc32/v1.21/bin/../lib/gcc/pic32mx/4.5.2/../../../../pic32mx/lib/size\libmchp_peripheral_32MX695F512H.a(spi_chn_data_rdy_lib.o)
 .bss           0x00000000        0x0 c:/program files (x86)/microchip/xc32/v1.21/bin/../lib/gcc/pic32mx/4.5.2/../../../../pic32mx/lib/size\libmchp_peripheral_32MX695F512H.a(spi_chn_data_rdy_lib.o)
 .reginfo       0x00000000       0x18 c:/program files (x86)/microchip/xc32/v1.21/bin/../lib/gcc/pic32mx/4.5.2/../../../../pic32mx/lib/size\libmchp_peripheral_32MX695F512H.a(spi_chn_data_rdy_lib.o)
 .pdr           0x00000000       0x20 c:/program files (x86)/microchip/xc32/v1.21/bin/../lib/gcc/pic32mx/4.5.2/../../../../pic32mx/lib/size\libmchp_peripheral_32MX695F512H.a(spi_chn_data_rdy_lib.o)
 .text          0x00000000        0x0 c:/program files (x86)/microchip/xc32/v1.21/bin/../lib/gcc/pic32mx/4.5.2/../../../../pic32mx/lib/size\libmchp_peripheral_32MX695F512H.a(spi_chn_getc_lib.o)
 .data          0x00000000        0x0 c:/program files (x86)/microchip/xc32/v1.21/bin/../lib/gcc/pic32mx/4.5.2/../../../../pic32mx/lib/size\libmchp_peripheral_32MX695F512H.a(spi_chn_getc_lib.o)
 .bss           0x00000000        0x0 c:/program files (x86)/microchip/xc32/v1.21/bin/../lib/gcc/pic32mx/4.5.2/../../../../pic32mx/lib/size\libmchp_peripheral_32MX695F512H.a(spi_chn_getc_lib.o)
 .reginfo       0x00000000       0x18 c:/program files (x86)/microchip/xc32/v1.21/bin/../lib/gcc/pic32mx/4.5.2/../../../../pic32mx/lib/size\libmchp_peripheral_32MX695F512H.a(spi_chn_getc_lib.o)
 .pdr           0x00000000       0x40 c:/program files (x86)/microchip/xc32/v1.21/bin/../lib/gcc/pic32mx/4.5.2/../../../../pic32mx/lib/size\libmchp_peripheral_32MX695F512H.a(spi_chn_getc_lib.o)
 .text.SpiChnGetC
                0x00000000       0x54 c:/program files (x86)/microchip/xc32/v1.21/bin/../lib/gcc/pic32mx/4.5.2/../../../../pic32mx/lib/size\libmchp_peripheral_32MX695F512H.a(spi_chn_getc_lib.o)
 .text          0x00000000        0x0 c:/program files (x86)/microchip/xc32/v1.21/bin/../lib/gcc/pic32mx/4.5.2/../../../../pic32mx/lib/size\libmchp_peripheral_32MX695F512H.a(spi_chn_open_lib.o)
 .data          0x00000000        0x0 c:/program files (x86)/microchip/xc32/v1.21/bin/../lib/gcc/pic32mx/4.5.2/../../../../pic32mx/lib/size\libmchp_peripheral_32MX695F512H.a(spi_chn_open_lib.o)
 .bss           0x00000000        0x0 c:/program files (x86)/microchip/xc32/v1.21/bin/../lib/gcc/pic32mx/4.5.2/../../../../pic32mx/lib/size\libmchp_peripheral_32MX695F512H.a(spi_chn_open_lib.o)
 .reginfo       0x00000000       0x18 c:/program files (x86)/microchip/xc32/v1.21/bin/../lib/gcc/pic32mx/4.5.2/../../../../pic32mx/lib/size\libmchp_peripheral_32MX695F512H.a(spi_chn_open_lib.o)
 .pdr           0x00000000       0x20 c:/program files (x86)/microchip/xc32/v1.21/bin/../lib/gcc/pic32mx/4.5.2/../../../../pic32mx/lib/size\libmchp_peripheral_32MX695F512H.a(spi_chn_open_lib.o)
 .text          0x00000000        0x0 c:/program files (x86)/microchip/xc32/v1.21/bin/../lib/gcc/pic32mx/4.5.2/../../../../pic32mx/lib/size\libmchp_peripheral_32MX695F512H.a(spi_chn_putc_lib.o)
 .data          0x00000000        0x0 c:/program files (x86)/microchip/xc32/v1.21/bin/../lib/gcc/pic32mx/4.5.2/../../../../pic32mx/lib/size\libmchp_peripheral_32MX695F512H.a(spi_chn_putc_lib.o)
 .bss           0x00000000        0x0 c:/program files (x86)/microchip/xc32/v1.21/bin/../lib/gcc/pic32mx/4.5.2/../../../../pic32mx/lib/size\libmchp_peripheral_32MX695F512H.a(spi_chn_putc_lib.o)
 .reginfo       0x00000000       0x18 c:/program files (x86)/microchip/xc32/v1.21/bin/../lib/gcc/pic32mx/4.5.2/../../../../pic32mx/lib/size\libmchp_peripheral_32MX695F512H.a(spi_chn_putc_lib.o)
 .pdr           0x00000000       0x60 c:/program files (x86)/microchip/xc32/v1.21/bin/../lib/gcc/pic32mx/4.5.2/../../../../pic32mx/lib/size\libmchp_peripheral_32MX695F512H.a(spi_chn_putc_lib.o)
 .text.SpiChnPutC
                0x00000000       0x54 c:/program files (x86)/microchip/xc32/v1.21/bin/../lib/gcc/pic32mx/4.5.2/../../../../pic32mx/lib/size\libmchp_peripheral_32MX695F512H.a(spi_chn_putc_lib.o)
 .text.SpiChnBuffer
                0x00000000       0x1c c:/program files (x86)/microchip/xc32/v1.21/bin/../lib/gcc/pic32mx/4.5.2/../../../../pic32mx/lib/size\libmchp_peripheral_32MX695F512H.a(spi_chn_putc_lib.o)
 .text          0x00000000        0x0 c:/program files (x86)/microchip/xc32/v1.21/bin/../lib/gcc/pic32mx/4.5.2/../../../../pic32mx/lib/size\libmchp_peripheral_32MX695F512H.a(spi_chn_tx_buff_empty_lib.o)
 .data          0x00000000        0x0 c:/program files (x86)/microchip/xc32/v1.21/bin/../lib/gcc/pic32mx/4.5.2/../../../../pic32mx/lib/size\libmchp_peripheral_32MX695F512H.a(spi_chn_tx_buff_empty_lib.o)
 .bss           0x00000000        0x0 c:/program files (x86)/microchip/xc32/v1.21/bin/../lib/gcc/pic32mx/4.5.2/../../../../pic32mx/lib/size\libmchp_peripheral_32MX695F512H.a(spi_chn_tx_buff_empty_lib.o)
 .reginfo       0x00000000       0x18 c:/program files (x86)/microchip/xc32/v1.21/bin/../lib/gcc/pic32mx/4.5.2/../../../../pic32mx/lib/size\libmchp_peripheral_32MX695F512H.a(spi_chn_tx_buff_empty_lib.o)
 .pdr           0x00000000       0x20 c:/program files (x86)/microchip/xc32/v1.21/bin/../lib/gcc/pic32mx/4.5.2/../../../../pic32mx/lib/size\libmchp_peripheral_32MX695F512H.a(spi_chn_tx_buff_empty_lib.o)
 .text          0x00000000        0x0 c:/program files (x86)/microchip/xc32/v1.21/bin/../lib/gcc/pic32mx/4.5.2/../../../../pic32mx/lib/size\libmchp_peripheral_32MX695F512H.a(spi_io_tbl_libp.o)
 .data          0x00000000        0x0 c:/program files (x86)/microchip/xc32/v1.21/bin/../lib/gcc/pic32mx/4.5.2/../../../../pic32mx/lib/size\libmchp_peripheral_32MX695F512H.a(spi_io_tbl_libp.o)
 .bss           0x00000000        0x0 c:/program files (x86)/microchip/xc32/v1.21/bin/../lib/gcc/pic32mx/4.5.2/../../../../pic32mx/lib/size\libmchp_peripheral_32MX695F512H.a(spi_io_tbl_libp.o)
 .reginfo       0x00000000       0x18 c:/program files (x86)/microchip/xc32/v1.21/bin/../lib/gcc/pic32mx/4.5.2/../../../../pic32mx/lib/size\libmchp_peripheral_32MX695F512H.a(spi_io_tbl_libp.o)
 .pdr           0x00000000        0x0 c:/program files (x86)/microchip/xc32/v1.21/bin/../lib/gcc/pic32mx/4.5.2/../../../../pic32mx/lib/size\libmchp_peripheral_32MX695F512H.a(spi_io_tbl_libp.o)
 .text          0x00000000        0x0 c:/program files (x86)/microchip/xc32/v1.21/bin/../lib/gcc/pic32mx/4.5.2/../../../../pic32mx/lib/size\libmchp_peripheral_32MX695F512H.a(spi_map_tbl_libp.o)
 .data          0x00000000        0x0 c:/program files (x86)/microchip/xc32/v1.21/bin/../lib/gcc/pic32mx/4.5.2/../../../../pic32mx/lib/size\libmchp_peripheral_32MX695F512H.a(spi_map_tbl_libp.o)
 .bss           0x00000000        0x0 c:/program files (x86)/microchip/xc32/v1.21/bin/../lib/gcc/pic32mx/4.5.2/../../../../pic32mx/lib/size\libmchp_peripheral_32MX695F512H.a(spi_map_tbl_libp.o)
 .reginfo       0x00000000       0x18 c:/program files (x86)/microchip/xc32/v1.21/bin/../lib/gcc/pic32mx/4.5.2/../../../../pic32mx/lib/size\libmchp_peripheral_32MX695F512H.a(spi_map_tbl_libp.o)
 .pdr           0x00000000        0x0 c:/program files (x86)/microchip/xc32/v1.21/bin/../lib/gcc/pic32mx/4.5.2/../../../../pic32mx/lib/size\libmchp_peripheral_32MX695F512H.a(spi_map_tbl_libp.o)
 .text          0x00000000        0x0 c:/program files (x86)/microchip/xc32/v1.21/bin/../lib/gcc/pic32mx/4.5.2/../../../../pic32mx/lib/size\libmchp_peripheral_32MX695F512H.a(port_set_pins_digital_in_lib.o)
 .data          0x00000000        0x0 c:/program files (x86)/microchip/xc32/v1.21/bin/../lib/gcc/pic32mx/4.5.2/../../../../pic32mx/lib/size\libmchp_peripheral_32MX695F512H.a(port_set_pins_digital_in_lib.o)
 .bss           0x00000000        0x0 c:/program files (x86)/microchip/xc32/v1.21/bin/../lib/gcc/pic32mx/4.5.2/../../../../pic32mx/lib/size\libmchp_peripheral_32MX695F512H.a(port_set_pins_digital_in_lib.o)
 .reginfo       0x00000000       0x18 c:/program files (x86)/microchip/xc32/v1.21/bin/../lib/gcc/pic32mx/4.5.2/../../../../pic32mx/lib/size\libmchp_peripheral_32MX695F512H.a(port_set_pins_digital_in_lib.o)
 .pdr           0x00000000       0x20 c:/program files (x86)/microchip/xc32/v1.21/bin/../lib/gcc/pic32mx/4.5.2/../../../../pic32mx/lib/size\libmchp_peripheral_32MX695F512H.a(port_set_pins_digital_in_lib.o)
 .text          0x00000000        0x0 c:/program files (x86)/microchip/xc32/v1.21/bin/../lib/gcc/pic32mx/4.5.2/../../../../pic32mx/lib/size\libmchp_peripheral_32MX695F512H.a(port_set_pins_digital_out_lib.o)
 .data          0x00000000        0x0 c:/program files (x86)/microchip/xc32/v1.21/bin/../lib/gcc/pic32mx/4.5.2/../../../../pic32mx/lib/size\libmchp_peripheral_32MX695F512H.a(port_set_pins_digital_out_lib.o)
 .bss           0x00000000        0x0 c:/program files (x86)/microchip/xc32/v1.21/bin/../lib/gcc/pic32mx/4.5.2/../../../../pic32mx/lib/size\libmchp_peripheral_32MX695F512H.a(port_set_pins_digital_out_lib.o)
 .reginfo       0x00000000       0x18 c:/program files (x86)/microchip/xc32/v1.21/bin/../lib/gcc/pic32mx/4.5.2/../../../../pic32mx/lib/size\libmchp_peripheral_32MX695F512H.a(port_set_pins_digital_out_lib.o)
 .pdr           0x00000000       0x20 c:/program files (x86)/microchip/xc32/v1.21/bin/../lib/gcc/pic32mx/4.5.2/../../../../pic32mx/lib/size\libmchp_peripheral_32MX695F512H.a(port_set_pins_digital_out_lib.o)
 .text          0x00000000        0x0 c:/program files (x86)/microchip/xc32/v1.21/bin/../lib/gcc/pic32mx/4.5.2/../../../../pic32mx/lib/size\libmchp_peripheral_32MX695F512H.a(_ports_tbl_libp.o)
 .data          0x00000000        0x0 c:/program files (x86)/microchip/xc32/v1.21/bin/../lib/gcc/pic32mx/4.5.2/../../../../pic32mx/lib/size\libmchp_peripheral_32MX695F512H.a(_ports_tbl_libp.o)
 .bss           0x00000000        0x0 c:/program files (x86)/microchip/xc32/v1.21/bin/../lib/gcc/pic32mx/4.5.2/../../../../pic32mx/lib/size\libmchp_peripheral_32MX695F512H.a(_ports_tbl_libp.o)
 .reginfo       0x00000000       0x18 c:/program files (x86)/microchip/xc32/v1.21/bin/../lib/gcc/pic32mx/4.5.2/../../../../pic32mx/lib/size\libmchp_peripheral_32MX695F512H.a(_ports_tbl_libp.o)
 .pdr           0x00000000        0x0 c:/program files (x86)/microchip/xc32/v1.21/bin/../lib/gcc/pic32mx/4.5.2/../../../../pic32mx/lib/size\libmchp_peripheral_32MX695F512H.a(_ports_tbl_libp.o)
 .text          0x00000000        0x0 c:/program files (x86)/microchip/xc32/v1.21/bin/../lib/gcc/pic32mx/4.5.2/../../../../pic32mx/lib/size\libmchp_peripheral_32MX695F512H.a(int_enable_interrupts_lib.o)
 .data          0x00000000        0x0 c:/program files (x86)/microchip/xc32/v1.21/bin/../lib/gcc/pic32mx/4.5.2/../../../../pic32mx/lib/size\libmchp_peripheral_32MX695F512H.a(int_enable_interrupts_lib.o)
 .bss           0x00000000        0x0 c:/program files (x86)/microchip/xc32/v1.21/bin/../lib/gcc/pic32mx/4.5.2/../../../../pic32mx/lib/size\libmchp_peripheral_32MX695F512H.a(int_enable_interrupts_lib.o)
 .reginfo       0x00000000       0x18 c:/program files (x86)/microchip/xc32/v1.21/bin/../lib/gcc/pic32mx/4.5.2/../../../../pic32mx/lib/size\libmchp_peripheral_32MX695F512H.a(int_enable_interrupts_lib.o)
 .pdr           0x00000000       0x20 c:/program files (x86)/microchip/xc32/v1.21/bin/../lib/gcc/pic32mx/4.5.2/../../../../pic32mx/lib/size\libmchp_peripheral_32MX695F512H.a(int_enable_interrupts_lib.o)
 .text          0x00000000        0x0 c:/program files (x86)/microchip/xc32/v1.21/bin/../lib/gcc/pic32mx/4.5.2/../../../../pic32mx/lib/size\libmchp_peripheral_32MX695F512H.a(_rtcc_wait_clock_off_lib.o)
 .data          0x00000000        0x0 c:/program files (x86)/microchip/xc32/v1.21/bin/../lib/gcc/pic32mx/4.5.2/../../../../pic32mx/lib/size\libmchp_peripheral_32MX695F512H.a(_rtcc_wait_clock_off_lib.o)
 .bss           0x00000000        0x0 c:/program files (x86)/microchip/xc32/v1.21/bin/../lib/gcc/pic32mx/4.5.2/../../../../pic32mx/lib/size\libmchp_peripheral_32MX695F512H.a(_rtcc_wait_clock_off_lib.o)
 .reginfo       0x00000000       0x18 c:/program files (x86)/microchip/xc32/v1.21/bin/../lib/gcc/pic32mx/4.5.2/../../../../pic32mx/lib/size\libmchp_peripheral_32MX695F512H.a(_rtcc_wait_clock_off_lib.o)
 .pdr           0x00000000       0x40 c:/program files (x86)/microchip/xc32/v1.21/bin/../lib/gcc/pic32mx/4.5.2/../../../../pic32mx/lib/size\libmchp_peripheral_32MX695F512H.a(_rtcc_wait_clock_off_lib.o)
 .text._RtccWaitClockOff
                0x00000000      0x104 c:/program files (x86)/microchip/xc32/v1.21/bin/../lib/gcc/pic32mx/4.5.2/../../../../pic32mx/lib/size\libmchp_peripheral_32MX695F512H.a(_rtcc_wait_clock_off_lib.o)
 .text._RtccSetClockWait
                0x00000000       0x14 c:/program files (x86)/microchip/xc32/v1.21/bin/../lib/gcc/pic32mx/4.5.2/../../../../pic32mx/lib/size\libmchp_peripheral_32MX695F512H.a(_rtcc_wait_clock_off_lib.o)
 .sdata         0x00000000        0x8 c:/program files (x86)/microchip/xc32/v1.21/bin/../lib/gcc/pic32mx/4.5.2/../../../../pic32mx/lib/size\libmchp_peripheral_32MX695F512H.a(_rtcc_wait_clock_off_lib.o)
 .text          0x00000000        0x0 c:/program files (x86)/microchip/xc32/v1.21/bin/../lib/gcc/pic32mx/4.5.2/../../../../pic32mx/lib/size\libmchp_peripheral_32MX695F512H.a(read_core_timer_lib.o)
 .data          0x00000000        0x0 c:/program files (x86)/microchip/xc32/v1.21/bin/../lib/gcc/pic32mx/4.5.2/../../../../pic32mx/lib/size\libmchp_peripheral_32MX695F512H.a(read_core_timer_lib.o)
 .bss           0x00000000        0x0 c:/program files (x86)/microchip/xc32/v1.21/bin/../lib/gcc/pic32mx/4.5.2/../../../../pic32mx/lib/size\libmchp_peripheral_32MX695F512H.a(read_core_timer_lib.o)
 .reginfo       0x00000000       0x18 c:/program files (x86)/microchip/xc32/v1.21/bin/../lib/gcc/pic32mx/4.5.2/../../../../pic32mx/lib/size\libmchp_peripheral_32MX695F512H.a(read_core_timer_lib.o)
 .pdr           0x00000000       0x20 c:/program files (x86)/microchip/xc32/v1.21/bin/../lib/gcc/pic32mx/4.5.2/../../../../pic32mx/lib/size\libmchp_peripheral_32MX695F512H.a(read_core_timer_lib.o)
 .text.ReadCoreTimer
                0x00000000        0x8 c:/program files (x86)/microchip/xc32/v1.21/bin/../lib/gcc/pic32mx/4.5.2/../../../../pic32mx/lib/size\libmchp_peripheral_32MX695F512H.a(read_core_timer_lib.o)
 .data          0x00000000        0x0 c:/program files (x86)/microchip/xc32/v1.21/bin/../lib/gcc/pic32mx/4.5.2/size\libgcc.a(_udivdi3.o)
 .bss           0x00000000        0x0 c:/program files (x86)/microchip/xc32/v1.21/bin/../lib/gcc/pic32mx/4.5.2/size\libgcc.a(_udivdi3.o)
 .reginfo       0x00000000       0x18 c:/program files (x86)/microchip/xc32/v1.21/bin/../lib/gcc/pic32mx/4.5.2/size\libgcc.a(_udivdi3.o)
 .pdr           0x00000000       0x20 c:/program files (x86)/microchip/xc32/v1.21/bin/../lib/gcc/pic32mx/4.5.2/size\libgcc.a(_udivdi3.o)
 .data          0x00000000        0x0 c:/program files (x86)/microchip/xc32/v1.21/bin/../lib/gcc/pic32mx/4.5.2/../../../../pic32mx/lib/size\libpic32.a(memcmp.o)
 .bss           0x00000000        0x0 c:/program files (x86)/microchip/xc32/v1.21/bin/../lib/gcc/pic32mx/4.5.2/../../../../pic32mx/lib/size\libpic32.a(memcmp.o)
 .reginfo       0x00000000       0x18 c:/program files (x86)/microchip/xc32/v1.21/bin/../lib/gcc/pic32mx/4.5.2/../../../../pic32mx/lib/size\libpic32.a(memcmp.o)
 .pdr           0x00000000       0x20 c:/program files (x86)/microchip/xc32/v1.21/bin/../lib/gcc/pic32mx/4.5.2/../../../../pic32mx/lib/size\libpic32.a(memcmp.o)
 .data          0x00000000        0x0 c:/program files (x86)/microchip/xc32/v1.21/bin/../lib/gcc/pic32mx/4.5.2/../../../../pic32mx/lib/size\libpic32.a(memcpy.o)
 .bss           0x00000000        0x0 c:/program files (x86)/microchip/xc32/v1.21/bin/../lib/gcc/pic32mx/4.5.2/../../../../pic32mx/lib/size\libpic32.a(memcpy.o)
 .reginfo       0x00000000       0x18 c:/program files (x86)/microchip/xc32/v1.21/bin/../lib/gcc/pic32mx/4.5.2/../../../../pic32mx/lib/size\libpic32.a(memcpy.o)
 .pdr           0x00000000       0x20 c:/program files (x86)/microchip/xc32/v1.21/bin/../lib/gcc/pic32mx/4.5.2/../../../../pic32mx/lib/size\libpic32.a(memcpy.o)
 .data          0x00000000        0x0 c:/program files (x86)/microchip/xc32/v1.21/bin/../lib/gcc/pic32mx/4.5.2/../../../../pic32mx/lib/size\libpic32.a(memset.o)
 .bss           0x00000000        0x0 c:/program files (x86)/microchip/xc32/v1.21/bin/../lib/gcc/pic32mx/4.5.2/../../../../pic32mx/lib/size\libpic32.a(memset.o)
 .reginfo       0x00000000       0x18 c:/program files (x86)/microchip/xc32/v1.21/bin/../lib/gcc/pic32mx/4.5.2/../../../../pic32mx/lib/size\libpic32.a(memset.o)
 .pdr           0x00000000       0x20 c:/program files (x86)/microchip/xc32/v1.21/bin/../lib/gcc/pic32mx/4.5.2/../../../../pic32mx/lib/size\libpic32.a(memset.o)
 .data          0x00000000        0x0 c:/program files (x86)/microchip/xc32/v1.21/bin/../lib/gcc/pic32mx/4.5.2/../../../../pic32mx/lib/size\libpic32.a(strcmp.o)
 .bss           0x00000000        0x0 c:/program files (x86)/microchip/xc32/v1.21/bin/../lib/gcc/pic32mx/4.5.2/../../../../pic32mx/lib/size\libpic32.a(strcmp.o)
 .reginfo       0x00000000       0x18 c:/program files (x86)/microchip/xc32/v1.21/bin/../lib/gcc/pic32mx/4.5.2/../../../../pic32mx/lib/size\libpic32.a(strcmp.o)
 .pdr           0x00000000       0x20 c:/program files (x86)/microchip/xc32/v1.21/bin/../lib/gcc/pic32mx/4.5.2/../../../../pic32mx/lib/size\libpic32.a(strcmp.o)
 .data          0x00000000        0x0 c:/program files (x86)/microchip/xc32/v1.21/bin/../lib/gcc/pic32mx/4.5.2/../../../../pic32mx/lib/size\libpic32.a(strcpy.o)
 .bss           0x00000000        0x0 c:/program files (x86)/microchip/xc32/v1.21/bin/../lib/gcc/pic32mx/4.5.2/../../../../pic32mx/lib/size\libpic32.a(strcpy.o)
 .reginfo       0x00000000       0x18 c:/program files (x86)/microchip/xc32/v1.21/bin/../lib/gcc/pic32mx/4.5.2/../../../../pic32mx/lib/size\libpic32.a(strcpy.o)
 .pdr           0x00000000       0x20 c:/program files (x86)/microchip/xc32/v1.21/bin/../lib/gcc/pic32mx/4.5.2/../../../../pic32mx/lib/size\libpic32.a(strcpy.o)
 .data          0x00000000        0x0 c:/program files (x86)/microchip/xc32/v1.21/bin/../lib/gcc/pic32mx/4.5.2/../../../../pic32mx/lib/size\libpic32.a(strlen.o)
 .bss           0x00000000        0x0 c:/program files (x86)/microchip/xc32/v1.21/bin/../lib/gcc/pic32mx/4.5.2/../../../../pic32mx/lib/size\libpic32.a(strlen.o)
 .reginfo       0x00000000       0x18 c:/program files (x86)/microchip/xc32/v1.21/bin/../lib/gcc/pic32mx/4.5.2/../../../../pic32mx/lib/size\libpic32.a(strlen.o)
 .pdr           0x00000000       0x20 c:/program files (x86)/microchip/xc32/v1.21/bin/../lib/gcc/pic32mx/4.5.2/../../../../pic32mx/lib/size\libpic32.a(strlen.o)
 .text          0x00000000        0x0 c:/program files (x86)/microchip/xc32/v1.21/bin/../lib/gcc/pic32mx/4.5.2/../../../../pic32mx/lib/size\libpic32.a(default-bootstrap-exception-handler.o)
 .data          0x00000000        0x0 c:/program files (x86)/microchip/xc32/v1.21/bin/../lib/gcc/pic32mx/4.5.2/../../../../pic32mx/lib/size\libpic32.a(default-bootstrap-exception-handler.o)
 .bss           0x00000000        0x0 c:/program files (x86)/microchip/xc32/v1.21/bin/../lib/gcc/pic32mx/4.5.2/../../../../pic32mx/lib/size\libpic32.a(default-bootstrap-exception-handler.o)
 .reginfo       0x00000000       0x18 c:/program files (x86)/microchip/xc32/v1.21/bin/../lib/gcc/pic32mx/4.5.2/../../../../pic32mx/lib/size\libpic32.a(default-bootstrap-exception-handler.o)
 .pdr           0x00000000       0x20 c:/program files (x86)/microchip/xc32/v1.21/bin/../lib/gcc/pic32mx/4.5.2/../../../../pic32mx/lib/size\libpic32.a(default-bootstrap-exception-handler.o)
 .text          0x00000000        0x0 c:/program files (x86)/microchip/xc32/v1.21/bin/../lib/gcc/pic32mx/4.5.2/../../../../pic32mx/lib/size\libpic32.a(default-on-reset.o)
 .data          0x00000000        0x0 c:/program files (x86)/microchip/xc32/v1.21/bin/../lib/gcc/pic32mx/4.5.2/../../../../pic32mx/lib/size\libpic32.a(default-on-reset.o)
 .bss           0x00000000        0x0 c:/program files (x86)/microchip/xc32/v1.21/bin/../lib/gcc/pic32mx/4.5.2/../../../../pic32mx/lib/size\libpic32.a(default-on-reset.o)
 .reginfo       0x00000000       0x18 c:/program files (x86)/microchip/xc32/v1.21/bin/../lib/gcc/pic32mx/4.5.2/../../../../pic32mx/lib/size\libpic32.a(default-on-reset.o)
 .pdr           0x00000000       0x20 c:/program files (x86)/microchip/xc32/v1.21/bin/../lib/gcc/pic32mx/4.5.2/../../../../pic32mx/lib/size\libpic32.a(default-on-reset.o)
 .text          0x00000000        0x0 c:/program files (x86)/microchip/xc32/v1.21/bin/../lib/gcc/pic32mx/4.5.2/../../../../pic32mx/lib/size\libpic32.a(default-on-bootstrap.o)
 .data          0x00000000        0x0 c:/program files (x86)/microchip/xc32/v1.21/bin/../lib/gcc/pic32mx/4.5.2/../../../../pic32mx/lib/size\libpic32.a(default-on-bootstrap.o)
 .bss           0x00000000        0x0 c:/program files (x86)/microchip/xc32/v1.21/bin/../lib/gcc/pic32mx/4.5.2/../../../../pic32mx/lib/size\libpic32.a(default-on-bootstrap.o)
 .reginfo       0x00000000       0x18 c:/program files (x86)/microchip/xc32/v1.21/bin/../lib/gcc/pic32mx/4.5.2/../../../../pic32mx/lib/size\libpic32.a(default-on-bootstrap.o)
 .pdr           0x00000000       0x20 c:/program files (x86)/microchip/xc32/v1.21/bin/../lib/gcc/pic32mx/4.5.2/../../../../pic32mx/lib/size\libpic32.a(default-on-bootstrap.o)
 .data          0x00000000        0x0 c:/program files (x86)/microchip/xc32/v1.21/bin/../lib/gcc/pic32mx/4.5.2/../../../../pic32mx/lib/size\libpic32.a(default-nmi-handler.o)
 .bss           0x00000000        0x0 c:/program files (x86)/microchip/xc32/v1.21/bin/../lib/gcc/pic32mx/4.5.2/../../../../pic32mx/lib/size\libpic32.a(default-nmi-handler.o)
 .reginfo       0x00000000       0x18 c:/program files (x86)/microchip/xc32/v1.21/bin/../lib/gcc/pic32mx/4.5.2/../../../../pic32mx/lib/size\libpic32.a(default-nmi-handler.o)
 .pdr           0x00000000       0x20 c:/program files (x86)/microchip/xc32/v1.21/bin/../lib/gcc/pic32mx/4.5.2/../../../../pic32mx/lib/size\libpic32.a(default-nmi-handler.o)
 .text          0x00000000        0x0 c:/program files (x86)/microchip/xc32/v1.21/bin/../lib/gcc/pic32mx/4.5.2/../../../../pic32mx/lib/size\libpic32.a(general-exception.o)
 .data          0x00000000        0x0 c:/program files (x86)/microchip/xc32/v1.21/bin/../lib/gcc/pic32mx/4.5.2/../../../../pic32mx/lib/size\libpic32.a(general-exception.o)
 .bss           0x00000000        0x0 c:/program files (x86)/microchip/xc32/v1.21/bin/../lib/gcc/pic32mx/4.5.2/../../../../pic32mx/lib/size\libpic32.a(general-exception.o)
 .reginfo       0x00000000       0x18 c:/program files (x86)/microchip/xc32/v1.21/bin/../lib/gcc/pic32mx/4.5.2/../../../../pic32mx/lib/size\libpic32.a(general-exception.o)
 .pdr           0x00000000       0x20 c:/program files (x86)/microchip/xc32/v1.21/bin/../lib/gcc/pic32mx/4.5.2/../../../../pic32mx/lib/size\libpic32.a(general-exception.o)
 .text          0x00000000        0x0 c:/program files (x86)/microchip/xc32/v1.21/bin/../lib/gcc/pic32mx/4.5.2/../../../../pic32mx/lib/size\libpic32.a(vector1.o)
 .data          0x00000000        0x0 c:/program files (x86)/microchip/xc32/v1.21/bin/../lib/gcc/pic32mx/4.5.2/../../../../pic32mx/lib/size\libpic32.a(vector1.o)
 .bss           0x00000000        0x0 c:/program files (x86)/microchip/xc32/v1.21/bin/../lib/gcc/pic32mx/4.5.2/../../../../pic32mx/lib/size\libpic32.a(vector1.o)
 .reginfo       0x00000000       0x18 c:/program files (x86)/microchip/xc32/v1.21/bin/../lib/gcc/pic32mx/4.5.2/../../../../pic32mx/lib/size\libpic32.a(vector1.o)
 .pdr           0x00000000       0x20 c:/program files (x86)/microchip/xc32/v1.21/bin/../lib/gcc/pic32mx/4.5.2/../../../../pic32mx/lib/size\libpic32.a(vector1.o)
 .text          0x00000000        0x0 c:/program files (x86)/microchip/xc32/v1.21/bin/../lib/gcc/pic32mx/4.5.2/../../../../pic32mx/lib/size\libpic32.a(vector2.o)
 .data          0x00000000        0x0 c:/program files (x86)/microchip/xc32/v1.21/bin/../lib/gcc/pic32mx/4.5.2/../../../../pic32mx/lib/size\libpic32.a(vector2.o)
 .bss           0x00000000        0x0 c:/program files (x86)/microchip/xc32/v1.21/bin/../lib/gcc/pic32mx/4.5.2/../../../../pic32mx/lib/size\libpic32.a(vector2.o)
 .reginfo       0x00000000       0x18 c:/program files (x86)/microchip/xc32/v1.21/bin/../lib/gcc/pic32mx/4.5.2/../../../../pic32mx/lib/size\libpic32.a(vector2.o)
 .pdr           0x00000000       0x20 c:/program files (x86)/microchip/xc32/v1.21/bin/../lib/gcc/pic32mx/4.5.2/../../../../pic32mx/lib/size\libpic32.a(vector2.o)
 .text          0x00000000        0x0 c:/program files (x86)/microchip/xc32/v1.21/bin/../lib/gcc/pic32mx/4.5.2/../../../../pic32mx/lib/size\libpic32.a(vector3.o)
 .data          0x00000000        0x0 c:/program files (x86)/microchip/xc32/v1.21/bin/../lib/gcc/pic32mx/4.5.2/../../../../pic32mx/lib/size\libpic32.a(vector3.o)
 .bss           0x00000000        0x0 c:/program files (x86)/microchip/xc32/v1.21/bin/../lib/gcc/pic32mx/4.5.2/../../../../pic32mx/lib/size\libpic32.a(vector3.o)
 .reginfo       0x00000000       0x18 c:/program files (x86)/microchip/xc32/v1.21/bin/../lib/gcc/pic32mx/4.5.2/../../../../pic32mx/lib/size\libpic32.a(vector3.o)
 .pdr           0x00000000       0x20 c:/program files (x86)/microchip/xc32/v1.21/bin/../lib/gcc/pic32mx/4.5.2/../../../../pic32mx/lib/size\libpic32.a(vector3.o)
 .text          0x00000000        0x0 c:/program files (x86)/microchip/xc32/v1.21/bin/../lib/gcc/pic32mx/4.5.2/../../../../pic32mx/lib/size\libpic32.a(vector4.o)
 .data          0x00000000        0x0 c:/program files (x86)/microchip/xc32/v1.21/bin/../lib/gcc/pic32mx/4.5.2/../../../../pic32mx/lib/size\libpic32.a(vector4.o)
 .bss           0x00000000        0x0 c:/program files (x86)/microchip/xc32/v1.21/bin/../lib/gcc/pic32mx/4.5.2/../../../../pic32mx/lib/size\libpic32.a(vector4.o)
 .reginfo       0x00000000       0x18 c:/program files (x86)/microchip/xc32/v1.21/bin/../lib/gcc/pic32mx/4.5.2/../../../../pic32mx/lib/size\libpic32.a(vector4.o)
 .pdr           0x00000000       0x20 c:/program files (x86)/microchip/xc32/v1.21/bin/../lib/gcc/pic32mx/4.5.2/../../../../pic32mx/lib/size\libpic32.a(vector4.o)
 .text          0x00000000        0x0 c:/program files (x86)/microchip/xc32/v1.21/bin/../lib/gcc/pic32mx/4.5.2/../../../../pic32mx/lib/size\libpic32.a(vector5.o)
 .data          0x00000000        0x0 c:/program files (x86)/microchip/xc32/v1.21/bin/../lib/gcc/pic32mx/4.5.2/../../../../pic32mx/lib/size\libpic32.a(vector5.o)
 .bss           0x00000000        0x0 c:/program files (x86)/microchip/xc32/v1.21/bin/../lib/gcc/pic32mx/4.5.2/../../../../pic32mx/lib/size\libpic32.a(vector5.o)
 .reginfo       0x00000000       0x18 c:/program files (x86)/microchip/xc32/v1.21/bin/../lib/gcc/pic32mx/4.5.2/../../../../pic32mx/lib/size\libpic32.a(vector5.o)
 .pdr           0x00000000       0x20 c:/program files (x86)/microchip/xc32/v1.21/bin/../lib/gcc/pic32mx/4.5.2/../../../../pic32mx/lib/size\libpic32.a(vector5.o)
 .text          0x00000000        0x0 c:/program files (x86)/microchip/xc32/v1.21/bin/../lib/gcc/pic32mx/4.5.2/../../../../pic32mx/lib/size\libpic32.a(vector6.o)
 .data          0x00000000        0x0 c:/program files (x86)/microchip/xc32/v1.21/bin/../lib/gcc/pic32mx/4.5.2/../../../../pic32mx/lib/size\libpic32.a(vector6.o)
 .bss           0x00000000        0x0 c:/program files (x86)/microchip/xc32/v1.21/bin/../lib/gcc/pic32mx/4.5.2/../../../../pic32mx/lib/size\libpic32.a(vector6.o)
 .reginfo       0x00000000       0x18 c:/program files (x86)/microchip/xc32/v1.21/bin/../lib/gcc/pic32mx/4.5.2/../../../../pic32mx/lib/size\libpic32.a(vector6.o)
 .pdr           0x00000000       0x20 c:/program files (x86)/microchip/xc32/v1.21/bin/../lib/gcc/pic32mx/4.5.2/../../../../pic32mx/lib/size\libpic32.a(vector6.o)
 .text          0x00000000        0x0 c:/program files (x86)/microchip/xc32/v1.21/bin/../lib/gcc/pic32mx/4.5.2/../../../../pic32mx/lib/size\libpic32.a(vector8.o)
 .data          0x00000000        0x0 c:/program files (x86)/microchip/xc32/v1.21/bin/../lib/gcc/pic32mx/4.5.2/../../../../pic32mx/lib/size\libpic32.a(vector8.o)
 .bss           0x00000000        0x0 c:/program files (x86)/microchip/xc32/v1.21/bin/../lib/gcc/pic32mx/4.5.2/../../../../pic32mx/lib/size\libpic32.a(vector8.o)
 .reginfo       0x00000000       0x18 c:/program files (x86)/microchip/xc32/v1.21/bin/../lib/gcc/pic32mx/4.5.2/../../../../pic32mx/lib/size\libpic32.a(vector8.o)
 .pdr           0x00000000       0x20 c:/program files (x86)/microchip/xc32/v1.21/bin/../lib/gcc/pic32mx/4.5.2/../../../../pic32mx/lib/size\libpic32.a(vector8.o)
 .text          0x00000000        0x0 c:/program files (x86)/microchip/xc32/v1.21/bin/../lib/gcc/pic32mx/4.5.2/../../../../pic32mx/lib/size\libpic32.a(vector9.o)
 .data          0x00000000        0x0 c:/program files (x86)/microchip/xc32/v1.21/bin/../lib/gcc/pic32mx/4.5.2/../../../../pic32mx/lib/size\libpic32.a(vector9.o)
 .bss           0x00000000        0x0 c:/program files (x86)/microchip/xc32/v1.21/bin/../lib/gcc/pic32mx/4.5.2/../../../../pic32mx/lib/size\libpic32.a(vector9.o)
 .reginfo       0x00000000       0x18 c:/program files (x86)/microchip/xc32/v1.21/bin/../lib/gcc/pic32mx/4.5.2/../../../../pic32mx/lib/size\libpic32.a(vector9.o)
 .pdr           0x00000000       0x20 c:/program files (x86)/microchip/xc32/v1.21/bin/../lib/gcc/pic32mx/4.5.2/../../../../pic32mx/lib/size\libpic32.a(vector9.o)
 .text          0x00000000        0x0 c:/program files (x86)/microchip/xc32/v1.21/bin/../lib/gcc/pic32mx/4.5.2/../../../../pic32mx/lib/size\libpic32.a(vector10.o)
 .data          0x00000000        0x0 c:/program files (x86)/microchip/xc32/v1.21/bin/../lib/gcc/pic32mx/4.5.2/../../../../pic32mx/lib/size\libpic32.a(vector10.o)
 .bss           0x00000000        0x0 c:/program files (x86)/microchip/xc32/v1.21/bin/../lib/gcc/pic32mx/4.5.2/../../../../pic32mx/lib/size\libpic32.a(vector10.o)
 .reginfo       0x00000000       0x18 c:/program files (x86)/microchip/xc32/v1.21/bin/../lib/gcc/pic32mx/4.5.2/../../../../pic32mx/lib/size\libpic32.a(vector10.o)
 .pdr           0x00000000       0x20 c:/program files (x86)/microchip/xc32/v1.21/bin/../lib/gcc/pic32mx/4.5.2/../../../../pic32mx/lib/size\libpic32.a(vector10.o)
 .text          0x00000000        0x0 c:/program files (x86)/microchip/xc32/v1.21/bin/../lib/gcc/pic32mx/4.5.2/../../../../pic32mx/lib/size\libpic32.a(vector11.o)
 .data          0x00000000        0x0 c:/program files (x86)/microchip/xc32/v1.21/bin/../lib/gcc/pic32mx/4.5.2/../../../../pic32mx/lib/size\libpic32.a(vector11.o)
 .bss           0x00000000        0x0 c:/program files (x86)/microchip/xc32/v1.21/bin/../lib/gcc/pic32mx/4.5.2/../../../../pic32mx/lib/size\libpic32.a(vector11.o)
 .reginfo       0x00000000       0x18 c:/program files (x86)/microchip/xc32/v1.21/bin/../lib/gcc/pic32mx/4.5.2/../../../../pic32mx/lib/size\libpic32.a(vector11.o)
 .pdr           0x00000000       0x20 c:/program files (x86)/microchip/xc32/v1.21/bin/../lib/gcc/pic32mx/4.5.2/../../../../pic32mx/lib/size\libpic32.a(vector11.o)
 .text          0x00000000        0x0 c:/program files (x86)/microchip/xc32/v1.21/bin/../lib/gcc/pic32mx/4.5.2/../../../../pic32mx/lib/size\libpic32.a(vector12.o)
 .data          0x00000000        0x0 c:/program files (x86)/microchip/xc32/v1.21/bin/../lib/gcc/pic32mx/4.5.2/../../../../pic32mx/lib/size\libpic32.a(vector12.o)
 .bss           0x00000000        0x0 c:/program files (x86)/microchip/xc32/v1.21/bin/../lib/gcc/pic32mx/4.5.2/../../../../pic32mx/lib/size\libpic32.a(vector12.o)
 .reginfo       0x00000000       0x18 c:/program files (x86)/microchip/xc32/v1.21/bin/../lib/gcc/pic32mx/4.5.2/../../../../pic32mx/lib/size\libpic32.a(vector12.o)
 .pdr           0x00000000       0x20 c:/program files (x86)/microchip/xc32/v1.21/bin/../lib/gcc/pic32mx/4.5.2/../../../../pic32mx/lib/size\libpic32.a(vector12.o)
 .text          0x00000000        0x0 c:/program files (x86)/microchip/xc32/v1.21/bin/../lib/gcc/pic32mx/4.5.2/../../../../pic32mx/lib/size\libpic32.a(vector13.o)
 .data          0x00000000        0x0 c:/program files (x86)/microchip/xc32/v1.21/bin/../lib/gcc/pic32mx/4.5.2/../../../../pic32mx/lib/size\libpic32.a(vector13.o)
 .bss           0x00000000        0x0 c:/program files (x86)/microchip/xc32/v1.21/bin/../lib/gcc/pic32mx/4.5.2/../../../../pic32mx/lib/size\libpic32.a(vector13.o)
 .reginfo       0x00000000       0x18 c:/program files (x86)/microchip/xc32/v1.21/bin/../lib/gcc/pic32mx/4.5.2/../../../../pic32mx/lib/size\libpic32.a(vector13.o)
 .pdr           0x00000000       0x20 c:/program files (x86)/microchip/xc32/v1.21/bin/../lib/gcc/pic32mx/4.5.2/../../../../pic32mx/lib/size\libpic32.a(vector13.o)
 .text          0x00000000        0x0 c:/program files (x86)/microchip/xc32/v1.21/bin/../lib/gcc/pic32mx/4.5.2/../../../../pic32mx/lib/size\libpic32.a(vector14.o)
 .data          0x00000000        0x0 c:/program files (x86)/microchip/xc32/v1.21/bin/../lib/gcc/pic32mx/4.5.2/../../../../pic32mx/lib/size\libpic32.a(vector14.o)
 .bss           0x00000000        0x0 c:/program files (x86)/microchip/xc32/v1.21/bin/../lib/gcc/pic32mx/4.5.2/../../../../pic32mx/lib/size\libpic32.a(vector14.o)
 .reginfo       0x00000000       0x18 c:/program files (x86)/microchip/xc32/v1.21/bin/../lib/gcc/pic32mx/4.5.2/../../../../pic32mx/lib/size\libpic32.a(vector14.o)
 .pdr           0x00000000       0x20 c:/program files (x86)/microchip/xc32/v1.21/bin/../lib/gcc/pic32mx/4.5.2/../../../../pic32mx/lib/size\libpic32.a(vector14.o)
 .text          0x00000000        0x0 c:/program files (x86)/microchip/xc32/v1.21/bin/../lib/gcc/pic32mx/4.5.2/../../../../pic32mx/lib/size\libpic32.a(vector16.o)
 .data          0x00000000        0x0 c:/program files (x86)/microchip/xc32/v1.21/bin/../lib/gcc/pic32mx/4.5.2/../../../../pic32mx/lib/size\libpic32.a(vector16.o)
 .bss           0x00000000        0x0 c:/program files (x86)/microchip/xc32/v1.21/bin/../lib/gcc/pic32mx/4.5.2/../../../../pic32mx/lib/size\libpic32.a(vector16.o)
 .reginfo       0x00000000       0x18 c:/program files (x86)/microchip/xc32/v1.21/bin/../lib/gcc/pic32mx/4.5.2/../../../../pic32mx/lib/size\libpic32.a(vector16.o)
 .pdr           0x00000000       0x20 c:/program files (x86)/microchip/xc32/v1.21/bin/../lib/gcc/pic32mx/4.5.2/../../../../pic32mx/lib/size\libpic32.a(vector16.o)
 .text          0x00000000        0x0 c:/program files (x86)/microchip/xc32/v1.21/bin/../lib/gcc/pic32mx/4.5.2/../../../../pic32mx/lib/size\libpic32.a(vector17.o)
 .data          0x00000000        0x0 c:/program files (x86)/microchip/xc32/v1.21/bin/../lib/gcc/pic32mx/4.5.2/../../../../pic32mx/lib/size\libpic32.a(vector17.o)
 .bss           0x00000000        0x0 c:/program files (x86)/microchip/xc32/v1.21/bin/../lib/gcc/pic32mx/4.5.2/../../../../pic32mx/lib/size\libpic32.a(vector17.o)
 .reginfo       0x00000000       0x18 c:/program files (x86)/microchip/xc32/v1.21/bin/../lib/gcc/pic32mx/4.5.2/../../../../pic32mx/lib/size\libpic32.a(vector17.o)
 .pdr           0x00000000       0x20 c:/program files (x86)/microchip/xc32/v1.21/bin/../lib/gcc/pic32mx/4.5.2/../../../../pic32mx/lib/size\libpic32.a(vector17.o)
 .text          0x00000000        0x0 c:/program files (x86)/microchip/xc32/v1.21/bin/../lib/gcc/pic32mx/4.5.2/../../../../pic32mx/lib/size\libpic32.a(vector18.o)
 .data          0x00000000        0x0 c:/program files (x86)/microchip/xc32/v1.21/bin/../lib/gcc/pic32mx/4.5.2/../../../../pic32mx/lib/size\libpic32.a(vector18.o)
 .bss           0x00000000        0x0 c:/program files (x86)/microchip/xc32/v1.21/bin/../lib/gcc/pic32mx/4.5.2/../../../../pic32mx/lib/size\libpic32.a(vector18.o)
 .reginfo       0x00000000       0x18 c:/program files (x86)/microchip/xc32/v1.21/bin/../lib/gcc/pic32mx/4.5.2/../../../../pic32mx/lib/size\libpic32.a(vector18.o)
 .pdr           0x00000000       0x20 c:/program files (x86)/microchip/xc32/v1.21/bin/../lib/gcc/pic32mx/4.5.2/../../../../pic32mx/lib/size\libpic32.a(vector18.o)
 .text          0x00000000        0x0 c:/program files (x86)/microchip/xc32/v1.21/bin/../lib/gcc/pic32mx/4.5.2/../../../../pic32mx/lib/size\libpic32.a(vector19.o)
 .data          0x00000000        0x0 c:/program files (x86)/microchip/xc32/v1.21/bin/../lib/gcc/pic32mx/4.5.2/../../../../pic32mx/lib/size\libpic32.a(vector19.o)
 .bss           0x00000000        0x0 c:/program files (x86)/microchip/xc32/v1.21/bin/../lib/gcc/pic32mx/4.5.2/../../../../pic32mx/lib/size\libpic32.a(vector19.o)
 .reginfo       0x00000000       0x18 c:/program files (x86)/microchip/xc32/v1.21/bin/../lib/gcc/pic32mx/4.5.2/../../../../pic32mx/lib/size\libpic32.a(vector19.o)
 .pdr           0x00000000       0x20 c:/program files (x86)/microchip/xc32/v1.21/bin/../lib/gcc/pic32mx/4.5.2/../../../../pic32mx/lib/size\libpic32.a(vector19.o)
 .text          0x00000000        0x0 c:/program files (x86)/microchip/xc32/v1.21/bin/../lib/gcc/pic32mx/4.5.2/../../../../pic32mx/lib/size\libpic32.a(vector20.o)
 .data          0x00000000        0x0 c:/program files (x86)/microchip/xc32/v1.21/bin/../lib/gcc/pic32mx/4.5.2/../../../../pic32mx/lib/size\libpic32.a(vector20.o)
 .bss           0x00000000        0x0 c:/program files (x86)/microchip/xc32/v1.21/bin/../lib/gcc/pic32mx/4.5.2/../../../../pic32mx/lib/size\libpic32.a(vector20.o)
 .reginfo       0x00000000       0x18 c:/program files (x86)/microchip/xc32/v1.21/bin/../lib/gcc/pic32mx/4.5.2/../../../../pic32mx/lib/size\libpic32.a(vector20.o)
 .pdr           0x00000000       0x20 c:/program files (x86)/microchip/xc32/v1.21/bin/../lib/gcc/pic32mx/4.5.2/../../../../pic32mx/lib/size\libpic32.a(vector20.o)
 .text          0x00000000        0x0 c:/program files (x86)/microchip/xc32/v1.21/bin/../lib/gcc/pic32mx/4.5.2/../../../../pic32mx/lib/size\libpic32.a(vector21.o)
 .data          0x00000000        0x0 c:/program files (x86)/microchip/xc32/v1.21/bin/../lib/gcc/pic32mx/4.5.2/../../../../pic32mx/lib/size\libpic32.a(vector21.o)
 .bss           0x00000000        0x0 c:/program files (x86)/microchip/xc32/v1.21/bin/../lib/gcc/pic32mx/4.5.2/../../../../pic32mx/lib/size\libpic32.a(vector21.o)
 .reginfo       0x00000000       0x18 c:/program files (x86)/microchip/xc32/v1.21/bin/../lib/gcc/pic32mx/4.5.2/../../../../pic32mx/lib/size\libpic32.a(vector21.o)
 .pdr           0x00000000       0x20 c:/program files (x86)/microchip/xc32/v1.21/bin/../lib/gcc/pic32mx/4.5.2/../../../../pic32mx/lib/size\libpic32.a(vector21.o)
 .text          0x00000000        0x0 c:/program files (x86)/microchip/xc32/v1.21/bin/../lib/gcc/pic32mx/4.5.2/../../../../pic32mx/lib/size\libpic32.a(vector22.o)
 .data          0x00000000        0x0 c:/program files (x86)/microchip/xc32/v1.21/bin/../lib/gcc/pic32mx/4.5.2/../../../../pic32mx/lib/size\libpic32.a(vector22.o)
 .bss           0x00000000        0x0 c:/program files (x86)/microchip/xc32/v1.21/bin/../lib/gcc/pic32mx/4.5.2/../../../../pic32mx/lib/size\libpic32.a(vector22.o)
 .reginfo       0x00000000       0x18 c:/program files (x86)/microchip/xc32/v1.21/bin/../lib/gcc/pic32mx/4.5.2/../../../../pic32mx/lib/size\libpic32.a(vector22.o)
 .pdr           0x00000000       0x20 c:/program files (x86)/microchip/xc32/v1.21/bin/../lib/gcc/pic32mx/4.5.2/../../../../pic32mx/lib/size\libpic32.a(vector22.o)
 .text          0x00000000        0x0 c:/program files (x86)/microchip/xc32/v1.21/bin/../lib/gcc/pic32mx/4.5.2/../../../../pic32mx/lib/size\libpic32.a(vector23.o)
 .data          0x00000000        0x0 c:/program files (x86)/microchip/xc32/v1.21/bin/../lib/gcc/pic32mx/4.5.2/../../../../pic32mx/lib/size\libpic32.a(vector23.o)
 .bss           0x00000000        0x0 c:/program files (x86)/microchip/xc32/v1.21/bin/../lib/gcc/pic32mx/4.5.2/../../../../pic32mx/lib/size\libpic32.a(vector23.o)
 .reginfo       0x00000000       0x18 c:/program files (x86)/microchip/xc32/v1.21/bin/../lib/gcc/pic32mx/4.5.2/../../../../pic32mx/lib/size\libpic32.a(vector23.o)
 .pdr           0x00000000       0x20 c:/program files (x86)/microchip/xc32/v1.21/bin/../lib/gcc/pic32mx/4.5.2/../../../../pic32mx/lib/size\libpic32.a(vector23.o)
 .text          0x00000000        0x0 c:/program files (x86)/microchip/xc32/v1.21/bin/../lib/gcc/pic32mx/4.5.2/../../../../pic32mx/lib/size\libpic32.a(vector24.o)
 .data          0x00000000        0x0 c:/program files (x86)/microchip/xc32/v1.21/bin/../lib/gcc/pic32mx/4.5.2/../../../../pic32mx/lib/size\libpic32.a(vector24.o)
 .bss           0x00000000        0x0 c:/program files (x86)/microchip/xc32/v1.21/bin/../lib/gcc/pic32mx/4.5.2/../../../../pic32mx/lib/size\libpic32.a(vector24.o)
 .reginfo       0x00000000       0x18 c:/program files (x86)/microchip/xc32/v1.21/bin/../lib/gcc/pic32mx/4.5.2/../../../../pic32mx/lib/size\libpic32.a(vector24.o)
 .pdr           0x00000000       0x20 c:/program files (x86)/microchip/xc32/v1.21/bin/../lib/gcc/pic32mx/4.5.2/../../../../pic32mx/lib/size\libpic32.a(vector24.o)
 .text          0x00000000        0x0 c:/program files (x86)/microchip/xc32/v1.21/bin/../lib/gcc/pic32mx/4.5.2/../../../../pic32mx/lib/size\libpic32.a(vector25.o)
 .data          0x00000000        0x0 c:/program files (x86)/microchip/xc32/v1.21/bin/../lib/gcc/pic32mx/4.5.2/../../../../pic32mx/lib/size\libpic32.a(vector25.o)
 .bss           0x00000000        0x0 c:/program files (x86)/microchip/xc32/v1.21/bin/../lib/gcc/pic32mx/4.5.2/../../../../pic32mx/lib/size\libpic32.a(vector25.o)
 .reginfo       0x00000000       0x18 c:/program files (x86)/microchip/xc32/v1.21/bin/../lib/gcc/pic32mx/4.5.2/../../../../pic32mx/lib/size\libpic32.a(vector25.o)
 .pdr           0x00000000       0x20 c:/program files (x86)/microchip/xc32/v1.21/bin/../lib/gcc/pic32mx/4.5.2/../../../../pic32mx/lib/size\libpic32.a(vector25.o)
 .text          0x00000000        0x0 c:/program files (x86)/microchip/xc32/v1.21/bin/../lib/gcc/pic32mx/4.5.2/../../../../pic32mx/lib/size\libpic32.a(vector27.o)
 .data          0x00000000        0x0 c:/program files (x86)/microchip/xc32/v1.21/bin/../lib/gcc/pic32mx/4.5.2/../../../../pic32mx/lib/size\libpic32.a(vector27.o)
 .bss           0x00000000        0x0 c:/program files (x86)/microchip/xc32/v1.21/bin/../lib/gcc/pic32mx/4.5.2/../../../../pic32mx/lib/size\libpic32.a(vector27.o)
 .reginfo       0x00000000       0x18 c:/program files (x86)/microchip/xc32/v1.21/bin/../lib/gcc/pic32mx/4.5.2/../../../../pic32mx/lib/size\libpic32.a(vector27.o)
 .pdr           0x00000000       0x20 c:/program files (x86)/microchip/xc32/v1.21/bin/../lib/gcc/pic32mx/4.5.2/../../../../pic32mx/lib/size\libpic32.a(vector27.o)
 .text          0x00000000        0x0 c:/program files (x86)/microchip/xc32/v1.21/bin/../lib/gcc/pic32mx/4.5.2/../../../../pic32mx/lib/size\libpic32.a(vector28.o)
 .data          0x00000000        0x0 c:/program files (x86)/microchip/xc32/v1.21/bin/../lib/gcc/pic32mx/4.5.2/../../../../pic32mx/lib/size\libpic32.a(vector28.o)
 .bss           0x00000000        0x0 c:/program files (x86)/microchip/xc32/v1.21/bin/../lib/gcc/pic32mx/4.5.2/../../../../pic32mx/lib/size\libpic32.a(vector28.o)
 .reginfo       0x00000000       0x18 c:/program files (x86)/microchip/xc32/v1.21/bin/../lib/gcc/pic32mx/4.5.2/../../../../pic32mx/lib/size\libpic32.a(vector28.o)
 .pdr           0x00000000       0x20 c:/program files (x86)/microchip/xc32/v1.21/bin/../lib/gcc/pic32mx/4.5.2/../../../../pic32mx/lib/size\libpic32.a(vector28.o)
 .text          0x00000000        0x0 c:/program files (x86)/microchip/xc32/v1.21/bin/../lib/gcc/pic32mx/4.5.2/../../../../pic32mx/lib/size\libpic32.a(vector29.o)
 .data          0x00000000        0x0 c:/program files (x86)/microchip/xc32/v1.21/bin/../lib/gcc/pic32mx/4.5.2/../../../../pic32mx/lib/size\libpic32.a(vector29.o)
 .bss           0x00000000        0x0 c:/program files (x86)/microchip/xc32/v1.21/bin/../lib/gcc/pic32mx/4.5.2/../../../../pic32mx/lib/size\libpic32.a(vector29.o)
 .reginfo       0x00000000       0x18 c:/program files (x86)/microchip/xc32/v1.21/bin/../lib/gcc/pic32mx/4.5.2/../../../../pic32mx/lib/size\libpic32.a(vector29.o)
 .pdr           0x00000000       0x20 c:/program files (x86)/microchip/xc32/v1.21/bin/../lib/gcc/pic32mx/4.5.2/../../../../pic32mx/lib/size\libpic32.a(vector29.o)
 .text          0x00000000        0x0 c:/program files (x86)/microchip/xc32/v1.21/bin/../lib/gcc/pic32mx/4.5.2/../../../../pic32mx/lib/size\libpic32.a(vector30.o)
 .data          0x00000000        0x0 c:/program files (x86)/microchip/xc32/v1.21/bin/../lib/gcc/pic32mx/4.5.2/../../../../pic32mx/lib/size\libpic32.a(vector30.o)
 .bss           0x00000000        0x0 c:/program files (x86)/microchip/xc32/v1.21/bin/../lib/gcc/pic32mx/4.5.2/../../../../pic32mx/lib/size\libpic32.a(vector30.o)
 .reginfo       0x00000000       0x18 c:/program files (x86)/microchip/xc32/v1.21/bin/../lib/gcc/pic32mx/4.5.2/../../../../pic32mx/lib/size\libpic32.a(vector30.o)
 .pdr           0x00000000       0x20 c:/program files (x86)/microchip/xc32/v1.21/bin/../lib/gcc/pic32mx/4.5.2/../../../../pic32mx/lib/size\libpic32.a(vector30.o)
 .text          0x00000000        0x0 c:/program files (x86)/microchip/xc32/v1.21/bin/../lib/gcc/pic32mx/4.5.2/../../../../pic32mx/lib/size\libpic32.a(vector31.o)
 .data          0x00000000        0x0 c:/program files (x86)/microchip/xc32/v1.21/bin/../lib/gcc/pic32mx/4.5.2/../../../../pic32mx/lib/size\libpic32.a(vector31.o)
 .bss           0x00000000        0x0 c:/program files (x86)/microchip/xc32/v1.21/bin/../lib/gcc/pic32mx/4.5.2/../../../../pic32mx/lib/size\libpic32.a(vector31.o)
 .reginfo       0x00000000       0x18 c:/program files (x86)/microchip/xc32/v1.21/bin/../lib/gcc/pic32mx/4.5.2/../../../../pic32mx/lib/size\libpic32.a(vector31.o)
 .pdr           0x00000000       0x20 c:/program files (x86)/microchip/xc32/v1.21/bin/../lib/gcc/pic32mx/4.5.2/../../../../pic32mx/lib/size\libpic32.a(vector31.o)
 .text          0x00000000        0x0 c:/program files (x86)/microchip/xc32/v1.21/bin/../lib/gcc/pic32mx/4.5.2/../../../../pic32mx/lib/size\libpic32.a(vector32.o)
 .data          0x00000000        0x0 c:/program files (x86)/microchip/xc32/v1.21/bin/../lib/gcc/pic32mx/4.5.2/../../../../pic32mx/lib/size\libpic32.a(vector32.o)
 .bss           0x00000000        0x0 c:/program files (x86)/microchip/xc32/v1.21/bin/../lib/gcc/pic32mx/4.5.2/../../../../pic32mx/lib/size\libpic32.a(vector32.o)
 .reginfo       0x00000000       0x18 c:/program files (x86)/microchip/xc32/v1.21/bin/../lib/gcc/pic32mx/4.5.2/../../../../pic32mx/lib/size\libpic32.a(vector32.o)
 .pdr           0x00000000       0x20 c:/program files (x86)/microchip/xc32/v1.21/bin/../lib/gcc/pic32mx/4.5.2/../../../../pic32mx/lib/size\libpic32.a(vector32.o)
 .text          0x00000000        0x0 c:/program files (x86)/microchip/xc32/v1.21/bin/../lib/gcc/pic32mx/4.5.2/../../../../pic32mx/lib/size\libpic32.a(vector33.o)
 .data          0x00000000        0x0 c:/program files (x86)/microchip/xc32/v1.21/bin/../lib/gcc/pic32mx/4.5.2/../../../../pic32mx/lib/size\libpic32.a(vector33.o)
 .bss           0x00000000        0x0 c:/program files (x86)/microchip/xc32/v1.21/bin/../lib/gcc/pic32mx/4.5.2/../../../../pic32mx/lib/size\libpic32.a(vector33.o)
 .reginfo       0x00000000       0x18 c:/program files (x86)/microchip/xc32/v1.21/bin/../lib/gcc/pic32mx/4.5.2/../../../../pic32mx/lib/size\libpic32.a(vector33.o)
 .pdr           0x00000000       0x20 c:/program files (x86)/microchip/xc32/v1.21/bin/../lib/gcc/pic32mx/4.5.2/../../../../pic32mx/lib/size\libpic32.a(vector33.o)
 .text          0x00000000        0x0 c:/program files (x86)/microchip/xc32/v1.21/bin/../lib/gcc/pic32mx/4.5.2/../../../../pic32mx/lib/size\libpic32.a(vector34.o)
 .data          0x00000000        0x0 c:/program files (x86)/microchip/xc32/v1.21/bin/../lib/gcc/pic32mx/4.5.2/../../../../pic32mx/lib/size\libpic32.a(vector34.o)
 .bss           0x00000000        0x0 c:/program files (x86)/microchip/xc32/v1.21/bin/../lib/gcc/pic32mx/4.5.2/../../../../pic32mx/lib/size\libpic32.a(vector34.o)
 .reginfo       0x00000000       0x18 c:/program files (x86)/microchip/xc32/v1.21/bin/../lib/gcc/pic32mx/4.5.2/../../../../pic32mx/lib/size\libpic32.a(vector34.o)
 .pdr           0x00000000       0x20 c:/program files (x86)/microchip/xc32/v1.21/bin/../lib/gcc/pic32mx/4.5.2/../../../../pic32mx/lib/size\libpic32.a(vector34.o)
 .text          0x00000000        0x0 c:/program files (x86)/microchip/xc32/v1.21/bin/../lib/gcc/pic32mx/4.5.2/../../../../pic32mx/lib/size\libpic32.a(vector35.o)
 .data          0x00000000        0x0 c:/program files (x86)/microchip/xc32/v1.21/bin/../lib/gcc/pic32mx/4.5.2/../../../../pic32mx/lib/size\libpic32.a(vector35.o)
 .bss           0x00000000        0x0 c:/program files (x86)/microchip/xc32/v1.21/bin/../lib/gcc/pic32mx/4.5.2/../../../../pic32mx/lib/size\libpic32.a(vector35.o)
 .reginfo       0x00000000       0x18 c:/program files (x86)/microchip/xc32/v1.21/bin/../lib/gcc/pic32mx/4.5.2/../../../../pic32mx/lib/size\libpic32.a(vector35.o)
 .pdr           0x00000000       0x20 c:/program files (x86)/microchip/xc32/v1.21/bin/../lib/gcc/pic32mx/4.5.2/../../../../pic32mx/lib/size\libpic32.a(vector35.o)
 .text          0x00000000        0x0 c:/program files (x86)/microchip/xc32/v1.21/bin/../lib/gcc/pic32mx/4.5.2/../../../../pic32mx/lib/size\libpic32.a(vector36.o)
 .data          0x00000000        0x0 c:/program files (x86)/microchip/xc32/v1.21/bin/../lib/gcc/pic32mx/4.5.2/../../../../pic32mx/lib/size\libpic32.a(vector36.o)
 .bss           0x00000000        0x0 c:/program files (x86)/microchip/xc32/v1.21/bin/../lib/gcc/pic32mx/4.5.2/../../../../pic32mx/lib/size\libpic32.a(vector36.o)
 .reginfo       0x00000000       0x18 c:/program files (x86)/microchip/xc32/v1.21/bin/../lib/gcc/pic32mx/4.5.2/../../../../pic32mx/lib/size\libpic32.a(vector36.o)
 .pdr           0x00000000       0x20 c:/program files (x86)/microchip/xc32/v1.21/bin/../lib/gcc/pic32mx/4.5.2/../../../../pic32mx/lib/size\libpic32.a(vector36.o)
 .text          0x00000000        0x0 c:/program files (x86)/microchip/xc32/v1.21/bin/../lib/gcc/pic32mx/4.5.2/../../../../pic32mx/lib/size\libpic32.a(vector37.o)
 .data          0x00000000        0x0 c:/program files (x86)/microchip/xc32/v1.21/bin/../lib/gcc/pic32mx/4.5.2/../../../../pic32mx/lib/size\libpic32.a(vector37.o)
 .bss           0x00000000        0x0 c:/program files (x86)/microchip/xc32/v1.21/bin/../lib/gcc/pic32mx/4.5.2/../../../../pic32mx/lib/size\libpic32.a(vector37.o)
 .reginfo       0x00000000       0x18 c:/program files (x86)/microchip/xc32/v1.21/bin/../lib/gcc/pic32mx/4.5.2/../../../../pic32mx/lib/size\libpic32.a(vector37.o)
 .pdr           0x00000000       0x20 c:/program files (x86)/microchip/xc32/v1.21/bin/../lib/gcc/pic32mx/4.5.2/../../../../pic32mx/lib/size\libpic32.a(vector37.o)
 .text          0x00000000        0x0 c:/program files (x86)/microchip/xc32/v1.21/bin/../lib/gcc/pic32mx/4.5.2/../../../../pic32mx/lib/size\libpic32.a(vector38.o)
 .data          0x00000000        0x0 c:/program files (x86)/microchip/xc32/v1.21/bin/../lib/gcc/pic32mx/4.5.2/../../../../pic32mx/lib/size\libpic32.a(vector38.o)
 .bss           0x00000000        0x0 c:/program files (x86)/microchip/xc32/v1.21/bin/../lib/gcc/pic32mx/4.5.2/../../../../pic32mx/lib/size\libpic32.a(vector38.o)
 .reginfo       0x00000000       0x18 c:/program files (x86)/microchip/xc32/v1.21/bin/../lib/gcc/pic32mx/4.5.2/../../../../pic32mx/lib/size\libpic32.a(vector38.o)
 .pdr           0x00000000       0x20 c:/program files (x86)/microchip/xc32/v1.21/bin/../lib/gcc/pic32mx/4.5.2/../../../../pic32mx/lib/size\libpic32.a(vector38.o)
 .text          0x00000000        0x0 c:/program files (x86)/microchip/xc32/v1.21/bin/../lib/gcc/pic32mx/4.5.2/../../../../pic32mx/lib/size\libpic32.a(vector39.o)
 .data          0x00000000        0x0 c:/program files (x86)/microchip/xc32/v1.21/bin/../lib/gcc/pic32mx/4.5.2/../../../../pic32mx/lib/size\libpic32.a(vector39.o)
 .bss           0x00000000        0x0 c:/program files (x86)/microchip/xc32/v1.21/bin/../lib/gcc/pic32mx/4.5.2/../../../../pic32mx/lib/size\libpic32.a(vector39.o)
 .reginfo       0x00000000       0x18 c:/program files (x86)/microchip/xc32/v1.21/bin/../lib/gcc/pic32mx/4.5.2/../../../../pic32mx/lib/size\libpic32.a(vector39.o)
 .pdr           0x00000000       0x20 c:/program files (x86)/microchip/xc32/v1.21/bin/../lib/gcc/pic32mx/4.5.2/../../../../pic32mx/lib/size\libpic32.a(vector39.o)
 .text          0x00000000        0x0 c:/program files (x86)/microchip/xc32/v1.21/bin/../lib/gcc/pic32mx/4.5.2/../../../../pic32mx/lib/size\libpic32.a(vector40.o)
 .data          0x00000000        0x0 c:/program files (x86)/microchip/xc32/v1.21/bin/../lib/gcc/pic32mx/4.5.2/../../../../pic32mx/lib/size\libpic32.a(vector40.o)
 .bss           0x00000000        0x0 c:/program files (x86)/microchip/xc32/v1.21/bin/../lib/gcc/pic32mx/4.5.2/../../../../pic32mx/lib/size\libpic32.a(vector40.o)
 .reginfo       0x00000000       0x18 c:/program files (x86)/microchip/xc32/v1.21/bin/../lib/gcc/pic32mx/4.5.2/../../../../pic32mx/lib/size\libpic32.a(vector40.o)
 .pdr           0x00000000       0x20 c:/program files (x86)/microchip/xc32/v1.21/bin/../lib/gcc/pic32mx/4.5.2/../../../../pic32mx/lib/size\libpic32.a(vector40.o)
 .text          0x00000000        0x0 c:/program files (x86)/microchip/xc32/v1.21/bin/../lib/gcc/pic32mx/4.5.2/../../../../pic32mx/lib/size\libpic32.a(vector41.o)
 .data          0x00000000        0x0 c:/program files (x86)/microchip/xc32/v1.21/bin/../lib/gcc/pic32mx/4.5.2/../../../../pic32mx/lib/size\libpic32.a(vector41.o)
 .bss           0x00000000        0x0 c:/program files (x86)/microchip/xc32/v1.21/bin/../lib/gcc/pic32mx/4.5.2/../../../../pic32mx/lib/size\libpic32.a(vector41.o)
 .reginfo       0x00000000       0x18 c:/program files (x86)/microchip/xc32/v1.21/bin/../lib/gcc/pic32mx/4.5.2/../../../../pic32mx/lib/size\libpic32.a(vector41.o)
 .pdr           0x00000000       0x20 c:/program files (x86)/microchip/xc32/v1.21/bin/../lib/gcc/pic32mx/4.5.2/../../../../pic32mx/lib/size\libpic32.a(vector41.o)
 .text          0x00000000        0x0 c:/program files (x86)/microchip/xc32/v1.21/bin/../lib/gcc/pic32mx/4.5.2/../../../../pic32mx/lib/size\libpic32.a(vector42.o)
 .data          0x00000000        0x0 c:/program files (x86)/microchip/xc32/v1.21/bin/../lib/gcc/pic32mx/4.5.2/../../../../pic32mx/lib/size\libpic32.a(vector42.o)
 .bss           0x00000000        0x0 c:/program files (x86)/microchip/xc32/v1.21/bin/../lib/gcc/pic32mx/4.5.2/../../../../pic32mx/lib/size\libpic32.a(vector42.o)
 .reginfo       0x00000000       0x18 c:/program files (x86)/microchip/xc32/v1.21/bin/../lib/gcc/pic32mx/4.5.2/../../../../pic32mx/lib/size\libpic32.a(vector42.o)
 .pdr           0x00000000       0x20 c:/program files (x86)/microchip/xc32/v1.21/bin/../lib/gcc/pic32mx/4.5.2/../../../../pic32mx/lib/size\libpic32.a(vector42.o)
 .text          0x00000000        0x0 c:/program files (x86)/microchip/xc32/v1.21/bin/../lib/gcc/pic32mx/4.5.2/../../../../pic32mx/lib/size\libpic32.a(vector43.o)
 .data          0x00000000        0x0 c:/program files (x86)/microchip/xc32/v1.21/bin/../lib/gcc/pic32mx/4.5.2/../../../../pic32mx/lib/size\libpic32.a(vector43.o)
 .bss           0x00000000        0x0 c:/program files (x86)/microchip/xc32/v1.21/bin/../lib/gcc/pic32mx/4.5.2/../../../../pic32mx/lib/size\libpic32.a(vector43.o)
 .reginfo       0x00000000       0x18 c:/program files (x86)/microchip/xc32/v1.21/bin/../lib/gcc/pic32mx/4.5.2/../../../../pic32mx/lib/size\libpic32.a(vector43.o)
 .pdr           0x00000000       0x20 c:/program files (x86)/microchip/xc32/v1.21/bin/../lib/gcc/pic32mx/4.5.2/../../../../pic32mx/lib/size\libpic32.a(vector43.o)
 .text          0x00000000        0x0 c:/program files (x86)/microchip/xc32/v1.21/bin/../lib/gcc/pic32mx/4.5.2/../../../../pic32mx/lib/size\libpic32.a(vector44.o)
 .data          0x00000000        0x0 c:/program files (x86)/microchip/xc32/v1.21/bin/../lib/gcc/pic32mx/4.5.2/../../../../pic32mx/lib/size\libpic32.a(vector44.o)
 .bss           0x00000000        0x0 c:/program files (x86)/microchip/xc32/v1.21/bin/../lib/gcc/pic32mx/4.5.2/../../../../pic32mx/lib/size\libpic32.a(vector44.o)
 .reginfo       0x00000000       0x18 c:/program files (x86)/microchip/xc32/v1.21/bin/../lib/gcc/pic32mx/4.5.2/../../../../pic32mx/lib/size\libpic32.a(vector44.o)
 .pdr           0x00000000       0x20 c:/program files (x86)/microchip/xc32/v1.21/bin/../lib/gcc/pic32mx/4.5.2/../../../../pic32mx/lib/size\libpic32.a(vector44.o)
 .text          0x00000000        0x0 c:/program files (x86)/microchip/xc32/v1.21/bin/../lib/gcc/pic32mx/4.5.2/../../../../pic32mx/lib/size\libpic32.a(vector45.o)
 .data          0x00000000        0x0 c:/program files (x86)/microchip/xc32/v1.21/bin/../lib/gcc/pic32mx/4.5.2/../../../../pic32mx/lib/size\libpic32.a(vector45.o)
 .bss           0x00000000        0x0 c:/program files (x86)/microchip/xc32/v1.21/bin/../lib/gcc/pic32mx/4.5.2/../../../../pic32mx/lib/size\libpic32.a(vector45.o)
 .reginfo       0x00000000       0x18 c:/program files (x86)/microchip/xc32/v1.21/bin/../lib/gcc/pic32mx/4.5.2/../../../../pic32mx/lib/size\libpic32.a(vector45.o)
 .pdr           0x00000000       0x20 c:/program files (x86)/microchip/xc32/v1.21/bin/../lib/gcc/pic32mx/4.5.2/../../../../pic32mx/lib/size\libpic32.a(vector45.o)
 .text          0x00000000        0x0 c:/program files (x86)/microchip/xc32/v1.21/bin/../lib/gcc/pic32mx/4.5.2/../../../../pic32mx/lib/size\libpic32.a(vector46.o)
 .data          0x00000000        0x0 c:/program files (x86)/microchip/xc32/v1.21/bin/../lib/gcc/pic32mx/4.5.2/../../../../pic32mx/lib/size\libpic32.a(vector46.o)
 .bss           0x00000000        0x0 c:/program files (x86)/microchip/xc32/v1.21/bin/../lib/gcc/pic32mx/4.5.2/../../../../pic32mx/lib/size\libpic32.a(vector46.o)
 .reginfo       0x00000000       0x18 c:/program files (x86)/microchip/xc32/v1.21/bin/../lib/gcc/pic32mx/4.5.2/../../../../pic32mx/lib/size\libpic32.a(vector46.o)
 .pdr           0x00000000       0x20 c:/program files (x86)/microchip/xc32/v1.21/bin/../lib/gcc/pic32mx/4.5.2/../../../../pic32mx/lib/size\libpic32.a(vector46.o)
 .text          0x00000000        0x0 c:/program files (x86)/microchip/xc32/v1.21/bin/../lib/gcc/pic32mx/4.5.2/../../../../pic32mx/lib/size\libpic32.a(vector47.o)
 .data          0x00000000        0x0 c:/program files (x86)/microchip/xc32/v1.21/bin/../lib/gcc/pic32mx/4.5.2/../../../../pic32mx/lib/size\libpic32.a(vector47.o)
 .bss           0x00000000        0x0 c:/program files (x86)/microchip/xc32/v1.21/bin/../lib/gcc/pic32mx/4.5.2/../../../../pic32mx/lib/size\libpic32.a(vector47.o)
 .reginfo       0x00000000       0x18 c:/program files (x86)/microchip/xc32/v1.21/bin/../lib/gcc/pic32mx/4.5.2/../../../../pic32mx/lib/size\libpic32.a(vector47.o)
 .pdr           0x00000000       0x20 c:/program files (x86)/microchip/xc32/v1.21/bin/../lib/gcc/pic32mx/4.5.2/../../../../pic32mx/lib/size\libpic32.a(vector47.o)
 .text          0x00000000        0x0 c:/program files (x86)/microchip/xc32/v1.21/bin/../lib/gcc/pic32mx/4.5.2/../../../../pic32mx/lib/size\libpic32.a(vector48.o)
 .data          0x00000000        0x0 c:/program files (x86)/microchip/xc32/v1.21/bin/../lib/gcc/pic32mx/4.5.2/../../../../pic32mx/lib/size\libpic32.a(vector48.o)
 .bss           0x00000000        0x0 c:/program files (x86)/microchip/xc32/v1.21/bin/../lib/gcc/pic32mx/4.5.2/../../../../pic32mx/lib/size\libpic32.a(vector48.o)
 .reginfo       0x00000000       0x18 c:/program files (x86)/microchip/xc32/v1.21/bin/../lib/gcc/pic32mx/4.5.2/../../../../pic32mx/lib/size\libpic32.a(vector48.o)
 .pdr           0x00000000       0x20 c:/program files (x86)/microchip/xc32/v1.21/bin/../lib/gcc/pic32mx/4.5.2/../../../../pic32mx/lib/size\libpic32.a(vector48.o)
 .text          0x00000000        0x0 c:/program files (x86)/microchip/xc32/v1.21/bin/../lib/gcc/pic32mx/4.5.2/../../../../pic32mx/lib/size\libpic32.a(vector49.o)
 .data          0x00000000        0x0 c:/program files (x86)/microchip/xc32/v1.21/bin/../lib/gcc/pic32mx/4.5.2/../../../../pic32mx/lib/size\libpic32.a(vector49.o)
 .bss           0x00000000        0x0 c:/program files (x86)/microchip/xc32/v1.21/bin/../lib/gcc/pic32mx/4.5.2/../../../../pic32mx/lib/size\libpic32.a(vector49.o)
 .reginfo       0x00000000       0x18 c:/program files (x86)/microchip/xc32/v1.21/bin/../lib/gcc/pic32mx/4.5.2/../../../../pic32mx/lib/size\libpic32.a(vector49.o)
 .pdr           0x00000000       0x20 c:/program files (x86)/microchip/xc32/v1.21/bin/../lib/gcc/pic32mx/4.5.2/../../../../pic32mx/lib/size\libpic32.a(vector49.o)
 .text          0x00000000        0x0 c:/program files (x86)/microchip/xc32/v1.21/bin/../lib/gcc/pic32mx/4.5.2/../../../../pic32mx/lib/size\libpic32.a(vector50.o)
 .data          0x00000000        0x0 c:/program files (x86)/microchip/xc32/v1.21/bin/../lib/gcc/pic32mx/4.5.2/../../../../pic32mx/lib/size\libpic32.a(vector50.o)
 .bss           0x00000000        0x0 c:/program files (x86)/microchip/xc32/v1.21/bin/../lib/gcc/pic32mx/4.5.2/../../../../pic32mx/lib/size\libpic32.a(vector50.o)
 .reginfo       0x00000000       0x18 c:/program files (x86)/microchip/xc32/v1.21/bin/../lib/gcc/pic32mx/4.5.2/../../../../pic32mx/lib/size\libpic32.a(vector50.o)
 .pdr           0x00000000       0x20 c:/program files (x86)/microchip/xc32/v1.21/bin/../lib/gcc/pic32mx/4.5.2/../../../../pic32mx/lib/size\libpic32.a(vector50.o)
 .text          0x00000000        0x0 c:/program files (x86)/microchip/xc32/v1.21/bin/../lib/gcc/pic32mx/4.5.2/../../../../pic32mx/lib/size\libpic32.a(vector51.o)
 .data          0x00000000        0x0 c:/program files (x86)/microchip/xc32/v1.21/bin/../lib/gcc/pic32mx/4.5.2/../../../../pic32mx/lib/size\libpic32.a(vector51.o)
 .bss           0x00000000        0x0 c:/program files (x86)/microchip/xc32/v1.21/bin/../lib/gcc/pic32mx/4.5.2/../../../../pic32mx/lib/size\libpic32.a(vector51.o)
 .reginfo       0x00000000       0x18 c:/program files (x86)/microchip/xc32/v1.21/bin/../lib/gcc/pic32mx/4.5.2/../../../../pic32mx/lib/size\libpic32.a(vector51.o)
 .pdr           0x00000000       0x20 c:/program files (x86)/microchip/xc32/v1.21/bin/../lib/gcc/pic32mx/4.5.2/../../../../pic32mx/lib/size\libpic32.a(vector51.o)
 .text          0x00000000        0x0 c:/program files (x86)/microchip/xc32/v1.21/bin/../lib/gcc/pic32mx/4.5.2/../../../../pic32mx/lib/size\libpic32.a(vector52.o)
 .data          0x00000000        0x0 c:/program files (x86)/microchip/xc32/v1.21/bin/../lib/gcc/pic32mx/4.5.2/../../../../pic32mx/lib/size\libpic32.a(vector52.o)
 .bss           0x00000000        0x0 c:/program files (x86)/microchip/xc32/v1.21/bin/../lib/gcc/pic32mx/4.5.2/../../../../pic32mx/lib/size\libpic32.a(vector52.o)
 .reginfo       0x00000000       0x18 c:/program files (x86)/microchip/xc32/v1.21/bin/../lib/gcc/pic32mx/4.5.2/../../../../pic32mx/lib/size\libpic32.a(vector52.o)
 .pdr           0x00000000       0x20 c:/program files (x86)/microchip/xc32/v1.21/bin/../lib/gcc/pic32mx/4.5.2/../../../../pic32mx/lib/size\libpic32.a(vector52.o)
 .text          0x00000000        0x0 c:/program files (x86)/microchip/xc32/v1.21/bin/../lib/gcc/pic32mx/4.5.2/../../../../pic32mx/lib/size\libpic32.a(vector53.o)
 .data          0x00000000        0x0 c:/program files (x86)/microchip/xc32/v1.21/bin/../lib/gcc/pic32mx/4.5.2/../../../../pic32mx/lib/size\libpic32.a(vector53.o)
 .bss           0x00000000        0x0 c:/program files (x86)/microchip/xc32/v1.21/bin/../lib/gcc/pic32mx/4.5.2/../../../../pic32mx/lib/size\libpic32.a(vector53.o)
 .reginfo       0x00000000       0x18 c:/program files (x86)/microchip/xc32/v1.21/bin/../lib/gcc/pic32mx/4.5.2/../../../../pic32mx/lib/size\libpic32.a(vector53.o)
 .pdr           0x00000000       0x20 c:/program files (x86)/microchip/xc32/v1.21/bin/../lib/gcc/pic32mx/4.5.2/../../../../pic32mx/lib/size\libpic32.a(vector53.o)
 .text          0x00000000        0x0 c:/program files (x86)/microchip/xc32/v1.21/bin/../lib/gcc/pic32mx/4.5.2/../../../../pic32mx/lib/size\libpic32.a(vector54.o)
 .data          0x00000000        0x0 c:/program files (x86)/microchip/xc32/v1.21/bin/../lib/gcc/pic32mx/4.5.2/../../../../pic32mx/lib/size\libpic32.a(vector54.o)
 .bss           0x00000000        0x0 c:/program files (x86)/microchip/xc32/v1.21/bin/../lib/gcc/pic32mx/4.5.2/../../../../pic32mx/lib/size\libpic32.a(vector54.o)
 .reginfo       0x00000000       0x18 c:/program files (x86)/microchip/xc32/v1.21/bin/../lib/gcc/pic32mx/4.5.2/../../../../pic32mx/lib/size\libpic32.a(vector54.o)
 .pdr           0x00000000       0x20 c:/program files (x86)/microchip/xc32/v1.21/bin/../lib/gcc/pic32mx/4.5.2/../../../../pic32mx/lib/size\libpic32.a(vector54.o)
 .text          0x00000000        0x0 c:/program files (x86)/microchip/xc32/v1.21/bin/../lib/gcc/pic32mx/4.5.2/../../../../pic32mx/lib/size\libpic32.a(vector55.o)
 .data          0x00000000        0x0 c:/program files (x86)/microchip/xc32/v1.21/bin/../lib/gcc/pic32mx/4.5.2/../../../../pic32mx/lib/size\libpic32.a(vector55.o)
 .bss           0x00000000        0x0 c:/program files (x86)/microchip/xc32/v1.21/bin/../lib/gcc/pic32mx/4.5.2/../../../../pic32mx/lib/size\libpic32.a(vector55.o)
 .reginfo       0x00000000       0x18 c:/program files (x86)/microchip/xc32/v1.21/bin/../lib/gcc/pic32mx/4.5.2/../../../../pic32mx/lib/size\libpic32.a(vector55.o)
 .pdr           0x00000000       0x20 c:/program files (x86)/microchip/xc32/v1.21/bin/../lib/gcc/pic32mx/4.5.2/../../../../pic32mx/lib/size\libpic32.a(vector55.o)
 .text          0x00000000        0x0 c:/program files (x86)/microchip/xc32/v1.21/bin/../lib/gcc/pic32mx/4.5.2/../../../../pic32mx/lib/size\libpic32.a(vector56.o)
 .data          0x00000000        0x0 c:/program files (x86)/microchip/xc32/v1.21/bin/../lib/gcc/pic32mx/4.5.2/../../../../pic32mx/lib/size\libpic32.a(vector56.o)
 .bss           0x00000000        0x0 c:/program files (x86)/microchip/xc32/v1.21/bin/../lib/gcc/pic32mx/4.5.2/../../../../pic32mx/lib/size\libpic32.a(vector56.o)
 .reginfo       0x00000000       0x18 c:/program files (x86)/microchip/xc32/v1.21/bin/../lib/gcc/pic32mx/4.5.2/../../../../pic32mx/lib/size\libpic32.a(vector56.o)
 .pdr           0x00000000       0x20 c:/program files (x86)/microchip/xc32/v1.21/bin/../lib/gcc/pic32mx/4.5.2/../../../../pic32mx/lib/size\libpic32.a(vector56.o)
 .text          0x00000000        0x0 c:/program files (x86)/microchip/xc32/v1.21/bin/../lib/gcc/pic32mx/4.5.2/../../../../pic32mx/lib/size\libpic32.a(vector57.o)
 .data          0x00000000        0x0 c:/program files (x86)/microchip/xc32/v1.21/bin/../lib/gcc/pic32mx/4.5.2/../../../../pic32mx/lib/size\libpic32.a(vector57.o)
 .bss           0x00000000        0x0 c:/program files (x86)/microchip/xc32/v1.21/bin/../lib/gcc/pic32mx/4.5.2/../../../../pic32mx/lib/size\libpic32.a(vector57.o)
 .reginfo       0x00000000       0x18 c:/program files (x86)/microchip/xc32/v1.21/bin/../lib/gcc/pic32mx/4.5.2/../../../../pic32mx/lib/size\libpic32.a(vector57.o)
 .pdr           0x00000000       0x20 c:/program files (x86)/microchip/xc32/v1.21/bin/../lib/gcc/pic32mx/4.5.2/../../../../pic32mx/lib/size\libpic32.a(vector57.o)
 .text          0x00000000        0x0 c:/program files (x86)/microchip/xc32/v1.21/bin/../lib/gcc/pic32mx/4.5.2/../../../../pic32mx/lib/size\libpic32.a(vector58.o)
 .data          0x00000000        0x0 c:/program files (x86)/microchip/xc32/v1.21/bin/../lib/gcc/pic32mx/4.5.2/../../../../pic32mx/lib/size\libpic32.a(vector58.o)
 .bss           0x00000000        0x0 c:/program files (x86)/microchip/xc32/v1.21/bin/../lib/gcc/pic32mx/4.5.2/../../../../pic32mx/lib/size\libpic32.a(vector58.o)
 .reginfo       0x00000000       0x18 c:/program files (x86)/microchip/xc32/v1.21/bin/../lib/gcc/pic32mx/4.5.2/../../../../pic32mx/lib/size\libpic32.a(vector58.o)
 .pdr           0x00000000       0x20 c:/program files (x86)/microchip/xc32/v1.21/bin/../lib/gcc/pic32mx/4.5.2/../../../../pic32mx/lib/size\libpic32.a(vector58.o)
 .text          0x00000000        0x0 c:/program files (x86)/microchip/xc32/v1.21/bin/../lib/gcc/pic32mx/4.5.2/../../../../pic32mx/lib/size\libpic32.a(vector59.o)
 .data          0x00000000        0x0 c:/program files (x86)/microchip/xc32/v1.21/bin/../lib/gcc/pic32mx/4.5.2/../../../../pic32mx/lib/size\libpic32.a(vector59.o)
 .bss           0x00000000        0x0 c:/program files (x86)/microchip/xc32/v1.21/bin/../lib/gcc/pic32mx/4.5.2/../../../../pic32mx/lib/size\libpic32.a(vector59.o)
 .reginfo       0x00000000       0x18 c:/program files (x86)/microchip/xc32/v1.21/bin/../lib/gcc/pic32mx/4.5.2/../../../../pic32mx/lib/size\libpic32.a(vector59.o)
 .pdr           0x00000000       0x20 c:/program files (x86)/microchip/xc32/v1.21/bin/../lib/gcc/pic32mx/4.5.2/../../../../pic32mx/lib/size\libpic32.a(vector59.o)
 .text          0x00000000        0x0 c:/program files (x86)/microchip/xc32/v1.21/bin/../lib/gcc/pic32mx/4.5.2/../../../../pic32mx/lib/size\libpic32.a(vector60.o)
 .data          0x00000000        0x0 c:/program files (x86)/microchip/xc32/v1.21/bin/../lib/gcc/pic32mx/4.5.2/../../../../pic32mx/lib/size\libpic32.a(vector60.o)
 .bss           0x00000000        0x0 c:/program files (x86)/microchip/xc32/v1.21/bin/../lib/gcc/pic32mx/4.5.2/../../../../pic32mx/lib/size\libpic32.a(vector60.o)
 .reginfo       0x00000000       0x18 c:/program files (x86)/microchip/xc32/v1.21/bin/../lib/gcc/pic32mx/4.5.2/../../../../pic32mx/lib/size\libpic32.a(vector60.o)
 .pdr           0x00000000       0x20 c:/program files (x86)/microchip/xc32/v1.21/bin/../lib/gcc/pic32mx/4.5.2/../../../../pic32mx/lib/size\libpic32.a(vector60.o)
 .text          0x00000000        0x0 c:/program files (x86)/microchip/xc32/v1.21/bin/../lib/gcc/pic32mx/4.5.2/../../../../pic32mx/lib/size\libpic32.a(vector61.o)
 .data          0x00000000        0x0 c:/program files (x86)/microchip/xc32/v1.21/bin/../lib/gcc/pic32mx/4.5.2/../../../../pic32mx/lib/size\libpic32.a(vector61.o)
 .bss           0x00000000        0x0 c:/program files (x86)/microchip/xc32/v1.21/bin/../lib/gcc/pic32mx/4.5.2/../../../../pic32mx/lib/size\libpic32.a(vector61.o)
 .reginfo       0x00000000       0x18 c:/program files (x86)/microchip/xc32/v1.21/bin/../lib/gcc/pic32mx/4.5.2/../../../../pic32mx/lib/size\libpic32.a(vector61.o)
 .pdr           0x00000000       0x20 c:/program files (x86)/microchip/xc32/v1.21/bin/../lib/gcc/pic32mx/4.5.2/../../../../pic32mx/lib/size\libpic32.a(vector61.o)
 .text          0x00000000        0x0 c:/program files (x86)/microchip/xc32/v1.21/bin/../lib/gcc/pic32mx/4.5.2/../../../../pic32mx/lib/size\libpic32.a(vector62.o)
 .data          0x00000000        0x0 c:/program files (x86)/microchip/xc32/v1.21/bin/../lib/gcc/pic32mx/4.5.2/../../../../pic32mx/lib/size\libpic32.a(vector62.o)
 .bss           0x00000000        0x0 c:/program files (x86)/microchip/xc32/v1.21/bin/../lib/gcc/pic32mx/4.5.2/../../../../pic32mx/lib/size\libpic32.a(vector62.o)
 .reginfo       0x00000000       0x18 c:/program files (x86)/microchip/xc32/v1.21/bin/../lib/gcc/pic32mx/4.5.2/../../../../pic32mx/lib/size\libpic32.a(vector62.o)
 .pdr           0x00000000       0x20 c:/program files (x86)/microchip/xc32/v1.21/bin/../lib/gcc/pic32mx/4.5.2/../../../../pic32mx/lib/size\libpic32.a(vector62.o)
 .text          0x00000000        0x0 c:/program files (x86)/microchip/xc32/v1.21/bin/../lib/gcc/pic32mx/4.5.2/../../../../pic32mx/lib/size\libpic32.a(vector63.o)
 .data          0x00000000        0x0 c:/program files (x86)/microchip/xc32/v1.21/bin/../lib/gcc/pic32mx/4.5.2/../../../../pic32mx/lib/size\libpic32.a(vector63.o)
 .bss           0x00000000        0x0 c:/program files (x86)/microchip/xc32/v1.21/bin/../lib/gcc/pic32mx/4.5.2/../../../../pic32mx/lib/size\libpic32.a(vector63.o)
 .reginfo       0x00000000       0x18 c:/program files (x86)/microchip/xc32/v1.21/bin/../lib/gcc/pic32mx/4.5.2/../../../../pic32mx/lib/size\libpic32.a(vector63.o)
 .pdr           0x00000000       0x20 c:/program files (x86)/microchip/xc32/v1.21/bin/../lib/gcc/pic32mx/4.5.2/../../../../pic32mx/lib/size\libpic32.a(vector63.o)
 .text          0x00000000        0x0 c:/program files (x86)/microchip/xc32/v1.21/bin/../lib/gcc/pic32mx/4.5.2/../../../../pic32mx/lib/size\libpic32.a(defaultinterrupt.o)
 .data          0x00000000        0x0 c:/program files (x86)/microchip/xc32/v1.21/bin/../lib/gcc/pic32mx/4.5.2/../../../../pic32mx/lib/size\libpic32.a(defaultinterrupt.o)
 .bss           0x00000000        0x0 c:/program files (x86)/microchip/xc32/v1.21/bin/../lib/gcc/pic32mx/4.5.2/../../../../pic32mx/lib/size\libpic32.a(defaultinterrupt.o)
 .reginfo       0x00000000       0x18 c:/program files (x86)/microchip/xc32/v1.21/bin/../lib/gcc/pic32mx/4.5.2/../../../../pic32mx/lib/size\libpic32.a(defaultinterrupt.o)
 .pdr           0x00000000       0x20 c:/program files (x86)/microchip/xc32/v1.21/bin/../lib/gcc/pic32mx/4.5.2/../../../../pic32mx/lib/size\libpic32.a(defaultinterrupt.o)
 .text          0x00000000        0x0 c:/program files (x86)/microchip/xc32/v1.21/bin/../lib/gcc/pic32mx/4.5.2/../../../../pic32mx/lib/size\libc.a(atoi.o)
 .data          0x00000000        0x0 c:/program files (x86)/microchip/xc32/v1.21/bin/../lib/gcc/pic32mx/4.5.2/../../../../pic32mx/lib/size\libc.a(atoi.o)
 .bss           0x00000000        0x0 c:/program files (x86)/microchip/xc32/v1.21/bin/../lib/gcc/pic32mx/4.5.2/../../../../pic32mx/lib/size\libc.a(atoi.o)
 .reginfo       0x00000000       0x18 c:/program files (x86)/microchip/xc32/v1.21/bin/../lib/gcc/pic32mx/4.5.2/../../../../pic32mx/lib/size\libc.a(atoi.o)
 .pdr           0x00000000       0x20 c:/program files (x86)/microchip/xc32/v1.21/bin/../lib/gcc/pic32mx/4.5.2/../../../../pic32mx/lib/size\libc.a(atoi.o)
 .text          0x00000000        0x0 c:/program files (x86)/microchip/xc32/v1.21/bin/../lib/gcc/pic32mx/4.5.2/../../../../pic32mx/lib/size\libc.a(ctype.o)
 .data          0x00000000        0x0 c:/program files (x86)/microchip/xc32/v1.21/bin/../lib/gcc/pic32mx/4.5.2/../../../../pic32mx/lib/size\libc.a(ctype.o)
 .bss           0x00000000        0x0 c:/program files (x86)/microchip/xc32/v1.21/bin/../lib/gcc/pic32mx/4.5.2/../../../../pic32mx/lib/size\libc.a(ctype.o)
 .reginfo       0x00000000       0x18 c:/program files (x86)/microchip/xc32/v1.21/bin/../lib/gcc/pic32mx/4.5.2/../../../../pic32mx/lib/size\libc.a(ctype.o)
 .pdr           0x00000000        0x0 c:/program files (x86)/microchip/xc32/v1.21/bin/../lib/gcc/pic32mx/4.5.2/../../../../pic32mx/lib/size\libc.a(ctype.o)
 .text          0x00000000        0x0 c:/program files (x86)/microchip/xc32/v1.21/bin/../lib/gcc/pic32mx/4.5.2/../../../../pic32mx/lib/size\libc.a(malloc.o)
 .data          0x00000000        0x0 c:/program files (x86)/microchip/xc32/v1.21/bin/../lib/gcc/pic32mx/4.5.2/../../../../pic32mx/lib/size\libc.a(malloc.o)
 .reginfo       0x00000000       0x18 c:/program files (x86)/microchip/xc32/v1.21/bin/../lib/gcc/pic32mx/4.5.2/../../../../pic32mx/lib/size\libc.a(malloc.o)
 .pdr           0x00000000       0x60 c:/program files (x86)/microchip/xc32/v1.21/bin/../lib/gcc/pic32mx/4.5.2/../../../../pic32mx/lib/size\libc.a(malloc.o)
 .text.realloc  0x00000000      0x130 c:/program files (x86)/microchip/xc32/v1.21/bin/../lib/gcc/pic32mx/4.5.2/../../../../pic32mx/lib/size\libc.a(malloc.o)
 .text          0x00000000        0x0 c:/program files (x86)/microchip/xc32/v1.21/bin/../lib/gcc/pic32mx/4.5.2/../../../../pic32mx/lib/size\libc.a(rand.o)
 .data          0x00000000        0x0 c:/program files (x86)/microchip/xc32/v1.21/bin/../lib/gcc/pic32mx/4.5.2/../../../../pic32mx/lib/size\libc.a(rand.o)
 .reginfo       0x00000000       0x18 c:/program files (x86)/microchip/xc32/v1.21/bin/../lib/gcc/pic32mx/4.5.2/../../../../pic32mx/lib/size\libc.a(rand.o)
 .pdr           0x00000000       0x40 c:/program files (x86)/microchip/xc32/v1.21/bin/../lib/gcc/pic32mx/4.5.2/../../../../pic32mx/lib/size\libc.a(rand.o)
 .text          0x00000000        0x0 c:/program files (x86)/microchip/xc32/v1.21/bin/../lib/gcc/pic32mx/4.5.2/../../../../pic32mx/lib/size\libc.a(strcat.o)
 .data          0x00000000        0x0 c:/program files (x86)/microchip/xc32/v1.21/bin/../lib/gcc/pic32mx/4.5.2/../../../../pic32mx/lib/size\libc.a(strcat.o)
 .bss           0x00000000        0x0 c:/program files (x86)/microchip/xc32/v1.21/bin/../lib/gcc/pic32mx/4.5.2/../../../../pic32mx/lib/size\libc.a(strcat.o)
 .reginfo       0x00000000       0x18 c:/program files (x86)/microchip/xc32/v1.21/bin/../lib/gcc/pic32mx/4.5.2/../../../../pic32mx/lib/size\libc.a(strcat.o)
 .pdr           0x00000000       0x20 c:/program files (x86)/microchip/xc32/v1.21/bin/../lib/gcc/pic32mx/4.5.2/../../../../pic32mx/lib/size\libc.a(strcat.o)
 .text          0x00000000        0x0 c:/program files (x86)/microchip/xc32/v1.21/bin/../lib/gcc/pic32mx/4.5.2/../../../../pic32mx/lib/size\libc.a(strchr.o)
 .data          0x00000000        0x0 c:/program files (x86)/microchip/xc32/v1.21/bin/../lib/gcc/pic32mx/4.5.2/../../../../pic32mx/lib/size\libc.a(strchr.o)
 .bss           0x00000000        0x0 c:/program files (x86)/microchip/xc32/v1.21/bin/../lib/gcc/pic32mx/4.5.2/../../../../pic32mx/lib/size\libc.a(strchr.o)
 .reginfo       0x00000000       0x18 c:/program files (x86)/microchip/xc32/v1.21/bin/../lib/gcc/pic32mx/4.5.2/../../../../pic32mx/lib/size\libc.a(strchr.o)
 .pdr           0x00000000       0x20 c:/program files (x86)/microchip/xc32/v1.21/bin/../lib/gcc/pic32mx/4.5.2/../../../../pic32mx/lib/size\libc.a(strchr.o)
 .text          0x00000000        0x0 c:/program files (x86)/microchip/xc32/v1.21/bin/../lib/gcc/pic32mx/4.5.2/../../../../pic32mx/lib/size\libc.a(strncat.o)
 .data          0x00000000        0x0 c:/program files (x86)/microchip/xc32/v1.21/bin/../lib/gcc/pic32mx/4.5.2/../../../../pic32mx/lib/size\libc.a(strncat.o)
 .bss           0x00000000        0x0 c:/program files (x86)/microchip/xc32/v1.21/bin/../lib/gcc/pic32mx/4.5.2/../../../../pic32mx/lib/size\libc.a(strncat.o)
 .reginfo       0x00000000       0x18 c:/program files (x86)/microchip/xc32/v1.21/bin/../lib/gcc/pic32mx/4.5.2/../../../../pic32mx/lib/size\libc.a(strncat.o)
 .pdr           0x00000000       0x20 c:/program files (x86)/microchip/xc32/v1.21/bin/../lib/gcc/pic32mx/4.5.2/../../../../pic32mx/lib/size\libc.a(strncat.o)
 .text          0x00000000        0x0 c:/program files (x86)/microchip/xc32/v1.21/bin/../lib/gcc/pic32mx/4.5.2/../../../../pic32mx/lib/size\libc.a(strncpy.o)
 .data          0x00000000        0x0 c:/program files (x86)/microchip/xc32/v1.21/bin/../lib/gcc/pic32mx/4.5.2/../../../../pic32mx/lib/size\libc.a(strncpy.o)
 .bss           0x00000000        0x0 c:/program files (x86)/microchip/xc32/v1.21/bin/../lib/gcc/pic32mx/4.5.2/../../../../pic32mx/lib/size\libc.a(strncpy.o)
 .reginfo       0x00000000       0x18 c:/program files (x86)/microchip/xc32/v1.21/bin/../lib/gcc/pic32mx/4.5.2/../../../../pic32mx/lib/size\libc.a(strncpy.o)
 .pdr           0x00000000       0x20 c:/program files (x86)/microchip/xc32/v1.21/bin/../lib/gcc/pic32mx/4.5.2/../../../../pic32mx/lib/size\libc.a(strncpy.o)
 .text.strncpy  0x00000000       0x50 c:/program files (x86)/microchip/xc32/v1.21/bin/../lib/gcc/pic32mx/4.5.2/../../../../pic32mx/lib/size\libc.a(strncpy.o)
 .text          0x00000000        0x0 c:/program files (x86)/microchip/xc32/v1.21/bin/../lib/gcc/pic32mx/4.5.2/../../../../pic32mx/lib/size\libc.a(strstr.o)
 .data          0x00000000        0x0 c:/program files (x86)/microchip/xc32/v1.21/bin/../lib/gcc/pic32mx/4.5.2/../../../../pic32mx/lib/size\libc.a(strstr.o)
 .bss           0x00000000        0x0 c:/program files (x86)/microchip/xc32/v1.21/bin/../lib/gcc/pic32mx/4.5.2/../../../../pic32mx/lib/size\libc.a(strstr.o)
 .reginfo       0x00000000       0x18 c:/program files (x86)/microchip/xc32/v1.21/bin/../lib/gcc/pic32mx/4.5.2/../../../../pic32mx/lib/size\libc.a(strstr.o)
 .pdr           0x00000000       0x20 c:/program files (x86)/microchip/xc32/v1.21/bin/../lib/gcc/pic32mx/4.5.2/../../../../pic32mx/lib/size\libc.a(strstr.o)
 .text          0x00000000        0x0 c:/program files (x86)/microchip/xc32/v1.21/bin/../lib/gcc/pic32mx/4.5.2/../../../../pic32mx/lib/size\libc.a(strtol.o)
 .data          0x00000000        0x0 c:/program files (x86)/microchip/xc32/v1.21/bin/../lib/gcc/pic32mx/4.5.2/../../../../pic32mx/lib/size\libc.a(strtol.o)
 .bss           0x00000000        0x0 c:/program files (x86)/microchip/xc32/v1.21/bin/../lib/gcc/pic32mx/4.5.2/../../../../pic32mx/lib/size\libc.a(strtol.o)
 .reginfo       0x00000000       0x18 c:/program files (x86)/microchip/xc32/v1.21/bin/../lib/gcc/pic32mx/4.5.2/../../../../pic32mx/lib/size\libc.a(strtol.o)
 .pdr           0x00000000       0x40 c:/program files (x86)/microchip/xc32/v1.21/bin/../lib/gcc/pic32mx/4.5.2/../../../../pic32mx/lib/size\libc.a(strtol.o)
 .text          0x00000000        0x0 c:/program files (x86)/microchip/xc32/v1.21/bin/../lib/gcc/pic32mx/4.5.2/../../../../pic32mx/lib/size\libc.a(snprintf_cdnopsuxX.eo)
 .data          0x00000000        0x0 c:/program files (x86)/microchip/xc32/v1.21/bin/../lib/gcc/pic32mx/4.5.2/../../../../pic32mx/lib/size\libc.a(snprintf_cdnopsuxX.eo)
 .bss           0x00000000        0x0 c:/program files (x86)/microchip/xc32/v1.21/bin/../lib/gcc/pic32mx/4.5.2/../../../../pic32mx/lib/size\libc.a(snprintf_cdnopsuxX.eo)
 .reginfo       0x00000000       0x18 c:/program files (x86)/microchip/xc32/v1.21/bin/../lib/gcc/pic32mx/4.5.2/../../../../pic32mx/lib/size\libc.a(snprintf_cdnopsuxX.eo)
 .pdr           0x00000000       0x20 c:/program files (x86)/microchip/xc32/v1.21/bin/../lib/gcc/pic32mx/4.5.2/../../../../pic32mx/lib/size\libc.a(snprintf_cdnopsuxX.eo)
 .text          0x00000000        0x0 c:/program files (x86)/microchip/xc32/v1.21/bin/../lib/gcc/pic32mx/4.5.2/../../../../pic32mx/lib/size\libc.a(sprintf_cdnopsuxX.eo)
 .data          0x00000000        0x0 c:/program files (x86)/microchip/xc32/v1.21/bin/../lib/gcc/pic32mx/4.5.2/../../../../pic32mx/lib/size\libc.a(sprintf_cdnopsuxX.eo)
 .bss           0x00000000        0x0 c:/program files (x86)/microchip/xc32/v1.21/bin/../lib/gcc/pic32mx/4.5.2/../../../../pic32mx/lib/size\libc.a(sprintf_cdnopsuxX.eo)
 .reginfo       0x00000000       0x18 c:/program files (x86)/microchip/xc32/v1.21/bin/../lib/gcc/pic32mx/4.5.2/../../../../pic32mx/lib/size\libc.a(sprintf_cdnopsuxX.eo)
 .pdr           0x00000000       0x20 c:/program files (x86)/microchip/xc32/v1.21/bin/../lib/gcc/pic32mx/4.5.2/../../../../pic32mx/lib/size\libc.a(sprintf_cdnopsuxX.eo)
 .text          0x00000000        0x0 c:/program files (x86)/microchip/xc32/v1.21/bin/../lib/gcc/pic32mx/4.5.2/../../../../pic32mx/lib/size\libc.a(vsnprintf_cdnopsuxX.eo)
 .data          0x00000000        0x0 c:/program files (x86)/microchip/xc32/v1.21/bin/../lib/gcc/pic32mx/4.5.2/../../../../pic32mx/lib/size\libc.a(vsnprintf_cdnopsuxX.eo)
 .bss           0x00000000        0x0 c:/program files (x86)/microchip/xc32/v1.21/bin/../lib/gcc/pic32mx/4.5.2/../../../../pic32mx/lib/size\libc.a(vsnprintf_cdnopsuxX.eo)
 .reginfo       0x00000000       0x18 c:/program files (x86)/microchip/xc32/v1.21/bin/../lib/gcc/pic32mx/4.5.2/../../../../pic32mx/lib/size\libc.a(vsnprintf_cdnopsuxX.eo)
 .pdr           0x00000000       0x20 c:/program files (x86)/microchip/xc32/v1.21/bin/../lib/gcc/pic32mx/4.5.2/../../../../pic32mx/lib/size\libc.a(vsnprintf_cdnopsuxX.eo)
 .text          0x00000000        0x0 c:/program files (x86)/microchip/xc32/v1.21/bin/../lib/gcc/pic32mx/4.5.2/../../../../pic32mx/lib/size\libc.a(vsnprintf.o)
 .data          0x00000000        0x0 c:/program files (x86)/microchip/xc32/v1.21/bin/../lib/gcc/pic32mx/4.5.2/../../../../pic32mx/lib/size\libc.a(vsnprintf.o)
 .bss           0x00000000        0x0 c:/program files (x86)/microchip/xc32/v1.21/bin/../lib/gcc/pic32mx/4.5.2/../../../../pic32mx/lib/size\libc.a(vsnprintf.o)
 .reginfo       0x00000000       0x18 c:/program files (x86)/microchip/xc32/v1.21/bin/../lib/gcc/pic32mx/4.5.2/../../../../pic32mx/lib/size\libc.a(vsnprintf.o)
 .pdr           0x00000000       0x20 c:/program files (x86)/microchip/xc32/v1.21/bin/../lib/gcc/pic32mx/4.5.2/../../../../pic32mx/lib/size\libc.a(vsnprintf.o)
 .text          0x00000000        0x0 c:/program files (x86)/microchip/xc32/v1.21/bin/../lib/gcc/pic32mx/4.5.2/../../../../pic32mx/lib/size\libc.a(ctypef.o)
 .data          0x00000000        0x0 c:/program files (x86)/microchip/xc32/v1.21/bin/../lib/gcc/pic32mx/4.5.2/../../../../pic32mx/lib/size\libc.a(ctypef.o)
 .bss           0x00000000        0x0 c:/program files (x86)/microchip/xc32/v1.21/bin/../lib/gcc/pic32mx/4.5.2/../../../../pic32mx/lib/size\libc.a(ctypef.o)
 .reginfo       0x00000000       0x18 c:/program files (x86)/microchip/xc32/v1.21/bin/../lib/gcc/pic32mx/4.5.2/../../../../pic32mx/lib/size\libc.a(ctypef.o)
 .pdr           0x00000000      0x220 c:/program files (x86)/microchip/xc32/v1.21/bin/../lib/gcc/pic32mx/4.5.2/../../../../pic32mx/lib/size\libc.a(ctypef.o)
 .text.tolower  0x00000000       0x24 c:/program files (x86)/microchip/xc32/v1.21/bin/../lib/gcc/pic32mx/4.5.2/../../../../pic32mx/lib/size\libc.a(ctypef.o)
 .text.isalnum  0x00000000       0x18 c:/program files (x86)/microchip/xc32/v1.21/bin/../lib/gcc/pic32mx/4.5.2/../../../../pic32mx/lib/size\libc.a(ctypef.o)
 .text.isalpha  0x00000000       0x18 c:/program files (x86)/microchip/xc32/v1.21/bin/../lib/gcc/pic32mx/4.5.2/../../../../pic32mx/lib/size\libc.a(ctypef.o)
 .text.isascii  0x00000000        0x8 c:/program files (x86)/microchip/xc32/v1.21/bin/../lib/gcc/pic32mx/4.5.2/../../../../pic32mx/lib/size\libc.a(ctypef.o)
 .text.iscntrl  0x00000000       0x18 c:/program files (x86)/microchip/xc32/v1.21/bin/../lib/gcc/pic32mx/4.5.2/../../../../pic32mx/lib/size\libc.a(ctypef.o)
 .text.isdigit  0x00000000       0x18 c:/program files (x86)/microchip/xc32/v1.21/bin/../lib/gcc/pic32mx/4.5.2/../../../../pic32mx/lib/size\libc.a(ctypef.o)
 .text.isgraph  0x00000000       0x18 c:/program files (x86)/microchip/xc32/v1.21/bin/../lib/gcc/pic32mx/4.5.2/../../../../pic32mx/lib/size\libc.a(ctypef.o)
 .text.islower  0x00000000       0x18 c:/program files (x86)/microchip/xc32/v1.21/bin/../lib/gcc/pic32mx/4.5.2/../../../../pic32mx/lib/size\libc.a(ctypef.o)
 .text.isprint  0x00000000       0x18 c:/program files (x86)/microchip/xc32/v1.21/bin/../lib/gcc/pic32mx/4.5.2/../../../../pic32mx/lib/size\libc.a(ctypef.o)
 .text.ispunct  0x00000000       0x18 c:/program files (x86)/microchip/xc32/v1.21/bin/../lib/gcc/pic32mx/4.5.2/../../../../pic32mx/lib/size\libc.a(ctypef.o)
 .text.isspace  0x00000000       0x18 c:/program files (x86)/microchip/xc32/v1.21/bin/../lib/gcc/pic32mx/4.5.2/../../../../pic32mx/lib/size\libc.a(ctypef.o)
 .text.isupper  0x00000000       0x18 c:/program files (x86)/microchip/xc32/v1.21/bin/../lib/gcc/pic32mx/4.5.2/../../../../pic32mx/lib/size\libc.a(ctypef.o)
 .text.isxdigit
                0x00000000       0x18 c:/program files (x86)/microchip/xc32/v1.21/bin/../lib/gcc/pic32mx/4.5.2/../../../../pic32mx/lib/size\libc.a(ctypef.o)
 .text.toascii  0x00000000        0x8 c:/program files (x86)/microchip/xc32/v1.21/bin/../lib/gcc/pic32mx/4.5.2/../../../../pic32mx/lib/size\libc.a(ctypef.o)
 .text._tolower
                0x00000000        0x8 c:/program files (x86)/microchip/xc32/v1.21/bin/../lib/gcc/pic32mx/4.5.2/../../../../pic32mx/lib/size\libc.a(ctypef.o)
 .text._toupper
                0x00000000        0x8 c:/program files (x86)/microchip/xc32/v1.21/bin/../lib/gcc/pic32mx/4.5.2/../../../../pic32mx/lib/size\libc.a(ctypef.o)
 .text          0x00000000        0x0 c:/program files (x86)/microchip/xc32/v1.21/bin/../lib/gcc/pic32mx/4.5.2/../../../../pic32mx/lib/size\libc.a(errno.o)
 .data          0x00000000        0x0 c:/program files (x86)/microchip/xc32/v1.21/bin/../lib/gcc/pic32mx/4.5.2/../../../../pic32mx/lib/size\libc.a(errno.o)
 .bss           0x00000000        0x0 c:/program files (x86)/microchip/xc32/v1.21/bin/../lib/gcc/pic32mx/4.5.2/../../../../pic32mx/lib/size\libc.a(errno.o)
 .reginfo       0x00000000       0x18 c:/program files (x86)/microchip/xc32/v1.21/bin/../lib/gcc/pic32mx/4.5.2/../../../../pic32mx/lib/size\libc.a(errno.o)
 .pdr           0x00000000        0x0 c:/program files (x86)/microchip/xc32/v1.21/bin/../lib/gcc/pic32mx/4.5.2/../../../../pic32mx/lib/size\libc.a(errno.o)
 .text          0x00000000        0x0 c:/program files (x86)/microchip/xc32/v1.21/bin/../lib/gcc/pic32mx/4.5.2/../../../../pic32mx/lib/size\libc.a(strncmp.o)
 .data          0x00000000        0x0 c:/program files (x86)/microchip/xc32/v1.21/bin/../lib/gcc/pic32mx/4.5.2/../../../../pic32mx/lib/size\libc.a(strncmp.o)
 .bss           0x00000000        0x0 c:/program files (x86)/microchip/xc32/v1.21/bin/../lib/gcc/pic32mx/4.5.2/../../../../pic32mx/lib/size\libc.a(strncmp.o)
 .reginfo       0x00000000       0x18 c:/program files (x86)/microchip/xc32/v1.21/bin/../lib/gcc/pic32mx/4.5.2/../../../../pic32mx/lib/size\libc.a(strncmp.o)
 .pdr           0x00000000       0x20 c:/program files (x86)/microchip/xc32/v1.21/bin/../lib/gcc/pic32mx/4.5.2/../../../../pic32mx/lib/size\libc.a(strncmp.o)
 .text          0x00000000        0x0 c:/program files (x86)/microchip/xc32/v1.21/bin/../lib/gcc/pic32mx/4.5.2/../../../../pic32mx/lib/size\libc.a(doprnt_cdnopsuxX.eo)
 .data          0x00000000        0x0 c:/program files (x86)/microchip/xc32/v1.21/bin/../lib/gcc/pic32mx/4.5.2/../../../../pic32mx/lib/size\libc.a(doprnt_cdnopsuxX.eo)
 .bss           0x00000000        0x0 c:/program files (x86)/microchip/xc32/v1.21/bin/../lib/gcc/pic32mx/4.5.2/../../../../pic32mx/lib/size\libc.a(doprnt_cdnopsuxX.eo)
 .reginfo       0x00000000       0x18 c:/program files (x86)/microchip/xc32/v1.21/bin/../lib/gcc/pic32mx/4.5.2/../../../../pic32mx/lib/size\libc.a(doprnt_cdnopsuxX.eo)
 .pdr           0x00000000       0x20 c:/program files (x86)/microchip/xc32/v1.21/bin/../lib/gcc/pic32mx/4.5.2/../../../../pic32mx/lib/size\libc.a(doprnt_cdnopsuxX.eo)
 .text          0x00000000        0x0 c:/program files (x86)/microchip/xc32/v1.21/bin/../lib/gcc/pic32mx/4.5.2/../../../../pic32mx/lib/size\libc.a(doprnt.o)
 .data          0x00000000        0x0 c:/program files (x86)/microchip/xc32/v1.21/bin/../lib/gcc/pic32mx/4.5.2/../../../../pic32mx/lib/size\libc.a(doprnt.o)
 .bss           0x00000000        0x0 c:/program files (x86)/microchip/xc32/v1.21/bin/../lib/gcc/pic32mx/4.5.2/../../../../pic32mx/lib/size\libc.a(doprnt.o)
 .reginfo       0x00000000       0x18 c:/program files (x86)/microchip/xc32/v1.21/bin/../lib/gcc/pic32mx/4.5.2/../../../../pic32mx/lib/size\libc.a(doprnt.o)
 .pdr           0x00000000       0x60 c:/program files (x86)/microchip/xc32/v1.21/bin/../lib/gcc/pic32mx/4.5.2/../../../../pic32mx/lib/size\libc.a(doprnt.o)
 .text          0x00000000        0x0 c:/program files (x86)/microchip/xc32/v1.21/bin/../lib/gcc/pic32mx/4.5.2/../../../../pic32mx/lib/size\libc.a(_fputc_simple.o)
 .data          0x00000000        0x0 c:/program files (x86)/microchip/xc32/v1.21/bin/../lib/gcc/pic32mx/4.5.2/../../../../pic32mx/lib/size\libc.a(_fputc_simple.o)
 .bss           0x00000000        0x0 c:/program files (x86)/microchip/xc32/v1.21/bin/../lib/gcc/pic32mx/4.5.2/../../../../pic32mx/lib/size\libc.a(_fputc_simple.o)
 .reginfo       0x00000000       0x18 c:/program files (x86)/microchip/xc32/v1.21/bin/../lib/gcc/pic32mx/4.5.2/../../../../pic32mx/lib/size\libc.a(_fputc_simple.o)
 .pdr           0x00000000       0x20 c:/program files (x86)/microchip/xc32/v1.21/bin/../lib/gcc/pic32mx/4.5.2/../../../../pic32mx/lib/size\libc.a(_fputc_simple.o)
 .text          0x00000000        0x0 c:/program files (x86)/microchip/xc32/v1.21/bin/../lib/gcc/pic32mx/4.5.2/../../../../pic32mx/lib/size\libc.a(powersf.o)
 .data          0x00000000        0x0 c:/program files (x86)/microchip/xc32/v1.21/bin/../lib/gcc/pic32mx/4.5.2/../../../../pic32mx/lib/size\libc.a(powersf.o)
 .bss           0x00000000        0x0 c:/program files (x86)/microchip/xc32/v1.21/bin/../lib/gcc/pic32mx/4.5.2/../../../../pic32mx/lib/size\libc.a(powersf.o)
 .reginfo       0x00000000       0x18 c:/program files (x86)/microchip/xc32/v1.21/bin/../lib/gcc/pic32mx/4.5.2/../../../../pic32mx/lib/size\libc.a(powersf.o)
 .pdr           0x00000000        0x0 c:/program files (x86)/microchip/xc32/v1.21/bin/../lib/gcc/pic32mx/4.5.2/../../../../pic32mx/lib/size\libc.a(powersf.o)
 .text          0x00000000        0x0 c:/program files (x86)/microchip/xc32/v1.21/bin/../lib/gcc/pic32mx/4.5.2/../../../../pic32mx/lib/size\libc.a(_iob.o)
 .data          0x00000000       0xa0 c:/program files (x86)/microchip/xc32/v1.21/bin/../lib/gcc/pic32mx/4.5.2/../../../../pic32mx/lib/size\libc.a(_iob.o)
 .reginfo       0x00000000       0x18 c:/program files (x86)/microchip/xc32/v1.21/bin/../lib/gcc/pic32mx/4.5.2/../../../../pic32mx/lib/size\libc.a(_iob.o)
 .pdr           0x00000000        0x0 c:/program files (x86)/microchip/xc32/v1.21/bin/../lib/gcc/pic32mx/4.5.2/../../../../pic32mx/lib/size\libc.a(_iob.o)
 .sdata         0x00000000        0x4 c:/program files (x86)/microchip/xc32/v1.21/bin/../lib/gcc/pic32mx/4.5.2/../../../../pic32mx/lib/size\libc.a(_iob.o)
 .text          0x00000000        0x0 c:/program files (x86)/microchip/xc32/v1.21/bin/../lib/gcc/pic32mx/4.5.2/../../../../pic32mx/lib/size\libc.a(_flsbuf_simple.o)
 .data          0x00000000        0x0 c:/program files (x86)/microchip/xc32/v1.21/bin/../lib/gcc/pic32mx/4.5.2/../../../../pic32mx/lib/size\libc.a(_flsbuf_simple.o)
 .bss           0x00000000        0x0 c:/program files (x86)/microchip/xc32/v1.21/bin/../lib/gcc/pic32mx/4.5.2/../../../../pic32mx/lib/size\libc.a(_flsbuf_simple.o)
 .reginfo       0x00000000       0x18 c:/program files (x86)/microchip/xc32/v1.21/bin/../lib/gcc/pic32mx/4.5.2/../../../../pic32mx/lib/size\libc.a(_flsbuf_simple.o)
 .pdr           0x00000000       0x20 c:/program files (x86)/microchip/xc32/v1.21/bin/../lib/gcc/pic32mx/4.5.2/../../../../pic32mx/lib/size\libc.a(_flsbuf_simple.o)
 .text          0x00000000        0x0 c:/program files (x86)/microchip/xc32/v1.21/bin/../lib/gcc/pic32mx/4.5.2/../../../../pic32mx/lib/size\libpic32.a(sbrk.o)
 .data          0x00000000        0x0 c:/program files (x86)/microchip/xc32/v1.21/bin/../lib/gcc/pic32mx/4.5.2/../../../../pic32mx/lib/size\libpic32.a(sbrk.o)
 .reginfo       0x00000000       0x18 c:/program files (x86)/microchip/xc32/v1.21/bin/../lib/gcc/pic32mx/4.5.2/../../../../pic32mx/lib/size\libpic32.a(sbrk.o)
 .pdr           0x00000000       0xa0 c:/program files (x86)/microchip/xc32/v1.21/bin/../lib/gcc/pic32mx/4.5.2/../../../../pic32mx/lib/size\libpic32.a(sbrk.o)
 .text.getpagesize
                0x00000000        0x8 c:/program files (x86)/microchip/xc32/v1.21/bin/../lib/gcc/pic32mx/4.5.2/../../../../pic32mx/lib/size\libpic32.a(sbrk.o)
 .text          0x00000000        0x0 c:/program files (x86)/microchip/xc32/v1.21/bin/../lib/gcc/pic32mx/4.5.2/../../../../pic32mx/lib/size\libpic32.a(write.o)
 .data          0x00000000        0x0 c:/program files (x86)/microchip/xc32/v1.21/bin/../lib/gcc/pic32mx/4.5.2/../../../../pic32mx/lib/size\libpic32.a(write.o)
 .bss           0x00000000        0x0 c:/program files (x86)/microchip/xc32/v1.21/bin/../lib/gcc/pic32mx/4.5.2/../../../../pic32mx/lib/size\libpic32.a(write.o)
 .reginfo       0x00000000       0x18 c:/program files (x86)/microchip/xc32/v1.21/bin/../lib/gcc/pic32mx/4.5.2/../../../../pic32mx/lib/size\libpic32.a(write.o)
 .pdr           0x00000000       0x20 c:/program files (x86)/microchip/xc32/v1.21/bin/../lib/gcc/pic32mx/4.5.2/../../../../pic32mx/lib/size\libpic32.a(write.o)
 .text          0x00000000        0x0 c:/program files (x86)/microchip/xc32/v1.21/bin/../lib/gcc/pic32mx/4.5.2/../../../../pic32mx/lib/size\libpic32.a(_mon_putc.o)
 .data          0x00000000        0x0 c:/program files (x86)/microchip/xc32/v1.21/bin/../lib/gcc/pic32mx/4.5.2/../../../../pic32mx/lib/size\libpic32.a(_mon_putc.o)
 .bss           0x00000000        0x0 c:/program files (x86)/microchip/xc32/v1.21/bin/../lib/gcc/pic32mx/4.5.2/../../../../pic32mx/lib/size\libpic32.a(_mon_putc.o)
 .reginfo       0x00000000       0x18 c:/program files (x86)/microchip/xc32/v1.21/bin/../lib/gcc/pic32mx/4.5.2/../../../../pic32mx/lib/size\libpic32.a(_mon_putc.o)
 .pdr           0x00000000       0x20 c:/program files (x86)/microchip/xc32/v1.21/bin/../lib/gcc/pic32mx/4.5.2/../../../../pic32mx/lib/size\libpic32.a(_mon_putc.o)
 .text          0x00000000        0x0 c:/program files (x86)/microchip/xc32/v1.21/bin/../lib/gcc/pic32mx/4.5.2/../../../../pic32mx/lib/size\libpic32.a(xc32_uart.o)
 .data          0x00000000        0x0 c:/program files (x86)/microchip/xc32/v1.21/bin/../lib/gcc/pic32mx/4.5.2/../../../../pic32mx/lib/size\libpic32.a(xc32_uart.o)
 .bss           0x00000000        0x0 c:/program files (x86)/microchip/xc32/v1.21/bin/../lib/gcc/pic32mx/4.5.2/../../../../pic32mx/lib/size\libpic32.a(xc32_uart.o)
 .reginfo       0x00000000       0x18 c:/program files (x86)/microchip/xc32/v1.21/bin/../lib/gcc/pic32mx/4.5.2/../../../../pic32mx/lib/size\libpic32.a(xc32_uart.o)
 .pdr           0x00000000        0x0 c:/program files (x86)/microchip/xc32/v1.21/bin/../lib/gcc/pic32mx/4.5.2/../../../../pic32mx/lib/size\libpic32.a(xc32_uart.o)
 .data          0x00000000        0x0 c:/program files (x86)/microchip/xc32/v1.21/bin/../lib/gcc/pic32mx/4.5.2/../../../../pic32mx/lib/size\libm.a(fpmod32.o)
 .bss           0x00000000        0x0 c:/program files (x86)/microchip/xc32/v1.21/bin/../lib/gcc/pic32mx/4.5.2/../../../../pic32mx/lib/size\libm.a(fpmod32.o)
 .reginfo       0x00000000       0x18 c:/program files (x86)/microchip/xc32/v1.21/bin/../lib/gcc/pic32mx/4.5.2/../../../../pic32mx/lib/size\libm.a(fpmod32.o)
 .pdr           0x00000000        0x0 c:/program files (x86)/microchip/xc32/v1.21/bin/../lib/gcc/pic32mx/4.5.2/../../../../pic32mx/lib/size\libm.a(fpmod32.o)
 .data          0x00000000        0x0 c:/program files (x86)/microchip/xc32/v1.21/bin/../lib/gcc/pic32mx/4.5.2/../../../../pic32mx/lib/size\libm.a(fp32.o)
 .bss           0x00000000        0x0 c:/program files (x86)/microchip/xc32/v1.21/bin/../lib/gcc/pic32mx/4.5.2/../../../../pic32mx/lib/size\libm.a(fp32.o)
 .reginfo       0x00000000       0x18 c:/program files (x86)/microchip/xc32/v1.21/bin/../lib/gcc/pic32mx/4.5.2/../../../../pic32mx/lib/size\libm.a(fp32.o)
 .pdr           0x00000000        0x0 c:/program files (x86)/microchip/xc32/v1.21/bin/../lib/gcc/pic32mx/4.5.2/../../../../pic32mx/lib/size\libm.a(fp32.o)
 .text          0x00000000        0x0 c:/program files (x86)/microchip/xc32/v1.21/bin/../lib/gcc/pic32mx/4.5.2/../../../../pic32mx/lib/size\libe.a(_floatdisf.o)
 .data          0x00000000        0x0 c:/program files (x86)/microchip/xc32/v1.21/bin/../lib/gcc/pic32mx/4.5.2/../../../../pic32mx/lib/size\libe.a(_floatdisf.o)
 .bss           0x00000000        0x0 c:/program files (x86)/microchip/xc32/v1.21/bin/../lib/gcc/pic32mx/4.5.2/../../../../pic32mx/lib/size\libe.a(_floatdisf.o)
 .reginfo       0x00000000       0x18 c:/program files (x86)/microchip/xc32/v1.21/bin/../lib/gcc/pic32mx/4.5.2/../../../../pic32mx/lib/size\libe.a(_floatdisf.o)
 .pdr           0x00000000       0x20 c:/program files (x86)/microchip/xc32/v1.21/bin/../lib/gcc/pic32mx/4.5.2/../../../../pic32mx/lib/size\libe.a(_floatdisf.o)
 .data          0x00000000        0x0 c:/program files (x86)/microchip/xc32/v1.21/bin/../lib/gcc/pic32mx/4.5.2/size\libgcc.a(_lshrdi3.o)
 .bss           0x00000000        0x0 c:/program files (x86)/microchip/xc32/v1.21/bin/../lib/gcc/pic32mx/4.5.2/size\libgcc.a(_lshrdi3.o)
 .reginfo       0x00000000       0x18 c:/program files (x86)/microchip/xc32/v1.21/bin/../lib/gcc/pic32mx/4.5.2/size\libgcc.a(_lshrdi3.o)
 .pdr           0x00000000       0x20 c:/program files (x86)/microchip/xc32/v1.21/bin/../lib/gcc/pic32mx/4.5.2/size\libgcc.a(_lshrdi3.o)
 .data          0x00000000        0x0 c:/program files (x86)/microchip/xc32/v1.21/bin/../lib/gcc/pic32mx/4.5.2/size\libgcc.a(_floatundisf.o)
 .bss           0x00000000        0x0 c:/program files (x86)/microchip/xc32/v1.21/bin/../lib/gcc/pic32mx/4.5.2/size\libgcc.a(_floatundisf.o)
 .reginfo       0x00000000       0x18 c:/program files (x86)/microchip/xc32/v1.21/bin/../lib/gcc/pic32mx/4.5.2/size\libgcc.a(_floatundisf.o)
 .pdr           0x00000000       0x20 c:/program files (x86)/microchip/xc32/v1.21/bin/../lib/gcc/pic32mx/4.5.2/size\libgcc.a(_floatundisf.o)
 .data          0x00000000        0x0 c:/program files (x86)/microchip/xc32/v1.21/bin/../lib/gcc/pic32mx/4.5.2/size\libgcc.a(_umoddi3.o)
 .bss           0x00000000        0x0 c:/program files (x86)/microchip/xc32/v1.21/bin/../lib/gcc/pic32mx/4.5.2/size\libgcc.a(_umoddi3.o)
 .reginfo       0x00000000       0x18 c:/program files (x86)/microchip/xc32/v1.21/bin/../lib/gcc/pic32mx/4.5.2/size\libgcc.a(_umoddi3.o)
 .pdr           0x00000000       0x20 c:/program files (x86)/microchip/xc32/v1.21/bin/../lib/gcc/pic32mx/4.5.2/size\libgcc.a(_umoddi3.o)
 .data          0x00000000        0x0 c:/program files (x86)/microchip/xc32/v1.21/bin/../lib/gcc/pic32mx/4.5.2/size\libgcc.a(floatunsisf.o)
 .bss           0x00000000        0x0 c:/program files (x86)/microchip/xc32/v1.21/bin/../lib/gcc/pic32mx/4.5.2/size\libgcc.a(floatunsisf.o)
 .reginfo       0x00000000       0x18 c:/program files (x86)/microchip/xc32/v1.21/bin/../lib/gcc/pic32mx/4.5.2/size\libgcc.a(floatunsisf.o)
 .pdr           0x00000000       0x20 c:/program files (x86)/microchip/xc32/v1.21/bin/../lib/gcc/pic32mx/4.5.2/size\libgcc.a(floatunsisf.o)

Memory Configuration

Name             Origin             Length             Attributes
kseg0_program_mem 0x9d000000         0x00080000         xr
kseg0_boot_mem   0x9fc00490         0x00000970
exception_mem    0x9fc01000         0x00001000
kseg1_boot_mem   0xbfc00000         0x00000490
debug_exec_mem   0xbfc02000         0x00000ff0
config3          0xbfc02ff0         0x00000004
config2          0xbfc02ff4         0x00000004
config1          0xbfc02ff8         0x00000004
config0          0xbfc02ffc         0x00000004
kseg1_data_mem   0xa0000000         0x00020000         w !x
sfrs             0xbf800000         0x00100000
configsfrs       0xbfc02ff0         0x00000010
*default*        0x00000000         0xffffffff

Linker script and memory map

LOAD c:/program files (x86)/microchip/xc32/v1.21/bin/../lib/gcc/pic32mx/4.5.2/../../../../pic32mx/lib/size/crt0.o
LOAD build/WiFIG/production/_ext/1293749816/bsp.o
LOAD build/WiFIG/production/_ext/101875047/hashes.o
LOAD build/WiFIG/production/_ext/101875047/lfsr.o
LOAD build/WiFIG/production/_ext/101875047/big_int.o
LOAD build/WiFIG/production/_ext/101875047/big_int_helper_c32.o
LOAD build/WiFIG/production/_ext/101875047/helpers.o
LOAD build/WiFIG/production/_ext/1472/berkeley_tcp_client_demo.o
LOAD build/WiFIG/production/_ext/1472/berkeley_tcp_server_demo.o
LOAD build/WiFIG/production/_ext/1472/berkeley_udp_client_demo.o
LOAD build/WiFIG/production/_ext/1472/generic_tcp_client.o
LOAD build/WiFIG/production/_ext/1472/generic_tcp_server.o
LOAD build/WiFIG/production/_ext/1472/ping_demo.o
LOAD build/WiFIG/production/_ext/1472/smtp_demo.o
LOAD build/WiFIG/production/_ext/365611741/system_services.o
LOAD build/WiFIG/production/_ext/365611741/system_debug.o
LOAD build/WiFIG/production/_ext/365611741/system_random.o
LOAD build/WiFIG/production/_ext/365611741/system_command.o
LOAD build/WiFIG/production/_ext/365611741/system_userio.o
LOAD build/WiFIG/production/_ext/97638081/sys_fs.o
LOAD build/WiFIG/production/_ext/97638081/mpfs2.o
LOAD build/WiFIG/production/_ext/792872985/usart.o
LOAD build/WiFIG/production/_ext/792872985/lcd.o
LOAD build/WiFIG/production/_ext/792872985/drv_spi.o
LOAD build/WiFIG/production/_ext/792872985/db_appio.o
LOAD build/WiFIG/production/_ext/792872985/spi_ram.o
LOAD build/WiFIG/production/_ext/792872985/spi_eeprom.o
LOAD build/WiFIG/production/_ext/792872985/spi_flash.o
LOAD build/WiFIG/production/_ext/792872985/drv_media.o
LOAD build/WiFIG/production/_ext/427700826/tcpip_announce.o
LOAD build/WiFIG/production/_ext/427700826/http2.o
LOAD build/WiFIG/production/_ext/427700826/arcfour.o
LOAD build/WiFIG/production/_ext/427700826/arp.o
LOAD build/WiFIG/production/_ext/427700826/berkeley_api.o
LOAD build/WiFIG/production/_ext/427700826/dhcp.o
LOAD build/WiFIG/production/_ext/427700826/dhcps.o
LOAD build/WiFIG/production/_ext/427700826/dns.o
LOAD build/WiFIG/production/_ext/427700826/dnss.o
LOAD build/WiFIG/production/_ext/427700826/dyn_dns.o
LOAD build/WiFIG/production/_ext/427700826/enc28_mac.o
LOAD build/WiFIG/production/_ext/427700826/enc28j60.o
LOAD build/WiFIG/production/_ext/427700826/encs24j600.o
LOAD build/WiFIG/production/_ext/427700826/encx24_mac.o
LOAD build/WiFIG/production/_ext/427700826/eth_pic32_ext_phy.o
LOAD build/WiFIG/production/_ext/427700826/eth_pic32_ext_phy_dp83848.o
LOAD build/WiFIG/production/_ext/427700826/eth_pic32_int_mac.o
LOAD build/WiFIG/production/_ext/427700826/ftp.o
LOAD build/WiFIG/production/_ext/427700826/hash_fnv.o
LOAD build/WiFIG/production/_ext/427700826/hash_tbl.o
LOAD build/WiFIG/production/_ext/427700826/icmp.o
LOAD build/WiFIG/production/_ext/427700826/icmpv6.o
LOAD build/WiFIG/production/_ext/427700826/ipv4.o
LOAD build/WiFIG/production/_ext/427700826/ipv6.o
LOAD build/WiFIG/production/_ext/427700826/mac_events_pic32.o
LOAD build/WiFIG/production/_ext/427700826/nbns.o
LOAD build/WiFIG/production/_ext/427700826/ndp.o
LOAD build/WiFIG/production/_ext/427700826/tcpip_reboot.o
LOAD build/WiFIG/production/_ext/427700826/rsa.o
LOAD build/WiFIG/production/_ext/427700826/smtp.o
LOAD build/WiFIG/production/_ext/427700826/snmp.o
LOAD build/WiFIG/production/_ext/427700826/snmpv3.o
LOAD build/WiFIG/production/_ext/427700826/snmpv3_usm.o
LOAD build/WiFIG/production/_ext/427700826/sntp.o
LOAD build/WiFIG/production/_ext/427700826/ssl.o
LOAD build/WiFIG/production/_ext/427700826/tcp.o
LOAD build/WiFIG/production/_ext/427700826/tcpip_heap_alloc.o
LOAD build/WiFIG/production/_ext/427700826/tcpip_storage.o
LOAD build/WiFIG/production/_ext/427700826/telnet.o
LOAD build/WiFIG/production/_ext/427700826/tftpc.o
LOAD build/WiFIG/production/_ext/427700826/udp.o
LOAD build/WiFIG/production/_ext/427700826/tcpip_mac_object.o
LOAD build/WiFIG/production/_ext/427700826/tcpip_manager.o
LOAD build/WiFIG/production/_ext/427700826/tcpip_helpers.o
LOAD build/WiFIG/production/_ext/427700826/tcpip_commands.o
LOAD build/WiFIG/production/_ext/427700826/iperf.o
LOAD build/WiFIG/production/_ext/427700826/tcpip_helper_c32.o
LOAD build/WiFIG/production/_ext/427700826/tcpip_notify.o
LOAD build/WiFIG/production/_ext/427700826/zero_conf_helper.o
LOAD build/WiFIG/production/_ext/427700826/zero_conf_link_local.o
LOAD build/WiFIG/production/_ext/427700826/zero_conf_multicast_dns.o
LOAD build/WiFIG/production/_ext/334706090/wf_tx_power.o
LOAD build/WiFIG/production/_ext/334706090/wf_connect.o
LOAD build/WiFIG/production/_ext/334706090/wf_connection_algorithm.o
LOAD build/WiFIG/production/_ext/334706090/wf_connection_manager.o
LOAD build/WiFIG/production/_ext/334706090/wf_connection_profile.o
LOAD build/WiFIG/production/_ext/334706090/wf_easy_config.o
LOAD build/WiFIG/production/_ext/334706090/wf_eint.o
LOAD build/WiFIG/production/_ext/334706090/wf_event_handler.o
LOAD build/WiFIG/production/_ext/334706090/wf_init.o
LOAD build/WiFIG/production/_ext/334706090/wf_power_save.o
LOAD build/WiFIG/production/_ext/334706090/wf_scan.o
LOAD build/WiFIG/production/_ext/334706090/wf_spi.o
LOAD build/WiFIG/production/_ext/334706090/mrf24w_mac_pic32.o
LOAD build/WiFIG/production/_ext/334706090/mrf24w_events.o
LOAD build/WiFIG/production/_ext/334706090/wf_debug_output.o
LOAD build/WiFIG/production/_ext/334706090/wf_commands.o
LOAD build/WiFIG/production/_ext/334706090/wf_pbkdf2.o
LOAD build/WiFIG/production/_ext/334706090/wf_driver_com_24g.o
LOAD build/WiFIG/production/_ext/334706090/wf_driver_raw_24g.o
LOAD build/WiFIG/production/_ext/334706090/wf_mac_24g.o
LOAD build/WiFIG/production/_ext/334706090/wf_mgmt_msg_24g.o
LOAD build/WiFIG/production/_ext/334706090/wf_param_msg_24g.o
LOAD build/WiFIG/production/_ext/334706090/wf_configData.o
LOAD build/WiFIG/production/_ext/1472/main_demo.o
LOAD build/WiFIG/production/_ext/1472/custom_snmp_app.o
LOAD build/WiFIG/production/_ext/1472/custom_ssl_cert.o
LOAD build/WiFIG/production/_ext/1472/mpfs_img2.o
LOAD build/WiFIG/production/_ext/1472/wf_config.o
LOAD build/WiFIG/production/_ext/1472/custom_http_app.o
LOAD build/WiFIG/production/_ext/1472/tcp6_demo_app.o
                0x00000001                __MPLAB_BUILD = 0x1
                0x00005208                _min_heap_size = 0x5208
                0x00000800                _min_stack_size = 0x800
LOAD c:/program files (x86)/microchip/xc32/v1.21/bin/../lib/gcc/pic32mx/4.5.2/../../../../pic32mx/lib/./proc/32MX695F512H\default_isr_vectors.o
                0x00000400                PROVIDE (_min_stack_size, 0x400)
LOAD c:/program files (x86)/microchip/xc32/v1.21/bin/../lib/gcc/pic32mx/4.5.2/../../../../pic32mx/lib/./proc/32MX695F512H\processor.o
START GROUP
LOAD c:/program files (x86)/microchip/xc32/v1.21/bin/../lib/gcc/pic32mx/4.5.2/../../../../pic32mx/lib/size\libmchp_peripheral.a
END GROUP
START GROUP
LOAD c:/program files (x86)/microchip/xc32/v1.21/bin/../lib/gcc/pic32mx/4.5.2/../../../../pic32mx/lib/size\libmchp_peripheral_32MX695F512H.a
END GROUP
                0x00000001                PROVIDE (_vector_spacing, 0x1)
                0x9fc01000                _ebase_address = 0x9fc01000
                0xbfc00000                _RESET_ADDR = 0xbfc00000
                0xbfc00380                _BEV_EXCPT_ADDR = 0xbfc00380
                0xbfc00480                _DBG_EXCPT_ADDR = 0xbfc00480
                0xbfc02000                _DBG_CODE_ADDR = 0xbfc02000
                0x00000ff0                _DBG_CODE_SIZE = 0xff0
                0x9fc01180                _GEN_EXCPT_ADDR = (_ebase_address + 0x180)

.config_BFC02FF0
 *(.config_BFC02FF0)

.config_BFC02FF4
                0xbfc02ff4        0x4
 *(.config_BFC02FF4)
 .config_BFC02FF4
                0xbfc02ff4        0x4 build/WiFIG/production/_ext/1293749816/bsp.o

.config_BFC02FF8
                0xbfc02ff8        0x4
 *(.config_BFC02FF8)
 .config_BFC02FF8
                0xbfc02ff8        0x4 build/WiFIG/production/_ext/1293749816/bsp.o

.config_BFC02FFC
                0xbfc02ffc        0x4
 *(.config_BFC02FFC)
 .config_BFC02FFC
                0xbfc02ffc        0x4 build/WiFIG/production/_ext/1293749816/bsp.o
                0xbfc02000                PROVIDE (_DBG_CODE_ADDR, 0xbfc02000)
                0x00000ff0                PROVIDE (_DBG_CODE_SIZE, 0xff0)

.reset          0xbfc00000      0x1f4
 *(.reset)
 .reset         0xbfc00000       0x10 c:/program files (x86)/microchip/xc32/v1.21/bin/../lib/gcc/pic32mx/4.5.2/../../../../pic32mx/lib/size/crt0.o
                0xbfc00000                _reset
 *(.reset.startup)
 .reset.startup
                0xbfc00010      0x1e4 c:/program files (x86)/microchip/xc32/v1.21/bin/../lib/gcc/pic32mx/4.5.2/../../../../pic32mx/lib/size/crt0.o

.bev_excpt      0xbfc00380       0x10
 *(.bev_handler)
 .bev_handler   0xbfc00380       0x10 c:/program files (x86)/microchip/xc32/v1.21/bin/../lib/gcc/pic32mx/4.5.2/../../../../pic32mx/lib/size/crt0.o

.dbg_excpt      0xbfc00480        0x0
                0xbfc00480                . = (. + DEFINED (_DEBUGGER)?0x8:0x0)

.dbg_code       0xbfc02000        0x0
                0xbfc02000                . = (. + DEFINED (_DEBUGGER)?_DBG_CODE_SIZE:0x0)

.app_excpt      0x9fc01180       0x10
 *(.gen_handler)
 .gen_handler   0x9fc01180       0x10 c:/program files (x86)/microchip/xc32/v1.21/bin/../lib/gcc/pic32mx/4.5.2/../../../../pic32mx/lib/size/crt0.o

.vector_0       0x9fc01200        0x8
 *(.vector_0)
 .vector_0      0x9fc01200        0x8 build/WiFIG/production/_ext/365611741/system_services.o
                0x9fc01200                __vector_dispatch_0
                0x00000001                ASSERT (((_vector_spacing == 0x0) || (SIZEOF (.vector_0) <= (_vector_spacing << 0x5))), function at exception vector 0 too large)

.vector_1       0x9fc01220        0x8
 *(.vector_1)
 .vector_1      0x9fc01220        0x8 c:/program files (x86)/microchip/xc32/v1.21/bin/../lib/gcc/pic32mx/4.5.2/../../../../pic32mx/lib/size\libpic32.a(vector1.o)
                0x9fc01220                __vector_dispatch_1
                0x00000001                ASSERT (((_vector_spacing == 0x0) || (SIZEOF (.vector_1) <= (_vector_spacing << 0x5))), function at exception vector 1 too large)

.vector_2       0x9fc01240        0x8
 *(.vector_2)
 .vector_2      0x9fc01240        0x8 c:/program files (x86)/microchip/xc32/v1.21/bin/../lib/gcc/pic32mx/4.5.2/../../../../pic32mx/lib/size\libpic32.a(vector2.o)
                0x9fc01240                __vector_dispatch_2
                0x00000001                ASSERT (((_vector_spacing == 0x0) || (SIZEOF (.vector_2) <= (_vector_spacing << 0x5))), function at exception vector 2 too large)

.vector_3       0x9fc01260        0x8
 *(.vector_3)
 .vector_3      0x9fc01260        0x8 c:/program files (x86)/microchip/xc32/v1.21/bin/../lib/gcc/pic32mx/4.5.2/../../../../pic32mx/lib/size\libpic32.a(vector3.o)
                0x9fc01260                __vector_dispatch_3
                0x00000001                ASSERT (((_vector_spacing == 0x0) || (SIZEOF (.vector_3) <= (_vector_spacing << 0x5))), function at exception vector 3 too large)

.vector_4       0x9fc01280        0x8
 *(.vector_4)
 .vector_4      0x9fc01280        0x8 c:/program files (x86)/microchip/xc32/v1.21/bin/../lib/gcc/pic32mx/4.5.2/../../../../pic32mx/lib/size\libpic32.a(vector4.o)
                0x9fc01280                __vector_dispatch_4
                0x00000001                ASSERT (((_vector_spacing == 0x0) || (SIZEOF (.vector_4) <= (_vector_spacing << 0x5))), function at exception vector 4 too large)

.vector_5       0x9fc012a0        0x8
 *(.vector_5)
 .vector_5      0x9fc012a0        0x8 c:/program files (x86)/microchip/xc32/v1.21/bin/../lib/gcc/pic32mx/4.5.2/../../../../pic32mx/lib/size\libpic32.a(vector5.o)
                0x9fc012a0                __vector_dispatch_5
                0x00000001                ASSERT (((_vector_spacing == 0x0) || (SIZEOF (.vector_5) <= (_vector_spacing << 0x5))), function at exception vector 5 too large)

.vector_6       0x9fc012c0        0x8
 *(.vector_6)
 .vector_6      0x9fc012c0        0x8 c:/program files (x86)/microchip/xc32/v1.21/bin/../lib/gcc/pic32mx/4.5.2/../../../../pic32mx/lib/size\libpic32.a(vector6.o)
                0x9fc012c0                __vector_dispatch_6
                0x00000001                ASSERT (((_vector_spacing == 0x0) || (SIZEOF (.vector_6) <= (_vector_spacing << 0x5))), function at exception vector 6 too large)

.vector_7       0x9fc012e0        0x8
 *(.vector_7)
 .vector_7      0x9fc012e0        0x8 build/WiFIG/production/_ext/365611741/system_services.o
                0x9fc012e0                __vector_dispatch_7
                0x00000001                ASSERT (((_vector_spacing == 0x0) || (SIZEOF (.vector_7) <= (_vector_spacing << 0x5))), function at exception vector 7 too large)

.vector_8       0x9fc01300        0x8
 *(.vector_8)
 .vector_8      0x9fc01300        0x8 c:/program files (x86)/microchip/xc32/v1.21/bin/../lib/gcc/pic32mx/4.5.2/../../../../pic32mx/lib/size\libpic32.a(vector8.o)
                0x9fc01300                __vector_dispatch_8
                0x00000001                ASSERT (((_vector_spacing == 0x0) || (SIZEOF (.vector_8) <= (_vector_spacing << 0x5))), function at exception vector 8 too large)

.vector_9       0x9fc01320        0x8
 *(.vector_9)
 .vector_9      0x9fc01320        0x8 c:/program files (x86)/microchip/xc32/v1.21/bin/../lib/gcc/pic32mx/4.5.2/../../../../pic32mx/lib/size\libpic32.a(vector9.o)
                0x9fc01320                __vector_dispatch_9
                0x00000001                ASSERT (((_vector_spacing == 0x0) || (SIZEOF (.vector_9) <= (_vector_spacing << 0x5))), function at exception vector 9 too large)

.vector_10      0x9fc01340        0x8
 *(.vector_10)
 .vector_10     0x9fc01340        0x8 c:/program files (x86)/microchip/xc32/v1.21/bin/../lib/gcc/pic32mx/4.5.2/../../../../pic32mx/lib/size\libpic32.a(vector10.o)
                0x9fc01340                __vector_dispatch_10
                0x00000001                ASSERT (((_vector_spacing == 0x0) || (SIZEOF (.vector_10) <= (_vector_spacing << 0x5))), function at exception vector 10 too large)

.vector_11      0x9fc01360        0x8
 *(.vector_11)
 .vector_11     0x9fc01360        0x8 c:/program files (x86)/microchip/xc32/v1.21/bin/../lib/gcc/pic32mx/4.5.2/../../../../pic32mx/lib/size\libpic32.a(vector11.o)
                0x9fc01360                __vector_dispatch_11
                0x00000001                ASSERT (((_vector_spacing == 0x0) || (SIZEOF (.vector_11) <= (_vector_spacing << 0x5))), function at exception vector 11 too large)

.vector_12      0x9fc01380        0x8
 *(.vector_12)
 .vector_12     0x9fc01380        0x8 c:/program files (x86)/microchip/xc32/v1.21/bin/../lib/gcc/pic32mx/4.5.2/../../../../pic32mx/lib/size\libpic32.a(vector12.o)
                0x9fc01380                __vector_dispatch_12
                0x00000001                ASSERT (((_vector_spacing == 0x0) || (SIZEOF (.vector_12) <= (_vector_spacing << 0x5))), function at exception vector 12 too large)

.vector_13      0x9fc013a0        0x8
 *(.vector_13)
 .vector_13     0x9fc013a0        0x8 c:/program files (x86)/microchip/xc32/v1.21/bin/../lib/gcc/pic32mx/4.5.2/../../../../pic32mx/lib/size\libpic32.a(vector13.o)
                0x9fc013a0                __vector_dispatch_13
                0x00000001                ASSERT (((_vector_spacing == 0x0) || (SIZEOF (.vector_13) <= (_vector_spacing << 0x5))), function at exception vector 13 too large)

.vector_14      0x9fc013c0        0x8
 *(.vector_14)
 .vector_14     0x9fc013c0        0x8 c:/program files (x86)/microchip/xc32/v1.21/bin/../lib/gcc/pic32mx/4.5.2/../../../../pic32mx/lib/size\libpic32.a(vector14.o)
                0x9fc013c0                __vector_dispatch_14
                0x00000001                ASSERT (((_vector_spacing == 0x0) || (SIZEOF (.vector_14) <= (_vector_spacing << 0x5))), function at exception vector 14 too large)

.vector_15      0x9fc013e0        0x8
 *(.vector_15)
 .vector_15     0x9fc013e0        0x8 build/WiFIG/production/_ext/365611741/system_services.o
                0x9fc013e0                __vector_dispatch_15
                0x00000001                ASSERT (((_vector_spacing == 0x0) || (SIZEOF (.vector_15) <= (_vector_spacing << 0x5))), function at exception vector 15 too large)

.vector_16      0x9fc01400        0x8
 *(.vector_16)
 .vector_16     0x9fc01400        0x8 c:/program files (x86)/microchip/xc32/v1.21/bin/../lib/gcc/pic32mx/4.5.2/../../../../pic32mx/lib/size\libpic32.a(vector16.o)
                0x9fc01400                __vector_dispatch_16
                0x00000001                ASSERT (((_vector_spacing == 0x0) || (SIZEOF (.vector_16) <= (_vector_spacing << 0x5))), function at exception vector 16 too large)

.vector_17      0x9fc01420        0x8
 *(.vector_17)
 .vector_17     0x9fc01420        0x8 c:/program files (x86)/microchip/xc32/v1.21/bin/../lib/gcc/pic32mx/4.5.2/../../../../pic32mx/lib/size\libpic32.a(vector17.o)
                0x9fc01420                __vector_dispatch_17
                0x00000001                ASSERT (((_vector_spacing == 0x0) || (SIZEOF (.vector_17) <= (_vector_spacing << 0x5))), function at exception vector 17 too large)

.vector_18      0x9fc01440        0x8
 *(.vector_18)
 .vector_18     0x9fc01440        0x8 c:/program files (x86)/microchip/xc32/v1.21/bin/../lib/gcc/pic32mx/4.5.2/../../../../pic32mx/lib/size\libpic32.a(vector18.o)
                0x9fc01440                __vector_dispatch_18
                0x00000001                ASSERT (((_vector_spacing == 0x0) || (SIZEOF (.vector_18) <= (_vector_spacing << 0x5))), function at exception vector 18 too large)

.vector_19      0x9fc01460        0x8
 *(.vector_19)
 .vector_19     0x9fc01460        0x8 c:/program files (x86)/microchip/xc32/v1.21/bin/../lib/gcc/pic32mx/4.5.2/../../../../pic32mx/lib/size\libpic32.a(vector19.o)
                0x9fc01460                __vector_dispatch_19
                0x00000001                ASSERT (((_vector_spacing == 0x0) || (SIZEOF (.vector_19) <= (_vector_spacing << 0x5))), function at exception vector 19 too large)

.vector_20      0x9fc01480        0x8
 *(.vector_20)
 .vector_20     0x9fc01480        0x8 c:/program files (x86)/microchip/xc32/v1.21/bin/../lib/gcc/pic32mx/4.5.2/../../../../pic32mx/lib/size\libpic32.a(vector20.o)
                0x9fc01480                __vector_dispatch_20
                0x00000001                ASSERT (((_vector_spacing == 0x0) || (SIZEOF (.vector_20) <= (_vector_spacing << 0x5))), function at exception vector 20 too large)

.vector_21      0x9fc014a0        0x8
 *(.vector_21)
 .vector_21     0x9fc014a0        0x8 c:/program files (x86)/microchip/xc32/v1.21/bin/../lib/gcc/pic32mx/4.5.2/../../../../pic32mx/lib/size\libpic32.a(vector21.o)
                0x9fc014a0                __vector_dispatch_21
                0x00000001                ASSERT (((_vector_spacing == 0x0) || (SIZEOF (.vector_21) <= (_vector_spacing << 0x5))), function at exception vector 21 too large)

.vector_22      0x9fc014c0        0x8
 *(.vector_22)
 .vector_22     0x9fc014c0        0x8 c:/program files (x86)/microchip/xc32/v1.21/bin/../lib/gcc/pic32mx/4.5.2/../../../../pic32mx/lib/size\libpic32.a(vector22.o)
                0x9fc014c0                __vector_dispatch_22
                0x00000001                ASSERT (((_vector_spacing == 0x0) || (SIZEOF (.vector_22) <= (_vector_spacing << 0x5))), function at exception vector 22 too large)

.vector_23      0x9fc014e0        0x8
 *(.vector_23)
 .vector_23     0x9fc014e0        0x8 c:/program files (x86)/microchip/xc32/v1.21/bin/../lib/gcc/pic32mx/4.5.2/../../../../pic32mx/lib/size\libpic32.a(vector23.o)
                0x9fc014e0                __vector_dispatch_23
                0x00000001                ASSERT (((_vector_spacing == 0x0) || (SIZEOF (.vector_23) <= (_vector_spacing << 0x5))), function at exception vector 23 too large)

.vector_24      0x9fc01500        0x8
 *(.vector_24)
 .vector_24     0x9fc01500        0x8 c:/program files (x86)/microchip/xc32/v1.21/bin/../lib/gcc/pic32mx/4.5.2/../../../../pic32mx/lib/size\libpic32.a(vector24.o)
                0x9fc01500                __vector_dispatch_24
                0x00000001                ASSERT (((_vector_spacing == 0x0) || (SIZEOF (.vector_24) <= (_vector_spacing << 0x5))), function at exception vector 24 too large)

.vector_25      0x9fc01520        0x8
 *(.vector_25)
 .vector_25     0x9fc01520        0x8 c:/program files (x86)/microchip/xc32/v1.21/bin/../lib/gcc/pic32mx/4.5.2/../../../../pic32mx/lib/size\libpic32.a(vector25.o)
                0x9fc01520                __vector_dispatch_25
                0x00000001                ASSERT (((_vector_spacing == 0x0) || (SIZEOF (.vector_25) <= (_vector_spacing << 0x5))), function at exception vector 25 too large)

.vector_26      0x9fc01540        0x8
 *(.vector_26)
 .vector_26     0x9fc01540        0x8 build/WiFIG/production/_ext/365611741/system_services.o
                0x9fc01540                __vector_dispatch_26
                0x00000001                ASSERT (((_vector_spacing == 0x0) || (SIZEOF (.vector_26) <= (_vector_spacing << 0x5))), function at exception vector 26 too large)

.vector_27      0x9fc01560        0x8
 *(.vector_27)
 .vector_27     0x9fc01560        0x8 c:/program files (x86)/microchip/xc32/v1.21/bin/../lib/gcc/pic32mx/4.5.2/../../../../pic32mx/lib/size\libpic32.a(vector27.o)
                0x9fc01560                __vector_dispatch_27
                0x00000001                ASSERT (((_vector_spacing == 0x0) || (SIZEOF (.vector_27) <= (_vector_spacing << 0x5))), function at exception vector 27 too large)

.vector_28      0x9fc01580        0x8
 *(.vector_28)
 .vector_28     0x9fc01580        0x8 c:/program files (x86)/microchip/xc32/v1.21/bin/../lib/gcc/pic32mx/4.5.2/../../../../pic32mx/lib/size\libpic32.a(vector28.o)
                0x9fc01580                __vector_dispatch_28
                0x00000001                ASSERT (((_vector_spacing == 0x0) || (SIZEOF (.vector_28) <= (_vector_spacing << 0x5))), function at exception vector 28 too large)

.vector_29      0x9fc015a0        0x8
 *(.vector_29)
 .vector_29     0x9fc015a0        0x8 c:/program files (x86)/microchip/xc32/v1.21/bin/../lib/gcc/pic32mx/4.5.2/../../../../pic32mx/lib/size\libpic32.a(vector29.o)
                0x9fc015a0                __vector_dispatch_29
                0x00000001                ASSERT (((_vector_spacing == 0x0) || (SIZEOF (.vector_29) <= (_vector_spacing << 0x5))), function at exception vector 29 too large)

.vector_30      0x9fc015c0        0x8
 *(.vector_30)
 .vector_30     0x9fc015c0        0x8 c:/program files (x86)/microchip/xc32/v1.21/bin/../lib/gcc/pic32mx/4.5.2/../../../../pic32mx/lib/size\libpic32.a(vector30.o)
                0x9fc015c0                __vector_dispatch_30
                0x00000001                ASSERT (((_vector_spacing == 0x0) || (SIZEOF (.vector_30) <= (_vector_spacing << 0x5))), function at exception vector 30 too large)

.vector_31      0x9fc015e0        0x8
 *(.vector_31)
 .vector_31     0x9fc015e0        0x8 c:/program files (x86)/microchip/xc32/v1.21/bin/../lib/gcc/pic32mx/4.5.2/../../../../pic32mx/lib/size\libpic32.a(vector31.o)
                0x9fc015e0                __vector_dispatch_31
                0x00000001                ASSERT (((_vector_spacing == 0x0) || (SIZEOF (.vector_31) <= (_vector_spacing << 0x5))), function at exception vector 31 too large)

.vector_32      0x9fc01600        0x8
 *(.vector_32)
 .vector_32     0x9fc01600        0x8 c:/program files (x86)/microchip/xc32/v1.21/bin/../lib/gcc/pic32mx/4.5.2/../../../../pic32mx/lib/size\libpic32.a(vector32.o)
                0x9fc01600                __vector_dispatch_32
                0x00000001                ASSERT (((_vector_spacing == 0x0) || (SIZEOF (.vector_32) <= (_vector_spacing << 0x5))), function at exception vector 32 too large)

.vector_33      0x9fc01620        0x8
 *(.vector_33)
 .vector_33     0x9fc01620        0x8 c:/program files (x86)/microchip/xc32/v1.21/bin/../lib/gcc/pic32mx/4.5.2/../../../../pic32mx/lib/size\libpic32.a(vector33.o)
                0x9fc01620                __vector_dispatch_33
                0x00000001                ASSERT (((_vector_spacing == 0x0) || (SIZEOF (.vector_33) <= (_vector_spacing << 0x5))), function at exception vector 33 too large)

.vector_34      0x9fc01640        0x8
 *(.vector_34)
 .vector_34     0x9fc01640        0x8 c:/program files (x86)/microchip/xc32/v1.21/bin/../lib/gcc/pic32mx/4.5.2/../../../../pic32mx/lib/size\libpic32.a(vector34.o)
                0x9fc01640                __vector_dispatch_34
                0x00000001                ASSERT (((_vector_spacing == 0x0) || (SIZEOF (.vector_34) <= (_vector_spacing << 0x5))), function at exception vector 34 too large)

.vector_35      0x9fc01660        0x8
 *(.vector_35)
 .vector_35     0x9fc01660        0x8 c:/program files (x86)/microchip/xc32/v1.21/bin/../lib/gcc/pic32mx/4.5.2/../../../../pic32mx/lib/size\libpic32.a(vector35.o)
                0x9fc01660                __vector_dispatch_35
                0x00000001                ASSERT (((_vector_spacing == 0x0) || (SIZEOF (.vector_35) <= (_vector_spacing << 0x5))), function at exception vector 35 too large)

.vector_36      0x9fc01680        0x8
 *(.vector_36)
 .vector_36     0x9fc01680        0x8 c:/program files (x86)/microchip/xc32/v1.21/bin/../lib/gcc/pic32mx/4.5.2/../../../../pic32mx/lib/size\libpic32.a(vector36.o)
                0x9fc01680                __vector_dispatch_36
                0x00000001                ASSERT (((_vector_spacing == 0x0) || (SIZEOF (.vector_36) <= (_vector_spacing << 0x5))), function at exception vector 36 too large)

.vector_37      0x9fc016a0        0x8
 *(.vector_37)
 .vector_37     0x9fc016a0        0x8 c:/program files (x86)/microchip/xc32/v1.21/bin/../lib/gcc/pic32mx/4.5.2/../../../../pic32mx/lib/size\libpic32.a(vector37.o)
                0x9fc016a0                __vector_dispatch_37
                0x00000001                ASSERT (((_vector_spacing == 0x0) || (SIZEOF (.vector_37) <= (_vector_spacing << 0x5))), function at exception vector 37 too large)

.vector_38      0x9fc016c0        0x8
 *(.vector_38)
 .vector_38     0x9fc016c0        0x8 c:/program files (x86)/microchip/xc32/v1.21/bin/../lib/gcc/pic32mx/4.5.2/../../../../pic32mx/lib/size\libpic32.a(vector38.o)
                0x9fc016c0                __vector_dispatch_38
                0x00000001                ASSERT (((_vector_spacing == 0x0) || (SIZEOF (.vector_38) <= (_vector_spacing << 0x5))), function at exception vector 38 too large)

.vector_39      0x9fc016e0        0x8
 *(.vector_39)
 .vector_39     0x9fc016e0        0x8 c:/program files (x86)/microchip/xc32/v1.21/bin/../lib/gcc/pic32mx/4.5.2/../../../../pic32mx/lib/size\libpic32.a(vector39.o)
                0x9fc016e0                __vector_dispatch_39
                0x00000001                ASSERT (((_vector_spacing == 0x0) || (SIZEOF (.vector_39) <= (_vector_spacing << 0x5))), function at exception vector 39 too large)

.vector_40      0x9fc01700        0x8
 *(.vector_40)
 .vector_40     0x9fc01700        0x8 c:/program files (x86)/microchip/xc32/v1.21/bin/../lib/gcc/pic32mx/4.5.2/../../../../pic32mx/lib/size\libpic32.a(vector40.o)
                0x9fc01700                __vector_dispatch_40
                0x00000001                ASSERT (((_vector_spacing == 0x0) || (SIZEOF (.vector_40) <= (_vector_spacing << 0x5))), function at exception vector 40 too large)

.vector_41      0x9fc01720        0x8
 *(.vector_41)
 .vector_41     0x9fc01720        0x8 c:/program files (x86)/microchip/xc32/v1.21/bin/../lib/gcc/pic32mx/4.5.2/../../../../pic32mx/lib/size\libpic32.a(vector41.o)
                0x9fc01720                __vector_dispatch_41
                0x00000001                ASSERT (((_vector_spacing == 0x0) || (SIZEOF (.vector_41) <= (_vector_spacing << 0x5))), function at exception vector 41 too large)

.vector_42      0x9fc01740        0x8
 *(.vector_42)
 .vector_42     0x9fc01740        0x8 c:/program files (x86)/microchip/xc32/v1.21/bin/../lib/gcc/pic32mx/4.5.2/../../../../pic32mx/lib/size\libpic32.a(vector42.o)
                0x9fc01740                __vector_dispatch_42
                0x00000001                ASSERT (((_vector_spacing == 0x0) || (SIZEOF (.vector_42) <= (_vector_spacing << 0x5))), function at exception vector 42 too large)

.vector_43      0x9fc01760        0x8
 *(.vector_43)
 .vector_43     0x9fc01760        0x8 c:/program files (x86)/microchip/xc32/v1.21/bin/../lib/gcc/pic32mx/4.5.2/../../../../pic32mx/lib/size\libpic32.a(vector43.o)
                0x9fc01760                __vector_dispatch_43
                0x00000001                ASSERT (((_vector_spacing == 0x0) || (SIZEOF (.vector_43) <= (_vector_spacing << 0x5))), function at exception vector 43 too large)

.vector_44      0x9fc01780        0x8
 *(.vector_44)
 .vector_44     0x9fc01780        0x8 c:/program files (x86)/microchip/xc32/v1.21/bin/../lib/gcc/pic32mx/4.5.2/../../../../pic32mx/lib/size\libpic32.a(vector44.o)
                0x9fc01780                __vector_dispatch_44
                0x00000001                ASSERT (((_vector_spacing == 0x0) || (SIZEOF (.vector_44) <= (_vector_spacing << 0x5))), function at exception vector 44 too large)

.vector_45      0x9fc017a0        0x8
 *(.vector_45)
 .vector_45     0x9fc017a0        0x8 c:/program files (x86)/microchip/xc32/v1.21/bin/../lib/gcc/pic32mx/4.5.2/../../../../pic32mx/lib/size\libpic32.a(vector45.o)
                0x9fc017a0                __vector_dispatch_45
                0x00000001                ASSERT (((_vector_spacing == 0x0) || (SIZEOF (.vector_45) <= (_vector_spacing << 0x5))), function at exception vector 45 too large)

.vector_46      0x9fc017c0        0x8
 *(.vector_46)
 .vector_46     0x9fc017c0        0x8 c:/program files (x86)/microchip/xc32/v1.21/bin/../lib/gcc/pic32mx/4.5.2/../../../../pic32mx/lib/size\libpic32.a(vector46.o)
                0x9fc017c0                __vector_dispatch_46
                0x00000001                ASSERT (((_vector_spacing == 0x0) || (SIZEOF (.vector_46) <= (_vector_spacing << 0x5))), function at exception vector 46 too large)

.vector_47      0x9fc017e0        0x8
 *(.vector_47)
 .vector_47     0x9fc017e0        0x8 c:/program files (x86)/microchip/xc32/v1.21/bin/../lib/gcc/pic32mx/4.5.2/../../../../pic32mx/lib/size\libpic32.a(vector47.o)
                0x9fc017e0                __vector_dispatch_47
                0x00000001                ASSERT (((_vector_spacing == 0x0) || (SIZEOF (.vector_47) <= (_vector_spacing << 0x5))), function at exception vector 47 too large)

.vector_48      0x9fc01800        0x8
 *(.vector_48)
 .vector_48     0x9fc01800        0x8 c:/program files (x86)/microchip/xc32/v1.21/bin/../lib/gcc/pic32mx/4.5.2/../../../../pic32mx/lib/size\libpic32.a(vector48.o)
                0x9fc01800                __vector_dispatch_48
                0x00000001                ASSERT (((_vector_spacing == 0x0) || (SIZEOF (.vector_48) <= (_vector_spacing << 0x5))), function at exception vector 48 too large)

.vector_49      0x9fc01820        0x8
 *(.vector_49)
 .vector_49     0x9fc01820        0x8 c:/program files (x86)/microchip/xc32/v1.21/bin/../lib/gcc/pic32mx/4.5.2/../../../../pic32mx/lib/size\libpic32.a(vector49.o)
                0x9fc01820                __vector_dispatch_49
                0x00000001                ASSERT (((_vector_spacing == 0x0) || (SIZEOF (.vector_49) <= (_vector_spacing << 0x5))), function at exception vector 49 too large)

.vector_50      0x9fc01840        0x8
 *(.vector_50)
 .vector_50     0x9fc01840        0x8 c:/program files (x86)/microchip/xc32/v1.21/bin/../lib/gcc/pic32mx/4.5.2/../../../../pic32mx/lib/size\libpic32.a(vector50.o)
                0x9fc01840                __vector_dispatch_50
                0x00000001                ASSERT (((_vector_spacing == 0x0) || (SIZEOF (.vector_50) <= (_vector_spacing << 0x5))), function at exception vector 50 too large)

.vector_51      0x9fc01860        0x8
 *(.vector_51)
 .vector_51     0x9fc01860        0x8 c:/program files (x86)/microchip/xc32/v1.21/bin/../lib/gcc/pic32mx/4.5.2/../../../../pic32mx/lib/size\libpic32.a(vector51.o)
                0x9fc01860                __vector_dispatch_51
                0x00000001                ASSERT (((_vector_spacing == 0x0) || (SIZEOF (.vector_51) <= (_vector_spacing << 0x5))), function at exception vector 51 too large)

.vector_52      0x9fc01880        0x8
 *(.vector_52)
 .vector_52     0x9fc01880        0x8 c:/program files (x86)/microchip/xc32/v1.21/bin/../lib/gcc/pic32mx/4.5.2/../../../../pic32mx/lib/size\libpic32.a(vector52.o)
                0x9fc01880                __vector_dispatch_52
                0x00000001                ASSERT (((_vector_spacing == 0x0) || (SIZEOF (.vector_52) <= (_vector_spacing << 0x5))), function at exception vector 52 too large)

.vector_53      0x9fc018a0        0x8
 *(.vector_53)
 .vector_53     0x9fc018a0        0x8 c:/program files (x86)/microchip/xc32/v1.21/bin/../lib/gcc/pic32mx/4.5.2/../../../../pic32mx/lib/size\libpic32.a(vector53.o)
                0x9fc018a0                __vector_dispatch_53
                0x00000001                ASSERT (((_vector_spacing == 0x0) || (SIZEOF (.vector_53) <= (_vector_spacing << 0x5))), function at exception vector 53 too large)

.vector_54      0x9fc018c0        0x8
 *(.vector_54)
 .vector_54     0x9fc018c0        0x8 c:/program files (x86)/microchip/xc32/v1.21/bin/../lib/gcc/pic32mx/4.5.2/../../../../pic32mx/lib/size\libpic32.a(vector54.o)
                0x9fc018c0                __vector_dispatch_54
                0x00000001                ASSERT (((_vector_spacing == 0x0) || (SIZEOF (.vector_54) <= (_vector_spacing << 0x5))), function at exception vector 54 too large)

.vector_55      0x9fc018e0        0x8
 *(.vector_55)
 .vector_55     0x9fc018e0        0x8 c:/program files (x86)/microchip/xc32/v1.21/bin/../lib/gcc/pic32mx/4.5.2/../../../../pic32mx/lib/size\libpic32.a(vector55.o)
                0x9fc018e0                __vector_dispatch_55
                0x00000001                ASSERT (((_vector_spacing == 0x0) || (SIZEOF (.vector_55) <= (_vector_spacing << 0x5))), function at exception vector 55 too large)

.vector_56      0x9fc01900        0x8
 *(.vector_56)
 .vector_56     0x9fc01900        0x8 c:/program files (x86)/microchip/xc32/v1.21/bin/../lib/gcc/pic32mx/4.5.2/../../../../pic32mx/lib/size\libpic32.a(vector56.o)
                0x9fc01900                __vector_dispatch_56
                0x00000001                ASSERT (((_vector_spacing == 0x0) || (SIZEOF (.vector_56) <= (_vector_spacing << 0x5))), function at exception vector 56 too large)

.vector_57      0x9fc01920        0x8
 *(.vector_57)
 .vector_57     0x9fc01920        0x8 c:/program files (x86)/microchip/xc32/v1.21/bin/../lib/gcc/pic32mx/4.5.2/../../../../pic32mx/lib/size\libpic32.a(vector57.o)
                0x9fc01920                __vector_dispatch_57
                0x00000001                ASSERT (((_vector_spacing == 0x0) || (SIZEOF (.vector_57) <= (_vector_spacing << 0x5))), function at exception vector 57 too large)

.vector_58      0x9fc01940        0x8
 *(.vector_58)
 .vector_58     0x9fc01940        0x8 c:/program files (x86)/microchip/xc32/v1.21/bin/../lib/gcc/pic32mx/4.5.2/../../../../pic32mx/lib/size\libpic32.a(vector58.o)
                0x9fc01940                __vector_dispatch_58
                0x00000001                ASSERT (((_vector_spacing == 0x0) || (SIZEOF (.vector_58) <= (_vector_spacing << 0x5))), function at exception vector 58 too large)

.vector_59      0x9fc01960        0x8
 *(.vector_59)
 .vector_59     0x9fc01960        0x8 c:/program files (x86)/microchip/xc32/v1.21/bin/../lib/gcc/pic32mx/4.5.2/../../../../pic32mx/lib/size\libpic32.a(vector59.o)
                0x9fc01960                __vector_dispatch_59
                0x00000001                ASSERT (((_vector_spacing == 0x0) || (SIZEOF (.vector_59) <= (_vector_spacing << 0x5))), function at exception vector 59 too large)

.vector_60      0x9fc01980        0x8
 *(.vector_60)
 .vector_60     0x9fc01980        0x8 c:/program files (x86)/microchip/xc32/v1.21/bin/../lib/gcc/pic32mx/4.5.2/../../../../pic32mx/lib/size\libpic32.a(vector60.o)
                0x9fc01980                __vector_dispatch_60
                0x00000001                ASSERT (((_vector_spacing == 0x0) || (SIZEOF (.vector_60) <= (_vector_spacing << 0x5))), function at exception vector 60 too large)

.vector_61      0x9fc019a0        0x8
 *(.vector_61)
 .vector_61     0x9fc019a0        0x8 c:/program files (x86)/microchip/xc32/v1.21/bin/../lib/gcc/pic32mx/4.5.2/../../../../pic32mx/lib/size\libpic32.a(vector61.o)
                0x9fc019a0                __vector_dispatch_61
                0x00000001                ASSERT (((_vector_spacing == 0x0) || (SIZEOF (.vector_61) <= (_vector_spacing << 0x5))), function at exception vector 61 too large)

.vector_62      0x9fc019c0        0x8
 *(.vector_62)
 .vector_62     0x9fc019c0        0x8 c:/program files (x86)/microchip/xc32/v1.21/bin/../lib/gcc/pic32mx/4.5.2/../../../../pic32mx/lib/size\libpic32.a(vector62.o)
                0x9fc019c0                __vector_dispatch_62
                0x00000001                ASSERT (((_vector_spacing == 0x0) || (SIZEOF (.vector_62) <= (_vector_spacing << 0x5))), function at exception vector 62 too large)

.vector_63      0x9fc019e0        0x8
 *(.vector_63)
 .vector_63     0x9fc019e0        0x8 c:/program files (x86)/microchip/xc32/v1.21/bin/../lib/gcc/pic32mx/4.5.2/../../../../pic32mx/lib/size\libpic32.a(vector63.o)
                0x9fc019e0                __vector_dispatch_63
                0x00000001                ASSERT (((_vector_spacing == 0x0) || (SIZEOF (.vector_63) <= (_vector_spacing << 0x5))), function at exception vector 63 too large)

.startup
 *(.startup)

.text           0x9d000000        0x0
 *(.stub .gnu.linkonce.t.*)
 *(.text.*personality*)
 *(.mips16.fn.*)
 *(.mips16.call.*)
 *(.gnu.warning)
                0x9d000000                . = ALIGN (0x4)

.init           0x9d000000        0x0
 *crti.o(.init)
 *crtbegin.o(.init)
 *(EXCLUDE_FILE(*crtn.o *crtend?.o *crtend.o) .init)
 *crtend.o(.init)
 *crtn.o(.init)
                0x9d000000                . = ALIGN (0x4)

.fini           0x9d000000        0x0
 *(.fini)
                0x9d000000                . = ALIGN (0x4)

.preinit_array  0x9d000000        0x0
                0x9d000000                PROVIDE (__preinit_array_start, .)
 *(.preinit_array)
                0x9d000000                PROVIDE (__preinit_array_end, .)
                0x9d000000                . = ALIGN (0x4)

.init_array     0x9d000000        0x0
                0x9d000000                PROVIDE (__init_array_start, .)
 *(SORT(.init_array.*))
 *(.init_array)
                0x9d000000                PROVIDE (__init_array_end, .)
                0x9d000000                . = ALIGN (0x4)

.fini_array     0x9d000000        0x0
                0x9d000000                PROVIDE (__fini_array_start, .)
 *(SORT(.fini_array.*))
 *(.fini_array)
                0x9d000000                PROVIDE (__fini_array_end, .)
                0x9d000000                . = ALIGN (0x4)

.ctors          0x9d000000        0x0
 *crtbegin.o(.ctors)
 *crtbegin?.o(.ctors)
 *(EXCLUDE_FILE(*crtend?.o *crtend.o) .ctors)
 *(SORT(.ctors.*))
 *(.ctors)
                0x9d000000                . = ALIGN (0x4)

.dtors          0x9d000000        0x0
 *crtbegin.o(.dtors)
 *crtbegin?.o(.dtors)
 *(EXCLUDE_FILE(*crtend?.o *crtend.o) .dtors)
 *(SORT(.dtors.*))
 *(.dtors)
                0x9d000000                . = ALIGN (0x4)

.rodata         0x9d000000        0x0
 *(.gnu.linkonce.r.*)
 *(.rodata1)
                0x9d000000                . = ALIGN (0x4)

.sdata2         0x9fc00490        0x0
 *(.sdata2 .sdata2.* .gnu.linkonce.s2.*)
                0x9fc00490                . = ALIGN (0x4)

.sbss2          0x9fc00490        0x0
 *(.sbss2 .sbss2.* .gnu.linkonce.sb2.*)
                0x9fc00490                . = ALIGN (0x4)

.eh_frame_hdr
 *(.eh_frame_hdr)
                0x9fc00490                . = ALIGN (0x4)

.eh_frame
 *(.eh_frame)
                0x9fc00490                . = ALIGN (0x4)

.gcc_except_table
 *(.gcc_except_table .gcc_except_table.*)
                0x9fc00490                . = ALIGN (0x4)

.dbg_data       0xa0000000        0x0
                0xa0000000                . = (. + DEFINED (_DEBUGGER)?0x200:0x0)

.jcr            0xa0000000        0x0
 *(.jcr)
                0xa0000000                . = ALIGN (0x4)

.eh_frame       0xa0000000       0x30
 *(.eh_frame)
 .eh_frame      0xa0000000       0x20 c:/program files (x86)/microchip/xc32/v1.21/bin/../lib/gcc/pic32mx/4.5.2/size\libgcc.a(_udivdi3.o)
 .eh_frame      0xa0000020       0x10 c:/program files (x86)/microchip/xc32/v1.21/bin/../lib/gcc/pic32mx/4.5.2/size\libgcc.a(_umoddi3.o)
                0xa0000030                . = ALIGN (0x4)

.gcc_except_table
 *(.gcc_except_table .gcc_except_table.*)
                0xa0000030                . = ALIGN (0x4)

.persist        0xa0000030        0x0
                0xa0000030                _persist_begin = .
 *(.persist .persist.*)
 *(.pbss .pbss.*)
                0xa0000030                . = ALIGN (0x4)
                0xa0000030                _persist_end = .

.data           0xa0000030        0x0
 *(.gnu.linkonce.d.*)
 *(.data1)
                0xa0000030                . = ALIGN (0x4)
                0xa0000030                . = .
                0xa0008020                _gp = (ALIGN (0x10) + 0x7ff0)

.got            0xa0000030        0x0
 *(.got.plt)
 *(.got)
                0xa0000030                . = ALIGN (0x4)

.sdata          0xa0000030      0x1bc
                0xa0000030                _sdata_begin = .
 *(.sdata .sdata.* .gnu.linkonce.s.*)
 .sdata         0xa0000030        0x4 build/WiFIG/production/_ext/101875047/lfsr.o
 .sdata         0xa0000034       0x10 build/WiFIG/production/_ext/365611741/system_services.o
                0xa0000034                MEDIA_STORAGE_PARTITION_TABLE
 .sdata         0xa0000044       0x60 build/WiFIG/production/_ext/365611741/system_debug.o
 .sdata         0xa00000a4       0x1c build/WiFIG/production/_ext/792872985/usart.o
                0xa00000a4                _usart_cdev_obj
 .sdata         0xa00000c0        0x8 build/WiFIG/production/_ext/427700826/arp.o
 .sdata         0xa00000c8        0x2 build/WiFIG/production/_ext/427700826/dns.o
 *fill*         0xa00000ca        0x2 00
 .sdata         0xa00000cc        0x4 build/WiFIG/production/_ext/427700826/tcpip_heap_alloc.o
 .sdata         0xa00000d0        0x1 build/WiFIG/production/_ext/334706090/wf_connection_algorithm.o
 .sdata         0xa00000d1        0x1 build/WiFIG/production/_ext/334706090/wf_power_save.o
 *fill*         0xa00000d2        0x2 00
 .sdata         0xa00000d4        0xc build/WiFIG/production/_ext/334706090/mrf24w_mac_pic32.o
 .sdata         0xa00000e0      0x100 build/WiFIG/production/_ext/334706090/wf_debug_output.o
                0xa00000e0                connectionLostStrings
                0xa00000f8                wpsState
                0xa0000134                wpsConfigErr
 .sdata         0xa00001e0        0x4 build/WiFIG/production/_ext/334706090/wf_configData.o
                0xa00001e0                p_wifi_ConfigData
 .sdata         0xa00001e4        0x2 build/WiFIG/production/_ext/1472/tcp6_demo_app.o
                0xa00001e4                mySocket
 *fill*         0xa00001e6        0x2 00
 .sdata         0xa00001e8        0x4 c:/program files (x86)/microchip/xc32/v1.21/bin/../lib/gcc/pic32mx/4.5.2/../../../../pic32mx/lib/size\libpic32.a(xc32_uart.o)
                0xa00001e8                __XC_UART
                0xa00001ec                . = ALIGN (0x4)
                0xa00001ec                _sdata_end = .

.lit8
 *(.lit8)

.lit4
 *(.lit4)
                0xa00001ec                . = ALIGN (0x4)
                0xa00001ec                _data_end = .
                0xa00001ec                _bss_begin = .

.sbss           0xa00001ec      0x310
                0xa00001ec                _sbss_begin = .
 *(.dynsbss)
 *(.sbss .sbss.* .gnu.linkonce.sb.*)
 .sbss          0xa00001ec       0x34 build/WiFIG/production/_ext/365611741/system_services.o
                0xa00001ec                _SystemTickCount
                0xa00001f0                _SystemTickResolution
 .sbss          0xa0000220        0x8 build/WiFIG/production/_ext/365611741/system_debug.o
 .sbss          0xa0000228       0x18 build/WiFIG/production/_ext/365611741/system_random.o
 .sbss          0xa0000240       0x30 build/WiFIG/production/_ext/365611741/system_userio.o
 .sbss          0xa0000270       0x1c build/WiFIG/production/_ext/427700826/tcpip_announce.o
 .sbss          0xa000028c       0x3c build/WiFIG/production/_ext/427700826/arp.o
 .sbss          0xa00002c8       0x20 build/WiFIG/production/_ext/427700826/dhcp.o
 .sbss          0xa00002e8       0x3c build/WiFIG/production/_ext/427700826/dns.o
 .sbss          0xa0000324        0x8 build/WiFIG/production/_ext/427700826/icmp.o
 .sbss          0xa000032c       0x20 build/WiFIG/production/_ext/427700826/ipv4.o
                0xa000033c                ipv4QueuedPackets
 .sbss          0xa000034c        0xc build/WiFIG/production/_ext/427700826/nbns.o
 .sbss          0xa0000358       0x20 build/WiFIG/production/_ext/427700826/tcp.o
 .sbss          0xa0000378       0x18 build/WiFIG/production/_ext/427700826/udp.o
                0xa0000378                UDPSocketDcpt
 .sbss          0xa0000390       0x3c build/WiFIG/production/_ext/427700826/tcpip_manager.o
 .sbss          0xa00003cc        0x1 build/WiFIG/production/_ext/334706090/wf_connection_manager.o
 .sbss          0xa00003cd        0x1 build/WiFIG/production/_ext/334706090/wf_connection_profile.o
 .sbss          0xa00003ce        0x2 build/WiFIG/production/_ext/334706090/wf_event_handler.o
                0xa00003ce                g_DhcpRenew
                0xa00003cf                g_asyncTaskFlags
 .sbss          0xa00003d0        0x3 build/WiFIG/production/_ext/334706090/wf_power_save.o
 .sbss          0xa00003d3        0x1 build/WiFIG/production/_ext/334706090/wf_spi.o
 .sbss          0xa00003d4       0x18 build/WiFIG/production/_ext/334706090/mrf24w_events.o
 .sbss          0xa00003ec        0x1 build/WiFIG/production/_ext/334706090/wf_debug_output.o
                0xa00003ec                g_outputConnectionContext
 *fill*         0xa00003ed        0x3 00
 .sbss          0xa00003f0       0x14 build/WiFIG/production/_ext/334706090/wf_driver_com_24g.o
                0xa00003fd                g_DhcpSuccessful
                0xa00003fe                g_WiFiConnectionChanged
                0xa00003ff                g_WiFiConnection
                0xa0000400                g_dhcpInProgress
 .sbss          0xa0000404        0x2 build/WiFIG/production/_ext/334706090/wf_driver_raw_24g.o
                0xa0000404                g_HostRAWDataPacketReceived
                0xa0000405                g_RawIndexPastEnd
 *fill*         0xa0000406        0x2 00
 .sbss          0xa0000408        0xc build/WiFIG/production/_ext/334706090/wf_mac_24g.o
 .sbss          0xa0000414        0x3 build/WiFIG/production/_ext/334706090/wf_mgmt_msg_24g.o
                0xa0000415                g_WaitingForMgmtResponse
 *fill*         0xa0000417        0x1 00
 .sbss          0xa0000418       0x1c build/WiFIG/production/_ext/1472/main_demo.o
                0xa0000418                stackNotifyCnt
                0xa000041c                stackTotEvents
                0xa0000420                mrf_txEvents
                0xa0000422                mrf_txEventInfo
                0xa0000424                mrf_mgmtEvents
                0xa0000426                mrf_mgmtEventInfo
                0xa0000428                mrf_EventCnt
 .sbss          0xa0000434       0x18 build/WiFIG/production/_ext/1472/tcp6_demo_app.o
                0xa0000434                bWiFiConnected
                0xa0000438                nAttempts
                0xa000043c                httpTransactionIndex
                0xa0000440                WaitDispatch2Timer
                0xa0000444                WaitAssociate
                0xa0000448                smMyDemoAppTasks
 .sbss          0xa000044c       0x10 c:/program files (x86)/microchip/xc32/v1.21/bin/../lib/gcc/pic32mx/4.5.2/../../../../pic32mx/lib/size\libc.a(malloc.o)
                0xa000044c                __allocp
                0xa0000450                __alloct
                0xa0000454                __allocx
 .sbss          0xa000045c        0x4 c:/program files (x86)/microchip/xc32/v1.21/bin/../lib/gcc/pic32mx/4.5.2/../../../../pic32mx/lib/size\libc.a(errno.o)
                0xa000045c                errno
 .sbss          0xa0000460        0x1 c:/program files (x86)/microchip/xc32/v1.21/bin/../lib/gcc/pic32mx/4.5.2/../../../../pic32mx/lib/size\libc.a(_iob.o)
                0xa0000460                _outdone
 *fill*         0xa0000461        0x3 00
 .sbss          0xa0000464        0x8 c:/program files (x86)/microchip/xc32/v1.21/bin/../lib/gcc/pic32mx/4.5.2/../../../../pic32mx/lib/size\libpic32.a(sbrk.o)
                0xa0000464                _minbrk
                0xa0000468                _maxbrk
 *(.scommon)
 .scommon       0xa000046c       0x1c build/WiFIG/production/_ext/1472/ping_demo.o
                0xa000046c                pingTimer
                0xa0000470                targetHostName
                0xa0000474                targetMACAddr
                0xa000047a                pingCount
                0xa000047c                targetAddressIPv4
                0xa0000480                firstHopAddress
                0xa0000484                pNetIf
 .scommon       0xa0000488        0x8 build/WiFIG/production/_ext/334706090/wf_event_handler.o
                0xa0000488                g_softAPEvent
 .scommon       0xa0000490        0x6 build/WiFIG/production/_ext/334706090/wf_power_save.o
                0xa0000490                g_savedPsPollContext
 *fill*         0xa0000496        0x2 00
 .scommon       0xa0000498        0x4 build/WiFIG/production/_ext/334706090/wf_scan.o
                0xa0000498                hMac_softap_connect
 .scommon       0xa000049c        0x3 build/WiFIG/production/_ext/334706090/wf_commands.o
                0xa000049c                iwconfigCb
 *fill*         0xa000049f        0x1 00
 .scommon       0xa00004a0        0x3 build/WiFIG/production/_ext/334706090/wf_driver_com_24g.o
                0xa00004a0                RawMoveState
                0xa00004a2                g_powerSaveState
 *fill*         0xa00004a3        0x1 00
 .scommon       0xa00004a4        0x2 build/WiFIG/production/_ext/334706090/wf_driver_raw_24g.o
                0xa00004a4                RawWindowState
 *fill*         0xa00004a6        0x2 00
 .scommon       0xa00004a8       0x10 build/WiFIG/production/_ext/334706090/wf_mac_24g.o
                0xa00004a8                g_rxBufferLength
                0xa00004ac                g_pNetIf
                0xa00004b0                g_gratArpContext
 .scommon       0xa00004b8        0x4 build/WiFIG/production/_ext/1472/main_demo.o
                0xa00004b8                stackNotifyHandle
 .scommon       0xa00004bc       0x40 build/WiFIG/production/_ext/1472/tcp6_demo_app.o
                0xa00004bc                serverIP
                0xa00004c0                j
                0xa00004c4                TCPReadByte
                0xa00004c8                dnsRes
                0xa00004cc                mac_addr
                0xa00004d4                clientTimer
                0xa00004d8                myNetHandle
                0xa00004dc                i
                0xa00004e0                toggleLed
                0xa00004e4                TCPIsPutReadyCnt
                0xa00004e6                serverPort
                0xa00004e8                TCPInBufPtr
                0xa00004ec                TCPInBufferIndex
                0xa00004f0                HTTPReplyDelay
                0xa00004f4                HTTPReplyLineCnt
                0xa00004f8                mac_addr_ptr
                0xa00004fc                _sbss_end = .
                0xa00004fc                . = ALIGN (0x4)

.bss            0xa00004fc     0x1bc4
 *(.dynbss)
 *(COMMON)
 COMMON         0xa00004fc       0x40 build/WiFIG/production/_ext/101875047/hashes.o
                0xa00004fc                lastBlock
 COMMON         0xa000053c        0xa build/WiFIG/production/_ext/427700826/tcpip_manager.o
                0xa000053c                remoteNode
 *fill*         0xa0000546        0x2 00
 COMMON         0xa0000548       0x8a build/WiFIG/production/_ext/334706090/wf_configData.o
                0xa0000548                wifi_ConfigData
 *fill*         0xa00005d2        0x2 00
 COMMON         0xa00005d4     0x1aec build/WiFIG/production/_ext/1472/tcp6_demo_app.o
                0xa00005d4                httpTransaction
                0xa0000a84                TCPInBuffer
                0xa0001a84                mac_addr_string
                0xa0001a94                TCPOutBuffer
                0xa0001c94                mysrc
                0xa0001d14                myb64
                0xa0001d94                temp
                0xa0001de4                OutString
                0xa0001fe4                mySocketInfo
                0xa000200c                myResourceState
                0xa00020c0                . = ALIGN ((. != 0x0)?0x4:0x1)
                0xa00020c0                . = ALIGN (0x4)
                0xa00020c0                _end = .
                0xa00020c0                _bss_end = .
                0x00020000                _bmxdudba_address = 0x20000
                0x00020000                _bmxdupba_address = 0x20000

/DISCARD/
 *(.pdr)
 *(.rel.dyn)
 *(.note.GNU-stack)
 *(.note.GNU-stack)
 *(.gnu_debuglink)
 *(.gnu.lto_*)
 *(.discard)

.gptab.sdata
 *(.gptab.data)
 *(.gptab.sdata)

.gptab.sbss
 *(.gptab.bss)
 *(.gptab.sbss)

.mdebug.abi32   0xa00020c0        0x0
 *(.mdebug.abi32)
 .mdebug.abi32  0xa00020c0        0x0 build/WiFIG/production/_ext/1293749816/bsp.o
 .mdebug.abi32  0xa00020c0        0x0 build/WiFIG/production/_ext/101875047/hashes.o
 .mdebug.abi32  0xa00020c0        0x0 build/WiFIG/production/_ext/101875047/lfsr.o
 .mdebug.abi32  0xa00020c0        0x0 build/WiFIG/production/_ext/101875047/big_int.o
 .mdebug.abi32  0xa00020c0        0x0 build/WiFIG/production/_ext/101875047/helpers.o
 .mdebug.abi32  0xa00020c0        0x0 build/WiFIG/production/_ext/1472/berkeley_tcp_client_demo.o
 .mdebug.abi32  0xa00020c0        0x0 build/WiFIG/production/_ext/1472/berkeley_tcp_server_demo.o
 .mdebug.abi32  0xa00020c0        0x0 build/WiFIG/production/_ext/1472/berkeley_udp_client_demo.o
 .mdebug.abi32  0xa00020c0        0x0 build/WiFIG/production/_ext/1472/generic_tcp_client.o
 .mdebug.abi32  0xa00020c0        0x0 build/WiFIG/production/_ext/1472/generic_tcp_server.o
 .mdebug.abi32  0xa00020c0        0x0 build/WiFIG/production/_ext/1472/ping_demo.o
 .mdebug.abi32  0xa00020c0        0x0 build/WiFIG/production/_ext/1472/smtp_demo.o
 .mdebug.abi32  0xa00020c0        0x0 build/WiFIG/production/_ext/365611741/system_services.o
 .mdebug.abi32  0xa00020c0        0x0 build/WiFIG/production/_ext/365611741/system_debug.o
 .mdebug.abi32  0xa00020c0        0x0 build/WiFIG/production/_ext/365611741/system_random.o
 .mdebug.abi32  0xa00020c0        0x0 build/WiFIG/production/_ext/365611741/system_command.o
 .mdebug.abi32  0xa00020c0        0x0 build/WiFIG/production/_ext/365611741/system_userio.o
 .mdebug.abi32  0xa00020c0        0x0 build/WiFIG/production/_ext/97638081/sys_fs.o
 .mdebug.abi32  0xa00020c0        0x0 build/WiFIG/production/_ext/97638081/mpfs2.o
 .mdebug.abi32  0xa00020c0        0x0 build/WiFIG/production/_ext/792872985/usart.o
 .mdebug.abi32  0xa00020c0        0x0 build/WiFIG/production/_ext/792872985/lcd.o
 .mdebug.abi32  0xa00020c0        0x0 build/WiFIG/production/_ext/792872985/drv_spi.o
 .mdebug.abi32  0xa00020c0        0x0 build/WiFIG/production/_ext/792872985/db_appio.o
 .mdebug.abi32  0xa00020c0        0x0 build/WiFIG/production/_ext/792872985/spi_ram.o
 .mdebug.abi32  0xa00020c0        0x0 build/WiFIG/production/_ext/792872985/spi_eeprom.o
 .mdebug.abi32  0xa00020c0        0x0 build/WiFIG/production/_ext/792872985/spi_flash.o
 .mdebug.abi32  0xa00020c0        0x0 build/WiFIG/production/_ext/792872985/drv_media.o
 .mdebug.abi32  0xa00020c0        0x0 build/WiFIG/production/_ext/427700826/tcpip_announce.o
 .mdebug.abi32  0xa00020c0        0x0 build/WiFIG/production/_ext/427700826/http2.o
 .mdebug.abi32  0xa00020c0        0x0 build/WiFIG/production/_ext/427700826/arcfour.o
 .mdebug.abi32  0xa00020c0        0x0 build/WiFIG/production/_ext/427700826/arp.o
 .mdebug.abi32  0xa00020c0        0x0 build/WiFIG/production/_ext/427700826/berkeley_api.o
 .mdebug.abi32  0xa00020c0        0x0 build/WiFIG/production/_ext/427700826/dhcp.o
 .mdebug.abi32  0xa00020c0        0x0 build/WiFIG/production/_ext/427700826/dhcps.o
 .mdebug.abi32  0xa00020c0        0x0 build/WiFIG/production/_ext/427700826/dns.o
 .mdebug.abi32  0xa00020c0        0x0 build/WiFIG/production/_ext/427700826/dnss.o
 .mdebug.abi32  0xa00020c0        0x0 build/WiFIG/production/_ext/427700826/dyn_dns.o
 .mdebug.abi32  0xa00020c0        0x0 build/WiFIG/production/_ext/427700826/enc28_mac.o
 .mdebug.abi32  0xa00020c0        0x0 build/WiFIG/production/_ext/427700826/enc28j60.o
 .mdebug.abi32  0xa00020c0        0x0 build/WiFIG/production/_ext/427700826/encs24j600.o
 .mdebug.abi32  0xa00020c0        0x0 build/WiFIG/production/_ext/427700826/encx24_mac.o
 .mdebug.abi32  0xa00020c0        0x0 build/WiFIG/production/_ext/427700826/eth_pic32_ext_phy.o
 .mdebug.abi32  0xa00020c0        0x0 build/WiFIG/production/_ext/427700826/eth_pic32_ext_phy_dp83848.o
 .mdebug.abi32  0xa00020c0        0x0 build/WiFIG/production/_ext/427700826/eth_pic32_int_mac.o
 .mdebug.abi32  0xa00020c0        0x0 build/WiFIG/production/_ext/427700826/ftp.o
 .mdebug.abi32  0xa00020c0        0x0 build/WiFIG/production/_ext/427700826/hash_fnv.o
 .mdebug.abi32  0xa00020c0        0x0 build/WiFIG/production/_ext/427700826/hash_tbl.o
 .mdebug.abi32  0xa00020c0        0x0 build/WiFIG/production/_ext/427700826/icmp.o
 .mdebug.abi32  0xa00020c0        0x0 build/WiFIG/production/_ext/427700826/icmpv6.o
 .mdebug.abi32  0xa00020c0        0x0 build/WiFIG/production/_ext/427700826/ipv4.o
 .mdebug.abi32  0xa00020c0        0x0 build/WiFIG/production/_ext/427700826/ipv6.o
 .mdebug.abi32  0xa00020c0        0x0 build/WiFIG/production/_ext/427700826/mac_events_pic32.o
 .mdebug.abi32  0xa00020c0        0x0 build/WiFIG/production/_ext/427700826/nbns.o
 .mdebug.abi32  0xa00020c0        0x0 build/WiFIG/production/_ext/427700826/ndp.o
 .mdebug.abi32  0xa00020c0        0x0 build/WiFIG/production/_ext/427700826/tcpip_reboot.o
 .mdebug.abi32  0xa00020c0        0x0 build/WiFIG/production/_ext/427700826/rsa.o
 .mdebug.abi32  0xa00020c0        0x0 build/WiFIG/production/_ext/427700826/smtp.o
 .mdebug.abi32  0xa00020c0        0x0 build/WiFIG/production/_ext/427700826/snmp.o
 .mdebug.abi32  0xa00020c0        0x0 build/WiFIG/production/_ext/427700826/snmpv3.o
 .mdebug.abi32  0xa00020c0        0x0 build/WiFIG/production/_ext/427700826/snmpv3_usm.o
 .mdebug.abi32  0xa00020c0        0x0 build/WiFIG/production/_ext/427700826/sntp.o
 .mdebug.abi32  0xa00020c0        0x0 build/WiFIG/production/_ext/427700826/ssl.o
 .mdebug.abi32  0xa00020c0        0x0 build/WiFIG/production/_ext/427700826/tcp.o
 .mdebug.abi32  0xa00020c0        0x0 build/WiFIG/production/_ext/427700826/tcpip_heap_alloc.o
 .mdebug.abi32  0xa00020c0        0x0 build/WiFIG/production/_ext/427700826/tcpip_storage.o
 .mdebug.abi32  0xa00020c0        0x0 build/WiFIG/production/_ext/427700826/telnet.o
 .mdebug.abi32  0xa00020c0        0x0 build/WiFIG/production/_ext/427700826/tftpc.o
 .mdebug.abi32  0xa00020c0        0x0 build/WiFIG/production/_ext/427700826/udp.o
 .mdebug.abi32  0xa00020c0        0x0 build/WiFIG/production/_ext/427700826/tcpip_mac_object.o
 .mdebug.abi32  0xa00020c0        0x0 build/WiFIG/production/_ext/427700826/tcpip_manager.o
 .mdebug.abi32  0xa00020c0        0x0 build/WiFIG/production/_ext/427700826/tcpip_helpers.o
 .mdebug.abi32  0xa00020c0        0x0 build/WiFIG/production/_ext/427700826/tcpip_commands.o
 .mdebug.abi32  0xa00020c0        0x0 build/WiFIG/production/_ext/427700826/iperf.o
 .mdebug.abi32  0xa00020c0        0x0 build/WiFIG/production/_ext/427700826/tcpip_notify.o
 .mdebug.abi32  0xa00020c0        0x0 build/WiFIG/production/_ext/427700826/zero_conf_helper.o
 .mdebug.abi32  0xa00020c0        0x0 build/WiFIG/production/_ext/427700826/zero_conf_link_local.o
 .mdebug.abi32  0xa00020c0        0x0 build/WiFIG/production/_ext/427700826/zero_conf_multicast_dns.o
 .mdebug.abi32  0xa00020c0        0x0 build/WiFIG/production/_ext/334706090/wf_tx_power.o
 .mdebug.abi32  0xa00020c0        0x0 build/WiFIG/production/_ext/334706090/wf_connect.o
 .mdebug.abi32  0xa00020c0        0x0 build/WiFIG/production/_ext/334706090/wf_connection_algorithm.o
 .mdebug.abi32  0xa00020c0        0x0 build/WiFIG/production/_ext/334706090/wf_connection_manager.o
 .mdebug.abi32  0xa00020c0        0x0 build/WiFIG/production/_ext/334706090/wf_connection_profile.o
 .mdebug.abi32  0xa00020c0        0x0 build/WiFIG/production/_ext/334706090/wf_easy_config.o
 .mdebug.abi32  0xa00020c0        0x0 build/WiFIG/production/_ext/334706090/wf_eint.o
 .mdebug.abi32  0xa00020c0        0x0 build/WiFIG/production/_ext/334706090/wf_event_handler.o
 .mdebug.abi32  0xa00020c0        0x0 build/WiFIG/production/_ext/334706090/wf_init.o
 .mdebug.abi32  0xa00020c0        0x0 build/WiFIG/production/_ext/334706090/wf_power_save.o
 .mdebug.abi32  0xa00020c0        0x0 build/WiFIG/production/_ext/334706090/wf_scan.o
 .mdebug.abi32  0xa00020c0        0x0 build/WiFIG/production/_ext/334706090/wf_spi.o
 .mdebug.abi32  0xa00020c0        0x0 build/WiFIG/production/_ext/334706090/mrf24w_mac_pic32.o
 .mdebug.abi32  0xa00020c0        0x0 build/WiFIG/production/_ext/334706090/mrf24w_events.o
 .mdebug.abi32  0xa00020c0        0x0 build/WiFIG/production/_ext/334706090/wf_debug_output.o
 .mdebug.abi32  0xa00020c0        0x0 build/WiFIG/production/_ext/334706090/wf_commands.o
 .mdebug.abi32  0xa00020c0        0x0 build/WiFIG/production/_ext/334706090/wf_pbkdf2.o
 .mdebug.abi32  0xa00020c0        0x0 build/WiFIG/production/_ext/334706090/wf_driver_com_24g.o
 .mdebug.abi32  0xa00020c0        0x0 build/WiFIG/production/_ext/334706090/wf_driver_raw_24g.o
 .mdebug.abi32  0xa00020c0        0x0 build/WiFIG/production/_ext/334706090/wf_mac_24g.o
 .mdebug.abi32  0xa00020c0        0x0 build/WiFIG/production/_ext/334706090/wf_mgmt_msg_24g.o
 .mdebug.abi32  0xa00020c0        0x0 build/WiFIG/production/_ext/334706090/wf_param_msg_24g.o
 .mdebug.abi32  0xa00020c0        0x0 build/WiFIG/production/_ext/334706090/wf_configData.o
 .mdebug.abi32  0xa00020c0        0x0 build/WiFIG/production/_ext/1472/main_demo.o
 .mdebug.abi32  0xa00020c0        0x0 build/WiFIG/production/_ext/1472/custom_snmp_app.o
 .mdebug.abi32  0xa00020c0        0x0 build/WiFIG/production/_ext/1472/custom_ssl_cert.o
 .mdebug.abi32  0xa00020c0        0x0 build/WiFIG/production/_ext/1472/mpfs_img2.o
 .mdebug.abi32  0xa00020c0        0x0 build/WiFIG/production/_ext/1472/wf_config.o
 .mdebug.abi32  0xa00020c0        0x0 build/WiFIG/production/_ext/1472/custom_http_app.o
 .mdebug.abi32  0xa00020c0        0x0 build/WiFIG/production/_ext/1472/tcp6_demo_app.o
 .mdebug.abi32  0xa00020c0        0x0 c:/program files (x86)/microchip/xc32/v1.21/bin/../lib/gcc/pic32mx/4.5.2/../../../../pic32mx/lib/size\libmchp_peripheral.a(open_core_timer_lib.o)
 .mdebug.abi32  0xa00020c0        0x0 c:/program files (x86)/microchip/xc32/v1.21/bin/../lib/gcc/pic32mx/4.5.2/../../../../pic32mx/lib/size\libmchp_peripheral_32MX695F512H.a(soft_reset_lib.o)
 .mdebug.abi32  0xa00020c0        0x0 c:/program files (x86)/microchip/xc32/v1.21/bin/../lib/gcc/pic32mx/4.5.2/../../../../pic32mx/lib/size\libmchp_peripheral_32MX695F512H.a(pcache.o)
 .mdebug.abi32  0xa00020c0        0x0 c:/program files (x86)/microchip/xc32/v1.21/bin/../lib/gcc/pic32mx/4.5.2/../../../../pic32mx/lib/size\libmchp_peripheral_32MX695F512H.a(int_disable_interrupts_lib.o)
 .mdebug.abi32  0xa00020c0        0x0 c:/program files (x86)/microchip/xc32/v1.21/bin/../lib/gcc/pic32mx/4.5.2/../../../../pic32mx/lib/size\libmchp_peripheral_32MX695F512H.a(int_restore_interrupts_lib.o)
 .mdebug.abi32  0xa00020c0        0x0 c:/program files (x86)/microchip/xc32/v1.21/bin/../lib/gcc/pic32mx/4.5.2/../../../../pic32mx/lib/size\libmchp_peripheral_32MX695F512H.a(int_enable_mv_int_lib.o)
 .mdebug.abi32  0xa00020c0        0x0 c:/program files (x86)/microchip/xc32/v1.21/bin/../lib/gcc/pic32mx/4.5.2/../../../../pic32mx/lib/size\libmchp_peripheral_32MX695F512H.a(int_tbl_lib.o)
 .mdebug.abi32  0xa00020c0        0x0 c:/program files (x86)/microchip/xc32/v1.21/bin/../lib/gcc/pic32mx/4.5.2/../../../../pic32mx/lib/size\libmchp_peripheral_32MX695F512H.a(rtcc_init_lib.o)
 .mdebug.abi32  0xa00020c0        0x0 c:/program files (x86)/microchip/xc32/v1.21/bin/../lib/gcc/pic32mx/4.5.2/../../../../pic32mx/lib/size\libmchp_peripheral_32MX695F512H.a(rtcc_open_lib.o)
 .mdebug.abi32  0xa00020c0        0x0 c:/program files (x86)/microchip/xc32/v1.21/bin/../lib/gcc/pic32mx/4.5.2/../../../../pic32mx/lib/size\libmchp_peripheral_32MX695F512H.a(spi_chn_data_rdy_lib.o)
 .mdebug.abi32  0xa00020c0        0x0 c:/program files (x86)/microchip/xc32/v1.21/bin/../lib/gcc/pic32mx/4.5.2/../../../../pic32mx/lib/size\libmchp_peripheral_32MX695F512H.a(spi_chn_getc_lib.o)
 .mdebug.abi32  0xa00020c0        0x0 c:/program files (x86)/microchip/xc32/v1.21/bin/../lib/gcc/pic32mx/4.5.2/../../../../pic32mx/lib/size\libmchp_peripheral_32MX695F512H.a(spi_chn_open_lib.o)
 .mdebug.abi32  0xa00020c0        0x0 c:/program files (x86)/microchip/xc32/v1.21/bin/../lib/gcc/pic32mx/4.5.2/../../../../pic32mx/lib/size\libmchp_peripheral_32MX695F512H.a(spi_chn_putc_lib.o)
 .mdebug.abi32  0xa00020c0        0x0 c:/program files (x86)/microchip/xc32/v1.21/bin/../lib/gcc/pic32mx/4.5.2/../../../../pic32mx/lib/size\libmchp_peripheral_32MX695F512H.a(spi_chn_tx_buff_empty_lib.o)
 .mdebug.abi32  0xa00020c0        0x0 c:/program files (x86)/microchip/xc32/v1.21/bin/../lib/gcc/pic32mx/4.5.2/../../../../pic32mx/lib/size\libmchp_peripheral_32MX695F512H.a(spi_io_tbl_libp.o)
 .mdebug.abi32  0xa00020c0        0x0 c:/program files (x86)/microchip/xc32/v1.21/bin/../lib/gcc/pic32mx/4.5.2/../../../../pic32mx/lib/size\libmchp_peripheral_32MX695F512H.a(spi_map_tbl_libp.o)
 .mdebug.abi32  0xa00020c0        0x0 c:/program files (x86)/microchip/xc32/v1.21/bin/../lib/gcc/pic32mx/4.5.2/../../../../pic32mx/lib/size\libmchp_peripheral_32MX695F512H.a(port_set_pins_digital_in_lib.o)
 .mdebug.abi32  0xa00020c0        0x0 c:/program files (x86)/microchip/xc32/v1.21/bin/../lib/gcc/pic32mx/4.5.2/../../../../pic32mx/lib/size\libmchp_peripheral_32MX695F512H.a(port_set_pins_digital_out_lib.o)
 .mdebug.abi32  0xa00020c0        0x0 c:/program files (x86)/microchip/xc32/v1.21/bin/../lib/gcc/pic32mx/4.5.2/../../../../pic32mx/lib/size\libmchp_peripheral_32MX695F512H.a(_ports_tbl_libp.o)
 .mdebug.abi32  0xa00020c0        0x0 c:/program files (x86)/microchip/xc32/v1.21/bin/../lib/gcc/pic32mx/4.5.2/../../../../pic32mx/lib/size\libmchp_peripheral_32MX695F512H.a(int_enable_interrupts_lib.o)
 .mdebug.abi32  0xa00020c0        0x0 c:/program files (x86)/microchip/xc32/v1.21/bin/../lib/gcc/pic32mx/4.5.2/../../../../pic32mx/lib/size\libmchp_peripheral_32MX695F512H.a(_rtcc_wait_clock_off_lib.o)
 .mdebug.abi32  0xa00020c0        0x0 c:/program files (x86)/microchip/xc32/v1.21/bin/../lib/gcc/pic32mx/4.5.2/../../../../pic32mx/lib/size\libmchp_peripheral_32MX695F512H.a(read_core_timer_lib.o)
 .mdebug.abi32  0xa00020c0        0x0 c:/program files (x86)/microchip/xc32/v1.21/bin/../lib/gcc/pic32mx/4.5.2/size\libgcc.a(_udivdi3.o)
 .mdebug.abi32  0xa00020c0        0x0 c:/program files (x86)/microchip/xc32/v1.21/bin/../lib/gcc/pic32mx/4.5.2/../../../../pic32mx/lib/size\libpic32.a(default-bootstrap-exception-handler.o)
 .mdebug.abi32  0xa00020c0        0x0 c:/program files (x86)/microchip/xc32/v1.21/bin/../lib/gcc/pic32mx/4.5.2/../../../../pic32mx/lib/size\libpic32.a(default-on-reset.o)
 .mdebug.abi32  0xa00020c0        0x0 c:/program files (x86)/microchip/xc32/v1.21/bin/../lib/gcc/pic32mx/4.5.2/../../../../pic32mx/lib/size\libpic32.a(default-on-bootstrap.o)
 .mdebug.abi32  0xa00020c0        0x0 c:/program files (x86)/microchip/xc32/v1.21/bin/../lib/gcc/pic32mx/4.5.2/../../../../pic32mx/lib/size\libpic32.a(defaultinterrupt.o)
 .mdebug.abi32  0xa00020c0        0x0 c:/program files (x86)/microchip/xc32/v1.21/bin/../lib/gcc/pic32mx/4.5.2/../../../../pic32mx/lib/size\libc.a(atoi.o)
 .mdebug.abi32  0xa00020c0        0x0 c:/program files (x86)/microchip/xc32/v1.21/bin/../lib/gcc/pic32mx/4.5.2/../../../../pic32mx/lib/size\libc.a(ctype.o)
 .mdebug.abi32  0xa00020c0        0x0 c:/program files (x86)/microchip/xc32/v1.21/bin/../lib/gcc/pic32mx/4.5.2/../../../../pic32mx/lib/size\libc.a(malloc.o)
 .mdebug.abi32  0xa00020c0        0x0 c:/program files (x86)/microchip/xc32/v1.21/bin/../lib/gcc/pic32mx/4.5.2/../../../../pic32mx/lib/size\libc.a(rand.o)
 .mdebug.abi32  0xa00020c0        0x0 c:/program files (x86)/microchip/xc32/v1.21/bin/../lib/gcc/pic32mx/4.5.2/../../../../pic32mx/lib/size\libc.a(strcat.o)
 .mdebug.abi32  0xa00020c0        0x0 c:/program files (x86)/microchip/xc32/v1.21/bin/../lib/gcc/pic32mx/4.5.2/../../../../pic32mx/lib/size\libc.a(strchr.o)
 .mdebug.abi32  0xa00020c0        0x0 c:/program files (x86)/microchip/xc32/v1.21/bin/../lib/gcc/pic32mx/4.5.2/../../../../pic32mx/lib/size\libc.a(strncat.o)
 .mdebug.abi32  0xa00020c0        0x0 c:/program files (x86)/microchip/xc32/v1.21/bin/../lib/gcc/pic32mx/4.5.2/../../../../pic32mx/lib/size\libc.a(strncpy.o)
 .mdebug.abi32  0xa00020c0        0x0 c:/program files (x86)/microchip/xc32/v1.21/bin/../lib/gcc/pic32mx/4.5.2/../../../../pic32mx/lib/size\libc.a(strstr.o)
 .mdebug.abi32  0xa00020c0        0x0 c:/program files (x86)/microchip/xc32/v1.21/bin/../lib/gcc/pic32mx/4.5.2/../../../../pic32mx/lib/size\libc.a(strtol.o)
 .mdebug.abi32  0xa00020c0        0x0 c:/program files (x86)/microchip/xc32/v1.21/bin/../lib/gcc/pic32mx/4.5.2/../../../../pic32mx/lib/size\libc.a(snprintf_cdnopsuxX.eo)
 .mdebug.abi32  0xa00020c0        0x0 c:/program files (x86)/microchip/xc32/v1.21/bin/../lib/gcc/pic32mx/4.5.2/../../../../pic32mx/lib/size\libc.a(sprintf_cdnopsuxX.eo)
 .mdebug.abi32  0xa00020c0        0x0 c:/program files (x86)/microchip/xc32/v1.21/bin/../lib/gcc/pic32mx/4.5.2/../../../../pic32mx/lib/size\libc.a(vsnprintf_cdnopsuxX.eo)
 .mdebug.abi32  0xa00020c0        0x0 c:/program files (x86)/microchip/xc32/v1.21/bin/../lib/gcc/pic32mx/4.5.2/../../../../pic32mx/lib/size\libc.a(vsnprintf.o)
 .mdebug.abi32  0xa00020c0        0x0 c:/program files (x86)/microchip/xc32/v1.21/bin/../lib/gcc/pic32mx/4.5.2/../../../../pic32mx/lib/size\libc.a(ctypef.o)
 .mdebug.abi32  0xa00020c0        0x0 c:/program files (x86)/microchip/xc32/v1.21/bin/../lib/gcc/pic32mx/4.5.2/../../../../pic32mx/lib/size\libc.a(errno.o)
 .mdebug.abi32  0xa00020c0        0x0 c:/program files (x86)/microchip/xc32/v1.21/bin/../lib/gcc/pic32mx/4.5.2/../../../../pic32mx/lib/size\libc.a(strncmp.o)
 .mdebug.abi32  0xa00020c0        0x0 c:/program files (x86)/microchip/xc32/v1.21/bin/../lib/gcc/pic32mx/4.5.2/../../../../pic32mx/lib/size\libc.a(doprnt_cdnopsuxX.eo)
 .mdebug.abi32  0xa00020c0        0x0 c:/program files (x86)/microchip/xc32/v1.21/bin/../lib/gcc/pic32mx/4.5.2/../../../../pic32mx/lib/size\libc.a(doprnt.o)
 .mdebug.abi32  0xa00020c0        0x0 c:/program files (x86)/microchip/xc32/v1.21/bin/../lib/gcc/pic32mx/4.5.2/../../../../pic32mx/lib/size\libc.a(_fputc_simple.o)
 .mdebug.abi32  0xa00020c0        0x0 c:/program files (x86)/microchip/xc32/v1.21/bin/../lib/gcc/pic32mx/4.5.2/../../../../pic32mx/lib/size\libc.a(powersf.o)
 .mdebug.abi32  0xa00020c0        0x0 c:/program files (x86)/microchip/xc32/v1.21/bin/../lib/gcc/pic32mx/4.5.2/../../../../pic32mx/lib/size\libc.a(_iob.o)
 .mdebug.abi32  0xa00020c0        0x0 c:/program files (x86)/microchip/xc32/v1.21/bin/../lib/gcc/pic32mx/4.5.2/../../../../pic32mx/lib/size\libc.a(_flsbuf_simple.o)
 .mdebug.abi32  0xa00020c0        0x0 c:/program files (x86)/microchip/xc32/v1.21/bin/../lib/gcc/pic32mx/4.5.2/../../../../pic32mx/lib/size\libpic32.a(sbrk.o)
 .mdebug.abi32  0xa00020c0        0x0 c:/program files (x86)/microchip/xc32/v1.21/bin/../lib/gcc/pic32mx/4.5.2/../../../../pic32mx/lib/size\libpic32.a(write.o)
 .mdebug.abi32  0xa00020c0        0x0 c:/program files (x86)/microchip/xc32/v1.21/bin/../lib/gcc/pic32mx/4.5.2/../../../../pic32mx/lib/size\libpic32.a(_mon_putc.o)
 .mdebug.abi32  0xa00020c0        0x0 c:/program files (x86)/microchip/xc32/v1.21/bin/../lib/gcc/pic32mx/4.5.2/../../../../pic32mx/lib/size\libpic32.a(xc32_uart.o)
 .mdebug.abi32  0xa00020c0        0x0 c:/program files (x86)/microchip/xc32/v1.21/bin/../lib/gcc/pic32mx/4.5.2/../../../../pic32mx/lib/size\libe.a(_floatdisf.o)
 .mdebug.abi32  0xa00020c0        0x0 c:/program files (x86)/microchip/xc32/v1.21/bin/../lib/gcc/pic32mx/4.5.2/size\libgcc.a(_lshrdi3.o)
 .mdebug.abi32  0xa00020c0        0x0 c:/program files (x86)/microchip/xc32/v1.21/bin/../lib/gcc/pic32mx/4.5.2/size\libgcc.a(_floatundisf.o)
 .mdebug.abi32  0xa00020c0        0x0 c:/program files (x86)/microchip/xc32/v1.21/bin/../lib/gcc/pic32mx/4.5.2/size\libgcc.a(_umoddi3.o)
 .mdebug.abi32  0xa00020c0        0x0 c:/program files (x86)/microchip/xc32/v1.21/bin/../lib/gcc/pic32mx/4.5.2/size\libgcc.a(floatunsisf.o)

.mdebug.abiN32
 *(.mdebug.abiN32)

.mdebug.abi64
 *(.mdebug.abi64)

.mdebug.abiO64
 *(.mdebug.abiO64)

.mdebug.eabi32
 *(.mdebug.eabi32)

.mdebug.eabi64
 *(.mdebug.eabi64)

.gcc_compiled_long32
 *(.gcc_compiled_long32)

.gcc_compiled_long64
 *(.gcc_compiled_long64)

.stab
 *(.stab)

.stabstr
 *(.stabstr)

.stab.excl
 *(.stab.excl)

.stab.exclstr
 *(.stab.exclstr)

.stab.index
 *(.stab.index)

.stab.indexstr
 *(.stab.indexstr)

.comment        0x00000000      0x2b5
 *(.comment)
 .comment       0x00000000       0x3c build/WiFIG/production/_ext/1293749816/bsp.o
                                 0x3d (size before relaxing)
 .comment       0x00000000       0x3d build/WiFIG/production/_ext/101875047/hashes.o
 .comment       0x00000000       0x3d build/WiFIG/production/_ext/101875047/lfsr.o
 .comment       0x00000000       0x3d build/WiFIG/production/_ext/101875047/big_int.o
 .comment       0x00000000       0x3d build/WiFIG/production/_ext/101875047/helpers.o
 .comment       0x00000000       0x3d build/WiFIG/production/_ext/1472/berkeley_tcp_client_demo.o
 .comment       0x00000000       0x3d build/WiFIG/production/_ext/1472/berkeley_tcp_server_demo.o
 .comment       0x00000000       0x3d build/WiFIG/production/_ext/1472/berkeley_udp_client_demo.o
 .comment       0x00000000       0x3d build/WiFIG/production/_ext/1472/generic_tcp_client.o
 .comment       0x00000000       0x3d build/WiFIG/production/_ext/1472/generic_tcp_server.o
 .comment       0x00000000       0x3d build/WiFIG/production/_ext/1472/ping_demo.o
 .comment       0x00000000       0x3d build/WiFIG/production/_ext/1472/smtp_demo.o
 .comment       0x00000000       0x3d build/WiFIG/production/_ext/365611741/system_services.o
 .comment       0x00000000       0x3d build/WiFIG/production/_ext/365611741/system_debug.o
 .comment       0x00000000       0x3d build/WiFIG/production/_ext/365611741/system_random.o
 .comment       0x00000000       0x3d build/WiFIG/production/_ext/365611741/system_command.o
 .comment       0x00000000       0x3d build/WiFIG/production/_ext/365611741/system_userio.o
 .comment       0x00000000       0x3d build/WiFIG/production/_ext/97638081/sys_fs.o
 .comment       0x00000000       0x3d build/WiFIG/production/_ext/97638081/mpfs2.o
 .comment       0x00000000       0x3d build/WiFIG/production/_ext/792872985/usart.o
 .comment       0x00000000       0x3d build/WiFIG/production/_ext/792872985/lcd.o
 .comment       0x00000000       0x3d build/WiFIG/production/_ext/792872985/drv_spi.o
 .comment       0x00000000       0x3d build/WiFIG/production/_ext/792872985/db_appio.o
 .comment       0x00000000       0x3d build/WiFIG/production/_ext/792872985/spi_ram.o
 .comment       0x00000000       0x3d build/WiFIG/production/_ext/792872985/spi_eeprom.o
 .comment       0x00000000       0x3d build/WiFIG/production/_ext/792872985/spi_flash.o
 .comment       0x00000000       0x3d build/WiFIG/production/_ext/792872985/drv_media.o
 .comment       0x00000000       0x3d build/WiFIG/production/_ext/427700826/tcpip_announce.o
 .comment       0x00000000       0x3d build/WiFIG/production/_ext/427700826/http2.o
 .comment       0x00000000       0x3d build/WiFIG/production/_ext/427700826/arcfour.o
 .comment       0x00000000       0x3d build/WiFIG/production/_ext/427700826/arp.o
 .comment       0x00000000       0x3d build/WiFIG/production/_ext/427700826/berkeley_api.o
 .comment       0x00000000       0x3d build/WiFIG/production/_ext/427700826/dhcp.o
 .comment       0x00000000       0x3d build/WiFIG/production/_ext/427700826/dhcps.o
 .comment       0x00000000       0x3d build/WiFIG/production/_ext/427700826/dns.o
 .comment       0x00000000       0x3d build/WiFIG/production/_ext/427700826/dnss.o
 .comment       0x00000000       0x3d build/WiFIG/production/_ext/427700826/dyn_dns.o
 .comment       0x00000000       0x3d build/WiFIG/production/_ext/427700826/enc28_mac.o
 .comment       0x00000000       0x3d build/WiFIG/production/_ext/427700826/enc28j60.o
 .comment       0x00000000       0x3d build/WiFIG/production/_ext/427700826/encs24j600.o
 .comment       0x00000000       0x3d build/WiFIG/production/_ext/427700826/encx24_mac.o
 .comment       0x00000000       0x3d build/WiFIG/production/_ext/427700826/eth_pic32_ext_phy.o
 .comment       0x00000000       0x3d build/WiFIG/production/_ext/427700826/eth_pic32_ext_phy_dp83848.o
 .comment       0x00000000       0x3d build/WiFIG/production/_ext/427700826/eth_pic32_int_mac.o
 .comment       0x00000000       0x3d build/WiFIG/production/_ext/427700826/ftp.o
 .comment       0x00000000       0x3d build/WiFIG/production/_ext/427700826/hash_fnv.o
 .comment       0x00000000       0x3d build/WiFIG/production/_ext/427700826/hash_tbl.o
 .comment       0x00000000       0x3d build/WiFIG/production/_ext/427700826/icmp.o
 .comment       0x00000000       0x3d build/WiFIG/production/_ext/427700826/icmpv6.o
 .comment       0x00000000       0x3d build/WiFIG/production/_ext/427700826/ipv4.o
 .comment       0x00000000       0x3d build/WiFIG/production/_ext/427700826/ipv6.o
 .comment       0x00000000       0x3d build/WiFIG/production/_ext/427700826/mac_events_pic32.o
 .comment       0x00000000       0x3d build/WiFIG/production/_ext/427700826/nbns.o
 .comment       0x00000000       0x3d build/WiFIG/production/_ext/427700826/ndp.o
 .comment       0x00000000       0x3d build/WiFIG/production/_ext/427700826/tcpip_reboot.o
 .comment       0x00000000       0x3d build/WiFIG/production/_ext/427700826/rsa.o
 .comment       0x00000000       0x3d build/WiFIG/production/_ext/427700826/smtp.o
 .comment       0x00000000       0x3d build/WiFIG/production/_ext/427700826/snmp.o
 .comment       0x00000000       0x3d build/WiFIG/production/_ext/427700826/snmpv3.o
 .comment       0x00000000       0x3d build/WiFIG/production/_ext/427700826/snmpv3_usm.o
 .comment       0x00000000       0x3d build/WiFIG/production/_ext/427700826/sntp.o
 .comment       0x00000000       0x3d build/WiFIG/production/_ext/427700826/ssl.o
 .comment       0x00000000       0x3d build/WiFIG/production/_ext/427700826/tcp.o
 .comment       0x00000000       0x3d build/WiFIG/production/_ext/427700826/tcpip_heap_alloc.o
 .comment       0x00000000       0x3d build/WiFIG/production/_ext/427700826/tcpip_storage.o
 .comment       0x00000000       0x3d build/WiFIG/production/_ext/427700826/telnet.o
 .comment       0x00000000       0x3d build/WiFIG/production/_ext/427700826/tftpc.o
 .comment       0x00000000       0x3d build/WiFIG/production/_ext/427700826/udp.o
 .comment       0x00000000       0x3d build/WiFIG/production/_ext/427700826/tcpip_mac_object.o
 .comment       0x00000000       0x3d build/WiFIG/production/_ext/427700826/tcpip_manager.o
 .comment       0x00000000       0x3d build/WiFIG/production/_ext/427700826/tcpip_helpers.o
 .comment       0x00000000       0x3d build/WiFIG/production/_ext/427700826/tcpip_commands.o
 .comment       0x00000000       0x3d build/WiFIG/production/_ext/427700826/iperf.o
 .comment       0x00000000       0x3d build/WiFIG/production/_ext/427700826/tcpip_notify.o
 .comment       0x00000000       0x3d build/WiFIG/production/_ext/427700826/zero_conf_helper.o
 .comment       0x00000000       0x3d build/WiFIG/production/_ext/427700826/zero_conf_link_local.o
 .comment       0x00000000       0x3d build/WiFIG/production/_ext/427700826/zero_conf_multicast_dns.o
 .comment       0x00000000       0x3d build/WiFIG/production/_ext/334706090/wf_tx_power.o
 .comment       0x00000000       0x3d build/WiFIG/production/_ext/334706090/wf_connect.o
 .comment       0x00000000       0x3d build/WiFIG/production/_ext/334706090/wf_connection_algorithm.o
 .comment       0x00000000       0x3d build/WiFIG/production/_ext/334706090/wf_connection_manager.o
 .comment       0x00000000       0x3d build/WiFIG/production/_ext/334706090/wf_connection_profile.o
 .comment       0x00000000       0x3d build/WiFIG/production/_ext/334706090/wf_easy_config.o
 .comment       0x00000000       0x3d build/WiFIG/production/_ext/334706090/wf_eint.o
 .comment       0x00000000       0x3d build/WiFIG/production/_ext/334706090/wf_event_handler.o
 .comment       0x00000000       0x3d build/WiFIG/production/_ext/334706090/wf_init.o
 .comment       0x00000000       0x3d build/WiFIG/production/_ext/334706090/wf_power_save.o
 .comment       0x00000000       0x3d build/WiFIG/production/_ext/334706090/wf_scan.o
 .comment       0x00000000       0x3d build/WiFIG/production/_ext/334706090/wf_spi.o
 .comment       0x00000000       0x3d build/WiFIG/production/_ext/334706090/mrf24w_mac_pic32.o
 .comment       0x00000000       0x3d build/WiFIG/production/_ext/334706090/mrf24w_events.o
 .comment       0x00000000       0x3d build/WiFIG/production/_ext/334706090/wf_debug_output.o
 .comment       0x00000000       0x3d build/WiFIG/production/_ext/334706090/wf_commands.o
 .comment       0x00000000       0x3d build/WiFIG/production/_ext/334706090/wf_pbkdf2.o
 .comment       0x00000000       0x3d build/WiFIG/production/_ext/334706090/wf_driver_com_24g.o
 .comment       0x00000000       0x3d build/WiFIG/production/_ext/334706090/wf_driver_raw_24g.o
 .comment       0x00000000       0x3d build/WiFIG/production/_ext/334706090/wf_mac_24g.o
 .comment       0x00000000       0x3d build/WiFIG/production/_ext/334706090/wf_mgmt_msg_24g.o
 .comment       0x00000000       0x3d build/WiFIG/production/_ext/334706090/wf_param_msg_24g.o
 .comment       0x00000000       0x3d build/WiFIG/production/_ext/334706090/wf_configData.o
 .comment       0x00000000       0x3d build/WiFIG/production/_ext/1472/main_demo.o
 .comment       0x00000000       0x3d build/WiFIG/production/_ext/1472/custom_snmp_app.o
 .comment       0x00000000       0x3d build/WiFIG/production/_ext/1472/custom_ssl_cert.o
 .comment       0x00000000       0x3d build/WiFIG/production/_ext/1472/mpfs_img2.o
 .comment       0x00000000       0x3d build/WiFIG/production/_ext/1472/wf_config.o
 .comment       0x00000000       0x3d build/WiFIG/production/_ext/1472/custom_http_app.o
 .comment       0x00000000       0x3d build/WiFIG/production/_ext/1472/tcp6_demo_app.o
 .comment       0x0000003c       0x3c c:/program files (x86)/microchip/xc32/v1.21/bin/../lib/gcc/pic32mx/4.5.2/../../../../pic32mx/lib/size\libmchp_peripheral.a(open_core_timer_lib.o)
                                 0x3d (size before relaxing)
 .comment       0x00000000       0x3d c:/program files (x86)/microchip/xc32/v1.21/bin/../lib/gcc/pic32mx/4.5.2/../../../../pic32mx/lib/size\libmchp_peripheral_32MX695F512H.a(soft_reset_lib.o)
 .comment       0x00000000       0x3d c:/program files (x86)/microchip/xc32/v1.21/bin/../lib/gcc/pic32mx/4.5.2/../../../../pic32mx/lib/size\libmchp_peripheral_32MX695F512H.a(pcache.o)
 .comment       0x00000000       0x3d c:/program files (x86)/microchip/xc32/v1.21/bin/../lib/gcc/pic32mx/4.5.2/../../../../pic32mx/lib/size\libmchp_peripheral_32MX695F512H.a(int_disable_interrupts_lib.o)
 .comment       0x00000000       0x3d c:/program files (x86)/microchip/xc32/v1.21/bin/../lib/gcc/pic32mx/4.5.2/../../../../pic32mx/lib/size\libmchp_peripheral_32MX695F512H.a(int_restore_interrupts_lib.o)
 .comment       0x00000000       0x3d c:/program files (x86)/microchip/xc32/v1.21/bin/../lib/gcc/pic32mx/4.5.2/../../../../pic32mx/lib/size\libmchp_peripheral_32MX695F512H.a(int_enable_mv_int_lib.o)
 .comment       0x00000000       0x3d c:/program files (x86)/microchip/xc32/v1.21/bin/../lib/gcc/pic32mx/4.5.2/../../../../pic32mx/lib/size\libmchp_peripheral_32MX695F512H.a(int_tbl_lib.o)
 .comment       0x00000000       0x3d c:/program files (x86)/microchip/xc32/v1.21/bin/../lib/gcc/pic32mx/4.5.2/../../../../pic32mx/lib/size\libmchp_peripheral_32MX695F512H.a(rtcc_init_lib.o)
 .comment       0x00000000       0x3d c:/program files (x86)/microchip/xc32/v1.21/bin/../lib/gcc/pic32mx/4.5.2/../../../../pic32mx/lib/size\libmchp_peripheral_32MX695F512H.a(rtcc_open_lib.o)
 .comment       0x00000000       0x3d c:/program files (x86)/microchip/xc32/v1.21/bin/../lib/gcc/pic32mx/4.5.2/../../../../pic32mx/lib/size\libmchp_peripheral_32MX695F512H.a(spi_chn_data_rdy_lib.o)
 .comment       0x00000000       0x3d c:/program files (x86)/microchip/xc32/v1.21/bin/../lib/gcc/pic32mx/4.5.2/../../../../pic32mx/lib/size\libmchp_peripheral_32MX695F512H.a(spi_chn_getc_lib.o)
 .comment       0x00000000       0x3d c:/program files (x86)/microchip/xc32/v1.21/bin/../lib/gcc/pic32mx/4.5.2/../../../../pic32mx/lib/size\libmchp_peripheral_32MX695F512H.a(spi_chn_open_lib.o)
 .comment       0x00000000       0x3d c:/program files (x86)/microchip/xc32/v1.21/bin/../lib/gcc/pic32mx/4.5.2/../../../../pic32mx/lib/size\libmchp_peripheral_32MX695F512H.a(spi_chn_putc_lib.o)
 .comment       0x00000000       0x3d c:/program files (x86)/microchip/xc32/v1.21/bin/../lib/gcc/pic32mx/4.5.2/../../../../pic32mx/lib/size\libmchp_peripheral_32MX695F512H.a(spi_chn_tx_buff_empty_lib.o)
 .comment       0x00000000       0x3d c:/program files (x86)/microchip/xc32/v1.21/bin/../lib/gcc/pic32mx/4.5.2/../../../../pic32mx/lib/size\libmchp_peripheral_32MX695F512H.a(spi_io_tbl_libp.o)
 .comment       0x00000000       0x3d c:/program files (x86)/microchip/xc32/v1.21/bin/../lib/gcc/pic32mx/4.5.2/../../../../pic32mx/lib/size\libmchp_peripheral_32MX695F512H.a(spi_map_tbl_libp.o)
 .comment       0x00000000       0x3d c:/program files (x86)/microchip/xc32/v1.21/bin/../lib/gcc/pic32mx/4.5.2/../../../../pic32mx/lib/size\libmchp_peripheral_32MX695F512H.a(port_set_pins_digital_in_lib.o)
 .comment       0x00000000       0x3d c:/program files (x86)/microchip/xc32/v1.21/bin/../lib/gcc/pic32mx/4.5.2/../../../../pic32mx/lib/size\libmchp_peripheral_32MX695F512H.a(port_set_pins_digital_out_lib.o)
 .comment       0x00000000       0x3d c:/program files (x86)/microchip/xc32/v1.21/bin/../lib/gcc/pic32mx/4.5.2/../../../../pic32mx/lib/size\libmchp_peripheral_32MX695F512H.a(_ports_tbl_libp.o)
 .comment       0x00000000       0x3d c:/program files (x86)/microchip/xc32/v1.21/bin/../lib/gcc/pic32mx/4.5.2/../../../../pic32mx/lib/size\libmchp_peripheral_32MX695F512H.a(int_enable_interrupts_lib.o)
 .comment       0x00000000       0x3d c:/program files (x86)/microchip/xc32/v1.21/bin/../lib/gcc/pic32mx/4.5.2/../../../../pic32mx/lib/size\libmchp_peripheral_32MX695F512H.a(_rtcc_wait_clock_off_lib.o)
 .comment       0x00000000       0x3d c:/program files (x86)/microchip/xc32/v1.21/bin/../lib/gcc/pic32mx/4.5.2/../../../../pic32mx/lib/size\libmchp_peripheral_32MX695F512H.a(read_core_timer_lib.o)
 .comment       0x00000000       0x3d c:/program files (x86)/microchip/xc32/v1.21/bin/../lib/gcc/pic32mx/4.5.2/size\libgcc.a(_udivdi3.o)
 .comment       0x00000078       0x18 c:/program files (x86)/microchip/xc32/v1.21/bin/../lib/gcc/pic32mx/4.5.2/../../../../pic32mx/lib/size\libpic32.a(memcmp.o)
                                 0x19 (size before relaxing)
 .comment       0x00000090       0x18 c:/program files (x86)/microchip/xc32/v1.21/bin/../lib/gcc/pic32mx/4.5.2/../../../../pic32mx/lib/size\libpic32.a(memset.o)
                                 0x19 (size before relaxing)
 .comment       0x000000a8       0x55 c:/program files (x86)/microchip/xc32/v1.21/bin/../lib/gcc/pic32mx/4.5.2/../../../../pic32mx/lib/size\libpic32.a(strcmp.o)
                                 0x56 (size before relaxing)
 .comment       0x000000fd       0x19 c:/program files (x86)/microchip/xc32/v1.21/bin/../lib/gcc/pic32mx/4.5.2/../../../../pic32mx/lib/size\libpic32.a(strcpy.o)
                                 0x1a (size before relaxing)
 .comment       0x00000116       0x19 c:/program files (x86)/microchip/xc32/v1.21/bin/../lib/gcc/pic32mx/4.5.2/../../../../pic32mx/lib/size\libpic32.a(strlen.o)
                                 0x1a (size before relaxing)
 .comment       0x00000000       0x3d c:/program files (x86)/microchip/xc32/v1.21/bin/../lib/gcc/pic32mx/4.5.2/../../../../pic32mx/lib/size\libpic32.a(default-bootstrap-exception-handler.o)
 .comment       0x00000000       0x3d c:/program files (x86)/microchip/xc32/v1.21/bin/../lib/gcc/pic32mx/4.5.2/../../../../pic32mx/lib/size\libpic32.a(default-on-reset.o)
 .comment       0x00000000       0x3d c:/program files (x86)/microchip/xc32/v1.21/bin/../lib/gcc/pic32mx/4.5.2/../../../../pic32mx/lib/size\libpic32.a(default-on-bootstrap.o)
 .comment       0x00000000       0x3d c:/program files (x86)/microchip/xc32/v1.21/bin/../lib/gcc/pic32mx/4.5.2/../../../../pic32mx/lib/size\libpic32.a(defaultinterrupt.o)
 .comment       0x00000000       0x3d c:/program files (x86)/microchip/xc32/v1.21/bin/../lib/gcc/pic32mx/4.5.2/../../../../pic32mx/lib/size\libc.a(atoi.o)
 .comment       0x0000012f       0x4e c:/program files (x86)/microchip/xc32/v1.21/bin/../lib/gcc/pic32mx/4.5.2/../../../../pic32mx/lib/size\libc.a(ctype.o)
                                 0x8b (size before relaxing)
 .comment       0x00000000       0x3d c:/program files (x86)/microchip/xc32/v1.21/bin/../lib/gcc/pic32mx/4.5.2/../../../../pic32mx/lib/size\libc.a(malloc.o)
 .comment       0x00000000       0x3d c:/program files (x86)/microchip/xc32/v1.21/bin/../lib/gcc/pic32mx/4.5.2/../../../../pic32mx/lib/size\libc.a(rand.o)
 .comment       0x00000000       0x3d c:/program files (x86)/microchip/xc32/v1.21/bin/../lib/gcc/pic32mx/4.5.2/../../../../pic32mx/lib/size\libc.a(strcat.o)
 .comment       0x00000000       0x3d c:/program files (x86)/microchip/xc32/v1.21/bin/../lib/gcc/pic32mx/4.5.2/../../../../pic32mx/lib/size\libc.a(strchr.o)
 .comment       0x00000000       0x3d c:/program files (x86)/microchip/xc32/v1.21/bin/../lib/gcc/pic32mx/4.5.2/../../../../pic32mx/lib/size\libc.a(strncat.o)
 .comment       0x00000000       0x3d c:/program files (x86)/microchip/xc32/v1.21/bin/../lib/gcc/pic32mx/4.5.2/../../../../pic32mx/lib/size\libc.a(strncpy.o)
 .comment       0x00000000       0x3d c:/program files (x86)/microchip/xc32/v1.21/bin/../lib/gcc/pic32mx/4.5.2/../../../../pic32mx/lib/size\libc.a(strstr.o)
 .comment       0x00000000       0x3d c:/program files (x86)/microchip/xc32/v1.21/bin/../lib/gcc/pic32mx/4.5.2/../../../../pic32mx/lib/size\libc.a(strtol.o)
 .comment       0x00000000       0x3d c:/program files (x86)/microchip/xc32/v1.21/bin/../lib/gcc/pic32mx/4.5.2/../../../../pic32mx/lib/size\libc.a(snprintf_cdnopsuxX.eo)
 .comment       0x00000000       0x3d c:/program files (x86)/microchip/xc32/v1.21/bin/../lib/gcc/pic32mx/4.5.2/../../../../pic32mx/lib/size\libc.a(sprintf_cdnopsuxX.eo)
 .comment       0x00000000       0x3d c:/program files (x86)/microchip/xc32/v1.21/bin/../lib/gcc/pic32mx/4.5.2/../../../../pic32mx/lib/size\libc.a(vsnprintf_cdnopsuxX.eo)
 .comment       0x00000000       0x3d c:/program files (x86)/microchip/xc32/v1.21/bin/../lib/gcc/pic32mx/4.5.2/../../../../pic32mx/lib/size\libc.a(vsnprintf.o)
 .comment       0x0000017d       0x4f c:/program files (x86)/microchip/xc32/v1.21/bin/../lib/gcc/pic32mx/4.5.2/../../../../pic32mx/lib/size\libc.a(ctypef.o)
                                 0x8c (size before relaxing)
 .comment       0x00000000       0x3d c:/program files (x86)/microchip/xc32/v1.21/bin/../lib/gcc/pic32mx/4.5.2/../../../../pic32mx/lib/size\libc.a(errno.o)
 .comment       0x00000000       0x3d c:/program files (x86)/microchip/xc32/v1.21/bin/../lib/gcc/pic32mx/4.5.2/../../../../pic32mx/lib/size\libc.a(strncmp.o)
 .comment       0x00000000       0x3d c:/program files (x86)/microchip/xc32/v1.21/bin/../lib/gcc/pic32mx/4.5.2/../../../../pic32mx/lib/size\libc.a(doprnt_cdnopsuxX.eo)
 .comment       0x00000000       0x3d c:/program files (x86)/microchip/xc32/v1.21/bin/../lib/gcc/pic32mx/4.5.2/../../../../pic32mx/lib/size\libc.a(doprnt.o)
 .comment       0x00000000       0x3d c:/program files (x86)/microchip/xc32/v1.21/bin/../lib/gcc/pic32mx/4.5.2/../../../../pic32mx/lib/size\libc.a(_fputc_simple.o)
 .comment       0x00000000       0x3d c:/program files (x86)/microchip/xc32/v1.21/bin/../lib/gcc/pic32mx/4.5.2/../../../../pic32mx/lib/size\libc.a(powersf.o)
 .comment       0x00000000       0x3d c:/program files (x86)/microchip/xc32/v1.21/bin/../lib/gcc/pic32mx/4.5.2/../../../../pic32mx/lib/size\libc.a(_iob.o)
 .comment       0x00000000       0x3d c:/program files (x86)/microchip/xc32/v1.21/bin/../lib/gcc/pic32mx/4.5.2/../../../../pic32mx/lib/size\libc.a(_flsbuf_simple.o)
 .comment       0x000001cc       0x4b c:/program files (x86)/microchip/xc32/v1.21/bin/../lib/gcc/pic32mx/4.5.2/../../../../pic32mx/lib/size\libpic32.a(sbrk.o)
                                 0x88 (size before relaxing)
 .comment       0x00000000       0x3d c:/program files (x86)/microchip/xc32/v1.21/bin/../lib/gcc/pic32mx/4.5.2/../../../../pic32mx/lib/size\libpic32.a(write.o)
 .comment       0x00000000       0x3d c:/program files (x86)/microchip/xc32/v1.21/bin/../lib/gcc/pic32mx/4.5.2/../../../../pic32mx/lib/size\libpic32.a(_mon_putc.o)
 .comment       0x00000000       0x3d c:/program files (x86)/microchip/xc32/v1.21/bin/../lib/gcc/pic32mx/4.5.2/../../../../pic32mx/lib/size\libpic32.a(xc32_uart.o)
 .comment       0x00000217       0x9e c:/program files (x86)/microchip/xc32/v1.21/bin/../lib/gcc/pic32mx/4.5.2/../../../../pic32mx/lib/size\libe.a(_floatdisf.o)
                                 0xdb (size before relaxing)
 .comment       0x00000000       0x3d c:/program files (x86)/microchip/xc32/v1.21/bin/../lib/gcc/pic32mx/4.5.2/size\libgcc.a(_lshrdi3.o)
 .comment       0x00000000       0x3d c:/program files (x86)/microchip/xc32/v1.21/bin/../lib/gcc/pic32mx/4.5.2/size\libgcc.a(_floatundisf.o)
 .comment       0x00000000       0x3d c:/program files (x86)/microchip/xc32/v1.21/bin/../lib/gcc/pic32mx/4.5.2/size\libgcc.a(_umoddi3.o)
 .comment       0x00000000       0x3d c:/program files (x86)/microchip/xc32/v1.21/bin/../lib/gcc/pic32mx/4.5.2/size\libgcc.a(floatunsisf.o)

.debug
 *(.debug)

.line
 *(.line)

.debug_srcinfo
 *(.debug_srcinfo)

.debug_sfnames
 *(.debug_sfnames)

.debug_aranges  0x00000000     0x2668
 *(.debug_aranges)
 .debug_aranges
                0x00000000       0x20 build/WiFIG/production/_ext/1293749816/bsp.o
 .debug_aranges
                0x00000020       0x60 build/WiFIG/production/_ext/101875047/hashes.o
 .debug_aranges
                0x00000080       0x28 build/WiFIG/production/_ext/101875047/lfsr.o
 .debug_aranges
                0x000000a8       0x80 build/WiFIG/production/_ext/101875047/big_int.o
 .debug_aranges
                0x00000128       0x20 build/WiFIG/production/_ext/101875047/big_int_helper_c32.o
 .debug_aranges
                0x00000148       0x58 build/WiFIG/production/_ext/101875047/helpers.o
 .debug_aranges
                0x000001a0       0x30 build/WiFIG/production/_ext/1472/ping_demo.o
 .debug_aranges
                0x000001d0      0x100 build/WiFIG/production/_ext/365611741/system_services.o
 .debug_aranges
                0x000002d0       0xa0 build/WiFIG/production/_ext/365611741/system_debug.o
 .debug_aranges
                0x00000370       0x40 build/WiFIG/production/_ext/365611741/system_random.o
 .debug_aranges
                0x000003b0       0x58 build/WiFIG/production/_ext/365611741/system_userio.o
 .debug_aranges
                0x00000408       0x50 build/WiFIG/production/_ext/792872985/usart.o
 .debug_aranges
                0x00000458       0x30 build/WiFIG/production/_ext/792872985/drv_spi.o
 .debug_aranges
                0x00000488       0x50 build/WiFIG/production/_ext/427700826/tcpip_announce.o
 .debug_aranges
                0x000004d8      0x138 build/WiFIG/production/_ext/427700826/arp.o
 .debug_aranges
                0x00000610       0xb0 build/WiFIG/production/_ext/427700826/dhcp.o
 .debug_aranges
                0x000006c0       0x30 build/WiFIG/production/_ext/427700826/dhcps.o
 .debug_aranges
                0x000006f0       0x70 build/WiFIG/production/_ext/427700826/dns.o
 .debug_aranges
                0x00000760       0x28 build/WiFIG/production/_ext/427700826/hash_fnv.o
 .debug_aranges
                0x00000788       0x58 build/WiFIG/production/_ext/427700826/hash_tbl.o
 .debug_aranges
                0x000007e0       0x50 build/WiFIG/production/_ext/427700826/icmp.o
 .debug_aranges
                0x00000830      0x150 build/WiFIG/production/_ext/427700826/ipv4.o
 .debug_aranges
                0x00000980       0x40 build/WiFIG/production/_ext/427700826/nbns.o
 .debug_aranges
                0x000009c0      0x288 build/WiFIG/production/_ext/427700826/tcp.o
 .debug_aranges
                0x00000c48       0x98 build/WiFIG/production/_ext/427700826/tcpip_heap_alloc.o
 .debug_aranges
                0x00000ce0      0x170 build/WiFIG/production/_ext/427700826/udp.o
 .debug_aranges
                0x00000e50       0xd8 build/WiFIG/production/_ext/427700826/tcpip_mac_object.o
 .debug_aranges
                0x00000f28      0x298 build/WiFIG/production/_ext/427700826/tcpip_manager.o
 .debug_aranges
                0x000011c0       0xe8 build/WiFIG/production/_ext/427700826/tcpip_helpers.o
 .debug_aranges
                0x000012a8       0x20 build/WiFIG/production/_ext/427700826/tcpip_helper_c32.o
 .debug_aranges
                0x000012c8       0x30 build/WiFIG/production/_ext/427700826/tcpip_notify.o
 .debug_aranges
                0x000012f8       0x30 build/WiFIG/production/_ext/427700826/zero_conf_link_local.o
 .debug_aranges
                0x00001328       0x30 build/WiFIG/production/_ext/334706090/wf_tx_power.o
 .debug_aranges
                0x00001358       0x40 build/WiFIG/production/_ext/334706090/wf_connect.o
 .debug_aranges
                0x00001398       0xa8 build/WiFIG/production/_ext/334706090/wf_connection_algorithm.o
 .debug_aranges
                0x00001440       0x50 build/WiFIG/production/_ext/334706090/wf_connection_manager.o
 .debug_aranges
                0x00001490       0xd8 build/WiFIG/production/_ext/334706090/wf_connection_profile.o
 .debug_aranges
                0x00001568       0x20 build/WiFIG/production/_ext/334706090/wf_easy_config.o
 .debug_aranges
                0x00001588       0x40 build/WiFIG/production/_ext/334706090/wf_eint.o
 .debug_aranges
                0x000015c8       0x68 build/WiFIG/production/_ext/334706090/wf_event_handler.o
 .debug_aranges
                0x00001630       0x40 build/WiFIG/production/_ext/334706090/wf_init.o
 .debug_aranges
                0x00001670       0x90 build/WiFIG/production/_ext/334706090/wf_power_save.o
 .debug_aranges
                0x00001700       0x30 build/WiFIG/production/_ext/334706090/wf_scan.o
 .debug_aranges
                0x00001730       0x40 build/WiFIG/production/_ext/334706090/wf_spi.o
 .debug_aranges
                0x00001770      0x108 build/WiFIG/production/_ext/334706090/mrf24w_mac_pic32.o
 .debug_aranges
                0x00001878       0x70 build/WiFIG/production/_ext/334706090/mrf24w_events.o
 .debug_aranges
                0x000018e8       0xb8 build/WiFIG/production/_ext/334706090/wf_debug_output.o
 .debug_aranges
                0x000019a0       0x90 build/WiFIG/production/_ext/334706090/wf_commands.o
 .debug_aranges
                0x00001a30       0xd8 build/WiFIG/production/_ext/334706090/wf_driver_com_24g.o
 .debug_aranges
                0x00001b08       0xc0 build/WiFIG/production/_ext/334706090/wf_driver_raw_24g.o
 .debug_aranges
                0x00001bc8      0x110 build/WiFIG/production/_ext/334706090/wf_mac_24g.o
 .debug_aranges
                0x00001cd8       0x40 build/WiFIG/production/_ext/334706090/wf_mgmt_msg_24g.o
 .debug_aranges
                0x00001d18       0xe8 build/WiFIG/production/_ext/334706090/wf_param_msg_24g.o
 .debug_aranges
                0x00001e00       0x38 build/WiFIG/production/_ext/334706090/wf_configData.o
 .debug_aranges
                0x00001e38       0x38 build/WiFIG/production/_ext/1472/main_demo.o
 .debug_aranges
                0x00001e70       0x20 build/WiFIG/production/_ext/1472/wf_config.o
 .debug_aranges
                0x00001e90       0x40 build/WiFIG/production/_ext/1472/tcp6_demo_app.o
 .debug_aranges
                0x00001ed0       0x20 c:/program files (x86)/microchip/xc32/v1.21/bin/../lib/gcc/pic32mx/4.5.2/../../../../pic32mx/lib/size\libmchp_peripheral.a(open_core_timer_lib.o)
 .debug_aranges
                0x00001ef0       0x20 c:/program files (x86)/microchip/xc32/v1.21/bin/../lib/gcc/pic32mx/4.5.2/../../../../pic32mx/lib/size\libmchp_peripheral_32MX695F512H.a(soft_reset_lib.o)
 .debug_aranges
                0x00001f10       0x28 c:/program files (x86)/microchip/xc32/v1.21/bin/../lib/gcc/pic32mx/4.5.2/../../../../pic32mx/lib/size\libmchp_peripheral_32MX695F512H.a(pcache.o)
 .debug_aranges
                0x00001f38       0x20 c:/program files (x86)/microchip/xc32/v1.21/bin/../lib/gcc/pic32mx/4.5.2/../../../../pic32mx/lib/size\libmchp_peripheral_32MX695F512H.a(int_disable_interrupts_lib.o)
 .debug_aranges
                0x00001f58       0x20 c:/program files (x86)/microchip/xc32/v1.21/bin/../lib/gcc/pic32mx/4.5.2/../../../../pic32mx/lib/size\libmchp_peripheral_32MX695F512H.a(int_restore_interrupts_lib.o)
 .debug_aranges
                0x00001f78       0x20 c:/program files (x86)/microchip/xc32/v1.21/bin/../lib/gcc/pic32mx/4.5.2/../../../../pic32mx/lib/size\libmchp_peripheral_32MX695F512H.a(int_enable_mv_int_lib.o)
 .debug_aranges
                0x00001f98       0x60 c:/program files (x86)/microchip/xc32/v1.21/bin/../lib/gcc/pic32mx/4.5.2/../../../../pic32mx/lib/size\libmchp_peripheral_32MX695F512H.a(int_tbl_lib.o)
 .debug_aranges
                0x00001ff8       0x20 c:/program files (x86)/microchip/xc32/v1.21/bin/../lib/gcc/pic32mx/4.5.2/../../../../pic32mx/lib/size\libmchp_peripheral_32MX695F512H.a(rtcc_init_lib.o)
 .debug_aranges
                0x00002018       0x20 c:/program files (x86)/microchip/xc32/v1.21/bin/../lib/gcc/pic32mx/4.5.2/../../../../pic32mx/lib/size\libmchp_peripheral_32MX695F512H.a(rtcc_open_lib.o)
 .debug_aranges
                0x00002038       0x20 c:/program files (x86)/microchip/xc32/v1.21/bin/../lib/gcc/pic32mx/4.5.2/../../../../pic32mx/lib/size\libmchp_peripheral_32MX695F512H.a(spi_chn_data_rdy_lib.o)
 .debug_aranges
                0x00002058       0x28 c:/program files (x86)/microchip/xc32/v1.21/bin/../lib/gcc/pic32mx/4.5.2/../../../../pic32mx/lib/size\libmchp_peripheral_32MX695F512H.a(spi_chn_getc_lib.o)
 .debug_aranges
                0x00002080       0x20 c:/program files (x86)/microchip/xc32/v1.21/bin/../lib/gcc/pic32mx/4.5.2/../../../../pic32mx/lib/size\libmchp_peripheral_32MX695F512H.a(spi_chn_open_lib.o)
 .debug_aranges
                0x000020a0       0x30 c:/program files (x86)/microchip/xc32/v1.21/bin/../lib/gcc/pic32mx/4.5.2/../../../../pic32mx/lib/size\libmchp_peripheral_32MX695F512H.a(spi_chn_putc_lib.o)
 .debug_aranges
                0x000020d0       0x20 c:/program files (x86)/microchip/xc32/v1.21/bin/../lib/gcc/pic32mx/4.5.2/../../../../pic32mx/lib/size\libmchp_peripheral_32MX695F512H.a(spi_chn_tx_buff_empty_lib.o)
 .debug_aranges
                0x000020f0       0x20 c:/program files (x86)/microchip/xc32/v1.21/bin/../lib/gcc/pic32mx/4.5.2/../../../../pic32mx/lib/size\libmchp_peripheral_32MX695F512H.a(port_set_pins_digital_in_lib.o)
 .debug_aranges
                0x00002110       0x20 c:/program files (x86)/microchip/xc32/v1.21/bin/../lib/gcc/pic32mx/4.5.2/../../../../pic32mx/lib/size\libmchp_peripheral_32MX695F512H.a(port_set_pins_digital_out_lib.o)
 .debug_aranges
                0x00002130       0x20 c:/program files (x86)/microchip/xc32/v1.21/bin/../lib/gcc/pic32mx/4.5.2/../../../../pic32mx/lib/size\libmchp_peripheral_32MX695F512H.a(int_enable_interrupts_lib.o)
 .debug_aranges
                0x00002150       0x28 c:/program files (x86)/microchip/xc32/v1.21/bin/../lib/gcc/pic32mx/4.5.2/../../../../pic32mx/lib/size\libmchp_peripheral_32MX695F512H.a(_rtcc_wait_clock_off_lib.o)
 .debug_aranges
                0x00002178       0x20 c:/program files (x86)/microchip/xc32/v1.21/bin/../lib/gcc/pic32mx/4.5.2/../../../../pic32mx/lib/size\libmchp_peripheral_32MX695F512H.a(read_core_timer_lib.o)
 .debug_aranges
                0x00002198       0x20 c:/program files (x86)/microchip/xc32/v1.21/bin/../lib/gcc/pic32mx/4.5.2/size\libgcc.a(_udivdi3.o)
 .debug_aranges
                0x000021b8       0x20 c:/program files (x86)/microchip/xc32/v1.21/bin/../lib/gcc/pic32mx/4.5.2/../../../../pic32mx/lib/size\libpic32.a(default-bootstrap-exception-handler.o)
 .debug_aranges
                0x000021d8       0x20 c:/program files (x86)/microchip/xc32/v1.21/bin/../lib/gcc/pic32mx/4.5.2/../../../../pic32mx/lib/size\libpic32.a(default-on-reset.o)
 .debug_aranges
                0x000021f8       0x20 c:/program files (x86)/microchip/xc32/v1.21/bin/../lib/gcc/pic32mx/4.5.2/../../../../pic32mx/lib/size\libpic32.a(default-on-bootstrap.o)
 .debug_aranges
                0x00002218       0x20 c:/program files (x86)/microchip/xc32/v1.21/bin/../lib/gcc/pic32mx/4.5.2/../../../../pic32mx/lib/size\libpic32.a(defaultinterrupt.o)
 .debug_aranges
                0x00002238       0x20 c:/program files (x86)/microchip/xc32/v1.21/bin/../lib/gcc/pic32mx/4.5.2/../../../../pic32mx/lib/size\libc.a(atoi.o)
 .debug_aranges
                0x00002258       0x30 c:/program files (x86)/microchip/xc32/v1.21/bin/../lib/gcc/pic32mx/4.5.2/../../../../pic32mx/lib/size\libc.a(malloc.o)
 .debug_aranges
                0x00002288       0x28 c:/program files (x86)/microchip/xc32/v1.21/bin/../lib/gcc/pic32mx/4.5.2/../../../../pic32mx/lib/size\libc.a(rand.o)
 .debug_aranges
                0x000022b0       0x20 c:/program files (x86)/microchip/xc32/v1.21/bin/../lib/gcc/pic32mx/4.5.2/../../../../pic32mx/lib/size\libc.a(strcat.o)
 .debug_aranges
                0x000022d0       0x20 c:/program files (x86)/microchip/xc32/v1.21/bin/../lib/gcc/pic32mx/4.5.2/../../../../pic32mx/lib/size\libc.a(strchr.o)
 .debug_aranges
                0x000022f0       0x20 c:/program files (x86)/microchip/xc32/v1.21/bin/../lib/gcc/pic32mx/4.5.2/../../../../pic32mx/lib/size\libc.a(strncat.o)
 .debug_aranges
                0x00002310       0x20 c:/program files (x86)/microchip/xc32/v1.21/bin/../lib/gcc/pic32mx/4.5.2/../../../../pic32mx/lib/size\libc.a(strncpy.o)
 .debug_aranges
                0x00002330       0x20 c:/program files (x86)/microchip/xc32/v1.21/bin/../lib/gcc/pic32mx/4.5.2/../../../../pic32mx/lib/size\libc.a(strstr.o)
 .debug_aranges
                0x00002350       0x28 c:/program files (x86)/microchip/xc32/v1.21/bin/../lib/gcc/pic32mx/4.5.2/../../../../pic32mx/lib/size\libc.a(strtol.o)
 .debug_aranges
                0x00002378       0x20 c:/program files (x86)/microchip/xc32/v1.21/bin/../lib/gcc/pic32mx/4.5.2/../../../../pic32mx/lib/size\libc.a(snprintf_cdnopsuxX.eo)
 .debug_aranges
                0x00002398       0x20 c:/program files (x86)/microchip/xc32/v1.21/bin/../lib/gcc/pic32mx/4.5.2/../../../../pic32mx/lib/size\libc.a(sprintf_cdnopsuxX.eo)
 .debug_aranges
                0x000023b8       0x20 c:/program files (x86)/microchip/xc32/v1.21/bin/../lib/gcc/pic32mx/4.5.2/../../../../pic32mx/lib/size\libc.a(vsnprintf_cdnopsuxX.eo)
 .debug_aranges
                0x000023d8       0x20 c:/program files (x86)/microchip/xc32/v1.21/bin/../lib/gcc/pic32mx/4.5.2/../../../../pic32mx/lib/size\libc.a(vsnprintf.o)
 .debug_aranges
                0x000023f8       0xa0 c:/program files (x86)/microchip/xc32/v1.21/bin/../lib/gcc/pic32mx/4.5.2/../../../../pic32mx/lib/size\libc.a(ctypef.o)
 .debug_aranges
                0x00002498       0x20 c:/program files (x86)/microchip/xc32/v1.21/bin/../lib/gcc/pic32mx/4.5.2/../../../../pic32mx/lib/size\libc.a(strncmp.o)
 .debug_aranges
                0x000024b8       0x20 c:/program files (x86)/microchip/xc32/v1.21/bin/../lib/gcc/pic32mx/4.5.2/../../../../pic32mx/lib/size\libc.a(doprnt_cdnopsuxX.eo)
 .debug_aranges
                0x000024d8       0x30 c:/program files (x86)/microchip/xc32/v1.21/bin/../lib/gcc/pic32mx/4.5.2/../../../../pic32mx/lib/size\libc.a(doprnt.o)
 .debug_aranges
                0x00002508       0x20 c:/program files (x86)/microchip/xc32/v1.21/bin/../lib/gcc/pic32mx/4.5.2/../../../../pic32mx/lib/size\libc.a(_fputc_simple.o)
 .debug_aranges
                0x00002528       0x20 c:/program files (x86)/microchip/xc32/v1.21/bin/../lib/gcc/pic32mx/4.5.2/../../../../pic32mx/lib/size\libc.a(_flsbuf_simple.o)
 .debug_aranges
                0x00002548       0x40 c:/program files (x86)/microchip/xc32/v1.21/bin/../lib/gcc/pic32mx/4.5.2/../../../../pic32mx/lib/size\libpic32.a(sbrk.o)
 .debug_aranges
                0x00002588       0x20 c:/program files (x86)/microchip/xc32/v1.21/bin/../lib/gcc/pic32mx/4.5.2/../../../../pic32mx/lib/size\libpic32.a(write.o)
 .debug_aranges
                0x000025a8       0x20 c:/program files (x86)/microchip/xc32/v1.21/bin/../lib/gcc/pic32mx/4.5.2/../../../../pic32mx/lib/size\libpic32.a(_mon_putc.o)
 .debug_aranges
                0x000025c8       0x20 c:/program files (x86)/microchip/xc32/v1.21/bin/../lib/gcc/pic32mx/4.5.2/../../../../pic32mx/lib/size\libe.a(_floatdisf.o)
 .debug_aranges
                0x000025e8       0x20 c:/program files (x86)/microchip/xc32/v1.21/bin/../lib/gcc/pic32mx/4.5.2/size\libgcc.a(_lshrdi3.o)
 .debug_aranges
                0x00002608       0x20 c:/program files (x86)/microchip/xc32/v1.21/bin/../lib/gcc/pic32mx/4.5.2/size\libgcc.a(_floatundisf.o)
 .debug_aranges
                0x00002628       0x20 c:/program files (x86)/microchip/xc32/v1.21/bin/../lib/gcc/pic32mx/4.5.2/size\libgcc.a(_umoddi3.o)
 .debug_aranges
                0x00002648       0x20 c:/program files (x86)/microchip/xc32/v1.21/bin/../lib/gcc/pic32mx/4.5.2/size\libgcc.a(floatunsisf.o)

.debug_pubnames
                0x00000000     0x4c31
 *(.debug_pubnames)
 .debug_pubnames
                0x00000000       0x25 build/WiFIG/production/_ext/1293749816/bsp.o
 .debug_pubnames
                0x00000025       0x97 build/WiFIG/production/_ext/101875047/hashes.o
 .debug_pubnames
                0x000000bc       0x30 build/WiFIG/production/_ext/101875047/lfsr.o
 .debug_pubnames
                0x000000ec       0xeb build/WiFIG/production/_ext/101875047/big_int.o
 .debug_pubnames
                0x000001d7       0x81 build/WiFIG/production/_ext/101875047/helpers.o
 .debug_pubnames
                0x00000258       0xc4 build/WiFIG/production/_ext/1472/ping_demo.o
 .debug_pubnames
                0x0000031c      0x393 build/WiFIG/production/_ext/365611741/system_services.o
 .debug_pubnames
                0x000006af      0x168 build/WiFIG/production/_ext/365611741/system_debug.o
 .debug_pubnames
                0x00000817       0x83 build/WiFIG/production/_ext/365611741/system_random.o
 .debug_pubnames
                0x0000089a       0xc8 build/WiFIG/production/_ext/365611741/system_userio.o
 .debug_pubnames
                0x00000962       0x94 build/WiFIG/production/_ext/792872985/usart.o
 .debug_pubnames
                0x000009f6       0x3a build/WiFIG/production/_ext/792872985/drv_spi.o
 .debug_pubnames
                0x00000a30       0x93 build/WiFIG/production/_ext/427700826/tcpip_announce.o
 .debug_pubnames
                0x00000ac3      0x1ba build/WiFIG/production/_ext/427700826/arp.o
 .debug_pubnames
                0x00000c7d       0xfb build/WiFIG/production/_ext/427700826/dhcp.o
 .debug_pubnames
                0x00000d78       0x55 build/WiFIG/production/_ext/427700826/dhcps.o
 .debug_pubnames
                0x00000dcd       0x8d build/WiFIG/production/_ext/427700826/dns.o
 .debug_pubnames
                0x00000e5a       0x33 build/WiFIG/production/_ext/427700826/hash_fnv.o
 .debug_pubnames
                0x00000e8d       0x86 build/WiFIG/production/_ext/427700826/hash_tbl.o
 .debug_pubnames
                0x00000f13       0x7e build/WiFIG/production/_ext/427700826/icmp.o
 .debug_pubnames
                0x00000f91      0x47f build/WiFIG/production/_ext/427700826/ipv4.o
 .debug_pubnames
                0x00001410       0x3b build/WiFIG/production/_ext/427700826/nbns.o
 .debug_pubnames
                0x0000144b      0x2b3 build/WiFIG/production/_ext/427700826/tcp.o
 .debug_pubnames
                0x000016fe      0x18c build/WiFIG/production/_ext/427700826/tcpip_heap_alloc.o
 .debug_pubnames
                0x0000188a      0x25a build/WiFIG/production/_ext/427700826/udp.o
 .debug_pubnames
                0x00001ae4      0x1f9 build/WiFIG/production/_ext/427700826/tcpip_mac_object.o
 .debug_pubnames
                0x00001cdd      0x781 build/WiFIG/production/_ext/427700826/tcpip_manager.o
 .debug_pubnames
                0x0000245e      0x2e1 build/WiFIG/production/_ext/427700826/tcpip_helpers.o
 .debug_pubnames
                0x0000273f       0x69 build/WiFIG/production/_ext/427700826/tcpip_notify.o
 .debug_pubnames
                0x000027a8       0x43 build/WiFIG/production/_ext/427700826/zero_conf_link_local.o
 .debug_pubnames
                0x000027eb       0x58 build/WiFIG/production/_ext/334706090/wf_tx_power.o
 .debug_pubnames
                0x00002843       0x23 build/WiFIG/production/_ext/334706090/wf_connect.o
 .debug_pubnames
                0x00002866      0x175 build/WiFIG/production/_ext/334706090/wf_connection_algorithm.o
 .debug_pubnames
                0x000029db       0x96 build/WiFIG/production/_ext/334706090/wf_connection_manager.o
 .debug_pubnames
                0x00002a71      0x1ad build/WiFIG/production/_ext/334706090/wf_connection_profile.o
 .debug_pubnames
                0x00002c1e       0x3b build/WiFIG/production/_ext/334706090/wf_easy_config.o
 .debug_pubnames
                0x00002c59       0x72 build/WiFIG/production/_ext/334706090/wf_eint.o
 .debug_pubnames
                0x00002ccb       0xf9 build/WiFIG/production/_ext/334706090/wf_event_handler.o
 .debug_pubnames
                0x00002dc4       0x6d build/WiFIG/production/_ext/334706090/wf_init.o
 .debug_pubnames
                0x00002e31      0x149 build/WiFIG/production/_ext/334706090/wf_power_save.o
 .debug_pubnames
                0x00002f7a       0x4b build/WiFIG/production/_ext/334706090/wf_scan.o
 .debug_pubnames
                0x00002fc5       0x67 build/WiFIG/production/_ext/334706090/wf_spi.o
 .debug_pubnames
                0x0000302c       0x87 build/WiFIG/production/_ext/334706090/mrf24w_mac_pic32.o
 .debug_pubnames
                0x000030b3      0x142 build/WiFIG/production/_ext/334706090/mrf24w_events.o
 .debug_pubnames
                0x000031f5      0x139 build/WiFIG/production/_ext/334706090/wf_debug_output.o
 .debug_pubnames
                0x0000332e       0x8a build/WiFIG/production/_ext/334706090/wf_commands.o
 .debug_pubnames
                0x000033b8      0x1f4 build/WiFIG/production/_ext/334706090/wf_driver_com_24g.o
 .debug_pubnames
                0x000035ac      0x1ef build/WiFIG/production/_ext/334706090/wf_driver_raw_24g.o
 .debug_pubnames
                0x0000379b      0x2ed build/WiFIG/production/_ext/334706090/wf_mac_24g.o
 .debug_pubnames
                0x00003a88       0xb0 build/WiFIG/production/_ext/334706090/wf_mgmt_msg_24g.o
 .debug_pubnames
                0x00003b38      0x26d build/WiFIG/production/_ext/334706090/wf_param_msg_24g.o
 .debug_pubnames
                0x00003da5       0x93 build/WiFIG/production/_ext/334706090/wf_configData.o
 .debug_pubnames
                0x00003e38      0x1cc build/WiFIG/production/_ext/1472/main_demo.o
 .debug_pubnames
                0x00004004       0x26 build/WiFIG/production/_ext/1472/wf_config.o
 .debug_pubnames
                0x0000402a      0x2e1 build/WiFIG/production/_ext/1472/tcp6_demo_app.o
 .debug_pubnames
                0x0000430b       0x24 c:/program files (x86)/microchip/xc32/v1.21/bin/../lib/gcc/pic32mx/4.5.2/../../../../pic32mx/lib/size\libmchp_peripheral.a(open_core_timer_lib.o)
 .debug_pubnames
                0x0000432f       0x20 c:/program files (x86)/microchip/xc32/v1.21/bin/../lib/gcc/pic32mx/4.5.2/../../../../pic32mx/lib/size\libmchp_peripheral_32MX695F512H.a(soft_reset_lib.o)
 .debug_pubnames
                0x0000434f       0x3b c:/program files (x86)/microchip/xc32/v1.21/bin/../lib/gcc/pic32mx/4.5.2/../../../../pic32mx/lib/size\libmchp_peripheral_32MX695F512H.a(pcache.o)
 .debug_pubnames
                0x0000438a       0x2b c:/program files (x86)/microchip/xc32/v1.21/bin/../lib/gcc/pic32mx/4.5.2/../../../../pic32mx/lib/size\libmchp_peripheral_32MX695F512H.a(int_disable_interrupts_lib.o)
 .debug_pubnames
                0x000043b5       0x2b c:/program files (x86)/microchip/xc32/v1.21/bin/../lib/gcc/pic32mx/4.5.2/../../../../pic32mx/lib/size\libmchp_peripheral_32MX695F512H.a(int_restore_interrupts_lib.o)
 .debug_pubnames
                0x000043e0       0x36 c:/program files (x86)/microchip/xc32/v1.21/bin/../lib/gcc/pic32mx/4.5.2/../../../../pic32mx/lib/size\libmchp_peripheral_32MX695F512H.a(int_enable_mv_int_lib.o)
 .debug_pubnames
                0x00004416       0xca c:/program files (x86)/microchip/xc32/v1.21/bin/../lib/gcc/pic32mx/4.5.2/../../../../pic32mx/lib/size\libmchp_peripheral_32MX695F512H.a(int_tbl_lib.o)
 .debug_pubnames
                0x000044e0       0x1f c:/program files (x86)/microchip/xc32/v1.21/bin/../lib/gcc/pic32mx/4.5.2/../../../../pic32mx/lib/size\libmchp_peripheral_32MX695F512H.a(rtcc_init_lib.o)
 .debug_pubnames
                0x000044ff       0x1f c:/program files (x86)/microchip/xc32/v1.21/bin/../lib/gcc/pic32mx/4.5.2/../../../../pic32mx/lib/size\libmchp_peripheral_32MX695F512H.a(rtcc_open_lib.o)
 .debug_pubnames
                0x0000451e       0x24 c:/program files (x86)/microchip/xc32/v1.21/bin/../lib/gcc/pic32mx/4.5.2/../../../../pic32mx/lib/size\libmchp_peripheral_32MX695F512H.a(spi_chn_data_rdy_lib.o)
 .debug_pubnames
                0x00004542       0x31 c:/program files (x86)/microchip/xc32/v1.21/bin/../lib/gcc/pic32mx/4.5.2/../../../../pic32mx/lib/size\libmchp_peripheral_32MX695F512H.a(spi_chn_getc_lib.o)
 .debug_pubnames
                0x00004573       0x21 c:/program files (x86)/microchip/xc32/v1.21/bin/../lib/gcc/pic32mx/4.5.2/../../../../pic32mx/lib/size\libmchp_peripheral_32MX695F512H.a(spi_chn_open_lib.o)
 .debug_pubnames
                0x00004594       0x43 c:/program files (x86)/microchip/xc32/v1.21/bin/../lib/gcc/pic32mx/4.5.2/../../../../pic32mx/lib/size\libmchp_peripheral_32MX695F512H.a(spi_chn_putc_lib.o)
 .debug_pubnames
                0x000045d7       0x28 c:/program files (x86)/microchip/xc32/v1.21/bin/../lib/gcc/pic32mx/4.5.2/../../../../pic32mx/lib/size\libmchp_peripheral_32MX695F512H.a(spi_chn_tx_buff_empty_lib.o)
 .debug_pubnames
                0x000045ff       0x2b c:/program files (x86)/microchip/xc32/v1.21/bin/../lib/gcc/pic32mx/4.5.2/../../../../pic32mx/lib/size\libmchp_peripheral_32MX695F512H.a(port_set_pins_digital_in_lib.o)
 .debug_pubnames
                0x0000462a       0x2c c:/program files (x86)/microchip/xc32/v1.21/bin/../lib/gcc/pic32mx/4.5.2/../../../../pic32mx/lib/size\libmchp_peripheral_32MX695F512H.a(port_set_pins_digital_out_lib.o)
 .debug_pubnames
                0x00004656       0x2a c:/program files (x86)/microchip/xc32/v1.21/bin/../lib/gcc/pic32mx/4.5.2/../../../../pic32mx/lib/size\libmchp_peripheral_32MX695F512H.a(int_enable_interrupts_lib.o)
 .debug_pubnames
                0x00004680       0x3e c:/program files (x86)/microchip/xc32/v1.21/bin/../lib/gcc/pic32mx/4.5.2/../../../../pic32mx/lib/size\libmchp_peripheral_32MX695F512H.a(_rtcc_wait_clock_off_lib.o)
 .debug_pubnames
                0x000046be       0x24 c:/program files (x86)/microchip/xc32/v1.21/bin/../lib/gcc/pic32mx/4.5.2/../../../../pic32mx/lib/size\libmchp_peripheral_32MX695F512H.a(read_core_timer_lib.o)
 .debug_pubnames
                0x000046e2       0x20 c:/program files (x86)/microchip/xc32/v1.21/bin/../lib/gcc/pic32mx/4.5.2/size\libgcc.a(_udivdi3.o)
 .debug_pubnames
                0x00004702       0x33 c:/program files (x86)/microchip/xc32/v1.21/bin/../lib/gcc/pic32mx/4.5.2/../../../../pic32mx/lib/size\libpic32.a(default-bootstrap-exception-handler.o)
 .debug_pubnames
                0x00004735       0x20 c:/program files (x86)/microchip/xc32/v1.21/bin/../lib/gcc/pic32mx/4.5.2/../../../../pic32mx/lib/size\libpic32.a(default-on-reset.o)
 .debug_pubnames
                0x00004755       0x24 c:/program files (x86)/microchip/xc32/v1.21/bin/../lib/gcc/pic32mx/4.5.2/../../../../pic32mx/lib/size\libpic32.a(default-on-bootstrap.o)
 .debug_pubnames
                0x00004779       0x28 c:/program files (x86)/microchip/xc32/v1.21/bin/../lib/gcc/pic32mx/4.5.2/../../../../pic32mx/lib/size\libpic32.a(defaultinterrupt.o)
 .debug_pubnames
                0x000047a1       0x1b c:/program files (x86)/microchip/xc32/v1.21/bin/../lib/gcc/pic32mx/4.5.2/../../../../pic32mx/lib/size\libc.a(atoi.o)
 .debug_pubnames
                0x000047bc       0x32 c:/program files (x86)/microchip/xc32/v1.21/bin/../lib/gcc/pic32mx/4.5.2/../../../../pic32mx/lib/size\libc.a(malloc.o)
 .debug_pubnames
                0x000047ee       0x25 c:/program files (x86)/microchip/xc32/v1.21/bin/../lib/gcc/pic32mx/4.5.2/../../../../pic32mx/lib/size\libc.a(rand.o)
 .debug_pubnames
                0x00004813       0x1d c:/program files (x86)/microchip/xc32/v1.21/bin/../lib/gcc/pic32mx/4.5.2/../../../../pic32mx/lib/size\libc.a(strcat.o)
 .debug_pubnames
                0x00004830       0x1d c:/program files (x86)/microchip/xc32/v1.21/bin/../lib/gcc/pic32mx/4.5.2/../../../../pic32mx/lib/size\libc.a(strchr.o)
 .debug_pubnames
                0x0000484d       0x1e c:/program files (x86)/microchip/xc32/v1.21/bin/../lib/gcc/pic32mx/4.5.2/../../../../pic32mx/lib/size\libc.a(strncat.o)
 .debug_pubnames
                0x0000486b       0x1e c:/program files (x86)/microchip/xc32/v1.21/bin/../lib/gcc/pic32mx/4.5.2/../../../../pic32mx/lib/size\libc.a(strncpy.o)
 .debug_pubnames
                0x00004889       0x1d c:/program files (x86)/microchip/xc32/v1.21/bin/../lib/gcc/pic32mx/4.5.2/../../../../pic32mx/lib/size\libc.a(strstr.o)
 .debug_pubnames
                0x000048a6       0x29 c:/program files (x86)/microchip/xc32/v1.21/bin/../lib/gcc/pic32mx/4.5.2/../../../../pic32mx/lib/size\libc.a(strtol.o)
 .debug_pubnames
                0x000048cf       0x2a c:/program files (x86)/microchip/xc32/v1.21/bin/../lib/gcc/pic32mx/4.5.2/../../../../pic32mx/lib/size\libc.a(snprintf_cdnopsuxX.eo)
 .debug_pubnames
                0x000048f9       0x29 c:/program files (x86)/microchip/xc32/v1.21/bin/../lib/gcc/pic32mx/4.5.2/../../../../pic32mx/lib/size\libc.a(sprintf_cdnopsuxX.eo)
 .debug_pubnames
                0x00004922       0x2b c:/program files (x86)/microchip/xc32/v1.21/bin/../lib/gcc/pic32mx/4.5.2/../../../../pic32mx/lib/size\libc.a(vsnprintf_cdnopsuxX.eo)
 .debug_pubnames
                0x0000494d       0x20 c:/program files (x86)/microchip/xc32/v1.21/bin/../lib/gcc/pic32mx/4.5.2/../../../../pic32mx/lib/size\libc.a(vsnprintf.o)
 .debug_pubnames
                0x0000496d       0xe1 c:/program files (x86)/microchip/xc32/v1.21/bin/../lib/gcc/pic32mx/4.5.2/../../../../pic32mx/lib/size\libc.a(ctypef.o)
 .debug_pubnames
                0x00004a4e       0x1e c:/program files (x86)/microchip/xc32/v1.21/bin/../lib/gcc/pic32mx/4.5.2/../../../../pic32mx/lib/size\libc.a(strncmp.o)
 .debug_pubnames
                0x00004a6c       0x2a c:/program files (x86)/microchip/xc32/v1.21/bin/../lib/gcc/pic32mx/4.5.2/../../../../pic32mx/lib/size\libc.a(doprnt_cdnopsuxX.eo)
 .debug_pubnames
                0x00004a96       0x1f c:/program files (x86)/microchip/xc32/v1.21/bin/../lib/gcc/pic32mx/4.5.2/../../../../pic32mx/lib/size\libc.a(doprnt.o)
 .debug_pubnames
                0x00004ab5       0x1c c:/program files (x86)/microchip/xc32/v1.21/bin/../lib/gcc/pic32mx/4.5.2/../../../../pic32mx/lib/size\libc.a(_fputc_simple.o)
 .debug_pubnames
                0x00004ad1       0x1e c:/program files (x86)/microchip/xc32/v1.21/bin/../lib/gcc/pic32mx/4.5.2/../../../../pic32mx/lib/size\libc.a(_flsbuf_simple.o)
 .debug_pubnames
                0x00004aef       0x5c c:/program files (x86)/microchip/xc32/v1.21/bin/../lib/gcc/pic32mx/4.5.2/../../../../pic32mx/lib/size\libpic32.a(sbrk.o)
 .debug_pubnames
                0x00004b4b       0x1c c:/program files (x86)/microchip/xc32/v1.21/bin/../lib/gcc/pic32mx/4.5.2/../../../../pic32mx/lib/size\libpic32.a(write.o)
 .debug_pubnames
                0x00004b67       0x20 c:/program files (x86)/microchip/xc32/v1.21/bin/../lib/gcc/pic32mx/4.5.2/../../../../pic32mx/lib/size\libpic32.a(_mon_putc.o)
 .debug_pubnames
                0x00004b87       0x22 c:/program files (x86)/microchip/xc32/v1.21/bin/../lib/gcc/pic32mx/4.5.2/../../../../pic32mx/lib/size\libe.a(_floatdisf.o)
 .debug_pubnames
                0x00004ba9       0x20 c:/program files (x86)/microchip/xc32/v1.21/bin/../lib/gcc/pic32mx/4.5.2/size\libgcc.a(_lshrdi3.o)
 .debug_pubnames
                0x00004bc9       0x24 c:/program files (x86)/microchip/xc32/v1.21/bin/../lib/gcc/pic32mx/4.5.2/size\libgcc.a(_floatundisf.o)
 .debug_pubnames
                0x00004bed       0x20 c:/program files (x86)/microchip/xc32/v1.21/bin/../lib/gcc/pic32mx/4.5.2/size\libgcc.a(_umoddi3.o)
 .debug_pubnames
                0x00004c0d       0x24 c:/program files (x86)/microchip/xc32/v1.21/bin/../lib/gcc/pic32mx/4.5.2/size\libgcc.a(floatunsisf.o)

.debug_info     0x00000000    0xa8249
 *(.debug_info .gnu.linkonce.wi.*)
 .debug_info    0x00000000     0x1702 build/WiFIG/production/_ext/1293749816/bsp.o
 .debug_info    0x00001702      0x827 build/WiFIG/production/_ext/101875047/hashes.o
 .debug_info    0x00001f29      0x21e build/WiFIG/production/_ext/101875047/lfsr.o
 .debug_info    0x00002147     0x173c build/WiFIG/production/_ext/101875047/big_int.o
 .debug_info    0x00003883       0xb8 build/WiFIG/production/_ext/101875047/big_int_helper_c32.o
 .debug_info    0x0000393b      0x510 build/WiFIG/production/_ext/101875047/helpers.o
 .debug_info    0x00003e4b        0x0 build/WiFIG/production/_ext/1472/berkeley_tcp_client_demo.o
 .debug_info    0x00003e4b        0x0 build/WiFIG/production/_ext/1472/berkeley_tcp_server_demo.o
 .debug_info    0x00003e4b        0x0 build/WiFIG/production/_ext/1472/berkeley_udp_client_demo.o
 .debug_info    0x00003e4b     0x11cb build/WiFIG/production/_ext/1472/generic_tcp_client.o
 .debug_info    0x00005016     0x11cb build/WiFIG/production/_ext/1472/generic_tcp_server.o
 .debug_info    0x000061e1     0x1a66 build/WiFIG/production/_ext/1472/ping_demo.o
 .debug_info    0x00007c47        0x0 build/WiFIG/production/_ext/1472/smtp_demo.o
 .debug_info    0x00007c47     0x3318 build/WiFIG/production/_ext/365611741/system_services.o
 .debug_info    0x0000af5f     0x15c7 build/WiFIG/production/_ext/365611741/system_debug.o
 .debug_info    0x0000c526     0x1c4f build/WiFIG/production/_ext/365611741/system_random.o
 .debug_info    0x0000e175      0xc15 build/WiFIG/production/_ext/365611741/system_command.o
 .debug_info    0x0000ed8a     0x20c0 build/WiFIG/production/_ext/365611741/system_userio.o
 .debug_info    0x00010e4a      0xc10 build/WiFIG/production/_ext/97638081/sys_fs.o
 .debug_info    0x00011a5a     0x1181 build/WiFIG/production/_ext/97638081/mpfs2.o
 .debug_info    0x00012bdb     0x166b build/WiFIG/production/_ext/792872985/usart.o
 .debug_info    0x00014246        0x0 build/WiFIG/production/_ext/792872985/lcd.o
 .debug_info    0x00014246     0x1682 build/WiFIG/production/_ext/792872985/drv_spi.o
 .debug_info    0x000158c8        0x0 build/WiFIG/production/_ext/792872985/db_appio.o
 .debug_info    0x000158c8     0x1188 build/WiFIG/production/_ext/792872985/spi_ram.o
 .debug_info    0x00016a50     0x118b build/WiFIG/production/_ext/792872985/spi_eeprom.o
 .debug_info    0x00017bdb     0x118a build/WiFIG/production/_ext/792872985/spi_flash.o
 .debug_info    0x00018d65     0x118a build/WiFIG/production/_ext/792872985/drv_media.o
 .debug_info    0x00019eef     0x2323 build/WiFIG/production/_ext/427700826/tcpip_announce.o
 .debug_info    0x0001c212     0x1387 build/WiFIG/production/_ext/427700826/http2.o
 .debug_info    0x0001d599     0x1389 build/WiFIG/production/_ext/427700826/arcfour.o
 .debug_info    0x0001e922     0x3c55 build/WiFIG/production/_ext/427700826/arp.o
 .debug_info    0x00022577     0x138e build/WiFIG/production/_ext/427700826/berkeley_api.o
 .debug_info    0x00023905     0x3838 build/WiFIG/production/_ext/427700826/dhcp.o
 .debug_info    0x0002713d     0x145c build/WiFIG/production/_ext/427700826/dhcps.o
 .debug_info    0x00028599     0x29d2 build/WiFIG/production/_ext/427700826/dns.o
 .debug_info    0x0002af6b     0x1386 build/WiFIG/production/_ext/427700826/dnss.o
 .debug_info    0x0002c2f1     0x1389 build/WiFIG/production/_ext/427700826/dyn_dns.o
 .debug_info    0x0002d67a     0x138b build/WiFIG/production/_ext/427700826/enc28_mac.o
 .debug_info    0x0002ea05     0x138a build/WiFIG/production/_ext/427700826/enc28j60.o
 .debug_info    0x0002fd8f     0x138c build/WiFIG/production/_ext/427700826/encs24j600.o
 .debug_info    0x0003111b     0x138c build/WiFIG/production/_ext/427700826/encx24_mac.o
 .debug_info    0x000324a7     0x1393 build/WiFIG/production/_ext/427700826/eth_pic32_ext_phy.o
 .debug_info    0x0003383a     0x139b build/WiFIG/production/_ext/427700826/eth_pic32_ext_phy_dp83848.o
 .debug_info    0x00034bd5     0x1393 build/WiFIG/production/_ext/427700826/eth_pic32_int_mac.o
 .debug_info    0x00035f68     0x1385 build/WiFIG/production/_ext/427700826/ftp.o
 .debug_info    0x000372ed      0x27a build/WiFIG/production/_ext/427700826/hash_fnv.o
 .debug_info    0x00037567      0x798 build/WiFIG/production/_ext/427700826/hash_tbl.o
 .debug_info    0x00037cff     0x279a build/WiFIG/production/_ext/427700826/icmp.o
 .debug_info    0x0003a499     0x1388 build/WiFIG/production/_ext/427700826/icmpv6.o
 .debug_info    0x0003b821     0x3baa build/WiFIG/production/_ext/427700826/ipv4.o
 .debug_info    0x0003f3cb     0x1386 build/WiFIG/production/_ext/427700826/ipv6.o
 .debug_info    0x00040751     0x1392 build/WiFIG/production/_ext/427700826/mac_events_pic32.o
 .debug_info    0x00041ae3     0x27c8 build/WiFIG/production/_ext/427700826/nbns.o
 .debug_info    0x000442ab     0x1385 build/WiFIG/production/_ext/427700826/ndp.o
 .debug_info    0x00045630     0x138e build/WiFIG/production/_ext/427700826/tcpip_reboot.o
 .debug_info    0x000469be     0x1385 build/WiFIG/production/_ext/427700826/rsa.o
 .debug_info    0x00047d43     0x1386 build/WiFIG/production/_ext/427700826/smtp.o
 .debug_info    0x000490c9     0x1386 build/WiFIG/production/_ext/427700826/snmp.o
 .debug_info    0x0004a44f     0x1388 build/WiFIG/production/_ext/427700826/snmpv3.o
 .debug_info    0x0004b7d7     0x138c build/WiFIG/production/_ext/427700826/snmpv3_usm.o
 .debug_info    0x0004cb63     0x1386 build/WiFIG/production/_ext/427700826/sntp.o
 .debug_info    0x0004dee9     0x1385 build/WiFIG/production/_ext/427700826/ssl.o
 .debug_info    0x0004f26e     0x58d6 build/WiFIG/production/_ext/427700826/tcp.o
 .debug_info    0x00054b44     0x1eee build/WiFIG/production/_ext/427700826/tcpip_heap_alloc.o
 .debug_info    0x00056a32     0x138f build/WiFIG/production/_ext/427700826/tcpip_storage.o
 .debug_info    0x00057dc1     0x1388 build/WiFIG/production/_ext/427700826/telnet.o
 .debug_info    0x00059149     0x1387 build/WiFIG/production/_ext/427700826/tftpc.o
 .debug_info    0x0005a4d0     0x4272 build/WiFIG/production/_ext/427700826/udp.o
 .debug_info    0x0005e742     0x2221 build/WiFIG/production/_ext/427700826/tcpip_mac_object.o
 .debug_info    0x00060963     0x52a1 build/WiFIG/production/_ext/427700826/tcpip_manager.o
 .debug_info    0x00065c04     0x2658 build/WiFIG/production/_ext/427700826/tcpip_helpers.o
 .debug_info    0x0006825c     0x1390 build/WiFIG/production/_ext/427700826/tcpip_commands.o
 .debug_info    0x000695ec     0x1387 build/WiFIG/production/_ext/427700826/iperf.o
 .debug_info    0x0006a973       0xb5 build/WiFIG/production/_ext/427700826/tcpip_helper_c32.o
 .debug_info    0x0006aa28      0x38d build/WiFIG/production/_ext/427700826/tcpip_notify.o
 .debug_info    0x0006adb5     0x1392 build/WiFIG/production/_ext/427700826/zero_conf_helper.o
 .debug_info    0x0006c147     0x1453 build/WiFIG/production/_ext/427700826/zero_conf_link_local.o
 .debug_info    0x0006d59a     0x1399 build/WiFIG/production/_ext/427700826/zero_conf_multicast_dns.o
 .debug_info    0x0006e933     0x1901 build/WiFIG/production/_ext/334706090/wf_tx_power.o
 .debug_info    0x00070234     0x1b4b build/WiFIG/production/_ext/334706090/wf_connect.o
 .debug_info    0x00071d7f     0x216b build/WiFIG/production/_ext/334706090/wf_connection_algorithm.o
 .debug_info    0x00073eea     0x2451 build/WiFIG/production/_ext/334706090/wf_connection_manager.o
 .debug_info    0x0007633b     0x264a build/WiFIG/production/_ext/334706090/wf_connection_profile.o
 .debug_info    0x00078985     0x17d4 build/WiFIG/production/_ext/334706090/wf_easy_config.o
 .debug_info    0x0007a159     0x1f29 build/WiFIG/production/_ext/334706090/wf_eint.o
 .debug_info    0x0007c082     0x1a9e build/WiFIG/production/_ext/334706090/wf_event_handler.o
 .debug_info    0x0007db20     0x1c95 build/WiFIG/production/_ext/334706090/wf_init.o
 .debug_info    0x0007f7b5     0x1ee3 build/WiFIG/production/_ext/334706090/wf_power_save.o
 .debug_info    0x00081698     0x207f build/WiFIG/production/_ext/334706090/wf_scan.o
 .debug_info    0x00083717     0x1a0f build/WiFIG/production/_ext/334706090/wf_spi.o
 .debug_info    0x00085126     0x3423 build/WiFIG/production/_ext/334706090/mrf24w_mac_pic32.o
 .debug_info    0x00088549     0x1dd8 build/WiFIG/production/_ext/334706090/mrf24w_events.o
 .debug_info    0x0008a321     0x2906 build/WiFIG/production/_ext/334706090/wf_debug_output.o
 .debug_info    0x0008cc27     0x2288 build/WiFIG/production/_ext/334706090/wf_commands.o
 .debug_info    0x0008eeaf     0x1390 build/WiFIG/production/_ext/334706090/wf_pbkdf2.o
 .debug_info    0x0009023f     0x2837 build/WiFIG/production/_ext/334706090/wf_driver_com_24g.o
 .debug_info    0x00092a76     0x1dc8 build/WiFIG/production/_ext/334706090/wf_driver_raw_24g.o
 .debug_info    0x0009483e     0x2704 build/WiFIG/production/_ext/334706090/wf_mac_24g.o
 .debug_info    0x00096f42     0x1ead build/WiFIG/production/_ext/334706090/wf_mgmt_msg_24g.o
 .debug_info    0x00098def     0x292e build/WiFIG/production/_ext/334706090/wf_param_msg_24g.o
 .debug_info    0x0009b71d     0x1c65 build/WiFIG/production/_ext/334706090/wf_configData.o
 .debug_info    0x0009d382     0x273e build/WiFIG/production/_ext/1472/main_demo.o
 .debug_info    0x0009fac0        0x0 build/WiFIG/production/_ext/1472/custom_snmp_app.o
 .debug_info    0x0009fac0        0x0 build/WiFIG/production/_ext/1472/custom_ssl_cert.o
 .debug_info    0x0009fac0     0x116b build/WiFIG/production/_ext/1472/mpfs_img2.o
 .debug_info    0x000a0c2b     0x1401 build/WiFIG/production/_ext/1472/wf_config.o
 .debug_info    0x000a202c        0x0 build/WiFIG/production/_ext/1472/custom_http_app.o
 .debug_info    0x000a202c     0x2612 build/WiFIG/production/_ext/1472/tcp6_demo_app.o
 .debug_info    0x000a463e       0xaa c:/program files (x86)/microchip/xc32/v1.21/bin/../lib/gcc/pic32mx/4.5.2/../../../../pic32mx/lib/size\libmchp_peripheral.a(open_core_timer_lib.o)
 .debug_info    0x000a46e8       0xb2 c:/program files (x86)/microchip/xc32/v1.21/bin/../lib/gcc/pic32mx/4.5.2/../../../../pic32mx/lib/size\libmchp_peripheral_32MX695F512H.a(soft_reset_lib.o)
 .debug_info    0x000a479a       0xbf c:/program files (x86)/microchip/xc32/v1.21/bin/../lib/gcc/pic32mx/4.5.2/../../../../pic32mx/lib/size\libmchp_peripheral_32MX695F512H.a(pcache.o)
 .debug_info    0x000a4859       0xb6 c:/program files (x86)/microchip/xc32/v1.21/bin/../lib/gcc/pic32mx/4.5.2/../../../../pic32mx/lib/size\libmchp_peripheral_32MX695F512H.a(int_disable_interrupts_lib.o)
 .debug_info    0x000a490f       0xb6 c:/program files (x86)/microchip/xc32/v1.21/bin/../lib/gcc/pic32mx/4.5.2/../../../../pic32mx/lib/size\libmchp_peripheral_32MX695F512H.a(int_restore_interrupts_lib.o)
 .debug_info    0x000a49c5       0xbc c:/program files (x86)/microchip/xc32/v1.21/bin/../lib/gcc/pic32mx/4.5.2/../../../../pic32mx/lib/size\libmchp_peripheral_32MX695F512H.a(int_enable_mv_int_lib.o)
 .debug_info    0x000a4a81      0x196 c:/program files (x86)/microchip/xc32/v1.21/bin/../lib/gcc/pic32mx/4.5.2/../../../../pic32mx/lib/size\libmchp_peripheral_32MX695F512H.a(int_tbl_lib.o)
 .debug_info    0x000a4c17      0x10c c:/program files (x86)/microchip/xc32/v1.21/bin/../lib/gcc/pic32mx/4.5.2/../../../../pic32mx/lib/size\libmchp_peripheral_32MX695F512H.a(rtcc_init_lib.o)
 .debug_info    0x000a4d23      0x10c c:/program files (x86)/microchip/xc32/v1.21/bin/../lib/gcc/pic32mx/4.5.2/../../../../pic32mx/lib/size\libmchp_peripheral_32MX695F512H.a(rtcc_open_lib.o)
 .debug_info    0x000a4e2f       0xbc c:/program files (x86)/microchip/xc32/v1.21/bin/../lib/gcc/pic32mx/4.5.2/../../../../pic32mx/lib/size\libmchp_peripheral_32MX695F512H.a(spi_chn_data_rdy_lib.o)
 .debug_info    0x000a4eeb       0xcf c:/program files (x86)/microchip/xc32/v1.21/bin/../lib/gcc/pic32mx/4.5.2/../../../../pic32mx/lib/size\libmchp_peripheral_32MX695F512H.a(spi_chn_getc_lib.o)
 .debug_info    0x000a4fba       0xa2 c:/program files (x86)/microchip/xc32/v1.21/bin/../lib/gcc/pic32mx/4.5.2/../../../../pic32mx/lib/size\libmchp_peripheral_32MX695F512H.a(spi_chn_open_lib.o)
 .debug_info    0x000a505c       0xeb c:/program files (x86)/microchip/xc32/v1.21/bin/../lib/gcc/pic32mx/4.5.2/../../../../pic32mx/lib/size\libmchp_peripheral_32MX695F512H.a(spi_chn_putc_lib.o)
 .debug_info    0x000a5147       0xb2 c:/program files (x86)/microchip/xc32/v1.21/bin/../lib/gcc/pic32mx/4.5.2/../../../../pic32mx/lib/size\libmchp_peripheral_32MX695F512H.a(spi_chn_tx_buff_empty_lib.o)
 .debug_info    0x000a51f9        0x0 c:/program files (x86)/microchip/xc32/v1.21/bin/../lib/gcc/pic32mx/4.5.2/../../../../pic32mx/lib/size\libmchp_peripheral_32MX695F512H.a(spi_io_tbl_libp.o)
 .debug_info    0x000a51f9        0x0 c:/program files (x86)/microchip/xc32/v1.21/bin/../lib/gcc/pic32mx/4.5.2/../../../../pic32mx/lib/size\libmchp_peripheral_32MX695F512H.a(spi_map_tbl_libp.o)
 .debug_info    0x000a51f9       0xba c:/program files (x86)/microchip/xc32/v1.21/bin/../lib/gcc/pic32mx/4.5.2/../../../../pic32mx/lib/size\libmchp_peripheral_32MX695F512H.a(port_set_pins_digital_in_lib.o)
 .debug_info    0x000a52b3       0xbc c:/program files (x86)/microchip/xc32/v1.21/bin/../lib/gcc/pic32mx/4.5.2/../../../../pic32mx/lib/size\libmchp_peripheral_32MX695F512H.a(port_set_pins_digital_out_lib.o)
 .debug_info    0x000a536f        0x0 c:/program files (x86)/microchip/xc32/v1.21/bin/../lib/gcc/pic32mx/4.5.2/../../../../pic32mx/lib/size\libmchp_peripheral_32MX695F512H.a(_ports_tbl_libp.o)
 .debug_info    0x000a536f       0xb4 c:/program files (x86)/microchip/xc32/v1.21/bin/../lib/gcc/pic32mx/4.5.2/../../../../pic32mx/lib/size\libmchp_peripheral_32MX695F512H.a(int_enable_interrupts_lib.o)
 .debug_info    0x000a5423       0xe7 c:/program files (x86)/microchip/xc32/v1.21/bin/../lib/gcc/pic32mx/4.5.2/../../../../pic32mx/lib/size\libmchp_peripheral_32MX695F512H.a(_rtcc_wait_clock_off_lib.o)
 .debug_info    0x000a550a       0xaa c:/program files (x86)/microchip/xc32/v1.21/bin/../lib/gcc/pic32mx/4.5.2/../../../../pic32mx/lib/size\libmchp_peripheral_32MX695F512H.a(read_core_timer_lib.o)
 .debug_info    0x000a55b4      0x760 c:/program files (x86)/microchip/xc32/v1.21/bin/../lib/gcc/pic32mx/4.5.2/size\libgcc.a(_udivdi3.o)
 .debug_info    0x000a5d14       0xe8 c:/program files (x86)/microchip/xc32/v1.21/bin/../lib/gcc/pic32mx/4.5.2/../../../../pic32mx/lib/size\libpic32.a(default-bootstrap-exception-handler.o)
 .debug_info    0x000a5dfc       0xc2 c:/program files (x86)/microchip/xc32/v1.21/bin/../lib/gcc/pic32mx/4.5.2/../../../../pic32mx/lib/size\libpic32.a(default-on-reset.o)
 .debug_info    0x000a5ebe       0xca c:/program files (x86)/microchip/xc32/v1.21/bin/../lib/gcc/pic32mx/4.5.2/../../../../pic32mx/lib/size\libpic32.a(default-on-bootstrap.o)
 .debug_info    0x000a5f88       0xdc c:/program files (x86)/microchip/xc32/v1.21/bin/../lib/gcc/pic32mx/4.5.2/../../../../pic32mx/lib/size\libpic32.a(defaultinterrupt.o)
 .debug_info    0x000a6064       0xb3 c:/program files (x86)/microchip/xc32/v1.21/bin/../lib/gcc/pic32mx/4.5.2/../../../../pic32mx/lib/size\libc.a(atoi.o)
 .debug_info    0x000a6117        0x0 c:/program files (x86)/microchip/xc32/v1.21/bin/../lib/gcc/pic32mx/4.5.2/../../../../pic32mx/lib/size\libc.a(ctype.o)
 .debug_info    0x000a6117       0xe0 c:/program files (x86)/microchip/xc32/v1.21/bin/../lib/gcc/pic32mx/4.5.2/../../../../pic32mx/lib/size\libc.a(malloc.o)
 .debug_info    0x000a61f7       0xc7 c:/program files (x86)/microchip/xc32/v1.21/bin/../lib/gcc/pic32mx/4.5.2/../../../../pic32mx/lib/size\libc.a(rand.o)
 .debug_info    0x000a62be       0xb7 c:/program files (x86)/microchip/xc32/v1.21/bin/../lib/gcc/pic32mx/4.5.2/../../../../pic32mx/lib/size\libc.a(strcat.o)
 .debug_info    0x000a6375       0xb7 c:/program files (x86)/microchip/xc32/v1.21/bin/../lib/gcc/pic32mx/4.5.2/../../../../pic32mx/lib/size\libc.a(strchr.o)
 .debug_info    0x000a642c       0xb9 c:/program files (x86)/microchip/xc32/v1.21/bin/../lib/gcc/pic32mx/4.5.2/../../../../pic32mx/lib/size\libc.a(strncat.o)
 .debug_info    0x000a64e5       0xb9 c:/program files (x86)/microchip/xc32/v1.21/bin/../lib/gcc/pic32mx/4.5.2/../../../../pic32mx/lib/size\libc.a(strncpy.o)
 .debug_info    0x000a659e       0xb7 c:/program files (x86)/microchip/xc32/v1.21/bin/../lib/gcc/pic32mx/4.5.2/../../../../pic32mx/lib/size\libc.a(strstr.o)
 .debug_info    0x000a6655       0xcd c:/program files (x86)/microchip/xc32/v1.21/bin/../lib/gcc/pic32mx/4.5.2/../../../../pic32mx/lib/size\libc.a(strtol.o)
 .debug_info    0x000a6722       0xc6 c:/program files (x86)/microchip/xc32/v1.21/bin/../lib/gcc/pic32mx/4.5.2/../../../../pic32mx/lib/size\libc.a(snprintf_cdnopsuxX.eo)
 .debug_info    0x000a67e8       0xc4 c:/program files (x86)/microchip/xc32/v1.21/bin/../lib/gcc/pic32mx/4.5.2/../../../../pic32mx/lib/size\libc.a(sprintf_cdnopsuxX.eo)
 .debug_info    0x000a68ac       0xc8 c:/program files (x86)/microchip/xc32/v1.21/bin/../lib/gcc/pic32mx/4.5.2/../../../../pic32mx/lib/size\libc.a(vsnprintf_cdnopsuxX.eo)
 .debug_info    0x000a6974       0xbd c:/program files (x86)/microchip/xc32/v1.21/bin/../lib/gcc/pic32mx/4.5.2/../../../../pic32mx/lib/size\libc.a(vsnprintf.o)
 .debug_info    0x000a6a31      0x21b c:/program files (x86)/microchip/xc32/v1.21/bin/../lib/gcc/pic32mx/4.5.2/../../../../pic32mx/lib/size\libc.a(ctypef.o)
 .debug_info    0x000a6c4c        0x0 c:/program files (x86)/microchip/xc32/v1.21/bin/../lib/gcc/pic32mx/4.5.2/../../../../pic32mx/lib/size\libc.a(errno.o)
 .debug_info    0x000a6c4c       0xb9 c:/program files (x86)/microchip/xc32/v1.21/bin/../lib/gcc/pic32mx/4.5.2/../../../../pic32mx/lib/size\libc.a(strncmp.o)
 .debug_info    0x000a6d05       0xc5 c:/program files (x86)/microchip/xc32/v1.21/bin/../lib/gcc/pic32mx/4.5.2/../../../../pic32mx/lib/size\libc.a(doprnt_cdnopsuxX.eo)
 .debug_info    0x000a6dca       0xe3 c:/program files (x86)/microchip/xc32/v1.21/bin/../lib/gcc/pic32mx/4.5.2/../../../../pic32mx/lib/size\libc.a(doprnt.o)
 .debug_info    0x000a6ead       0xb5 c:/program files (x86)/microchip/xc32/v1.21/bin/../lib/gcc/pic32mx/4.5.2/../../../../pic32mx/lib/size\libc.a(_fputc_simple.o)
 .debug_info    0x000a6f62        0x0 c:/program files (x86)/microchip/xc32/v1.21/bin/../lib/gcc/pic32mx/4.5.2/../../../../pic32mx/lib/size\libc.a(powersf.o)
 .debug_info    0x000a6f62        0x0 c:/program files (x86)/microchip/xc32/v1.21/bin/../lib/gcc/pic32mx/4.5.2/../../../../pic32mx/lib/size\libc.a(_iob.o)
 .debug_info    0x000a6f62       0xb8 c:/program files (x86)/microchip/xc32/v1.21/bin/../lib/gcc/pic32mx/4.5.2/../../../../pic32mx/lib/size\libc.a(_flsbuf_simple.o)
 .debug_info    0x000a701a      0x11b c:/program files (x86)/microchip/xc32/v1.21/bin/../lib/gcc/pic32mx/4.5.2/../../../../pic32mx/lib/size\libpic32.a(sbrk.o)
 .debug_info    0x000a7135       0xb3 c:/program files (x86)/microchip/xc32/v1.21/bin/../lib/gcc/pic32mx/4.5.2/../../../../pic32mx/lib/size\libpic32.a(write.o)
 .debug_info    0x000a71e8       0xbb c:/program files (x86)/microchip/xc32/v1.21/bin/../lib/gcc/pic32mx/4.5.2/../../../../pic32mx/lib/size\libpic32.a(_mon_putc.o)
 .debug_info    0x000a72a3        0x0 c:/program files (x86)/microchip/xc32/v1.21/bin/../lib/gcc/pic32mx/4.5.2/../../../../pic32mx/lib/size\libpic32.a(xc32_uart.o)
 .debug_info    0x000a72a3       0xd1 c:/program files (x86)/microchip/xc32/v1.21/bin/../lib/gcc/pic32mx/4.5.2/../../../../pic32mx/lib/size\libe.a(_floatdisf.o)
 .debug_info    0x000a7374      0x326 c:/program files (x86)/microchip/xc32/v1.21/bin/../lib/gcc/pic32mx/4.5.2/size\libgcc.a(_lshrdi3.o)
 .debug_info    0x000a769a      0x2ad c:/program files (x86)/microchip/xc32/v1.21/bin/../lib/gcc/pic32mx/4.5.2/size\libgcc.a(_floatundisf.o)
 .debug_info    0x000a7947      0x79d c:/program files (x86)/microchip/xc32/v1.21/bin/../lib/gcc/pic32mx/4.5.2/size\libgcc.a(_umoddi3.o)
 .debug_info    0x000a80e4      0x165 c:/program files (x86)/microchip/xc32/v1.21/bin/../lib/gcc/pic32mx/4.5.2/size\libgcc.a(floatunsisf.o)

.debug_abbrev   0x00000000     0xd3eb
 *(.debug_abbrev)
 .debug_abbrev  0x00000000      0x17d build/WiFIG/production/_ext/1293749816/bsp.o
 .debug_abbrev  0x0000017d      0x18e build/WiFIG/production/_ext/101875047/hashes.o
 .debug_abbrev  0x0000030b       0x65 build/WiFIG/production/_ext/101875047/lfsr.o
 .debug_abbrev  0x00000370      0x218 build/WiFIG/production/_ext/101875047/big_int.o
 .debug_abbrev  0x00000588       0x14 build/WiFIG/production/_ext/101875047/big_int_helper_c32.o
 .debug_abbrev  0x0000059c       0xfd build/WiFIG/production/_ext/101875047/helpers.o
 .debug_abbrev  0x00000699        0x1 build/WiFIG/production/_ext/1472/berkeley_tcp_client_demo.o
 .debug_abbrev  0x0000069a        0x1 build/WiFIG/production/_ext/1472/berkeley_tcp_server_demo.o
 .debug_abbrev  0x0000069b        0x1 build/WiFIG/production/_ext/1472/berkeley_udp_client_demo.o
 .debug_abbrev  0x0000069c      0x166 build/WiFIG/production/_ext/1472/generic_tcp_client.o
 .debug_abbrev  0x00000802      0x166 build/WiFIG/production/_ext/1472/generic_tcp_server.o
 .debug_abbrev  0x00000968      0x265 build/WiFIG/production/_ext/1472/ping_demo.o
 .debug_abbrev  0x00000bcd        0x1 build/WiFIG/production/_ext/1472/smtp_demo.o
 .debug_abbrev  0x00000bce      0x3ff build/WiFIG/production/_ext/365611741/system_services.o
 .debug_abbrev  0x00000fcd      0x2d8 build/WiFIG/production/_ext/365611741/system_debug.o
 .debug_abbrev  0x000012a5      0x230 build/WiFIG/production/_ext/365611741/system_random.o
 .debug_abbrev  0x000014d5      0x139 build/WiFIG/production/_ext/365611741/system_command.o
 .debug_abbrev  0x0000160e      0x26c build/WiFIG/production/_ext/365611741/system_userio.o
 .debug_abbrev  0x0000187a      0x139 build/WiFIG/production/_ext/97638081/sys_fs.o
 .debug_abbrev  0x000019b3      0x166 build/WiFIG/production/_ext/97638081/mpfs2.o
 .debug_abbrev  0x00001b19      0x218 build/WiFIG/production/_ext/792872985/usart.o
 .debug_abbrev  0x00001d31        0x1 build/WiFIG/production/_ext/792872985/lcd.o
 .debug_abbrev  0x00001d32      0x1e1 build/WiFIG/production/_ext/792872985/drv_spi.o
 .debug_abbrev  0x00001f13        0x1 build/WiFIG/production/_ext/792872985/db_appio.o
 .debug_abbrev  0x00001f14      0x166 build/WiFIG/production/_ext/792872985/spi_ram.o
 .debug_abbrev  0x0000207a      0x166 build/WiFIG/production/_ext/792872985/spi_eeprom.o
 .debug_abbrev  0x000021e0      0x166 build/WiFIG/production/_ext/792872985/spi_flash.o
 .debug_abbrev  0x00002346      0x166 build/WiFIG/production/_ext/792872985/drv_media.o
 .debug_abbrev  0x000024ac      0x36c build/WiFIG/production/_ext/427700826/tcpip_announce.o
 .debug_abbrev  0x00002818      0x18b build/WiFIG/production/_ext/427700826/http2.o
 .debug_abbrev  0x000029a3      0x18b build/WiFIG/production/_ext/427700826/arcfour.o
 .debug_abbrev  0x00002b2e      0x3f8 build/WiFIG/production/_ext/427700826/arp.o
 .debug_abbrev  0x00002f26      0x18b build/WiFIG/production/_ext/427700826/berkeley_api.o
 .debug_abbrev  0x000030b1      0x3a3 build/WiFIG/production/_ext/427700826/dhcp.o
 .debug_abbrev  0x00003454      0x1ba build/WiFIG/production/_ext/427700826/dhcps.o
 .debug_abbrev  0x0000360e      0x36c build/WiFIG/production/_ext/427700826/dns.o
 .debug_abbrev  0x0000397a      0x18b build/WiFIG/production/_ext/427700826/dnss.o
 .debug_abbrev  0x00003b05      0x18b build/WiFIG/production/_ext/427700826/dyn_dns.o
 .debug_abbrev  0x00003c90      0x18b build/WiFIG/production/_ext/427700826/enc28_mac.o
 .debug_abbrev  0x00003e1b      0x18b build/WiFIG/production/_ext/427700826/enc28j60.o
 .debug_abbrev  0x00003fa6      0x18b build/WiFIG/production/_ext/427700826/encs24j600.o
 .debug_abbrev  0x00004131      0x18b build/WiFIG/production/_ext/427700826/encx24_mac.o
 .debug_abbrev  0x000042bc      0x18b build/WiFIG/production/_ext/427700826/eth_pic32_ext_phy.o
 .debug_abbrev  0x00004447      0x18b build/WiFIG/production/_ext/427700826/eth_pic32_ext_phy_dp83848.o
 .debug_abbrev  0x000045d2      0x18b build/WiFIG/production/_ext/427700826/eth_pic32_int_mac.o
 .debug_abbrev  0x0000475d      0x18b build/WiFIG/production/_ext/427700826/ftp.o
 .debug_abbrev  0x000048e8       0x8c build/WiFIG/production/_ext/427700826/hash_fnv.o
 .debug_abbrev  0x00004974      0x1ca build/WiFIG/production/_ext/427700826/hash_tbl.o
 .debug_abbrev  0x00004b3e      0x2ff build/WiFIG/production/_ext/427700826/icmp.o
 .debug_abbrev  0x00004e3d      0x18b build/WiFIG/production/_ext/427700826/icmpv6.o
 .debug_abbrev  0x00004fc8      0x3c7 build/WiFIG/production/_ext/427700826/ipv4.o
 .debug_abbrev  0x0000538f      0x18b build/WiFIG/production/_ext/427700826/ipv6.o
 .debug_abbrev  0x0000551a      0x18b build/WiFIG/production/_ext/427700826/mac_events_pic32.o
 .debug_abbrev  0x000056a5      0x2c2 build/WiFIG/production/_ext/427700826/nbns.o
 .debug_abbrev  0x00005967      0x18b build/WiFIG/production/_ext/427700826/ndp.o
 .debug_abbrev  0x00005af2      0x18b build/WiFIG/production/_ext/427700826/tcpip_reboot.o
 .debug_abbrev  0x00005c7d      0x18b build/WiFIG/production/_ext/427700826/rsa.o
 .debug_abbrev  0x00005e08      0x18b build/WiFIG/production/_ext/427700826/smtp.o
 .debug_abbrev  0x00005f93      0x18b build/WiFIG/production/_ext/427700826/snmp.o
 .debug_abbrev  0x0000611e      0x18b build/WiFIG/production/_ext/427700826/snmpv3.o
 .debug_abbrev  0x000062a9      0x18b build/WiFIG/production/_ext/427700826/snmpv3_usm.o
 .debug_abbrev  0x00006434      0x18b build/WiFIG/production/_ext/427700826/sntp.o
 .debug_abbrev  0x000065bf      0x18b build/WiFIG/production/_ext/427700826/ssl.o
 .debug_abbrev  0x0000674a      0x39d build/WiFIG/production/_ext/427700826/tcp.o
 .debug_abbrev  0x00006ae7      0x295 build/WiFIG/production/_ext/427700826/tcpip_heap_alloc.o
 .debug_abbrev  0x00006d7c      0x18b build/WiFIG/production/_ext/427700826/tcpip_storage.o
 .debug_abbrev  0x00006f07      0x18b build/WiFIG/production/_ext/427700826/telnet.o
 .debug_abbrev  0x00007092      0x18b build/WiFIG/production/_ext/427700826/tftpc.o
 .debug_abbrev  0x0000721d      0x3ad build/WiFIG/production/_ext/427700826/udp.o
 .debug_abbrev  0x000075ca      0x22e build/WiFIG/production/_ext/427700826/tcpip_mac_object.o
 .debug_abbrev  0x000077f8      0x3d5 build/WiFIG/production/_ext/427700826/tcpip_manager.o
 .debug_abbrev  0x00007bcd      0x28d build/WiFIG/production/_ext/427700826/tcpip_helpers.o
 .debug_abbrev  0x00007e5a      0x18b build/WiFIG/production/_ext/427700826/tcpip_commands.o
 .debug_abbrev  0x00007fe5      0x18b build/WiFIG/production/_ext/427700826/iperf.o
 .debug_abbrev  0x00008170       0x14 build/WiFIG/production/_ext/427700826/tcpip_helper_c32.o
 .debug_abbrev  0x00008184       0xd9 build/WiFIG/production/_ext/427700826/tcpip_notify.o
 .debug_abbrev  0x0000825d      0x18b build/WiFIG/production/_ext/427700826/zero_conf_helper.o
 .debug_abbrev  0x000083e8      0x1ba build/WiFIG/production/_ext/427700826/zero_conf_link_local.o
 .debug_abbrev  0x000085a2      0x18b build/WiFIG/production/_ext/427700826/zero_conf_multicast_dns.o
 .debug_abbrev  0x0000872d      0x1da build/WiFIG/production/_ext/334706090/wf_tx_power.o
 .debug_abbrev  0x00008907      0x267 build/WiFIG/production/_ext/334706090/wf_connect.o
 .debug_abbrev  0x00008b6e      0x277 build/WiFIG/production/_ext/334706090/wf_connection_algorithm.o
 .debug_abbrev  0x00008de5      0x263 build/WiFIG/production/_ext/334706090/wf_connection_manager.o
 .debug_abbrev  0x00009048      0x2d5 build/WiFIG/production/_ext/334706090/wf_connection_profile.o
 .debug_abbrev  0x0000931d      0x1d2 build/WiFIG/production/_ext/334706090/wf_easy_config.o
 .debug_abbrev  0x000094ef      0x1b9 build/WiFIG/production/_ext/334706090/wf_eint.o
 .debug_abbrev  0x000096a8      0x2a8 build/WiFIG/production/_ext/334706090/wf_event_handler.o
 .debug_abbrev  0x00009950      0x284 build/WiFIG/production/_ext/334706090/wf_init.o
 .debug_abbrev  0x00009bd4      0x29b build/WiFIG/production/_ext/334706090/wf_power_save.o
 .debug_abbrev  0x00009e6f      0x21e build/WiFIG/production/_ext/334706090/wf_scan.o
 .debug_abbrev  0x0000a08d      0x22a build/WiFIG/production/_ext/334706090/wf_spi.o
 .debug_abbrev  0x0000a2b7      0x310 build/WiFIG/production/_ext/334706090/mrf24w_mac_pic32.o
 .debug_abbrev  0x0000a5c7      0x259 build/WiFIG/production/_ext/334706090/mrf24w_events.o
 .debug_abbrev  0x0000a820      0x316 build/WiFIG/production/_ext/334706090/wf_debug_output.o
 .debug_abbrev  0x0000ab36      0x2f8 build/WiFIG/production/_ext/334706090/wf_commands.o
 .debug_abbrev  0x0000ae2e      0x18b build/WiFIG/production/_ext/334706090/wf_pbkdf2.o
 .debug_abbrev  0x0000afb9      0x37a build/WiFIG/production/_ext/334706090/wf_driver_com_24g.o
 .debug_abbrev  0x0000b333      0x281 build/WiFIG/production/_ext/334706090/wf_driver_raw_24g.o
 .debug_abbrev  0x0000b5b4      0x356 build/WiFIG/production/_ext/334706090/wf_mac_24g.o
 .debug_abbrev  0x0000b90a      0x24e build/WiFIG/production/_ext/334706090/wf_mgmt_msg_24g.o
 .debug_abbrev  0x0000bb58      0x267 build/WiFIG/production/_ext/334706090/wf_param_msg_24g.o
 .debug_abbrev  0x0000bdbf      0x271 build/WiFIG/production/_ext/334706090/wf_configData.o
 .debug_abbrev  0x0000c030      0x281 build/WiFIG/production/_ext/1472/main_demo.o
 .debug_abbrev  0x0000c2b1        0x1 build/WiFIG/production/_ext/1472/custom_snmp_app.o
 .debug_abbrev  0x0000c2b2        0x1 build/WiFIG/production/_ext/1472/custom_ssl_cert.o
 .debug_abbrev  0x0000c2b3      0x166 build/WiFIG/production/_ext/1472/mpfs_img2.o
 .debug_abbrev  0x0000c419      0x1bc build/WiFIG/production/_ext/1472/wf_config.o
 .debug_abbrev  0x0000c5d5        0x1 build/WiFIG/production/_ext/1472/custom_http_app.o
 .debug_abbrev  0x0000c5d6      0x25d build/WiFIG/production/_ext/1472/tcp6_demo_app.o
 .debug_abbrev  0x0000c833       0x25 c:/program files (x86)/microchip/xc32/v1.21/bin/../lib/gcc/pic32mx/4.5.2/../../../../pic32mx/lib/size\libmchp_peripheral.a(open_core_timer_lib.o)
 .debug_abbrev  0x0000c858       0x34 c:/program files (x86)/microchip/xc32/v1.21/bin/../lib/gcc/pic32mx/4.5.2/../../../../pic32mx/lib/size\libmchp_peripheral_32MX695F512H.a(soft_reset_lib.o)
 .debug_abbrev  0x0000c88c       0x25 c:/program files (x86)/microchip/xc32/v1.21/bin/../lib/gcc/pic32mx/4.5.2/../../../../pic32mx/lib/size\libmchp_peripheral_32MX695F512H.a(pcache.o)
 .debug_abbrev  0x0000c8b1       0x25 c:/program files (x86)/microchip/xc32/v1.21/bin/../lib/gcc/pic32mx/4.5.2/../../../../pic32mx/lib/size\libmchp_peripheral_32MX695F512H.a(int_disable_interrupts_lib.o)
 .debug_abbrev  0x0000c8d6       0x25 c:/program files (x86)/microchip/xc32/v1.21/bin/../lib/gcc/pic32mx/4.5.2/../../../../pic32mx/lib/size\libmchp_peripheral_32MX695F512H.a(int_restore_interrupts_lib.o)
 .debug_abbrev  0x0000c8fb       0x25 c:/program files (x86)/microchip/xc32/v1.21/bin/../lib/gcc/pic32mx/4.5.2/../../../../pic32mx/lib/size\libmchp_peripheral_32MX695F512H.a(int_enable_mv_int_lib.o)
 .debug_abbrev  0x0000c920       0x25 c:/program files (x86)/microchip/xc32/v1.21/bin/../lib/gcc/pic32mx/4.5.2/../../../../pic32mx/lib/size\libmchp_peripheral_32MX695F512H.a(int_tbl_lib.o)
 .debug_abbrev  0x0000c945       0x41 c:/program files (x86)/microchip/xc32/v1.21/bin/../lib/gcc/pic32mx/4.5.2/../../../../pic32mx/lib/size\libmchp_peripheral_32MX695F512H.a(rtcc_init_lib.o)
 .debug_abbrev  0x0000c986       0x41 c:/program files (x86)/microchip/xc32/v1.21/bin/../lib/gcc/pic32mx/4.5.2/../../../../pic32mx/lib/size\libmchp_peripheral_32MX695F512H.a(rtcc_open_lib.o)
 .debug_abbrev  0x0000c9c7       0x34 c:/program files (x86)/microchip/xc32/v1.21/bin/../lib/gcc/pic32mx/4.5.2/../../../../pic32mx/lib/size\libmchp_peripheral_32MX695F512H.a(spi_chn_data_rdy_lib.o)
 .debug_abbrev  0x0000c9fb       0x34 c:/program files (x86)/microchip/xc32/v1.21/bin/../lib/gcc/pic32mx/4.5.2/../../../../pic32mx/lib/size\libmchp_peripheral_32MX695F512H.a(spi_chn_getc_lib.o)
 .debug_abbrev  0x0000ca2f       0x25 c:/program files (x86)/microchip/xc32/v1.21/bin/../lib/gcc/pic32mx/4.5.2/../../../../pic32mx/lib/size\libmchp_peripheral_32MX695F512H.a(spi_chn_open_lib.o)
 .debug_abbrev  0x0000ca54       0x34 c:/program files (x86)/microchip/xc32/v1.21/bin/../lib/gcc/pic32mx/4.5.2/../../../../pic32mx/lib/size\libmchp_peripheral_32MX695F512H.a(spi_chn_putc_lib.o)
 .debug_abbrev  0x0000ca88       0x25 c:/program files (x86)/microchip/xc32/v1.21/bin/../lib/gcc/pic32mx/4.5.2/../../../../pic32mx/lib/size\libmchp_peripheral_32MX695F512H.a(spi_chn_tx_buff_empty_lib.o)
 .debug_abbrev  0x0000caad        0x1 c:/program files (x86)/microchip/xc32/v1.21/bin/../lib/gcc/pic32mx/4.5.2/../../../../pic32mx/lib/size\libmchp_peripheral_32MX695F512H.a(spi_io_tbl_libp.o)
 .debug_abbrev  0x0000caae        0x1 c:/program files (x86)/microchip/xc32/v1.21/bin/../lib/gcc/pic32mx/4.5.2/../../../../pic32mx/lib/size\libmchp_peripheral_32MX695F512H.a(spi_map_tbl_libp.o)
 .debug_abbrev  0x0000caaf       0x25 c:/program files (x86)/microchip/xc32/v1.21/bin/../lib/gcc/pic32mx/4.5.2/../../../../pic32mx/lib/size\libmchp_peripheral_32MX695F512H.a(port_set_pins_digital_in_lib.o)
 .debug_abbrev  0x0000cad4       0x25 c:/program files (x86)/microchip/xc32/v1.21/bin/../lib/gcc/pic32mx/4.5.2/../../../../pic32mx/lib/size\libmchp_peripheral_32MX695F512H.a(port_set_pins_digital_out_lib.o)
 .debug_abbrev  0x0000caf9        0x1 c:/program files (x86)/microchip/xc32/v1.21/bin/../lib/gcc/pic32mx/4.5.2/../../../../pic32mx/lib/size\libmchp_peripheral_32MX695F512H.a(_ports_tbl_libp.o)
 .debug_abbrev  0x0000cafa       0x25 c:/program files (x86)/microchip/xc32/v1.21/bin/../lib/gcc/pic32mx/4.5.2/../../../../pic32mx/lib/size\libmchp_peripheral_32MX695F512H.a(int_enable_interrupts_lib.o)
 .debug_abbrev  0x0000cb1f       0x34 c:/program files (x86)/microchip/xc32/v1.21/bin/../lib/gcc/pic32mx/4.5.2/../../../../pic32mx/lib/size\libmchp_peripheral_32MX695F512H.a(_rtcc_wait_clock_off_lib.o)
 .debug_abbrev  0x0000cb53       0x25 c:/program files (x86)/microchip/xc32/v1.21/bin/../lib/gcc/pic32mx/4.5.2/../../../../pic32mx/lib/size\libmchp_peripheral_32MX695F512H.a(read_core_timer_lib.o)
 .debug_abbrev  0x0000cb78      0x13d c:/program files (x86)/microchip/xc32/v1.21/bin/../lib/gcc/pic32mx/4.5.2/size\libgcc.a(_udivdi3.o)
 .debug_abbrev  0x0000ccb5       0x25 c:/program files (x86)/microchip/xc32/v1.21/bin/../lib/gcc/pic32mx/4.5.2/../../../../pic32mx/lib/size\libpic32.a(default-bootstrap-exception-handler.o)
 .debug_abbrev  0x0000ccda       0x25 c:/program files (x86)/microchip/xc32/v1.21/bin/../lib/gcc/pic32mx/4.5.2/../../../../pic32mx/lib/size\libpic32.a(default-on-reset.o)
 .debug_abbrev  0x0000ccff       0x25 c:/program files (x86)/microchip/xc32/v1.21/bin/../lib/gcc/pic32mx/4.5.2/../../../../pic32mx/lib/size\libpic32.a(default-on-bootstrap.o)
 .debug_abbrev  0x0000cd24       0x25 c:/program files (x86)/microchip/xc32/v1.21/bin/../lib/gcc/pic32mx/4.5.2/../../../../pic32mx/lib/size\libpic32.a(defaultinterrupt.o)
 .debug_abbrev  0x0000cd49       0x25 c:/program files (x86)/microchip/xc32/v1.21/bin/../lib/gcc/pic32mx/4.5.2/../../../../pic32mx/lib/size\libc.a(atoi.o)
 .debug_abbrev  0x0000cd6e        0x1 c:/program files (x86)/microchip/xc32/v1.21/bin/../lib/gcc/pic32mx/4.5.2/../../../../pic32mx/lib/size\libc.a(ctype.o)
 .debug_abbrev  0x0000cd6f       0x25 c:/program files (x86)/microchip/xc32/v1.21/bin/../lib/gcc/pic32mx/4.5.2/../../../../pic32mx/lib/size\libc.a(malloc.o)
 .debug_abbrev  0x0000cd94       0x25 c:/program files (x86)/microchip/xc32/v1.21/bin/../lib/gcc/pic32mx/4.5.2/../../../../pic32mx/lib/size\libc.a(rand.o)
 .debug_abbrev  0x0000cdb9       0x25 c:/program files (x86)/microchip/xc32/v1.21/bin/../lib/gcc/pic32mx/4.5.2/../../../../pic32mx/lib/size\libc.a(strcat.o)
 .debug_abbrev  0x0000cdde       0x25 c:/program files (x86)/microchip/xc32/v1.21/bin/../lib/gcc/pic32mx/4.5.2/../../../../pic32mx/lib/size\libc.a(strchr.o)
 .debug_abbrev  0x0000ce03       0x25 c:/program files (x86)/microchip/xc32/v1.21/bin/../lib/gcc/pic32mx/4.5.2/../../../../pic32mx/lib/size\libc.a(strncat.o)
 .debug_abbrev  0x0000ce28       0x25 c:/program files (x86)/microchip/xc32/v1.21/bin/../lib/gcc/pic32mx/4.5.2/../../../../pic32mx/lib/size\libc.a(strncpy.o)
 .debug_abbrev  0x0000ce4d       0x25 c:/program files (x86)/microchip/xc32/v1.21/bin/../lib/gcc/pic32mx/4.5.2/../../../../pic32mx/lib/size\libc.a(strstr.o)
 .debug_abbrev  0x0000ce72       0x25 c:/program files (x86)/microchip/xc32/v1.21/bin/../lib/gcc/pic32mx/4.5.2/../../../../pic32mx/lib/size\libc.a(strtol.o)
 .debug_abbrev  0x0000ce97       0x25 c:/program files (x86)/microchip/xc32/v1.21/bin/../lib/gcc/pic32mx/4.5.2/../../../../pic32mx/lib/size\libc.a(snprintf_cdnopsuxX.eo)
 .debug_abbrev  0x0000cebc       0x25 c:/program files (x86)/microchip/xc32/v1.21/bin/../lib/gcc/pic32mx/4.5.2/../../../../pic32mx/lib/size\libc.a(sprintf_cdnopsuxX.eo)
 .debug_abbrev  0x0000cee1       0x25 c:/program files (x86)/microchip/xc32/v1.21/bin/../lib/gcc/pic32mx/4.5.2/../../../../pic32mx/lib/size\libc.a(vsnprintf_cdnopsuxX.eo)
 .debug_abbrev  0x0000cf06       0x25 c:/program files (x86)/microchip/xc32/v1.21/bin/../lib/gcc/pic32mx/4.5.2/../../../../pic32mx/lib/size\libc.a(vsnprintf.o)
 .debug_abbrev  0x0000cf2b       0x25 c:/program files (x86)/microchip/xc32/v1.21/bin/../lib/gcc/pic32mx/4.5.2/../../../../pic32mx/lib/size\libc.a(ctypef.o)
 .debug_abbrev  0x0000cf50        0x1 c:/program files (x86)/microchip/xc32/v1.21/bin/../lib/gcc/pic32mx/4.5.2/../../../../pic32mx/lib/size\libc.a(errno.o)
 .debug_abbrev  0x0000cf51       0x25 c:/program files (x86)/microchip/xc32/v1.21/bin/../lib/gcc/pic32mx/4.5.2/../../../../pic32mx/lib/size\libc.a(strncmp.o)
 .debug_abbrev  0x0000cf76       0x25 c:/program files (x86)/microchip/xc32/v1.21/bin/../lib/gcc/pic32mx/4.5.2/../../../../pic32mx/lib/size\libc.a(doprnt_cdnopsuxX.eo)
 .debug_abbrev  0x0000cf9b       0x36 c:/program files (x86)/microchip/xc32/v1.21/bin/../lib/gcc/pic32mx/4.5.2/../../../../pic32mx/lib/size\libc.a(doprnt.o)
 .debug_abbrev  0x0000cfd1       0x25 c:/program files (x86)/microchip/xc32/v1.21/bin/../lib/gcc/pic32mx/4.5.2/../../../../pic32mx/lib/size\libc.a(_fputc_simple.o)
 .debug_abbrev  0x0000cff6        0x1 c:/program files (x86)/microchip/xc32/v1.21/bin/../lib/gcc/pic32mx/4.5.2/../../../../pic32mx/lib/size\libc.a(powersf.o)
 .debug_abbrev  0x0000cff7        0x1 c:/program files (x86)/microchip/xc32/v1.21/bin/../lib/gcc/pic32mx/4.5.2/../../../../pic32mx/lib/size\libc.a(_iob.o)
 .debug_abbrev  0x0000cff8       0x25 c:/program files (x86)/microchip/xc32/v1.21/bin/../lib/gcc/pic32mx/4.5.2/../../../../pic32mx/lib/size\libc.a(_flsbuf_simple.o)
 .debug_abbrev  0x0000d01d       0x38 c:/program files (x86)/microchip/xc32/v1.21/bin/../lib/gcc/pic32mx/4.5.2/../../../../pic32mx/lib/size\libpic32.a(sbrk.o)
 .debug_abbrev  0x0000d055       0x25 c:/program files (x86)/microchip/xc32/v1.21/bin/../lib/gcc/pic32mx/4.5.2/../../../../pic32mx/lib/size\libpic32.a(write.o)
 .debug_abbrev  0x0000d07a       0x25 c:/program files (x86)/microchip/xc32/v1.21/bin/../lib/gcc/pic32mx/4.5.2/../../../../pic32mx/lib/size\libpic32.a(_mon_putc.o)
 .debug_abbrev  0x0000d09f        0x1 c:/program files (x86)/microchip/xc32/v1.21/bin/../lib/gcc/pic32mx/4.5.2/../../../../pic32mx/lib/size\libpic32.a(xc32_uart.o)
 .debug_abbrev  0x0000d0a0       0x32 c:/program files (x86)/microchip/xc32/v1.21/bin/../lib/gcc/pic32mx/4.5.2/../../../../pic32mx/lib/size\libe.a(_floatdisf.o)
 .debug_abbrev  0x0000d0d2       0xe3 c:/program files (x86)/microchip/xc32/v1.21/bin/../lib/gcc/pic32mx/4.5.2/size\libgcc.a(_lshrdi3.o)
 .debug_abbrev  0x0000d1b5       0x79 c:/program files (x86)/microchip/xc32/v1.21/bin/../lib/gcc/pic32mx/4.5.2/size\libgcc.a(_floatundisf.o)
 .debug_abbrev  0x0000d22e      0x15c c:/program files (x86)/microchip/xc32/v1.21/bin/../lib/gcc/pic32mx/4.5.2/size\libgcc.a(_umoddi3.o)
 .debug_abbrev  0x0000d38a       0x61 c:/program files (x86)/microchip/xc32/v1.21/bin/../lib/gcc/pic32mx/4.5.2/size\libgcc.a(floatunsisf.o)

.debug_line     0x00000000    0x184b9
 *(.debug_line)
 .debug_line    0x00000000      0x1d6 build/WiFIG/production/_ext/1293749816/bsp.o
 .debug_line    0x000001d6      0x2e4 build/WiFIG/production/_ext/101875047/hashes.o
 .debug_line    0x000004ba       0xf0 build/WiFIG/production/_ext/101875047/lfsr.o
 .debug_line    0x000005aa      0x3eb build/WiFIG/production/_ext/101875047/big_int.o
 .debug_line    0x00000995      0x14f build/WiFIG/production/_ext/101875047/big_int_helper_c32.o
 .debug_line    0x00000ae4      0x24e build/WiFIG/production/_ext/101875047/helpers.o
 .debug_line    0x00000d32        0x0 build/WiFIG/production/_ext/1472/berkeley_tcp_client_demo.o
 .debug_line    0x00000d32        0x0 build/WiFIG/production/_ext/1472/berkeley_tcp_server_demo.o
 .debug_line    0x00000d32        0x0 build/WiFIG/production/_ext/1472/berkeley_udp_client_demo.o
 .debug_line    0x00000d32      0x1c5 build/WiFIG/production/_ext/1472/generic_tcp_client.o
 .debug_line    0x00000ef7      0x1c5 build/WiFIG/production/_ext/1472/generic_tcp_server.o
 .debug_line    0x000010bc      0x31e build/WiFIG/production/_ext/1472/ping_demo.o
 .debug_line    0x000013da        0x0 build/WiFIG/production/_ext/1472/smtp_demo.o
 .debug_line    0x000013da      0x6f4 build/WiFIG/production/_ext/365611741/system_services.o
 .debug_line    0x00001ace      0x3f8 build/WiFIG/production/_ext/365611741/system_debug.o
 .debug_line    0x00001ec6      0x35d build/WiFIG/production/_ext/365611741/system_random.o
 .debug_line    0x00002223       0xd1 build/WiFIG/production/_ext/365611741/system_command.o
 .debug_line    0x000022f4      0x387 build/WiFIG/production/_ext/365611741/system_userio.o
 .debug_line    0x0000267b       0xd1 build/WiFIG/production/_ext/97638081/sys_fs.o
 .debug_line    0x0000274c      0x18e build/WiFIG/production/_ext/97638081/mpfs2.o
 .debug_line    0x000028da      0x272 build/WiFIG/production/_ext/792872985/usart.o
 .debug_line    0x00002b4c        0x0 build/WiFIG/production/_ext/792872985/lcd.o
 .debug_line    0x00002b4c      0x2e9 build/WiFIG/production/_ext/792872985/drv_spi.o
 .debug_line    0x00002e35        0x0 build/WiFIG/production/_ext/792872985/db_appio.o
 .debug_line    0x00002e35      0x18e build/WiFIG/production/_ext/792872985/spi_ram.o
 .debug_line    0x00002fc3      0x18e build/WiFIG/production/_ext/792872985/spi_eeprom.o
 .debug_line    0x00003151      0x18e build/WiFIG/production/_ext/792872985/spi_flash.o
 .debug_line    0x000032df      0x18e build/WiFIG/production/_ext/792872985/drv_media.o
 .debug_line    0x0000346d      0x497 build/WiFIG/production/_ext/427700826/tcpip_announce.o
 .debug_line    0x00003904      0x230 build/WiFIG/production/_ext/427700826/http2.o
 .debug_line    0x00003b34      0x230 build/WiFIG/production/_ext/427700826/arcfour.o
 .debug_line    0x00003d64      0x920 build/WiFIG/production/_ext/427700826/arp.o
 .debug_line    0x00004684      0x230 build/WiFIG/production/_ext/427700826/berkeley_api.o
 .debug_line    0x000048b4      0x86e build/WiFIG/production/_ext/427700826/dhcp.o
 .debug_line    0x00005122      0x29a build/WiFIG/production/_ext/427700826/dhcps.o
 .debug_line    0x000053bc      0x662 build/WiFIG/production/_ext/427700826/dns.o
 .debug_line    0x00005a1e      0x230 build/WiFIG/production/_ext/427700826/dnss.o
 .debug_line    0x00005c4e      0x230 build/WiFIG/production/_ext/427700826/dyn_dns.o
 .debug_line    0x00005e7e      0x230 build/WiFIG/production/_ext/427700826/enc28_mac.o
 .debug_line    0x000060ae      0x230 build/WiFIG/production/_ext/427700826/enc28j60.o
 .debug_line    0x000062de      0x230 build/WiFIG/production/_ext/427700826/encs24j600.o
 .debug_line    0x0000650e      0x230 build/WiFIG/production/_ext/427700826/encx24_mac.o
 .debug_line    0x0000673e      0x230 build/WiFIG/production/_ext/427700826/eth_pic32_ext_phy.o
 .debug_line    0x0000696e      0x230 build/WiFIG/production/_ext/427700826/eth_pic32_ext_phy_dp83848.o
 .debug_line    0x00006b9e      0x230 build/WiFIG/production/_ext/427700826/eth_pic32_int_mac.o
 .debug_line    0x00006dce      0x230 build/WiFIG/production/_ext/427700826/ftp.o
 .debug_line    0x00006ffe      0x173 build/WiFIG/production/_ext/427700826/hash_fnv.o
 .debug_line    0x00007171      0x263 build/WiFIG/production/_ext/427700826/hash_tbl.o
 .debug_line    0x000073d4      0x411 build/WiFIG/production/_ext/427700826/icmp.o
 .debug_line    0x000077e5      0x230 build/WiFIG/production/_ext/427700826/icmpv6.o
 .debug_line    0x00007a15      0x89f build/WiFIG/production/_ext/427700826/ipv4.o
 .debug_line    0x000082b4      0x230 build/WiFIG/production/_ext/427700826/ipv6.o
 .debug_line    0x000084e4      0x230 build/WiFIG/production/_ext/427700826/mac_events_pic32.o
 .debug_line    0x00008714      0x4a3 build/WiFIG/production/_ext/427700826/nbns.o
 .debug_line    0x00008bb7      0x230 build/WiFIG/production/_ext/427700826/ndp.o
 .debug_line    0x00008de7      0x230 build/WiFIG/production/_ext/427700826/tcpip_reboot.o
 .debug_line    0x00009017      0x230 build/WiFIG/production/_ext/427700826/rsa.o
 .debug_line    0x00009247      0x230 build/WiFIG/production/_ext/427700826/smtp.o
 .debug_line    0x00009477      0x230 build/WiFIG/production/_ext/427700826/snmp.o
 .debug_line    0x000096a7      0x230 build/WiFIG/production/_ext/427700826/snmpv3.o
 .debug_line    0x000098d7      0x230 build/WiFIG/production/_ext/427700826/snmpv3_usm.o
 .debug_line    0x00009b07      0x230 build/WiFIG/production/_ext/427700826/sntp.o
 .debug_line    0x00009d37      0x230 build/WiFIG/production/_ext/427700826/ssl.o
 .debug_line    0x00009f67     0x1437 build/WiFIG/production/_ext/427700826/tcp.o
 .debug_line    0x0000b39e      0x536 build/WiFIG/production/_ext/427700826/tcpip_heap_alloc.o
 .debug_line    0x0000b8d4      0x230 build/WiFIG/production/_ext/427700826/tcpip_storage.o
 .debug_line    0x0000bb04      0x230 build/WiFIG/production/_ext/427700826/telnet.o
 .debug_line    0x0000bd34      0x230 build/WiFIG/production/_ext/427700826/tftpc.o
 .debug_line    0x0000bf64      0xa27 build/WiFIG/production/_ext/427700826/udp.o
 .debug_line    0x0000c98b      0x50b build/WiFIG/production/_ext/427700826/tcpip_mac_object.o
 .debug_line    0x0000ce96      0xedc build/WiFIG/production/_ext/427700826/tcpip_manager.o
 .debug_line    0x0000dd72      0x691 build/WiFIG/production/_ext/427700826/tcpip_helpers.o
 .debug_line    0x0000e403      0x230 build/WiFIG/production/_ext/427700826/tcpip_commands.o
 .debug_line    0x0000e633      0x230 build/WiFIG/production/_ext/427700826/iperf.o
 .debug_line    0x0000e863       0xee build/WiFIG/production/_ext/427700826/tcpip_helper_c32.o
 .debug_line    0x0000e951      0x120 build/WiFIG/production/_ext/427700826/tcpip_notify.o
 .debug_line    0x0000ea71      0x230 build/WiFIG/production/_ext/427700826/zero_conf_helper.o
 .debug_line    0x0000eca1      0x2a9 build/WiFIG/production/_ext/427700826/zero_conf_link_local.o
 .debug_line    0x0000ef4a      0x230 build/WiFIG/production/_ext/427700826/zero_conf_multicast_dns.o
 .debug_line    0x0000f17a      0x367 build/WiFIG/production/_ext/334706090/wf_tx_power.o
 .debug_line    0x0000f4e1      0x3a6 build/WiFIG/production/_ext/334706090/wf_connect.o
 .debug_line    0x0000f887      0x4ea build/WiFIG/production/_ext/334706090/wf_connection_algorithm.o
 .debug_line    0x0000fd71      0x3d6 build/WiFIG/production/_ext/334706090/wf_connection_manager.o
 .debug_line    0x00010147      0x59a build/WiFIG/production/_ext/334706090/wf_connection_profile.o
 .debug_line    0x000106e1      0x34a build/WiFIG/production/_ext/334706090/wf_easy_config.o
 .debug_line    0x00010a2b      0x2c0 build/WiFIG/production/_ext/334706090/wf_eint.o
 .debug_line    0x00010ceb      0x498 build/WiFIG/production/_ext/334706090/wf_event_handler.o
 .debug_line    0x00011183      0x3dc build/WiFIG/production/_ext/334706090/wf_init.o
 .debug_line    0x0001155f      0x46f build/WiFIG/production/_ext/334706090/wf_power_save.o
 .debug_line    0x000119ce      0x388 build/WiFIG/production/_ext/334706090/wf_scan.o
 .debug_line    0x00011d56      0x365 build/WiFIG/production/_ext/334706090/wf_spi.o
 .debug_line    0x000120bb      0x613 build/WiFIG/production/_ext/334706090/mrf24w_mac_pic32.o
 .debug_line    0x000126ce      0x42d build/WiFIG/production/_ext/334706090/mrf24w_events.o
 .debug_line    0x00012afb      0x623 build/WiFIG/production/_ext/334706090/wf_debug_output.o
 .debug_line    0x0001311e      0x626 build/WiFIG/production/_ext/334706090/wf_commands.o
 .debug_line    0x00013744      0x230 build/WiFIG/production/_ext/334706090/wf_pbkdf2.o
 .debug_line    0x00013974      0x6a2 build/WiFIG/production/_ext/334706090/wf_driver_com_24g.o
 .debug_line    0x00014016      0x5ca build/WiFIG/production/_ext/334706090/wf_driver_raw_24g.o
 .debug_line    0x000145e0      0x6b0 build/WiFIG/production/_ext/334706090/wf_mac_24g.o
 .debug_line    0x00014c90      0x402 build/WiFIG/production/_ext/334706090/wf_mgmt_msg_24g.o
 .debug_line    0x00015092      0x5b3 build/WiFIG/production/_ext/334706090/wf_param_msg_24g.o
 .debug_line    0x00015645      0x3ee build/WiFIG/production/_ext/334706090/wf_configData.o
 .debug_line    0x00015a33      0x4c3 build/WiFIG/production/_ext/1472/main_demo.o
 .debug_line    0x00015ef6        0x0 build/WiFIG/production/_ext/1472/custom_snmp_app.o
 .debug_line    0x00015ef6        0x0 build/WiFIG/production/_ext/1472/custom_ssl_cert.o
 .debug_line    0x00015ef6      0x18e build/WiFIG/production/_ext/1472/mpfs_img2.o
 .debug_line    0x00016084      0x2ac build/WiFIG/production/_ext/1472/wf_config.o
 .debug_line    0x00016330        0x0 build/WiFIG/production/_ext/1472/custom_http_app.o
 .debug_line    0x00016330      0x56c build/WiFIG/production/_ext/1472/tcp6_demo_app.o
 .debug_line    0x0001689c       0x6e c:/program files (x86)/microchip/xc32/v1.21/bin/../lib/gcc/pic32mx/4.5.2/../../../../pic32mx/lib/size\libmchp_peripheral.a(open_core_timer_lib.o)
 .debug_line    0x0001690a       0xbf c:/program files (x86)/microchip/xc32/v1.21/bin/../lib/gcc/pic32mx/4.5.2/../../../../pic32mx/lib/size\libmchp_peripheral_32MX695F512H.a(soft_reset_lib.o)
 .debug_line    0x000169c9       0x62 c:/program files (x86)/microchip/xc32/v1.21/bin/../lib/gcc/pic32mx/4.5.2/../../../../pic32mx/lib/size\libmchp_peripheral_32MX695F512H.a(pcache.o)
 .debug_line    0x00016a2b       0x73 c:/program files (x86)/microchip/xc32/v1.21/bin/../lib/gcc/pic32mx/4.5.2/../../../../pic32mx/lib/size\libmchp_peripheral_32MX695F512H.a(int_disable_interrupts_lib.o)
 .debug_line    0x00016a9e       0x73 c:/program files (x86)/microchip/xc32/v1.21/bin/../lib/gcc/pic32mx/4.5.2/../../../../pic32mx/lib/size\libmchp_peripheral_32MX695F512H.a(int_restore_interrupts_lib.o)
 .debug_line    0x00016b11       0x6e c:/program files (x86)/microchip/xc32/v1.21/bin/../lib/gcc/pic32mx/4.5.2/../../../../pic32mx/lib/size\libmchp_peripheral_32MX695F512H.a(int_enable_mv_int_lib.o)
 .debug_line    0x00016b7f       0x64 c:/program files (x86)/microchip/xc32/v1.21/bin/../lib/gcc/pic32mx/4.5.2/../../../../pic32mx/lib/size\libmchp_peripheral_32MX695F512H.a(int_tbl_lib.o)
 .debug_line    0x00016be3       0xda c:/program files (x86)/microchip/xc32/v1.21/bin/../lib/gcc/pic32mx/4.5.2/../../../../pic32mx/lib/size\libmchp_peripheral_32MX695F512H.a(rtcc_init_lib.o)
 .debug_line    0x00016cbd       0xda c:/program files (x86)/microchip/xc32/v1.21/bin/../lib/gcc/pic32mx/4.5.2/../../../../pic32mx/lib/size\libmchp_peripheral_32MX695F512H.a(rtcc_open_lib.o)
 .debug_line    0x00016d97       0x7f c:/program files (x86)/microchip/xc32/v1.21/bin/../lib/gcc/pic32mx/4.5.2/../../../../pic32mx/lib/size\libmchp_peripheral_32MX695F512H.a(spi_chn_data_rdy_lib.o)
 .debug_line    0x00016e16       0x7b c:/program files (x86)/microchip/xc32/v1.21/bin/../lib/gcc/pic32mx/4.5.2/../../../../pic32mx/lib/size\libmchp_peripheral_32MX695F512H.a(spi_chn_getc_lib.o)
 .debug_line    0x00016e91       0x69 c:/program files (x86)/microchip/xc32/v1.21/bin/../lib/gcc/pic32mx/4.5.2/../../../../pic32mx/lib/size\libmchp_peripheral_32MX695F512H.a(spi_chn_open_lib.o)
 .debug_line    0x00016efa       0x7b c:/program files (x86)/microchip/xc32/v1.21/bin/../lib/gcc/pic32mx/4.5.2/../../../../pic32mx/lib/size\libmchp_peripheral_32MX695F512H.a(spi_chn_putc_lib.o)
 .debug_line    0x00016f75       0x72 c:/program files (x86)/microchip/xc32/v1.21/bin/../lib/gcc/pic32mx/4.5.2/../../../../pic32mx/lib/size\libmchp_peripheral_32MX695F512H.a(spi_chn_tx_buff_empty_lib.o)
 .debug_line    0x00016fe7        0x0 c:/program files (x86)/microchip/xc32/v1.21/bin/../lib/gcc/pic32mx/4.5.2/../../../../pic32mx/lib/size\libmchp_peripheral_32MX695F512H.a(spi_io_tbl_libp.o)
 .debug_line    0x00016fe7        0x0 c:/program files (x86)/microchip/xc32/v1.21/bin/../lib/gcc/pic32mx/4.5.2/../../../../pic32mx/lib/size\libmchp_peripheral_32MX695F512H.a(spi_map_tbl_libp.o)
 .debug_line    0x00016fe7       0x77 c:/program files (x86)/microchip/xc32/v1.21/bin/../lib/gcc/pic32mx/4.5.2/../../../../pic32mx/lib/size\libmchp_peripheral_32MX695F512H.a(port_set_pins_digital_in_lib.o)
 .debug_line    0x0001705e       0x78 c:/program files (x86)/microchip/xc32/v1.21/bin/../lib/gcc/pic32mx/4.5.2/../../../../pic32mx/lib/size\libmchp_peripheral_32MX695F512H.a(port_set_pins_digital_out_lib.o)
 .debug_line    0x000170d6        0x0 c:/program files (x86)/microchip/xc32/v1.21/bin/../lib/gcc/pic32mx/4.5.2/../../../../pic32mx/lib/size\libmchp_peripheral_32MX695F512H.a(_ports_tbl_libp.o)
 .debug_line    0x000170d6       0x72 c:/program files (x86)/microchip/xc32/v1.21/bin/../lib/gcc/pic32mx/4.5.2/../../../../pic32mx/lib/size\libmchp_peripheral_32MX695F512H.a(int_enable_interrupts_lib.o)
 .debug_line    0x00017148       0xbd c:/program files (x86)/microchip/xc32/v1.21/bin/../lib/gcc/pic32mx/4.5.2/../../../../pic32mx/lib/size\libmchp_peripheral_32MX695F512H.a(_rtcc_wait_clock_off_lib.o)
 .debug_line    0x00017205       0x6e c:/program files (x86)/microchip/xc32/v1.21/bin/../lib/gcc/pic32mx/4.5.2/../../../../pic32mx/lib/size\libmchp_peripheral_32MX695F512H.a(read_core_timer_lib.o)
 .debug_line    0x00017273      0x119 c:/program files (x86)/microchip/xc32/v1.21/bin/../lib/gcc/pic32mx/4.5.2/size\libgcc.a(_udivdi3.o)
 .debug_line    0x0001738c       0x9d c:/program files (x86)/microchip/xc32/v1.21/bin/../lib/gcc/pic32mx/4.5.2/../../../../pic32mx/lib/size\libpic32.a(default-bootstrap-exception-handler.o)
 .debug_line    0x00017429       0x8a c:/program files (x86)/microchip/xc32/v1.21/bin/../lib/gcc/pic32mx/4.5.2/../../../../pic32mx/lib/size\libpic32.a(default-on-reset.o)
 .debug_line    0x000174b3       0x8e c:/program files (x86)/microchip/xc32/v1.21/bin/../lib/gcc/pic32mx/4.5.2/../../../../pic32mx/lib/size\libpic32.a(default-on-bootstrap.o)
 .debug_line    0x00017541       0x9c c:/program files (x86)/microchip/xc32/v1.21/bin/../lib/gcc/pic32mx/4.5.2/../../../../pic32mx/lib/size\libpic32.a(defaultinterrupt.o)
 .debug_line    0x000175dd       0x80 c:/program files (x86)/microchip/xc32/v1.21/bin/../lib/gcc/pic32mx/4.5.2/../../../../pic32mx/lib/size\libc.a(atoi.o)
 .debug_line    0x0001765d        0x0 c:/program files (x86)/microchip/xc32/v1.21/bin/../lib/gcc/pic32mx/4.5.2/../../../../pic32mx/lib/size\libc.a(ctype.o)
 .debug_line    0x0001765d       0x82 c:/program files (x86)/microchip/xc32/v1.21/bin/../lib/gcc/pic32mx/4.5.2/../../../../pic32mx/lib/size\libc.a(malloc.o)
 .debug_line    0x000176df       0x80 c:/program files (x86)/microchip/xc32/v1.21/bin/../lib/gcc/pic32mx/4.5.2/../../../../pic32mx/lib/size\libc.a(rand.o)
 .debug_line    0x0001775f       0x82 c:/program files (x86)/microchip/xc32/v1.21/bin/../lib/gcc/pic32mx/4.5.2/../../../../pic32mx/lib/size\libc.a(strcat.o)
 .debug_line    0x000177e1       0x82 c:/program files (x86)/microchip/xc32/v1.21/bin/../lib/gcc/pic32mx/4.5.2/../../../../pic32mx/lib/size\libc.a(strchr.o)
 .debug_line    0x00017863       0x83 c:/program files (x86)/microchip/xc32/v1.21/bin/../lib/gcc/pic32mx/4.5.2/../../../../pic32mx/lib/size\libc.a(strncat.o)
 .debug_line    0x000178e6       0x83 c:/program files (x86)/microchip/xc32/v1.21/bin/../lib/gcc/pic32mx/4.5.2/../../../../pic32mx/lib/size\libc.a(strncpy.o)
 .debug_line    0x00017969       0x82 c:/program files (x86)/microchip/xc32/v1.21/bin/../lib/gcc/pic32mx/4.5.2/../../../../pic32mx/lib/size\libc.a(strstr.o)
 .debug_line    0x000179eb       0x82 c:/program files (x86)/microchip/xc32/v1.21/bin/../lib/gcc/pic32mx/4.5.2/../../../../pic32mx/lib/size\libc.a(strtol.o)
 .debug_line    0x00017a6d       0x84 c:/program files (x86)/microchip/xc32/v1.21/bin/../lib/gcc/pic32mx/4.5.2/../../../../pic32mx/lib/size\libc.a(snprintf_cdnopsuxX.eo)
 .debug_line    0x00017af1       0x83 c:/program files (x86)/microchip/xc32/v1.21/bin/../lib/gcc/pic32mx/4.5.2/../../../../pic32mx/lib/size\libc.a(sprintf_cdnopsuxX.eo)
 .debug_line    0x00017b74       0x85 c:/program files (x86)/microchip/xc32/v1.21/bin/../lib/gcc/pic32mx/4.5.2/../../../../pic32mx/lib/size\libc.a(vsnprintf_cdnopsuxX.eo)
 .debug_line    0x00017bf9       0x85 c:/program files (x86)/microchip/xc32/v1.21/bin/../lib/gcc/pic32mx/4.5.2/../../../../pic32mx/lib/size\libc.a(vsnprintf.o)
 .debug_line    0x00017c7e       0x82 c:/program files (x86)/microchip/xc32/v1.21/bin/../lib/gcc/pic32mx/4.5.2/../../../../pic32mx/lib/size\libc.a(ctypef.o)
 .debug_line    0x00017d00        0x0 c:/program files (x86)/microchip/xc32/v1.21/bin/../lib/gcc/pic32mx/4.5.2/../../../../pic32mx/lib/size\libc.a(errno.o)
 .debug_line    0x00017d00       0x83 c:/program files (x86)/microchip/xc32/v1.21/bin/../lib/gcc/pic32mx/4.5.2/../../../../pic32mx/lib/size\libc.a(strncmp.o)
 .debug_line    0x00017d83       0x82 c:/program files (x86)/microchip/xc32/v1.21/bin/../lib/gcc/pic32mx/4.5.2/../../../../pic32mx/lib/size\libc.a(doprnt_cdnopsuxX.eo)
 .debug_line    0x00017e05       0x82 c:/program files (x86)/microchip/xc32/v1.21/bin/../lib/gcc/pic32mx/4.5.2/../../../../pic32mx/lib/size\libc.a(doprnt.o)
 .debug_line    0x00017e87       0x81 c:/program files (x86)/microchip/xc32/v1.21/bin/../lib/gcc/pic32mx/4.5.2/../../../../pic32mx/lib/size\libc.a(_fputc_simple.o)
 .debug_line    0x00017f08        0x0 c:/program files (x86)/microchip/xc32/v1.21/bin/../lib/gcc/pic32mx/4.5.2/../../../../pic32mx/lib/size\libc.a(powersf.o)
 .debug_line    0x00017f08        0x0 c:/program files (x86)/microchip/xc32/v1.21/bin/../lib/gcc/pic32mx/4.5.2/../../../../pic32mx/lib/size\libc.a(_iob.o)
 .debug_line    0x00017f08       0x82 c:/program files (x86)/microchip/xc32/v1.21/bin/../lib/gcc/pic32mx/4.5.2/../../../../pic32mx/lib/size\libc.a(_flsbuf_simple.o)
 .debug_line    0x00017f8a       0x7e c:/program files (x86)/microchip/xc32/v1.21/bin/../lib/gcc/pic32mx/4.5.2/../../../../pic32mx/lib/size\libpic32.a(sbrk.o)
 .debug_line    0x00018008       0x7f c:/program files (x86)/microchip/xc32/v1.21/bin/../lib/gcc/pic32mx/4.5.2/../../../../pic32mx/lib/size\libpic32.a(write.o)
 .debug_line    0x00018087       0x83 c:/program files (x86)/microchip/xc32/v1.21/bin/../lib/gcc/pic32mx/4.5.2/../../../../pic32mx/lib/size\libpic32.a(_mon_putc.o)
 .debug_line    0x0001810a        0x0 c:/program files (x86)/microchip/xc32/v1.21/bin/../lib/gcc/pic32mx/4.5.2/../../../../pic32mx/lib/size\libpic32.a(xc32_uart.o)
 .debug_line    0x0001810a       0x99 c:/program files (x86)/microchip/xc32/v1.21/bin/../lib/gcc/pic32mx/4.5.2/../../../../pic32mx/lib/size\libe.a(_floatdisf.o)
 .debug_line    0x000181a3       0xbe c:/program files (x86)/microchip/xc32/v1.21/bin/../lib/gcc/pic32mx/4.5.2/size\libgcc.a(_lshrdi3.o)
 .debug_line    0x00018261       0xc9 c:/program files (x86)/microchip/xc32/v1.21/bin/../lib/gcc/pic32mx/4.5.2/size\libgcc.a(_floatundisf.o)
 .debug_line    0x0001832a      0x11f c:/program files (x86)/microchip/xc32/v1.21/bin/../lib/gcc/pic32mx/4.5.2/size\libgcc.a(_umoddi3.o)
 .debug_line    0x00018449       0x70 c:/program files (x86)/microchip/xc32/v1.21/bin/../lib/gcc/pic32mx/4.5.2/size\libgcc.a(floatunsisf.o)

.debug_frame    0x00000000     0x6818
 *(.debug_frame)
 .debug_frame   0x00000000       0x2c build/WiFIG/production/_ext/1293749816/bsp.o
 .debug_frame   0x0000002c      0x10c build/WiFIG/production/_ext/101875047/hashes.o
 .debug_frame   0x00000138       0x48 build/WiFIG/production/_ext/101875047/lfsr.o
 .debug_frame   0x00000180      0x188 build/WiFIG/production/_ext/101875047/big_int.o
 .debug_frame   0x00000308       0xf0 build/WiFIG/production/_ext/101875047/helpers.o
 .debug_frame   0x000003f8       0x64 build/WiFIG/production/_ext/1472/ping_demo.o
 .debug_frame   0x0000045c      0x3e8 build/WiFIG/production/_ext/365611741/system_services.o
 .debug_frame   0x00000844      0x1ec build/WiFIG/production/_ext/365611741/system_debug.o
 .debug_frame   0x00000a30       0xa0 build/WiFIG/production/_ext/365611741/system_random.o
 .debug_frame   0x00000ad0       0xf0 build/WiFIG/production/_ext/365611741/system_userio.o
 .debug_frame   0x00000bc0       0xd8 build/WiFIG/production/_ext/792872985/usart.o
 .debug_frame   0x00000c98       0x64 build/WiFIG/production/_ext/792872985/drv_spi.o
 .debug_frame   0x00000cfc       0xd8 build/WiFIG/production/_ext/427700826/tcpip_announce.o
 .debug_frame   0x00000dd4      0x42c build/WiFIG/production/_ext/427700826/arp.o
 .debug_frame   0x00001200      0x240 build/WiFIG/production/_ext/427700826/dhcp.o
 .debug_frame   0x00001440       0x64 build/WiFIG/production/_ext/427700826/dhcps.o
 .debug_frame   0x000014a4      0x148 build/WiFIG/production/_ext/427700826/dns.o
 .debug_frame   0x000015ec       0x48 build/WiFIG/production/_ext/427700826/hash_fnv.o
 .debug_frame   0x00001634       0xf0 build/WiFIG/production/_ext/427700826/hash_tbl.o
 .debug_frame   0x00001724       0xd4 build/WiFIG/production/_ext/427700826/icmp.o
 .debug_frame   0x000017f8      0x458 build/WiFIG/production/_ext/427700826/ipv4.o
 .debug_frame   0x00001c50       0x9c build/WiFIG/production/_ext/427700826/nbns.o
 .debug_frame   0x00001cec      0x8ac build/WiFIG/production/_ext/427700826/tcp.o
 .debug_frame   0x00002598      0x1d0 build/WiFIG/production/_ext/427700826/tcpip_heap_alloc.o
 .debug_frame   0x00002768      0x4e0 build/WiFIG/production/_ext/427700826/udp.o
 .debug_frame   0x00002c48      0x2b0 build/WiFIG/production/_ext/427700826/tcpip_mac_object.o
 .debug_frame   0x00002ef8      0x8d0 build/WiFIG/production/_ext/427700826/tcpip_manager.o
 .debug_frame   0x000037c8      0x2e8 build/WiFIG/production/_ext/427700826/tcpip_helpers.o
 .debug_frame   0x00003ab0       0x64 build/WiFIG/production/_ext/427700826/tcpip_notify.o
 .debug_frame   0x00003b14       0x64 build/WiFIG/production/_ext/427700826/zero_conf_link_local.o
 .debug_frame   0x00003b78       0x64 build/WiFIG/production/_ext/334706090/wf_tx_power.o
 .debug_frame   0x00003bdc       0x9c build/WiFIG/production/_ext/334706090/wf_connect.o
 .debug_frame   0x00003c78      0x208 build/WiFIG/production/_ext/334706090/wf_connection_algorithm.o
 .debug_frame   0x00003e80       0xd4 build/WiFIG/production/_ext/334706090/wf_connection_manager.o
 .debug_frame   0x00003f54      0x2b0 build/WiFIG/production/_ext/334706090/wf_connection_profile.o
 .debug_frame   0x00004204       0x2c build/WiFIG/production/_ext/334706090/wf_easy_config.o
 .debug_frame   0x00004230       0x9c build/WiFIG/production/_ext/334706090/wf_eint.o
 .debug_frame   0x000042cc      0x128 build/WiFIG/production/_ext/334706090/wf_event_handler.o
 .debug_frame   0x000043f4       0x9c build/WiFIG/production/_ext/334706090/wf_init.o
 .debug_frame   0x00004490      0x1b4 build/WiFIG/production/_ext/334706090/wf_power_save.o
 .debug_frame   0x00004644       0x64 build/WiFIG/production/_ext/334706090/wf_scan.o
 .debug_frame   0x000046a8       0x9c build/WiFIG/production/_ext/334706090/wf_spi.o
 .debug_frame   0x00004744      0x358 build/WiFIG/production/_ext/334706090/mrf24w_mac_pic32.o
 .debug_frame   0x00004a9c      0x144 build/WiFIG/production/_ext/334706090/mrf24w_events.o
 .debug_frame   0x00004be0      0x240 build/WiFIG/production/_ext/334706090/wf_debug_output.o
 .debug_frame   0x00004e20      0x1bc build/WiFIG/production/_ext/334706090/wf_commands.o
 .debug_frame   0x00004fdc      0x2b0 build/WiFIG/production/_ext/334706090/wf_driver_com_24g.o
 .debug_frame   0x0000528c      0x25c build/WiFIG/production/_ext/334706090/wf_driver_raw_24g.o
 .debug_frame   0x000054e8      0x374 build/WiFIG/production/_ext/334706090/wf_mac_24g.o
 .debug_frame   0x0000585c       0x9c build/WiFIG/production/_ext/334706090/wf_mgmt_msg_24g.o
 .debug_frame   0x000058f8      0x2e8 build/WiFIG/production/_ext/334706090/wf_param_msg_24g.o
 .debug_frame   0x00005be0       0x80 build/WiFIG/production/_ext/334706090/wf_configData.o
 .debug_frame   0x00005c60       0x84 build/WiFIG/production/_ext/1472/main_demo.o
 .debug_frame   0x00005ce4       0x2c build/WiFIG/production/_ext/1472/wf_config.o
 .debug_frame   0x00005d10       0xa0 build/WiFIG/production/_ext/1472/tcp6_demo_app.o
 .debug_frame   0x00005db0       0x20 c:/program files (x86)/microchip/xc32/v1.21/bin/../lib/gcc/pic32mx/4.5.2/../../../../pic32mx/lib/size\libmchp_peripheral.a(open_core_timer_lib.o)
 .debug_frame   0x00005dd0       0x28 c:/program files (x86)/microchip/xc32/v1.21/bin/../lib/gcc/pic32mx/4.5.2/../../../../pic32mx/lib/size\libmchp_peripheral_32MX695F512H.a(soft_reset_lib.o)
 .debug_frame   0x00005df8       0x30 c:/program files (x86)/microchip/xc32/v1.21/bin/../lib/gcc/pic32mx/4.5.2/../../../../pic32mx/lib/size\libmchp_peripheral_32MX695F512H.a(pcache.o)
 .debug_frame   0x00005e28       0x20 c:/program files (x86)/microchip/xc32/v1.21/bin/../lib/gcc/pic32mx/4.5.2/../../../../pic32mx/lib/size\libmchp_peripheral_32MX695F512H.a(int_disable_interrupts_lib.o)
 .debug_frame   0x00005e48       0x20 c:/program files (x86)/microchip/xc32/v1.21/bin/../lib/gcc/pic32mx/4.5.2/../../../../pic32mx/lib/size\libmchp_peripheral_32MX695F512H.a(int_restore_interrupts_lib.o)
 .debug_frame   0x00005e68       0x28 c:/program files (x86)/microchip/xc32/v1.21/bin/../lib/gcc/pic32mx/4.5.2/../../../../pic32mx/lib/size\libmchp_peripheral_32MX695F512H.a(int_enable_mv_int_lib.o)
 .debug_frame   0x00005e90       0xa0 c:/program files (x86)/microchip/xc32/v1.21/bin/../lib/gcc/pic32mx/4.5.2/../../../../pic32mx/lib/size\libmchp_peripheral_32MX695F512H.a(int_tbl_lib.o)
 .debug_frame   0x00005f30       0x2c c:/program files (x86)/microchip/xc32/v1.21/bin/../lib/gcc/pic32mx/4.5.2/../../../../pic32mx/lib/size\libmchp_peripheral_32MX695F512H.a(rtcc_init_lib.o)
 .debug_frame   0x00005f5c       0x34 c:/program files (x86)/microchip/xc32/v1.21/bin/../lib/gcc/pic32mx/4.5.2/../../../../pic32mx/lib/size\libmchp_peripheral_32MX695F512H.a(rtcc_open_lib.o)
 .debug_frame   0x00005f90       0x20 c:/program files (x86)/microchip/xc32/v1.21/bin/../lib/gcc/pic32mx/4.5.2/../../../../pic32mx/lib/size\libmchp_peripheral_32MX695F512H.a(spi_chn_data_rdy_lib.o)
 .debug_frame   0x00005fb0       0x30 c:/program files (x86)/microchip/xc32/v1.21/bin/../lib/gcc/pic32mx/4.5.2/../../../../pic32mx/lib/size\libmchp_peripheral_32MX695F512H.a(spi_chn_getc_lib.o)
 .debug_frame   0x00005fe0       0x3c c:/program files (x86)/microchip/xc32/v1.21/bin/../lib/gcc/pic32mx/4.5.2/../../../../pic32mx/lib/size\libmchp_peripheral_32MX695F512H.a(spi_chn_open_lib.o)
 .debug_frame   0x0000601c       0x40 c:/program files (x86)/microchip/xc32/v1.21/bin/../lib/gcc/pic32mx/4.5.2/../../../../pic32mx/lib/size\libmchp_peripheral_32MX695F512H.a(spi_chn_putc_lib.o)
 .debug_frame   0x0000605c       0x20 c:/program files (x86)/microchip/xc32/v1.21/bin/../lib/gcc/pic32mx/4.5.2/../../../../pic32mx/lib/size\libmchp_peripheral_32MX695F512H.a(spi_chn_tx_buff_empty_lib.o)
 .debug_frame   0x0000607c       0x20 c:/program files (x86)/microchip/xc32/v1.21/bin/../lib/gcc/pic32mx/4.5.2/../../../../pic32mx/lib/size\libmchp_peripheral_32MX695F512H.a(port_set_pins_digital_in_lib.o)
 .debug_frame   0x0000609c       0x20 c:/program files (x86)/microchip/xc32/v1.21/bin/../lib/gcc/pic32mx/4.5.2/../../../../pic32mx/lib/size\libmchp_peripheral_32MX695F512H.a(port_set_pins_digital_out_lib.o)
 .debug_frame   0x000060bc       0x20 c:/program files (x86)/microchip/xc32/v1.21/bin/../lib/gcc/pic32mx/4.5.2/../../../../pic32mx/lib/size\libmchp_peripheral_32MX695F512H.a(int_enable_interrupts_lib.o)
 .debug_frame   0x000060dc       0x48 c:/program files (x86)/microchip/xc32/v1.21/bin/../lib/gcc/pic32mx/4.5.2/../../../../pic32mx/lib/size\libmchp_peripheral_32MX695F512H.a(_rtcc_wait_clock_off_lib.o)
 .debug_frame   0x00006124       0x20 c:/program files (x86)/microchip/xc32/v1.21/bin/../lib/gcc/pic32mx/4.5.2/../../../../pic32mx/lib/size\libmchp_peripheral_32MX695F512H.a(read_core_timer_lib.o)
 .debug_frame   0x00006144       0x20 c:/program files (x86)/microchip/xc32/v1.21/bin/../lib/gcc/pic32mx/4.5.2/size\libgcc.a(_udivdi3.o)
 .debug_frame   0x00006164       0x20 c:/program files (x86)/microchip/xc32/v1.21/bin/../lib/gcc/pic32mx/4.5.2/../../../../pic32mx/lib/size\libpic32.a(default-bootstrap-exception-handler.o)
 .debug_frame   0x00006184       0x20 c:/program files (x86)/microchip/xc32/v1.21/bin/../lib/gcc/pic32mx/4.5.2/../../../../pic32mx/lib/size\libpic32.a(default-on-reset.o)
 .debug_frame   0x000061a4       0x20 c:/program files (x86)/microchip/xc32/v1.21/bin/../lib/gcc/pic32mx/4.5.2/../../../../pic32mx/lib/size\libpic32.a(default-on-bootstrap.o)
 .debug_frame   0x000061c4       0x20 c:/program files (x86)/microchip/xc32/v1.21/bin/../lib/gcc/pic32mx/4.5.2/../../../../pic32mx/lib/size\libpic32.a(defaultinterrupt.o)
 .debug_frame   0x000061e4       0x20 c:/program files (x86)/microchip/xc32/v1.21/bin/../lib/gcc/pic32mx/4.5.2/../../../../pic32mx/lib/size\libc.a(atoi.o)
 .debug_frame   0x00006204       0x6c c:/program files (x86)/microchip/xc32/v1.21/bin/../lib/gcc/pic32mx/4.5.2/../../../../pic32mx/lib/size\libc.a(malloc.o)
 .debug_frame   0x00006270       0x38 c:/program files (x86)/microchip/xc32/v1.21/bin/../lib/gcc/pic32mx/4.5.2/../../../../pic32mx/lib/size\libc.a(rand.o)
 .debug_frame   0x000062a8       0x20 c:/program files (x86)/microchip/xc32/v1.21/bin/../lib/gcc/pic32mx/4.5.2/../../../../pic32mx/lib/size\libc.a(strcat.o)
 .debug_frame   0x000062c8       0x20 c:/program files (x86)/microchip/xc32/v1.21/bin/../lib/gcc/pic32mx/4.5.2/../../../../pic32mx/lib/size\libc.a(strchr.o)
 .debug_frame   0x000062e8       0x20 c:/program files (x86)/microchip/xc32/v1.21/bin/../lib/gcc/pic32mx/4.5.2/../../../../pic32mx/lib/size\libc.a(strncat.o)
 .debug_frame   0x00006308       0x20 c:/program files (x86)/microchip/xc32/v1.21/bin/../lib/gcc/pic32mx/4.5.2/../../../../pic32mx/lib/size\libc.a(strncpy.o)
 .debug_frame   0x00006328       0x2c c:/program files (x86)/microchip/xc32/v1.21/bin/../lib/gcc/pic32mx/4.5.2/../../../../pic32mx/lib/size\libc.a(strstr.o)
 .debug_frame   0x00006354       0x58 c:/program files (x86)/microchip/xc32/v1.21/bin/../lib/gcc/pic32mx/4.5.2/../../../../pic32mx/lib/size\libc.a(strtol.o)
 .debug_frame   0x000063ac       0x28 c:/program files (x86)/microchip/xc32/v1.21/bin/../lib/gcc/pic32mx/4.5.2/../../../../pic32mx/lib/size\libc.a(snprintf_cdnopsuxX.eo)
 .debug_frame   0x000063d4       0x2c c:/program files (x86)/microchip/xc32/v1.21/bin/../lib/gcc/pic32mx/4.5.2/../../../../pic32mx/lib/size\libc.a(sprintf_cdnopsuxX.eo)
 .debug_frame   0x00006400       0x28 c:/program files (x86)/microchip/xc32/v1.21/bin/../lib/gcc/pic32mx/4.5.2/../../../../pic32mx/lib/size\libc.a(vsnprintf_cdnopsuxX.eo)
 .debug_frame   0x00006428       0x28 c:/program files (x86)/microchip/xc32/v1.21/bin/../lib/gcc/pic32mx/4.5.2/../../../../pic32mx/lib/size\libc.a(vsnprintf.o)
 .debug_frame   0x00006450      0x120 c:/program files (x86)/microchip/xc32/v1.21/bin/../lib/gcc/pic32mx/4.5.2/../../../../pic32mx/lib/size\libc.a(ctypef.o)
 .debug_frame   0x00006570       0x20 c:/program files (x86)/microchip/xc32/v1.21/bin/../lib/gcc/pic32mx/4.5.2/../../../../pic32mx/lib/size\libc.a(strncmp.o)
 .debug_frame   0x00006590       0x38 c:/program files (x86)/microchip/xc32/v1.21/bin/../lib/gcc/pic32mx/4.5.2/../../../../pic32mx/lib/size\libc.a(doprnt_cdnopsuxX.eo)
 .debug_frame   0x000065c8       0x74 c:/program files (x86)/microchip/xc32/v1.21/bin/../lib/gcc/pic32mx/4.5.2/../../../../pic32mx/lib/size\libc.a(doprnt.o)
 .debug_frame   0x0000663c       0x2c c:/program files (x86)/microchip/xc32/v1.21/bin/../lib/gcc/pic32mx/4.5.2/../../../../pic32mx/lib/size\libc.a(_fputc_simple.o)
 .debug_frame   0x00006668       0x28 c:/program files (x86)/microchip/xc32/v1.21/bin/../lib/gcc/pic32mx/4.5.2/../../../../pic32mx/lib/size\libc.a(_flsbuf_simple.o)
 .debug_frame   0x00006690       0x88 c:/program files (x86)/microchip/xc32/v1.21/bin/../lib/gcc/pic32mx/4.5.2/../../../../pic32mx/lib/size\libpic32.a(sbrk.o)
 .debug_frame   0x00006718       0x2c c:/program files (x86)/microchip/xc32/v1.21/bin/../lib/gcc/pic32mx/4.5.2/../../../../pic32mx/lib/size\libpic32.a(write.o)
 .debug_frame   0x00006744       0x20 c:/program files (x86)/microchip/xc32/v1.21/bin/../lib/gcc/pic32mx/4.5.2/../../../../pic32mx/lib/size\libpic32.a(_mon_putc.o)
 .debug_frame   0x00006764       0x20 c:/program files (x86)/microchip/xc32/v1.21/bin/../lib/gcc/pic32mx/4.5.2/../../../../pic32mx/lib/size\libe.a(_floatdisf.o)
 .debug_frame   0x00006784       0x20 c:/program files (x86)/microchip/xc32/v1.21/bin/../lib/gcc/pic32mx/4.5.2/size\libgcc.a(_lshrdi3.o)
 .debug_frame   0x000067a4       0x2c c:/program files (x86)/microchip/xc32/v1.21/bin/../lib/gcc/pic32mx/4.5.2/size\libgcc.a(_floatundisf.o)
 .debug_frame   0x000067d0       0x20 c:/program files (x86)/microchip/xc32/v1.21/bin/../lib/gcc/pic32mx/4.5.2/size\libgcc.a(_umoddi3.o)
 .debug_frame   0x000067f0       0x28 c:/program files (x86)/microchip/xc32/v1.21/bin/../lib/gcc/pic32mx/4.5.2/size\libgcc.a(floatunsisf.o)

.debug_str      0x00000000     0x9534
 *(.debug_str)
 .debug_str     0x00000000      0x16c build/WiFIG/production/_ext/1293749816/bsp.o
 .debug_str     0x0000016c       0x1a build/WiFIG/production/_ext/101875047/hashes.o
 .debug_str     0x00000186        0x0 build/WiFIG/production/_ext/101875047/lfsr.o
 .debug_str     0x00000186      0x12f build/WiFIG/production/_ext/101875047/big_int.o
 .debug_str     0x000002b5        0x0 build/WiFIG/production/_ext/101875047/helpers.o
 .debug_str     0x000002b5        0x0 build/WiFIG/production/_ext/1472/berkeley_tcp_client_demo.o
 .debug_str     0x000002b5        0x0 build/WiFIG/production/_ext/1472/berkeley_tcp_server_demo.o
 .debug_str     0x000002b5        0x0 build/WiFIG/production/_ext/1472/berkeley_udp_client_demo.o
 .debug_str     0x000002b5      0x156 build/WiFIG/production/_ext/1472/generic_tcp_client.o
 .debug_str     0x0000040b      0x156 build/WiFIG/production/_ext/1472/generic_tcp_server.o
 .debug_str     0x00000561      0x18b build/WiFIG/production/_ext/1472/ping_demo.o
 .debug_str     0x000006ec        0x0 build/WiFIG/production/_ext/1472/smtp_demo.o
 .debug_str     0x000006ec      0x239 build/WiFIG/production/_ext/365611741/system_services.o
 .debug_str     0x00000925      0x156 build/WiFIG/production/_ext/365611741/system_debug.o
 .debug_str     0x00000a7b      0x15f build/WiFIG/production/_ext/365611741/system_random.o
 .debug_str     0x00000bda       0xfe build/WiFIG/production/_ext/365611741/system_command.o
 .debug_str     0x00000cd8      0x172 build/WiFIG/production/_ext/365611741/system_userio.o
 .debug_str     0x00000e4a       0xfe build/WiFIG/production/_ext/97638081/sys_fs.o
 .debug_str     0x00000f48      0x12f build/WiFIG/production/_ext/97638081/mpfs2.o
 .debug_str     0x00001077      0x11a build/WiFIG/production/_ext/792872985/usart.o
 .debug_str     0x00001191        0x0 build/WiFIG/production/_ext/792872985/lcd.o
 .debug_str     0x00001191      0x156 build/WiFIG/production/_ext/792872985/drv_spi.o
 .debug_str     0x000012e7        0x0 build/WiFIG/production/_ext/792872985/db_appio.o
 .debug_str     0x000012e7      0x12f build/WiFIG/production/_ext/792872985/spi_ram.o
 .debug_str     0x00001416      0x12f build/WiFIG/production/_ext/792872985/spi_eeprom.o
 .debug_str     0x00001545      0x12f build/WiFIG/production/_ext/792872985/spi_flash.o
 .debug_str     0x00001674      0x12f build/WiFIG/production/_ext/792872985/drv_media.o
 .debug_str     0x000017a3      0x196 build/WiFIG/production/_ext/427700826/tcpip_announce.o
 .debug_str     0x00001939      0x170 build/WiFIG/production/_ext/427700826/http2.o
 .debug_str     0x00001aa9      0x170 build/WiFIG/production/_ext/427700826/arcfour.o
 .debug_str     0x00001c19      0x234 build/WiFIG/production/_ext/427700826/arp.o
 .debug_str     0x00001e4d      0x170 build/WiFIG/production/_ext/427700826/berkeley_api.o
 .debug_str     0x00001fbd      0x1c6 build/WiFIG/production/_ext/427700826/dhcp.o
 .debug_str     0x00002183      0x170 build/WiFIG/production/_ext/427700826/dhcps.o
 .debug_str     0x000022f3      0x18f build/WiFIG/production/_ext/427700826/dns.o
 .debug_str     0x00002482      0x170 build/WiFIG/production/_ext/427700826/dnss.o
 .debug_str     0x000025f2      0x170 build/WiFIG/production/_ext/427700826/dyn_dns.o
 .debug_str     0x00002762      0x170 build/WiFIG/production/_ext/427700826/enc28_mac.o
 .debug_str     0x000028d2      0x170 build/WiFIG/production/_ext/427700826/enc28j60.o
 .debug_str     0x00002a42      0x170 build/WiFIG/production/_ext/427700826/encs24j600.o
 .debug_str     0x00002bb2      0x170 build/WiFIG/production/_ext/427700826/encx24_mac.o
 .debug_str     0x00002d22      0x170 build/WiFIG/production/_ext/427700826/eth_pic32_ext_phy.o
 .debug_str     0x00002e92      0x170 build/WiFIG/production/_ext/427700826/eth_pic32_ext_phy_dp83848.o
 .debug_str     0x00003002      0x170 build/WiFIG/production/_ext/427700826/eth_pic32_int_mac.o
 .debug_str     0x00003172      0x170 build/WiFIG/production/_ext/427700826/ftp.o
 .debug_str     0x000032e2        0x0 build/WiFIG/production/_ext/427700826/hash_fnv.o
 .debug_str     0x000032e2        0xa build/WiFIG/production/_ext/427700826/hash_tbl.o
 .debug_str     0x000032ec      0x1a8 build/WiFIG/production/_ext/427700826/icmp.o
 .debug_str     0x00003494      0x170 build/WiFIG/production/_ext/427700826/icmpv6.o
 .debug_str     0x00003604      0x227 build/WiFIG/production/_ext/427700826/ipv4.o
 .debug_str     0x0000382b      0x170 build/WiFIG/production/_ext/427700826/ipv6.o
 .debug_str     0x0000399b      0x170 build/WiFIG/production/_ext/427700826/mac_events_pic32.o
 .debug_str     0x00003b0b      0x1b1 build/WiFIG/production/_ext/427700826/nbns.o
 .debug_str     0x00003cbc      0x170 build/WiFIG/production/_ext/427700826/ndp.o
 .debug_str     0x00003e2c      0x170 build/WiFIG/production/_ext/427700826/tcpip_reboot.o
 .debug_str     0x00003f9c      0x170 build/WiFIG/production/_ext/427700826/rsa.o
 .debug_str     0x0000410c      0x170 build/WiFIG/production/_ext/427700826/smtp.o
 .debug_str     0x0000427c      0x170 build/WiFIG/production/_ext/427700826/snmp.o
 .debug_str     0x000043ec      0x170 build/WiFIG/production/_ext/427700826/snmpv3.o
 .debug_str     0x0000455c      0x170 build/WiFIG/production/_ext/427700826/snmpv3_usm.o
 .debug_str     0x000046cc      0x170 build/WiFIG/production/_ext/427700826/sntp.o
 .debug_str     0x0000483c      0x170 build/WiFIG/production/_ext/427700826/ssl.o
 .debug_str     0x000049ac      0x26b build/WiFIG/production/_ext/427700826/tcp.o
 .debug_str     0x00004c17      0x195 build/WiFIG/production/_ext/427700826/tcpip_heap_alloc.o
 .debug_str     0x00004dac      0x170 build/WiFIG/production/_ext/427700826/tcpip_storage.o
 .debug_str     0x00004f1c      0x170 build/WiFIG/production/_ext/427700826/telnet.o
 .debug_str     0x0000508c      0x170 build/WiFIG/production/_ext/427700826/tftpc.o
 .debug_str     0x000051fc      0x247 build/WiFIG/production/_ext/427700826/udp.o
 .debug_str     0x00005443      0x31b build/WiFIG/production/_ext/427700826/tcpip_mac_object.o
 .debug_str     0x0000575e      0x347 build/WiFIG/production/_ext/427700826/tcpip_manager.o
 .debug_str     0x00005aa5      0x181 build/WiFIG/production/_ext/427700826/tcpip_helpers.o
 .debug_str     0x00005c26      0x170 build/WiFIG/production/_ext/427700826/tcpip_commands.o
 .debug_str     0x00005d96      0x170 build/WiFIG/production/_ext/427700826/iperf.o
 .debug_str     0x00005f06        0xb build/WiFIG/production/_ext/427700826/tcpip_notify.o
 .debug_str     0x00005f11      0x170 build/WiFIG/production/_ext/427700826/zero_conf_helper.o
 .debug_str     0x00006081      0x170 build/WiFIG/production/_ext/427700826/zero_conf_link_local.o
 .debug_str     0x000061f1      0x170 build/WiFIG/production/_ext/427700826/zero_conf_multicast_dns.o
 .debug_str     0x00006361      0x178 build/WiFIG/production/_ext/334706090/wf_tx_power.o
 .debug_str     0x000064d9      0x1ba build/WiFIG/production/_ext/334706090/wf_connect.o
 .debug_str     0x00006693      0x1b2 build/WiFIG/production/_ext/334706090/wf_connection_algorithm.o
 .debug_str     0x00006845      0x177 build/WiFIG/production/_ext/334706090/wf_connection_manager.o
 .debug_str     0x000069bc      0x200 build/WiFIG/production/_ext/334706090/wf_connection_profile.o
 .debug_str     0x00006bbc      0x17a build/WiFIG/production/_ext/334706090/wf_easy_config.o
 .debug_str     0x00006d36      0x18c build/WiFIG/production/_ext/334706090/wf_eint.o
 .debug_str     0x00006ec2      0x1ac build/WiFIG/production/_ext/334706090/wf_event_handler.o
 .debug_str     0x0000706e      0x242 build/WiFIG/production/_ext/334706090/wf_init.o
 .debug_str     0x000072b0      0x1a4 build/WiFIG/production/_ext/334706090/wf_power_save.o
 .debug_str     0x00007454      0x170 build/WiFIG/production/_ext/334706090/wf_scan.o
 .debug_str     0x000075c4      0x183 build/WiFIG/production/_ext/334706090/wf_spi.o
 .debug_str     0x00007747      0x1b3 build/WiFIG/production/_ext/334706090/mrf24w_mac_pic32.o
 .debug_str     0x000078fa      0x18b build/WiFIG/production/_ext/334706090/mrf24w_events.o
 .debug_str     0x00007a85      0x2e1 build/WiFIG/production/_ext/334706090/wf_debug_output.o
 .debug_str     0x00007d66      0x1bc build/WiFIG/production/_ext/334706090/wf_commands.o
 .debug_str     0x00007f22      0x170 build/WiFIG/production/_ext/334706090/wf_pbkdf2.o
 .debug_str     0x00008092      0x241 build/WiFIG/production/_ext/334706090/wf_driver_com_24g.o
 .debug_str     0x000082d3      0x22f build/WiFIG/production/_ext/334706090/wf_driver_raw_24g.o
 .debug_str     0x00008502      0x241 build/WiFIG/production/_ext/334706090/wf_mac_24g.o
 .debug_str     0x00008743      0x1b5 build/WiFIG/production/_ext/334706090/wf_mgmt_msg_24g.o
 .debug_str     0x000088f8      0x1e0 build/WiFIG/production/_ext/334706090/wf_param_msg_24g.o
 .debug_str     0x00008ad8      0x239 build/WiFIG/production/_ext/334706090/wf_configData.o
 .debug_str     0x00008d11      0x27b build/WiFIG/production/_ext/1472/main_demo.o
 .debug_str     0x00008f8c        0x0 build/WiFIG/production/_ext/1472/custom_snmp_app.o
 .debug_str     0x00008f8c        0x0 build/WiFIG/production/_ext/1472/custom_ssl_cert.o
 .debug_str     0x00008f8c      0x12f build/WiFIG/production/_ext/1472/mpfs_img2.o
 .debug_str     0x000090bb      0x156 build/WiFIG/production/_ext/1472/wf_config.o
 .debug_str     0x00009211        0x0 build/WiFIG/production/_ext/1472/custom_http_app.o
 .debug_str     0x00009211      0x323 build/WiFIG/production/_ext/1472/tcp6_demo_app.o
 .debug_str     0x00009534        0x0 c:/program files (x86)/microchip/xc32/v1.21/bin/../lib/gcc/pic32mx/4.5.2/../../../../pic32mx/lib/size\libmchp_peripheral.a(open_core_timer_lib.o)
 .debug_str     0x00009534        0x0 c:/program files (x86)/microchip/xc32/v1.21/bin/../lib/gcc/pic32mx/4.5.2/../../../../pic32mx/lib/size\libmchp_peripheral_32MX695F512H.a(soft_reset_lib.o)
 .debug_str     0x00009534        0x0 c:/program files (x86)/microchip/xc32/v1.21/bin/../lib/gcc/pic32mx/4.5.2/../../../../pic32mx/lib/size\libmchp_peripheral_32MX695F512H.a(pcache.o)
 .debug_str     0x00009534        0x0 c:/program files (x86)/microchip/xc32/v1.21/bin/../lib/gcc/pic32mx/4.5.2/../../../../pic32mx/lib/size\libmchp_peripheral_32MX695F512H.a(int_disable_interrupts_lib.o)
 .debug_str     0x00009534        0x0 c:/program files (x86)/microchip/xc32/v1.21/bin/../lib/gcc/pic32mx/4.5.2/../../../../pic32mx/lib/size\libmchp_peripheral_32MX695F512H.a(int_restore_interrupts_lib.o)
 .debug_str     0x00009534        0x0 c:/program files (x86)/microchip/xc32/v1.21/bin/../lib/gcc/pic32mx/4.5.2/../../../../pic32mx/lib/size\libmchp_peripheral_32MX695F512H.a(int_enable_mv_int_lib.o)
 .debug_str     0x00009534        0x0 c:/program files (x86)/microchip/xc32/v1.21/bin/../lib/gcc/pic32mx/4.5.2/../../../../pic32mx/lib/size\libmchp_peripheral_32MX695F512H.a(int_tbl_lib.o)
 .debug_str     0x00009534        0x0 c:/program files (x86)/microchip/xc32/v1.21/bin/../lib/gcc/pic32mx/4.5.2/../../../../pic32mx/lib/size\libmchp_peripheral_32MX695F512H.a(rtcc_init_lib.o)
 .debug_str     0x00009534        0x0 c:/program files (x86)/microchip/xc32/v1.21/bin/../lib/gcc/pic32mx/4.5.2/../../../../pic32mx/lib/size\libmchp_peripheral_32MX695F512H.a(rtcc_open_lib.o)
 .debug_str     0x00009534        0x0 c:/program files (x86)/microchip/xc32/v1.21/bin/../lib/gcc/pic32mx/4.5.2/../../../../pic32mx/lib/size\libmchp_peripheral_32MX695F512H.a(spi_chn_data_rdy_lib.o)
 .debug_str     0x00009534        0x0 c:/program files (x86)/microchip/xc32/v1.21/bin/../lib/gcc/pic32mx/4.5.2/../../../../pic32mx/lib/size\libmchp_peripheral_32MX695F512H.a(spi_chn_getc_lib.o)
 .debug_str     0x00009534        0x0 c:/program files (x86)/microchip/xc32/v1.21/bin/../lib/gcc/pic32mx/4.5.2/../../../../pic32mx/lib/size\libmchp_peripheral_32MX695F512H.a(spi_chn_open_lib.o)
 .debug_str     0x00009534        0x0 c:/program files (x86)/microchip/xc32/v1.21/bin/../lib/gcc/pic32mx/4.5.2/../../../../pic32mx/lib/size\libmchp_peripheral_32MX695F512H.a(spi_chn_putc_lib.o)
 .debug_str     0x00009534        0x0 c:/program files (x86)/microchip/xc32/v1.21/bin/../lib/gcc/pic32mx/4.5.2/../../../../pic32mx/lib/size\libmchp_peripheral_32MX695F512H.a(spi_chn_tx_buff_empty_lib.o)
 .debug_str     0x00009534        0x0 c:/program files (x86)/microchip/xc32/v1.21/bin/../lib/gcc/pic32mx/4.5.2/../../../../pic32mx/lib/size\libmchp_peripheral_32MX695F512H.a(spi_io_tbl_libp.o)
 .debug_str     0x00009534        0x0 c:/program files (x86)/microchip/xc32/v1.21/bin/../lib/gcc/pic32mx/4.5.2/../../../../pic32mx/lib/size\libmchp_peripheral_32MX695F512H.a(spi_map_tbl_libp.o)
 .debug_str     0x00009534        0x0 c:/program files (x86)/microchip/xc32/v1.21/bin/../lib/gcc/pic32mx/4.5.2/../../../../pic32mx/lib/size\libmchp_peripheral_32MX695F512H.a(port_set_pins_digital_in_lib.o)
 .debug_str     0x00009534        0x0 c:/program files (x86)/microchip/xc32/v1.21/bin/../lib/gcc/pic32mx/4.5.2/../../../../pic32mx/lib/size\libmchp_peripheral_32MX695F512H.a(port_set_pins_digital_out_lib.o)
 .debug_str     0x00009534        0x0 c:/program files (x86)/microchip/xc32/v1.21/bin/../lib/gcc/pic32mx/4.5.2/../../../../pic32mx/lib/size\libmchp_peripheral_32MX695F512H.a(_ports_tbl_libp.o)
 .debug_str     0x00009534        0x0 c:/program files (x86)/microchip/xc32/v1.21/bin/../lib/gcc/pic32mx/4.5.2/../../../../pic32mx/lib/size\libmchp_peripheral_32MX695F512H.a(int_enable_interrupts_lib.o)
 .debug_str     0x00009534        0x0 c:/program files (x86)/microchip/xc32/v1.21/bin/../lib/gcc/pic32mx/4.5.2/../../../../pic32mx/lib/size\libmchp_peripheral_32MX695F512H.a(_rtcc_wait_clock_off_lib.o)
 .debug_str     0x00009534        0x0 c:/program files (x86)/microchip/xc32/v1.21/bin/../lib/gcc/pic32mx/4.5.2/../../../../pic32mx/lib/size\libmchp_peripheral_32MX695F512H.a(read_core_timer_lib.o)
 .debug_str     0x00009534        0x0 c:/program files (x86)/microchip/xc32/v1.21/bin/../lib/gcc/pic32mx/4.5.2/size\libgcc.a(_udivdi3.o)
 .debug_str     0x00009534        0x0 c:/program files (x86)/microchip/xc32/v1.21/bin/../lib/gcc/pic32mx/4.5.2/../../../../pic32mx/lib/size\libpic32.a(default-bootstrap-exception-handler.o)
 .debug_str     0x00009534        0x0 c:/program files (x86)/microchip/xc32/v1.21/bin/../lib/gcc/pic32mx/4.5.2/../../../../pic32mx/lib/size\libpic32.a(default-on-reset.o)
 .debug_str     0x00009534        0x0 c:/program files (x86)/microchip/xc32/v1.21/bin/../lib/gcc/pic32mx/4.5.2/../../../../pic32mx/lib/size\libpic32.a(default-on-bootstrap.o)
 .debug_str     0x00009534        0x0 c:/program files (x86)/microchip/xc32/v1.21/bin/../lib/gcc/pic32mx/4.5.2/../../../../pic32mx/lib/size\libpic32.a(defaultinterrupt.o)
 .debug_str     0x00009534        0x0 c:/program files (x86)/microchip/xc32/v1.21/bin/../lib/gcc/pic32mx/4.5.2/../../../../pic32mx/lib/size\libc.a(atoi.o)
 .debug_str     0x00009534        0x0 c:/program files (x86)/microchip/xc32/v1.21/bin/../lib/gcc/pic32mx/4.5.2/../../../../pic32mx/lib/size\libc.a(ctype.o)
 .debug_str     0x00009534        0x0 c:/program files (x86)/microchip/xc32/v1.21/bin/../lib/gcc/pic32mx/4.5.2/../../../../pic32mx/lib/size\libc.a(malloc.o)
 .debug_str     0x00009534        0x0 c:/program files (x86)/microchip/xc32/v1.21/bin/../lib/gcc/pic32mx/4.5.2/../../../../pic32mx/lib/size\libc.a(rand.o)
 .debug_str     0x00009534        0x0 c:/program files (x86)/microchip/xc32/v1.21/bin/../lib/gcc/pic32mx/4.5.2/../../../../pic32mx/lib/size\libc.a(strcat.o)
 .debug_str     0x00009534        0x0 c:/program files (x86)/microchip/xc32/v1.21/bin/../lib/gcc/pic32mx/4.5.2/../../../../pic32mx/lib/size\libc.a(strchr.o)
 .debug_str     0x00009534        0x0 c:/program files (x86)/microchip/xc32/v1.21/bin/../lib/gcc/pic32mx/4.5.2/../../../../pic32mx/lib/size\libc.a(strncat.o)
 .debug_str     0x00009534        0x0 c:/program files (x86)/microchip/xc32/v1.21/bin/../lib/gcc/pic32mx/4.5.2/../../../../pic32mx/lib/size\libc.a(strncpy.o)
 .debug_str     0x00009534        0x0 c:/program files (x86)/microchip/xc32/v1.21/bin/../lib/gcc/pic32mx/4.5.2/../../../../pic32mx/lib/size\libc.a(strstr.o)
 .debug_str     0x00009534        0x0 c:/program files (x86)/microchip/xc32/v1.21/bin/../lib/gcc/pic32mx/4.5.2/../../../../pic32mx/lib/size\libc.a(strtol.o)
 .debug_str     0x00009534        0x0 c:/program files (x86)/microchip/xc32/v1.21/bin/../lib/gcc/pic32mx/4.5.2/../../../../pic32mx/lib/size\libc.a(snprintf_cdnopsuxX.eo)
 .debug_str     0x00009534        0x0 c:/program files (x86)/microchip/xc32/v1.21/bin/../lib/gcc/pic32mx/4.5.2/../../../../pic32mx/lib/size\libc.a(sprintf_cdnopsuxX.eo)
 .debug_str     0x00009534        0x0 c:/program files (x86)/microchip/xc32/v1.21/bin/../lib/gcc/pic32mx/4.5.2/../../../../pic32mx/lib/size\libc.a(vsnprintf_cdnopsuxX.eo)
 .debug_str     0x00009534        0x0 c:/program files (x86)/microchip/xc32/v1.21/bin/../lib/gcc/pic32mx/4.5.2/../../../../pic32mx/lib/size\libc.a(vsnprintf.o)
 .debug_str     0x00009534        0x0 c:/program files (x86)/microchip/xc32/v1.21/bin/../lib/gcc/pic32mx/4.5.2/../../../../pic32mx/lib/size\libc.a(ctypef.o)
 .debug_str     0x00009534        0x0 c:/program files (x86)/microchip/xc32/v1.21/bin/../lib/gcc/pic32mx/4.5.2/../../../../pic32mx/lib/size\libc.a(errno.o)
 .debug_str     0x00009534        0x0 c:/program files (x86)/microchip/xc32/v1.21/bin/../lib/gcc/pic32mx/4.5.2/../../../../pic32mx/lib/size\libc.a(strncmp.o)
 .debug_str     0x00009534        0x0 c:/program files (x86)/microchip/xc32/v1.21/bin/../lib/gcc/pic32mx/4.5.2/../../../../pic32mx/lib/size\libc.a(doprnt_cdnopsuxX.eo)
 .debug_str     0x00009534        0x0 c:/program files (x86)/microchip/xc32/v1.21/bin/../lib/gcc/pic32mx/4.5.2/../../../../pic32mx/lib/size\libc.a(doprnt.o)
 .debug_str     0x00009534        0x0 c:/program files (x86)/microchip/xc32/v1.21/bin/../lib/gcc/pic32mx/4.5.2/../../../../pic32mx/lib/size\libc.a(_fputc_simple.o)
 .debug_str     0x00009534        0x0 c:/program files (x86)/microchip/xc32/v1.21/bin/../lib/gcc/pic32mx/4.5.2/../../../../pic32mx/lib/size\libc.a(powersf.o)
 .debug_str     0x00009534        0x0 c:/program files (x86)/microchip/xc32/v1.21/bin/../lib/gcc/pic32mx/4.5.2/../../../../pic32mx/lib/size\libc.a(_iob.o)
 .debug_str     0x00009534        0x0 c:/program files (x86)/microchip/xc32/v1.21/bin/../lib/gcc/pic32mx/4.5.2/../../../../pic32mx/lib/size\libc.a(_flsbuf_simple.o)
 .debug_str     0x00009534        0x0 c:/program files (x86)/microchip/xc32/v1.21/bin/../lib/gcc/pic32mx/4.5.2/../../../../pic32mx/lib/size\libpic32.a(sbrk.o)
 .debug_str     0x00009534        0x0 c:/program files (x86)/microchip/xc32/v1.21/bin/../lib/gcc/pic32mx/4.5.2/../../../../pic32mx/lib/size\libpic32.a(write.o)
 .debug_str     0x00009534        0x0 c:/program files (x86)/microchip/xc32/v1.21/bin/../lib/gcc/pic32mx/4.5.2/../../../../pic32mx/lib/size\libpic32.a(_mon_putc.o)
 .debug_str     0x00009534        0x0 c:/program files (x86)/microchip/xc32/v1.21/bin/../lib/gcc/pic32mx/4.5.2/../../../../pic32mx/lib/size\libpic32.a(xc32_uart.o)
 .debug_str     0x00009534        0x0 c:/program files (x86)/microchip/xc32/v1.21/bin/../lib/gcc/pic32mx/4.5.2/../../../../pic32mx/lib/size\libe.a(_floatdisf.o)
 .debug_str     0x00009534        0x0 c:/program files (x86)/microchip/xc32/v1.21/bin/../lib/gcc/pic32mx/4.5.2/size\libgcc.a(_lshrdi3.o)
 .debug_str     0x00009534        0x0 c:/program files (x86)/microchip/xc32/v1.21/bin/../lib/gcc/pic32mx/4.5.2/size\libgcc.a(_floatundisf.o)
 .debug_str     0x00009534        0x0 c:/program files (x86)/microchip/xc32/v1.21/bin/../lib/gcc/pic32mx/4.5.2/size\libgcc.a(_umoddi3.o)
 .debug_str     0x00009534        0x0 c:/program files (x86)/microchip/xc32/v1.21/bin/../lib/gcc/pic32mx/4.5.2/size\libgcc.a(floatunsisf.o)

.debug_loc      0x00000000     0x166a
 *(.debug_loc)
 .debug_loc     0x00000000      0xa67 c:/program files (x86)/microchip/xc32/v1.21/bin/../lib/gcc/pic32mx/4.5.2/size\libgcc.a(_udivdi3.o)
 .debug_loc     0x00000a67       0x5f c:/program files (x86)/microchip/xc32/v1.21/bin/../lib/gcc/pic32mx/4.5.2/size\libgcc.a(_lshrdi3.o)
 .debug_loc     0x00000ac6       0xc9 c:/program files (x86)/microchip/xc32/v1.21/bin/../lib/gcc/pic32mx/4.5.2/size\libgcc.a(_floatundisf.o)
 .debug_loc     0x00000b8f      0xa73 c:/program files (x86)/microchip/xc32/v1.21/bin/../lib/gcc/pic32mx/4.5.2/size\libgcc.a(_umoddi3.o)
 .debug_loc     0x00001602       0x68 c:/program files (x86)/microchip/xc32/v1.21/bin/../lib/gcc/pic32mx/4.5.2/size\libgcc.a(floatunsisf.o)

.debug_macinfo
 *(.debug_macinfo)

.debug_weaknames
 *(.debug_weaknames)

.debug_funcnames
 *(.debug_funcnames)

.debug_typenames
 *(.debug_typenames)

.debug_varnames
 *(.debug_varnames)

.debug_pubtypes
                0x00000000     0xa517
 *(.debug_pubtypes)
 .debug_pubtypes
                0x00000000      0x132 build/WiFIG/production/_ext/1293749816/bsp.o
 .debug_pubtypes
                0x00000132       0x6d build/WiFIG/production/_ext/101875047/hashes.o
 .debug_pubtypes
                0x0000019f       0x3e build/WiFIG/production/_ext/101875047/lfsr.o
 .debug_pubtypes
                0x000001dd      0x13a build/WiFIG/production/_ext/101875047/big_int.o
 .debug_pubtypes
                0x00000317       0x68 build/WiFIG/production/_ext/101875047/helpers.o
 .debug_pubtypes
                0x0000037f       0xf4 build/WiFIG/production/_ext/1472/generic_tcp_client.o
 .debug_pubtypes
                0x00000473       0xf4 build/WiFIG/production/_ext/1472/generic_tcp_server.o
 .debug_pubtypes
                0x00000567      0x17a build/WiFIG/production/_ext/1472/ping_demo.o
 .debug_pubtypes
                0x000006e1      0x290 build/WiFIG/production/_ext/365611741/system_services.o
 .debug_pubtypes
                0x00000971      0x1a8 build/WiFIG/production/_ext/365611741/system_debug.o
 .debug_pubtypes
                0x00000b19      0x14c build/WiFIG/production/_ext/365611741/system_random.o
 .debug_pubtypes
                0x00000c65       0x94 build/WiFIG/production/_ext/365611741/system_command.o
 .debug_pubtypes
                0x00000cf9      0x1fd build/WiFIG/production/_ext/365611741/system_userio.o
 .debug_pubtypes
                0x00000ef6       0x94 build/WiFIG/production/_ext/97638081/sys_fs.o
 .debug_pubtypes
                0x00000f8a       0xe7 build/WiFIG/production/_ext/97638081/mpfs2.o
 .debug_pubtypes
                0x00001071      0x1a7 build/WiFIG/production/_ext/792872985/usart.o
 .debug_pubtypes
                0x00001218      0x131 build/WiFIG/production/_ext/792872985/drv_spi.o
 .debug_pubtypes
                0x00001349       0xe7 build/WiFIG/production/_ext/792872985/spi_ram.o
 .debug_pubtypes
                0x00001430       0xe7 build/WiFIG/production/_ext/792872985/spi_eeprom.o
 .debug_pubtypes
                0x00001517       0xe7 build/WiFIG/production/_ext/792872985/spi_flash.o
 .debug_pubtypes
                0x000015fe       0xe7 build/WiFIG/production/_ext/792872985/drv_media.o
 .debug_pubtypes
                0x000016e5      0x32f build/WiFIG/production/_ext/427700826/tcpip_announce.o
 .debug_pubtypes
                0x00001a14      0x12c build/WiFIG/production/_ext/427700826/http2.o
 .debug_pubtypes
                0x00001b40      0x12c build/WiFIG/production/_ext/427700826/arcfour.o
 .debug_pubtypes
                0x00001c6c      0x483 build/WiFIG/production/_ext/427700826/arp.o
 .debug_pubtypes
                0x000020ef      0x12c build/WiFIG/production/_ext/427700826/berkeley_api.o
 .debug_pubtypes
                0x0000221b      0x392 build/WiFIG/production/_ext/427700826/dhcp.o
 .debug_pubtypes
                0x000025ad      0x141 build/WiFIG/production/_ext/427700826/dhcps.o
 .debug_pubtypes
                0x000026ee      0x34b build/WiFIG/production/_ext/427700826/dns.o
 .debug_pubtypes
                0x00002a39      0x12c build/WiFIG/production/_ext/427700826/dnss.o
 .debug_pubtypes
                0x00002b65      0x12c build/WiFIG/production/_ext/427700826/dyn_dns.o
 .debug_pubtypes
                0x00002c91      0x12c build/WiFIG/production/_ext/427700826/enc28_mac.o
 .debug_pubtypes
                0x00002dbd      0x12c build/WiFIG/production/_ext/427700826/enc28j60.o
 .debug_pubtypes
                0x00002ee9      0x12c build/WiFIG/production/_ext/427700826/encs24j600.o
 .debug_pubtypes
                0x00003015      0x12c build/WiFIG/production/_ext/427700826/encx24_mac.o
 .debug_pubtypes
                0x00003141      0x12c build/WiFIG/production/_ext/427700826/eth_pic32_ext_phy.o
 .debug_pubtypes
                0x0000326d      0x12c build/WiFIG/production/_ext/427700826/eth_pic32_ext_phy_dp83848.o
 .debug_pubtypes
                0x00003399      0x12c build/WiFIG/production/_ext/427700826/eth_pic32_int_mac.o
 .debug_pubtypes
                0x000034c5      0x12c build/WiFIG/production/_ext/427700826/ftp.o
 .debug_pubtypes
                0x000035f1       0x3a build/WiFIG/production/_ext/427700826/hash_fnv.o
 .debug_pubtypes
                0x0000362b       0xe1 build/WiFIG/production/_ext/427700826/hash_tbl.o
 .debug_pubtypes
                0x0000370c      0x360 build/WiFIG/production/_ext/427700826/icmp.o
 .debug_pubtypes
                0x00003a6c      0x12c build/WiFIG/production/_ext/427700826/icmpv6.o
 .debug_pubtypes
                0x00003b98      0x399 build/WiFIG/production/_ext/427700826/ipv4.o
 .debug_pubtypes
                0x00003f31      0x12c build/WiFIG/production/_ext/427700826/ipv6.o
 .debug_pubtypes
                0x0000405d      0x12c build/WiFIG/production/_ext/427700826/mac_events_pic32.o
 .debug_pubtypes
                0x00004189      0x3f7 build/WiFIG/production/_ext/427700826/nbns.o
 .debug_pubtypes
                0x00004580      0x12c build/WiFIG/production/_ext/427700826/ndp.o
 .debug_pubtypes
                0x000046ac      0x12c build/WiFIG/production/_ext/427700826/tcpip_reboot.o
 .debug_pubtypes
                0x000047d8      0x12c build/WiFIG/production/_ext/427700826/rsa.o
 .debug_pubtypes
                0x00004904      0x12c build/WiFIG/production/_ext/427700826/smtp.o
 .debug_pubtypes
                0x00004a30      0x12c build/WiFIG/production/_ext/427700826/snmp.o
 .debug_pubtypes
                0x00004b5c      0x12c build/WiFIG/production/_ext/427700826/snmpv3.o
 .debug_pubtypes
                0x00004c88      0x12c build/WiFIG/production/_ext/427700826/snmpv3_usm.o
 .debug_pubtypes
                0x00004db4      0x12c build/WiFIG/production/_ext/427700826/sntp.o
 .debug_pubtypes
                0x00004ee0      0x12c build/WiFIG/production/_ext/427700826/ssl.o
 .debug_pubtypes
                0x0000500c      0x4a1 build/WiFIG/production/_ext/427700826/tcp.o
 .debug_pubtypes
                0x000054ad      0x203 build/WiFIG/production/_ext/427700826/tcpip_heap_alloc.o
 .debug_pubtypes
                0x000056b0      0x12c build/WiFIG/production/_ext/427700826/tcpip_storage.o
 .debug_pubtypes
                0x000057dc      0x12c build/WiFIG/production/_ext/427700826/telnet.o
 .debug_pubtypes
                0x00005908      0x12c build/WiFIG/production/_ext/427700826/tftpc.o
 .debug_pubtypes
                0x00005a34      0x44b build/WiFIG/production/_ext/427700826/udp.o
 .debug_pubtypes
                0x00005e7f      0x238 build/WiFIG/production/_ext/427700826/tcpip_mac_object.o
 .debug_pubtypes
                0x000060b7      0x5c4 build/WiFIG/production/_ext/427700826/tcpip_manager.o
 .debug_pubtypes
                0x0000667b      0x262 build/WiFIG/production/_ext/427700826/tcpip_helpers.o
 .debug_pubtypes
                0x000068dd      0x12c build/WiFIG/production/_ext/427700826/tcpip_commands.o
 .debug_pubtypes
                0x00006a09      0x12c build/WiFIG/production/_ext/427700826/iperf.o
 .debug_pubtypes
                0x00006b35       0x6c build/WiFIG/production/_ext/427700826/tcpip_notify.o
 .debug_pubtypes
                0x00006ba1      0x12c build/WiFIG/production/_ext/427700826/zero_conf_helper.o
 .debug_pubtypes
                0x00006ccd      0x141 build/WiFIG/production/_ext/427700826/zero_conf_link_local.o
 .debug_pubtypes
                0x00006e0e      0x12c build/WiFIG/production/_ext/427700826/zero_conf_multicast_dns.o
 .debug_pubtypes
                0x00006f3a      0x155 build/WiFIG/production/_ext/334706090/wf_tx_power.o
 .debug_pubtypes
                0x0000708f      0x20c build/WiFIG/production/_ext/334706090/wf_connect.o
 .debug_pubtypes
                0x0000729b      0x1f9 build/WiFIG/production/_ext/334706090/wf_connection_algorithm.o
 .debug_pubtypes
                0x00007494      0x17b build/WiFIG/production/_ext/334706090/wf_connection_manager.o
 .debug_pubtypes
                0x0000760f      0x27f build/WiFIG/production/_ext/334706090/wf_connection_profile.o
 .debug_pubtypes
                0x0000788e      0x1c0 build/WiFIG/production/_ext/334706090/wf_easy_config.o
 .debug_pubtypes
                0x00007a4e      0x160 build/WiFIG/production/_ext/334706090/wf_eint.o
 .debug_pubtypes
                0x00007bae      0x21b build/WiFIG/production/_ext/334706090/wf_event_handler.o
 .debug_pubtypes
                0x00007dc9      0x22c build/WiFIG/production/_ext/334706090/wf_init.o
 .debug_pubtypes
                0x00007ff5      0x1bf build/WiFIG/production/_ext/334706090/wf_power_save.o
 .debug_pubtypes
                0x000081b4      0x171 build/WiFIG/production/_ext/334706090/wf_scan.o
 .debug_pubtypes
                0x00008325      0x16c build/WiFIG/production/_ext/334706090/wf_spi.o
 .debug_pubtypes
                0x00008491      0x343 build/WiFIG/production/_ext/334706090/mrf24w_mac_pic32.o
 .debug_pubtypes
                0x000087d4      0x1e2 build/WiFIG/production/_ext/334706090/mrf24w_events.o
 .debug_pubtypes
                0x000089b6      0x295 build/WiFIG/production/_ext/334706090/wf_debug_output.o
 .debug_pubtypes
                0x00008c4b      0x2b8 build/WiFIG/production/_ext/334706090/wf_commands.o
 .debug_pubtypes
                0x00008f03      0x12c build/WiFIG/production/_ext/334706090/wf_pbkdf2.o
 .debug_pubtypes
                0x0000902f      0x26e build/WiFIG/production/_ext/334706090/wf_driver_com_24g.o
 .debug_pubtypes
                0x0000929d      0x16a build/WiFIG/production/_ext/334706090/wf_driver_raw_24g.o
 .debug_pubtypes
                0x00009407      0x295 build/WiFIG/production/_ext/334706090/wf_mac_24g.o
 .debug_pubtypes
                0x0000969c      0x17e build/WiFIG/production/_ext/334706090/wf_mgmt_msg_24g.o
 .debug_pubtypes
                0x0000981a      0x21b build/WiFIG/production/_ext/334706090/wf_param_msg_24g.o
 .debug_pubtypes
                0x00009a35      0x217 build/WiFIG/production/_ext/334706090/wf_configData.o
 .debug_pubtypes
                0x00009c4c      0x2e3 build/WiFIG/production/_ext/1472/main_demo.o
 .debug_pubtypes
                0x00009f2f       0xe7 build/WiFIG/production/_ext/1472/mpfs_img2.o
 .debug_pubtypes
                0x0000a016      0x111 build/WiFIG/production/_ext/1472/wf_config.o
 .debug_pubtypes
                0x0000a127      0x268 build/WiFIG/production/_ext/1472/tcp6_demo_app.o
 .debug_pubtypes
                0x0000a38f       0x59 c:/program files (x86)/microchip/xc32/v1.21/bin/../lib/gcc/pic32mx/4.5.2/size\libgcc.a(_udivdi3.o)
 .debug_pubtypes
                0x0000a3e8       0x62 c:/program files (x86)/microchip/xc32/v1.21/bin/../lib/gcc/pic32mx/4.5.2/size\libgcc.a(_lshrdi3.o)
 .debug_pubtypes
                0x0000a44a       0x40 c:/program files (x86)/microchip/xc32/v1.21/bin/../lib/gcc/pic32mx/4.5.2/size\libgcc.a(_floatundisf.o)
 .debug_pubtypes
                0x0000a48a       0x59 c:/program files (x86)/microchip/xc32/v1.21/bin/../lib/gcc/pic32mx/4.5.2/size\libgcc.a(_umoddi3.o)
 .debug_pubtypes
                0x0000a4e3       0x34 c:/program files (x86)/microchip/xc32/v1.21/bin/../lib/gcc/pic32mx/4.5.2/size\libgcc.a(floatunsisf.o)

.debug_ranges   0x00000000     0x2138
 *(.debug_ranges)
 .debug_ranges  0x00000000       0x10 build/WiFIG/production/_ext/1293749816/bsp.o
 .debug_ranges  0x00000010       0x50 build/WiFIG/production/_ext/101875047/hashes.o
 .debug_ranges  0x00000060       0x18 build/WiFIG/production/_ext/101875047/lfsr.o
 .debug_ranges  0x00000078       0x70 build/WiFIG/production/_ext/101875047/big_int.o
 .debug_ranges  0x000000e8       0x48 build/WiFIG/production/_ext/101875047/helpers.o
 .debug_ranges  0x00000130       0x20 build/WiFIG/production/_ext/1472/ping_demo.o
 .debug_ranges  0x00000150      0x150 build/WiFIG/production/_ext/365611741/system_services.o
 .debug_ranges  0x000002a0       0x90 build/WiFIG/production/_ext/365611741/system_debug.o
 .debug_ranges  0x00000330       0x30 build/WiFIG/production/_ext/365611741/system_random.o
 .debug_ranges  0x00000360       0x48 build/WiFIG/production/_ext/365611741/system_userio.o
 .debug_ranges  0x000003a8       0x40 build/WiFIG/production/_ext/792872985/usart.o
 .debug_ranges  0x000003e8       0x20 build/WiFIG/production/_ext/792872985/drv_spi.o
 .debug_ranges  0x00000408       0x40 build/WiFIG/production/_ext/427700826/tcpip_announce.o
 .debug_ranges  0x00000448      0x128 build/WiFIG/production/_ext/427700826/arp.o
 .debug_ranges  0x00000570       0xa0 build/WiFIG/production/_ext/427700826/dhcp.o
 .debug_ranges  0x00000610       0x20 build/WiFIG/production/_ext/427700826/dhcps.o
 .debug_ranges  0x00000630       0x60 build/WiFIG/production/_ext/427700826/dns.o
 .debug_ranges  0x00000690       0x18 build/WiFIG/production/_ext/427700826/hash_fnv.o
 .debug_ranges  0x000006a8       0x48 build/WiFIG/production/_ext/427700826/hash_tbl.o
 .debug_ranges  0x000006f0       0x40 build/WiFIG/production/_ext/427700826/icmp.o
 .debug_ranges  0x00000730      0x140 build/WiFIG/production/_ext/427700826/ipv4.o
 .debug_ranges  0x00000870       0x30 build/WiFIG/production/_ext/427700826/nbns.o
 .debug_ranges  0x000008a0      0x290 build/WiFIG/production/_ext/427700826/tcp.o
 .debug_ranges  0x00000b30       0x88 build/WiFIG/production/_ext/427700826/tcpip_heap_alloc.o
 .debug_ranges  0x00000bb8      0x160 build/WiFIG/production/_ext/427700826/udp.o
 .debug_ranges  0x00000d18       0xc8 build/WiFIG/production/_ext/427700826/tcpip_mac_object.o
 .debug_ranges  0x00000de0      0x288 build/WiFIG/production/_ext/427700826/tcpip_manager.o
 .debug_ranges  0x00001068       0xd8 build/WiFIG/production/_ext/427700826/tcpip_helpers.o
 .debug_ranges  0x00001140       0x20 build/WiFIG/production/_ext/427700826/tcpip_notify.o
 .debug_ranges  0x00001160       0x20 build/WiFIG/production/_ext/427700826/zero_conf_link_local.o
 .debug_ranges  0x00001180       0x20 build/WiFIG/production/_ext/334706090/wf_tx_power.o
 .debug_ranges  0x000011a0       0x30 build/WiFIG/production/_ext/334706090/wf_connect.o
 .debug_ranges  0x000011d0       0x98 build/WiFIG/production/_ext/334706090/wf_connection_algorithm.o
 .debug_ranges  0x00001268       0x40 build/WiFIG/production/_ext/334706090/wf_connection_manager.o
 .debug_ranges  0x000012a8       0xc8 build/WiFIG/production/_ext/334706090/wf_connection_profile.o
 .debug_ranges  0x00001370       0x10 build/WiFIG/production/_ext/334706090/wf_easy_config.o
 .debug_ranges  0x00001380       0x30 build/WiFIG/production/_ext/334706090/wf_eint.o
 .debug_ranges  0x000013b0       0x58 build/WiFIG/production/_ext/334706090/wf_event_handler.o
 .debug_ranges  0x00001408       0x30 build/WiFIG/production/_ext/334706090/wf_init.o
 .debug_ranges  0x00001438       0x80 build/WiFIG/production/_ext/334706090/wf_power_save.o
 .debug_ranges  0x000014b8       0x20 build/WiFIG/production/_ext/334706090/wf_scan.o
 .debug_ranges  0x000014d8       0x30 build/WiFIG/production/_ext/334706090/wf_spi.o
 .debug_ranges  0x00001508       0xf8 build/WiFIG/production/_ext/334706090/mrf24w_mac_pic32.o
 .debug_ranges  0x00001600       0x60 build/WiFIG/production/_ext/334706090/mrf24w_events.o
 .debug_ranges  0x00001660       0xa8 build/WiFIG/production/_ext/334706090/wf_debug_output.o
 .debug_ranges  0x00001708       0x80 build/WiFIG/production/_ext/334706090/wf_commands.o
 .debug_ranges  0x00001788       0xc8 build/WiFIG/production/_ext/334706090/wf_driver_com_24g.o
 .debug_ranges  0x00001850       0xb0 build/WiFIG/production/_ext/334706090/wf_driver_raw_24g.o
 .debug_ranges  0x00001900      0x100 build/WiFIG/production/_ext/334706090/wf_mac_24g.o
 .debug_ranges  0x00001a00       0x30 build/WiFIG/production/_ext/334706090/wf_mgmt_msg_24g.o
 .debug_ranges  0x00001a30       0xd8 build/WiFIG/production/_ext/334706090/wf_param_msg_24g.o
 .debug_ranges  0x00001b08       0x28 build/WiFIG/production/_ext/334706090/wf_configData.o
 .debug_ranges  0x00001b30       0x28 build/WiFIG/production/_ext/1472/main_demo.o
 .debug_ranges  0x00001b58       0x10 build/WiFIG/production/_ext/1472/wf_config.o
 .debug_ranges  0x00001b68       0x30 build/WiFIG/production/_ext/1472/tcp6_demo_app.o
 .debug_ranges  0x00001b98       0x10 c:/program files (x86)/microchip/xc32/v1.21/bin/../lib/gcc/pic32mx/4.5.2/../../../../pic32mx/lib/size\libmchp_peripheral.a(open_core_timer_lib.o)
 .debug_ranges  0x00001ba8       0x10 c:/program files (x86)/microchip/xc32/v1.21/bin/../lib/gcc/pic32mx/4.5.2/../../../../pic32mx/lib/size\libmchp_peripheral_32MX695F512H.a(soft_reset_lib.o)
 .debug_ranges  0x00001bb8       0x18 c:/program files (x86)/microchip/xc32/v1.21/bin/../lib/gcc/pic32mx/4.5.2/../../../../pic32mx/lib/size\libmchp_peripheral_32MX695F512H.a(pcache.o)
 .debug_ranges  0x00001bd0       0x10 c:/program files (x86)/microchip/xc32/v1.21/bin/../lib/gcc/pic32mx/4.5.2/../../../../pic32mx/lib/size\libmchp_peripheral_32MX695F512H.a(int_disable_interrupts_lib.o)
 .debug_ranges  0x00001be0       0x10 c:/program files (x86)/microchip/xc32/v1.21/bin/../lib/gcc/pic32mx/4.5.2/../../../../pic32mx/lib/size\libmchp_peripheral_32MX695F512H.a(int_restore_interrupts_lib.o)
 .debug_ranges  0x00001bf0       0x10 c:/program files (x86)/microchip/xc32/v1.21/bin/../lib/gcc/pic32mx/4.5.2/../../../../pic32mx/lib/size\libmchp_peripheral_32MX695F512H.a(int_enable_mv_int_lib.o)
 .debug_ranges  0x00001c00       0x50 c:/program files (x86)/microchip/xc32/v1.21/bin/../lib/gcc/pic32mx/4.5.2/../../../../pic32mx/lib/size\libmchp_peripheral_32MX695F512H.a(int_tbl_lib.o)
 .debug_ranges  0x00001c50       0x10 c:/program files (x86)/microchip/xc32/v1.21/bin/../lib/gcc/pic32mx/4.5.2/../../../../pic32mx/lib/size\libmchp_peripheral_32MX695F512H.a(rtcc_init_lib.o)
 .debug_ranges  0x00001c60       0x10 c:/program files (x86)/microchip/xc32/v1.21/bin/../lib/gcc/pic32mx/4.5.2/../../../../pic32mx/lib/size\libmchp_peripheral_32MX695F512H.a(rtcc_open_lib.o)
 .debug_ranges  0x00001c70       0x10 c:/program files (x86)/microchip/xc32/v1.21/bin/../lib/gcc/pic32mx/4.5.2/../../../../pic32mx/lib/size\libmchp_peripheral_32MX695F512H.a(spi_chn_data_rdy_lib.o)
 .debug_ranges  0x00001c80       0x18 c:/program files (x86)/microchip/xc32/v1.21/bin/../lib/gcc/pic32mx/4.5.2/../../../../pic32mx/lib/size\libmchp_peripheral_32MX695F512H.a(spi_chn_getc_lib.o)
 .debug_ranges  0x00001c98       0x10 c:/program files (x86)/microchip/xc32/v1.21/bin/../lib/gcc/pic32mx/4.5.2/../../../../pic32mx/lib/size\libmchp_peripheral_32MX695F512H.a(spi_chn_open_lib.o)
 .debug_ranges  0x00001ca8       0x20 c:/program files (x86)/microchip/xc32/v1.21/bin/../lib/gcc/pic32mx/4.5.2/../../../../pic32mx/lib/size\libmchp_peripheral_32MX695F512H.a(spi_chn_putc_lib.o)
 .debug_ranges  0x00001cc8       0x10 c:/program files (x86)/microchip/xc32/v1.21/bin/../lib/gcc/pic32mx/4.5.2/../../../../pic32mx/lib/size\libmchp_peripheral_32MX695F512H.a(spi_chn_tx_buff_empty_lib.o)
 .debug_ranges  0x00001cd8       0x10 c:/program files (x86)/microchip/xc32/v1.21/bin/../lib/gcc/pic32mx/4.5.2/../../../../pic32mx/lib/size\libmchp_peripheral_32MX695F512H.a(port_set_pins_digital_in_lib.o)
 .debug_ranges  0x00001ce8       0x10 c:/program files (x86)/microchip/xc32/v1.21/bin/../lib/gcc/pic32mx/4.5.2/../../../../pic32mx/lib/size\libmchp_peripheral_32MX695F512H.a(port_set_pins_digital_out_lib.o)
 .debug_ranges  0x00001cf8       0x10 c:/program files (x86)/microchip/xc32/v1.21/bin/../lib/gcc/pic32mx/4.5.2/../../../../pic32mx/lib/size\libmchp_peripheral_32MX695F512H.a(int_enable_interrupts_lib.o)
 .debug_ranges  0x00001d08       0x18 c:/program files (x86)/microchip/xc32/v1.21/bin/../lib/gcc/pic32mx/4.5.2/../../../../pic32mx/lib/size\libmchp_peripheral_32MX695F512H.a(_rtcc_wait_clock_off_lib.o)
 .debug_ranges  0x00001d20       0x10 c:/program files (x86)/microchip/xc32/v1.21/bin/../lib/gcc/pic32mx/4.5.2/../../../../pic32mx/lib/size\libmchp_peripheral_32MX695F512H.a(read_core_timer_lib.o)
 .debug_ranges  0x00001d30       0xc0 c:/program files (x86)/microchip/xc32/v1.21/bin/../lib/gcc/pic32mx/4.5.2/size\libgcc.a(_udivdi3.o)
 .debug_ranges  0x00001df0       0x10 c:/program files (x86)/microchip/xc32/v1.21/bin/../lib/gcc/pic32mx/4.5.2/../../../../pic32mx/lib/size\libpic32.a(default-bootstrap-exception-handler.o)
 .debug_ranges  0x00001e00       0x10 c:/program files (x86)/microchip/xc32/v1.21/bin/../lib/gcc/pic32mx/4.5.2/../../../../pic32mx/lib/size\libpic32.a(default-on-reset.o)
 .debug_ranges  0x00001e10       0x10 c:/program files (x86)/microchip/xc32/v1.21/bin/../lib/gcc/pic32mx/4.5.2/../../../../pic32mx/lib/size\libpic32.a(default-on-bootstrap.o)
 .debug_ranges  0x00001e20       0x10 c:/program files (x86)/microchip/xc32/v1.21/bin/../lib/gcc/pic32mx/4.5.2/../../../../pic32mx/lib/size\libpic32.a(defaultinterrupt.o)
 .debug_ranges  0x00001e30       0x10 c:/program files (x86)/microchip/xc32/v1.21/bin/../lib/gcc/pic32mx/4.5.2/../../../../pic32mx/lib/size\libc.a(atoi.o)
 .debug_ranges  0x00001e40       0x20 c:/program files (x86)/microchip/xc32/v1.21/bin/../lib/gcc/pic32mx/4.5.2/../../../../pic32mx/lib/size\libc.a(malloc.o)
 .debug_ranges  0x00001e60       0x18 c:/program files (x86)/microchip/xc32/v1.21/bin/../lib/gcc/pic32mx/4.5.2/../../../../pic32mx/lib/size\libc.a(rand.o)
 .debug_ranges  0x00001e78       0x10 c:/program files (x86)/microchip/xc32/v1.21/bin/../lib/gcc/pic32mx/4.5.2/../../../../pic32mx/lib/size\libc.a(strcat.o)
 .debug_ranges  0x00001e88       0x10 c:/program files (x86)/microchip/xc32/v1.21/bin/../lib/gcc/pic32mx/4.5.2/../../../../pic32mx/lib/size\libc.a(strchr.o)
 .debug_ranges  0x00001e98       0x10 c:/program files (x86)/microchip/xc32/v1.21/bin/../lib/gcc/pic32mx/4.5.2/../../../../pic32mx/lib/size\libc.a(strncat.o)
 .debug_ranges  0x00001ea8       0x10 c:/program files (x86)/microchip/xc32/v1.21/bin/../lib/gcc/pic32mx/4.5.2/../../../../pic32mx/lib/size\libc.a(strncpy.o)
 .debug_ranges  0x00001eb8       0x10 c:/program files (x86)/microchip/xc32/v1.21/bin/../lib/gcc/pic32mx/4.5.2/../../../../pic32mx/lib/size\libc.a(strstr.o)
 .debug_ranges  0x00001ec8       0x18 c:/program files (x86)/microchip/xc32/v1.21/bin/../lib/gcc/pic32mx/4.5.2/../../../../pic32mx/lib/size\libc.a(strtol.o)
 .debug_ranges  0x00001ee0       0x10 c:/program files (x86)/microchip/xc32/v1.21/bin/../lib/gcc/pic32mx/4.5.2/../../../../pic32mx/lib/size\libc.a(snprintf_cdnopsuxX.eo)
 .debug_ranges  0x00001ef0       0x10 c:/program files (x86)/microchip/xc32/v1.21/bin/../lib/gcc/pic32mx/4.5.2/../../../../pic32mx/lib/size\libc.a(sprintf_cdnopsuxX.eo)
 .debug_ranges  0x00001f00       0x10 c:/program files (x86)/microchip/xc32/v1.21/bin/../lib/gcc/pic32mx/4.5.2/../../../../pic32mx/lib/size\libc.a(vsnprintf_cdnopsuxX.eo)
 .debug_ranges  0x00001f10       0x10 c:/program files (x86)/microchip/xc32/v1.21/bin/../lib/gcc/pic32mx/4.5.2/../../../../pic32mx/lib/size\libc.a(vsnprintf.o)
 .debug_ranges  0x00001f20       0x90 c:/program files (x86)/microchip/xc32/v1.21/bin/../lib/gcc/pic32mx/4.5.2/../../../../pic32mx/lib/size\libc.a(ctypef.o)
 .debug_ranges  0x00001fb0       0x10 c:/program files (x86)/microchip/xc32/v1.21/bin/../lib/gcc/pic32mx/4.5.2/../../../../pic32mx/lib/size\libc.a(strncmp.o)
 .debug_ranges  0x00001fc0       0x10 c:/program files (x86)/microchip/xc32/v1.21/bin/../lib/gcc/pic32mx/4.5.2/../../../../pic32mx/lib/size\libc.a(doprnt_cdnopsuxX.eo)
 .debug_ranges  0x00001fd0       0x20 c:/program files (x86)/microchip/xc32/v1.21/bin/../lib/gcc/pic32mx/4.5.2/../../../../pic32mx/lib/size\libc.a(doprnt.o)
 .debug_ranges  0x00001ff0       0x10 c:/program files (x86)/microchip/xc32/v1.21/bin/../lib/gcc/pic32mx/4.5.2/../../../../pic32mx/lib/size\libc.a(_fputc_simple.o)
 .debug_ranges  0x00002000       0x10 c:/program files (x86)/microchip/xc32/v1.21/bin/../lib/gcc/pic32mx/4.5.2/../../../../pic32mx/lib/size\libc.a(_flsbuf_simple.o)
 .debug_ranges  0x00002010       0x30 c:/program files (x86)/microchip/xc32/v1.21/bin/../lib/gcc/pic32mx/4.5.2/../../../../pic32mx/lib/size\libpic32.a(sbrk.o)
 .debug_ranges  0x00002040       0x10 c:/program files (x86)/microchip/xc32/v1.21/bin/../lib/gcc/pic32mx/4.5.2/../../../../pic32mx/lib/size\libpic32.a(write.o)
 .debug_ranges  0x00002050       0x10 c:/program files (x86)/microchip/xc32/v1.21/bin/../lib/gcc/pic32mx/4.5.2/../../../../pic32mx/lib/size\libpic32.a(_mon_putc.o)
 .debug_ranges  0x00002060       0x10 c:/program files (x86)/microchip/xc32/v1.21/bin/../lib/gcc/pic32mx/4.5.2/../../../../pic32mx/lib/size\libe.a(_floatdisf.o)
 .debug_ranges  0x00002070       0xc8 c:/program files (x86)/microchip/xc32/v1.21/bin/../lib/gcc/pic32mx/4.5.2/size\libgcc.a(_umoddi3.o)

.gnu.attributes
                0x00000000       0x10
 *(.gnu.attributes)
 .gnu.attributes
                0x00000000       0x10 build/WiFIG/production/_ext/1293749816/bsp.o
 .gnu.attributes
                0x00000010       0x10 build/WiFIG/production/_ext/101875047/hashes.o
 .gnu.attributes
                0x00000020       0x10 build/WiFIG/production/_ext/101875047/lfsr.o
 .gnu.attributes
                0x00000030       0x10 build/WiFIG/production/_ext/101875047/big_int.o
 .gnu.attributes
                0x00000040       0x10 build/WiFIG/production/_ext/101875047/helpers.o
 .gnu.attributes
                0x00000050       0x10 build/WiFIG/production/_ext/1472/berkeley_tcp_client_demo.o
 .gnu.attributes
                0x00000060       0x10 build/WiFIG/production/_ext/1472/berkeley_tcp_server_demo.o
 .gnu.attributes
                0x00000070       0x10 build/WiFIG/production/_ext/1472/berkeley_udp_client_demo.o
 .gnu.attributes
                0x00000080       0x10 build/WiFIG/production/_ext/1472/generic_tcp_client.o
 .gnu.attributes
                0x00000090       0x10 build/WiFIG/production/_ext/1472/generic_tcp_server.o
 .gnu.attributes
                0x000000a0       0x10 build/WiFIG/production/_ext/1472/ping_demo.o
 .gnu.attributes
                0x000000b0       0x10 build/WiFIG/production/_ext/1472/smtp_demo.o
 .gnu.attributes
                0x000000c0       0x10 build/WiFIG/production/_ext/365611741/system_services.o
 .gnu.attributes
                0x000000d0       0x10 build/WiFIG/production/_ext/365611741/system_debug.o
 .gnu.attributes
                0x000000e0       0x10 build/WiFIG/production/_ext/365611741/system_random.o
 .gnu.attributes
                0x000000f0       0x10 build/WiFIG/production/_ext/365611741/system_command.o
 .gnu.attributes
                0x00000100       0x10 build/WiFIG/production/_ext/365611741/system_userio.o
 .gnu.attributes
                0x00000110       0x10 build/WiFIG/production/_ext/97638081/sys_fs.o
 .gnu.attributes
                0x00000120       0x10 build/WiFIG/production/_ext/97638081/mpfs2.o
 .gnu.attributes
                0x00000130       0x10 build/WiFIG/production/_ext/792872985/usart.o
 .gnu.attributes
                0x00000140       0x10 build/WiFIG/production/_ext/792872985/lcd.o
 .gnu.attributes
                0x00000150       0x10 build/WiFIG/production/_ext/792872985/drv_spi.o
 .gnu.attributes
                0x00000160       0x10 build/WiFIG/production/_ext/792872985/db_appio.o
 .gnu.attributes
                0x00000170       0x10 build/WiFIG/production/_ext/792872985/spi_ram.o
 .gnu.attributes
                0x00000180       0x10 build/WiFIG/production/_ext/792872985/spi_eeprom.o
 .gnu.attributes
                0x00000190       0x10 build/WiFIG/production/_ext/792872985/spi_flash.o
 .gnu.attributes
                0x000001a0       0x10 build/WiFIG/production/_ext/792872985/drv_media.o
 .gnu.attributes
                0x000001b0       0x10 build/WiFIG/production/_ext/427700826/tcpip_announce.o
 .gnu.attributes
                0x000001c0       0x10 build/WiFIG/production/_ext/427700826/http2.o
 .gnu.attributes
                0x000001d0       0x10 build/WiFIG/production/_ext/427700826/arcfour.o
 .gnu.attributes
                0x000001e0       0x10 build/WiFIG/production/_ext/427700826/arp.o
 .gnu.attributes
                0x000001f0       0x10 build/WiFIG/production/_ext/427700826/berkeley_api.o
 .gnu.attributes
                0x00000200       0x10 build/WiFIG/production/_ext/427700826/dhcp.o
 .gnu.attributes
                0x00000210       0x10 build/WiFIG/production/_ext/427700826/dhcps.o
 .gnu.attributes
                0x00000220       0x10 build/WiFIG/production/_ext/427700826/dns.o
 .gnu.attributes
                0x00000230       0x10 build/WiFIG/production/_ext/427700826/dnss.o
 .gnu.attributes
                0x00000240       0x10 build/WiFIG/production/_ext/427700826/dyn_dns.o
 .gnu.attributes
                0x00000250       0x10 build/WiFIG/production/_ext/427700826/enc28_mac.o
 .gnu.attributes
                0x00000260       0x10 build/WiFIG/production/_ext/427700826/enc28j60.o
 .gnu.attributes
                0x00000270       0x10 build/WiFIG/production/_ext/427700826/encs24j600.o
 .gnu.attributes
                0x00000280       0x10 build/WiFIG/production/_ext/427700826/encx24_mac.o
 .gnu.attributes
                0x00000290       0x10 build/WiFIG/production/_ext/427700826/eth_pic32_ext_phy.o
 .gnu.attributes
                0x000002a0       0x10 build/WiFIG/production/_ext/427700826/eth_pic32_ext_phy_dp83848.o
 .gnu.attributes
                0x000002b0       0x10 build/WiFIG/production/_ext/427700826/eth_pic32_int_mac.o
 .gnu.attributes
                0x000002c0       0x10 build/WiFIG/production/_ext/427700826/ftp.o
 .gnu.attributes
                0x000002d0       0x10 build/WiFIG/production/_ext/427700826/hash_fnv.o
 .gnu.attributes
                0x000002e0       0x10 build/WiFIG/production/_ext/427700826/hash_tbl.o
 .gnu.attributes
                0x000002f0       0x10 build/WiFIG/production/_ext/427700826/icmp.o
 .gnu.attributes
                0x00000300       0x10 build/WiFIG/production/_ext/427700826/icmpv6.o
 .gnu.attributes
                0x00000310       0x10 build/WiFIG/production/_ext/427700826/ipv4.o
 .gnu.attributes
                0x00000320       0x10 build/WiFIG/production/_ext/427700826/ipv6.o
 .gnu.attributes
                0x00000330       0x10 build/WiFIG/production/_ext/427700826/mac_events_pic32.o
 .gnu.attributes
                0x00000340       0x10 build/WiFIG/production/_ext/427700826/nbns.o
 .gnu.attributes
                0x00000350       0x10 build/WiFIG/production/_ext/427700826/ndp.o
 .gnu.attributes
                0x00000360       0x10 build/WiFIG/production/_ext/427700826/tcpip_reboot.o
 .gnu.attributes
                0x00000370       0x10 build/WiFIG/production/_ext/427700826/rsa.o
 .gnu.attributes
                0x00000380       0x10 build/WiFIG/production/_ext/427700826/smtp.o
 .gnu.attributes
                0x00000390       0x10 build/WiFIG/production/_ext/427700826/snmp.o
 .gnu.attributes
                0x000003a0       0x10 build/WiFIG/production/_ext/427700826/snmpv3.o
 .gnu.attributes
                0x000003b0       0x10 build/WiFIG/production/_ext/427700826/snmpv3_usm.o
 .gnu.attributes
                0x000003c0       0x10 build/WiFIG/production/_ext/427700826/sntp.o
 .gnu.attributes
                0x000003d0       0x10 build/WiFIG/production/_ext/427700826/ssl.o
 .gnu.attributes
                0x000003e0       0x10 build/WiFIG/production/_ext/427700826/tcp.o
 .gnu.attributes
                0x000003f0       0x10 build/WiFIG/production/_ext/427700826/tcpip_heap_alloc.o
 .gnu.attributes
                0x00000400       0x10 build/WiFIG/production/_ext/427700826/tcpip_storage.o
 .gnu.attributes
                0x00000410       0x10 build/WiFIG/production/_ext/427700826/telnet.o
 .gnu.attributes
                0x00000420       0x10 build/WiFIG/production/_ext/427700826/tftpc.o
 .gnu.attributes
                0x00000430       0x10 build/WiFIG/production/_ext/427700826/udp.o
 .gnu.attributes
                0x00000440       0x10 build/WiFIG/production/_ext/427700826/tcpip_mac_object.o
 .gnu.attributes
                0x00000450       0x10 build/WiFIG/production/_ext/427700826/tcpip_manager.o
 .gnu.attributes
                0x00000460       0x10 build/WiFIG/production/_ext/427700826/tcpip_helpers.o
 .gnu.attributes
                0x00000470       0x10 build/WiFIG/production/_ext/427700826/tcpip_commands.o
 .gnu.attributes
                0x00000480       0x10 build/WiFIG/production/_ext/427700826/iperf.o
 .gnu.attributes
                0x00000490       0x10 build/WiFIG/production/_ext/427700826/tcpip_notify.o
 .gnu.attributes
                0x000004a0       0x10 build/WiFIG/production/_ext/427700826/zero_conf_helper.o
 .gnu.attributes
                0x000004b0       0x10 build/WiFIG/production/_ext/427700826/zero_conf_link_local.o
 .gnu.attributes
                0x000004c0       0x10 build/WiFIG/production/_ext/427700826/zero_conf_multicast_dns.o
 .gnu.attributes
                0x000004d0       0x10 build/WiFIG/production/_ext/334706090/wf_tx_power.o
 .gnu.attributes
                0x000004e0       0x10 build/WiFIG/production/_ext/334706090/wf_connect.o
 .gnu.attributes
                0x000004f0       0x10 build/WiFIG/production/_ext/334706090/wf_connection_algorithm.o
 .gnu.attributes
                0x00000500       0x10 build/WiFIG/production/_ext/334706090/wf_connection_manager.o
 .gnu.attributes
                0x00000510       0x10 build/WiFIG/production/_ext/334706090/wf_connection_profile.o
 .gnu.attributes
                0x00000520       0x10 build/WiFIG/production/_ext/334706090/wf_easy_config.o
 .gnu.attributes
                0x00000530       0x10 build/WiFIG/production/_ext/334706090/wf_eint.o
 .gnu.attributes
                0x00000540       0x10 build/WiFIG/production/_ext/334706090/wf_event_handler.o
 .gnu.attributes
                0x00000550       0x10 build/WiFIG/production/_ext/334706090/wf_init.o
 .gnu.attributes
                0x00000560       0x10 build/WiFIG/production/_ext/334706090/wf_power_save.o
 .gnu.attributes
                0x00000570       0x10 build/WiFIG/production/_ext/334706090/wf_scan.o
 .gnu.attributes
                0x00000580       0x10 build/WiFIG/production/_ext/334706090/wf_spi.o
 .gnu.attributes
                0x00000590       0x10 build/WiFIG/production/_ext/334706090/mrf24w_mac_pic32.o
 .gnu.attributes
                0x000005a0       0x10 build/WiFIG/production/_ext/334706090/mrf24w_events.o
 .gnu.attributes
                0x000005b0       0x10 build/WiFIG/production/_ext/334706090/wf_debug_output.o
 .gnu.attributes
                0x000005c0       0x10 build/WiFIG/production/_ext/334706090/wf_commands.o
 .gnu.attributes
                0x000005d0       0x10 build/WiFIG/production/_ext/334706090/wf_pbkdf2.o
 .gnu.attributes
                0x000005e0       0x10 build/WiFIG/production/_ext/334706090/wf_driver_com_24g.o
 .gnu.attributes
                0x000005f0       0x10 build/WiFIG/production/_ext/334706090/wf_driver_raw_24g.o
 .gnu.attributes
                0x00000600       0x10 build/WiFIG/production/_ext/334706090/wf_mac_24g.o
 .gnu.attributes
                0x00000610       0x10 build/WiFIG/production/_ext/334706090/wf_mgmt_msg_24g.o
 .gnu.attributes
                0x00000620       0x10 build/WiFIG/production/_ext/334706090/wf_param_msg_24g.o
 .gnu.attributes
                0x00000630       0x10 build/WiFIG/production/_ext/334706090/wf_configData.o
 .gnu.attributes
                0x00000640       0x10 build/WiFIG/production/_ext/1472/main_demo.o
 .gnu.attributes
                0x00000650       0x10 build/WiFIG/production/_ext/1472/custom_snmp_app.o
 .gnu.attributes
                0x00000660       0x10 build/WiFIG/production/_ext/1472/custom_ssl_cert.o
 .gnu.attributes
                0x00000670       0x10 build/WiFIG/production/_ext/1472/mpfs_img2.o
 .gnu.attributes
                0x00000680       0x10 build/WiFIG/production/_ext/1472/wf_config.o
 .gnu.attributes
                0x00000690       0x10 build/WiFIG/production/_ext/1472/custom_http_app.o
 .gnu.attributes
                0x000006a0       0x10 build/WiFIG/production/_ext/1472/tcp6_demo_app.o
 .gnu.attributes
                0x000006b0       0x10 c:/program files (x86)/microchip/xc32/v1.21/bin/../lib/gcc/pic32mx/4.5.2/../../../../pic32mx/lib/size\libmchp_peripheral.a(open_core_timer_lib.o)
 .gnu.attributes
                0x000006c0       0x10 c:/program files (x86)/microchip/xc32/v1.21/bin/../lib/gcc/pic32mx/4.5.2/../../../../pic32mx/lib/size\libmchp_peripheral_32MX695F512H.a(soft_reset_lib.o)
 .gnu.attributes
                0x000006d0       0x10 c:/program files (x86)/microchip/xc32/v1.21/bin/../lib/gcc/pic32mx/4.5.2/../../../../pic32mx/lib/size\libmchp_peripheral_32MX695F512H.a(pcache.o)
 .gnu.attributes
                0x000006e0       0x10 c:/program files (x86)/microchip/xc32/v1.21/bin/../lib/gcc/pic32mx/4.5.2/../../../../pic32mx/lib/size\libmchp_peripheral_32MX695F512H.a(int_disable_interrupts_lib.o)
 .gnu.attributes
                0x000006f0       0x10 c:/program files (x86)/microchip/xc32/v1.21/bin/../lib/gcc/pic32mx/4.5.2/../../../../pic32mx/lib/size\libmchp_peripheral_32MX695F512H.a(int_restore_interrupts_lib.o)
 .gnu.attributes
                0x00000700       0x10 c:/program files (x86)/microchip/xc32/v1.21/bin/../lib/gcc/pic32mx/4.5.2/../../../../pic32mx/lib/size\libmchp_peripheral_32MX695F512H.a(int_enable_mv_int_lib.o)
 .gnu.attributes
                0x00000710       0x10 c:/program files (x86)/microchip/xc32/v1.21/bin/../lib/gcc/pic32mx/4.5.2/../../../../pic32mx/lib/size\libmchp_peripheral_32MX695F512H.a(int_tbl_lib.o)
 .gnu.attributes
                0x00000720       0x10 c:/program files (x86)/microchip/xc32/v1.21/bin/../lib/gcc/pic32mx/4.5.2/../../../../pic32mx/lib/size\libmchp_peripheral_32MX695F512H.a(rtcc_init_lib.o)
 .gnu.attributes
                0x00000730       0x10 c:/program files (x86)/microchip/xc32/v1.21/bin/../lib/gcc/pic32mx/4.5.2/../../../../pic32mx/lib/size\libmchp_peripheral_32MX695F512H.a(rtcc_open_lib.o)
 .gnu.attributes
                0x00000740       0x10 c:/program files (x86)/microchip/xc32/v1.21/bin/../lib/gcc/pic32mx/4.5.2/../../../../pic32mx/lib/size\libmchp_peripheral_32MX695F512H.a(spi_chn_data_rdy_lib.o)
 .gnu.attributes
                0x00000750       0x10 c:/program files (x86)/microchip/xc32/v1.21/bin/../lib/gcc/pic32mx/4.5.2/../../../../pic32mx/lib/size\libmchp_peripheral_32MX695F512H.a(spi_chn_getc_lib.o)
 .gnu.attributes
                0x00000760       0x10 c:/program files (x86)/microchip/xc32/v1.21/bin/../lib/gcc/pic32mx/4.5.2/../../../../pic32mx/lib/size\libmchp_peripheral_32MX695F512H.a(spi_chn_open_lib.o)
 .gnu.attributes
                0x00000770       0x10 c:/program files (x86)/microchip/xc32/v1.21/bin/../lib/gcc/pic32mx/4.5.2/../../../../pic32mx/lib/size\libmchp_peripheral_32MX695F512H.a(spi_chn_putc_lib.o)
 .gnu.attributes
                0x00000780       0x10 c:/program files (x86)/microchip/xc32/v1.21/bin/../lib/gcc/pic32mx/4.5.2/../../../../pic32mx/lib/size\libmchp_peripheral_32MX695F512H.a(spi_chn_tx_buff_empty_lib.o)
 .gnu.attributes
                0x00000790       0x10 c:/program files (x86)/microchip/xc32/v1.21/bin/../lib/gcc/pic32mx/4.5.2/../../../../pic32mx/lib/size\libmchp_peripheral_32MX695F512H.a(spi_io_tbl_libp.o)
 .gnu.attributes
                0x000007a0       0x10 c:/program files (x86)/microchip/xc32/v1.21/bin/../lib/gcc/pic32mx/4.5.2/../../../../pic32mx/lib/size\libmchp_peripheral_32MX695F512H.a(spi_map_tbl_libp.o)
 .gnu.attributes
                0x000007b0       0x10 c:/program files (x86)/microchip/xc32/v1.21/bin/../lib/gcc/pic32mx/4.5.2/../../../../pic32mx/lib/size\libmchp_peripheral_32MX695F512H.a(port_set_pins_digital_in_lib.o)
 .gnu.attributes
                0x000007c0       0x10 c:/program files (x86)/microchip/xc32/v1.21/bin/../lib/gcc/pic32mx/4.5.2/../../../../pic32mx/lib/size\libmchp_peripheral_32MX695F512H.a(port_set_pins_digital_out_lib.o)
 .gnu.attributes
                0x000007d0       0x10 c:/program files (x86)/microchip/xc32/v1.21/bin/../lib/gcc/pic32mx/4.5.2/../../../../pic32mx/lib/size\libmchp_peripheral_32MX695F512H.a(_ports_tbl_libp.o)
 .gnu.attributes
                0x000007e0       0x10 c:/program files (x86)/microchip/xc32/v1.21/bin/../lib/gcc/pic32mx/4.5.2/../../../../pic32mx/lib/size\libmchp_peripheral_32MX695F512H.a(int_enable_interrupts_lib.o)
 .gnu.attributes
                0x000007f0       0x10 c:/program files (x86)/microchip/xc32/v1.21/bin/../lib/gcc/pic32mx/4.5.2/../../../../pic32mx/lib/size\libmchp_peripheral_32MX695F512H.a(_rtcc_wait_clock_off_lib.o)
 .gnu.attributes
                0x00000800       0x10 c:/program files (x86)/microchip/xc32/v1.21/bin/../lib/gcc/pic32mx/4.5.2/../../../../pic32mx/lib/size\libmchp_peripheral_32MX695F512H.a(read_core_timer_lib.o)
 .gnu.attributes
                0x00000810       0x10 c:/program files (x86)/microchip/xc32/v1.21/bin/../lib/gcc/pic32mx/4.5.2/size\libgcc.a(_udivdi3.o)
 .gnu.attributes
                0x00000820       0x10 c:/program files (x86)/microchip/xc32/v1.21/bin/../lib/gcc/pic32mx/4.5.2/../../../../pic32mx/lib/size\libpic32.a(default-bootstrap-exception-handler.o)
 .gnu.attributes
                0x00000830       0x10 c:/program files (x86)/microchip/xc32/v1.21/bin/../lib/gcc/pic32mx/4.5.2/../../../../pic32mx/lib/size\libpic32.a(default-on-reset.o)
 .gnu.attributes
                0x00000840       0x10 c:/program files (x86)/microchip/xc32/v1.21/bin/../lib/gcc/pic32mx/4.5.2/../../../../pic32mx/lib/size\libpic32.a(default-on-bootstrap.o)
 .gnu.attributes
                0x00000850       0x10 c:/program files (x86)/microchip/xc32/v1.21/bin/../lib/gcc/pic32mx/4.5.2/../../../../pic32mx/lib/size\libpic32.a(defaultinterrupt.o)
 .gnu.attributes
                0x00000860       0x10 c:/program files (x86)/microchip/xc32/v1.21/bin/../lib/gcc/pic32mx/4.5.2/../../../../pic32mx/lib/size\libc.a(atoi.o)
 .gnu.attributes
                0x00000870       0x10 c:/program files (x86)/microchip/xc32/v1.21/bin/../lib/gcc/pic32mx/4.5.2/../../../../pic32mx/lib/size\libc.a(ctype.o)
 .gnu.attributes
                0x00000880       0x10 c:/program files (x86)/microchip/xc32/v1.21/bin/../lib/gcc/pic32mx/4.5.2/../../../../pic32mx/lib/size\libc.a(malloc.o)
 .gnu.attributes
                0x00000890       0x10 c:/program files (x86)/microchip/xc32/v1.21/bin/../lib/gcc/pic32mx/4.5.2/../../../../pic32mx/lib/size\libc.a(rand.o)
 .gnu.attributes
                0x000008a0       0x10 c:/program files (x86)/microchip/xc32/v1.21/bin/../lib/gcc/pic32mx/4.5.2/../../../../pic32mx/lib/size\libc.a(strcat.o)
 .gnu.attributes
                0x000008b0       0x10 c:/program files (x86)/microchip/xc32/v1.21/bin/../lib/gcc/pic32mx/4.5.2/../../../../pic32mx/lib/size\libc.a(strchr.o)
 .gnu.attributes
                0x000008c0       0x10 c:/program files (x86)/microchip/xc32/v1.21/bin/../lib/gcc/pic32mx/4.5.2/../../../../pic32mx/lib/size\libc.a(strncat.o)
 .gnu.attributes
                0x000008d0       0x10 c:/program files (x86)/microchip/xc32/v1.21/bin/../lib/gcc/pic32mx/4.5.2/../../../../pic32mx/lib/size\libc.a(strncpy.o)
 .gnu.attributes
                0x000008e0       0x10 c:/program files (x86)/microchip/xc32/v1.21/bin/../lib/gcc/pic32mx/4.5.2/../../../../pic32mx/lib/size\libc.a(strstr.o)
 .gnu.attributes
                0x000008f0       0x10 c:/program files (x86)/microchip/xc32/v1.21/bin/../lib/gcc/pic32mx/4.5.2/../../../../pic32mx/lib/size\libc.a(strtol.o)
 .gnu.attributes
                0x00000900       0x10 c:/program files (x86)/microchip/xc32/v1.21/bin/../lib/gcc/pic32mx/4.5.2/../../../../pic32mx/lib/size\libc.a(snprintf_cdnopsuxX.eo)
 .gnu.attributes
                0x00000910       0x10 c:/program files (x86)/microchip/xc32/v1.21/bin/../lib/gcc/pic32mx/4.5.2/../../../../pic32mx/lib/size\libc.a(sprintf_cdnopsuxX.eo)
 .gnu.attributes
                0x00000920       0x10 c:/program files (x86)/microchip/xc32/v1.21/bin/../lib/gcc/pic32mx/4.5.2/../../../../pic32mx/lib/size\libc.a(vsnprintf_cdnopsuxX.eo)
 .gnu.attributes
                0x00000930       0x10 c:/program files (x86)/microchip/xc32/v1.21/bin/../lib/gcc/pic32mx/4.5.2/../../../../pic32mx/lib/size\libc.a(vsnprintf.o)
 .gnu.attributes
                0x00000940       0x10 c:/program files (x86)/microchip/xc32/v1.21/bin/../lib/gcc/pic32mx/4.5.2/../../../../pic32mx/lib/size\libc.a(ctypef.o)
 .gnu.attributes
                0x00000950       0x10 c:/program files (x86)/microchip/xc32/v1.21/bin/../lib/gcc/pic32mx/4.5.2/../../../../pic32mx/lib/size\libc.a(errno.o)
 .gnu.attributes
                0x00000960       0x10 c:/program files (x86)/microchip/xc32/v1.21/bin/../lib/gcc/pic32mx/4.5.2/../../../../pic32mx/lib/size\libc.a(strncmp.o)
 .gnu.attributes
                0x00000970       0x10 c:/program files (x86)/microchip/xc32/v1.21/bin/../lib/gcc/pic32mx/4.5.2/../../../../pic32mx/lib/size\libc.a(doprnt_cdnopsuxX.eo)
 .gnu.attributes
                0x00000980       0x10 c:/program files (x86)/microchip/xc32/v1.21/bin/../lib/gcc/pic32mx/4.5.2/../../../../pic32mx/lib/size\libc.a(doprnt.o)
 .gnu.attributes
                0x00000990       0x10 c:/program files (x86)/microchip/xc32/v1.21/bin/../lib/gcc/pic32mx/4.5.2/../../../../pic32mx/lib/size\libc.a(_fputc_simple.o)
 .gnu.attributes
                0x000009a0       0x10 c:/program files (x86)/microchip/xc32/v1.21/bin/../lib/gcc/pic32mx/4.5.2/../../../../pic32mx/lib/size\libc.a(powersf.o)
 .gnu.attributes
                0x000009b0       0x10 c:/program files (x86)/microchip/xc32/v1.21/bin/../lib/gcc/pic32mx/4.5.2/../../../../pic32mx/lib/size\libc.a(_iob.o)
 .gnu.attributes
                0x000009c0       0x10 c:/program files (x86)/microchip/xc32/v1.21/bin/../lib/gcc/pic32mx/4.5.2/../../../../pic32mx/lib/size\libc.a(_flsbuf_simple.o)
 .gnu.attributes
                0x000009d0       0x10 c:/program files (x86)/microchip/xc32/v1.21/bin/../lib/gcc/pic32mx/4.5.2/../../../../pic32mx/lib/size\libpic32.a(sbrk.o)
 .gnu.attributes
                0x000009e0       0x10 c:/program files (x86)/microchip/xc32/v1.21/bin/../lib/gcc/pic32mx/4.5.2/../../../../pic32mx/lib/size\libpic32.a(write.o)
 .gnu.attributes
                0x000009f0       0x10 c:/program files (x86)/microchip/xc32/v1.21/bin/../lib/gcc/pic32mx/4.5.2/../../../../pic32mx/lib/size\libpic32.a(_mon_putc.o)
 .gnu.attributes
                0x00000a00       0x10 c:/program files (x86)/microchip/xc32/v1.21/bin/../lib/gcc/pic32mx/4.5.2/../../../../pic32mx/lib/size\libpic32.a(xc32_uart.o)
 .gnu.attributes
                0x00000a10       0x10 c:/program files (x86)/microchip/xc32/v1.21/bin/../lib/gcc/pic32mx/4.5.2/../../../../pic32mx/lib/size\libe.a(_floatdisf.o)
 .gnu.attributes
                0x00000a20       0x10 c:/program files (x86)/microchip/xc32/v1.21/bin/../lib/gcc/pic32mx/4.5.2/size\libgcc.a(_lshrdi3.o)
 .gnu.attributes
                0x00000a30       0x10 c:/program files (x86)/microchip/xc32/v1.21/bin/../lib/gcc/pic32mx/4.5.2/size\libgcc.a(_floatundisf.o)
 .gnu.attributes
                0x00000a40       0x10 c:/program files (x86)/microchip/xc32/v1.21/bin/../lib/gcc/pic32mx/4.5.2/size\libgcc.a(_umoddi3.o)
 .gnu.attributes
                0x00000a50       0x10 c:/program files (x86)/microchip/xc32/v1.21/bin/../lib/gcc/pic32mx/4.5.2/size\libgcc.a(floatunsisf.o)
LOAD c:/program files (x86)/microchip/xc32/v1.21/bin/../lib/gcc/pic32mx/4.5.2/size\libgcc.a
START GROUP
LOAD c:/program files (x86)/microchip/xc32/v1.21/bin/../lib/gcc/pic32mx/4.5.2/../../../../pic32mx/lib/size\libpic32.a
LOAD c:/program files (x86)/microchip/xc32/v1.21/bin/../lib/gcc/pic32mx/4.5.2/../../../../pic32mx/lib/size\libdebug.a
LOAD c:/program files (x86)/microchip/xc32/v1.21/bin/../lib/gcc/pic32mx/4.5.2/../../../../pic32mx/lib/size\libm.a
LOAD c:/program files (x86)/microchip/xc32/v1.21/bin/../lib/gcc/pic32mx/4.5.2/../../../../pic32mx/lib/size\libe.a
LOAD c:/program files (x86)/microchip/xc32/v1.21/bin/../lib/gcc/pic32mx/4.5.2/../../../../pic32mx/lib/size\libdsp.a
LOAD c:/program files (x86)/microchip/xc32/v1.21/bin/../lib/gcc/pic32mx/4.5.2/size\libgcc.a
LOAD c:/program files (x86)/microchip/xc32/v1.21/bin/../lib/gcc/pic32mx/4.5.2/../../../../pic32mx/lib/size\libpic32.a
LOAD c:/program files (x86)/microchip/xc32/v1.21/bin/../lib/gcc/pic32mx/4.5.2/../../../../pic32mx/lib/size\libc.a
LOAD c:/program files (x86)/microchip/xc32/v1.21/bin/../lib/gcc/pic32mx/4.5.2/../../../../pic32mx/lib/size\libpic32.a
END GROUP
LOAD c:/program files (x86)/microchip/xc32/v1.21/bin/../lib/gcc/pic32mx/4.5.2/size\libgcc.a
OUTPUT(dist/WiFIG/production/tcp6_demo_app_wifi.X.production.elf elf32-tradlittlemips)
LOAD stack
LOAD data_init

.reginfo        0x9d000000       0x18
 .reginfo       0x9d000000       0x18 c:/program files (x86)/microchip/xc32/v1.21/bin/../lib/gcc/pic32mx/4.5.2/../../../../pic32mx/lib/size/crt0.o

.stack          0xa0007618      0x800
 .stack         0xa0007618      0x800 stack

.data           0xa00020c0      0x208
 .data          0xa00020c0      0x174 build/WiFIG/production/_ext/334706090/wf_debug_output.o
                0xa00020c0                connectionFailureStrings
                0xa0002110                deauthDisssocReasonCodes
                0xa0002174                statusCodes
 .data          0xa0002234       0x94 build/WiFIG/production/_ext/1472/tcp6_demo_app.o
                0xa0002234                WeatherString
                0xa0002284                b64

.bss            0xa00022c8      0x128
 .bss           0xa00022c8       0x5c build/WiFIG/production/_ext/365611741/system_random.o
 .bss           0xa0002324       0x50 build/WiFIG/production/_ext/365611741/system_userio.o
 .bss           0xa0002374       0x40 c:/program files (x86)/microchip/xc32/v1.21/bin/../lib/gcc/pic32mx/4.5.2/../../../../pic32mx/lib/size\libc.a(_iob.o)
                0xa0002374                _sibuf
                0xa0002394                _sobuf
 .bss           0xa00023b4       0x1c c:/program files (x86)/microchip/xc32/v1.21/bin/../lib/gcc/pic32mx/4.5.2/../../../../pic32mx/lib/size\libpic32.a(sbrk.o)
 .bss           0xa00023d0       0x10 c:/program files (x86)/microchip/xc32/v1.21/bin/../lib/gcc/pic32mx/4.5.2/../../../../pic32mx/lib/size\libc.a(malloc.o)
                0xa00023d0                __allocs
 .bss           0xa00023e0       0x10 c:/program files (x86)/microchip/xc32/v1.21/bin/../lib/gcc/pic32mx/4.5.2/../../../../pic32mx/lib/size\libc.a(rand.o)

.text._TcpHandleSeg
                0x9d000020     0x1778
 .text._TcpHandleSeg
                0x9d000020     0x1778 build/WiFIG/production/_ext/427700826/tcp.o

.text.vfprintf  0x9d001798     0x15a8
 .text.vfprintf
                0x9d001798     0x15a8 c:/program files (x86)/microchip/xc32/v1.21/bin/../lib/gcc/pic32mx/4.5.2/../../../../pic32mx/lib/size\libc.a(doprnt.o)
                0x9d001798                vfprintf

.text.DNSClientTask
                0x9d002d40     0x1144
 .text.DNSClientTask
                0x9d002d40     0x1144 build/WiFIG/production/_ext/427700826/dns.o
                0x9d002d40                DNSClientTask

.text.tcp6_demo_app_tasks
                0x9d003e84     0x10f0
 .text.tcp6_demo_app_tasks
                0x9d003e84     0x10f0 build/WiFIG/production/_ext/1472/tcp6_demo_app.o
                0x9d003e84                tcp6_demo_app_tasks

.rodata         0x9d004f74     0x1084
 .rodata        0x9d004f74     0x1084 build/WiFIG/production/_ext/334706090/wf_debug_output.o

.text.DHCPTask  0x9d005ff8      0xa74
 .text.DHCPTask
                0x9d005ff8      0xa74 build/WiFIG/production/_ext/427700826/dhcp.o
                0x9d005ff8                DHCPTask

.text._TcpSend  0x9d006a6c      0xa40
 .text._TcpSend
                0x9d006a6c      0xa40 build/WiFIG/production/_ext/427700826/tcp.o

.text           0x9d0074ac      0x8ec
 .text          0x9d0074ac      0x8ec c:/program files (x86)/microchip/xc32/v1.21/bin/../lib/gcc/pic32mx/4.5.2/../../../../pic32mx/lib/size\libm.a(fp32.o)
                0x9d0074ac                fpsub
                0x9d0074ac                __subsf3
                0x9d0074b4                __addsf3
                0x9d0074b4                fpadd
                0x9d007720                __mulsf3
                0x9d007720                fpmul
                0x9d0078d8                fpdiv
                0x9d0078d8                __divsf3
                0x9d007b04                sitofp
                0x9d007b04                litofp
                0x9d007b04                __floatsisf
                0x9d007b60                ultofp
                0x9d007b60                uitofp
                0x9d007bac                fptosi
                0x9d007bac                fptoli
                0x9d007bac                __fixsfsi
                0x9d007c24                fptoui
                0x9d007c24                __fixunssfsi
                0x9d007c24                fptoul
                0x9d007c98                __nesf2
                0x9d007c98                fpcmp
                0x9d007c98                __eqsf2
                0x9d007c98                __gesf2
                0x9d007c98                __ltsf2
                0x9d007c98                __gtsf2
                0x9d007c98                __lesf2
                0x9d007d2c                fpfabs
                0x9d007d2c                fabsf
                0x9d007d3c                __negsf2
                0x9d007d4c                fpnan
                0x9d007d4c                nanf

.text._vfprintf_cdnopsuxX
                0x9d007d98      0x8b8
 .text._vfprintf_cdnopsuxX
                0x9d007d98      0x8b8 c:/program files (x86)/microchip/xc32/v1.21/bin/../lib/gcc/pic32mx/4.5.2/../../../../pic32mx/lib/size\libc.a(doprnt_cdnopsuxX.eo)
                0x9d007d98                _vfprintf_cdnopsuxX
                0x9d007d98                _vfprintf_cdnopuxX

.text.TCPTick   0x9d008650      0x890
 .text.TCPTick  0x9d008650      0x890 build/WiFIG/production/_ext/427700826/tcp.o
                0x9d008650                TCPTick

.rodata         0x9d008ee0      0x7d4
 .rodata        0x9d008ee0      0x7d4 c:/program files (x86)/microchip/xc32/v1.21/bin/../lib/gcc/pic32mx/4.5.2/../../../../pic32mx/lib/size\libmchp_peripheral_32MX695F512H.a(int_tbl_lib.o)
                0x9d008ee0                __IntSrcTbl
                0x9d0093fc                __IntVectorTbl

.text._DHCPReceive
                0x9d0096b4      0x748
 .text._DHCPReceive
                0x9d0096b4      0x748 build/WiFIG/production/_ext/427700826/dhcp.o

.text.NBNSTask  0x9d009dfc      0x73c
 .text.NBNSTask
                0x9d009dfc      0x73c build/WiFIG/production/_ext/427700826/nbns.o
                0x9d009dfc                NBNSTask

.dinit          0x9d00a538      0x6d0
 .dinit         0x9d00a538      0x6d0 data_init

.text._DHCPSend
                0x9d00ac08      0x5c8
 .text._DHCPSend
                0x9d00ac08      0x5c8 build/WiFIG/production/_ext/427700826/dhcp.o

.text.SHA1HashBlock
                0x9d00b1d0      0x4fc
 .text.SHA1HashBlock
                0x9d00b1d0      0x4fc build/WiFIG/production/_ext/101875047/hashes.o

.rodata         0x9d00b6cc      0x4f4
 .rodata        0x9d00b6cc      0x4f4 build/WiFIG/production/_ext/1472/tcp6_demo_app.o
                0x9d00b6cc                Version
                0x9d00b6d0                CompileDate
                0x9d00b6dc                CompileTime
                0x9d00b804                HTTP_TRANSACTION_LIST

.text.TCPIP_ANNOUNCE_Send
                0x9d00bbc0      0x490
 .text.TCPIP_ANNOUNCE_Send
                0x9d00bbc0      0x490 build/WiFIG/production/_ext/427700826/tcpip_announce.o
                0x9d00bbc0                TCPIP_ANNOUNCE_Send

.text._TCPIP_HEAP_Free
                0x9d00c050      0x490
 .text._TCPIP_HEAP_Free
                0x9d00c050      0x490 build/WiFIG/production/_ext/427700826/tcpip_heap_alloc.o
                0x9d00c050                _TCPIP_HEAP_Free

.text.TCPIP_STACK_Init
                0x9d00c4e0      0x464
 .text.TCPIP_STACK_Init
                0x9d00c4e0      0x464 build/WiFIG/production/_ext/427700826/tcpip_manager.o
                0x9d00c4e0                TCPIP_STACK_Init

.text           0x9d00c944      0x8a0
 .text          0x9d00c944      0x460 c:/program files (x86)/microchip/xc32/v1.21/bin/../lib/gcc/pic32mx/4.5.2/size\libgcc.a(_umoddi3.o)
                0x9d00c944                __umoddi3
 .text          0x9d00cda4      0x440 c:/program files (x86)/microchip/xc32/v1.21/bin/../lib/gcc/pic32mx/4.5.2/size\libgcc.a(_udivdi3.o)
                0x9d00cda4                __udivdi3

.text.TCPIP_STACK_BringNetUp
                0x9d00d1e4      0x438
 .text.TCPIP_STACK_BringNetUp
                0x9d00d1e4      0x438 build/WiFIG/production/_ext/427700826/tcpip_manager.o

.text.TCPOpen   0x9d00d61c      0x420
 .text.TCPOpen  0x9d00d61c      0x420 build/WiFIG/production/_ext/427700826/tcp.o

.rodata         0x9d00da3c      0x3fc
 .rodata        0x9d00da3c      0x3fc build/WiFIG/production/_ext/427700826/tcpip_manager.o

.text.ARPInitialize
                0x9d00de38      0x3f4
 .text.ARPInitialize
                0x9d00de38      0x3f4 build/WiFIG/production/_ext/427700826/arp.o
                0x9d00de38                ARPInitialize

.text._TcpFindMatchingSocket
                0x9d00e22c      0x3e8
 .text._TcpFindMatchingSocket
                0x9d00e22c      0x3e8 build/WiFIG/production/_ext/427700826/tcp.o

.text           0x9d00e614      0x3dc
 .text          0x9d00e614      0x3dc c:/program files (x86)/microchip/xc32/v1.21/bin/../lib/gcc/pic32mx/4.5.2/../../../../pic32mx/lib/size\libm.a(fpmod32.o)
                0x9d00e614                fpfmod
                0x9d00e614                fmodf
                0x9d00e758                fpfrexp
                0x9d00e758                frexpf
                0x9d00e7dc                fpldexp
                0x9d00e7dc                __mchp_ldexpf
                0x9d00e920                fpmodf
                0x9d00e920                modff

.text.WFProcessMgmtIndicateMsg
                0x9d00e9f0      0x3b0
 .text.WFProcessMgmtIndicateMsg
                0x9d00e9f0      0x3b0 build/WiFIG/production/_ext/334706090/wf_event_handler.o
                0x9d00e9f0                WFProcessMgmtIndicateMsg

.text.SYS_Initialize
                0x9d00eda0      0x3a8
 .text.SYS_Initialize
                0x9d00eda0      0x3a8 build/WiFIG/production/_ext/365611741/system_services.o
                0x9d00eda0                SYS_Initialize

.text.FindMatchingSocket
                0x9d00f148      0x39c
 .text.FindMatchingSocket
                0x9d00f148      0x39c build/WiFIG/production/_ext/427700826/udp.o

.text.OutputSecurityMode
                0x9d00f4e4      0x38c
 .text.OutputSecurityMode
                0x9d00f4e4      0x38c build/WiFIG/production/_ext/334706090/wf_debug_output.o

.text.TCPIP_STACK_Task
                0x9d00f870      0x35c
 .text.TCPIP_STACK_Task
                0x9d00f870      0x35c build/WiFIG/production/_ext/427700826/tcpip_manager.o
                0x9d00f870                TCPIP_STACK_Task

.text.main      0x9d00fbcc      0x358
 .text.main     0x9d00fbcc      0x358 build/WiFIG/production/_ext/1472/main_demo.o
                0x9d00fbcc                main

.text.UDPOpen   0x9d00ff24      0x330
 .text.UDPOpen  0x9d00ff24      0x330 build/WiFIG/production/_ext/427700826/udp.o

.text.TCPIP_HELPER_StringToIPAddress
                0x9d010254      0x31c
 .text.TCPIP_HELPER_StringToIPAddress
                0x9d010254      0x31c build/WiFIG/production/_ext/427700826/tcpip_helpers.o
                0x9d010254                TCPIP_HELPER_StringToIPAddress

.text.OutputConnectionFailedMsg
                0x9d010570      0x31c
 .text.OutputConnectionFailedMsg
                0x9d010570      0x31c build/WiFIG/production/_ext/334706090/wf_debug_output.o

.text.ARPTask   0x9d01088c      0x310
 .text.ARPTask  0x9d01088c      0x310 build/WiFIG/production/_ext/427700826/arp.o
                0x9d01088c                ARPTask

.text.TCPIP_IPV4_PutArrayHelper
                0x9d010b9c      0x310
 .text.TCPIP_IPV4_PutArrayHelper
                0x9d010b9c      0x310 build/WiFIG/production/_ext/427700826/ipv4.o
                0x9d010b9c                TCPIP_IPV4_PutArrayHelper

.text.UDPInit   0x9d010eac      0x300
 .text.UDPInit  0x9d010eac      0x300 build/WiFIG/production/_ext/427700826/udp.o
                0x9d010eac                UDPInit

.text.tcp6_demo_app_init
                0x9d0111ac      0x2c4
 .text.tcp6_demo_app_init
                0x9d0111ac      0x2c4 build/WiFIG/production/_ext/1472/tcp6_demo_app.o
                0x9d0111ac                tcp6_demo_app_init

.text.ICMPProcess
                0x9d011470      0x2ac
 .text.ICMPProcess
                0x9d011470      0x2ac build/WiFIG/production/_ext/427700826/icmp.o
                0x9d011470                ICMPProcess

.text.TCPPutArray
                0x9d01171c      0x2ac
 .text.TCPPutArray
                0x9d01171c      0x2ac build/WiFIG/production/_ext/427700826/tcp.o
                0x9d01171c                TCPPutArray

.text.Wifi_Connect
                0x9d0119c8      0x284
 .text.Wifi_Connect
                0x9d0119c8      0x284 build/WiFIG/production/_ext/334706090/wf_connect.o
                0x9d0119c8                Wifi_Connect

.text.UDPProcessIPv4
                0x9d011c4c      0x278
 .text.UDPProcessIPv4
                0x9d011c4c      0x278 build/WiFIG/production/_ext/427700826/udp.o
                0x9d011c4c                UDPProcessIPv4

.text.SyncENCPtrRAWState
                0x9d011ec4      0x278
 .text.SyncENCPtrRAWState
                0x9d011ec4      0x278 build/WiFIG/production/_ext/334706090/wf_mac_24g.o

.text.GetMaxSegSizeOption
                0x9d01213c      0x274
 .text.GetMaxSegSizeOption
                0x9d01213c      0x274 build/WiFIG/production/_ext/427700826/tcp.o

.text.WriteAnalogRegisterBitBang
                0x9d0123b0      0x270
 .text.WriteAnalogRegisterBitBang
                0x9d0123b0      0x270 build/WiFIG/production/_ext/334706090/wf_driver_com_24g.o

.text.TCPIP_IPV4_CalculatePayloadChecksum
                0x9d012620      0x268
 .text.TCPIP_IPV4_CalculatePayloadChecksum
                0x9d012620      0x268 build/WiFIG/production/_ext/427700826/ipv4.o
                0x9d012620                TCPIP_IPV4_CalculatePayloadChecksum

.text.TCPGetArray
                0x9d012888      0x260
 .text.TCPGetArray
                0x9d012888      0x260 build/WiFIG/production/_ext/427700826/tcp.o
                0x9d012888                TCPGetArray

.text.SYS_GENERATE_RANDOM_DWORD
                0x9d012ae8      0x25c
 .text.SYS_GENERATE_RANDOM_DWORD
                0x9d012ae8      0x25c build/WiFIG/production/_ext/365611741/system_random.o
                0x9d012ae8                SYS_GENERATE_RANDOM_DWORD

.text.SYS_CLK_OscClockGet
                0x9d012d44      0x254
 .text.SYS_CLK_OscClockGet
                0x9d012d44      0x254 build/WiFIG/production/_ext/365611741/system_services.o
                0x9d012d44                SYS_CLK_OscClockGet

.text.TCPIP_IPV4_CopyTxPacketStruct
                0x9d012f98      0x250
 .text.TCPIP_IPV4_CopyTxPacketStruct
                0x9d012f98      0x250 build/WiFIG/production/_ext/427700826/ipv4.o
                0x9d012f98                TCPIP_IPV4_CopyTxPacketStruct

.text           0x9d0131e8      0x248
 .text          0x9d0131e8      0x248 build/WiFIG/production/_ext/427700826/tcpip_helper_c32.o
                0x9d0131e8                TCPIP_HELPER_htonl
                0x9d0131f4                TCPIP_HELPER_htons
                0x9d013200                TCPIP_Helper_CalcIPChecksum

.text.LoadDefaultConfig
                0x9d013430      0x244
 .text.LoadDefaultConfig
                0x9d013430      0x244 build/WiFIG/production/_ext/427700826/tcpip_manager.o

.text.ProcessTCPIPMacEvents
                0x9d013674      0x240
 .text.ProcessTCPIPMacEvents
                0x9d013674      0x240 build/WiFIG/production/_ext/427700826/tcpip_manager.o

.text.malloc    0x9d0138b4      0x240
 .text.malloc   0x9d0138b4      0x240 c:/program files (x86)/microchip/xc32/v1.21/bin/../lib/gcc/pic32mx/4.5.2/../../../../pic32mx/lib/size\libc.a(malloc.o)
                0x9d0138b4                malloc

.text.ARPEntryRemoveNet
                0x9d013af4      0x224
 .text.ARPEntryRemoveNet
                0x9d013af4      0x224 build/WiFIG/production/_ext/427700826/arp.o
                0x9d013af4                ARPEntryRemoveNet

.text.TCPIP_IPV4_GetDataSegmentByType
                0x9d013d18      0x224
 .text.TCPIP_IPV4_GetDataSegmentByType
                0x9d013d18      0x224 build/WiFIG/production/_ext/427700826/ipv4.o
                0x9d013d18                TCPIP_IPV4_GetDataSegmentByType

.text.__floatdisf
                0x9d013f3c      0x220
 .text.__floatdisf
                0x9d013f3c      0x220 c:/program files (x86)/microchip/xc32/v1.21/bin/../lib/gcc/pic32mx/4.5.2/../../../../pic32mx/lib/size\libe.a(_floatdisf.o)
                0x9d013f3c                __floatdisf

.text.TCPInit   0x9d01415c      0x210
 .text.TCPInit  0x9d01415c      0x210 build/WiFIG/production/_ext/427700826/tcp.o
                0x9d01415c                TCPInit

.text.DHCPInit  0x9d01436c      0x204
 .text.DHCPInit
                0x9d01436c      0x204 build/WiFIG/production/_ext/427700826/dhcp.o
                0x9d01436c                DHCPInit

.text._TcpDisconnect
                0x9d014570      0x204
 .text._TcpDisconnect
                0x9d014570      0x204 build/WiFIG/production/_ext/427700826/tcp.o

.text.UDPTask   0x9d014774      0x200
 .text.UDPTask  0x9d014774      0x200 build/WiFIG/production/_ext/427700826/udp.o
                0x9d014774                UDPTask

.text.TCPIP_ANNOUNCE_Task
                0x9d014974      0x1f8
 .text.TCPIP_ANNOUNCE_Task
                0x9d014974      0x1f8 build/WiFIG/production/_ext/427700826/tcpip_announce.o
                0x9d014974                TCPIP_ANNOUNCE_Task

.text.ARPProcess
                0x9d014b6c      0x1f0
 .text.ARPProcess
                0x9d014b6c      0x1f0 build/WiFIG/production/_ext/427700826/arp.o
                0x9d014b6c                ARPProcess

.text.TCPIP_IPV4_Flush
                0x9d014d5c      0x1ec
 .text.TCPIP_IPV4_Flush
                0x9d014d5c      0x1ec build/WiFIG/production/_ext/427700826/ipv4.o
                0x9d014d5c                TCPIP_IPV4_Flush

.text._TCPIP_HEAP_Malloc
                0x9d014f48      0x1e0
 .text._TCPIP_HEAP_Malloc
                0x9d014f48      0x1e0 build/WiFIG/production/_ext/427700826/tcpip_heap_alloc.o
                0x9d014f48                _TCPIP_HEAP_Malloc

.text.TCPProcessIPv4
                0x9d015128      0x1dc
 .text.TCPProcessIPv4
                0x9d015128      0x1dc build/WiFIG/production/_ext/427700826/tcp.o
                0x9d015128                TCPProcessIPv4

.text.TCPIP_IPV4_IsTxPutReady
                0x9d015304      0x1d8
 .text.TCPIP_IPV4_IsTxPutReady
                0x9d015304      0x1d8 build/WiFIG/production/_ext/427700826/ipv4.o
                0x9d015304                TCPIP_IPV4_IsTxPutReady

.text.UDPv4IsTxPutReady
                0x9d0154dc      0x1d0
 .text.UDPv4IsTxPutReady
                0x9d0154dc      0x1d0 build/WiFIG/production/_ext/427700826/udp.o

.text._TCPIsPutReady
                0x9d0156ac      0x1cc
 .text._TCPIsPutReady
                0x9d0156ac      0x1cc build/WiFIG/production/_ext/427700826/tcp.o

.text.UDPDeInit
                0x9d015878      0x1cc
 .text.UDPDeInit
                0x9d015878      0x1cc build/WiFIG/production/_ext/427700826/udp.o
                0x9d015878                UDPDeInit

.text.strtoul   0x9d015a44      0x1cc
 .text.strtoul  0x9d015a44      0x1cc c:/program files (x86)/microchip/xc32/v1.21/bin/../lib/gcc/pic32mx/4.5.2/../../../../pic32mx/lib/size\libc.a(strtol.o)
                0x9d015a44                strtoul

.text._TcpSocketSetIdleState
                0x9d015c10      0x1c8
 .text._TcpSocketSetIdleState
                0x9d015c10      0x1c8 build/WiFIG/production/_ext/427700826/tcp.o

.text.MRF24W_MACGetHeader
                0x9d015dd8      0x1b8
 .text.MRF24W_MACGetHeader
                0x9d015dd8      0x1b8 build/WiFIG/production/_ext/334706090/wf_mac_24g.o
                0x9d015dd8                MRF24W_MACGetHeader

.text.WF_ProcessEvent
                0x9d015f90      0x1b4
 .text.WF_ProcessEvent
                0x9d015f90      0x1b4 build/WiFIG/production/_ext/1472/wf_config.o
                0x9d015f90                WF_ProcessEvent

.text._SystemTickIntHandler
                0x9d016144      0x1b0
 .text._SystemTickIntHandler
                0x9d016144      0x1b0 build/WiFIG/production/_ext/365611741/system_services.o
                0x9d016144                _SystemTickIntHandler

.text.isNotifyApp
                0x9d0162f4      0x1a8
 .text.isNotifyApp
                0x9d0162f4      0x1a8 build/WiFIG/production/_ext/334706090/wf_event_handler.o

.rodata         0x9d01649c      0x1a8
 .rodata        0x9d01649c      0x1a8 build/WiFIG/production/_ext/1472/main_demo.o
                0x9d01649c                arpConfigData
                0x9d0164bc                dhcpConfigData
                0x9d0164cc                macPIC32INTConfigData
                0x9d0164dc                macMRF24WConfigData
                0x9d0164dc                mac97J60ConfigData
                0x9d0164dc                macENCJ600ConfigData
                0x9d0164dc                tcpConfigData
                0x9d0164dc                macENCJ60ConfigData
                0x9d0164e4                udpConfigData
                0x9d01653c                TCPIP_HOSTS_CONFIGURATION
                0x9d016564                TCPIP_STACK_MODULE_CONFIG_TBL

.text           0x9d016644      0x1a0
 .text          0x9d016644      0x1a0 c:/program files (x86)/microchip/xc32/v1.21/bin/../lib/gcc/pic32mx/4.5.2/../../../../pic32mx/lib/size\libpic32.a(strcpy.o)
                0x9d016644                strcpy

.text._TcpCloseSocket
                0x9d0167e4      0x198
 .text._TcpCloseSocket
                0x9d0167e4      0x198 build/WiFIG/production/_ext/427700826/tcp.o

.text.NBNSGetName
                0x9d01697c      0x194
 .text.NBNSGetName
                0x9d01697c      0x194 build/WiFIG/production/_ext/427700826/nbns.o

.text._Sys_Ext1_Isr
                0x9d016b10      0x190
 .text._Sys_Ext1_Isr
                0x9d016b10      0x190 build/WiFIG/production/_ext/365611741/system_services.o
                0x9d016b10                _Sys_Ext1_Isr

.text._Sys_Ext3_Isr
                0x9d016ca0      0x190
 .text._Sys_Ext3_Isr
                0x9d016ca0      0x190 build/WiFIG/production/_ext/365611741/system_services.o
                0x9d016ca0                _Sys_Ext3_Isr

.text._Sys_CN_Isr
                0x9d016e30      0x190
 .text._Sys_CN_Isr
                0x9d016e30      0x190 build/WiFIG/production/_ext/365611741/system_services.o
                0x9d016e30                _Sys_CN_Isr

.text.MRF24W_ChipReset
                0x9d016fc0      0x190
 .text.MRF24W_ChipReset
                0x9d016fc0      0x190 build/WiFIG/production/_ext/334706090/wf_driver_com_24g.o
                0x9d016fc0                MRF24W_ChipReset

.text.RawMove   0x9d017150      0x190
 .text.RawMove  0x9d017150      0x190 build/WiFIG/production/_ext/334706090/wf_driver_raw_24g.o

.text.TCPIP_HELPER_StringToMACAddress
                0x9d0172e0      0x18c
 .text.TCPIP_HELPER_StringToMACAddress
                0x9d0172e0      0x18c build/WiFIG/production/_ext/427700826/tcpip_helpers.o
                0x9d0172e0                TCPIP_HELPER_StringToMACAddress

.text.WaitForRawMoveComplete
                0x9d01746c      0x18c
 .text.WaitForRawMoveComplete
                0x9d01746c      0x18c build/WiFIG/production/_ext/334706090/wf_driver_raw_24g.o

.text.UDPGetArray
                0x9d0175f8      0x188
 .text.UDPGetArray
                0x9d0175f8      0x188 build/WiFIG/production/_ext/427700826/udp.o
                0x9d0175f8                UDPGetArray

.text.OutputBeaconTimeout
                0x9d017780      0x188
 .text.OutputBeaconTimeout
                0x9d017780      0x188 build/WiFIG/production/_ext/334706090/wf_debug_output.o

.text._OAHashFindBkt
                0x9d017908      0x180
 .text._OAHashFindBkt
                0x9d017908      0x180 build/WiFIG/production/_ext/427700826/hash_tbl.o

.text.ARPIsResolved
                0x9d017a88      0x178
 .text.ARPIsResolved
                0x9d017a88      0x178 build/WiFIG/production/_ext/427700826/arp.o
                0x9d017a88                ARPIsResolved

.text.TCPIP_IPV4_AllocateTxPacket
                0x9d017c00      0x178
 .text.TCPIP_IPV4_AllocateTxPacket
                0x9d017c00      0x178 build/WiFIG/production/_ext/427700826/ipv4.o
                0x9d017c00                TCPIP_IPV4_AllocateTxPacket

.text.TCPIP_HEAP_Create
                0x9d017d78      0x178
 .text.TCPIP_HEAP_Create
                0x9d017d78      0x178 build/WiFIG/production/_ext/427700826/tcpip_heap_alloc.o
                0x9d017d78                TCPIP_HEAP_Create

.text._ARPProbeAddress
                0x9d017ef0      0x170
 .text._ARPProbeAddress
                0x9d017ef0      0x170 build/WiFIG/production/_ext/427700826/arp.o

.text.SpiChnOpen
                0x9d018060      0x170
 .text.SpiChnOpen
                0x9d018060      0x170 c:/program files (x86)/microchip/xc32/v1.21/bin/../lib/gcc/pic32mx/4.5.2/../../../../pic32mx/lib/size\libmchp_peripheral_32MX695F512H.a(spi_chn_open_lib.o)
                0x9d018060                SpiChnOpen

.text.OAHashLookUpInsert
                0x9d0181d0      0x16c
 .text.OAHashLookUpInsert
                0x9d0181d0      0x16c build/WiFIG/production/_ext/427700826/hash_tbl.o
                0x9d0181d0                OAHashLookUpInsert

.text.UDPv4Flush
                0x9d01833c      0x16c
 .text.UDPv4Flush
                0x9d01833c      0x16c build/WiFIG/production/_ext/427700826/udp.o

.text.WFHardwareInit
                0x9d0184a8      0x168
 .text.WFHardwareInit
                0x9d0184a8      0x168 build/WiFIG/production/_ext/334706090/wf_driver_com_24g.o
                0x9d0184a8                WFHardwareInit

.text.RawSetIndex
                0x9d018610      0x168
 .text.RawSetIndex
                0x9d018610      0x168 build/WiFIG/production/_ext/334706090/wf_driver_raw_24g.o
                0x9d018610                RawSetIndex

.text           0x9d018778      0x2d0
 .text          0x9d018778      0x168 c:/program files (x86)/microchip/xc32/v1.21/bin/../lib/gcc/pic32mx/4.5.2/../../../../pic32mx/lib/size\libpic32.a(memcpy.o)
                0x9d018778                memcpy
 .text          0x9d0188e0      0x168 c:/program files (x86)/microchip/xc32/v1.21/bin/../lib/gcc/pic32mx/4.5.2/../../../../pic32mx/lib/size\libpic32.a(strlen.o)
                0x9d0188e0                strlen

.text.SYS_TICK_TimerDelete
                0x9d018a48      0x160
 .text.SYS_TICK_TimerDelete
                0x9d018a48      0x160 build/WiFIG/production/_ext/365611741/system_services.o
                0x9d018a48                SYS_TICK_TimerDelete

.text.USART_INIT
                0x9d018ba8      0x160
 .text.USART_INIT
                0x9d018ba8      0x160 build/WiFIG/production/_ext/792872985/usart.o
                0x9d018ba8                USART_INIT

.text.DRV_SPI_TxRx
                0x9d018d08      0x160
 .text.DRV_SPI_TxRx
                0x9d018d08      0x160 build/WiFIG/production/_ext/792872985/drv_spi.o
                0x9d018d08                DRV_SPI_TxRx

.text.DNSPutString
                0x9d018e68      0x160
 .text.DNSPutString
                0x9d018e68      0x160 build/WiFIG/production/_ext/427700826/dns.o

.text.TCPIP_IPV4_TransmitPacket
                0x9d018fc8      0x160
 .text.TCPIP_IPV4_TransmitPacket
                0x9d018fc8      0x160 build/WiFIG/production/_ext/427700826/ipv4.o
                0x9d018fc8                TCPIP_IPV4_TransmitPacket

.text.UDPBind   0x9d019128      0x160
 .text.UDPBind  0x9d019128      0x160 build/WiFIG/production/_ext/427700826/udp.o
                0x9d019128                UDPBind

.text.WFEintHandler
                0x9d019288      0x160
 .text.WFEintHandler
                0x9d019288      0x160 build/WiFIG/production/_ext/334706090/wf_driver_com_24g.o
                0x9d019288                WFEintHandler

.text.encodeblock
                0x9d0193e8      0x160
 .text.encodeblock
                0x9d0193e8      0x160 build/WiFIG/production/_ext/1472/tcp6_demo_app.o
                0x9d0193e8                encodeblock

.text.ARP_SendIfPkt
                0x9d019548      0x15c
 .text.ARP_SendIfPkt
                0x9d019548      0x15c build/WiFIG/production/_ext/427700826/arp.o

.text.TCPIP_IPV4_GetHeader
                0x9d0196a4      0x15c
 .text.TCPIP_IPV4_GetHeader
                0x9d0196a4      0x15c build/WiFIG/production/_ext/427700826/ipv4.o
                0x9d0196a4                TCPIP_IPV4_GetHeader

.text.ProcessInterruptServiceResult
                0x9d019800      0x154
 .text.ProcessInterruptServiceResult
                0x9d019800      0x154 build/WiFIG/production/_ext/334706090/wf_driver_com_24g.o

.rodata         0x9d019954      0x150
 .rodata        0x9d019954      0x150 build/WiFIG/production/_ext/365611741/system_debug.o

.text._TCPIPStackIsLocalNetwork
                0x9d019aa4      0x150
 .text._TCPIPStackIsLocalNetwork
                0x9d019aa4      0x150 build/WiFIG/production/_ext/427700826/tcpip_manager.o
                0x9d019aa4                _TCPIPStackIsLocalNetwork

.text.TCPIP_Helper_CalcMACBufferIPChecksum
                0x9d019bf4      0x150
 .text.TCPIP_Helper_CalcMACBufferIPChecksum
                0x9d019bf4      0x150 build/WiFIG/production/_ext/427700826/tcpip_helpers.o
                0x9d019bf4                TCPIP_Helper_CalcMACBufferIPChecksum

.text.OutputChannelList
                0x9d019d44      0x150
 .text.OutputChannelList
                0x9d019d44      0x150 build/WiFIG/production/_ext/334706090/wf_debug_output.o

.text.scale     0x9d019e94      0x150
 .text.scale    0x9d019e94      0x150 c:/program files (x86)/microchip/xc32/v1.21/bin/../lib/gcc/pic32mx/4.5.2/../../../../pic32mx/lib/size\libc.a(doprnt.o)

.text._sbrk_init
                0x9d019fe4      0x14c
 .text._sbrk_init
                0x9d019fe4      0x14c c:/program files (x86)/microchip/xc32/v1.21/bin/../lib/gcc/pic32mx/4.5.2/../../../../pic32mx/lib/size\libpic32.a(sbrk.o)
                0x9d019fe4                _sbrk_init

.text.TCPIP_STACK_DeInit
                0x9d01a130      0x148
 .text.TCPIP_STACK_DeInit
                0x9d01a130      0x148 build/WiFIG/production/_ext/427700826/tcpip_manager.o
                0x9d01a130                TCPIP_STACK_DeInit

.text.OutputConnectionTempLostMsg
                0x9d01a278      0x148
 .text.OutputConnectionTempLostMsg
                0x9d01a278      0x148 build/WiFIG/production/_ext/334706090/wf_debug_output.o

.text.OutputConnectionPermLostMsg
                0x9d01a3c0      0x148
 .text.OutputConnectionPermLostMsg
                0x9d01a3c0      0x148 build/WiFIG/production/_ext/334706090/wf_debug_output.o

.text.SendMgmtMsg
                0x9d01a508      0x148
 .text.SendMgmtMsg
                0x9d01a508      0x148 build/WiFIG/production/_ext/334706090/wf_mgmt_msg_24g.o
                0x9d01a508                SendMgmtMsg

.text.OAHashLookUp
                0x9d01a650      0x144
 .text.OAHashLookUp
                0x9d01a650      0x144 build/WiFIG/production/_ext/427700826/hash_tbl.o
                0x9d01a650                OAHashLookUp

.text.UDPSocketSetNet
                0x9d01a794      0x140
 .text.UDPSocketSetNet
                0x9d01a794      0x140 build/WiFIG/production/_ext/427700826/udp.o
                0x9d01a794                UDPSocketSetNet

.text._WF_OutputConnectionContext
                0x9d01a8d4      0x140
 .text._WF_OutputConnectionContext
                0x9d01a8d4      0x140 build/WiFIG/production/_ext/334706090/wf_debug_output.o
                0x9d01a8d4                _WF_OutputConnectionContext

.text.PowerSaveTask
                0x9d01aa14      0x140
 .text.PowerSaveTask
                0x9d01aa14      0x140 build/WiFIG/production/_ext/334706090/wf_driver_com_24g.o
                0x9d01aa14                PowerSaveTask

.text.WF_SetMultiCastFilter
                0x9d01ab54      0x13c
 .text.WF_SetMultiCastFilter
                0x9d01ab54      0x13c build/WiFIG/production/_ext/334706090/wf_param_msg_24g.o
                0x9d01ab54                WF_SetMultiCastFilter

.text._ARPUpdateEntry
                0x9d01ac90      0x138
 .text._ARPUpdateEntry
                0x9d01ac90      0x138 build/WiFIG/production/_ext/427700826/arp.o

.text.TCPIP_IPV4_QueuedPacketTransmitTask
                0x9d01adc8      0x138
 .text.TCPIP_IPV4_QueuedPacketTransmitTask
                0x9d01adc8      0x138 build/WiFIG/production/_ext/427700826/ipv4.o

.text.UDPIsGetReady
                0x9d01af00      0x138
 .text.UDPIsGetReady
                0x9d01af00      0x138 build/WiFIG/production/_ext/427700826/udp.o
                0x9d01af00                UDPIsGetReady

.text._general_exception_handler
                0x9d01b038      0x134
 .text._general_exception_handler
                0x9d01b038      0x134 build/WiFIG/production/_ext/365611741/system_debug.o
                0x9d01b038                _general_exception_handler

.text.TCPIP_IPV4_InsertIPPacketSegment
                0x9d01b16c      0x134
 .text.TCPIP_IPV4_InsertIPPacketSegment
                0x9d01b16c      0x134 build/WiFIG/production/_ext/427700826/ipv4.o
                0x9d01b16c                TCPIP_IPV4_InsertIPPacketSegment

.text.SetSecurity
                0x9d01b2a0      0x134
 .text.SetSecurity
                0x9d01b2a0      0x134 build/WiFIG/production/_ext/334706090/wf_connection_profile.o

.text.uitoa     0x9d01b3d4      0x130
 .text.uitoa    0x9d01b3d4      0x130 build/WiFIG/production/_ext/101875047/helpers.o
                0x9d01b3d4                uitoa

.text.UDPSetBcastIPV4Address
                0x9d01b504      0x130
 .text.UDPSetBcastIPV4Address
                0x9d01b504      0x130 build/WiFIG/production/_ext/427700826/udp.o
                0x9d01b504                UDPSetBcastIPV4Address

.text.WF_ConfigDataLoad
                0x9d01b634      0x12c
 .text.WF_ConfigDataLoad
                0x9d01b634      0x12c build/WiFIG/production/_ext/334706090/wf_init.o
                0x9d01b634                WF_ConfigDataLoad

.text.DNSBeginUsage
                0x9d01b760      0x128
 .text.DNSBeginUsage
                0x9d01b760      0x128 build/WiFIG/production/_ext/427700826/dns.o
                0x9d01b760                DNSBeginUsage

.text.fputc     0x9d01b888      0x128
 .text.fputc    0x9d01b888      0x128 c:/program files (x86)/microchip/xc32/v1.21/bin/../lib/gcc/pic32mx/4.5.2/../../../../pic32mx/lib/size\libc.a(_fputc_simple.o)
                0x9d01b888                fputc

.text.SYS_USERIO_Initialize
                0x9d01b9b0      0x124
 .text.SYS_USERIO_Initialize
                0x9d01b9b0      0x124 build/WiFIG/production/_ext/365611741/system_userio.o
                0x9d01b9b0                SYS_USERIO_Initialize

.text._TCPSendWinIncUpdate
                0x9d01bad4      0x124
 .text._TCPSendWinIncUpdate
                0x9d01bad4      0x124 build/WiFIG/production/_ext/427700826/tcp.o

.text.WaitForMgmtResponse
                0x9d01bbf8      0x124
 .text.WaitForMgmtResponse
                0x9d01bbf8      0x124 build/WiFIG/production/_ext/334706090/wf_mgmt_msg_24g.o
                0x9d01bbf8                WaitForMgmtResponse

.text.strtol    0x9d01bd1c      0x124
 .text.strtol   0x9d01bd1c      0x124 c:/program files (x86)/microchip/xc32/v1.21/bin/../lib/gcc/pic32mx/4.5.2/../../../../pic32mx/lib/size\libc.a(strtol.o)
                0x9d01bd1c                strtol

.text.TCPIP_IPV4_QueuePacket
                0x9d01be40      0x120
 .text.TCPIP_IPV4_QueuePacket
                0x9d01be40      0x120 build/WiFIG/production/_ext/427700826/ipv4.o

.text.UDPOpenServer
                0x9d01bf60      0x120
 .text.UDPOpenServer
                0x9d01bf60      0x120 build/WiFIG/production/_ext/427700826/udp.o
                0x9d01bf60                UDPOpenServer

.text           0x9d01c080      0x120
 .text          0x9d01c080      0x120 c:/program files (x86)/microchip/xc32/v1.21/bin/../lib/gcc/pic32mx/4.5.2/../../../../pic32mx/lib/size\libpic32.a(strcmp.o)
                0x9d01c080                strcmp

.text.fround    0x9d01c1a0      0x120
 .text.fround   0x9d01c1a0      0x120 c:/program files (x86)/microchip/xc32/v1.21/bin/../lib/gcc/pic32mx/4.5.2/../../../../pic32mx/lib/size\libc.a(doprnt.o)

.text.SHA1AddData
                0x9d01c2c0      0x11c
 .text.SHA1AddData
                0x9d01c2c0      0x11c build/WiFIG/production/_ext/101875047/hashes.o
                0x9d01c2c0                SHA1AddData

.text.b64_encode
                0x9d01c3dc      0x11c
 .text.b64_encode
                0x9d01c3dc      0x11c build/WiFIG/production/_ext/1472/tcp6_demo_app.o
                0x9d01c3dc                b64_encode

.text.TCPIP_IPV4_Initialize
                0x9d01c4f8      0x118
 .text.TCPIP_IPV4_Initialize
                0x9d01c4f8      0x118 build/WiFIG/production/_ext/427700826/ipv4.o
                0x9d01c4f8                TCPIP_IPV4_Initialize

.text.TCPIP_IPV4_PutHeader
                0x9d01c610      0x114
 .text.TCPIP_IPV4_PutHeader
                0x9d01c610      0x114 build/WiFIG/production/_ext/427700826/ipv4.o
                0x9d01c610                TCPIP_IPV4_PutHeader

.text.WiFiAsyncTask
                0x9d01c724      0x110
 .text.WiFiAsyncTask
                0x9d01c724      0x110 build/WiFIG/production/_ext/334706090/wf_event_handler.o
                0x9d01c724                WiFiAsyncTask

.text.WF_PsPollEnable
                0x9d01c834      0x110
 .text.WF_PsPollEnable
                0x9d01c834      0x110 build/WiFIG/production/_ext/334706090/wf_power_save.o
                0x9d01c834                WF_PsPollEnable

.text._flsbuf   0x9d01c944      0x110
 .text._flsbuf  0x9d01c944      0x110 c:/program files (x86)/microchip/xc32/v1.21/bin/../lib/gcc/pic32mx/4.5.2/../../../../pic32mx/lib/size\libc.a(_flsbuf_simple.o)
                0x9d01c944                _flsbuf

.text._TcpSwapHeader
                0x9d01ca54      0x10c
 .text._TcpSwapHeader
                0x9d01ca54      0x10c build/WiFIG/production/_ext/427700826/tcp.o

.text.TCPIP_STACK_BringNetDown
                0x9d01cb60      0x108
 .text.TCPIP_STACK_BringNetDown
                0x9d01cb60      0x108 build/WiFIG/production/_ext/427700826/tcpip_manager.o

.text.OutputNetworkType
                0x9d01cc68      0x108
 .text.OutputNetworkType
                0x9d01cc68      0x108 build/WiFIG/production/_ext/334706090/wf_debug_output.o

.text._DHCPClose
                0x9d01cd70      0x104
 .text._DHCPClose
                0x9d01cd70      0x104 build/WiFIG/production/_ext/427700826/dhcp.o

.text.WF_ScanContextGet
                0x9d01ce74      0x104
 .text.WF_ScanContextGet
                0x9d01ce74      0x104 build/WiFIG/production/_ext/334706090/wf_connection_algorithm.o
                0x9d01ce74                WF_ScanContextGet

.rodata         0x9d01cf78      0x208
 .rodata        0x9d01cf78      0x104 build/WiFIG/production/_ext/1472/wf_config.o
 .rodata        0x9d01d07c      0x104 c:/program files (x86)/microchip/xc32/v1.21/bin/../lib/gcc/pic32mx/4.5.2/../../../../pic32mx/lib/size\libc.a(ctype.o)
                0x9d01d07c                _ctype

.text.hexatob   0x9d01d180      0x100
 .text.hexatob  0x9d01d180      0x100 build/WiFIG/production/_ext/101875047/helpers.o
                0x9d01d180                hexatob

.text.DisplayIPValue
                0x9d01d280      0x100
 .text.DisplayIPValue
                0x9d01d280      0x100 build/WiFIG/production/_ext/1472/main_demo.o
                0x9d01d280                DisplayIPValue

.text.WaitForMgmtResponseAndReadData
                0x9d01d380       0xfc
 .text.WaitForMgmtResponseAndReadData
                0x9d01d380       0xfc build/WiFIG/production/_ext/334706090/wf_mgmt_msg_24g.o
                0x9d01d380                WaitForMgmtResponseAndReadData

.text._TCPIPStackAddressServiceEvent
                0x9d01d47c       0xf8
 .text._TCPIPStackAddressServiceEvent
                0x9d01d47c       0xf8 build/WiFIG/production/_ext/427700826/tcpip_manager.o
                0x9d01d47c                _TCPIPStackAddressServiceEvent

.text.SingleListRemoveNode
                0x9d01d574       0xf8
 .text.SingleListRemoveNode
                0x9d01d574       0xf8 build/WiFIG/production/_ext/427700826/tcpip_helpers.o
                0x9d01d574                SingleListRemoveNode

.text.WF_Init   0x9d01d66c       0xf8
 .text.WF_Init  0x9d01d66c       0xf8 build/WiFIG/production/_ext/334706090/wf_init.o
                0x9d01d66c                WF_Init

.text.SYS_USERIO_DeviceDebounce
                0x9d01d764       0xf4
 .text.SYS_USERIO_DeviceDebounce
                0x9d01d764       0xf4 build/WiFIG/production/_ext/365611741/system_userio.o
                0x9d01d764                SYS_USERIO_DeviceDebounce

.text.UDPSetSourceIPAddress
                0x9d01d858       0xf4
 .text.UDPSetSourceIPAddress
                0x9d01d858       0xf4 build/WiFIG/production/_ext/427700826/udp.o
                0x9d01d858                UDPSetSourceIPAddress

.text.UDPSetDestinationIPAddress
                0x9d01d94c       0xf4
 .text.UDPSetDestinationIPAddress
                0x9d01d94c       0xf4 build/WiFIG/production/_ext/427700826/udp.o
                0x9d01d94c                UDPSetDestinationIPAddress

.text.WF_SecurityGet
                0x9d01da40       0xf4
 .text.WF_SecurityGet
                0x9d01da40       0xf4 build/WiFIG/production/_ext/334706090/wf_connection_profile.o
                0x9d01da40                WF_SecurityGet

.text.MRF24W_MACInitialize
                0x9d01db34       0xf4
 .text.MRF24W_MACInitialize
                0x9d01db34       0xf4 build/WiFIG/production/_ext/334706090/mrf24w_mac_pic32.o
                0x9d01db34                MRF24W_MACInitialize

.text._ARPAddCompleteEntry
                0x9d01dc28       0xf0
 .text._ARPAddCompleteEntry
                0x9d01dc28       0xf0 build/WiFIG/production/_ext/427700826/arp.o

.text.UDPDiscard
                0x9d01dd18       0xf0
 .text.UDPDiscard
                0x9d01dd18       0xf0 build/WiFIG/production/_ext/427700826/udp.o
                0x9d01dd18                UDPDiscard

.text.WF_ScanContextSet
                0x9d01de08       0xf0
 .text.WF_ScanContextSet
                0x9d01de08       0xf0 build/WiFIG/production/_ext/334706090/wf_connection_algorithm.o
                0x9d01de08                WF_ScanContextSet

.text.NBNSPutName
                0x9d01def8       0xec
 .text.NBNSPutName
                0x9d01def8       0xec build/WiFIG/production/_ext/427700826/nbns.o

.text.TCPIsPutReady
                0x9d01dfe4       0xec
 .text.TCPIsPutReady
                0x9d01dfe4       0xec build/WiFIG/production/_ext/427700826/tcp.o
                0x9d01dfe4                TCPIsPutReady

.text._TCPIP_HEAP_CallocDebug
                0x9d01e0d0       0xec
 .text._TCPIP_HEAP_CallocDebug
                0x9d01e0d0       0xec build/WiFIG/production/_ext/427700826/tcpip_heap_alloc.o
                0x9d01e0d0                _TCPIP_HEAP_CallocDebug

.text.AllocateDataTxBuffer
                0x9d01e1bc       0xec
 .text.AllocateDataTxBuffer
                0x9d01e1bc       0xec build/WiFIG/production/_ext/334706090/wf_driver_raw_24g.o
                0x9d01e1bc                AllocateDataTxBuffer

.text.DNSIsResolved
                0x9d01e2a8       0xe8
 .text.DNSIsResolved
                0x9d01e2a8       0xe8 build/WiFIG/production/_ext/427700826/dns.o
                0x9d01e2a8                DNSIsResolved

.text.TCPIP_IPV4_PutUpperLayerHeader
                0x9d01e390       0xe8
 .text.TCPIP_IPV4_PutUpperLayerHeader
                0x9d01e390       0xe8 build/WiFIG/production/_ext/427700826/ipv4.o
                0x9d01e390                TCPIP_IPV4_PutUpperLayerHeader

.text.UDPSetRxOffset
                0x9d01e478       0xe8
 .text.UDPSetRxOffset
                0x9d01e478       0xe8 build/WiFIG/production/_ext/427700826/udp.o
                0x9d01e478                UDPSetRxOffset

.text.ProcessTCPIPTickEvent
                0x9d01e560       0xe8
 .text.ProcessTCPIPTickEvent
                0x9d01e560       0xe8 build/WiFIG/production/_ext/427700826/tcpip_manager.o

.text.WF_GetDeviceInfo
                0x9d01e648       0xe8
 .text.WF_GetDeviceInfo
                0x9d01e648       0xe8 build/WiFIG/production/_ext/334706090/wf_param_msg_24g.o
                0x9d01e648                WF_GetDeviceInfo

.rodata         0x9d01e730       0xe8
 .rodata        0x9d01e730       0xe8 c:/program files (x86)/microchip/xc32/v1.21/bin/../lib/gcc/pic32mx/4.5.2/../../../../pic32mx/lib/size\libc.a(doprnt.o)

.text.TCPIP_IPV4_ResetTransmitPacketState
                0x9d01e818       0xe4
 .text.TCPIP_IPV4_ResetTransmitPacketState
                0x9d01e818       0xe4 build/WiFIG/production/_ext/427700826/ipv4.o
                0x9d01e818                TCPIP_IPV4_ResetTransmitPacketState

.text.TCPIP_IPV4_AllocateDataSegmentHeader
                0x9d01e8fc       0xe4
 .text.TCPIP_IPV4_AllocateDataSegmentHeader
                0x9d01e8fc       0xe4 build/WiFIG/production/_ext/427700826/ipv4.o
                0x9d01e8fc                TCPIP_IPV4_AllocateDataSegmentHeader

.text.TCPDeInit
                0x9d01e9e0       0xe4
 .text.TCPDeInit
                0x9d01e9e0       0xe4 build/WiFIG/production/_ext/427700826/tcp.o
                0x9d01e9e0                TCPDeInit

.text.TCPIP_HEAP_Delete
                0x9d01eac4       0xe4
 .text.TCPIP_HEAP_Delete
                0x9d01eac4       0xe4 build/WiFIG/production/_ext/427700826/tcpip_heap_alloc.o
                0x9d01eac4                TCPIP_HEAP_Delete

.text.SYS_TICK_TimerCreate
                0x9d01eba8       0xe0
 .text.SYS_TICK_TimerCreate
                0x9d01eba8       0xe0 build/WiFIG/production/_ext/365611741/system_services.o
                0x9d01eba8                SYS_TICK_TimerCreate

.text._ARPSetEntry
                0x9d01ec88       0xe0
 .text._ARPSetEntry
                0x9d01ec88       0xe0 build/WiFIG/production/_ext/427700826/arp.o

.text.ARPResolve
                0x9d01ed68       0xe0
 .text.ARPResolve
                0x9d01ed68       0xe0 build/WiFIG/production/_ext/427700826/arp.o
                0x9d01ed68                ARPResolve

.text.UDPPutArray
                0x9d01ee48       0xe0
 .text.UDPPutArray
                0x9d01ee48       0xe0 build/WiFIG/production/_ext/427700826/udp.o
                0x9d01ee48                UDPPutArray

.text.TCPIPMacEventCB
                0x9d01ef28       0xe0
 .text.TCPIPMacEventCB
                0x9d01ef28       0xe0 build/WiFIG/production/_ext/427700826/tcpip_manager.o

.text.ProcessNotification
                0x9d01f008       0xe0
 .text.ProcessNotification
                0x9d01f008       0xe0 build/WiFIG/production/_ext/1472/main_demo.o

.text._SYS_ERROR_PRINT
                0x9d01f0e8       0xdc
 .text._SYS_ERROR_PRINT
                0x9d01f0e8       0xdc build/WiFIG/production/_ext/365611741/system_debug.o
                0x9d01f0e8                _SYS_ERROR_PRINT

.text.ARPHashDeleteEntry
                0x9d01f1c4       0xdc
 .text.ARPHashDeleteEntry
                0x9d01f1c4       0xdc build/WiFIG/production/_ext/427700826/arp.o
                0x9d01f1c4                ARPHashDeleteEntry

.text.DHCPConnectionHandler
                0x9d01f2a0       0xdc
 .text.DHCPConnectionHandler
                0x9d01f2a0       0xdc build/WiFIG/production/_ext/427700826/dhcp.o
                0x9d01f2a0                DHCPConnectionHandler

.text._TcpCleanup
                0x9d01f37c       0xdc
 .text._TcpCleanup
                0x9d01f37c       0xdc build/WiFIG/production/_ext/427700826/tcp.o

.text.TCPOpenClient
                0x9d01f458       0xdc
 .text.TCPOpenClient
                0x9d01f458       0xdc build/WiFIG/production/_ext/427700826/tcp.o
                0x9d01f458                TCPOpenClient

.text.TcpAllocateEphemeralPort
                0x9d01f534       0xdc
 .text.TcpAllocateEphemeralPort
                0x9d01f534       0xdc build/WiFIG/production/_ext/427700826/tcp.o

.text.UDPOpenClient
                0x9d01f610       0xdc
 .text.UDPOpenClient
                0x9d01f610       0xdc build/WiFIG/production/_ext/427700826/udp.o
                0x9d01f610                UDPOpenClient

.text.UdpAllocateEphemeralPort
                0x9d01f6ec       0xdc
 .text.UdpAllocateEphemeralPort
                0x9d01f6ec       0xdc build/WiFIG/production/_ext/427700826/udp.o

.text.OutputTxMode
                0x9d01f7c8       0xdc
 .text.OutputTxMode
                0x9d01f7c8       0xdc build/WiFIG/production/_ext/334706090/wf_debug_output.o

.text.MACIFService
                0x9d01f8a4       0xdc
 .text.MACIFService
                0x9d01f8a4       0xdc build/WiFIG/production/_ext/334706090/wf_mac_24g.o

.text.DHCPEnable
                0x9d01f980       0xd8
 .text.DHCPEnable
                0x9d01f980       0xd8 build/WiFIG/production/_ext/427700826/dhcp.o
                0x9d01f980                DHCPEnable

.text.TCPIP_IPV4_GetPseudoHeaderChecksum
                0x9d01fa58       0xd8
 .text.TCPIP_IPV4_GetPseudoHeaderChecksum
                0x9d01fa58       0xd8 build/WiFIG/production/_ext/427700826/ipv4.o
                0x9d01fa58                TCPIP_IPV4_GetPseudoHeaderChecksum

.text._TCPIP_HEAP_MallocDebug
                0x9d01fb30       0xd8
 .text._TCPIP_HEAP_MallocDebug
                0x9d01fb30       0xd8 build/WiFIG/production/_ext/427700826/tcpip_heap_alloc.o
                0x9d01fb30                _TCPIP_HEAP_MallocDebug

.text._SYS_RANDOM_INIT
                0x9d01fc08       0xd4
 .text._SYS_RANDOM_INIT
                0x9d01fc08       0xd4 build/WiFIG/production/_ext/365611741/system_random.o
                0x9d01fc08                _SYS_RANDOM_INIT

.text.TCPIP_ANNOUNCE_Init
                0x9d01fcdc       0xd4
 .text.TCPIP_ANNOUNCE_Init
                0x9d01fcdc       0xd4 build/WiFIG/production/_ext/427700826/tcpip_announce.o
                0x9d01fcdc                TCPIP_ANNOUNCE_Init

.text._TcpAbort
                0x9d01fdb0       0xd4
 .text._TcpAbort
                0x9d01fdb0       0xd4 build/WiFIG/production/_ext/427700826/tcp.o

.text.TCPClose  0x9d01fe84       0xd4
 .text.TCPClose
                0x9d01fe84       0xd4 build/WiFIG/production/_ext/427700826/tcp.o
                0x9d01fe84                TCPClose

.text.OutputDomain
                0x9d01ff58       0xd4
 .text.OutputDomain
                0x9d01ff58       0xd4 build/WiFIG/production/_ext/334706090/wf_debug_output.o

.text.AllocateMgmtTxBuffer
                0x9d02002c       0xd4
 .text.AllocateMgmtTxBuffer
                0x9d02002c       0xd4 build/WiFIG/production/_ext/334706090/wf_driver_raw_24g.o
                0x9d02002c                AllocateMgmtTxBuffer

.text           0x9d020100       0xd4
 .text          0x9d020100       0xd4 c:/program files (x86)/microchip/xc32/v1.21/bin/../lib/gcc/pic32mx/4.5.2/size\libgcc.a(_floatundisf.o)
                0x9d020100                __floatundisf

.text.SYS_USERIO_SetLED
                0x9d0201d4       0xd0
 .text.SYS_USERIO_SetLED
                0x9d0201d4       0xd0 build/WiFIG/production/_ext/365611741/system_userio.o
                0x9d0201d4                SYS_USERIO_SetLED

.text._ARPDeleteResources
                0x9d0202a4       0xd0
 .text._ARPDeleteResources
                0x9d0202a4       0xd0 build/WiFIG/production/_ext/427700826/arp.o

.text.fnv_32_hash
                0x9d020374       0xd0
 .text.fnv_32_hash
                0x9d020374       0xd0 build/WiFIG/production/_ext/427700826/hash_fnv.o
                0x9d020374                fnv_32_hash

.text._TcpSocketInitialize
                0x9d020444       0xd0
 .text._TcpSocketInitialize
                0x9d020444       0xd0 build/WiFIG/production/_ext/427700826/tcp.o

.text.UDPSetOptions
                0x9d020514       0xd0
 .text.UDPSetOptions
                0x9d020514       0xd0 build/WiFIG/production/_ext/427700826/udp.o
                0x9d020514                UDPSetOptions

.text.TCPIP_STACK_RegisterHandler
                0x9d0205e4       0xd0
 .text.TCPIP_STACK_RegisterHandler
                0x9d0205e4       0xd0 build/WiFIG/production/_ext/427700826/tcpip_manager.o
                0x9d0205e4                TCPIP_STACK_RegisterHandler

.text.DhcpConfigTask
                0x9d0206b4       0xd0
 .text.DhcpConfigTask
                0x9d0206b4       0xd0 build/WiFIG/production/_ext/334706090/wf_connection_profile.o
                0x9d0206b4                DhcpConfigTask

.text.OutputDeviceInfo
                0x9d020784       0xd0
 .text.OutputDeviceInfo
                0x9d020784       0xd0 build/WiFIG/production/_ext/334706090/wf_debug_output.o

.text.MRF24W_MACPutHeader
                0x9d020854       0xd0
 .text.MRF24W_MACPutHeader
                0x9d020854       0xd0 build/WiFIG/production/_ext/334706090/wf_mac_24g.o
                0x9d020854                MRF24W_MACPutHeader

.text.general_exception
                0x9d020924       0xd0
 .text.general_exception
                0x9d020924       0xd0 c:/program files (x86)/microchip/xc32/v1.21/bin/../lib/gcc/pic32mx/4.5.2/../../../../pic32mx/lib/size\libpic32.a(general-exception.o)
                0x9d020924                _general_exception_context

.rodata         0x9d0209f8       0xd0
 .rodata        0x9d0209f8       0xd0 c:/program files (x86)/microchip/xc32/v1.21/bin/../lib/gcc/pic32mx/4.5.2/../../../../pic32mx/lib/size\libc.a(doprnt_cdnopsuxX.eo)

.text.TCPIP_IPV4_SetPayload
                0x9d020ac8       0xcc
 .text.TCPIP_IPV4_SetPayload
                0x9d020ac8       0xcc build/WiFIG/production/_ext/427700826/ipv4.o
                0x9d020ac8                TCPIP_IPV4_SetPayload

.text.BSP_Initialize
                0x9d020b94       0xc8
 .text.BSP_Initialize
                0x9d020b94       0xc8 build/WiFIG/production/_ext/1293749816/bsp.o
                0x9d020b94                BSP_Initialize

.text.DNSRetry  0x9d020c5c       0xc8
 .text.DNSRetry
                0x9d020c5c       0xc8 build/WiFIG/production/_ext/427700826/dns.o

.text.DNSDiscardName
                0x9d020d24       0xc8
 .text.DNSDiscardName
                0x9d020d24       0xc8 build/WiFIG/production/_ext/427700826/dns.o

.text.UDPClose  0x9d020dec       0xc8
 .text.UDPClose
                0x9d020dec       0xc8 build/WiFIG/production/_ext/427700826/udp.o
                0x9d020dec                UDPClose

.text.UDPSetTxOffset
                0x9d020eb4       0xc8
 .text.UDPSetTxOffset
                0x9d020eb4       0xc8 build/WiFIG/production/_ext/427700826/udp.o
                0x9d020eb4                UDPSetTxOffset

.text.InitNetConfig
                0x9d020f7c       0xc8
 .text.InitNetConfig
                0x9d020f7c       0xc8 build/WiFIG/production/_ext/427700826/tcpip_manager.o

.text.TCPIP_Helper_FormatNetBIOSName
                0x9d021044       0xc8
 .text.TCPIP_Helper_FormatNetBIOSName
                0x9d021044       0xc8 build/WiFIG/production/_ext/427700826/tcpip_helpers.o
                0x9d021044                TCPIP_Helper_FormatNetBIOSName

.text.OutputDemoHeader
                0x9d02110c       0xc8
 .text.OutputDemoHeader
                0x9d02110c       0xc8 build/WiFIG/production/_ext/334706090/wf_debug_output.o
                0x9d02110c                OutputDemoHeader

.text.HostInterruptRegInit
                0x9d0211d4       0xc8
 .text.HostInterruptRegInit
                0x9d0211d4       0xc8 build/WiFIG/production/_ext/334706090/wf_driver_com_24g.o

.text._DHCPEnable
                0x9d02129c       0xc4
 .text._DHCPEnable
                0x9d02129c       0xc4 build/WiFIG/production/_ext/427700826/dhcp.o

.text.MRF24W_MACGetArray
                0x9d021360       0xc4
 .text.MRF24W_MACGetArray
                0x9d021360       0xc4 build/WiFIG/production/_ext/334706090/wf_mac_24g.o
                0x9d021360                MRF24W_MACGetArray

.text.SYS_TICK_Initialize
                0x9d021424       0xc0
 .text.SYS_TICK_Initialize
                0x9d021424       0xc0 build/WiFIG/production/_ext/365611741/system_services.o
                0x9d021424                SYS_TICK_Initialize

.text.LowLevel_CPGetElement
                0x9d0214e4       0xc0
 .text.LowLevel_CPGetElement
                0x9d0214e4       0xc0 build/WiFIG/production/_ext/334706090/wf_connection_profile.o

.text.ProcessMgmtRxMsg
                0x9d0215a4       0xc0
 .text.ProcessMgmtRxMsg
                0x9d0215a4       0xc0 build/WiFIG/production/_ext/334706090/wf_driver_com_24g.o

.rodata         0x9d021664       0xbc
 .rodata        0x9d021664       0xbc build/WiFIG/production/_ext/365611741/system_services.o
                0x9d021674                MEDIA_STORAGE_WIFI_STORAGE_PARTITION
                0x9d021690                MEDIA_STORAGE_TCPIP_STORAGE_PARTITION
                0x9d0216a4                MEDIA_STORAGE_MPFS_IMAGE_PARTITION
                0x9d0216b8                MEDIA_STORAGE_CONFIGURATION

.text.SYS_INT_DynamicRegister
                0x9d021720       0xbc
 .text.SYS_INT_DynamicRegister
                0x9d021720       0xbc build/WiFIG/production/_ext/365611741/system_services.o
                0x9d021720                SYS_INT_DynamicRegister

.text._ARPRemoveEntry
                0x9d0217dc       0xbc
 .text._ARPRemoveEntry
                0x9d0217dc       0xbc build/WiFIG/production/_ext/427700826/arp.o

.text.OAHashRemoveAll
                0x9d021898       0xbc
 .text.OAHashRemoveAll
                0x9d021898       0xbc build/WiFIG/production/_ext/427700826/hash_tbl.o
                0x9d021898                OAHashRemoveAll

.text.UDPDiscardNet
                0x9d021954       0xbc
 .text.UDPDiscardNet
                0x9d021954       0xbc build/WiFIG/production/_ext/427700826/udp.o
                0x9d021954                UDPDiscardNet

.text.TCPIP_Helper_StringToPowerMode
                0x9d021a10       0xbc
 .text.TCPIP_Helper_StringToPowerMode
                0x9d021a10       0xbc build/WiFIG/production/_ext/427700826/tcpip_helpers.o
                0x9d021a10                TCPIP_Helper_StringToPowerMode

.text.LowLevel_CAGetElement
                0x9d021acc       0xbc
 .text.LowLevel_CAGetElement
                0x9d021acc       0xbc build/WiFIG/production/_ext/334706090/wf_connection_algorithm.o

.text.MRF24W_MACEventSetNotifyHandler
                0x9d021b88       0xbc
 .text.MRF24W_MACEventSetNotifyHandler
                0x9d021b88       0xbc build/WiFIG/production/_ext/334706090/mrf24w_events.o
                0x9d021b88                MRF24W_MACEventSetNotifyHandler

.text.OutputMacAddress
                0x9d021c44       0xbc
 .text.OutputMacAddress
                0x9d021c44       0xbc build/WiFIG/production/_ext/334706090/wf_debug_output.o

.text._SYS_DEBUG_INIT
                0x9d021d00       0xb8
 .text._SYS_DEBUG_INIT
                0x9d021d00       0xb8 build/WiFIG/production/_ext/365611741/system_debug.o
                0x9d021d00                _SYS_DEBUG_INIT

.text._SYS_CONSOLE_INIT
                0x9d021db8       0xb8
 .text._SYS_CONSOLE_INIT
                0x9d021db8       0xb8 build/WiFIG/production/_ext/365611741/system_debug.o
                0x9d021db8                _SYS_CONSOLE_INIT

.text.TCPv4AllocateTxPacketStruct
                0x9d021e70       0xb8
 .text.TCPv4AllocateTxPacketStruct
                0x9d021e70       0xb8 build/WiFIG/production/_ext/427700826/tcp.o

.text._TCPIsGetReady
                0x9d021f28       0xb8
 .text._TCPIsGetReady
                0x9d021f28       0xb8 build/WiFIG/production/_ext/427700826/tcp.o

.text.UDPGetTxCount
                0x9d021fe0       0xb8
 .text.UDPGetTxCount
                0x9d021fe0       0xb8 build/WiFIG/production/_ext/427700826/udp.o
                0x9d021fe0                UDPGetTxCount

.text.OutputScanType
                0x9d022098       0xb8
 .text.OutputScanType
                0x9d022098       0xb8 build/WiFIG/production/_ext/334706090/wf_debug_output.o

.text.RawGetByte
                0x9d022150       0xb8
 .text.RawGetByte
                0x9d022150       0xb8 build/WiFIG/production/_ext/334706090/wf_driver_raw_24g.o
                0x9d022150                RawGetByte

.text.RawSetByte
                0x9d022208       0xb8
 .text.RawSetByte
                0x9d022208       0xb8 build/WiFIG/production/_ext/334706090/wf_driver_raw_24g.o
                0x9d022208                RawSetByte

.text._TcpMac2RamCopy
                0x9d0222c0       0xb4
 .text._TcpMac2RamCopy
                0x9d0222c0       0xb4 build/WiFIG/production/_ext/427700826/tcp.o

.text.UDPv4AllocateTxPacketStruct
                0x9d022374       0xb4
 .text.UDPv4AllocateTxPacketStruct
                0x9d022374       0xb4 build/WiFIG/production/_ext/427700826/udp.o

.text.UDPIsTxPutReady
                0x9d022428       0xb4
 .text.UDPIsTxPutReady
                0x9d022428       0xb4 build/WiFIG/production/_ext/427700826/udp.o
                0x9d022428                UDPIsTxPutReady

.text.WF_SsidSet
                0x9d0224dc       0xb4
 .text.WF_SsidSet
                0x9d0224dc       0xb4 build/WiFIG/production/_ext/334706090/wf_connection_profile.o
                0x9d0224dc                WF_SsidSet

.text.MRF24W_MACEventInit
                0x9d022590       0xb4
 .text.MRF24W_MACEventInit
                0x9d022590       0xb4 build/WiFIG/production/_ext/334706090/mrf24w_events.o
                0x9d022590                MRF24W_MACEventInit

.text._mon_putc
                0x9d022644       0xb4
 .text._mon_putc
                0x9d022644       0xb4 c:/program files (x86)/microchip/xc32/v1.21/bin/../lib/gcc/pic32mx/4.5.2/../../../../pic32mx/lib/size\libpic32.a(_mon_putc.o)
                0x9d022644                _mon_putc

.text.TCPIP_ANNOUNCE_DeInit
                0x9d0226f8       0xb0
 .text.TCPIP_ANNOUNCE_DeInit
                0x9d0226f8       0xb0 build/WiFIG/production/_ext/427700826/tcpip_announce.o
                0x9d0226f8                TCPIP_ANNOUNCE_DeInit

.text._ARPRemoveCacheEntries
                0x9d0227a8       0xb0
 .text._ARPRemoveCacheEntries
                0x9d0227a8       0xb0 build/WiFIG/production/_ext/427700826/arp.o

.text._ARPNotifyClients
                0x9d022858       0xb0
 .text._ARPNotifyClients
                0x9d022858       0xb0 build/WiFIG/production/_ext/427700826/arp.o

.text._Tcpv4AckFnc
                0x9d022908       0xb0
 .text._Tcpv4AckFnc
                0x9d022908       0xb0 build/WiFIG/production/_ext/427700826/tcp.o

.text._TCPIPStackSetNetAddress
                0x9d0229b8       0xb0
 .text._TCPIPStackSetNetAddress
                0x9d0229b8       0xb0 build/WiFIG/production/_ext/427700826/tcpip_manager.o
                0x9d0229b8                _TCPIPStackSetNetAddress

.text._TCPIPStackIsBcastAddress
                0x9d022a68       0xb0
 .text._TCPIPStackIsBcastAddress
                0x9d022a68       0xb0 build/WiFIG/production/_ext/427700826/tcpip_manager.o
                0x9d022a68                _TCPIPStackIsBcastAddress

.text.HostInterrupt2RegInit
                0x9d022b18       0xb0
 .text.HostInterrupt2RegInit
                0x9d022b18       0xb0 build/WiFIG/production/_ext/334706090/wf_driver_com_24g.o

.rodata         0x9d022bc8       0xac
 .rodata        0x9d022bc8       0xac build/WiFIG/production/_ext/427700826/tcp.o

.text.TCPIsConnected
                0x9d022c74       0xac
 .text.TCPIsConnected
                0x9d022c74       0xac build/WiFIG/production/_ext/427700826/tcp.o
                0x9d022c74                TCPIsConnected

.text._SYS_ERROR
                0x9d022d20       0xa8
 .text._SYS_ERROR
                0x9d022d20       0xa8 build/WiFIG/production/_ext/365611741/system_debug.o
                0x9d022d20                _SYS_ERROR

.text.ARPDeinitialize
                0x9d022dc8       0xa8
 .text.ARPDeinitialize
                0x9d022dc8       0xa8 build/WiFIG/production/_ext/427700826/arp.o
                0x9d022dc8                ARPDeinitialize

.text._TCPIPStackStringToMACId
                0x9d022e70       0xa8
 .text._TCPIPStackStringToMACId
                0x9d022e70       0xa8 build/WiFIG/production/_ext/427700826/tcpip_manager.o
                0x9d022e70                _TCPIPStackStringToMACId

.text.WFConfigureLowPowerMode
                0x9d022f18       0xa8
 .text.WFConfigureLowPowerMode
                0x9d022f18       0xa8 build/WiFIG/production/_ext/334706090/wf_power_save.o
                0x9d022f18                WFConfigureLowPowerMode

.text.WF_OutputConnectionDebugMsg
                0x9d022fc0       0xa8
 .text.WF_OutputConnectionDebugMsg
                0x9d022fc0       0xa8 build/WiFIG/production/_ext/334706090/wf_debug_output.o
                0x9d022fc0                WF_OutputConnectionDebugMsg

.text           0x9d023068       0xa8
 .text          0x9d023068       0xa8 c:/program files (x86)/microchip/xc32/v1.21/bin/../lib/gcc/pic32mx/4.5.2/../../../../pic32mx/lib/size\libpic32.a(memset.o)
                0x9d023068                memset

.text.SYS_USERIO_ReadIO
                0x9d023110       0xa4
 .text.SYS_USERIO_ReadIO
                0x9d023110       0xa4 build/WiFIG/production/_ext/365611741/system_userio.o

.text.DNSResolve
                0x9d0231b4       0xa4
 .text.DNSResolve
                0x9d0231b4       0xa4 build/WiFIG/production/_ext/427700826/dns.o
                0x9d0231b4                DNSResolve

.text._ICMPAllocateTxPacketStruct
                0x9d023258       0xa4
 .text._ICMPAllocateTxPacketStruct
                0x9d023258       0xa4 build/WiFIG/production/_ext/427700826/icmp.o

.text.TCPIP_IPV4_DeInitialize
                0x9d0232fc       0xa4
 .text.TCPIP_IPV4_DeInitialize
                0x9d0232fc       0xa4 build/WiFIG/production/_ext/427700826/ipv4.o
                0x9d0232fc                TCPIP_IPV4_DeInitialize

.text._TCPIPStackNetByAddress
                0x9d0233a0       0xa4
 .text._TCPIPStackNetByAddress
                0x9d0233a0       0xa4 build/WiFIG/production/_ext/427700826/tcpip_manager.o
                0x9d0233a0                _TCPIPStackNetByAddress

.text.WF_ReconnectModeSet
                0x9d023444       0xa4
 .text.WF_ReconnectModeSet
                0x9d023444       0xa4 build/WiFIG/production/_ext/334706090/wf_connection_algorithm.o
                0x9d023444                WF_ReconnectModeSet

.text.WF_LibInitialize
                0x9d0234e8       0xa4
 .text.WF_LibInitialize
                0x9d0234e8       0xa4 build/WiFIG/production/_ext/334706090/wf_init.o
                0x9d0234e8                WF_LibInitialize

.text._sbrk     0x9d02358c       0xa4
 .text._sbrk    0x9d02358c       0xa4 c:/program files (x86)/microchip/xc32/v1.21/bin/../lib/gcc/pic32mx/4.5.2/../../../../pic32mx/lib/size\libpic32.a(sbrk.o)
                0x9d02358c                _sbrk

.text.USART_GETS
                0x9d023630       0xa0
 .text.USART_GETS
                0x9d023630       0xa0 build/WiFIG/production/_ext/792872985/usart.o
                0x9d023630                USART_GETS

.text._DHCPDiscard
                0x9d0236d0       0xa0
 .text._DHCPDiscard
                0x9d0236d0       0xa0 build/WiFIG/production/_ext/427700826/dhcp.o

.text._DHCPNotifyClients
                0x9d023770       0xa0
 .text._DHCPNotifyClients
                0x9d023770       0xa0 build/WiFIG/production/_ext/427700826/dhcp.o

.text._UdpSocketDcpt
                0x9d023810       0xa0
 .text._UdpSocketDcpt
                0x9d023810       0xa0 build/WiFIG/production/_ext/427700826/udp.o

.rodata         0x9d0238b0       0xa0
 .rodata        0x9d0238b0       0xa0 c:/program files (x86)/microchip/xc32/v1.21/bin/../lib/gcc/pic32mx/4.5.2/../../../../pic32mx/lib/size\libmchp_peripheral_32MX695F512H.a(spi_io_tbl_libp.o)
                0x9d0238b0                _SpiIoTbl

.text.strupr    0x9d023950       0x9c
 .text.strupr   0x9d023950       0x9c build/WiFIG/production/_ext/101875047/helpers.o
                0x9d023950                strupr

.text.ANNOUNCE_Notify
                0x9d0239ec       0x9c
 .text.ANNOUNCE_Notify
                0x9d0239ec       0x9c build/WiFIG/production/_ext/427700826/tcpip_announce.o

.text.DHCPRegisterHandler
                0x9d023a88       0x9c
 .text.DHCPRegisterHandler
                0x9d023a88       0x9c build/WiFIG/production/_ext/427700826/dhcp.o
                0x9d023a88                DHCPRegisterHandler

.text._TcpSocketKill
                0x9d023b24       0x9c
 .text._TcpSocketKill
                0x9d023b24       0x9c build/WiFIG/production/_ext/427700826/tcp.o

.text.TCPIsAvailablePort
                0x9d023bc0       0x9c
 .text.TCPIsAvailablePort
                0x9d023bc0       0x9c build/WiFIG/production/_ext/427700826/tcp.o

.text.UdpIsAvailablePort
                0x9d023c5c       0x9c
 .text.UdpIsAvailablePort
                0x9d023c5c       0x9c build/WiFIG/production/_ext/427700826/udp.o

.text._TCPIPStackMacIdToNet
                0x9d023cf8       0x9c
 .text._TCPIPStackMacIdToNet
                0x9d023cf8       0x9c build/WiFIG/production/_ext/427700826/tcpip_manager.o
                0x9d023cf8                _TCPIPStackMacIdToNet

.text.SingleListRemoveHead
                0x9d023d94       0x9c
 .text.SingleListRemoveHead
                0x9d023d94       0x9c build/WiFIG/production/_ext/427700826/tcpip_helpers.o
                0x9d023d94                SingleListRemoveHead

.text.SetWpsSecurity
                0x9d023e30       0x9c
 .text.SetWpsSecurity
                0x9d023e30       0x9c build/WiFIG/production/_ext/334706090/wf_connect.o

.text.WF_SpiTxRx
                0x9d023ecc       0x9c
 .text.WF_SpiTxRx
                0x9d023ecc       0x9c build/WiFIG/production/_ext/334706090/wf_spi.o
                0x9d023ecc                WF_SpiTxRx

.text.OutputIpAddress
                0x9d023f68       0x9c
 .text.OutputIpAddress
                0x9d023f68       0x9c build/WiFIG/production/_ext/334706090/wf_debug_output.o

.text.GetSpiPortWithBitBang
                0x9d024004       0x9c
 .text.GetSpiPortWithBitBang
                0x9d024004       0x9c build/WiFIG/production/_ext/334706090/wf_driver_com_24g.o

.text._SYS_DEBUG_OPEN
                0x9d0240a0       0x98
 .text._SYS_DEBUG_OPEN
                0x9d0240a0       0x98 build/WiFIG/production/_ext/365611741/system_debug.o
                0x9d0240a0                _SYS_DEBUG_OPEN

.text._SYS_ASSERT
                0x9d024138       0x98
 .text._SYS_ASSERT
                0x9d024138       0x98 build/WiFIG/production/_ext/365611741/system_debug.o
                0x9d024138                _SYS_ASSERT

.text._SYS_CONSOLE_OPEN
                0x9d0241d0       0x98
 .text._SYS_CONSOLE_OPEN
                0x9d0241d0       0x98 build/WiFIG/production/_ext/365611741/system_debug.o
                0x9d0241d0                _SYS_CONSOLE_OPEN

.text.TCPIP_STACK_VerifyPktIf
                0x9d024268       0x98
 .text.TCPIP_STACK_VerifyPktIf
                0x9d024268       0x98 build/WiFIG/production/_ext/427700826/tcpip_manager.o

.text.WF_ReconnectModeGet
                0x9d024300       0x98
 .text.WF_ReconnectModeGet
                0x9d024300       0x98 build/WiFIG/production/_ext/334706090/wf_connection_algorithm.o
                0x9d024300                WF_ReconnectModeGet

.text.WF_ChannelListGet
                0x9d024398       0x98
 .text.WF_ChannelListGet
                0x9d024398       0x98 build/WiFIG/production/_ext/334706090/wf_connection_algorithm.o
                0x9d024398                WF_ChannelListGet

.text           0x9d024430       0x98
 .text          0x9d024430       0x98 c:/program files (x86)/microchip/xc32/v1.21/bin/../lib/gcc/pic32mx/4.5.2/../../../../pic32mx/lib/size\libpic32.a(memcmp.o)
                0x9d024430                memcmp

.text.TCP_PutArray
                0x9d0244c8       0x94
 .text.TCP_PutArray
                0x9d0244c8       0x94 build/WiFIG/production/_ext/427700826/tcp.o

.text.SingleListAddTail
                0x9d02455c       0x94
 .text.SingleListAddTail
                0x9d02455c       0x94 build/WiFIG/production/_ext/427700826/tcpip_helpers.o
                0x9d02455c                SingleListAddTail

.text.LowLevel_CPSetElement
                0x9d0245f0       0x94
 .text.LowLevel_CPSetElement
                0x9d0245f0       0x94 build/WiFIG/production/_ext/334706090/wf_connection_profile.o

.text.MRF24W_SetUserEvents
                0x9d024684       0x94
 .text.MRF24W_SetUserEvents
                0x9d024684       0x94 build/WiFIG/production/_ext/334706090/mrf24w_events.o
                0x9d024684                MRF24W_SetUserEvents

.text.RawMountRxBuffer
                0x9d024718       0x94
 .text.RawMountRxBuffer
                0x9d024718       0x94 build/WiFIG/production/_ext/334706090/wf_driver_raw_24g.o
                0x9d024718                RawMountRxBuffer

.text.MRF24W_MACCalcRxChecksum
                0x9d0247ac       0x94
 .text.MRF24W_MACCalcRxChecksum
                0x9d0247ac       0x94 build/WiFIG/production/_ext/334706090/wf_mac_24g.o
                0x9d0247ac                MRF24W_MACCalcRxChecksum

.text.USART_PRINT
                0x9d024840       0x90
 .text.USART_PRINT
                0x9d024840       0x90 build/WiFIG/production/_ext/792872985/usart.o
                0x9d024840                USART_PRINT

.text.DHCPIsBound
                0x9d0248d0       0x90
 .text.DHCPIsBound
                0x9d0248d0       0x90 build/WiFIG/production/_ext/427700826/dhcp.o
                0x9d0248d0                DHCPIsBound

.text.TCPIP_IPV4_FreePacketData
                0x9d024960       0x90
 .text.TCPIP_IPV4_FreePacketData
                0x9d024960       0x90 build/WiFIG/production/_ext/427700826/ipv4.o
                0x9d024960                TCPIP_IPV4_FreePacketData

.text.NBNSDeInit
                0x9d0249f0       0x90
 .text.NBNSDeInit
                0x9d0249f0       0x90 build/WiFIG/production/_ext/427700826/nbns.o
                0x9d0249f0                NBNSDeInit

.text.TCP_SetPayload
                0x9d024a80       0x90
 .text.TCP_SetPayload
                0x9d024a80       0x90 build/WiFIG/production/_ext/427700826/tcp.o

.text._TCPIPStackIsNetBcastAddress
                0x9d024b10       0x90
 .text._TCPIPStackIsNetBcastAddress
                0x9d024b10       0x90 build/WiFIG/production/_ext/427700826/tcpip_manager.o
                0x9d024b10                _TCPIPStackIsNetBcastAddress

.text.OutputSsid
                0x9d024ba0       0x90
 .text.OutputSsid
                0x9d024ba0       0x90 build/WiFIG/production/_ext/334706090/wf_debug_output.o

.text.ReadWFArray
                0x9d024c30       0x90
 .text.ReadWFArray
                0x9d024c30       0x90 build/WiFIG/production/_ext/334706090/wf_driver_com_24g.o
                0x9d024c30                ReadWFArray

.text.SendGetParamMsg
                0x9d024cc0       0x90
 .text.SendGetParamMsg
                0x9d024cc0       0x90 build/WiFIG/production/_ext/334706090/wf_param_msg_24g.o
                0x9d024cc0                SendGetParamMsg

.text.SwapARPPacket
                0x9d024d50       0x8c
 .text.SwapARPPacket
                0x9d024d50       0x8c build/WiFIG/production/_ext/427700826/arp.o

.text.DHCPDisable
                0x9d024ddc       0x8c
 .text.DHCPDisable
                0x9d024ddc       0x8c build/WiFIG/production/_ext/427700826/dhcp.o
                0x9d024ddc                DHCPDisable

.text.DNSClientInit
                0x9d024e68       0x8c
 .text.DNSClientInit
                0x9d024e68       0x8c build/WiFIG/production/_ext/427700826/dns.o
                0x9d024e68                DNSClientInit

.text.SwapIPV4Header
                0x9d024ef4       0x8c
 .text.SwapIPV4Header
                0x9d024ef4       0x8c build/WiFIG/production/_ext/427700826/ipv4.o

.text.UDPFlush  0x9d024f80       0x8c
 .text.UDPFlush
                0x9d024f80       0x8c build/WiFIG/production/_ext/427700826/udp.o
                0x9d024f80                UDPFlush

.text.UDPRemoteBind
                0x9d02500c       0x8c
 .text.UDPRemoteBind
                0x9d02500c       0x8c build/WiFIG/production/_ext/427700826/udp.o
                0x9d02500c                UDPRemoteBind

.text.LowLevel_CASetElement
                0x9d025098       0x8c
 .text.LowLevel_CASetElement
                0x9d025098       0x8c build/WiFIG/production/_ext/334706090/wf_connection_algorithm.o

.text.write     0x9d025124       0x8c
 .text.write    0x9d025124       0x8c c:/program files (x86)/microchip/xc32/v1.21/bin/../lib/gcc/pic32mx/4.5.2/../../../../pic32mx/lib/size\libpic32.a(write.o)
                0x9d025124                write

.text.SHA1Initialize
                0x9d0251b0       0x88
 .text.SHA1Initialize
                0x9d0251b0       0x88 build/WiFIG/production/_ext/101875047/hashes.o
                0x9d0251b0                SHA1Initialize

.text._SysGetCDevEntry
                0x9d025238       0x88
 .text._SysGetCDevEntry
                0x9d025238       0x88 build/WiFIG/production/_ext/365611741/system_debug.o

.text.DHCPDeInit
                0x9d0252c0       0x88
 .text.DHCPDeInit
                0x9d0252c0       0x88 build/WiFIG/production/_ext/427700826/dhcp.o
                0x9d0252c0                DHCPDeInit

.text.TCP_IsTxPutReady
                0x9d025348       0x88
 .text.TCP_IsTxPutReady
                0x9d025348       0x88 build/WiFIG/production/_ext/427700826/tcp.o

.text.TCP_PutHeader
                0x9d0253d0       0x88
 .text.TCP_PutHeader
                0x9d0253d0       0x88 build/WiFIG/production/_ext/427700826/tcp.o

.text._TCPIPStackIpAddToNet
                0x9d025458       0x88
 .text._TCPIPStackIpAddToNet
                0x9d025458       0x88 build/WiFIG/production/_ext/427700826/tcpip_manager.o
                0x9d025458                _TCPIPStackIpAddToNet

.text._TCPIPStackMACIdToString
                0x9d0254e0       0x88
 .text._TCPIPStackMACIdToString
                0x9d0254e0       0x88 build/WiFIG/production/_ext/427700826/tcpip_manager.o
                0x9d0254e0                _TCPIPStackMACIdToString

.text.TCPIP_STACK_NetBcastAddress
                0x9d025568       0x88
 .text.TCPIP_STACK_NetBcastAddress
                0x9d025568       0x88 build/WiFIG/production/_ext/427700826/tcpip_manager.o
                0x9d025568                TCPIP_STACK_NetBcastAddress

.text.Read16BitWFRegister
                0x9d0255f0       0x88
 .text.Read16BitWFRegister
                0x9d0255f0       0x88 build/WiFIG/production/_ext/334706090/wf_driver_com_24g.o
                0x9d0255f0                Read16BitWFRegister

.text.Write16BitWFRegister
                0x9d025678       0x88
 .text.Write16BitWFRegister
                0x9d025678       0x88 build/WiFIG/production/_ext/334706090/wf_driver_com_24g.o
                0x9d025678                Write16BitWFRegister

.text.WriteWFArray
                0x9d025700       0x88
 .text.WriteWFArray
                0x9d025700       0x88 build/WiFIG/production/_ext/334706090/wf_driver_com_24g.o
                0x9d025700                WriteWFArray

.text.SendSetParamMsg
                0x9d025788       0x88
 .text.SendSetParamMsg
                0x9d025788       0x88 build/WiFIG/production/_ext/334706090/wf_param_msg_24g.o
                0x9d025788                SendSetParamMsg

.text.LFSRSeedRand
                0x9d025810       0x84
 .text.LFSRSeedRand
                0x9d025810       0x84 build/WiFIG/production/_ext/101875047/lfsr.o
                0x9d025810                LFSRSeedRand

.text._SYS_CONSOLE_PRINT
                0x9d025894       0x84
 .text._SYS_CONSOLE_PRINT
                0x9d025894       0x84 build/WiFIG/production/_ext/365611741/system_debug.o
                0x9d025894                _SYS_CONSOLE_PRINT

.text.OAHashInit
                0x9d025918       0x84
 .text.OAHashInit
                0x9d025918       0x84 build/WiFIG/production/_ext/427700826/hash_tbl.o
                0x9d025918                OAHashInit

.text._TCPIP_HEAP_Calloc
                0x9d02599c       0x84
 .text._TCPIP_HEAP_Calloc
                0x9d02599c       0x84 build/WiFIG/production/_ext/427700826/tcpip_heap_alloc.o
                0x9d02599c                _TCPIP_HEAP_Calloc

.text.TcpipStackFindModuleData
                0x9d025a20       0x84
 .text.TcpipStackFindModuleData
                0x9d025a20       0x84 build/WiFIG/production/_ext/427700826/tcpip_manager.o

.text.TcpipStackFindMacModule
                0x9d025aa4       0x84
 .text.TcpipStackFindMacModule
                0x9d025aa4       0x84 build/WiFIG/production/_ext/427700826/tcpip_manager.o

.text.mrf24w_MACPowerMode
                0x9d025b28       0x84
 .text.mrf24w_MACPowerMode
                0x9d025b28       0x84 build/WiFIG/production/_ext/334706090/mrf24w_mac_pic32.o

.text.MRF24W_ISR
                0x9d025bac       0x84
 .text.MRF24W_ISR
                0x9d025bac       0x84 build/WiFIG/production/_ext/334706090/mrf24w_events.o
                0x9d025bac                MRF24W_ISR

.rodata         0x9d025c30       0x84
 .rodata        0x9d025c30       0x84 build/WiFIG/production/_ext/334706090/wf_driver_raw_24g.o
                0x9d025c70                g_RawAccessOutOfBoundsMask

.text.atoi      0x9d025cb4       0x84
 .text.atoi     0x9d025cb4       0x84 c:/program files (x86)/microchip/xc32/v1.21/bin/../lib/gcc/pic32mx/4.5.2/../../../../pic32mx/lib/size\libc.a(atoi.o)
                0x9d025cb4                atoi

.text.TCPIP_IPV4_FlushDataSegments
                0x9d025d38       0x80
 .text.TCPIP_IPV4_FlushDataSegments
                0x9d025d38       0x80 build/WiFIG/production/_ext/427700826/ipv4.o
                0x9d025d38                TCPIP_IPV4_FlushDataSegments

.text.TCP_IsTxReady
                0x9d025db8       0x80
 .text.TCP_IsTxReady
                0x9d025db8       0x80 build/WiFIG/production/_ext/427700826/tcp.o

.text.TCP_CopyTxPacketStruct
                0x9d025e38       0x80
 .text.TCP_CopyTxPacketStruct
                0x9d025e38       0x80 build/WiFIG/production/_ext/427700826/tcp.o

.text._Udpv4AckFnc
                0x9d025eb8       0x80
 .text._Udpv4AckFnc
                0x9d025eb8       0x80 build/WiFIG/production/_ext/427700826/udp.o

.text.SetWpaSecurity
                0x9d025f38       0x80
 .text.SetWpaSecurity
                0x9d025f38       0x80 build/WiFIG/production/_ext/334706090/wf_connect.o

.text.ValidateConfig
                0x9d025fb8       0x80
 .text.ValidateConfig
                0x9d025fb8       0x80 build/WiFIG/production/_ext/334706090/wf_debug_output.o
                0x9d025fb8                ValidateConfig

.text.ScratchMount
                0x9d026038       0x80
 .text.ScratchMount
                0x9d026038       0x80 build/WiFIG/production/_ext/334706090/wf_driver_raw_24g.o
                0x9d026038                ScratchMount

.text.TCP_Flush
                0x9d0260b8       0x7c
 .text.TCP_Flush
                0x9d0260b8       0x7c build/WiFIG/production/_ext/427700826/tcp.o

.text._TCPIPStackAddressServiceSelect
                0x9d026134       0x7c
 .text._TCPIPStackAddressServiceSelect
                0x9d026134       0x7c build/WiFIG/production/_ext/427700826/tcpip_manager.o
                0x9d026134                _TCPIPStackAddressServiceSelect

.text.MRF24W_MACGetConfig
                0x9d0261b0       0x7c
 .text.MRF24W_MACGetConfig
                0x9d0261b0       0x7c build/WiFIG/production/_ext/334706090/mrf24w_mac_pic32.o
                0x9d0261b0                MRF24W_MACGetConfig

.text.DeallocateDataRxBuffer
                0x9d02622c       0x7c
 .text.DeallocateDataRxBuffer
                0x9d02622c       0x7c build/WiFIG/production/_ext/334706090/wf_driver_raw_24g.o
                0x9d02622c                DeallocateDataRxBuffer

.text.LFSRRand  0x9d0262a8       0x78
 .text.LFSRRand
                0x9d0262a8       0x78 build/WiFIG/production/_ext/101875047/lfsr.o
                0x9d0262a8                LFSRRand

.text.SYS_TICK_TimerSetRate
                0x9d026320       0x78
 .text.SYS_TICK_TimerSetRate
                0x9d026320       0x78 build/WiFIG/production/_ext/365611741/system_services.o
                0x9d026320                SYS_TICK_TimerSetRate

.text.DHCPDeRegisterHandler
                0x9d026398       0x78
 .text.DHCPDeRegisterHandler
                0x9d026398       0x78 build/WiFIG/production/_ext/427700826/dhcp.o
                0x9d026398                DHCPDeRegisterHandler

.text.DNSClientDeInit
                0x9d026410       0x78
 .text.DNSClientDeInit
                0x9d026410       0x78 build/WiFIG/production/_ext/427700826/dns.o
                0x9d026410                DNSClientDeInit

.text.SetWepSecurity
                0x9d026488       0x78
 .text.SetWepSecurity
                0x9d026488       0x78 build/WiFIG/production/_ext/334706090/wf_connect.o

.text.ResetPll  0x9d026500       0x78
 .text.ResetPll
                0x9d026500       0x78 build/WiFIG/production/_ext/334706090/wf_driver_com_24g.o

.text.SendRAWDataFrame
                0x9d026578       0x78
 .text.SendRAWDataFrame
                0x9d026578       0x78 build/WiFIG/production/_ext/334706090/wf_driver_raw_24g.o
                0x9d026578                SendRAWDataFrame

.text.MRF24W_MACFlush
                0x9d0265f0       0x78
 .text.MRF24W_MACFlush
                0x9d0265f0       0x78 build/WiFIG/production/_ext/334706090/wf_mac_24g.o
                0x9d0265f0                MRF24W_MACFlush

.text.rand      0x9d026668       0x78
 .text.rand     0x9d026668       0x78 c:/program files (x86)/microchip/xc32/v1.21/bin/../lib/gcc/pic32mx/4.5.2/../../../../pic32mx/lib/size\libc.a(rand.o)
                0x9d026668                rand

.text.strstr    0x9d0266e0       0x78
 .text.strstr   0x9d0266e0       0x78 c:/program files (x86)/microchip/xc32/v1.21/bin/../lib/gcc/pic32mx/4.5.2/../../../../pic32mx/lib/size\libc.a(strstr.o)
                0x9d0266e0                strstr

.text.SYS_RANDOM_ADD
                0x9d026758       0x74
 .text.SYS_RANDOM_ADD
                0x9d026758       0x74 build/WiFIG/production/_ext/365611741/system_random.o
                0x9d026758                SYS_RANDOM_ADD

.text.TCPIP_IPV4_SetTxBuffer
                0x9d0267cc       0x74
 .text.TCPIP_IPV4_SetTxBuffer
                0x9d0267cc       0x74 build/WiFIG/production/_ext/427700826/ipv4.o
                0x9d0267cc                TCPIP_IPV4_SetTxBuffer

.text.TCP_GetUpperLayerHeaderPtr
                0x9d026840       0x74
 .text.TCP_GetUpperLayerHeaderPtr
                0x9d026840       0x74 build/WiFIG/production/_ext/427700826/tcp.o

.text.TCP_IsPacketQueued
                0x9d0268b4       0x74
 .text.TCP_IsPacketQueued
                0x9d0268b4       0x74 build/WiFIG/production/_ext/427700826/tcp.o

.text.TCP_ResetTransmitPacketState
                0x9d026928       0x74
 .text.TCP_ResetTransmitPacketState
                0x9d026928       0x74 build/WiFIG/production/_ext/427700826/tcp.o

.text._TCPIP_HEAP_FreeDebug
                0x9d02699c       0x74
 .text._TCPIP_HEAP_FreeDebug
                0x9d02699c       0x74 build/WiFIG/production/_ext/427700826/tcpip_heap_alloc.o
                0x9d02699c                _TCPIP_HEAP_FreeDebug

.text.UDPIsConnected
                0x9d026a10       0x74
 .text.UDPIsConnected
                0x9d026a10       0x74 build/WiFIG/production/_ext/427700826/udp.o
                0x9d026a10                UDPIsConnected

.text._TCPIPStackIsAddressOfNet
                0x9d026a84       0x74
 .text._TCPIPStackIsAddressOfNet
                0x9d026a84       0x74 build/WiFIG/production/_ext/427700826/tcpip_manager.o
                0x9d026a84                _TCPIPStackIsAddressOfNet

.text.WF_PsPollDisable
                0x9d026af8       0x74
 .text.WF_PsPollDisable
                0x9d026af8       0x74 build/WiFIG/production/_ext/334706090/wf_power_save.o
                0x9d026af8                WF_PsPollDisable

.text.EnsureWFisAwake
                0x9d026b6c       0x74
 .text.EnsureWFisAwake
                0x9d026b6c       0x74 build/WiFIG/production/_ext/334706090/wf_power_save.o
                0x9d026b6c                EnsureWFisAwake

.text.RawRead   0x9d026be0       0x74
 .text.RawRead  0x9d026be0       0x74 build/WiFIG/production/_ext/334706090/wf_driver_raw_24g.o
                0x9d026be0                RawRead

.text.RawWrite  0x9d026c54       0x74
 .text.RawWrite
                0x9d026c54       0x74 build/WiFIG/production/_ext/334706090/wf_driver_raw_24g.o
                0x9d026c54                RawWrite

.text.RawInit   0x9d026cc8       0x74
 .text.RawInit  0x9d026cc8       0x74 build/WiFIG/production/_ext/334706090/wf_mac_24g.o
                0x9d026cc8                RawInit

.text.SYS_INT_SourceRestore
                0x9d026d3c       0x70
 .text.SYS_INT_SourceRestore
                0x9d026d3c       0x70 build/WiFIG/production/_ext/365611741/system_services.o
                0x9d026d3c                SYS_INT_SourceRestore

.text._ARPDeleteCache
                0x9d026dac       0x70
 .text._ARPDeleteCache
                0x9d026dac       0x70 build/WiFIG/production/_ext/427700826/arp.o

.text.ICMPInitialize
                0x9d026e1c       0x70
 .text.ICMPInitialize
                0x9d026e1c       0x70 build/WiFIG/production/_ext/427700826/icmp.o
                0x9d026e1c                ICMPInitialize

.text.TCPIP_IPV4_SingleListFree
                0x9d026e8c       0x70
 .text.TCPIP_IPV4_SingleListFree
                0x9d026e8c       0x70 build/WiFIG/production/_ext/427700826/ipv4.o
                0x9d026e8c                TCPIP_IPV4_SingleListFree

.text.NBNSInit  0x9d026efc       0x70
 .text.NBNSInit
                0x9d026efc       0x70 build/WiFIG/production/_ext/427700826/nbns.o
                0x9d026efc                NBNSInit

.text.TCPPutString
                0x9d026f6c       0x70
 .text.TCPPutString
                0x9d026f6c       0x70 build/WiFIG/production/_ext/427700826/tcp.o
                0x9d026f6c                TCPPutString

.text.WF_Connect
                0x9d026fdc       0x70
 .text.WF_Connect
                0x9d026fdc       0x70 build/WiFIG/production/_ext/334706090/wf_connection_manager.o
                0x9d026fdc                WF_Connect

.text.MRF24W_MACOpen
                0x9d02704c       0x70
 .text.MRF24W_MACOpen
                0x9d02704c       0x70 build/WiFIG/production/_ext/334706090/mrf24w_mac_pic32.o
                0x9d02704c                MRF24W_MACOpen

.text.Write8BitWFRegister
                0x9d0270bc       0x70
 .text.Write8BitWFRegister
                0x9d0270bc       0x70 build/WiFIG/production/_ext/334706090/wf_driver_com_24g.o
                0x9d0270bc                Write8BitWFRegister

.text._ARPRefreshEntry
                0x9d02712c       0x6c
 .text._ARPRefreshEntry
                0x9d02712c       0x6c build/WiFIG/production/_ext/427700826/arp.o

.text._TCPGetRxFIFOFree
                0x9d027198       0x6c
 .text._TCPGetRxFIFOFree
                0x9d027198       0x6c build/WiFIG/production/_ext/427700826/tcp.o

.text.TcpClientIpv4RemoteHash
                0x9d027204       0x6c
 .text.TcpClientIpv4RemoteHash
                0x9d027204       0x6c build/WiFIG/production/_ext/427700826/tcp.o

.text.TCPIP_HEAP_FreeSize
                0x9d027270       0x6c
 .text.TCPIP_HEAP_FreeSize
                0x9d027270       0x6c build/WiFIG/production/_ext/427700826/tcpip_heap_alloc.o
                0x9d027270                TCPIP_HEAP_FreeSize

.rodata         0x9d0272dc       0x6c
 .rodata        0x9d0272dc       0x6c build/WiFIG/production/_ext/427700826/udp.o

.text.ProcessTCPIPMacGeneric
                0x9d027348       0x6c
 .text.ProcessTCPIPMacGeneric
                0x9d027348       0x6c build/WiFIG/production/_ext/427700826/tcpip_manager.o

.text.TCPIP_STACK_NetBIOSName
                0x9d0273b4       0x6c
 .text.TCPIP_STACK_NetBIOSName
                0x9d0273b4       0x6c build/WiFIG/production/_ext/427700826/tcpip_manager.o
                0x9d0273b4                TCPIP_STACK_NetBIOSName

.text.TCPIP_STACK_FilterRxPkt
                0x9d027420       0x6c
 .text.TCPIP_STACK_FilterRxPkt
                0x9d027420       0x6c build/WiFIG/production/_ext/427700826/tcpip_manager.o

.text.TCPIP_NotificationRemove
                0x9d02748c       0x6c
 .text.TCPIP_NotificationRemove
                0x9d02748c       0x6c build/WiFIG/production/_ext/427700826/tcpip_notify.o
                0x9d02748c                TCPIP_NotificationRemove

.text.SendPowerModeMsg
                0x9d0274f8       0x6c
 .text.SendPowerModeMsg
                0x9d0274f8       0x6c build/WiFIG/production/_ext/334706090/wf_power_save.o

.text.Read8BitWFRegister
                0x9d027564       0x6c
 .text.Read8BitWFRegister
                0x9d027564       0x6c build/WiFIG/production/_ext/334706090/wf_driver_com_24g.o
                0x9d027564                Read8BitWFRegister

.text.MRF24W_MACInit
                0x9d0275d0       0x6c
 .text.MRF24W_MACInit
                0x9d0275d0       0x6c build/WiFIG/production/_ext/334706090/wf_mac_24g.o
                0x9d0275d0                MRF24W_MACInit

.text.OAHashGetEntry
                0x9d02763c       0x68
 .text.OAHashGetEntry
                0x9d02763c       0x68 build/WiFIG/production/_ext/427700826/hash_tbl.o
                0x9d02763c                OAHashGetEntry

.text.TCPIP_IPV4_FreePacket
                0x9d0276a4       0x68
 .text.TCPIP_IPV4_FreePacket
                0x9d0276a4       0x68 build/WiFIG/production/_ext/427700826/ipv4.o
                0x9d0276a4                TCPIP_IPV4_FreePacket

.text._TcpSocketBind
                0x9d02770c       0x68
 .text._TcpSocketBind
                0x9d02770c       0x68 build/WiFIG/production/_ext/427700826/tcp.o

.text._TcpSocketChk
                0x9d027774       0x68
 .text._TcpSocketChk
                0x9d027774       0x68 build/WiFIG/production/_ext/427700826/tcp.o

.text._TcpFlush
                0x9d0277dc       0x68
 .text._TcpFlush
                0x9d0277dc       0x68 build/WiFIG/production/_ext/427700826/tcp.o

.text._UdpSocketBind
                0x9d027844       0x68
 .text._UdpSocketBind
                0x9d027844       0x68 build/WiFIG/production/_ext/427700826/udp.o

.text.MACPutHeader
                0x9d0278ac       0x68
 .text.MACPutHeader
                0x9d0278ac       0x68 build/WiFIG/production/_ext/427700826/tcpip_mac_object.o
                0x9d0278ac                MACPutHeader

.text.TCPIP_STACK_NetName
                0x9d027914       0x68
 .text.TCPIP_STACK_NetName
                0x9d027914       0x68 build/WiFIG/production/_ext/427700826/tcpip_manager.o
                0x9d027914                TCPIP_STACK_NetName

.text.TCPIP_NotificationAdd
                0x9d02797c       0x68
 .text.TCPIP_NotificationAdd
                0x9d02797c       0x68 build/WiFIG/production/_ext/427700826/tcpip_notify.o
                0x9d02797c                TCPIP_NotificationAdd

.rodata         0x9d0279e4       0x68
 .rodata        0x9d0279e4       0x68 build/WiFIG/production/_ext/334706090/mrf24w_mac_pic32.o

.text.MRF24W_MACEventDeInit
                0x9d027a4c       0x68
 .text.MRF24W_MACEventDeInit
                0x9d027a4c       0x68 build/WiFIG/production/_ext/334706090/mrf24w_events.o
                0x9d027a4c                MRF24W_MACEventDeInit

.text.RawCalculateChecksum
                0x9d027ab4       0x68
 .text.RawCalculateChecksum
                0x9d027ab4       0x68 build/WiFIG/production/_ext/334706090/wf_driver_raw_24g.o
                0x9d027ab4                RawCalculateChecksum

.text.MRF24W_MACPutArray
                0x9d027b1c       0x68
 .text.MRF24W_MACPutArray
                0x9d027b1c       0x68 build/WiFIG/production/_ext/334706090/wf_mac_24g.o
                0x9d027b1c                MRF24W_MACPutArray

.rodata         0x9d027b84       0x68
 .rodata        0x9d027b84       0x68 c:/program files (x86)/microchip/xc32/v1.21/bin/../lib/gcc/pic32mx/4.5.2/../../../../pic32mx/lib/size\libc.a(powersf.o)
                0x9d027b84                _powers_f
                0x9d027bb8                _npowers_f

.text.TCPIP_IPV4_GetDataSegmentContentsByType
                0x9d027bec       0x64
 .text.TCPIP_IPV4_GetDataSegmentContentsByType
                0x9d027bec       0x64 build/WiFIG/production/_ext/427700826/ipv4.o
                0x9d027bec                TCPIP_IPV4_GetDataSegmentContentsByType

.text._TCPIPStackIsNetLinked
                0x9d027c50       0x64
 .text._TCPIPStackIsNetLinked
                0x9d027c50       0x64 build/WiFIG/production/_ext/427700826/tcpip_manager.o
                0x9d027c50                _TCPIPStackIsNetLinked

.text.TCPIP_NotificationRemoveAll
                0x9d027cb4       0x64
 .text.TCPIP_NotificationRemoveAll
                0x9d027cb4       0x64 build/WiFIG/production/_ext/427700826/tcpip_notify.o
                0x9d027cb4                TCPIP_NotificationRemoveAll

.text.WF_CPCreate
                0x9d027d18       0x64
 .text.WF_CPCreate
                0x9d027d18       0x64 build/WiFIG/production/_ext/334706090/wf_connection_profile.o
                0x9d027d18                WF_CPCreate

.text.MRF24W_MACEventSetNotifyEvents
                0x9d027d7c       0x64
 .text.MRF24W_MACEventSetNotifyEvents
                0x9d027d7c       0x64 build/WiFIG/production/_ext/334706090/mrf24w_events.o
                0x9d027d7c                MRF24W_MACEventSetNotifyEvents

.text._sprintf_cdnopsuxX
                0x9d027de0       0x64
 .text._sprintf_cdnopsuxX
                0x9d027de0       0x64 c:/program files (x86)/microchip/xc32/v1.21/bin/../lib/gcc/pic32mx/4.5.2/../../../../pic32mx/lib/size\libc.a(sprintf_cdnopsuxX.eo)
                0x9d027de0                _sprintf_cdnopsuxX
                0x9d027de0                _sprintf_cdnopuxX

.text.USART_PUTC
                0x9d027e44       0x60
 .text.USART_PUTC
                0x9d027e44       0x60 build/WiFIG/production/_ext/792872985/usart.o
                0x9d027e44                USART_PUTC

.text.ICMPDeinitialize
                0x9d027ea4       0x60
 .text.ICMPDeinitialize
                0x9d027ea4       0x60 build/WiFIG/production/_ext/427700826/icmp.o
                0x9d027ea4                ICMPDeinitialize

.text.TCPIP_IPV4_SetRxBuffer
                0x9d027f04       0x60
 .text.TCPIP_IPV4_SetRxBuffer
                0x9d027f04       0x60 build/WiFIG/production/_ext/427700826/ipv4.o
                0x9d027f04                TCPIP_IPV4_SetRxBuffer

.text.TCP_FreePacket
                0x9d027f64       0x60
 .text.TCP_FreePacket
                0x9d027f64       0x60 build/WiFIG/production/_ext/427700826/tcp.o

.text.MACCalcRxChecksum
                0x9d027fc4       0x60
 .text.MACCalcRxChecksum
                0x9d027fc4       0x60 build/WiFIG/production/_ext/427700826/tcpip_mac_object.o
                0x9d027fc4                MACCalcRxChecksum

.rodata         0x9d028024       0x60
 .rodata        0x9d028024       0x60 build/WiFIG/production/_ext/427700826/tcpip_helpers.o

.text.ConfigureSpiMRF24W
                0x9d028084       0x60
 .text.ConfigureSpiMRF24W
                0x9d028084       0x60 build/WiFIG/production/_ext/334706090/wf_spi.o

.text.MRF24W_MACDeinitialize
                0x9d0280e4       0x60
 .text.MRF24W_MACDeinitialize
                0x9d0280e4       0x60 build/WiFIG/production/_ext/334706090/mrf24w_mac_pic32.o
                0x9d0280e4                MRF24W_MACDeinitialize

.text.mrf24w_MACSetRXHashTableEntry
                0x9d028144       0x60
 .text.mrf24w_MACSetRXHashTableEntry
                0x9d028144       0x60 build/WiFIG/production/_ext/334706090/mrf24w_mac_pic32.o

.text.WiFi_EintTask
                0x9d0281a4       0x60
 .text.WiFi_EintTask
                0x9d0281a4       0x60 build/WiFIG/production/_ext/334706090/wf_driver_com_24g.o
                0x9d0281a4                WiFi_EintTask

.text.SYS_INT_SourceDisable
                0x9d028204       0x5c
 .text.SYS_INT_SourceDisable
                0x9d028204       0x5c build/WiFIG/production/_ext/365611741/system_services.o
                0x9d028204                SYS_INT_SourceDisable

.text.SYS_INT_PrioritySet
                0x9d028260       0x5c
 .text.SYS_INT_PrioritySet
                0x9d028260       0x5c build/WiFIG/production/_ext/365611741/system_services.o
                0x9d028260                SYS_INT_PrioritySet

.text.SYS_INT_SubprioritySet
                0x9d0282bc       0x5c
 .text.SYS_INT_SubprioritySet
                0x9d0282bc       0x5c build/WiFIG/production/_ext/365611741/system_services.o
                0x9d0282bc                SYS_INT_SubprioritySet

.text._DHCPCleanup
                0x9d028318       0x5c
 .text._DHCPCleanup
                0x9d028318       0x5c build/WiFIG/production/_ext/427700826/dhcp.o

.text.OAHashRemoveEntry
                0x9d028374       0x5c
 .text.OAHashRemoveEntry
                0x9d028374       0x5c build/WiFIG/production/_ext/427700826/hash_tbl.o
                0x9d028374                OAHashRemoveEntry

.text.TCPFlush  0x9d0283d0       0x5c
 .text.TCPFlush
                0x9d0283d0       0x5c build/WiFIG/production/_ext/427700826/tcp.o
                0x9d0283d0                TCPFlush

.text.MACGetArray
                0x9d02842c       0x5c
 .text.MACGetArray
                0x9d02842c       0x5c build/WiFIG/production/_ext/427700826/tcpip_mac_object.o
                0x9d02842c                MACGetArray

.text.MACPutArray
                0x9d028488       0x5c
 .text.MACPutArray
                0x9d028488       0x5c build/WiFIG/production/_ext/427700826/tcpip_mac_object.o
                0x9d028488                MACPutArray

.text.MACEventSetNotifyHandler
                0x9d0284e4       0x5c
 .text.MACEventSetNotifyHandler
                0x9d0284e4       0x5c build/WiFIG/production/_ext/427700826/tcpip_mac_object.o
                0x9d0284e4                MACEventSetNotifyHandler

.text._TCPIPStackNetAddress
                0x9d028540       0x5c
 .text._TCPIPStackNetAddress
                0x9d028540       0x5c build/WiFIG/production/_ext/427700826/tcpip_manager.o
                0x9d028540                _TCPIPStackNetAddress

.text._TCPIPStackNetMask
                0x9d02859c       0x5c
 .text._TCPIPStackNetMask
                0x9d02859c       0x5c build/WiFIG/production/_ext/427700826/tcpip_manager.o
                0x9d02859c                _TCPIPStackNetMask

.text._TCPIPStackNetMacAddress
                0x9d0285f8       0x5c
 .text._TCPIPStackNetMacAddress
                0x9d0285f8       0x5c build/WiFIG/production/_ext/427700826/tcpip_manager.o
                0x9d0285f8                _TCPIPStackNetMacAddress

.text.SetListenInterval
                0x9d028654       0x5c
 .text.SetListenInterval
                0x9d028654       0x5c build/WiFIG/production/_ext/334706090/wf_connection_algorithm.o
                0x9d028654                SetListenInterval

.text.SetDtimInterval
                0x9d0286b0       0x5c
 .text.SetDtimInterval
                0x9d0286b0       0x5c build/WiFIG/production/_ext/334706090/wf_connection_algorithm.o
                0x9d0286b0                SetDtimInterval

.text.WF_SecurityWepSet
                0x9d02870c       0x5c
 .text.WF_SecurityWepSet
                0x9d02870c       0x5c build/WiFIG/production/_ext/334706090/wf_connection_profile.o
                0x9d02870c                WF_SecurityWepSet

.text.WF_SecurityWpaSet
                0x9d028768       0x5c
 .text.WF_SecurityWpaSet
                0x9d028768       0x5c build/WiFIG/production/_ext/334706090/wf_connection_profile.o
                0x9d028768                WF_SecurityWpaSet

.text.WF_SecurityWpsSet
                0x9d0287c4       0x5c
 .text.WF_SecurityWpsSet
                0x9d0287c4       0x5c build/WiFIG/production/_ext/334706090/wf_connection_profile.o
                0x9d0287c4                WF_SecurityWpsSet

.text.WF_EintIsPending
                0x9d028820       0x5c
 .text.WF_EintIsPending
                0x9d028820       0x5c build/WiFIG/production/_ext/334706090/wf_eint.o
                0x9d028820                WF_EintIsPending

.text.mrf24w_MACPutHeader
                0x9d02887c       0x5c
 .text.mrf24w_MACPutHeader
                0x9d02887c       0x5c build/WiFIG/production/_ext/334706090/mrf24w_mac_pic32.o

.text.SignalWiFiConnectionChanged
                0x9d0288d8       0x5c
 .text.SignalWiFiConnectionChanged
                0x9d0288d8       0x5c build/WiFIG/production/_ext/334706090/wf_driver_com_24g.o
                0x9d0288d8                SignalWiFiConnectionChanged

.text.WF_StartGratuitousArp
                0x9d028934       0x5c
 .text.WF_StartGratuitousArp
                0x9d028934       0x5c build/WiFIG/production/_ext/334706090/wf_mac_24g.o
                0x9d028934                WF_StartGratuitousArp

.text.MRF24W_MACIsTxReady
                0x9d028990       0x5c
 .text.MRF24W_MACIsTxReady
                0x9d028990       0x5c build/WiFIG/production/_ext/334706090/wf_mac_24g.o
                0x9d028990                MRF24W_MACIsTxReady

.text.SYS_INT_SourceEnable
                0x9d0289ec       0x58
 .text.SYS_INT_SourceEnable
                0x9d0289ec       0x58 build/WiFIG/production/_ext/365611741/system_services.o
                0x9d0289ec                SYS_INT_SourceEnable

.text.USART_OPEN
                0x9d028a44       0x58
 .text.USART_OPEN
                0x9d028a44       0x58 build/WiFIG/production/_ext/792872985/usart.o
                0x9d028a44                USART_OPEN

.text.USART_GETC
                0x9d028a9c       0x58
 .text.USART_GETC
                0x9d028a9c       0x58 build/WiFIG/production/_ext/792872985/usart.o
                0x9d028a9c                USART_GETC

.text.WaitForDataByte
                0x9d028af4       0x58
 .text.WaitForDataByte
                0x9d028af4       0x58 build/WiFIG/production/_ext/792872985/drv_spi.o

.text.ARPHashKeyHash
                0x9d028b4c       0x58
 .text.ARPHashKeyHash
                0x9d028b4c       0x58 build/WiFIG/production/_ext/427700826/arp.o
                0x9d028b4c                ARPHashKeyHash

.text._TcpipHeapHandleToDcpt
                0x9d028ba4       0x58
 .text._TcpipHeapHandleToDcpt
                0x9d028ba4       0x58 build/WiFIG/production/_ext/427700826/tcpip_heap_alloc.o

.text.TCPIP_STACK_IxToNet
                0x9d028bfc       0x58
 .text.TCPIP_STACK_IxToNet
                0x9d028bfc       0x58 build/WiFIG/production/_ext/427700826/tcpip_manager.o
                0x9d028bfc                TCPIP_STACK_IxToNet

.text._TCPIPStackIsNetUp
                0x9d028c54       0x58
 .text._TCPIPStackIsNetUp
                0x9d028c54       0x58 build/WiFIG/production/_ext/427700826/tcpip_manager.o
                0x9d028c54                _TCPIPStackIsNetUp

.text.WF_NetworkTypeSet
                0x9d028cac       0x58
 .text.WF_NetworkTypeSet
                0x9d028cac       0x58 build/WiFIG/production/_ext/334706090/wf_connection_profile.o
                0x9d028cac                WF_NetworkTypeSet

.text.mrf24w_MACCalcRxChecksum
                0x9d028d04       0x58
 .text.mrf24w_MACCalcRxChecksum
                0x9d028d04       0x58 build/WiFIG/production/_ext/334706090/mrf24w_mac_pic32.o

.text.MRF24W_MACCalcIPBufferChecksum
                0x9d028d5c       0x58
 .text.MRF24W_MACCalcIPBufferChecksum
                0x9d028d5c       0x58 build/WiFIG/production/_ext/334706090/wf_mac_24g.o
                0x9d028d5c                MRF24W_MACCalcIPBufferChecksum

.text.SYS_INT_SourceStatusClear
                0x9d028db4       0x54
 .text.SYS_INT_SourceStatusClear
                0x9d028db4       0x54 build/WiFIG/production/_ext/365611741/system_services.o
                0x9d028db4                SYS_INT_SourceStatusClear

.text._ICMPAckPacket
                0x9d028e08       0x54
 .text._ICMPAckPacket
                0x9d028e08       0x54 build/WiFIG/production/_ext/427700826/icmp.o

.text._TcpDiscardTx
                0x9d028e5c       0x54
 .text._TcpDiscardTx
                0x9d028e5c       0x54 build/WiFIG/production/_ext/427700826/tcp.o

.text._UdpSocketInit
                0x9d028eb0       0x54
 .text._UdpSocketInit
                0x9d028eb0       0x54 build/WiFIG/production/_ext/427700826/udp.o

.text.UDPPut    0x9d028f04       0x54
 .text.UDPPut   0x9d028f04       0x54 build/WiFIG/production/_ext/427700826/udp.o
                0x9d028f04                UDPPut

.text.MACGetHeader
                0x9d028f58       0x54
 .text.MACGetHeader
                0x9d028f58       0x54 build/WiFIG/production/_ext/427700826/tcpip_mac_object.o
                0x9d028f58                MACGetHeader

.text.MACSetReadPtrInRx
                0x9d028fac       0x54
 .text.MACSetReadPtrInRx
                0x9d028fac       0x54 build/WiFIG/production/_ext/427700826/tcpip_mac_object.o
                0x9d028fac                MACSetReadPtrInRx

.text.MACCalcIPBufferChecksum
                0x9d029000       0x54
 .text.MACCalcIPBufferChecksum
                0x9d029000       0x54 build/WiFIG/production/_ext/427700826/tcpip_mac_object.o
                0x9d029000                MACCalcIPBufferChecksum

.text.MACEventSetNotifyEvents
                0x9d029054       0x54
 .text.MACEventSetNotifyEvents
                0x9d029054       0x54 build/WiFIG/production/_ext/427700826/tcpip_mac_object.o
                0x9d029054                MACEventSetNotifyEvents

.text.MACEventAck
                0x9d0290a8       0x54
 .text.MACEventAck
                0x9d0290a8       0x54 build/WiFIG/production/_ext/427700826/tcpip_mac_object.o
                0x9d0290a8                MACEventAck

.text._TCPIPStackAddressServiceCanStart
                0x9d0290fc       0x54
 .text._TCPIPStackAddressServiceCanStart
                0x9d0290fc       0x54 build/WiFIG/production/_ext/427700826/tcpip_manager.o
                0x9d0290fc                _TCPIPStackAddressServiceCanStart

.text._TCPIPStackAddressServiceSetDefault
                0x9d029150       0x54
 .text._TCPIPStackAddressServiceSetDefault
                0x9d029150       0x54 build/WiFIG/production/_ext/427700826/tcpip_manager.o
                0x9d029150                _TCPIPStackAddressServiceSetDefault

.text.mrf24w_MACDeinitialize
                0x9d0291a4       0x54
 .text.mrf24w_MACDeinitialize
                0x9d0291a4       0x54 build/WiFIG/production/_ext/334706090/mrf24w_mac_pic32.o

.text.GratuitousArpHandler
                0x9d0291f8       0x54
 .text.GratuitousArpHandler
                0x9d0291f8       0x54 build/WiFIG/production/_ext/334706090/wf_mac_24g.o

.text._vsnprintf_cdnopsuxX
                0x9d02924c       0x54
 .text._vsnprintf_cdnopsuxX
                0x9d02924c       0x54 c:/program files (x86)/microchip/xc32/v1.21/bin/../lib/gcc/pic32mx/4.5.2/../../../../pic32mx/lib/size\libc.a(vsnprintf_cdnopsuxX.eo)
                0x9d02924c                _vsnprintf_cdnopsuxX

.text.vsnprintf
                0x9d0292a0       0x54
 .text.vsnprintf
                0x9d0292a0       0x54 c:/program files (x86)/microchip/xc32/v1.21/bin/../lib/gcc/pic32mx/4.5.2/../../../../pic32mx/lib/size\libc.a(vsnprintf.o)
                0x9d0292a0                vsnprintf

.text._SYS_CONSOLE_MESSAGE
                0x9d0292f4       0x50
 .text._SYS_CONSOLE_MESSAGE
                0x9d0292f4       0x50 build/WiFIG/production/_ext/365611741/system_debug.o
                0x9d0292f4                _SYS_CONSOLE_MESSAGE

.text._TCPIP_AnnounceCleanup
                0x9d029344       0x50
 .text._TCPIP_AnnounceCleanup
                0x9d029344       0x50 build/WiFIG/production/_ext/427700826/tcpip_announce.o

.text.ARPHashKeyCompare
                0x9d029394       0x50
 .text.ARPHashKeyCompare
                0x9d029394       0x50 build/WiFIG/production/_ext/427700826/arp.o
                0x9d029394                ARPHashKeyCompare

.text._DNSReleaseSocket
                0x9d0293e4       0x50
 .text._DNSReleaseSocket
                0x9d0293e4       0x50 build/WiFIG/production/_ext/427700826/dns.o

.text.WF_EintInit
                0x9d029434       0x50
 .text.WF_EintInit
                0x9d029434       0x50 build/WiFIG/production/_ext/334706090/wf_eint.o
                0x9d029434                WF_EintInit

.text.WF_SpiInit
                0x9d029484       0x50
 .text.WF_SpiInit
                0x9d029484       0x50 build/WiFIG/production/_ext/334706090/wf_spi.o
                0x9d029484                WF_SpiInit

.text.mrf24w_MACEventSetNotifyHandler
                0x9d0294d4       0x50
 .text.mrf24w_MACEventSetNotifyHandler
                0x9d0294d4       0x50 build/WiFIG/production/_ext/334706090/mrf24w_mac_pic32.o

.text.MRF24W_GetTrafficEvents
                0x9d029524       0x50
 .text.MRF24W_GetTrafficEvents
                0x9d029524       0x50 build/WiFIG/production/_ext/334706090/mrf24w_events.o
                0x9d029524                MRF24W_GetTrafficEvents

.text.MRF24W_GetMgmtEvents
                0x9d029574       0x50
 .text.MRF24W_GetMgmtEvents
                0x9d029574       0x50 build/WiFIG/production/_ext/334706090/mrf24w_events.o
                0x9d029574                MRF24W_GetMgmtEvents

.text.SignalDHCPSuccessful
                0x9d0295c4       0x50
 .text.SignalDHCPSuccessful
                0x9d0295c4       0x50 build/WiFIG/production/_ext/334706090/wf_driver_com_24g.o
                0x9d0295c4                SignalDHCPSuccessful

.text.InitGratuitousArp
                0x9d029614       0x50
 .text.InitGratuitousArp
                0x9d029614       0x50 build/WiFIG/production/_ext/334706090/wf_mac_24g.o
                0x9d029614                InitGratuitousArp

.text.MRF24W_MACSetWritePtr
                0x9d029664       0x50
 .text.MRF24W_MACSetWritePtr
                0x9d029664       0x50 build/WiFIG/production/_ext/334706090/wf_mac_24g.o
                0x9d029664                MRF24W_MACSetWritePtr

.text.MRF24W_MACSetReadPtr
                0x9d0296b4       0x50
 .text.MRF24W_MACSetReadPtr
                0x9d0296b4       0x50 build/WiFIG/production/_ext/334706090/wf_mac_24g.o
                0x9d0296b4                MRF24W_MACSetReadPtr

.text.MRF24W_MACSetBaseReadPtr
                0x9d029704       0x50
 .text.MRF24W_MACSetBaseReadPtr
                0x9d029704       0x50 build/WiFIG/production/_ext/334706090/wf_mac_24g.o
                0x9d029704                MRF24W_MACSetBaseReadPtr

.text.StackNotification
                0x9d029754       0x50
 .text.StackNotification
                0x9d029754       0x50 build/WiFIG/production/_ext/1472/main_demo.o

.text.DRV_SPI_Initialize
                0x9d0297a4       0x4c
 .text.DRV_SPI_Initialize
                0x9d0297a4       0x4c build/WiFIG/production/_ext/792872985/drv_spi.o
                0x9d0297a4                DRV_SPI_Initialize

.text.TCPGet    0x9d0297f0       0x4c
 .text.TCPGet   0x9d0297f0       0x4c build/WiFIG/production/_ext/427700826/tcp.o
                0x9d0297f0                TCPGet

.text.UDPGet    0x9d02983c       0x4c
 .text.UDPGet   0x9d02983c       0x4c build/WiFIG/production/_ext/427700826/udp.o
                0x9d02983c                UDPGet

.text.MACSetWritePtr
                0x9d029888       0x4c
 .text.MACSetWritePtr
                0x9d029888       0x4c build/WiFIG/production/_ext/427700826/tcpip_mac_object.o
                0x9d029888                MACSetWritePtr

.text.MACSetReadPtr
                0x9d0298d4       0x4c
 .text.MACSetReadPtr
                0x9d0298d4       0x4c build/WiFIG/production/_ext/427700826/tcpip_mac_object.o
                0x9d0298d4                MACSetReadPtr

.text.MACEventGetPending
                0x9d029920       0x4c
 .text.MACEventGetPending
                0x9d029920       0x4c build/WiFIG/production/_ext/427700826/tcpip_mac_object.o
                0x9d029920                MACEventGetPending

.text.WF_ChannelListSet
                0x9d02996c       0x4c
 .text.WF_ChannelListSet
                0x9d02996c       0x4c build/WiFIG/production/_ext/334706090/wf_connection_algorithm.o
                0x9d02996c                WF_ChannelListSet

.text.WF_EintEnable
                0x9d0299b8       0x4c
 .text.WF_EintEnable
                0x9d0299b8       0x4c build/WiFIG/production/_ext/334706090/wf_eint.o
                0x9d0299b8                WF_EintEnable

.text.DhcpEventHandler
                0x9d029a04       0x4c
 .text.DhcpEventHandler
                0x9d029a04       0x4c build/WiFIG/production/_ext/334706090/wf_event_handler.o
                0x9d029a04                DhcpEventHandler

.text.mrf24w_MACPutArray
                0x9d029a50       0x4c
 .text.mrf24w_MACPutArray
                0x9d029a50       0x4c build/WiFIG/production/_ext/334706090/mrf24w_mac_pic32.o

.text.mrf24w_MACGetArray
                0x9d029a9c       0x4c
 .text.mrf24w_MACGetArray
                0x9d029a9c       0x4c build/WiFIG/production/_ext/334706090/mrf24w_mac_pic32.o

.text.MRF24W_MACEventAck
                0x9d029ae8       0x4c
 .text.MRF24W_MACEventAck
                0x9d029ae8       0x4c build/WiFIG/production/_ext/334706090/mrf24w_events.o
                0x9d029ae8                MRF24W_MACEventAck

.text.SendRAWManagementFrame
                0x9d029b34       0x4c
 .text.SendRAWManagementFrame
                0x9d029b34       0x4c build/WiFIG/production/_ext/334706090/wf_driver_raw_24g.o
                0x9d029b34                SendRAWManagementFrame

.text.ScratchUnmount
                0x9d029b80       0x4c
 .text.ScratchUnmount
                0x9d029b80       0x4c build/WiFIG/production/_ext/334706090/wf_driver_raw_24g.o
                0x9d029b80                ScratchUnmount

.text.MRF24W_MACSetReadPtrInRx
                0x9d029bcc       0x4c
 .text.MRF24W_MACSetReadPtrInRx
                0x9d029bcc       0x4c build/WiFIG/production/_ext/334706090/wf_mac_24g.o
                0x9d029bcc                MRF24W_MACSetReadPtrInRx

.text.INTEnable
                0x9d029c18       0x4c
 .text.INTEnable
                0x9d029c18       0x4c c:/program files (x86)/microchip/xc32/v1.21/bin/../lib/gcc/pic32mx/4.5.2/../../../../pic32mx/lib/size\libmchp_peripheral_32MX695F512H.a(int_tbl_lib.o)
                0x9d029c18                INTEnable

.text           0x9d029c64       0x4c
 .text          0x9d029c64       0x4c c:/program files (x86)/microchip/xc32/v1.21/bin/../lib/gcc/pic32mx/4.5.2/size\libgcc.a(floatunsisf.o)
                0x9d029c64                __floatunsisf

.text.SYS_CLK_PeripheralClockGet
                0x9d029cb0       0x48
 .text.SYS_CLK_PeripheralClockGet
                0x9d029cb0       0x48 build/WiFIG/production/_ext/365611741/system_services.o
                0x9d029cb0                SYS_CLK_PeripheralClockGet

.text.ARPHashKeyCopy
                0x9d029cf8       0x48
 .text.ARPHashKeyCopy
                0x9d029cf8       0x48 build/WiFIG/production/_ext/427700826/arp.o
                0x9d029cf8                ARPHashKeyCopy

.text.DNSEndUsage
                0x9d029d40       0x48
 .text.DNSEndUsage
                0x9d029d40       0x48 build/WiFIG/production/_ext/427700826/dns.o
                0x9d029d40                DNSEndUsage

.text.TCPIP_IPV4_SetSourceAddress
                0x9d029d88       0x48
 .text.TCPIP_IPV4_SetSourceAddress
                0x9d029d88       0x48 build/WiFIG/production/_ext/427700826/ipv4.o
                0x9d029d88                TCPIP_IPV4_SetSourceAddress

.text.TCPIP_STACK_NetAddress
                0x9d029dd0       0x48
 .text.TCPIP_STACK_NetAddress
                0x9d029dd0       0x48 build/WiFIG/production/_ext/427700826/tcpip_manager.o
                0x9d029dd0                TCPIP_STACK_NetAddress

.text.TCPIP_STACK_NetMacAddress
                0x9d029e18       0x48
 .text.TCPIP_STACK_NetMacAddress
                0x9d029e18       0x48 build/WiFIG/production/_ext/427700826/tcpip_manager.o
                0x9d029e18                TCPIP_STACK_NetMacAddress

.text.isEventNotifyBitSet
                0x9d029e60       0x48
 .text.isEventNotifyBitSet
                0x9d029e60       0x48 build/WiFIG/production/_ext/334706090/wf_event_handler.o

.rodata         0x9d029ea8       0x48
 .rodata        0x9d029ea8       0x48 build/WiFIG/production/_ext/334706090/wf_init.o

.text.mrf24w_MACCalcIPBufferChecksum
                0x9d029ef0       0x48
 .text.mrf24w_MACCalcIPBufferChecksum
                0x9d029ef0       0x48 build/WiFIG/production/_ext/334706090/mrf24w_mac_pic32.o

.text.mrf24w_MACEventSetNotifyEvents
                0x9d029f38       0x48
 .text.mrf24w_MACEventSetNotifyEvents
                0x9d029f38       0x48 build/WiFIG/production/_ext/334706090/mrf24w_mac_pic32.o

.text.mrf24w_MACEventClearNotifyEvents
                0x9d029f80       0x48
 .text.mrf24w_MACEventClearNotifyEvents
                0x9d029f80       0x48 build/WiFIG/production/_ext/334706090/mrf24w_mac_pic32.o

.text.mrf24w_MACEventAck
                0x9d029fc8       0x48
 .text.mrf24w_MACEventAck
                0x9d029fc8       0x48 build/WiFIG/production/_ext/334706090/mrf24w_mac_pic32.o

.text.MRF24W_MACEventClearNotifyEvents
                0x9d02a010       0x48
 .text.MRF24W_MACEventClearNotifyEvents
                0x9d02a010       0x48 build/WiFIG/production/_ext/334706090/mrf24w_events.o
                0x9d02a010                MRF24W_MACEventClearNotifyEvents

.text.OutputPowerSaveMode
                0x9d02a058       0x48
 .text.OutputPowerSaveMode
                0x9d02a058       0x48 build/WiFIG/production/_ext/334706090/wf_debug_output.o

.text.WFEnableMRF24WMode
                0x9d02a0a0       0x48
 .text.WFEnableMRF24WMode
                0x9d02a0a0       0x48 build/WiFIG/production/_ext/334706090/wf_param_msg_24g.o
                0x9d02a0a0                WFEnableMRF24WMode

.rodata         0x9d02a0e8       0x48
 .rodata        0x9d02a0e8       0x48 c:/program files (x86)/microchip/xc32/v1.21/bin/../lib/gcc/pic32mx/4.5.2/../../../../pic32mx/lib/size\libmchp_peripheral_32MX695F512H.a(_ports_tbl_libp.o)
                0x9d02a0e8                PortRegTbl

.text._DefaultInterrupt
                0x9d02a130       0x48
 .text._DefaultInterrupt
                0x9d02a130       0x48 c:/program files (x86)/microchip/xc32/v1.21/bin/../lib/gcc/pic32mx/4.5.2/../../../../pic32mx/lib/size\libpic32.a(defaultinterrupt.o)
                0x9d02a130                _DefaultInterrupt

.text.sbrk      0x9d02a178       0x48
 .text.sbrk     0x9d02a178       0x48 c:/program files (x86)/microchip/xc32/v1.21/bin/../lib/gcc/pic32mx/4.5.2/../../../../pic32mx/lib/size\libpic32.a(sbrk.o)
                0x9d02a178                sbrk

.text.SYS_CLK_ClockGet
                0x9d02a1c0       0x44
 .text.SYS_CLK_ClockGet
                0x9d02a1c0       0x44 build/WiFIG/production/_ext/365611741/system_services.o
                0x9d02a1c0                SYS_CLK_ClockGet

.text.USART_DATA_RDY
                0x9d02a204       0x44
 .text.USART_DATA_RDY
                0x9d02a204       0x44 build/WiFIG/production/_ext/792872985/usart.o
                0x9d02a204                USART_DATA_RDY

.text.TCPIP_IPV4_SetPacketIPProtocol
                0x9d02a248       0x44
 .text.TCPIP_IPV4_SetPacketIPProtocol
                0x9d02a248       0x44 build/WiFIG/production/_ext/427700826/ipv4.o
                0x9d02a248                TCPIP_IPV4_SetPacketIPProtocol

.text.MACClose  0x9d02a28c       0x44
 .text.MACClose
                0x9d02a28c       0x44 build/WiFIG/production/_ext/427700826/tcpip_mac_object.o
                0x9d02a28c                MACClose

.text.MACDiscardRx
                0x9d02a2d0       0x44
 .text.MACDiscardRx
                0x9d02a2d0       0x44 build/WiFIG/production/_ext/427700826/tcpip_mac_object.o
                0x9d02a2d0                MACDiscardRx

.text.MACIsTxReady
                0x9d02a314       0x44
 .text.MACIsTxReady
                0x9d02a314       0x44 build/WiFIG/production/_ext/427700826/tcpip_mac_object.o
                0x9d02a314                MACIsTxReady

.text.MACFlush  0x9d02a358       0x44
 .text.MACFlush
                0x9d02a358       0x44 build/WiFIG/production/_ext/427700826/tcpip_mac_object.o
                0x9d02a358                MACFlush

.text.MACCheckLink
                0x9d02a39c       0x44
 .text.MACCheckLink
                0x9d02a39c       0x44 build/WiFIG/production/_ext/427700826/tcpip_mac_object.o
                0x9d02a39c                MACCheckLink

.text.MACGetTxBaseAddr
                0x9d02a3e0       0x44
 .text.MACGetTxBaseAddr
                0x9d02a3e0       0x44 build/WiFIG/production/_ext/427700826/tcpip_mac_object.o
                0x9d02a3e0                MACGetTxBaseAddr

.text.TCPIP_STACK_NetHandle
                0x9d02a424       0x44
 .text.TCPIP_STACK_NetHandle
                0x9d02a424       0x44 build/WiFIG/production/_ext/427700826/tcpip_manager.o
                0x9d02a424                TCPIP_STACK_NetHandle

.text._TCPIPStackNetIx
                0x9d02a468       0x44
 .text._TCPIPStackNetIx
                0x9d02a468       0x44 build/WiFIG/production/_ext/427700826/tcpip_manager.o
                0x9d02a468                _TCPIPStackNetIx

.text._TCPIPStackSetGatewayAddress
                0x9d02a4ac       0x44
 .text._TCPIPStackSetGatewayAddress
                0x9d02a4ac       0x44 build/WiFIG/production/_ext/427700826/tcpip_manager.o
                0x9d02a4ac                _TCPIPStackSetGatewayAddress

.text._TCPIPStackSetPriDNSAddress
                0x9d02a4f0       0x44
 .text._TCPIPStackSetPriDNSAddress
                0x9d02a4f0       0x44 build/WiFIG/production/_ext/427700826/tcpip_manager.o
                0x9d02a4f0                _TCPIPStackSetPriDNSAddress

.text._TCPIPStackSetSecondDNSAddress
                0x9d02a534       0x44
 .text._TCPIPStackSetSecondDNSAddress
                0x9d02a534       0x44 build/WiFIG/production/_ext/427700826/tcpip_manager.o
                0x9d02a534                _TCPIPStackSetSecondDNSAddress

.text._TCPIPStackNetToMac
                0x9d02a578       0x44
 .text._TCPIPStackNetToMac
                0x9d02a578       0x44 build/WiFIG/production/_ext/427700826/tcpip_manager.o
                0x9d02a578                _TCPIPStackNetToMac

.text.SingleListInit
                0x9d02a5bc       0x44
 .text.SingleListInit
                0x9d02a5bc       0x44 build/WiFIG/production/_ext/427700826/tcpip_helpers.o
                0x9d02a5bc                SingleListInit

.text.WF_ConnectContextGet
                0x9d02a600       0x44
 .text.WF_ConnectContextGet
                0x9d02a600       0x44 build/WiFIG/production/_ext/334706090/wf_connection_manager.o
                0x9d02a600                WF_ConnectContextGet

.rodata         0x9d02a644       0x44
 .rodata        0x9d02a644       0x44 build/WiFIG/production/_ext/334706090/wf_connection_profile.o

.text.WF_NetworkTypeGet
                0x9d02a688       0x44
 .text.WF_NetworkTypeGet
                0x9d02a688       0x44 build/WiFIG/production/_ext/334706090/wf_connection_profile.o
                0x9d02a688                WF_NetworkTypeGet

.text.WF_WepKeyTypeGet
                0x9d02a6cc       0x44
 .text.WF_WepKeyTypeGet
                0x9d02a6cc       0x44 build/WiFIG/production/_ext/334706090/wf_connection_profile.o
                0x9d02a6cc                WF_WepKeyTypeGet

.text.mrf24w_MACGetHeader
                0x9d02a710       0x44
 .text.mrf24w_MACGetHeader
                0x9d02a710       0x44 build/WiFIG/production/_ext/334706090/mrf24w_mac_pic32.o

.text.mrf24w_MACSetReadPtrInRx
                0x9d02a754       0x44
 .text.mrf24w_MACSetReadPtrInRx
                0x9d02a754       0x44 build/WiFIG/production/_ext/334706090/mrf24w_mac_pic32.o

.text.WiFi_GratuitousArpTask
                0x9d02a798       0x44
 .text.WiFi_GratuitousArpTask
                0x9d02a798       0x44 build/WiFIG/production/_ext/334706090/wf_mac_24g.o
                0x9d02a798                WiFi_GratuitousArpTask

.text.MRF24W_MACProcess
                0x9d02a7dc       0x44
 .text.MRF24W_MACProcess
                0x9d02a7dc       0x44 build/WiFIG/production/_ext/334706090/wf_mac_24g.o
                0x9d02a7dc                MRF24W_MACProcess

.text.RawGetMgmtRxBuffer
                0x9d02a820       0x44
 .text.RawGetMgmtRxBuffer
                0x9d02a820       0x44 build/WiFIG/production/_ext/334706090/wf_mac_24g.o
                0x9d02a820                RawGetMgmtRxBuffer

.text.WF_SetWPATimeout
                0x9d02a864       0x44
 .text.WF_SetWPATimeout
                0x9d02a864       0x44 build/WiFIG/production/_ext/334706090/wf_param_msg_24g.o
                0x9d02a864                WF_SetWPATimeout

.text.WF_SetTxMode
                0x9d02a8a8       0x44
 .text.WF_SetTxMode
                0x9d02a8a8       0x44 build/WiFIG/production/_ext/334706090/wf_param_msg_24g.o
                0x9d02a8a8                WF_SetTxMode

.text.WF_SetTxDataConfirm
                0x9d02a8ec       0x44
 .text.WF_SetTxDataConfirm
                0x9d02a8ec       0x44 build/WiFIG/production/_ext/334706090/wf_param_msg_24g.o
                0x9d02a8ec                WF_SetTxDataConfirm

.text.strncat   0x9d02a930       0x44
 .text.strncat  0x9d02a930       0x44 c:/program files (x86)/microchip/xc32/v1.21/bin/../lib/gcc/pic32mx/4.5.2/../../../../pic32mx/lib/size\libc.a(strncat.o)
                0x9d02a930                strncat

.text.strncmp   0x9d02a974       0x44
 .text.strncmp  0x9d02a974       0x44 c:/program files (x86)/microchip/xc32/v1.21/bin/../lib/gcc/pic32mx/4.5.2/../../../../pic32mx/lib/size\libc.a(strncmp.o)
                0x9d02a974                strncmp

.text           0x9d02a9b8       0x44
 .text          0x9d02a9b8       0x44 c:/program files (x86)/microchip/xc32/v1.21/bin/../lib/gcc/pic32mx/4.5.2/size\libgcc.a(_lshrdi3.o)
                0x9d02a9b8                __lshrdi3

.text.TCPIP_IPV4_Task
                0x9d02a9fc       0x40
 .text.TCPIP_IPV4_Task
                0x9d02a9fc       0x40 build/WiFIG/production/_ext/427700826/ipv4.o
                0x9d02a9fc                TCPIP_IPV4_Task

.text.UDPResetHeader
                0x9d02aa3c       0x40
 .text.UDPResetHeader
                0x9d02aa3c       0x40 build/WiFIG/production/_ext/427700826/udp.o
                0x9d02aa3c                UDPResetHeader

.text.WF_CASetEventNotificationAction
                0x9d02aa7c       0x40
 .text.WF_CASetEventNotificationAction
                0x9d02aa7c       0x40 build/WiFIG/production/_ext/334706090/wf_connection_algorithm.o
                0x9d02aa7c                WF_CASetEventNotificationAction

.text.WF_SecurityOpenSet
                0x9d02aabc       0x40
 .text.WF_SecurityOpenSet
                0x9d02aabc       0x40 build/WiFIG/production/_ext/334706090/wf_connection_profile.o
                0x9d02aabc                WF_SecurityOpenSet

.text.MRF24W_MACConnect
                0x9d02aafc       0x40
 .text.MRF24W_MACConnect
                0x9d02aafc       0x40 build/WiFIG/production/_ext/334706090/mrf24w_mac_pic32.o
                0x9d02aafc                MRF24W_MACConnect

.text.mrf24w_MACEventGetPending
                0x9d02ab3c       0x40
 .text.mrf24w_MACEventGetPending
                0x9d02ab3c       0x40 build/WiFIG/production/_ext/334706090/mrf24w_mac_pic32.o

.text.DeallocateMgmtRxBuffer
                0x9d02ab7c       0x40
 .text.DeallocateMgmtRxBuffer
                0x9d02ab7c       0x40 build/WiFIG/production/_ext/334706090/wf_driver_raw_24g.o
                0x9d02ab7c                DeallocateMgmtRxBuffer

.text.MRF24W_MACDiscardRx
                0x9d02abbc       0x40
 .text.MRF24W_MACDiscardRx
                0x9d02abbc       0x40 build/WiFIG/production/_ext/334706090/wf_mac_24g.o
                0x9d02abbc                MRF24W_MACDiscardRx

.text.WF_GetTxMode
                0x9d02abfc       0x40
 .text.WF_GetTxMode
                0x9d02abfc       0x40 build/WiFIG/production/_ext/334706090/wf_param_msg_24g.o
                0x9d02abfc                WF_GetTxMode

.text.WF_MacAddressSet
                0x9d02ac3c       0x40
 .text.WF_MacAddressSet
                0x9d02ac3c       0x40 build/WiFIG/production/_ext/334706090/wf_param_msg_24g.o
                0x9d02ac3c                WF_MacAddressSet

.text.WF_MacAddressGet
                0x9d02ac7c       0x40
 .text.WF_MacAddressGet
                0x9d02ac7c       0x40 build/WiFIG/production/_ext/334706090/wf_param_msg_24g.o
                0x9d02ac7c                WF_MacAddressGet

.text.WF_RegionalDomainGet
                0x9d02acbc       0x40
 .text.WF_RegionalDomainGet
                0x9d02acbc       0x40 build/WiFIG/production/_ext/334706090/wf_param_msg_24g.o
                0x9d02acbc                WF_RegionalDomainGet

.text.SpiChnDataRdy
                0x9d02acfc       0x40
 .text.SpiChnDataRdy
                0x9d02acfc       0x40 c:/program files (x86)/microchip/xc32/v1.21/bin/../lib/gcc/pic32mx/4.5.2/../../../../pic32mx/lib/size\libmchp_peripheral_32MX695F512H.a(spi_chn_data_rdy_lib.o)
                0x9d02acfc                SpiChnDataRdy

.text._ARPDeleteClients
                0x9d02ad3c       0x3c
 .text._ARPDeleteClients
                0x9d02ad3c       0x3c build/WiFIG/production/_ext/427700826/arp.o

.text.ARPTmoHandler
                0x9d02ad78       0x3c
 .text.ARPTmoHandler
                0x9d02ad78       0x3c build/WiFIG/production/_ext/427700826/arp.o

.text.TCPIP_IPV4_GetUpperLayerHeaderPtr
                0x9d02adb4       0x3c
 .text.TCPIP_IPV4_GetUpperLayerHeaderPtr
                0x9d02adb4       0x3c build/WiFIG/production/_ext/427700826/ipv4.o
                0x9d02adb4                TCPIP_IPV4_GetUpperLayerHeaderPtr

.text.TCPIP_IPV4_GetPayloadLength
                0x9d02adf0       0x3c
 .text.TCPIP_IPV4_GetPayloadLength
                0x9d02adf0       0x3c build/WiFIG/production/_ext/427700826/ipv4.o
                0x9d02adf0                TCPIP_IPV4_GetPayloadLength

.rodata         0x9d02ae2c       0x3c
 .rodata        0x9d02ae2c       0x3c build/WiFIG/production/_ext/427700826/tcpip_heap_alloc.o

.text.WifiAsyncSetEventPending
                0x9d02ae68       0x3c
 .text.WifiAsyncSetEventPending
                0x9d02ae68       0x3c build/WiFIG/production/_ext/334706090/wf_event_handler.o
                0x9d02ae68                WifiAsyncSetEventPending

.text.mrf24w_MACSetWritePtr
                0x9d02aea4       0x3c
 .text.mrf24w_MACSetWritePtr
                0x9d02aea4       0x3c build/WiFIG/production/_ext/334706090/mrf24w_mac_pic32.o

.text.mrf24w_MACSetReadPtr
                0x9d02aee0       0x3c
 .text.mrf24w_MACSetReadPtr
                0x9d02aee0       0x3c build/WiFIG/production/_ext/334706090/mrf24w_mac_pic32.o

.text.mrf24w_MACSetBaseReadPtr
                0x9d02af1c       0x3c
 .text.mrf24w_MACSetBaseReadPtr
                0x9d02af1c       0x3c build/WiFIG/production/_ext/334706090/mrf24w_mac_pic32.o

.text.PORTSetPinsDigitalIn
                0x9d02af58       0x3c
 .text.PORTSetPinsDigitalIn
                0x9d02af58       0x3c c:/program files (x86)/microchip/xc32/v1.21/bin/../lib/gcc/pic32mx/4.5.2/../../../../pic32mx/lib/size\libmchp_peripheral_32MX695F512H.a(port_set_pins_digital_in_lib.o)
                0x9d02af58                PORTSetPinsDigitalIn

.text.PORTSetPinsDigitalOut
                0x9d02af94       0x3c
 .text.PORTSetPinsDigitalOut
                0x9d02af94       0x3c c:/program files (x86)/microchip/xc32/v1.21/bin/../lib/gcc/pic32mx/4.5.2/../../../../pic32mx/lib/size\libmchp_peripheral_32MX695F512H.a(port_set_pins_digital_out_lib.o)
                0x9d02af94                PORTSetPinsDigitalOut

.text           0x9d02afd0       0x38
 .text          0x9d02afd0       0x38 c:/program files (x86)/microchip/xc32/v1.21/bin/../lib/gcc/pic32mx/4.5.2/../../../../pic32mx/lib/size/crt0.o
                0x9d02affc                __crt0_exit

.text._OAHashProbeStep
                0x9d02b008       0x38
 .text._OAHashProbeStep
                0x9d02b008       0x38 build/WiFIG/production/_ext/427700826/hash_tbl.o

.rodata         0x9d02b040       0x38
 .rodata        0x9d02b040       0x38 build/WiFIG/production/_ext/334706090/wf_event_handler.o

.text.RenewDhcp
                0x9d02b078       0x38
 .text.RenewDhcp
                0x9d02b078       0x38 build/WiFIG/production/_ext/334706090/wf_event_handler.o

.text.mrf24w_MACClose
                0x9d02b0b0       0x38
 .text.mrf24w_MACClose
                0x9d02b0b0       0x38 build/WiFIG/production/_ext/334706090/mrf24w_mac_pic32.o

.rodata         0x9d02b0e8       0x70
 .rodata        0x9d02b0e8       0x38 build/WiFIG/production/_ext/334706090/wf_driver_com_24g.o
 .rodata        0x9d02b120       0x38 build/WiFIG/production/_ext/334706090/wf_param_msg_24g.o

.text.INTSetVectorPriority
                0x9d02b158       0x38
 .text.INTSetVectorPriority
                0x9d02b158       0x38 c:/program files (x86)/microchip/xc32/v1.21/bin/../lib/gcc/pic32mx/4.5.2/../../../../pic32mx/lib/size\libmchp_peripheral_32MX695F512H.a(int_tbl_lib.o)
                0x9d02b158                INTSetVectorPriority

.text.INTSetVectorSubPriority
                0x9d02b190       0x38
 .text.INTSetVectorSubPriority
                0x9d02b190       0x38 c:/program files (x86)/microchip/xc32/v1.21/bin/../lib/gcc/pic32mx/4.5.2/../../../../pic32mx/lib/size\libmchp_peripheral_32MX695F512H.a(int_tbl_lib.o)
                0x9d02b190                INTSetVectorSubPriority

.text.TCPIP_IPV4_SetDestAddress
                0x9d02b1c8       0x34
 .text.TCPIP_IPV4_SetDestAddress
                0x9d02b1c8       0x34 build/WiFIG/production/_ext/427700826/ipv4.o
                0x9d02b1c8                TCPIP_IPV4_SetDestAddress

.text.TCPIP_IPV4_GetDestAddress
                0x9d02b1fc       0x34
 .text.TCPIP_IPV4_GetDestAddress
                0x9d02b1fc       0x34 build/WiFIG/production/_ext/427700826/ipv4.o
                0x9d02b1fc                TCPIP_IPV4_GetDestAddress

.text.TCPIP_IPV4_GetSourceAddress
                0x9d02b230       0x34
 .text.TCPIP_IPV4_GetSourceAddress
                0x9d02b230       0x34 build/WiFIG/production/_ext/427700826/ipv4.o
                0x9d02b230                TCPIP_IPV4_GetSourceAddress

.text.ProcessTCPIPMacErrorEvents
                0x9d02b264       0x34
 .text.ProcessTCPIPMacErrorEvents
                0x9d02b264       0x34 build/WiFIG/production/_ext/427700826/tcpip_manager.o

.rodata         0x9d02b298       0x34
 .rodata        0x9d02b298       0x34 build/WiFIG/production/_ext/334706090/wf_connect.o

.text.WF_EintIsDisabled
                0x9d02b2cc       0x34
 .text.WF_EintIsDisabled
                0x9d02b2cc       0x34 build/WiFIG/production/_ext/334706090/wf_eint.o
                0x9d02b2cc                WF_EintIsDisabled

.text.WF_DeInit
                0x9d02b300       0x34
 .text.WF_DeInit
                0x9d02b300       0x34 build/WiFIG/production/_ext/334706090/wf_init.o
                0x9d02b300                WF_DeInit

.text.WF_SpiDisableChipSelect
                0x9d02b334       0x34
 .text.WF_SpiDisableChipSelect
                0x9d02b334       0x34 build/WiFIG/production/_ext/334706090/wf_spi.o
                0x9d02b334                WF_SpiDisableChipSelect

.text.mrf24w_MACGetReadPtrInRx
                0x9d02b368       0x34
 .text.mrf24w_MACGetReadPtrInRx
                0x9d02b368       0x34 build/WiFIG/production/_ext/334706090/mrf24w_mac_pic32.o

.text.mrf24w_MACIsTxReady
                0x9d02b39c       0x34
 .text.mrf24w_MACIsTxReady
                0x9d02b39c       0x34 build/WiFIG/production/_ext/334706090/mrf24w_mac_pic32.o

.text.mrf24w_MACFlush
                0x9d02b3d0       0x34
 .text.mrf24w_MACFlush
                0x9d02b3d0       0x34 build/WiFIG/production/_ext/334706090/mrf24w_mac_pic32.o

.text.mrf24w_MACDiscardRx
                0x9d02b404       0x34
 .text.mrf24w_MACDiscardRx
                0x9d02b404       0x34 build/WiFIG/production/_ext/334706090/mrf24w_mac_pic32.o

.text.mrf24w_MACCheckLink
                0x9d02b438       0x34
 .text.mrf24w_MACCheckLink
                0x9d02b438       0x34 build/WiFIG/production/_ext/334706090/mrf24w_mac_pic32.o

.text.SetNetworkConfig
                0x9d02b46c       0x34
 .text.SetNetworkConfig
                0x9d02b46c       0x34 build/WiFIG/production/_ext/334706090/wf_mac_24g.o
                0x9d02b46c                SetNetworkConfig

.rodata         0x9d02b4a0       0x34
 .rodata        0x9d02b4a0       0x34 build/WiFIG/production/_ext/334706090/wf_mgmt_msg_24g.o

.text.INTEnableSystemMultiVectoredInt
                0x9d02b4d4       0x34
 .text.INTEnableSystemMultiVectoredInt
                0x9d02b4d4       0x34 c:/program files (x86)/microchip/xc32/v1.21/bin/../lib/gcc/pic32mx/4.5.2/../../../../pic32mx/lib/size\libmchp_peripheral_32MX695F512H.a(int_enable_mv_int_lib.o)
                0x9d02b4d4                INTEnableSystemMultiVectoredInt

.text.SYS_Tasks
                0x9d02b508       0x30
 .text.SYS_Tasks
                0x9d02b508       0x30 build/WiFIG/production/_ext/365611741/system_services.o
                0x9d02b508                SYS_Tasks

.text.SYS_USERIO_Tasks
                0x9d02b538       0x30
 .text.SYS_USERIO_Tasks
                0x9d02b538       0x30 build/WiFIG/production/_ext/365611741/system_userio.o
                0x9d02b538                SYS_USERIO_Tasks

.text.TCPIP_IPV4_TmoHandler
                0x9d02b568       0x30
 .text.TCPIP_IPV4_TmoHandler
                0x9d02b568       0x30 build/WiFIG/production/_ext/427700826/ipv4.o
                0x9d02b568                TCPIP_IPV4_TmoHandler

.text._TcpTmoHandler
                0x9d02b598       0x30
 .text._TcpTmoHandler
                0x9d02b598       0x30 build/WiFIG/production/_ext/427700826/tcp.o

.text.TCPIP_STACK_TickHandler
                0x9d02b5c8       0x30
 .text.TCPIP_STACK_TickHandler
                0x9d02b5c8       0x30 build/WiFIG/production/_ext/427700826/tcpip_manager.o

.text.SetEventNotificationMask
                0x9d02b5f8       0x30
 .text.SetEventNotificationMask
                0x9d02b5f8       0x30 build/WiFIG/production/_ext/334706090/wf_connection_algorithm.o

.text.SetLogicalConnectionState
                0x9d02b628       0x30
 .text.SetLogicalConnectionState
                0x9d02b628       0x30 build/WiFIG/production/_ext/334706090/wf_connection_manager.o
                0x9d02b628                SetLogicalConnectionState

.text.SetAppPowerSaveMode
                0x9d02b658       0x30
 .text.SetAppPowerSaveMode
                0x9d02b658       0x30 build/WiFIG/production/_ext/334706090/wf_power_save.o
                0x9d02b658                SetAppPowerSaveMode

.text.WF_GetPowerSaveState
                0x9d02b688       0x30
 .text.WF_GetPowerSaveState
                0x9d02b688       0x30 build/WiFIG/production/_ext/334706090/wf_power_save.o
                0x9d02b688                WF_GetPowerSaveState

.text.SetPowerSaveState
                0x9d02b6b8       0x30
 .text.SetPowerSaveState
                0x9d02b6b8       0x30 build/WiFIG/production/_ext/334706090/wf_power_save.o

.text.WF_SpiEnableChipSelect
                0x9d02b6e8       0x30
 .text.WF_SpiEnableChipSelect
                0x9d02b6e8       0x30 build/WiFIG/production/_ext/334706090/wf_spi.o
                0x9d02b6e8                WF_SpiEnableChipSelect

.rodata         0x9d02b718       0x30
 .rodata        0x9d02b718       0x30 build/WiFIG/production/_ext/334706090/wf_mac_24g.o

.text.MRF24W_MACCheckLink
                0x9d02b748       0x30
 .text.MRF24W_MACCheckLink
                0x9d02b748       0x30 build/WiFIG/production/_ext/334706090/wf_mac_24g.o
                0x9d02b748                MRF24W_MACCheckLink

.text.WFStateNotify
                0x9d02b778       0x30
 .text.WFStateNotify
                0x9d02b778       0x30 build/WiFIG/production/_ext/1472/tcp6_demo_app.o
                0x9d02b778                WFStateNotify

.text.strcat    0x9d02b7a8       0x30
 .text.strcat   0x9d02b7a8       0x30 c:/program files (x86)/microchip/xc32/v1.21/bin/../lib/gcc/pic32mx/4.5.2/../../../../pic32mx/lib/size\libc.a(strcat.o)
                0x9d02b7a8                strcat

.text.SYS_WDT_Clear
                0x9d02b7d8       0x2c
 .text.SYS_WDT_Clear
                0x9d02b7d8       0x2c build/WiFIG/production/_ext/365611741/system_services.o
                0x9d02b7d8                SYS_WDT_Clear

.text.TCPIP_ANNOUNCE_TaskPending
                0x9d02b804       0x2c
 .text.TCPIP_ANNOUNCE_TaskPending
                0x9d02b804       0x2c build/WiFIG/production/_ext/427700826/tcpip_announce.o
                0x9d02b804                TCPIP_ANNOUNCE_TaskPending

.text.ARPTaskPending
                0x9d02b830       0x2c
 .text.ARPTaskPending
                0x9d02b830       0x2c build/WiFIG/production/_ext/427700826/arp.o
                0x9d02b830                ARPTaskPending

.text.TCPIP_IPV4_TaskPending
                0x9d02b85c       0x2c
 .text.TCPIP_IPV4_TaskPending
                0x9d02b85c       0x2c build/WiFIG/production/_ext/427700826/ipv4.o
                0x9d02b85c                TCPIP_IPV4_TaskPending

.text.TCPTaskPending
                0x9d02b888       0x2c
 .text.TCPTaskPending
                0x9d02b888       0x2c build/WiFIG/production/_ext/427700826/tcp.o
                0x9d02b888                TCPTaskPending

.text.WF_EintDisable
                0x9d02b8b4       0x2c
 .text.WF_EintDisable
                0x9d02b8b4       0x2c build/WiFIG/production/_ext/334706090/wf_eint.o
                0x9d02b8b4                WF_EintDisable

.text.WiFiAsyncTaskPending
                0x9d02b8e0       0x2c
 .text.WiFiAsyncTaskPending
                0x9d02b8e0       0x2c build/WiFIG/production/_ext/334706090/wf_event_handler.o
                0x9d02b8e0                WiFiAsyncTaskPending

.rodata         0x9d02b90c       0x2c
 .rodata        0x9d02b90c       0x2c build/WiFIG/production/_ext/334706090/wf_spi.o

.text.MRF24W_MACEventGetPending
                0x9d02b938       0x2c
 .text.MRF24W_MACEventGetPending
                0x9d02b938       0x2c build/WiFIG/production/_ext/334706090/mrf24w_events.o
                0x9d02b938                MRF24W_MACEventGetPending

.text.strchr    0x9d02b964       0x2c
 .text.strchr   0x9d02b964       0x2c c:/program files (x86)/microchip/xc32/v1.21/bin/../lib/gcc/pic32mx/4.5.2/../../../../pic32mx/lib/size\libc.a(strchr.o)
                0x9d02b964                strchr

.text._stub_sbd_memlayout
                0x9d02b990       0x2c
 .text._stub_sbd_memlayout
                0x9d02b990       0x2c c:/program files (x86)/microchip/xc32/v1.21/bin/../lib/gcc/pic32mx/4.5.2/../../../../pic32mx/lib/size\libpic32.a(sbrk.o)
                0x9d02b990                _sbd_memlayout
                0x9d02b990                _stub_sbd_memlayout

.rodata         0x9d02b9bc       0x28
 .rodata        0x9d02b9bc       0x28 build/WiFIG/production/_ext/792872985/usart.o

.text.DHCPServerDisable
                0x9d02b9e4       0x28
 .text.DHCPServerDisable
                0x9d02b9e4       0x28 build/WiFIG/production/_ext/427700826/dhcps.o
                0x9d02b9e4                DHCPServerDisable

.text.DHCPServerEnable
                0x9d02ba0c       0x28
 .text.DHCPServerEnable
                0x9d02ba0c       0x28 build/WiFIG/production/_ext/427700826/dhcps.o
                0x9d02ba0c                DHCPServerEnable

.text.ZCLLEnable
                0x9d02ba34       0x28
 .text.ZCLLEnable
                0x9d02ba34       0x28 build/WiFIG/production/_ext/427700826/zero_conf_link_local.o
                0x9d02ba34                ZCLLEnable

.text.SetSleepNeeded
                0x9d02ba5c       0x28
 .text.SetSleepNeeded
                0x9d02ba5c       0x28 build/WiFIG/production/_ext/334706090/wf_power_save.o
                0x9d02ba5c                SetSleepNeeded

.text.mrf24w_MACGetTxBaseAddr
                0x9d02ba84       0x28
 .text.mrf24w_MACGetTxBaseAddr
                0x9d02ba84       0x28 build/WiFIG/production/_ext/334706090/mrf24w_mac_pic32.o

.text.WF_OutputConnectionContext
                0x9d02baac       0x28
 .text.WF_OutputConnectionContext
                0x9d02baac       0x28 build/WiFIG/production/_ext/334706090/wf_debug_output.o
                0x9d02baac                WF_OutputConnectionContext

.text.SetDhcpProgressState
                0x9d02bad4       0x28
 .text.SetDhcpProgressState
                0x9d02bad4       0x28 build/WiFIG/production/_ext/334706090/wf_driver_com_24g.o
                0x9d02bad4                SetDhcpProgressState

.text.SignalMgmtConfirmReceivedEvent
                0x9d02bafc       0x28
 .text.SignalMgmtConfirmReceivedEvent
                0x9d02bafc       0x28 build/WiFIG/production/_ext/334706090/wf_mgmt_msg_24g.o
                0x9d02bafc                SignalMgmtConfirmReceivedEvent

.text.WiFiMemory_read
                0x9d02bb24       0x28
 .text.WiFiMemory_read
                0x9d02bb24       0x28 build/WiFIG/production/_ext/334706090/wf_configData.o
                0x9d02bb24                WiFiMemory_read

.text.INTClearFlag
                0x9d02bb4c       0x28
 .text.INTClearFlag
                0x9d02bb4c       0x28 c:/program files (x86)/microchip/xc32/v1.21/bin/../lib/gcc/pic32mx/4.5.2/../../../../pic32mx/lib/size\libmchp_peripheral_32MX695F512H.a(int_tbl_lib.o)
                0x9d02bb4c                INTClearFlag

.text.SYS_DRIVERS_Initialize
                0x9d02bb74       0x24
 .text.SYS_DRIVERS_Initialize
                0x9d02bb74       0x24 build/WiFIG/production/_ext/365611741/system_services.o
                0x9d02bb74                SYS_DRIVERS_Initialize

.text.TCPIP_STACK_GetDefaultNet
                0x9d02bb98       0x24
 .text.TCPIP_STACK_GetDefaultNet
                0x9d02bb98       0x24 build/WiFIG/production/_ext/427700826/tcpip_manager.o
                0x9d02bb98                TCPIP_STACK_GetDefaultNet

.text.TCPIP_STACK_NetworksNo
                0x9d02bbbc       0x24
 .text.TCPIP_STACK_NetworksNo
                0x9d02bbbc       0x24 build/WiFIG/production/_ext/427700826/tcpip_manager.o
                0x9d02bbbc                TCPIP_STACK_NetworksNo

.text.GetEventNotificationMask
                0x9d02bbe0       0x24
 .text.GetEventNotificationMask
                0x9d02bbe0       0x24 build/WiFIG/production/_ext/334706090/wf_connection_algorithm.o
                0x9d02bbe0                GetEventNotificationMask

.text.WFisConnected
                0x9d02bc04       0x24
 .text.WFisConnected
                0x9d02bc04       0x24 build/WiFIG/production/_ext/334706090/wf_connection_manager.o
                0x9d02bc04                WFisConnected

.text.GetWiFiNetworkType
                0x9d02bc28       0x24
 .text.GetWiFiNetworkType
                0x9d02bc28       0x24 build/WiFIG/production/_ext/334706090/wf_connection_profile.o
                0x9d02bc28                GetWiFiNetworkType

.text.WifiAsyncClearAllEvents
                0x9d02bc4c       0x24
 .text.WifiAsyncClearAllEvents
                0x9d02bc4c       0x24 build/WiFIG/production/_ext/334706090/wf_event_handler.o
                0x9d02bc4c                WifiAsyncClearAllEvents

.text.WF_ConfigDataSave
                0x9d02bc70       0x24
 .text.WF_ConfigDataSave
                0x9d02bc70       0x24 build/WiFIG/production/_ext/334706090/wf_init.o
                0x9d02bc70                WF_ConfigDataSave

.text.isSleepNeeded
                0x9d02bc94       0x24
 .text.isSleepNeeded
                0x9d02bc94       0x24 build/WiFIG/production/_ext/334706090/wf_power_save.o
                0x9d02bc94                isSleepNeeded

.text.ClearSleepNeeded
                0x9d02bcb8       0x24
 .text.ClearSleepNeeded
                0x9d02bcb8       0x24 build/WiFIG/production/_ext/334706090/wf_power_save.o
                0x9d02bcb8                ClearSleepNeeded

.text.GetAppPowerSaveMode
                0x9d02bcdc       0x24
 .text.GetAppPowerSaveMode
                0x9d02bcdc       0x24 build/WiFIG/production/_ext/334706090/wf_power_save.o
                0x9d02bcdc                GetAppPowerSaveMode

.text.InitPowerSaveTask
                0x9d02bd00       0x24
 .text.InitPowerSaveTask
                0x9d02bd00       0x24 build/WiFIG/production/_ext/334706090/wf_driver_com_24g.o
                0x9d02bd00                InitPowerSaveTask

.text.isDhcpInProgress
                0x9d02bd24       0x24
 .text.isDhcpInProgress
                0x9d02bd24       0x24 build/WiFIG/production/_ext/334706090/wf_driver_com_24g.o

.text.GetReadPtrRawWindow
                0x9d02bd48       0x24
 .text.GetReadPtrRawWindow
                0x9d02bd48       0x24 build/WiFIG/production/_ext/334706090/wf_mac_24g.o
                0x9d02bd48                GetReadPtrRawWindow

.text.GetNetworkConfig
                0x9d02bd6c       0x24
 .text.GetNetworkConfig
                0x9d02bd6c       0x24 build/WiFIG/production/_ext/334706090/wf_mac_24g.o
                0x9d02bd6c                GetNetworkConfig

.text.MRF24W_MACGetReadPtrInRx
                0x9d02bd90       0x24
 .text.MRF24W_MACGetReadPtrInRx
                0x9d02bd90       0x24 build/WiFIG/production/_ext/334706090/wf_mac_24g.o
                0x9d02bd90                MRF24W_MACGetReadPtrInRx

.text._snprintf_cdnopsuxX
                0x9d02bdb4       0x24
 .text._snprintf_cdnopsuxX
                0x9d02bdb4       0x24 c:/program files (x86)/microchip/xc32/v1.21/bin/../lib/gcc/pic32mx/4.5.2/../../../../pic32mx/lib/size\libc.a(snprintf_cdnopsuxX.eo)
                0x9d02bdb4                _snprintf_cdnopsuxX

.text.toupper   0x9d02bdd8       0x24
 .text.toupper  0x9d02bdd8       0x24 c:/program files (x86)/microchip/xc32/v1.21/bin/../lib/gcc/pic32mx/4.5.2/../../../../pic32mx/lib/size\libc.a(ctypef.o)
                0x9d02bdd8                toupper

.rodata         0x9d02bdfc       0x20
 .rodata        0x9d02bdfc       0x20 build/WiFIG/production/_ext/427700826/arp.o

.text.SetEapSecurity
                0x9d02be1c       0x20
 .text.SetEapSecurity
                0x9d02be1c       0x20 build/WiFIG/production/_ext/334706090/wf_connect.o

.text.MRF24W_MACPowerDown
                0x9d02be3c       0x20
 .text.MRF24W_MACPowerDown
                0x9d02be3c       0x20 build/WiFIG/production/_ext/334706090/wf_mac_24g.o
                0x9d02be3c                MRF24W_MACPowerDown

.text.MRF24W_MACPowerUp
                0x9d02be5c       0x20
 .text.MRF24W_MACPowerUp
                0x9d02be5c       0x20 build/WiFIG/production/_ext/334706090/wf_mac_24g.o
                0x9d02be5c                MRF24W_MACPowerUp

.text.SpiChnReadC
                0x9d02be7c       0x20
 .text.SpiChnReadC
                0x9d02be7c       0x20 c:/program files (x86)/microchip/xc32/v1.21/bin/../lib/gcc/pic32mx/4.5.2/../../../../pic32mx/lib/size\libmchp_peripheral_32MX695F512H.a(spi_chn_getc_lib.o)
                0x9d02be7c                SpiChnReadC

.text.SpiChnWriteC
                0x9d02be9c       0x20
 .text.SpiChnWriteC
                0x9d02be9c       0x20 c:/program files (x86)/microchip/xc32/v1.21/bin/../lib/gcc/pic32mx/4.5.2/../../../../pic32mx/lib/size\libmchp_peripheral_32MX695F512H.a(spi_chn_putc_lib.o)
                0x9d02be9c                SpiChnWriteC

.text.SpiChnTxBuffEmpty
                0x9d02bebc       0x20
 .text.SpiChnTxBuffEmpty
                0x9d02bebc       0x20 c:/program files (x86)/microchip/xc32/v1.21/bin/../lib/gcc/pic32mx/4.5.2/../../../../pic32mx/lib/size\libmchp_peripheral_32MX695F512H.a(spi_chn_tx_buff_empty_lib.o)
                0x9d02bebc                SpiChnTxBuffEmpty

.text.INTRestoreInterrupts
                0x9d02bedc       0x1c
 .text.INTRestoreInterrupts
                0x9d02bedc       0x1c c:/program files (x86)/microchip/xc32/v1.21/bin/../lib/gcc/pic32mx/4.5.2/../../../../pic32mx/lib/size\libmchp_peripheral_32MX695F512H.a(int_restore_interrupts_lib.o)
                0x9d02bedc                INTRestoreInterrupts

.text.free      0x9d02bef8       0x1c
 .text.free     0x9d02bef8       0x1c c:/program files (x86)/microchip/xc32/v1.21/bin/../lib/gcc/pic32mx/4.5.2/../../../../pic32mx/lib/size\libc.a(malloc.o)
                0x9d02bef8                free

.text.srand     0x9d02bf14       0x1c
 .text.srand    0x9d02bf14       0x1c c:/program files (x86)/microchip/xc32/v1.21/bin/../lib/gcc/pic32mx/4.5.2/../../../../pic32mx/lib/size\libc.a(rand.o)
                0x9d02bf14                srand

.text.CheKseg0CacheOn
                0x9d02bf30       0x18
 .text.CheKseg0CacheOn
                0x9d02bf30       0x18 c:/program files (x86)/microchip/xc32/v1.21/bin/../lib/gcc/pic32mx/4.5.2/../../../../pic32mx/lib/size\libmchp_peripheral_32MX695F512H.a(pcache.o)
                0x9d02bf30                CheKseg0CacheOn

.text           0x9d02bf48       0x18
 .text          0x9d02bf48       0x18 c:/program files (x86)/microchip/xc32/v1.21/bin/../lib/gcc/pic32mx/4.5.2/../../../../pic32mx/lib/size\libpic32.a(default-nmi-handler.o)
                0x9d02bf48                _nmi_handler

.rodata         0x9d02bf60       0x24
 .rodata        0x9d02bf60       0x14 c:/program files (x86)/microchip/xc32/v1.21/bin/../lib/gcc/pic32mx/4.5.2/../../../../pic32mx/lib/size\libmchp_peripheral_32MX695F512H.a(spi_map_tbl_libp.o)
                0x9d02bf60                _SpiMapTbl
 .rodata        0x9d02bf74       0x10 build/WiFIG/production/_ext/427700826/dhcp.o

.text.OpenCoreTimer
                0x9d02bf84        0xc
 .text.OpenCoreTimer
                0x9d02bf84        0xc c:/program files (x86)/microchip/xc32/v1.21/bin/../lib/gcc/pic32mx/4.5.2/../../../../pic32mx/lib/size\libmchp_peripheral.a(open_core_timer_lib.o)
                0x9d02bf84                OpenCoreTimer

.text._bootstrap_exception_handler
                0x9d02bf90        0xc
 .text._bootstrap_exception_handler
                0x9d02bf90        0xc c:/program files (x86)/microchip/xc32/v1.21/bin/../lib/gcc/pic32mx/4.5.2/../../../../pic32mx/lib/size\libpic32.a(default-bootstrap-exception-handler.o)
                0x9d02bf90                _bootstrap_exception_handler

.text.INTDisableInterrupts
                0x9d02bf9c        0x8
 .text.INTDisableInterrupts
                0x9d02bf9c        0x8 c:/program files (x86)/microchip/xc32/v1.21/bin/../lib/gcc/pic32mx/4.5.2/../../../../pic32mx/lib/size\libmchp_peripheral_32MX695F512H.a(int_disable_interrupts_lib.o)
                0x9d02bf9c                INTDisableInterrupts

.text.INTEnableInterrupts
                0x9d02bfa4        0x8
 .text.INTEnableInterrupts
                0x9d02bfa4        0x8 c:/program files (x86)/microchip/xc32/v1.21/bin/../lib/gcc/pic32mx/4.5.2/../../../../pic32mx/lib/size\libmchp_peripheral_32MX695F512H.a(int_enable_interrupts_lib.o)
                0x9d02bfa4                INTEnableInterrupts

.text._on_reset
                0x9d02bfac        0x8
 .text._on_reset
                0x9d02bfac        0x8 c:/program files (x86)/microchip/xc32/v1.21/bin/../lib/gcc/pic32mx/4.5.2/../../../../pic32mx/lib/size\libpic32.a(default-on-reset.o)
                0x9d02bfac                _on_reset

.text._on_bootstrap
                0x9d02bfb4        0x8
 .text._on_bootstrap
                0x9d02bfb4        0x8 c:/program files (x86)/microchip/xc32/v1.21/bin/../lib/gcc/pic32mx/4.5.2/../../../../pic32mx/lib/size\libpic32.a(default-on-bootstrap.o)
                0x9d02bfb4                _on_bootstrap

.rodata         0x9d02bfbc        0x8
 .rodata        0x9d02bfbc        0x8 c:/program files (x86)/microchip/xc32/v1.21/bin/../lib/gcc/pic32mx/4.5.2/size\libgcc.a(_floatundisf.o)

.rodata         0x9d0209f4        0x4
 .rodata        0x9d0209f4        0x4 build/WiFIG/production/_ext/427700826/tcpip_announce.o
